 eduke32

 Timestamp is 56d63510 (Tue Mar 01 19:34:24 2016)

 Preferred load address is 00400000

 Start         Length     Name                   Class
 0001:00000000 002a6220H .text                   CODE
 0001:002a6220 000073f4H .text$yc                CODE
 0002:00000000 0000212dH code                    CODE
 0003:00000000 00000720H .idata$5                DATA
 0003:00000720 00000004H .CRT$XCA                DATA
 0003:00000724 00000004H .CRT$XCAA               DATA
 0003:00000728 00000020H .CRT$XCU                DATA
 0003:00000748 00000004H .CRT$XCZ                DATA
 0003:0000074c 00000004H .CRT$XIA                DATA
 0003:00000750 00000004H .CRT$XIAA               DATA
 0003:00000754 00000004H .CRT$XIC                DATA
 0003:00000758 00000004H .CRT$XIY                DATA
 0003:0000075c 00000004H .CRT$XIZ                DATA
 0003:00000760 00059f80H .rdata                  DATA
 0003:0005a6e0 00000010H .rdata$CLSID_DirectDraw DATA
 0003:0005a6f0 00000010H .rdata$CLSID_DirectDraw7 DATA
 0003:0005a700 00000010H .rdata$CLSID_DirectDrawClipper DATA
 0003:0005a710 00000010H .rdata$CLSID_DirectInput DATA
 0003:0005a720 00000010H .rdata$CLSID_DirectInput8 DATA
 0003:0005a730 00000010H .rdata$CLSID_DirectInputDevice DATA
 0003:0005a740 00000010H .rdata$CLSID_DirectInputDevice8 DATA
 0003:0005a750 00000010H .rdata$CLSID_DirectSound DATA
 0003:0005a760 00000010H .rdata$CLSID_DirectSound8 DATA
 0003:0005a770 00000010H .rdata$CLSID_DirectSoundCapture DATA
 0003:0005a780 00000010H .rdata$CLSID_DirectSoundCapture8 DATA
 0003:0005a790 00000010H .rdata$CLSID_DirectSoundFullDuplex DATA
 0003:0005a7a0 00000010H .rdata$CLSID_XAudio2    DATA
 0003:0005a7b0 00000010H .rdata$CLSID_XAudio2_Debug DATA
 0003:0005a7c0 00000010H .rdata$DSDEVID_DefaultCapture DATA
 0003:0005a7d0 00000010H .rdata$DSDEVID_DefaultPlayback DATA
 0003:0005a7e0 00000010H .rdata$DSDEVID_DefaultVoiceCapture DATA
 0003:0005a7f0 00000010H .rdata$DSDEVID_DefaultVoicePlayback DATA
 0003:0005a800 00000010H .rdata$DSDEVID_WinePlayback DATA
 0003:0005a810 00000010H .rdata$GUID_Button      DATA
 0003:0005a820 00000010H .rdata$GUID_ConstantForce DATA
 0003:0005a830 00000010H .rdata$GUID_CustomForce DATA
 0003:0005a840 00000010H .rdata$GUID_Damper      DATA
 0003:0005a850 00000010H .rdata$GUID_Friction    DATA
 0003:0005a860 00000010H .rdata$GUID_Inertia     DATA
 0003:0005a870 00000010H .rdata$GUID_Joystick    DATA
 0003:0005a880 00000010H .rdata$GUID_Key         DATA
 0003:0005a890 00000010H .rdata$GUID_POV         DATA
 0003:0005a8a0 00000010H .rdata$GUID_RampForce   DATA
 0003:0005a8b0 00000010H .rdata$GUID_RxAxis      DATA
 0003:0005a8c0 00000010H .rdata$GUID_RyAxis      DATA
 0003:0005a8d0 00000010H .rdata$GUID_RzAxis      DATA
 0003:0005a8e0 00000010H .rdata$GUID_SawtoothDown DATA
 0003:0005a8f0 00000010H .rdata$GUID_SawtoothUp  DATA
 0003:0005a900 00000010H .rdata$GUID_Sine        DATA
 0003:0005a910 00000010H .rdata$GUID_Slider      DATA
 0003:0005a920 00000010H .rdata$GUID_Spring      DATA
 0003:0005a930 00000010H .rdata$GUID_Square      DATA
 0003:0005a940 00000010H .rdata$GUID_SysKeyboard DATA
 0003:0005a950 00000010H .rdata$GUID_SysKeyboardEm DATA
 0003:0005a960 00000010H .rdata$GUID_SysKeyboardEm2 DATA
 0003:0005a970 00000010H .rdata$GUID_SysMouse    DATA
 0003:0005a980 00000010H .rdata$GUID_SysMouseEm  DATA
 0003:0005a990 00000010H .rdata$GUID_SysMouseEm2 DATA
 0003:0005a9a0 00000010H .rdata$GUID_Triangle    DATA
 0003:0005a9b0 00000010H .rdata$GUID_Unknown     DATA
 0003:0005a9c0 00000010H .rdata$GUID_XAxis       DATA
 0003:0005a9d0 00000010H .rdata$GUID_YAxis       DATA
 0003:0005a9e0 00000010H .rdata$GUID_ZAxis       DATA
 0003:0005a9f0 00000010H .rdata$IID_AsyncIUnknown DATA
 0003:0005aa00 00000010H .rdata$IID_IAdviseSink  DATA
 0003:0005aa10 00000010H .rdata$IID_IBindCtx     DATA
 0003:0005aa20 00000010H .rdata$IID_IBindStatusCallback DATA
 0003:0005aa30 00000010H .rdata$IID_IBinding     DATA
 0003:0005aa40 00000010H .rdata$IID_IClassFactory DATA
 0003:0005aa50 00000010H .rdata$IID_ICreateTypeInfo DATA
 0003:0005aa60 00000010H .rdata$IID_IDataObject  DATA
 0003:0005aa70 00000010H .rdata$IID_IDirectDraw  DATA
 0003:0005aa80 00000010H .rdata$IID_IDirectDraw2 DATA
 0003:0005aa90 00000010H .rdata$IID_IDirectDraw3 DATA
 0003:0005aaa0 00000010H .rdata$IID_IDirectDraw4 DATA
 0003:0005aab0 00000010H .rdata$IID_IDirectDraw7 DATA
 0003:0005aac0 00000010H .rdata$IID_IDirectDrawClipper DATA
 0003:0005aad0 00000010H .rdata$IID_IDirectDrawColorControl DATA
 0003:0005aae0 00000010H .rdata$IID_IDirectDrawGammaControl DATA
 0003:0005aaf0 00000010H .rdata$IID_IDirectDrawPalette DATA
 0003:0005ab00 00000010H .rdata$IID_IDirectDrawSurface DATA
 0003:0005ab10 00000010H .rdata$IID_IDirectDrawSurface2 DATA
 0003:0005ab20 00000010H .rdata$IID_IDirectDrawSurface3 DATA
 0003:0005ab30 00000010H .rdata$IID_IDirectDrawSurface4 DATA
 0003:0005ab40 00000010H .rdata$IID_IDirectDrawSurface7 DATA
 0003:0005ab50 00000010H .rdata$IID_IDirectInput2A DATA
 0003:0005ab60 00000010H .rdata$IID_IDirectInput2W DATA
 0003:0005ab70 00000010H .rdata$IID_IDirectInput7A DATA
 0003:0005ab80 00000010H .rdata$IID_IDirectInput7W DATA
 0003:0005ab90 00000010H .rdata$IID_IDirectInput8A DATA
 0003:0005aba0 00000010H .rdata$IID_IDirectInput8W DATA
 0003:0005abb0 00000010H .rdata$IID_IDirectInputA DATA
 0003:0005abc0 00000010H .rdata$IID_IDirectInputDevice2A DATA
 0003:0005abd0 00000010H .rdata$IID_IDirectInputDevice2W DATA
 0003:0005abe0 00000010H .rdata$IID_IDirectInputDevice7A DATA
 0003:0005abf0 00000010H .rdata$IID_IDirectInputDevice7W DATA
 0003:0005ac00 00000010H .rdata$IID_IDirectInputDevice8A DATA
 0003:0005ac10 00000010H .rdata$IID_IDirectInputDevice8W DATA
 0003:0005ac20 00000010H .rdata$IID_IDirectInputDeviceA DATA
 0003:0005ac30 00000010H .rdata$IID_IDirectInputDeviceW DATA
 0003:0005ac40 00000010H .rdata$IID_IDirectInputEffect DATA
 0003:0005ac50 00000010H .rdata$IID_IDirectInputW DATA
 0003:0005ac60 00000010H .rdata$IID_IDirectSound DATA
 0003:0005ac70 00000010H .rdata$IID_IDirectSound3DBuffer DATA
 0003:0005ac80 00000010H .rdata$IID_IDirectSound3DListener DATA
 0003:0005ac90 00000010H .rdata$IID_IDirectSound8 DATA
 0003:0005aca0 00000010H .rdata$IID_IDirectSoundBuffer DATA
 0003:0005acb0 00000010H .rdata$IID_IDirectSoundBuffer8 DATA
 0003:0005acc0 00000010H .rdata$IID_IDirectSoundCapture DATA
 0003:0005acd0 00000010H .rdata$IID_IDirectSoundCaptureBuffer DATA
 0003:0005ace0 00000010H .rdata$IID_IDirectSoundCaptureBuffer8 DATA
 0003:0005acf0 00000010H .rdata$IID_IDirectSoundFullDuplex DATA
 0003:0005ad00 00000010H .rdata$IID_IDirectSoundNotify DATA
 0003:0005ad10 00000010H .rdata$IID_IDispatch    DATA
 0003:0005ad20 00000010H .rdata$IID_IEnumFORMATETC DATA
 0003:0005ad30 00000010H .rdata$IID_IEnumMoniker DATA
 0003:0005ad40 00000010H .rdata$IID_IEnumSTATDATA DATA
 0003:0005ad50 00000010H .rdata$IID_IEnumSTATSTG DATA
 0003:0005ad60 00000010H .rdata$IID_IEnumString  DATA
 0003:0005ad70 00000010H .rdata$IID_IEnumUnknown DATA
 0003:0005ad80 00000010H .rdata$IID_IEnumVARIANT DATA
 0003:0005ad90 00000010H .rdata$IID_IErrorLog    DATA
 0003:0005ada0 00000010H .rdata$IID_IKsPropertySet DATA
 0003:0005adb0 00000010H .rdata$IID_IMoniker     DATA
 0003:0005adc0 00000010H .rdata$IID_IPersist     DATA
 0003:0005add0 00000010H .rdata$IID_IPersistStream DATA
 0003:0005ade0 00000010H .rdata$IID_IPropertyBag DATA
 0003:0005adf0 00000010H .rdata$IID_IRecordInfo  DATA
 0003:0005ae00 00000010H .rdata$IID_IRunningObjectTable DATA
 0003:0005ae10 00000010H .rdata$IID_ISequentialStream DATA
 0003:0005ae20 00000010H .rdata$IID_IStorage     DATA
 0003:0005ae30 00000010H .rdata$IID_IStream      DATA
 0003:0005ae40 00000010H .rdata$IID_ITypeComp    DATA
 0003:0005ae50 00000010H .rdata$IID_ITypeInfo    DATA
 0003:0005ae60 00000010H .rdata$IID_ITypeLib     DATA
 0003:0005ae70 00000010H .rdata$IID_IUnknown     DATA
 0003:0005ae80 00000010H .rdata$IID_IXAudio2     DATA
 0003:0005ae90 0000003fH .rdata$debug            DATA
 0003:0005aed0 00002194H .rdata$zzz              DATA
 0003:0005d064 00000004H .rtc$IAA                DATA
 0003:0005d068 00000004H .rtc$IZZ                DATA
 0003:0005d06c 00000004H .rtc$TAA                DATA
 0003:0005d070 00000004H .rtc$TZZ                DATA
 0003:0005d078 0000005cH .xdata$x                DATA
 0003:0005d0d4 0000012cH .idata$2                DATA
 0003:0005d200 00000014H .idata$3                DATA
 0003:0005d214 00000720H .idata$4                DATA
 0003:0005d934 00001a8aH .idata$6                DATA
 0003:0005f3be 00000000H .edata                  DATA
 0004:00000000 0000f150H .data                   DATA
 0004:0000f160 10465be0H .bss                    DATA
 0005:00000000 00003e04H .drectve                DATA
 0006:00000000 0000994cH .eh_frame               DATA
 0007:00000000 00000a00H .rodata                 DATA
 0008:00000000 001d16d2H .debug_info             DATA
 0009:00000000 000185f3H .debug_abbrev           DATA
 000a:00000000 0012e7f0H .debug_loc              DATA
 000b:00000000 00000fe0H .debug_aranges          DATA
 000c:00000000 0001a028H .debug_ranges           DATA
 000d:00000000 000396e4H .debug_line             DATA
 000e:00000000 0000c29cH .debug_str              DATA
 000f:00000000 00020fd0H .debug_frame            DATA
 0010:00000000 000003d0H .rsrc$01                DATA
 0010:000003d0 00067ad0H .rsrc$02                DATA

  Address         Publics by Value              Rva+Base       Lib:Object

 0000:00000000       ___safe_se_handler_count   00000000     <absolute>
 0000:00000000       ___safe_se_handler_table   00000000     <absolute>
 0000:00000000       __except_list              00000000     <absolute>
 0000:00009876       __fltused                  00009876     <absolute>
 0000:00009876       __ldused                   00009876     <absolute>
 0000:00000000       ___ImageBase               00400000     <linker-defined>
 0001:00000040       _M32RunScript              00401040 f   game.obj
 0001:00000050       _G_DefaultRtsFile          00401050 f   game.obj
 0001:00000120       _P_SetGamePalette          00401120 f   game.obj
 0001:00000180       _G_HandleSpecialKeys       00401180 f   game.obj
 0001:00000380       _G_GameQuit                00401380 f   game.obj
 0001:000003f0       _A_CheckInventorySprite    004013f0 f   game.obj
 0001:00000450       _G_DrawTile                00401450 f   game.obj
 0001:000005b0       _G_DrawTilePal             004015b0 f   game.obj
 0001:000005e0       _G_DrawTileSmall           004015e0 f   game.obj
 0001:00000670       _G_DrawTilePalSmall        00401670 f   game.obj
 0001:000006a0       _G_FadePalette             004016a0 f   game.obj
 0001:00000700       _fadepal                   00401700 f   game.obj
 0001:000007a0       _G_GameExit                004017a0 f   game.obj
 0001:00000d60       _G_GetCrosshairColor       00401d60 f   game.obj
 0001:00000ea0       _G_SetCrosshairColor       00401ea0 f   game.obj
 0001:00001060       _G_DisplayRest             00402060 f   game.obj
 0001:00004d30       _G_HandleMirror            00405d30 f   game.obj
 0001:000050b0       _G_DrawRooms               004060b0 f   game.obj
 0001:00007540       _G_DumpDebugInfo           00408540 f   game.obj
 0001:00007a70       _A_InsertSprite            00408a70 f   game.obj
 0001:00007ec0       _Yax_SetBunchZs            00408ec0 f   game.obj
 0001:00007fd0       _A_Spawn                   00408fd0 f   game.obj
 0001:0000ed80       _G_DoSpriteAnimations      0040fd80 f   game.obj
 0001:00012270       _G_SetViewportShrink       00413270 f   game.obj
 0001:000122c0       _G_InitTimer               004132c0 f   game.obj
 0001:000122f0       _G_StartRTS                004132f0 f   game.obj
 0001:000123d0       _G_StartMusic              004133d0 f   game.obj
 0001:00012460       _G_HandleLocalKeys         00413460 f   game.obj
 0001:00013a60       _loaddefinitions_game      00414a60 f   game.obj
 0001:00014640       _G_UpdateAppTitle          00415640 f   game.obj
 0001:00014690       _G_Shutdown                00415690 f   game.obj
 0001:000148d0       _G_PostCreateGameState     004158d0 f   game.obj
 0001:00014c50       _G_UpdatePlayerFromMenu    00415c50 f   game.obj
 0001:00014e70       _G_BackToMenu              00415e70 f   game.obj
 0001:00014ed0       _app_crashhandler          00415ed0 f   game.obj
 0001:00014ef0       _G_MaybeAllocPlayer        00415ef0 f   game.obj
 0001:00014f90       _app_main                  00415f90 f   game.obj
 0001:000190f0       _G_DoMoveThings            0041a0f0 f   game.obj
 0001:00019910       _G_PrintYourTime           0041a910 f   game.obj
 0001:00019b80       _G_PrintParTime            0041ab80 f   game.obj
 0001:00019c00       _G_PrintDesignerTime       0041ac00 f   game.obj
 0001:00019c30       _G_PrintBestTime           0041ac30 f   game.obj
 0001:00019c50       _G_BonusScreen             0041ac50 f   game.obj
 0001:0001c350       _A_SpawnWallGlass          0041d350 f   game.obj
 0001:0001c6f0       _A_SpawnGlass              0041d6f0 f   game.obj
 0001:0001c800       _A_SpawnCeilingGlass       0041d800 f   game.obj
 0001:0001c9a0       _A_SpawnRandomGlass        0041d9a0 f   game.obj
 0001:0001d0c0       ?strchr@@YAPADPADH@Z       0041e0c0 f i game.obj
 0001:0001d0e0       ?strrchr@@YAPADPADH@Z      0041e0e0 f i game.obj
 0001:0001d100       ??I?$SectorTracker@H@@QAEPAHXZ 0041e100 f i game.obj
 0001:0001d100       ??I?$SectorTracker@G@@QAEPAGXZ 0041e100 f i game.obj
 0001:0001d120       ??4?$SectorTracker@F@@QAEFF@Z 0041e120 f i game.obj
 0001:0001d1c0       ??B?$SectorTracker@G@@QBEGXZ 0041e1c0 f i game.obj
 0001:0001d1c0       ?cast@?$SectorTracker@G@@QBEGXZ 0041e1c0 f i game.obj
 0001:0001d1c0       ??B?$SpriteTracker@F@@QBEFXZ 0041e1c0 f i game.obj
 0001:0001d1c0       ??B?$SectorTracker@F@@QBEFXZ 0041e1c0 f i game.obj
 0001:0001d1c0       ?cast@?$SpriteTracker@F@@QBEFXZ 0041e1c0 f i game.obj
 0001:0001d1c0       ??B?$WallTracker@F@@QBEFXZ 0041e1c0 f i game.obj
 0001:0001d1c0       ?cast@?$SectorTracker@F@@QBEFXZ 0041e1c0 f i game.obj
 0001:0001d1c0       ??B?$WallTracker@G@@QBEGXZ 0041e1c0 f i game.obj
 0001:0001d1c0       ??B?$SpriteTracker@G@@QBEGXZ 0041e1c0 f i game.obj
 0001:0001d1e0       ??4?$SectorTracker@H@@QAEHH@Z 0041e1e0 f i game.obj
 0001:0001d270       ??Y?$SectorTracker@H@@QAEHH@Z 0041e270 f i game.obj
 0001:0001d300       ??B?$SpriteTracker@H@@QBEHXZ 0041e300 f i game.obj
 0001:0001d300       ?cast@?$SpriteTracker@H@@QBEHXZ 0041e300 f i game.obj
 0001:0001d300       ??B?$SectorTracker@H@@QBEHXZ 0041e300 f i game.obj
 0001:0001d300       ??B?$WallTracker@H@@QBEHXZ 0041e300 f i game.obj
 0001:0001d300       ?cast@?$WallTracker@H@@QBEHXZ 0041e300 f i game.obj
 0001:0001d310       ??4?$SectorTracker@G@@QAEGG@Z 0041e310 f i game.obj
 0001:0001d3b0       ??_5?$SectorTracker@G@@QAEGG@Z 0041e3b0 f i game.obj
 0001:0001d450       ??_6?$SectorTracker@G@@QAEGG@Z 0041e450 f i game.obj
 0001:0001d4f0       ??4?$SectorTracker@C@@QAECC@Z 0041e4f0 f i game.obj
 0001:0001d580       ??4?$SectorTracker@E@@QAEEE@Z 0041e580 f i game.obj
 0001:0001d610       ??4?$WallTracker@G@@QAEGG@Z 0041e610 f i game.obj
 0001:0001d6b0       ??4?$WallTracker@C@@QAECC@Z 0041e6b0 f i game.obj
 0001:0001d740       ??4?$SpriteTracker@H@@QAEHH@Z 0041e740 f i game.obj
 0001:0001d7d0       ??Y?$SpriteTracker@H@@QAEHH@Z 0041e7d0 f i game.obj
 0001:0001d860       ??Z?$SpriteTracker@H@@QAEHH@Z 0041e860 f i game.obj
 0001:0001d8f0       ??4?$SpriteTracker@G@@QAEGG@Z 0041e8f0 f i game.obj
 0001:0001d990       ??_5?$SpriteTracker@G@@QAEGG@Z 0041e990 f i game.obj
 0001:0001da30       ??_4?$SpriteTracker@G@@QAEGG@Z 0041ea30 f i game.obj
 0001:0001dad0       ??_6?$SpriteTracker@G@@QAEGG@Z 0041ead0 f i game.obj
 0001:0001db70       ??_3?$SpriteTracker@G@@QAEGG@Z 0041eb70 f i game.obj
 0001:0001dc10       ??4?$SpriteTracker@F@@QAEFF@Z 0041ec10 f i game.obj
 0001:0001dcb0       ??Y?$SpriteTracker@F@@QAEFF@Z 0041ecb0 f i game.obj
 0001:0001dd50       ??_5?$SpriteTracker@F@@QAEFF@Z 0041ed50 f i game.obj
 0001:0001ddf0       ??_3?$SpriteTracker@F@@QAEFF@Z 0041edf0 f i game.obj
 0001:0001de90       ??4?$SpriteTracker@C@@QAECC@Z 0041ee90 f i game.obj
 0001:0001df20       ??B?$WallTracker@E@@QBEEXZ 0041ef20 f i gamevars.obj
 0001:0001df20       ??B?$SectorTracker@C@@QBECXZ 0041ef20 f i game.obj
 0001:0001df20       ??B?$SpriteTracker@E@@QBEEXZ 0041ef20 f i game.obj
 0001:0001df20       ??B?$WallTracker@C@@QBECXZ 0041ef20 f i game.obj
 0001:0001df20       ??B?$SpriteTracker@C@@QBECXZ 0041ef20 f i game.obj
 0001:0001df20       ??B?$SectorTracker@E@@QBEEXZ 0041ef20 f i game.obj
 0001:0001df30       ??4?$SpriteTracker@E@@QAEEE@Z 0041ef30 f i game.obj
 0001:0001dff0       _G_SetInterpolation        0041eff0 f   actors.obj
 0001:0001e070       _G_StopInterpolation       0041f070 f   actors.obj
 0001:0001e100       _G_DoInterpolations        0041f100 f   actors.obj
 0001:0001e1d0       _G_ClearCameraView         0041f1d0 f   actors.obj
 0001:0001e2a0       _A_RadiusDamage            0041f2a0 f   actors.obj
 0001:0001f010       _A_MoveSpriteClipdist      00420010 f   actors.obj
 0001:0001fa30       _G_Polymer_UnInit          00420a30 f   actors.obj
 0001:0001fac0       _A_DeleteSprite            00420ac0 f   actors.obj
 0001:0001fc10       _A_AddToDeleteQueue        00420c10 f   actors.obj
 0001:0001fca0       _A_SpawnMultiple           00420ca0 f   actors.obj
 0001:0001fd70       _A_DoGuts                  00420d70 f   actors.obj
 0001:0001ffa0       _A_DoGutsDir               00420fa0 f   actors.obj
 0001:00020130       _Sect_ToggleInterpolation  00421130 f   actors.obj
 0001:000202a0       _A_MoveSector              004212a0 f   actors.obj
 0001:000204c0       _G_AddGameLight            004214c0 f   actors.obj
 0001:00020890       _A_IncurDamage             00421890 f   actors.obj
 0001:00020d70       _A_MoveCyclers             00421d70 f   actors.obj
 0001:00020f30       _A_MoveDummyPlayers        00421f30 f   actors.obj
 0001:00021230       _A_PlayAlertSound          00422230 f   actors.obj
 0001:00021720       _A_CheckSwitchTile         00422720 f   actors.obj
 0001:000218e0       _G_RefreshLights           004228e0 f   actors.obj
 0001:00023000       _G_MoveWorld               00424000 f   actors.obj
 0001:0003b9e0       ??F?$SectorTracker@F@@QAEFH@Z 0043c9e0 f i actors.obj
 0001:0003ba20       ??I?$WallTracker@H@@QAEPAHXZ 0043ca20 f i actors.obj
 0001:0003ba40       ??E?$WallTracker@F@@QAEFH@Z 0043ca40 f i actors.obj
 0001:0003ba80       ??I?$SpriteTracker@F@@QAEPAFXZ 0043ca80 f i actors.obj
 0001:0003ba80       ??I?$SpriteTracker@H@@QAEPAHXZ 0043ca80 f i actors.obj
 0001:0003baa0       ??E?$SpriteTracker@G@@QAEGH@Z 0043caa0 f i actors.obj
 0001:0003baa0       ??E?$SpriteTracker@F@@QAEFH@Z 0043caa0 f i actors.obj
 0001:0003bae0       ??F?$SpriteTracker@F@@QAEFH@Z 0043cae0 f i actors.obj
 0001:0003bae0       ??F?$SpriteTracker@G@@QAEGH@Z 0043cae0 f i actors.obj
 0001:0003bb20       ??E?$SpriteTracker@C@@QAECXZ 0043cb20 f i actors.obj
 0001:0003bb50       ??E?$SpriteTracker@E@@QAEEH@Z 0043cb50 f i actors.obj
 0001:0003bb50       ??E?$SpriteTracker@C@@QAECH@Z 0043cb50 f i actors.obj
 0001:0003bb90       ??Y?$SectorTracker@F@@QAEFF@Z 0043cb90 f i actors.obj
 0001:0003bc30       ??Z?$SectorTracker@H@@QAEHH@Z 0043cc30 f i actors.obj
 0001:0003bcc0       ??Y?$SectorTracker@C@@QAECC@Z 0043ccc0 f i actors.obj
 0001:0003bd60       ??Z?$SectorTracker@C@@QAECC@Z 0043cd60 f i actors.obj
 0001:0003be00       ??Y?$SectorTracker@E@@QAEEE@Z 0043ce00 f i actors.obj
 0001:0003bea0       ??Z?$SectorTracker@E@@QAEEE@Z 0043cea0 f i actors.obj
 0001:0003bf40       ??4?$WallTracker@F@@QAEFF@Z 0043cf40 f i actors.obj
 0001:0003bfe0       ??_5?$WallTracker@G@@QAEGG@Z 0043cfe0 f i actors.obj
 0001:0003c080       ??_4?$WallTracker@G@@QAEGG@Z 0043d080 f i actors.obj
 0001:0003c120       ??Y?$WallTracker@C@@QAECC@Z 0043d120 f i actors.obj
 0001:0003c1c0       ??Z?$WallTracker@C@@QAECC@Z 0043d1c0 f i actors.obj
 0001:0003c260       ??4?$WallTracker@E@@QAEEE@Z 0043d260 f i actors.obj
 0001:0003c2f0       ??Y?$SpriteTracker@G@@QAEGG@Z 0043d2f0 f i actors.obj
 0001:0003c390       ??Z?$SpriteTracker@G@@QAEGG@Z 0043d390 f i actors.obj
 0001:0003c430       ??Z?$SpriteTracker@F@@QAEFF@Z 0043d430 f i actors.obj
 0001:0003c4d0       ??_4?$SpriteTracker@F@@QAEFF@Z 0043d4d0 f i actors.obj
 0001:0003c570       ??_2?$SpriteTracker@F@@QAEFF@Z 0043d570 f i actors.obj
 0001:0003c610       ??Y?$SpriteTracker@C@@QAECC@Z 0043d610 f i actors.obj
 0001:0003c6b0       ??Y?$SpriteTracker@E@@QAEEE@Z 0043d6b0 f i actors.obj
 0001:0003c750       ??Z?$SpriteTracker@E@@QAEEE@Z 0043d750 f i actors.obj
 0001:0003c7f0       ??_2?$SpriteTracker@E@@QAEEE@Z 0043d7f0 f i actors.obj
 0001:0003c890       ?Anim_Find@@YAPAUdukeanim_t@@PBD@Z 0043d890 f   anim.obj
 0001:0003c8c0       ?Anim_Setup@@YAPAUdukeanim_t@@PBDEP6AXH@Z@Z 0043d8c0 f   anim.obj
 0001:0003c970       ?Anim_Init@@YAXXZ          0043d970 f   anim.obj
 0001:0003ca70       ?Anim_Play@@YAHPBD@Z       0043da70 f   anim.obj
 0001:0003d220       ?endanimsounds@@YAXH@Z     0043e220 f   animsounds.obj
 0001:0003d510       ?logoanimsounds@@YAXH@Z    0043e510 f   animsounds.obj
 0001:0003d550       ?intro4animsounds@@YAXH@Z  0043e550 f   animsounds.obj
 0001:0003d5f0       ?first4animsounds@@YAXH@Z  0043e5f0 f   animsounds.obj
 0001:0003d690       ?intro42animsounds@@YAXH@Z 0043e690 f   animsounds.obj
 0001:0003d6c0       ?endanimvol41@@YAXH@Z      0043e6c0 f   animsounds.obj
 0001:0003d700       ?endanimvol42@@YAXH@Z      0043e700 f   animsounds.obj
 0001:0003d7b0       ?endanimvol43@@YAXH@Z      0043e7b0 f   animsounds.obj
 0001:0003d820       ?animvpx_read_ivf_header@@YAHHPAUanimvpx_ivf_header_t@@@Z 0043e820 f   animvpx.obj
 0001:0003da70       ?animvpx_init_codec@@YAHPBUanimvpx_ivf_header_t@@HPAUanimvpx_codec_ctx@@@Z 0043ea70 f   animvpx.obj
 0001:0003dc00       ?animvpx_uninit_codec@@YAHPAUanimvpx_codec_ctx@@@Z 0043ec00 f   animvpx.obj
 0001:0003dc70       ?animvpx_nextpic@@YAHPAUanimvpx_codec_ctx@@PAPAE@Z 0043ec70 f   animvpx.obj
 0001:0003e390       ?animvpx_setup_glstate@@YAXXZ 0043f390 f   animvpx.obj
 0001:0003e5e0       ?animvpx_restore_glstate@@YAXXZ 0043f5e0 f   animvpx.obj
 0001:0003e620       ?animvpx_render_frame@@YAHPAUanimvpx_codec_ctx@@@Z 0043f620 f   animvpx.obj
 0001:0003e8b0       ?animvpx_print_stats@@YAXPBUanimvpx_codec_ctx@@@Z 0043f8b0 f   animvpx.obj
 0001:0003e950       ?G_SetupCheats@@YAXXZ      0043f950 f   cheats.obj
 0001:0003ed20       ?G_DoCheats@@YAXXZ         0043fd20 f   cheats.obj
 0001:000402a0       ??_4?$SectorTracker@G@@QAEGG@Z 004412a0 f i cheats.obj
 0001:00040340       ?sbarsc@@YAHH@Z            00441340 f   sbar.obj
 0001:00040470       ?sbarx16@@YAHH@Z           00441470 f   sbar.obj
 0001:000404c0       ?sbary16@@YAHH@Z           004414c0 f   sbar.obj
 0001:000404f0       _G_DrawTXDigiNumZ          004414f0 f   sbar.obj
 0001:000405b0       ?G_DrawInventory@@YAXPBUDukePlayer_t@@@Z 004415b0 f   sbar.obj
 0001:00040aa0       _G_DrawFrags               00441aa0 f   sbar.obj
 0001:00040c50       ?G_DrawStatusBar@@YAXH@Z   00441c50 f   sbar.obj
 0001:00043b60       _G_DrawBackground          00444b60 f   sbar.obj
 0001:000445b0       ?textsc@@YAHH@Z            004455b0 f   screentext.obj
 0001:000447c0       ?G_GetStringLineLength@@YAHPBD0H@Z 004457c0 f   screentext.obj
 0001:00044800       ?G_GetStringNumLines@@YAHPBD0H@Z 00445800 f   screentext.obj
 0001:00044840       ?G_GetSubString@@YAPADPBD0HH@Z 00445840 f   screentext.obj
 0001:000448f0       ?G_GetStringTile@@YAHHPADH@Z 004458f0 f   screentext.obj
 0001:00044bb0       ?G_ScreenTextSize@@YA?AUvec2_t@@HHHHHPBDHHHHHHHHHH@Z 00445bb0 f   screentext.obj
 0001:00045450       ?G_AddCoordsFromRotation@@YAXPAUvec2_t@@PBU1@H@Z 00446450 f   screentext.obj
 0001:000454a0       ?G_ScreenText@@YA?AUvec2_t@@HHHHHHPBDHHHHHHHHHHHHH@Z 004464a0 f   screentext.obj
 0001:000462e0       ?G_ScreenTextShadow@@YA?AUvec2_t@@HHHHHHHHPBDHHHHHHHHHHHHH@Z 004472e0 f   screentext.obj
 0001:00046470       ?G_PrintGameText@@YAHHHHHPBDHHHHHHHHH@Z 00447470 f   screentext.obj
 0001:000465f0       ?G_GameTextLen@@YAHHPBD@Z  004475f0 f   screentext.obj
 0001:00046680       ?minitext_@@YAHHHPBDHHH@Z  00447680 f   screentext.obj
 0001:000467c0       _G_AddUserQuote            004477c0 f   screentext.obj
 0001:00046860       _G_PrintGameQuotes         00447860 f   screentext.obj
 0001:00046e10       _P_DoQuote                 00447e10 f   screentext.obj
 0001:00046f70       _clearGrpNamePtr           00447f70 f   common.obj
 0001:00046f90       _clearScriptNamePtr        00447f90 f   common.obj
 0001:00046fb0       _G_DefaultGrpFile          00447fb0 f   common.obj
 0001:00047010       _G_DefaultDefFile          00448010 f   common.obj
 0001:000470e0       _G_DefaultConFile          004480e0 f   common.obj
 0001:000471d0       _G_GrpFile                 004481d0 f   common.obj
 0001:000471f0       _G_DefFile                 004481f0 f   common.obj
 0001:00047210       _G_ConFile                 00448210 f   common.obj
 0001:00047230       _G_InitMultiPsky           00448230 f   common.obj
 0001:00047350       _G_SetupGlobalPsky         00448350 f   common.obj
 0001:00047420       _kopen4loadfrommod         00448420 f   common.obj
 0001:000474a0       _G_ExtPreInit              004484a0 f   common.obj
 0001:000474e0       _G_ExtInit                 004484e0 f   common.obj
 0001:000477d0       _G_ScanGroups              004487d0 f   common.obj
 0001:00047830       _G_LoadGroups              00448830 f   common.obj
 0001:00047cf0       _G_AddSearchPaths          00448cf0 f   common.obj
 0001:00048110       _G_CleanupSearchPaths      00449110 f   common.obj
 0001:00048150       _G_AddGroup                00449150 f   common.obj
 0001:000482b0       _G_AddPath                 004492b0 f   common.obj
 0001:00048350       _G_AddCon                  00449350 f   common.obj
 0001:00048380       _G_AddConModule            00449380 f   common.obj
 0001:00048430       _G_LoadGroupsInDir         00449430 f   common.obj
 0001:00048540       _G_DoAutoload              00449540 f   common.obj
 0001:00048590       _G_LoadLookups             00449590 f   common.obj
 0001:00048730       _S_OpenAudio               00449730 f   common.obj
 0001:000489f0       ?Demo_PrepareWarp@@YAXXZ   004499f0 f   demo.obj
 0001:00048a20       ?G_OpenDemoWrite@@YAXXZ    00449a20 f   demo.obj
 0001:00048e90       ?Demo_PlayFirst@@YAXHH@Z   00449e90 f   demo.obj
 0001:00048ed0       ?Demo_SetFirst@@YAXPBD@Z   00449ed0 f   demo.obj
 0001:00048f40       ?G_DemoRecord@@YAXXZ       00449f40 f   demo.obj
 0001:000490f0       ?G_CloseDemoWrite@@YAXXZ   0044a0f0 f   demo.obj
 0001:000491e0       ?Demo_IsProfiling@@YAHXZ   0044a1e0 f   demo.obj
 0001:00049200       ?G_PlaybackDemo@@YAHXZ     0044a200 f   demo.obj
 0001:0004abd0       ?C_InitHashes@@YAXXZ       0044bbd0 f   gamedef.obj
 0001:0004afa0       _G_DoGameStartup           0044bfa0 f   gamedef.obj
 0001:0004b3c0       _C_DefineMusic             0044c3c0 f   gamedef.obj
 0001:0004b540       _C_DefineVolumeFlags       0044c540 f   gamedef.obj
 0001:0004b570       _C_UndefineVolume          0044c570 f   gamedef.obj
 0001:0004b610       _C_UndefineSkill           0044c610 f   gamedef.obj
 0001:0004b690       _C_UndefineLevel           0044c690 f   gamedef.obj
 0001:0004b740       _C_AllocProjectile         0044c740 f   gamedef.obj
 0001:0004b790       _C_FreeProjectile          0044c790 f   gamedef.obj
 0001:0004b7d0       _C_AllocQuote              0044c7d0 f   gamedef.obj
 0001:0004b870       _C_InitQuotes              0044c870 f   gamedef.obj
 0001:0004bca0       _C_InitProjectiles         0044cca0 f   gamedef.obj
 0001:0004be10       ?C_PrintStats@@YAXXZ       0044ce10 f   gamedef.obj
 0001:0004bf60       _C_Compile                 0044cf60 f   gamedef.obj
 0001:00056a50       _C_ReportError             00457a50 f   gamedef.obj
 0001:00057010       ?strstr@@YAPADPADPBD@Z     00458010 f i gamedef.obj
 0001:00057060       _VM_ScriptInfo             00458060 f   gameexec.obj
 0001:00057210       _VM_OnEventWithBoth_       00458210 f   gameexec.obj
 0001:00057430       _VM_OnEventWithReturn_     00458430 f   gameexec.obj
 0001:00057450       _VM_OnEventWithDist_       00458450 f   gameexec.obj
 0001:00057470       _VM_OnEvent_               00458470 f   gameexec.obj
 0001:00057490       _A_Dodge                   00458490 f   gameexec.obj
 0001:000576e0       _A_GetFurthestAngle        004586e0 f   gameexec.obj
 0001:00057870       _A_FurthestVisiblePoint    00458870 f   gameexec.obj
 0001:00057aa0       _A_GetZLimits              00458aa0 f   gameexec.obj
 0001:00057e60       _A_Fall                    00458e60 f   gameexec.obj
 0001:00058280       _G_GetAngleDelta           00459280 f   gameexec.obj
 0001:000582f0       _G_GetTimeDate             004592f0 f   gameexec.obj
 0001:000583c0       _G_StartTrack              004593c0 f   gameexec.obj
 0001:0006a270       _A_LoadActor               0046b270 f   gameexec.obj
 0001:0006a380       _A_Execute                 0046b380 f   gameexec.obj
 0001:0006bab0       _G_SaveMapState            0046cab0 f   gameexec.obj
 0001:0006c180       _G_RestoreMapState         0046d180 f   gameexec.obj
 0001:0006cad0       ??I?$SpriteTracker@G@@QAEPAGXZ 0046dad0 f i gameexec.obj
 0001:0006cb10       ?VM_GetUserdef@@YIHH@Z     0046db10 f   gamevars.obj
 0001:0006d2b0       ?VM_SetUserdef@@YIXHH@Z    0046e2b0 f   gamevars.obj
 0001:0006da10       ?VM_GetActiveProjectile@@YIHHH@Z 0046ea10 f   gamevars.obj
 0001:0006dcd0       ?VM_SetActiveProjectile@@YIXHHH@Z 0046ecd0 f   gamevars.obj
 0001:0006df80       ?VM_GetPlayer@@YIHHHH@Z    0046ef80 f   gamevars.obj
 0001:0006ed40       ?VM_SetPlayer@@YIXHHHH@Z   0046fd40 f   gamevars.obj
 0001:0006fb40       ?VM_GetPlayerInput@@YIHHH@Z 00470b40 f   gamevars.obj
 0001:0006fc30       ?VM_SetPlayerInput@@YIXHHH@Z 00470c30 f   gamevars.obj
 0001:0006fd10       ?VM_GetWall@@YIHHH@Z       00470d10 f   gamevars.obj
 0001:0006ff60       ?VM_SetWall@@YIXHHH@Z      00470f60 f   gamevars.obj
 0001:000701a0       ?VM_GetSector@@YIHHH@Z     004711a0 f   gamevars.obj
 0001:00070580       ?VM_SetSector@@YIXHHH@Z    00471580 f   gamevars.obj
 0001:00070920       ?VM_SetSprite@@YIXHHHH@Z   00471920 f   gamevars.obj
 0001:00071050       ?VM_GetSprite@@YIHHHH@Z    00472050 f   gamevars.obj
 0001:000717e0       ?VM_GetTsprite@@YIHHH@Z    004727e0 f   gamevars.obj
 0001:00071ab0       ?VM_SetTsprite@@YIXHHH@Z   00472ab0 f   gamevars.obj
 0001:00071d70       ?VM_GetProjectile@@YIHHH@Z 00472d70 f   gamevars.obj
 0001:00072040       ?VM_SetProjectile@@YIXHHH@Z 00473040 f   gamevars.obj
 0001:00072300       ?VM_GetTileData@@YIHHH@Z   00473300 f   gamevars.obj
 0001:00072420       ?VM_GetPalData@@YIHHH@Z    00473420 f   gamevars.obj
 0001:00072490       ?Gv_ReadSave@@YAHHH@Z      00473490 f   gamevars.obj
 0001:00072e80       ?Gv_WriteSave@@YAXPAU_iobuf@@H@Z 00473e80 f   gamevars.obj
 0001:000732c0       ?Gv_DumpValues@@YAXXZ      004742c0 f   gamevars.obj
 0001:000734d0       ?Gv_ResetVars@@YAXXZ       004744d0 f   gamevars.obj
 0001:000735f0       ?Gv_NewArray@@YAHPBDPAXHI@Z 004745f0 f   gamevars.obj
 0001:000738a0       ?Gv_NewVar@@YAHPBDHI@Z     004748a0 f   gamevars.obj
 0001:00073c90       ?Gv_GetGameArrayValue@@YIHHH@Z 00474c90 f   gamevars.obj
 0001:00073d60       ?Gv_GetVar@@YIHHHH@Z       00474d60 f   gamevars.obj
 0001:000744b0       ?Gv_SetVar@@YIXHHHH@Z      004754b0 f   gamevars.obj
 0001:00074680       ?Gv_GetSpecialVarX@@YIHH@Z 00475680 f   gamevars.obj
 0001:00074dc0       ?Gv_GetVarX@@YIHH@Z        00475dc0 f   gamevars.obj
 0001:00074f70       ?Gv_GetManyVars@@YIXHQAH@Z 00475f70 f   gamevars.obj
 0001:00075170       ?Gv_SetVarX@@YIXHH@Z       00476170 f   gamevars.obj
 0001:000752d0       ?Gv_GetVarByLabel@@YAHPBDHHH@Z 004762d0 f   gamevars.obj
 0001:00075320       ?Gv_ResetSystemDefaults@@YAXXZ 00476320 f   gamevars.obj
 0001:00075940       ?Gv_FinalizeWeaponDefaults@@YAXXZ 00476940 f   gamevars.obj
 0001:00075d30       ?Gv_Init@@YAXXZ            00476d30 f   gamevars.obj
 0001:00076cd0       ?Gv_InitWeaponPointers@@YAXXZ 00477cd0 f   gamevars.obj
 0001:000770f0       ?Gv_RefreshPointers@@YAXXZ 004780f0 f   gamevars.obj
 0001:00077960       ??4?$WallTracker@H@@QAEHH@Z 00478960 f i gamevars.obj
 0001:000779f0       ?I_CheckAllInput@@YAHXZ    004789f0 f   input.obj
 0001:00077a30       ?I_ClearAllInput@@YAXXZ    00478a30 f   input.obj
 0001:00077a50       ?I_AdvanceTrigger@@YAHXZ   00478a50 f   input.obj
 0001:00077b10       ?I_AdvanceTriggerClear@@YAXXZ 00478b10 f   input.obj
 0001:00077b50       ?I_ReturnTrigger@@YAHXZ    00478b50 f   input.obj
 0001:00077bb0       ?I_ReturnTriggerClear@@YAXXZ 00478bb0 f   input.obj
 0001:00077be0       ?I_EscapeTrigger@@YAHXZ    00478be0 f   input.obj
 0001:00077c00       ?I_EscapeTriggerClear@@YAXXZ 00478c00 f   input.obj
 0001:00077c20       ?I_MenuUp@@YAHXZ           00478c20 f   input.obj
 0001:00077c90       ?I_MenuUpClear@@YAXXZ      00478c90 f   input.obj
 0001:00077cd0       ?I_MenuDown@@YAHXZ         00478cd0 f   input.obj
 0001:00077d50       ?I_MenuDownClear@@YAXXZ    00478d50 f   input.obj
 0001:00077d90       ?I_MenuLeft@@YAHXZ         00478d90 f   input.obj
 0001:00077e50       ?I_MenuLeftClear@@YAXXZ    00478e50 f   input.obj
 0001:00077e90       ?I_MenuRight@@YAHXZ        00478e90 f   input.obj
 0001:00077f60       ?I_MenuRightClear@@YAXXZ   00478f60 f   input.obj
 0001:00077fb0       ?I_PanelUp@@YAHXZ          00478fb0 f   input.obj
 0001:00077ff0       ?I_PanelUpClear@@YAXXZ     00478ff0 f   input.obj
 0001:00078010       ?I_PanelDown@@YAHXZ        00479010 f   input.obj
 0001:00078060       ?I_PanelDownClear@@YAXXZ   00479060 f   input.obj
 0001:00078080       ?I_SliderLeft@@YAHXZ       00479080 f   input.obj
 0001:000780d0       ?I_SliderLeftClear@@YAXXZ  004790d0 f   input.obj
 0001:000780f0       ?I_SliderRight@@YAHXZ      004790f0 f   input.obj
 0001:00078140       ?I_SliderRightClear@@YAXXZ 00479140 f   input.obj
 0001:00078160       ?I_EnterText@@YAHPADHH@Z   00479160 f   input.obj
 0001:00078260       _menutext_                 00479260 f   menus.obj
 0001:00078330       _M_Init                    00479330 f   menus.obj
 0001:000790b0       ?klistbookends@@YAXPAU_CACHE1D_FIND_REC@@@Z 0047a0b0 f   menus.obj
 0001:00079140       ?M_Anim_SinOutRight@@YAHPAUMenuAnimation_t@@@Z 0047a140 f   menus.obj
 0001:00079290       ?M_Anim_SinInRight@@YAHPAUMenuAnimation_t@@@Z 0047a290 f   menus.obj
 0001:000792d0       ?M_Anim_SinOutLeft@@YAHPAUMenuAnimation_t@@@Z 0047a2d0 f   menus.obj
 0001:00079310       ?M_Anim_SinInLeft@@YAHPAUMenuAnimation_t@@@Z 0047a310 f   menus.obj
 0001:00079350       _M_ChangeMenuAnimate       0047a350 f   menus.obj
 0001:00079450       _M_ChangeMenu              0047a450 f   menus.obj
 0001:00079a50       _G_CheckPlayerColor        0047aa50 f   menus.obj
 0001:00079a90       ?M_DetermineMenuSpecialState@@YAHPAUMenuEntry_t@@@Z 0047aa90 f   menus.obj
 0001:00079b00       _M_IsTextInput             0047ab00 f   menus.obj
 0001:00079b80       _M_OpenMenu                0047ab80 f   menus.obj
 0001:00079bf0       _M_CloseMenu               0047abf0 f   menus.obj
 0001:00079cd0       _M_DisplayMenus            0047acd0 f   menus.obj
 0001:000865c0       ?G_ProcessDynamicTileMapping@@YAXPBDH@Z 004875c0 f   namesdyn.obj
 0001:00086650       ?inithashnames@@YAXXZ      00487650 f   namesdyn.obj
 0001:000866b0       ?freehashnames@@YAXXZ      004876b0 f   namesdyn.obj
 0001:000866d0       ?G_InitDynamicTiles@@YAXXZ 004876d0 f   namesdyn.obj
 0001:000868d0       ?Net_SyncPlayer@@YAXPAU_ENetEvent@@@Z 004878d0 f   net.obj
 0001:00086a70       ?Net_SpawnPlayer@@YAXH@Z   00487a70 f   net.obj
 0001:00086b10       _faketimerhandler          00487b10 f   net.obj
 0001:00086b60       ?Net_WaitForServer@@YAXXZ  00487b60 f   net.obj
 0001:00086dc0       ?Net_ResetPrediction@@YAXXZ 00487dc0 f   net.obj
 0001:00086f50       ?Net_Connect@@YAXPBD@Z     00487f50 f   net.obj
 0001:00087150       ?Net_Disconnect@@YAXXZ     00488150 f   net.obj
 0001:00087300       ?Net_ReceiveDisconnect@@YAXPAU_ENetEvent@@@Z 00488300 f   net.obj
 0001:00087410       ?Net_GetPackets@@YAXXZ     00488410 f   net.obj
 0001:00087480       ?Net_HandleClientPackets@@YAXXZ 00488480 f   net.obj
 0001:00087840       ?Net_HandleServerPackets@@YAXXZ 00488840 f   net.obj
 0001:000878b0       ?Net_ParseClientPacket@@YAXPAU_ENetEvent@@@Z 004888b0 f   net.obj
 0001:00087b60       ?Net_ParseServerPacket@@YAXPAU_ENetEvent@@@Z 00488b60 f   net.obj
 0001:00087e70       ?Net_ParsePacketCommon@@YAXPAEHH@Z 00488e70 f   net.obj
 0001:00087f30       ?Net_SendAcknowledge@@YAXPAU_ENetPeer@@@Z 00488f30 f   net.obj
 0001:00087f80       ?Net_ReceiveAcknowledge@@YAXPAEH@Z 00488f80 f   net.obj
 0001:00087f90       ?Net_SendChallenge@@YAXXZ  00488f90 f   net.obj
 0001:00088070       ?Net_ReceiveChallenge@@YAXPAEHPAU_ENetEvent@@@Z 00489070 f   net.obj
 0001:00088180       ?Net_SendNewPlayer@@YAXH@Z 00489180 f   net.obj
 0001:000881f0       ?Net_ReceiveNewPlayer@@YAXPAEH@Z 004891f0 f   net.obj
 0001:00088390       ?Net_SendPlayerIndex@@YAXHPAU_ENetPeer@@@Z 00489390 f   net.obj
 0001:000883d0       ?Net_ReceivePlayerIndex@@YAXPAEH@Z 004893d0 f   net.obj
 0001:00088400       ?Net_SendClientInfo@@YAXXZ 00489400 f   net.obj
 0001:000886a0       ?Net_ReceiveClientInfo@@YAXPAEHH@Z 004896a0 f   net.obj
 0001:00088840       ?Net_SendUserMapName@@YAXXZ 00489840 f   net.obj
 0001:00088920       ?Net_ReceiveUserMapName@@YAXPAEH@Z 00489920 f   net.obj
 0001:000889d0       ?Net_GetRevision@@YAPAUnetmapstate_t@@EE@Z 004899d0 f   net.obj
 0001:00088a80       ?Net_SendMapUpdate@@YAXXZ  00489a80 f   net.obj
 0001:00088c30       ?Net_ReceiveMapUpdate@@YAXPAU_ENetEvent@@@Z 00489c30 f   net.obj
 0001:00088c80       ?Net_SaveMapState@@YAXPAUnetmapstate_t@@@Z 00489c80 f   net.obj
 0001:00088db0       ?Net_FillMapDiff@@YAXII@Z  00489db0 f   net.obj
 0001:00089050       ?Net_RestoreMapState@@YAXXZ 0048a050 f   net.obj
 0001:00089130       ?Net_CopyToNet@@YAXHPAUnetactor_t@@@Z 0048a130 f   net.obj
 0001:000892a0       ?Net_CopyFromNet@@YAXHPAUnetactor_t@@@Z 0048a2a0 f   net.obj
 0001:000894c0       ?Net_ActorsAreDifferent@@YAHPAUnetactor_t@@0@Z 0048a4c0 f   net.obj
 0001:00089860       ?Net_IsRelevantSprite@@YAHH@Z 0048a860 f   net.obj
 0001:000898d0       ?Net_IsRelevantStat@@YAHH@Z 0048a8d0 f   net.obj
 0001:00089930       ?Net_InsertSprite@@YAHHH@Z 0048a930 f   net.obj
 0001:00089980       ?Net_DeleteSprite@@YAXH@Z  0048a980 f   net.obj
 0001:000899e0       ?Net_FillPlayerUpdate@@YAXPAUplayerupdate_t@@H@Z 0048a9e0 f   net.obj
 0001:00089b10       ?Net_ExtractPlayerUpdate@@YAXPAUplayerupdate_t@@H@Z 0048ab10 f   net.obj
 0001:00089c50       ?Net_SendServerUpdates@@YAXXZ 0048ac50 f   net.obj
 0001:0008a040       ?Net_ReceiveServerUpdate@@YAXPAU_ENetEvent@@@Z 0048b040 f   net.obj
 0001:0008a370       ?Net_SendClientUpdate@@YAXXZ 0048b370 f   net.obj
 0001:0008a400       ?Net_ReceiveClientUpdate@@YAXPAU_ENetEvent@@@Z 0048b400 f   net.obj
 0001:0008a4a0       ?Net_SendMessage@@YAXXZ    0048b4a0 f   net.obj
 0001:0008aee0       ?Net_ReceiveMessage@@YAXPAEH@Z 0048bee0 f   net.obj
 0001:0008af40       ?Net_StartNewGame@@YAXXZ   0048bf40 f   net.obj
 0001:0008aff0       ?Net_NotifyNewGame@@YAXXZ  0048bff0 f   net.obj
 0001:0008b0e0       ?Net_SendNewGame@@YAXHPAU_ENetPeer@@@Z 0048c0e0 f   net.obj
 0001:0008b160       ?Net_ReceiveNewGame@@YAXPAU_ENetEvent@@@Z 0048c160 f   net.obj
 0001:0008b210       ?Net_FillNewGame@@YAXPAUnewgame_t@@H@Z 0048c210 f   net.obj
 0001:0008b310       ?Net_ExtractNewGame@@YAXPAUnewgame_t@@H@Z 0048c310 f   net.obj
 0001:0008b420       ?Net_SendMapVoteInitiate@@YAXXZ 0048c420 f   net.obj
 0001:0008b490       ?Net_ReceiveMapVoteInitiate@@YAXPAE@Z 0048c490 f   net.obj
 0001:0008b5d0       ?Net_SendMapVote@@YAXH@Z   0048c5d0 f   net.obj
 0001:0008b690       ?Net_ReceiveMapVote@@YAXPAE@Z 0048c690 f   net.obj
 0001:0008b730       ?Net_CheckForEnoughVotes@@YAXXZ 0048c730 f   net.obj
 0001:0008b830       ?Net_SendMapVoteCancel@@YAXH@Z 0048c830 f   net.obj
 0001:0008b8f0       ?Net_ReceiveMapVoteCancel@@YAXPAE@Z 0048c8f0 f   net.obj
 0001:0008ba40       _P_UpdateScreenPal         0048ca40 f   player.obj
 0001:0008bb40       _P_QuickKill               0048cb40 f   player.obj
 0001:0008bc00       _A_GetHitscanRange         0048cc00 f   player.obj
 0001:0008bd50       _A_ShootWithZvel           0048cd50 f   player.obj
 0001:00091280       _P_GetHudPal               00492280 f   player.obj
 0001:00091300       _P_SetWeaponGamevars       00492300 f   player.obj
 0001:00091380       _P_DisplayScuba            00492380 f   player.obj
 0001:000916e0       _P_DisplayWeapon           004926e0 f   player.obj
 0001:00094da0       _P_GetInput                00495da0 f   player.obj
 0001:00096390       _P_DropWeapon              00497390 f   player.obj
 0001:00096430       _P_AddAmmo                 00497430 f   player.obj
 0001:000964a0       _P_AddWeapon               004974a0 f   player.obj
 0001:00096780       _P_SelectNextInvItem       00497780 f   player.obj
 0001:00096850       _P_CheckWeapon             00497850 f   player.obj
 0001:000969f0       _P_FindOtherPlayer         004979f0 f   player.obj
 0001:00096b20       _P_FragPlayer              00497b20 f   player.obj
 0001:00097130       _P_WeaponState             00498130 f   player.obj
 0001:00097290       _P_EndLevel                00498290 f   player.obj
 0001:00097340       _P_UpdatePosWhenViewingCam 00498340 f   player.obj
 0001:000973e0       _P_ProcessInput            004983e0 f   player.obj
 0001:0009dc90       ??_0?$SpriteTracker@F@@QAEFF@Z 0049ec90 f i player.obj
 0001:0009dd30       _G_CacheMapData            0049ed30 f   premap.obj
 0001:0009fc30       _G_UpdateScreenArea        004a0c30 f   premap.obj
 0001:0009fee0       _P_RandomSpawnPoint        004a0ee0 f   premap.obj
 0001:000a0160       _P_ResetPlayer             004a1160 f   premap.obj
 0001:000a05e0       _P_ResetStatus             004a15e0 f   premap.obj
 0001:000a0a90       _P_ResetWeapons            004a1a90 f   premap.obj
 0001:000a0b90       _P_ResetInventory          004a1b90 f   premap.obj
 0001:000a0c20       _G_NewGame                 004a1c20 f   premap.obj
 0001:000a0fd0       _G_ResetTimers             004a1fd0 f   premap.obj
 0001:000a1050       _G_ClearFIFO               004a2050 f   premap.obj
 0001:000a1160       _G_FindLevelByFile         004a2160 f   premap.obj
 0001:000a11f0       _G_SetupFilenameBasedMusic 004a21f0 f   premap.obj
 0001:000a1390       _G_EnterLevel              004a2390 f   premap.obj
 0001:000a4420       _G_FreeMapState            004a5420 f   premap.obj
 0001:000a45e0       _G_Util_PtrToIdx           004a55e0 f   savegame.obj
 0001:000a4690       _G_Util_PtrToIdx2          004a5690 f   savegame.obj
 0001:000a4740       _G_ResetInterpolations     004a5740 f   savegame.obj
 0001:000a4970       _ReadSaveGameHeaders       004a5970 f   savegame.obj
 0001:000a4aa0       _G_LoadSaveHeaderNew       004a5aa0 f   savegame.obj
 0001:000a4c30       _G_LoadPlayer              004a5c30 f   savegame.obj
 0001:000a50c0       _G_SavePlayer              004a60c0 f   savegame.obj
 0001:000a5350       _G_LoadPlayerMaybeMulti    004a6350 f   savegame.obj
 0001:000a53d0       _G_SavePlayerMaybeMulti    004a63d0 f   savegame.obj
 0001:000a5450       _sv_freemem                004a6450 f   savegame.obj
 0001:000a54b0       _sv_saveandmakesnapshot    004a64b0 f   savegame.obj
 0001:000a5db0       _sv_loadheader             004a6db0 f   savegame.obj
 0001:000a5fa0       _sv_loadsnapshot           004a6fa0 f   savegame.obj
 0001:000a6180       _sv_writediff              004a7180 f   savegame.obj
 0001:000a6e70       _sv_readdiff               004a7e70 f   savegame.obj
 0001:000a76b0       _sv_postyaxload            004a86b0 f   savegame.obj
 0001:000a8060       _sv_updatestate            004a9060 f   savegame.obj
 0001:000a9350       _S_FindMusicSFX            004aa350 f   sector.obj
 0001:000a93e0       _A_CallSound               004aa3e0 f   sector.obj
 0001:000a9640       _G_CheckActivatorMotion    004aa640 f   sector.obj
 0001:000a97d0       _CheckDoorTile             004aa7d0 f   sector.obj
 0001:000a9880       _isanunderoperator         004aa880 f   sector.obj
 0001:000a98d0       _isanearoperator           004aa8d0 f   sector.obj
 0001:000a9930       @A_FindPlayer@8            004aa930 f   sector.obj
 0001:000a9ab0       _G_DoSectorAnimations      004aaab0 f   sector.obj
 0001:000a9f20       _GetAnimationGoal          004aaf20 f   sector.obj
 0001:000a9f60       _SetAnimation              004aaf60 f   sector.obj
 0001:000aa040       _G_AnimateCamSprite        004ab040 f   sector.obj
 0001:000aa500       _G_AnimateWalls            004ab500 f   sector.obj
 0001:000aa920       _G_ActivateWarpElevators   004ab920 f   sector.obj
 0001:000aab30       _G_OperateSectors          004abb30 f   sector.obj
 0001:000ac480       _G_OperateRespawns         004ad480 f   sector.obj
 0001:000ac590       _G_OperateActivators       004ad590 f   sector.obj
 0001:000aca60       _G_OperateMasterSwitches   004ada60 f   sector.obj
 0001:000acb00       _G_OperateForceFields      004adb00 f   sector.obj
 0001:000acc50       _P_ActivateSwitch          004adc50 f   sector.obj
 0001:000addf0       _G_ActivateBySector        004aedf0 f   sector.obj
 0001:000ade90       _A_DamageWall              004aee90 f   sector.obj
 0001:000aedb0       _Sect_DamageCeilingOrFloor 004afdb0 f   sector.obj
 0001:000af280       _A_DamageObject            004b0280 f   sector.obj
 0001:000b1690       _G_AlignWarpElevators      004b2690 f   sector.obj
 0001:000b1830       _P_HandleSharedKeys        004b2830 f   sector.obj
 0001:000b2c00       _A_CheckHitSprite          004b3c00 f   sector.obj
 0001:000b2dc0       _P_CheckSectors            004b3dc0 f   sector.obj
 0001:000b4380       ??F?$WallTracker@F@@QAEFH@Z 004b5380 f i sector.obj
 0001:000b43c0       ??Z?$WallTracker@E@@QAEEE@Z 004b53c0 f i sector.obj
 0001:000b4460       ?RTS_Init@@YAXPBD@Z        004b5460 f   rts.obj
 0001:000b4770       ?RTS_IsInitialized@@YAHXZ  004b5770 f   rts.obj
 0001:000b4790       ?RTS_SoundLength@@YAHH@Z   004b5790 f   rts.obj
 0001:000b47d0       ?RTS_GetSound@@YAPAXH@Z    004b57d0 f   rts.obj
 0001:000b48e0       ?CONFIG_FunctionNameToNum@@YAHPBD@Z 004b58e0 f   config.obj
 0001:000b49a0       ?CONFIG_FunctionNumToName@@YAPADH@Z 004b59a0 f   config.obj
 0001:000b49c0       ?CONFIG_AnalogNameToNum@@YAHPBD@Z 004b59c0 f   config.obj
 0001:000b4a40       ?CONFIG_AnalogNumToName@@YAPBDH@Z 004b5a40 f   config.obj
 0001:000b4aa0       ?CONFIG_SetDefaultKeys@@YAXPAY0CA@$$CBD@Z 004b5aa0 f   config.obj
 0001:000b4b90       ?CONFIG_SetDefaults@@YAXXZ 004b5b90 f   config.obj
 0001:000b52b0       ?CONFIG_MapKey@@YAXHEEEE@Z 004b62b0 f   config.obj
 0001:000b5460       ?CONFIG_SetupMouse@@YAXXZ  004b6460 f   config.obj
 0001:000b5860       ?CONFIG_SetupJoystick@@YAXXZ 004b6860 f   config.obj
 0001:000b5cc0       ?CONFIG_ReadSetup@@YAHXZ   004b6cc0 f   config.obj
 0001:000b6310       ?CONFIG_WriteSettings@@YAXXZ 004b7310 f   config.obj
 0001:000b66c0       ?CONFIG_WriteSetup@@YAXI@Z 004b76c0 f   config.obj
 0001:000b7050       ?CONFIG_GetMapBestTime@@YAHPBDPBE@Z 004b8050 f   config.obj
 0001:000b7280       ?CONFIG_SetMapBestTime@@YAHPBEH@Z 004b8280 f   config.obj
 0001:000b7300       _ANIM_LoadAnim             004b8300 f   animlib.obj
 0001:000b76c0       _ANIM_FreeAnim             004b86c0 f   animlib.obj
 0001:000b76f0       _ANIM_NumFrames            004b86f0 f   animlib.obj
 0001:000b7700       _ANIM_DrawFrame            004b8700 f   animlib.obj
 0001:000b7b90       _ANIM_GetPalette           004b8b90 f   animlib.obj
 0001:000b7ba0       ?GAME_drawosdchar@@YAXHHDHH@Z 004b8ba0 f   osdfuncs.obj
 0001:000b7e10       ?GAME_drawosdstr@@YAXHHPBDHHH@Z 004b8e10 f   osdfuncs.obj
 0001:000b7fd0       ?GAME_drawosdcursor@@YAXHHHH@Z 004b8fd0 f   osdfuncs.obj
 0001:000b8130       ?GAME_getcolumnwidth@@YAHH@Z 004b9130 f   osdfuncs.obj
 0001:000b8170       ?GAME_getrowheight@@YAHH@Z 004b9170 f   osdfuncs.obj
 0001:000b81a0       ?GAME_onshowosd@@YAXH@Z    004b91a0 f   osdfuncs.obj
 0001:000b81d0       ?GAME_clearbackground@@YAXHH@Z 004b91d0 f   osdfuncs.obj
 0001:000b8400       _osdcmd_restartvid         004b9400 f   osdcmds.obj
 0001:000b8460       ?osdcmd_restartmap@@YAHPBUosdfuncparm_t@@@Z 004b9460 f   osdcmds.obj
 0001:000b84b0       _onvideomodechange         004b94b0 f   osdcmds.obj
 0001:000b85b0       _registerosdcommands       004b95b0 f   osdcmds.obj
 0001:000bc7a0       _FindGroup                 004bd7a0 f   grpscan.obj
 0001:000bc7e0       _ScanGroups                004bd7e0 f   grpscan.obj
 0001:000bd600       _FreeGroups                004be600 f   grpscan.obj
 0001:000be0c0       ?G_GetVersionFromWebsite@@YAHPAD@Z 004bf0c0 f   winbits.obj
 0001:000be390       _startwin_open             004bf390 f   startwin.game.obj
 0001:000bf7f0       _startwin_close            004c07f0 f   startwin.game.obj
 0001:000bf820       _startwin_puts             004c0820 f   startwin.game.obj
 0001:000bfa50       _startwin_settitle         004c0a50 f   startwin.game.obj
 0001:000bfa80       _startwin_idle             004c0a80 f   startwin.game.obj
 0001:000bfac0       _startwin_run              004c0ac0 f   startwin.game.obj
 0001:000bfda0       ?SafeOpen@@YAHPBDHH@Z      004c0da0 f   file_lib.obj
 0001:000bfe90       _SafeOpenRead              004c0e90 f   file_lib.obj
 0001:000bfef0       _SafeClose                 004c0ef0 f   file_lib.obj
 0001:000bff80       _SafeFileExists            004c0f80 f   file_lib.obj
 0001:000bffa0       _SafeFileLength            004c0fa0 f   file_lib.obj
 0001:000bffc0       _SafeRead                  004c0fc0 f   file_lib.obj
 0001:000c0050       _CONTROL_ClearAllBinds     004c1050 f   control.obj
 0001:000c00b0       _CONTROL_BindKey           004c10b0 f   control.obj
 0001:000c0110       _CONTROL_BindMouse         004c1110 f   control.obj
 0001:000c0170       _CONTROL_FreeKeyBind       004c1170 f   control.obj
 0001:000c01c0       _CONTROL_FreeMouseBind     004c11c0 f   control.obj
 0001:000c0210       _CONTROL_DefineFlag        004c1210 f   control.obj
 0001:000c0260       _CONTROL_FlagActive        004c1260 f   control.obj
 0001:000c0280       _CONTROL_MapButton         004c1280 f   control.obj
 0001:000c02f0       _CONTROL_MapAnalogAxis     004c12f0 f   control.obj
 0001:000c0350       _CONTROL_SetAnalogAxisScale 004c1350 f   control.obj
 0001:000c03a0       _CONTROL_MapDigitalAxis    004c13a0 f   control.obj
 0001:000c0440       _CONTROL_ClearAssignments  004c1440 f   control.obj
 0001:000c0530       _CONTROL_ClearButton       004c1530 f   control.obj
 0001:000c0580       _CONTROL_ProcessBinds      004c1580 f   control.obj
 0001:000c0620       _CONTROL_GetInput          004c1620 f   control.obj
 0001:000c1170       _CONTROL_Startup           004c2170 f   control.obj
 0001:000c1370       _CONTROL_Shutdown          004c2370 f   control.obj
 0001:000c13a0       _KB_ClearKeysDown          004c23a0 f   keyboard.obj
 0001:000c13c0       _KB_ScanCodeToString       004c23c0 f   keyboard.obj
 0001:000c1410       _KB_StringToScanCode       004c2410 f   keyboard.obj
 0001:000c1460       _KB_Startup                004c2460 f   keyboard.obj
 0001:000c14a0       _KB_Shutdown               004c24a0 f   keyboard.obj
 0001:000c14b0       _Mouse_Init                004c24b0 f   mouse.obj
 0001:000c14d0       _MOUSE_Shutdown            004c24d0 f   mouse.obj
 0001:000c14e0       _MOUSE_GetButtons          004c24e0 f   mouse.obj
 0001:000c1500       _JOYSTICK_GetButtons       004c2500 f   joystick.obj
 0001:000c1520       _JOYSTICK_ClearButton      004c2520 f   joystick.obj
 0001:000c1540       _JOYSTICK_ClearAllButtons  004c2540 f   joystick.obj
 0001:000c1550       _JOYSTICK_GetHat           004c2550 f   joystick.obj
 0001:000c15c0       _JOYSTICK_ClearHat         004c25c0 f   joystick.obj
 0001:000c15f0       _JOYSTICK_ClearAllHats     004c25f0 f   joystick.obj
 0001:000c1630       _JOYSTICK_GetAxis          004c2630 f   joystick.obj
 0001:000c1670       _JOYSTICK_ClearAxis        004c2670 f   joystick.obj
 0001:000c16a0       _JOYSTICK_ClearAllAxes     004c26a0 f   joystick.obj
 0001:000c16e0       _SCRIPT_New                004c26e0 f   scriplib.obj
 0001:000c1790       _SCRIPT_Delete             004c2790 f   scriplib.obj
 0001:000c1870       _SCRIPT_FreeSection        004c2870 f   scriplib.obj
 0001:000c1930       _SCRIPT_SectionExists      004c2930 f   scriplib.obj
 0001:000c19d0       _SCRIPT_AddSection         004c29d0 f   scriplib.obj
 0001:000c1af0       _SCRIPT_EntryExists        004c2af0 f   scriplib.obj
 0001:000c1b70       _SCRIPT_AddEntry           004c2b70 f   scriplib.obj
 0001:000c1cb0       ?SCRIPT_ParseBuffer@@YAHHPADH@Z 004c2cb0 f   scriplib.obj
 0001:000c2330       _SCRIPT_Init               004c3330 f   scriplib.obj
 0001:000c2370       _SCRIPT_Free               004c3370 f   scriplib.obj
 0001:000c2390       _SCRIPT_Load               004c3390 f   scriplib.obj
 0001:000c2460       _SCRIPT_Save               004c3460 f   scriplib.obj
 0001:000c25b0       _SCRIPT_NumberSections     004c35b0 f   scriplib.obj
 0001:000c2630       _SCRIPT_Section            004c3630 f   scriplib.obj
 0001:000c26b0       _SCRIPT_NumberEntries      004c36b0 f   scriplib.obj
 0001:000c2740       _SCRIPT_Entry              004c3740 f   scriplib.obj
 0001:000c27d0       _SCRIPT_GetRaw             004c37d0 f   scriplib.obj
 0001:000c2840       _SCRIPT_GetStringPtr       004c3840 f   scriplib.obj
 0001:000c2c00       _SCRIPT_GetString          004c3c00 f   scriplib.obj
 0001:000c2c20       _SCRIPT_GetDoubleString    004c3c20 f   scriplib.obj
 0001:000c2d00       _SCRIPT_GetNumber          004c3d00 f   scriplib.obj
 0001:000c2e40       _SCRIPT_GetBoolean         004c3e40 f   scriplib.obj
 0001:000c2f90       _SCRIPT_PutSection         004c3f90 f   scriplib.obj
 0001:000c2fb0       _SCRIPT_PutRaw             004c3fb0 f   scriplib.obj
 0001:000c2fd0       _SCRIPT_PutString          004c3fd0 f   scriplib.obj
 0001:000c31e0       _SCRIPT_PutDoubleString    004c41e0 f   scriplib.obj
 0001:000c35a0       _SCRIPT_PutNumber          004c45a0 f   scriplib.obj
 0001:000c3610       _SCRIPT_PutBoolean         004c4610 f   scriplib.obj
 0001:000c3650       _SCRIPT_PutDouble          004c4650 f   scriplib.obj
 0001:000c36a0       _S_SoundStartup            004c46a0 f   sounds.obj
 0001:000c3960       _S_SoundShutdown           004c4960 f   sounds.obj
 0001:000c39b0       _S_MusicStartup            004c49b0 f   sounds.obj
 0001:000c3a10       _S_MusicShutdown           004c4a10 f   sounds.obj
 0001:000c3a40       _S_PauseMusic              004c4a40 f   sounds.obj
 0001:000c3aa0       _S_PauseSounds             004c4aa0 f   sounds.obj
 0001:000c3b40       _S_MusicVolume             004c4b40 f   sounds.obj
 0001:000c3b80       _S_RestartMusic            004c4b80 f   sounds.obj
 0001:000c3c30       _S_MenuSound               004c4c30 f   sounds.obj
 0001:000c3d10       _S_PlayMusic               004c4d10 f   sounds.obj
 0001:000c3f20       _S_GetMusicPosition        004c4f20 f   sounds.obj
 0001:000c3f50       _S_SetMusicPosition        004c4f50 f   sounds.obj
 0001:000c3f80       _S_StopMusic               004c4f80 f   sounds.obj
 0001:000c3ff0       _S_Cleanup                 004c4ff0 f   sounds.obj
 0001:000c42a0       _S_LoadSound               004c52a0 f   sounds.obj
 0001:000c43b0       _S_PlaySound3D             004c53b0 f   sounds.obj
 0001:000c50f0       _S_PlaySound               004c60f0 f   sounds.obj
 0001:000c5490       _A_PlaySound               004c6490 f   sounds.obj
 0001:000c54f0       _S_StopEnvSound            004c64f0 f   sounds.obj
 0001:000c5610       _S_ChangeSoundPitch        004c6610 f   sounds.obj
 0001:000c56f0       _S_Update                  004c66f0 f   sounds.obj
 0001:000c5910       _S_Callback                004c6910 f   sounds.obj
 0001:000c5960       _S_ClearSoundLocks         004c6960 f   sounds.obj
 0001:000c59e0       _A_CheckSoundPlaying       004c69e0 f   sounds.obj
 0001:000c5a70       _A_CheckAnySoundPlaying    004c6a70 f   sounds.obj
 0001:000c5ae0       _S_CheckSoundPlaying       004c6ae0 f   sounds.obj
 0001:000c5b30       ?G_ProcessDynamicSoundMapping@@YAXPBDH@Z 004c6b30 f   soundsdyn.obj
 0001:000c5bc0       ?initsoundhashnames@@YAXXZ 004c6bc0 f   soundsdyn.obj
 0001:000c5c20       ?freesoundhashnames@@YAXXZ 004c6c20 f   soundsdyn.obj
 0001:000c5c40       ?G_InitDynamicSounds@@YAXXZ 004c6c40 f   soundsdyn.obj
 0001:000c5cb0       ??0MiniDumper@@QAE@PBD@Z   004c6cb0 f   mdump.obj
 0001:000c5d20       ?TopLevelFilter@MiniDumper@@CGJPAU_EXCEPTION_POINTERS@@@Z 004c6d20 f   mdump.obj
 0001:000c5f80       ?MIDI_AllNotesOff@@YAHXZ   004c6f80 f   midi.obj
 0001:000c6020       ?MIDI_Reset@@YAHXZ         004c7020 f   midi.obj
 0001:000c6150       ?MIDI_SetVolume@@YAHH@Z    004c7150 f   midi.obj
 0001:000c61d0       ?MIDI_ContinueSong@@YAXXZ  004c71d0 f   midi.obj
 0001:000c61f0       ?MIDI_PauseSong@@YAXXZ     004c71f0 f   midi.obj
 0001:000c6220       ?MIDI_SetMidiFuncs@@YAXPAUmidifuncs@@@Z 004c7220 f   midi.obj
 0001:000c6230       ?MIDI_StopSong@@YAXXZ      004c7230 f   midi.obj
 0001:000c6460       ?MIDI_PlaySong@@YAHPADH@Z  004c7460 f   midi.obj
 0001:000c7260       ?MIDI_SetTempo@@YAXH@Z     004c8260 f   midi.obj
 0001:000c72a0       ?MIDI_SetDivision@@YAXH@Z  004c82a0 f   midi.obj
 0001:000c78f0       ?MIDI_UpdateMusic@@YAXXZ   004c88f0 f   midi.obj
 0001:000c7920       ?MUSIC_ErrorString@@YAPBDH@Z 004c8920 f   music.obj
 0001:000c7990       ?MUSIC_Init@@YAHH@Z        004c8990 f   music.obj
 0001:000c79e0       ?MUSIC_Shutdown@@YAHXZ     004c89e0 f   music.obj
 0001:000c79f0       ?MUSIC_SetVolume@@YAXH@Z   004c89f0 f   music.obj
 0001:000c7a60       ?MUSIC_Continue@@YAXXZ     004c8a60 f   music.obj
 0001:000c7a70       ?MUSIC_Pause@@YAXXZ        004c8a70 f   music.obj
 0001:000c7a80       ?MUSIC_StopSong@@YAHXZ     004c8a80 f   music.obj
 0001:000c7aa0       ?MUSIC_PlaySong@@YAHPADH@Z 004c8aa0 f   music.obj
 0001:000c7ae0       ?MUSIC_InitMidi@@YAHPAUmidifuncs@@@Z 004c8ae0 f   music.obj
 0001:000c7b40       ?MUSIC_Update@@YAXXZ       004c8b40 f   music.obj
 0001:000c7b50       ?MPU_FinishBuffer@@YAXH@Z  004c8b50 f   mpu401.obj
 0001:000c7c10       ?MPU_BeginPlayback@@YAXXZ  004c8c10 f   mpu401.obj
 0001:000c7c40       ?MPU_Pause@@YAXXZ          004c8c40 f   mpu401.obj
 0001:000c7c60       ?MPU_Unpause@@YAXXZ        004c8c60 f   mpu401.obj
 0001:000c7c80       ?MPU_MIDICallback@@YGXPAUHMIDIOUT__@@IKKK@Z 004c8c80 f   mpu401.obj
 0001:000c7d00       ?MPU_GetNextBuffer@@YAHXZ  004c8d00 f   mpu401.obj
 0001:000c7d40       ?MPU_SendMidi@@YAXPADH@Z   004c8d40 f   mpu401.obj
 0001:000c7f80       ?MPU_Reset@@YAHXZ          004c8f80 f   mpu401.obj
 0001:000c7fa0       ?MPU_Init@@YAHH@Z          004c8fa0 f   mpu401.obj
 0001:000c8020       ?MPU_NoteOff@@YAXDDD@Z     004c9020 f   mpu401.obj
 0001:000c8050       ?MPU_NoteOn@@YAXDDD@Z      004c9050 f   mpu401.obj
 0001:000c8080       ?MPU_PolyAftertouch@@YAXDDD@Z 004c9080 f   mpu401.obj
 0001:000c80b0       ?MPU_ControlChange@@YAXDDD@Z 004c90b0 f   mpu401.obj
 0001:000c80e0       ?MPU_ProgramChange@@YAXDD@Z 004c90e0 f   mpu401.obj
 0001:000c8110       ?MPU_ChannelAftertouch@@YAXDD@Z 004c9110 f   mpu401.obj
 0001:000c8140       ?MPU_PitchBend@@YAXDDD@Z   004c9140 f   mpu401.obj
 0001:000c8170       ?MPU_SetTempo@@YAXH@Z      004c9170 f   mpu401.obj
 0001:000c81b0       ?MPU_SetDivision@@YAXH@Z   004c91b0 f   mpu401.obj
 0001:000c81e0       _mousepressstateadvance    004c91e0 f   baselayer.obj
 0001:000c8240       _setkeypresscallback       004c9240 f   baselayer.obj
 0001:000c8250       _setmousepresscallback     004c9250 f   baselayer.obj
 0001:000c8260       _setjoypresscallback       004c9260 f   baselayer.obj
 0001:000c8270       _GetKey                    004c9270 f   baselayer.obj
 0001:000c8290       _SetKey                    004c9290 f   baselayer.obj
 0001:000c82f0       _bgetchar                  004c92f0 f   baselayer.obj
 0001:000c8340       _bflushchars               004c9340 f   baselayer.obj
 0001:000c8370       _getkeyname                004c9370 f   baselayer.obj
 0001:000c83a0       _readmousexy               004c93a0 f   baselayer.obj
 0001:000c8410       _readmouseabsxy            004c9410 f   baselayer.obj
 0001:000c8610       _readmousebstatus          004c9610 f   baselayer.obj
 0001:000c8670       _readjoybstatus            004c9670 f   baselayer.obj
 0001:000c86a0       ?nx_unprotect@@YAHHH@Z     004c96a0 f   baselayer.obj
 0001:000c86e0       _calc_ylookup              004c96e0 f   baselayer.obj
 0001:000c8870       _makeasmwriteable          004c9870 f   baselayer.obj
 0001:000c8890       _fullscreen_tint_gl        004c9890 f   baselayer.obj
 0001:000c8990       _osdcmd_glinfo             004c9990 f   baselayer.obj
 0001:000c8d40       _baselayer_init            004c9d40 f   baselayer.obj
 0001:000c9410       _maybe_redirect_outputs    004ca410 f   baselayer.obj
 0001:000c94d0       _kpzbufloadfil             004ca4d0 f   cache1d.obj
 0001:000c9590       _kpzbufload                004ca590 f   cache1d.obj
 0001:000c95e0       _initcache                 004ca5e0 f   cache1d.obj
 0001:000c9690       _allocache                 004ca690 f   cache1d.obj
 0001:000c9a60       _agecache                  004caa60 f   cache1d.obj
 0001:000c9ca0       _listsearchpath            004caca0 f   cache1d.obj
 0001:000c9d00       _addsearchpath_user        004cad00 f   cache1d.obj
 0001:000c9f90       _removesearchpath          004caf90 f   cache1d.obj
 0001:000ca120       _removesearchpaths_withuser 004cb120 f   cache1d.obj
 0001:000ca1c0       _findfrompath              004cb1c0 f   cache1d.obj
 0001:000ca3f0       _openfrompath              004cb3f0 f   cache1d.obj
 0001:000ca470       _fopenfrompath             004cb470 f   cache1d.obj
 0001:000ca640       _cache1d_file_fromzip      004cb640 f   cache1d.obj
 0001:000ca660       _initgroupfile             004cb660 f   cache1d.obj
 0001:000caed0       _uninitgroupfile           004cbed0 f   cache1d.obj
 0001:000cb540       _krename                   004cc540 f   cache1d.obj
 0001:000cb5b0       _kfileparent               004cc5b0 f   cache1d.obj
 0001:000cb5f0       _kopen4load                004cc5f0 f   cache1d.obj
 0001:000cb6b0       ?kread_internal@@YAHHPAXHPAEPAH2@Z 004cc6b0 f   cache1d.obj
 0001:000cb900       ?klseek_internal@@YAHHHHPAEPAH1@Z 004cc900 f   cache1d.obj
 0001:000cba60       ?kfilelength_internal@@YAHHPAEPAH1@Z 004cca60 f   cache1d.obj
 0001:000cbb60       ?ktell_internal@@YAHHPAEPAH1@Z 004ccb60 f   cache1d.obj
 0001:000cbc30       ?kclose_internal@@YAXHPAEPAH@Z 004ccc30 f   cache1d.obj
 0001:000cbc90       _kread                     004ccc90 f   cache1d.obj
 0001:000cbcc0       _klseek                    004cccc0 f   cache1d.obj
 0001:000cbcf0       _kfilelength               004cccf0 f   cache1d.obj
 0001:000cbd10       _ktell                     004ccd10 f   cache1d.obj
 0001:000cbd30       _kclose                    004ccd30 f   cache1d.obj
 0001:000cbdd0       _klistfree                 004ccdd0 f   cache1d.obj
 0001:000cbe00       _klistpath                 004cce00 f   cache1d.obj
 0001:000cc880       _kdfread                   004cd880 f   cache1d.obj
 0001:000ccb20       _dfwrite                   004cdb20 f   cache1d.obj
 0001:000cd5a0       _clearDefNamePtr           004ce5a0 f   common.obj
 0001:000cd5c0       _G_AddDef                  004ce5c0 f   common.obj
 0001:000cd6a0       _G_AddDefModule            004ce6a0 f   common.obj
 0001:000cd780       _G_AddClipMap              004ce780 f   common.obj
 0001:000cd800       _getatoken                 004ce800 f   common.obj
 0001:000cd880       _G_CheckCmdSwitch          004ce880 f   common.obj
 0001:000cd8d0       _testkopen                 004ce8d0 f   common.obj
 0001:000cd910       _check_file_exist          004ce910 f   common.obj
 0001:000cd9d0       _fnlist_clearnames         004ce9d0 f   common.obj
 0001:000cda20       _fnlist_getnames           004cea20 f   common.obj
 0001:000cdae0       _maybe_append_ext          004ceae0 f   common.obj
 0001:000cdba0       _ldist                     004ceba0 f   common.obj
 0001:000cdc80       _dist                      004cec80 f   common.obj
 0001:000cdd80       _FindDistance2D            004ced80 f   common.obj
 0001:000cdda0       _FindDistance3D            004ceda0 f   common.obj
 0001:000cddc0       _COMMON_clearbackground    004cedc0 f   common.obj
 0001:000cdf30       _xalloc_set_location       004cef30 f   compat.obj
 0001:000cdf60       _handle_memerr             004cef60 f   compat.obj
 0001:000cdfc0       _set_memerr_handler        004cefc0 f   compat.obj
 0001:000cdfd0       _Bgethomedir               004cefd0 f   compat.obj
 0001:000ce0c0       _Bgetappdir                004cf0c0 f   compat.obj
 0001:000ce150       _Bcorrectfilename          004cf150 f   compat.obj
 0001:000ce3f0       _Bcanonicalisefilename     004cf3f0 f   compat.obj
 0001:000ce5e0       _Bgetsystemdrives          004cf5e0 f   compat.obj
 0001:000ce6e0       _Bfilelength               004cf6e0 f   compat.obj
 0001:000ce750       _Bopendir                  004cf750 f   compat.obj
 0001:000ce8c0       _Breaddir                  004cf8c0 f   compat.obj
 0001:000cea50       _Bclosedir                 004cfa50 f   compat.obj
 0001:000cea80       _Bstrtoken                 004cfa80 f   compat.obj
 0001:000ceb70       _Bstrtolower               004cfb70 f   compat.obj
 0001:000cebe0       _Bgetsysmemsize            004cfbe0 f   compat.obj
 0001:000cec90       ?libdivide_u32_gen@@YA?AUlibdivide_u32_t@@I@Z 004cfc90 f   compat.obj
 0001:000cee30       ?libdivide_u32_do@@YAIIPBUlibdivide_u32_t@@@Z 004cfe30 f   compat.obj
 0001:000cef00       ?libdivide_u32_get_algorithm@@YAHPBUlibdivide_u32_t@@@Z 004cff00 f   compat.obj
 0001:000cef40       ?libdivide_u32_do_alg0@@YAIIPBUlibdivide_u32_t@@@Z 004cff40 f   compat.obj
 0001:000cef60       ?libdivide_u32_do_alg1@@YAIIPBUlibdivide_u32_t@@@Z 004cff60 f   compat.obj
 0001:000cef90       ?libdivide_u32_do_alg2@@YAIIPBUlibdivide_u32_t@@@Z 004cff90 f   compat.obj
 0001:000cefd0       ?libdivide_u64_gen@@YA?AUlibdivide_u64_t@@_K@Z 004cffd0 f   compat.obj
 0001:000cf580       ?libdivide_u64_do@@YA_K_KPBUlibdivide_u64_t@@@Z 004d0580 f   compat.obj
 0001:000cf720       ?libdivide_u64_get_algorithm@@YAHPBUlibdivide_u64_t@@@Z 004d0720 f   compat.obj
 0001:000cf760       ?libdivide_u64_do_alg0@@YA_K_KPBUlibdivide_u64_t@@@Z 004d0760 f   compat.obj
 0001:000cf780       ?libdivide_u64_do_alg1@@YA_K_KPBUlibdivide_u64_t@@@Z 004d0780 f   compat.obj
 0001:000cf7c0       ?libdivide_u64_do_alg2@@YA_K_KPBUlibdivide_u64_t@@@Z 004d07c0 f   compat.obj
 0001:000cf820       ?libdivide_s32_gen@@YA?AUlibdivide_s32_t@@H@Z 004d0820 f   compat.obj
 0001:000cf960       ?libdivide_s32_do@@YAHHPBUlibdivide_s32_t@@@Z 004d0960 f   compat.obj
 0001:000cfa70       ?libdivide_s32_get_algorithm@@YAHPBUlibdivide_s32_t@@@Z 004d0a70 f   compat.obj
 0001:000cfad0       ?libdivide_s32_do_alg0@@YAHHPBUlibdivide_s32_t@@@Z 004d0ad0 f   compat.obj
 0001:000cfb10       ?libdivide_s32_do_alg1@@YAHHPBUlibdivide_s32_t@@@Z 004d0b10 f   compat.obj
 0001:000cfb50       ?libdivide_s32_do_alg2@@YAHHPBUlibdivide_s32_t@@@Z 004d0b50 f   compat.obj
 0001:000cfba0       ?libdivide_s32_do_alg3@@YAHHPBUlibdivide_s32_t@@@Z 004d0ba0 f   compat.obj
 0001:000cfbf0       ?libdivide_s32_do_alg4@@YAHHPBUlibdivide_s32_t@@@Z 004d0bf0 f   compat.obj
 0001:000cfc40       ?libdivide_s64_gen@@YA?AUlibdivide_s64_t@@_J@Z 004d0c40 f   compat.obj
 0001:000cfe90       ?libdivide_s64_do@@YA_J_JPBUlibdivide_s64_t@@@Z 004d0e90 f   compat.obj
 0001:000d00f0       ?libdivide_s64_get_algorithm@@YAHPBUlibdivide_s64_t@@@Z 004d10f0 f   compat.obj
 0001:000d0160       ?libdivide_s64_do_alg0@@YA_J_JPBUlibdivide_s64_t@@@Z 004d1160 f   compat.obj
 0001:000d01c0       ?libdivide_s64_do_alg1@@YA_J_JPBUlibdivide_s64_t@@@Z 004d11c0 f   compat.obj
 0001:000d0230       ?libdivide_s64_do_alg2@@YA_J_JPBUlibdivide_s64_t@@@Z 004d1230 f   compat.obj
 0001:000d02d0       ?libdivide_s64_do_alg3@@YA_J_JPBUlibdivide_s64_t@@@Z 004d12d0 f   compat.obj
 0001:000d0370       ?libdivide_s64_do_alg4@@YA_J_JPBUlibdivide_s64_t@@@Z 004d1370 f   compat.obj
 0001:000d0400       _Bcrc32                    004d1400 f   crc32.obj
 0001:000d04d0       _initcrc32table            004d14d0 f   crc32.obj
 0001:000d05f0       _loaddefinitionsfile       004d15f0 f   defs.obj
 0001:000d7f50       _initfastcolorlookup_scale 004d8f50 f   colmatch.obj
 0001:000d8010       _initfastcolorlookup_palette 004d9010 f   colmatch.obj
 0001:000d8130       _initfastcolorlookup_gridvectors 004d9130 f   colmatch.obj
 0001:000d8220       _getclosestcol_flush       004d9220 f   colmatch.obj
 0001:000d8250       _getclosestcol_lim         004d9250 f   colmatch.obj
 0001:000d8460       _getclosestcol_nocache_lim 004d9460 f   colmatch.obj
 0001:000d8750       _compare_usermaphacks      004d9750 f   engine.obj
 0001:000d8770       _get_alwaysshowgray        004d9770 f   engine.obj
 0001:000d87b0       _yax_updategrays           004d97b0 f   engine.obj
 0001:000d8b80       _yax_getbunch              004d9b80 f   engine.obj
 0001:000d8bf0       _yax_setbunch              004d9bf0 f   engine.obj
 0001:000d8d80       _yax_setbunches            004d9d80 f   engine.obj
 0001:000d8db0       _yax_getnextwall           004d9db0 f   engine.obj
 0001:000d8e50       _yax_setnextwall           004d9e50 f   engine.obj
 0001:000d8f20       _yax_vnextsec              004d9f20 f   engine.obj
 0001:000d8f80       _yax_update                004d9f80 f   engine.obj
 0001:000d9510       _yax_getneighborsect       004da510 f   engine.obj
 0001:000d95a0       _yax_tweakpicnums          004da5a0 f   engine.obj
 0001:000d9930       _yax_preparedrawrooms      004da930 f   engine.obj
 0001:000d9a50       _yax_drawrooms             004daa50 f   engine.obj
 0001:000daa60       _setslope                  004dba60 f   engine.obj
 0001:000dab90       _clipmapinfo_load          004dbb90 f   engine.obj
 0001:000dc5c0       _clipshape_idx_for_sprite  004dd5c0 f   engine.obj
 0001:000dc660       _checksectorpointer        004dd660 f   engine.obj
 0001:000dce60       _fade_screen_black         004dde60 f   engine.obj
 0001:000dcfc0       _engine_addtsprite         004ddfc0 f   engine.obj
 0001:000dde60       _wallfront                 004dee60 f   engine.obj
 0001:000de0c0       _animateoffs               004df0c0 f   engine.obj
 0001:000de190       _dorotspr_handle_bit2      004df190 f   engine.obj
 0001:000de4c0       _E_ReplaceTransparentColorWithBlack 004df4c0 f   engine.obj
 0001:000de5f0       _loadlookups               004df5f0 f   engine.obj
 0001:000de6f0       _generatefogpals           004df6f0 f   engine.obj
 0001:000de7c0       _fillemptylookups          004df7c0 f   engine.obj
 0001:000de860       _do_insertsprite_at_headofsect 004df860 f   engine.obj
 0001:000de8e0       _do_deletespritesect       004df8e0 f   engine.obj
 0001:000de970       _do_insertsprite_at_headofstat 004df970 f   engine.obj
 0001:000de9f0       _insertspritestat          004df9f0 f   engine.obj
 0001:000dea80       _insertsprite              004dfa80 f   engine.obj
 0001:000deaf0       _deletesprite              004dfaf0 f   engine.obj
 0001:000decd0       _changespritesect          004dfcd0 f   engine.obj
 0001:000ded60       _changespritestat          004dfd60 f   engine.obj
 0001:000dedf0       _lintersect                004dfdf0 f   engine.obj
 0001:000defd0       _rayintersect              004dffd0 f   engine.obj
 0001:000df330       _E_DefinePsky              004e0330 f   engine.obj
 0001:000df430       _preinitengine             004e0430 f   engine.obj
 0001:000df520       _initengine                004e0520 f   engine.obj
 0001:000e00e0       _E_PostInit                004e10e0 f   engine.obj
 0001:000e0390       _uninitengine              004e1390 f   engine.obj
 0001:000e0600       _initspritelists           004e1600 f   engine.obj
 0001:000e0760       _set_globalang             004e1760 f   engine.obj
 0001:000e07f0       _drawrooms                 004e17f0 f   engine.obj
 0001:000e8fd0       _wallvisible               004e9fd0 f   engine.obj
 0001:000e9080       _drawmasks                 004ea080 f   engine.obj
 0001:000f29e0       _drawmapview               004f39e0 f   engine.obj
 0001:000f57f0       _E_MapArt_Clear            004f67f0 f   engine.obj
 0001:000f5a00       _E_MapArt_Setup            004f6a00 f   engine.obj
 0001:000f5ba0       _loadboard                 004f6ba0 f   engine.obj
 0001:000f6f10       _loadoldboard              004f7f10 f   engine.obj
 0001:000f8340       _delete_maphack_lights     004f9340 f   engine.obj
 0001:000f83b0       _loadmaphack               004f93b0 f   engine.obj
 0001:000f8bb0       _saveboard                 004f9bb0 f   engine.obj
 0001:000f97e0       _setgamemode               004fa7e0 f   engine.obj
 0001:000f9dc0       _nextpage                  004fadc0 f   engine.obj
 0001:000fc580       _E_CreateDummyTile         004fd580 f   engine.obj
 0001:000fc5e0       _E_CreateFakeTile          004fd5e0 f   engine.obj
 0001:000fc700       _E_UndefineTile            004fd700 f   engine.obj
 0001:000fc840       _set_tilesiz               004fd840 f   engine.obj
 0001:000fc870       _tile_exists               004fd870 f   engine.obj
 0001:000fc8d0       _E_ReadArtFileHeader       004fd8d0 f   engine.obj
 0001:000fca10       _E_ReadArtFileHeaderFromBuffer 004fda10 f   engine.obj
 0001:000fcb00       _E_CheckUnitArtFileHeader  004fdb00 f   engine.obj
 0001:000fcb60       _E_ConvertARTv1picanmToMemory 004fdb60 f   engine.obj
 0001:000fcbd0       _E_ReadArtFileTileInfo     004fdbd0 f   engine.obj
 0001:000fcd30       _E_ReadArtFileIntoFakeData 004fdd30 f   engine.obj
 0001:000fd130       _loadpics                  004fe130 f   engine.obj
 0001:000fd290       _loadtile                  004fe290 f   engine.obj
 0001:000fd330       _E_LoadTileIntoBuffer      004fe330 f   engine.obj
 0001:000fd4c0       _E_RenderArtDataIntoBuffer 004fe4c0 f   engine.obj
 0001:000fd590       _allocatepermanenttile     004fe590 f   engine.obj
 0001:000fd630       _copytilepiece             004fe630 f   engine.obj
 0001:000fd7d0       _qloadkvx                  004fe7d0 f   engine.obj
 0001:000fd940       _clipinsidebox             004fe940 f   engine.obj
 0001:000fdaf0       _clipinsideboxline         004feaf0 f   engine.obj
 0001:000fdc50       _inside                    004fec50 f   engine.obj
 0001:000fde00       @getangle@8                004fee00 f   engine.obj
 0001:000fdf50       _ksqrt                     004fef50 f   engine.obj
 0001:000fdf70       _spriteheightofsptr        004fef70 f   engine.obj
 0001:000fe000       _setsprite                 004ff000 f   engine.obj
 0001:000fe0b0       _setspritez                004ff0b0 f   engine.obj
 0001:000fe170       _nextsectorneighborz       004ff170 f   engine.obj
 0001:000fe2c0       _cansee                    004ff2c0 f   engine.obj
 0001:000fed60       _hitscan                   004ffd60 f   engine.obj
 0001:001005b0       _neartag                   005015b0 f   engine.obj
 0001:00100b00       _dragpoint                 00501b00 f   engine.obj
 0001:00100e70       _lastwall                  00501e70 f   engine.obj
 0001:001013f0       _clipmovex                 005023f0 f   engine.obj
 0001:00101450       _clipmove                  00502450 f   engine.obj
 0001:00103500       _pushmove                  00504500 f   engine.obj
 0001:00103a70       _bfirst_search_init        00504a70 f   engine.obj
 0001:00103ad0       _bfirst_search_try         00504ad0 f   engine.obj
 0001:00103b50       _updatesector              00504b50 f   engine.obj
 0001:00103cb0       _updatesectorbreadth       00504cb0 f   engine.obj
 0001:00103e10       _updatesectorexclude       00504e10 f   engine.obj
 0001:00103fb0       _updatesectorz             00504fb0 f   engine.obj
 0001:00104260       _rotatepoint               00505260 f   engine.obj
 0001:00104300       _getmousevalues            00505300 f   engine.obj
 0001:00104330       _getzrange                 00505330 f   engine.obj
 0001:001055c0       _setaspect_new             005065c0 f   engine.obj
 0001:00105740       _setview                   00506740 f   engine.obj
 0001:001058f0       _setaspect                 005068f0 f   engine.obj
 0001:00105970       _flushperms                00506970 f   engine.obj
 0001:00105990       _rotatesprite_             00506990 f   engine.obj
 0001:00105f70       _setblendtab               00506f70 f   engine.obj
 0001:00105fd0       _removeblendtab            00506fd0 f   engine.obj
 0001:00106000       _setpalookup               00507000 f   engine.obj
 0001:00106050       _removepalookup            00507050 f   engine.obj
 0001:00106120       _makepalookup              00507120 f   engine.obj
 0001:00106390       _setbasepal                00507390 f   engine.obj
 0001:001063f0       _removebasepal             005073f0 f   engine.obj
 0001:00106440       _setbrightness             00507440 f   engine.obj
 0001:00106870       _setpalettefade            00507870 f   engine.obj
 0001:00106900       _clearview                 00507900 f   engine.obj
 0001:00106a40       _clearallviews             00507a40 f   engine.obj
 0001:00106b40       _plotpixel                 00507b40 f   engine.obj
 0001:00106d30       _plotlines2d               00507d30 f   engine.obj
 0001:00106e40       _getpixel                  00507e40 f   engine.obj
 0001:00106ea0       _setviewtotile             00507ea0 f   engine.obj
 0001:00107040       _setviewback               00508040 f   engine.obj
 0001:001071d0       _squarerotatetile          005081d0 f   engine.obj
 0001:00107470       _preparemirror             00508470 f   engine.obj
 0001:001075b0       _completemirror            005085b0 f   engine.obj
 0001:00107730       _sectorofwall              00508730 f   engine.obj
 0001:00107880       _sectorofwall_noquick      00508880 f   engine.obj
 0001:001078b0       _getceilzofslopeptr        005088b0 f   engine.obj
 0001:00107a10       _getflorzofslopeptr        00508a10 f   engine.obj
 0001:00107b40       _getzsofslopeptr           00508b40 f   engine.obj
 0001:00107ce0       _alignceilslope            00508ce0 f   engine.obj
 0001:00107e50       _alignflorslope            00508e50 f   engine.obj
 0001:00107fc0       _loopnumofsector           00508fc0 f   engine.obj
 0001:00108060       _setfirstwall              00509060 f   engine.obj
 0001:001084c0       _drawline256               005094c0 f   engine.obj
 0001:00108ab0       _drawline16                00509ab0 f   engine.obj
 0001:00109050       _drawcircle16              0050a050 f   engine.obj
 0001:001096e0       _qsetmodeany               0050a6e0 f   engine.obj
 0001:001097e0       _clear2dscreen             0050a7e0 f   engine.obj
 0001:00109840       _scalescreeny              0050a840 f   engine.obj
 0001:00109880       _screencoords              0050a880 f   engine.obj
 0001:00109900       _getinvdisplacement        0050a900 f   engine.obj
 0001:001099b0       _getscreenvdisp            0050a9b0 f   engine.obj
 0001:001099d0       _setup_sideview_sincos     0050a9d0 f   engine.obj
 0001:00109ab0       _draw2dgrid                0050aab0 f   engine.obj
 0001:0010a350       _getspritecol              0050b350 f   engine.obj
 0001:0010a5c0       _draw2dscreen              0050b5c0 f   engine.obj
 0001:0010c830       _printext16                0050d830 f   engine.obj
 0001:0010cda0       _printext256               0050dda0 f   engine.obj
 0001:0010cfd0       _screencapture             0050dfd0 f   engine.obj
 0001:0010d790       _setrendermode             0050e790 f   engine.obj
 0001:0010d900       _setrollangle              0050e900 f   engine.obj
 0001:0010d920       _invalidatetile            0050e920 f   engine.obj
 0001:0010da20       _setpolymost2dview         0050ea20 f   engine.obj
 0001:0010daf0       _hash_init                 0050eaf0 f   engine.obj
 0001:0010db40       _hash_loop                 0050eb40 f   engine.obj
 0001:0010dbb0       _hash_free                 0050ebb0 f   engine.obj
 0001:0010dc50       _hash_add                  0050ec50 f   engine.obj
 0001:0010de40       _hash_delete               0050ee40 f   engine.obj
 0001:0010df10       _hash_find                 0050ef10 f   engine.obj
 0001:0010df90       _hash_findcase             0050ef90 f   engine.obj
 0001:0010e010       _inthash_init              0050f010 f   engine.obj
 0001:0010e070       _inthash_loop              0050f070 f   engine.obj
 0001:0010e0e0       _inthash_free              0050f0e0 f   engine.obj
 0001:0010e100       _inthash_add               0050f100 f   engine.obj
 0001:0010e290       _inthash_delete            0050f290 f   engine.obj
 0001:0010e350       _inthash_find              0050f350 f   engine.obj
 0001:0010e640       _atanf                     0050f640 f i engine.obj
 0001:0010e660       _sinf                      0050f660 f i engine.obj
 0001:0010e680       _powf                      0050f680 f i engine.obj
 0001:0010e6b0       ??I?$SectorTracker@E@@QAEPAEXZ 0050f6b0 f i engine.obj
 0001:0010e6b0       ??I?$SectorTracker@F@@QAEPAFXZ 0050f6b0 f i engine.obj
 0001:0010e6d0       ??I?$WallTracker@G@@QAEPAGXZ 0050f6d0 f i engine.obj
 0001:0010e6d0       ??I?$WallTracker@F@@QAEPAFXZ 0050f6d0 f i engine.obj
 0001:0010e6f0       ??Y?$WallTracker@H@@QAEHH@Z 0050f6f0 f i engine.obj
 0001:0010e780       ??Z?$WallTracker@H@@QAEHH@Z 0050f780 f i engine.obj
 0001:0010e810       ??X?$WallTracker@H@@QAEHH@Z 0050f810 f i engine.obj
 0001:0010e8a0       ??Y?$WallTracker@F@@QAEFF@Z 0050f8a0 f i engine.obj
 0001:0010e940       ??Z?$WallTracker@F@@QAEFF@Z 0050f940 f i engine.obj
 0001:0010e9f0       ?loadgldriver@@YAHPBD@Z    0050f9f0 f   glbuild.obj
 0001:0010f4f0       ?loadglextensions@@YAHXZ   005104f0 f   glbuild.obj
 0001:00110180       ?unloadgldriver@@YAHXZ     00511180 f   glbuild.obj
 0001:00110a60       ?loadglulibrary@@YAHPBD@Z  00511a60 f   glbuild.obj
 0001:00110c80       ?unloadglulibrary@@YAHXZ   00511c80 f   glbuild.obj
 0001:00110d60       ?texcache_fetchmulti@@YAPAUpthtyp_t@@PAU1@PAUhicreplc_t@@HH@Z 00511d60 f   texcache.obj
 0001:00110f30       _texcache_fetch            00511f30 f   texcache.obj
 0001:00111650       _texcache_freeptrs         00512650 f   texcache.obj
 0001:00111740       _texcache_syncmemcache     00512740 f   texcache.obj
 0001:00111870       _texcache_init             00512870 f   texcache.obj
 0001:00111940       _texcache_openfiles        00512940 f   texcache.obj
 0001:00111a60       _texcache_checkgarbage     00512a60 f   texcache.obj
 0001:00111b70       _texcache_invalidate       00512b70 f   texcache.obj
 0001:00111bf0       _texcache_loadoffsets      00512bf0 f   texcache.obj
 0001:00111e60       _texcache_readdata         00512e60 f   texcache.obj
 0001:00111f00       _texcache_readtexheader    00512f00 f   texcache.obj
 0001:001122e0       _texcache_writetex         005132e0 f   texcache.obj
 0001:00112a10       _texcache_loadskin         00513a10 f   texcache.obj
 0001:00112e20       _texcache_loadtile         00513e20 f   texcache.obj
 0001:00112ec0       _texcache_setupmemcache    00513ec0 f   texcache.obj
 0001:001134d0       _kpgetdim                  005144d0 f   kplib.obj
 0001:00113a80       _kprender                  00514a80 f   kplib.obj
 0001:00119f00       _wildmatch                 0051af00 f   kplib.obj
 0001:0011a060       _kzuninit                  0051b060 f   kplib.obj
 0001:0011a0b0       _kzaddstack                0051b0b0 f   kplib.obj
 0001:0011aa00       ?kzsetfil@@YAXPAU_iobuf@@@Z 0051ba00 f   kplib.obj
 0001:0011aa60       _kzopen                    0051ba60 f   kplib.obj
 0001:0011b030       _kzfindfilestart           0051c030 f   kplib.obj
 0001:0011b0a0       _kzfindfile                0051c0a0 f   kplib.obj
 0001:0011b4a0       _kzread                    0051c4a0 f   kplib.obj
 0001:0011bf60       _kzseek                    0051cf60 f   kplib.obj
 0001:0011bff0       _kpzdecode                 0051cff0 f   kplib.obj
 0001:0011c0e0       _kpzload                   0051d0e0 f   kplib.obj
 0001:0011c110       _hicfindsubst              0051d110 f   hightile.obj
 0001:0011c190       _hicfindskybox             0051d190 f   hightile.obj
 0001:0011c210       _hicinit                   0051d210 f   hightile.obj
 0001:0011c340       _hicsetpalettetint         0051d340 f   hightile.obj
 0001:0011c3a0       _hicsetsubsttex            0051d3a0 f   hightile.obj
 0001:0011c5b0       _hicsetskybox              0051d5b0 f   hightile.obj
 0001:0011c780       _hicclearsubst             0051d780 f   hightile.obj
 0001:0011c8a0       _gltexinvalidate           0051d8a0 f   polymost.obj
 0001:0011c940       _gltexinvalidatetype       0051d940 f   polymost.obj
 0001:0011ca00       _gltexapplyprops           0051da00 f   polymost.obj
 0001:0011cce0       _polymost_glreset          0051dce0 f   polymost.obj
 0001:0011ced0       _polymost_glinit           0051ded0 f   polymost.obj
 0001:0011d030       _calc_and_apply_fog        0051e030 f   polymost.obj
 0001:0011d400       _calc_and_apply_fog_factor 0051e400 f   polymost.obj
 0001:0011d490       _uploadtexture             0051e490 f   polymost.obj
 0001:0011de10       _gloadtile_art             0051ee10 f   polymost.obj
 0001:0011eb70       _gloadtile_hi              0051fb70 f   polymost.obj
 0001:0011fb30       _polymost_setupdetailtexture 00520b30 f   polymost.obj
 0001:0011fc90       _polymost_setupglowtexture 00520c90 f   polymost.obj
 0001:0011fe10       ?polymost_editorfunc@@YAXXZ 00520e10 f   polymost.obj
 0001:00120bd0       _polymost_scansector       00521bd0 f   polymost.obj
 0001:00121340       _polymost_drawrooms        00522340 f   polymost.obj
 0001:0012abc0       _polymost_drawmaskwall     0052bbc0 f   polymost.obj
 0001:0012b9d0       ?polymost_lintersect@@YAHHHHHHHHH@Z 0052c9d0 f   polymost.obj
 0001:0012bac0       _polymost_drawsprite       0052cac0 f   polymost.obj
 0001:0012e210       ?polymost_dorotatespritemodel@@YAXHHHFFCDHEH@Z 0052f210 f   polymost.obj
 0001:0012eb30       _polymost_dorotatesprite   0052fb30 f   polymost.obj
 0001:0012f8b0       _polymost_fillpolygon      005308b0 f   polymost.obj
 0001:00130aa0       _polymost_drawtilescreen   00531aa0 f   polymost.obj
 0001:00130f90       _polymost_printext256      00531f90 f   polymost.obj
 0001:00131680       _polymost_initosdfuncs     00532680 f   polymost.obj
 0001:00132910       _polymost_precache         00533910 f   polymost.obj
 0001:00132a90       _fabsf                     00533a90 f i polymost.obj
 0001:00132ab0       _cosf                      00533ab0 f i polymost.obj
 0001:00132ad0       _sqrtf                     00533ad0 f i polymost.obj
 0001:00132af0       _floorf                    00533af0 f i polymost.obj
 0001:00132b10       _tanf                      00533b10 f i polymost.obj
 0001:00132b50       _polymer_init              00533b50 f   polymer.obj
 0001:00132ef0       _polymer_uninit            00533ef0 f   polymer.obj
 0001:00133000       _polymer_setaspect         00534000 f   polymer.obj
 0001:001330d0       _polymer_glinit            005340d0 f   polymer.obj
 0001:00133220       _polymer_resetlights       00534220 f   polymer.obj
 0001:00133360       _polymer_loadboard         00534360 f   polymer.obj
 0001:001334e0       _polymer_drawrooms         005344e0 f   polymer.obj
 0001:00133ba0       _polymer_drawmasks         00534ba0 f   polymer.obj
 0001:00133c70       _polymer_editorpick        00534c70 f   polymer.obj
 0001:00134420       _polymer_inb4rotatesprite  00535420 f   polymer.obj
 0001:00134480       _polymer_postrotatesprite  00535480 f   polymer.obj
 0001:001344a0       _polymer_drawmaskwall      005354a0 f   polymer.obj
 0001:00134680       _polymer_drawsprite        00535680 f   polymer.obj
 0001:00134d60       _polymer_setanimatesprites 00535d60 f   polymer.obj
 0001:00134d90       _polymer_addlight          00535d90 f   polymer.obj
 0001:00134fc0       _polymer_deletelight       00535fc0 f   polymer.obj
 0001:00135040       _polymer_invalidatelights  00536040 f   polymer.obj
 0001:001350a0       _polymer_texinvalidate     005360a0 f   polymer.obj
 0001:00135190       _polymer_definehighpalookup 00536190 f   polymer.obj
 0001:00135220       _polymer_havehighpalookup  00536220 f   polymer.obj
 0001:001381c0       _polymer_tesserror@4       005391c0 f   polymer.obj
 0001:00138200       _polymer_tessedgeflag@4    00539200 f   polymer.obj
 0001:00138210       _polymer_tessvertex@8      00539210 f   polymer.obj
 0001:00143b40       _polymer_debugoutputcallback@28 00544b40 f   polymer.obj
 0001:00143bd0       ?sqrt@@YAMM@Z              00544bd0 f i polymer.obj
 0001:00143bf0       ?cos@@YAMM@Z               00544bf0 f i polymer.obj
 0001:00143c10       ?sin@@YAMM@Z               00544c10 f i polymer.obj
 0001:00143c30       _Ptile2tile                00544c30 f   mdsprite.obj
 0001:00143c80       _md_freevbos               00544c80 f   mdsprite.obj
 0001:00143d50       _freeallmodels             00544d50 f   mdsprite.obj
 0001:00143e90       _clearskins                00544e90 f   mdsprite.obj
 0001:001441d0       _mdinit                    005451d0 f   mdsprite.obj
 0001:001441f0       _md_loadmodel              005451f0 f   mdsprite.obj
 0001:001442e0       _md_setmisc                005452e0 f   mdsprite.obj
 0001:00144350       _md_defineframe            00545350 f   mdsprite.obj
 0001:00144670       _md_defineanimation        00545670 f   mdsprite.obj
 0001:001447b0       _md_defineskin             005457b0 f   mdsprite.obj
 0001:001449b0       _md_definehud              005459b0 f   mdsprite.obj
 0001:00144a80       _md_undefinetile           00545a80 f   mdsprite.obj
 0001:00144b20       _md_undefinemodel          00545b20 f   mdsprite.obj
 0001:00144c10       _mdloadskin                00545c10 f   mdsprite.obj
 0001:001460b0       _updateanimation           005470b0 f   mdsprite.obj
 0001:00146680       ?partition@@YAHPAGPAMHH@Z  00547680 f   mdsprite.obj
 0001:001467e0       _md3postload_polymer       005477e0 f   mdsprite.obj
 0001:00147390       _md3_vox_calcmat_common    00548390 f   mdsprite.obj
 0001:00149100       ?md_allocvbos@@YAXXZ       0054a100 f   mdsprite.obj
 0001:00149280       _polymost_mddraw           0054a280 f   mdsprite.obj
 0001:0014b6a0       ?gloadtex@@YAIPAHHHHH@Z    0054c6a0 f   voxmodel.obj
 0001:0014b8e0       _voxfree                   0054c8e0 f   voxmodel.obj
 0001:0014b950       _voxload                   0054c950 f   voxmodel.obj
 0001:0014e550       _polymost_voxdraw          0054f550 f   voxmodel.obj
 0001:0014f010       ?dxtfilter@@YAHHPBUtexcachepic_t@@PBDPAXPADI@Z 00550010 f   dxtfilter.obj
 0001:0014f520       ?dedxtfilter@@YAHHPBUtexcachepic_t@@PADPAX1H@Z 00550520 f   dxtfilter.obj
 0001:0014fa60       _LZ4_versionNumber         00550a60 f   lz4.obj
 0001:0014fa70       _LZ4_compressBound         00550a70 f   lz4.obj
 0001:0014fab0       _LZ4_sizeofState           00550ab0 f   lz4.obj
 0001:0014fac0       _LZ4_compress_fast_extState 00550ac0 f   lz4.obj
 0001:00150890       _LZ4_compress_fast         00551890 f   lz4.obj
 0001:001508f0       _LZ4_compress_default      005518f0 f   lz4.obj
 0001:00150910       ?LZ4_compress_fast_force@@YAHPBDPADHHH@Z 00551910 f   lz4.obj
 0001:001509c0       _LZ4_compress_destSize     005519c0 f   lz4.obj
 0001:00151040       _LZ4_createStream          00552040 f   lz4.obj
 0001:00151070       _LZ4_resetStream           00552070 f   lz4.obj
 0001:00151090       _LZ4_freeStream            00552090 f   lz4.obj
 0001:001510b0       _LZ4_loadDict              005520b0 f   lz4.obj
 0001:001511d0       _LZ4_compress_fast_continue 005521d0 f   lz4.obj
 0001:00151510       ?LZ4_compress_forceExtDict@@YAHPAULZ4_stream_t@@PBDPADH@Z 00552510 f   lz4.obj
 0001:001515b0       _LZ4_saveDict              005525b0 f   lz4.obj
 0001:00151640       _LZ4_decompress_safe       00552640 f   lz4.obj
 0001:00151da0       _LZ4_decompress_safe_partial 00552da0 f   lz4.obj
 0001:00151dd0       _LZ4_decompress_fast       00552dd0 f   lz4.obj
 0001:00151e10       _LZ4_createStreamDecode    00552e10 f   lz4.obj
 0001:00151e30       _LZ4_freeStreamDecode      00552e30 f   lz4.obj
 0001:00151e50       _LZ4_setStreamDecode       00552e50 f   lz4.obj
 0001:00151e90       _LZ4_decompress_safe_continue 00552e90 f   lz4.obj
 0001:00151f90       _LZ4_decompress_fast_continue 00552f90 f   lz4.obj
 0001:00152090       _LZ4_decompress_safe_usingDict 00553090 f   lz4.obj
 0001:001521a0       _LZ4_decompress_fast_usingDict 005531a0 f   lz4.obj
 0001:001521d0       ?LZ4_decompress_safe_forceExtDict@@YAHPBDPADHH0H@Z 005531d0 f   lz4.obj
 0001:00152210       _LZ4_compress_limitedOutput 00553210 f   lz4.obj
 0001:00152230       _LZ4_compress              00553230 f   lz4.obj
 0001:00152260       _LZ4_compress_limitedOutput_withState 00553260 f   lz4.obj
 0001:00152290       _LZ4_compress_withState    00553290 f   lz4.obj
 0001:001522c0       _LZ4_compress_limitedOutput_continue 005532c0 f   lz4.obj
 0001:001522f0       _LZ4_compress_continue     005532f0 f   lz4.obj
 0001:00152320       ?LZ4_uncompress@@YAHPBDPADH@Z 00553320 f   lz4.obj
 0001:00152340       ?LZ4_uncompress_unknownOutputSize@@YAHPBDPADHH@Z 00553340 f   lz4.obj
 0001:00152360       _LZ4_sizeofStreamState     00553360 f   lz4.obj
 0001:00152370       _LZ4_resetStreamState      00553370 f   lz4.obj
 0001:001523d0       _LZ4_create                005533d0 f   lz4.obj
 0001:00152400       _LZ4_slideInputBuffer      00553400 f   lz4.obj
 0001:00152440       _LZ4_decompress_safe_withPrefix64k 00553440 f   lz4.obj
 0001:00152480       _LZ4_decompress_fast_withPrefix64k 00553480 f   lz4.obj
 0001:001524c0       _md4once                   005534c0 f   md4.obj
 0001:00152510       _md4init                   00553510 f   md4.obj
 0001:00152550       _md4block                  00553550 f   md4.obj
 0001:00152660       _md4finish                 00553660 f   md4.obj
 0001:00153180       ?isvalidipaddress@@YAHPBD@Z 00554180 f   mmulti_null.obj
 0001:00153190       ?initmultiplayersparms@@YAHHQBQBD@Z 00554190 f   mmulti_null.obj
 0001:001531a0       ?initmultiplayerscycle@@YAHXZ 005541a0 f   mmulti_null.obj
 0001:001531b0       ?initmultiplayers@@YAXHQBQBDEEE@Z 005541b0 f   mmulti_null.obj
 0001:001531e0       ?setpackettimeout@@YAXHH@Z 005541e0 f   mmulti_null.obj
 0001:001531f0       ?uninitmultiplayers@@YAXXZ 005541f0 f   mmulti_null.obj
 0001:00153200       ?sendlogon@@YAXXZ          00554200 f   mmulti_null.obj
 0001:00153210       ?sendlogoff@@YAXXZ         00554210 f   mmulti_null.obj
 0001:00153220       ?getoutputcirclesize@@YAHXZ 00554220 f   mmulti_null.obj
 0001:00153230       ?setsocket@@YAXH@Z         00554230 f   mmulti_null.obj
 0001:00153240       ?sendpacket@@YAXHPAEH@Z    00554240 f   mmulti_null.obj
 0001:00153250       ?getpacket@@YAHPAHPAE@Z    00554250 f   mmulti_null.obj
 0001:00153260       ?flushpackets@@YAXXZ       00554260 f   mmulti_null.obj
 0001:00153270       ?genericmultifunction@@YAXHPAEHH@Z 00554270 f   mmulti_null.obj
 0001:00153290       _OSD_RegisterCvar          00554290 f   osd.obj
 0001:00153590       _OSD_StripColors           00554590 f   osd.obj
 0001:00153690       _OSD_Exec                  00554690 f   osd.obj
 0001:00153860       _OSD_ParsingScript         00554860 f   osd.obj
 0001:00153870       _OSD_OSDKey                00554870 f   osd.obj
 0001:00153880       _OSD_GetCols               00554880 f   osd.obj
 0001:00153890       _OSD_IsMoving              00554890 f   osd.obj
 0001:001538d0       _OSD_GetRowsCur            005548d0 f   osd.obj
 0001:001538e0       _OSD_GetTextMode           005548e0 f   osd.obj
 0001:001538f0       _OSD_GetShadePal           005548f0 f   osd.obj
 0001:00153960       _OSD_SetTextMode           00554960 f   osd.obj
 0001:00153d00       _OSD_Cleanup               00554d00 f   osd.obj
 0001:00153e90       _OSD_Init                  00554e90 f   osd.obj
 0001:00155070       _OSD_SetLogFile            00556070 f   osd.obj
 0001:00155100       _OSD_SetFunctions          00556100 f   osd.obj
 0001:00155200       _OSD_SetParameters         00556200 f   osd.obj
 0001:00155260       _OSD_CaptureKey            00556260 f   osd.obj
 0001:00155280       _OSD_HandleChar            00556280 f   osd.obj
 0001:00156600       _OSD_HandleScanCode        00557600 f   osd.obj
 0001:00156e30       _OSD_ResizeDisplay         00557e30 f   osd.obj
 0001:00157040       _OSD_CaptureInput          00558040 f   osd.obj
 0001:001570b0       _OSD_ShowDisplay           005580b0 f   osd.obj
 0001:001570f0       _OSD_Draw                  005580f0 f   osd.obj
 0001:00157720       _OSD_Printf                00558720 f   osd.obj
 0001:00157760       _OSD_Puts                  00558760 f   osd.obj
 0001:00157c70       _OSD_DispatchQueued        00558c70 f   osd.obj
 0001:00157ce0       _OSD_Dispatch              00558ce0 f   osd.obj
 0001:001580b0       _OSD_RegisterFunction      005590b0 f   osd.obj
 0001:00158250       _OSD_SetVersion            00559250 f   osd.obj
 0001:001585b0       _osdcmd_cvar_set           005595b0 f   osd.obj
 0001:00158d40       _OSD_WriteAliases          00559d40 f   osd.obj
 0001:00158d90       _OSD_WriteCvars            00559d90 f   osd.obj
 0001:00158fe0       _initdivtables             00559fe0 f   pragmas.obj
 0001:001590d0       _divideu32_noinline        0055a0d0 f   pragmas.obj
 0001:00159150       _tabledivide32_noinline    0055a150 f   pragmas.obj
 0001:00159200       _tabledivide64_noinline    0055a200 f   pragmas.obj
 0001:001592f0       _scriptfile_gettoken       0055a2f0 f   scriptfile.obj
 0001:001593b0       _scriptfile_getstring      0055a3b0 f   scriptfile.obj
 0001:00159400       _scriptfile_getnumber      0055a400 f   scriptfile.obj
 0001:00159550       _scriptfile_getdouble      0055a550 f   scriptfile.obj
 0001:00159810       _scriptfile_getsymbol      0055a810 f   scriptfile.obj
 0001:001598b0       _scriptfile_getbraces      0055a8b0 f   scriptfile.obj
 0001:001599e0       _scriptfile_getlinum       0055a9e0 f   scriptfile.obj
 0001:00159a70       ?scriptfile_preparse@@YAXPAUscriptfile@@PADH@Z 0055aa70 f   scriptfile.obj
 0001:00159e30       _scriptfile_fromfile       0055ae30 f   scriptfile.obj
 0001:00159f60       _scriptfile_fromstring     0055af60 f   scriptfile.obj
 0001:0015a020       _scriptfile_close          0055b020 f   scriptfile.obj
 0001:0015a070       _scriptfile_eof            0055b070 f   scriptfile.obj
 0001:0015a0a0       _scriptfile_getsymbolvalue 0055b0a0 f   scriptfile.obj
 0001:0015a140       _scriptfile_addsymbolvalue 0055b140 f   scriptfile.obj
 0001:0015a320       _scriptfile_clearsymbols   0055b320 f   scriptfile.obj
 0001:0015a360       _mutex_init                0055b360 f   mutex.obj
 0001:0015a390       _mutex_lock                0055b390 f   mutex.obj
 0001:0015a3b0       _mutex_unlock              0055b3b0 f   mutex.obj
 0001:0015a3d0       ?CheckWinVersion@@YAHXZ    0055b3d0 f   winbits.obj
 0001:0015a460       ?win_allowtaskswitching@@YAXH@Z 0055b460 f   winbits.obj
 0001:0015a4c0       ?win_checkinstance@@YAHXZ  0055b4c0 f   winbits.obj
 0001:0015a4f0       ?win_inittimer@@YAHXZ      0055b4f0 f   winbits.obj
 0001:0015a540       ?win_getu64ticks@@YA_KXZ   0055b540 f   winbits.obj
 0001:0015a570       ?win_open@@YAXXZ           0055b570 f   winbits.obj
 0001:0015a5f0       ?win_init@@YAXXZ           0055b5f0 f   winbits.obj
 0001:0015a8b0       ?win_setvideomode@@YAXH@Z  0055b8b0 f   winbits.obj
 0001:0015a980       ?win_uninit@@YAXXZ         0055b980 f   winbits.obj
 0001:0015a990       ?win_close@@YAXXZ          0055b990 f   winbits.obj
 0001:0015a9b0       ?ShowErrorBox@@YAXPBD@Z    0055b9b0 f   winbits.obj
 0001:0015aa10       ?GetWindowsErrorMsg@@YAPADK@Z 0055ba10 f   winbits.obj
 0001:0015aa40       ?addsearchpath_ProgramFiles@@YAHPBD@Z 0055ba40 f   winbits.obj
 0001:0015ab10       ?win_buildargs@@YAHPAPAD@Z 0055bb10 f   winbits.obj
 0001:0015ac80       _XXH_versionNumber         0055bc80 f   xxhash.obj
 0001:0015ac90       _XXH32                     0055bc90 f   xxhash.obj
 0001:0015b010       _XXH64                     0055c010 f   xxhash.obj
 0001:0015b870       _XXH32_createState         0055c870 f   xxhash.obj
 0001:0015b8a0       _XXH32_freeState           0055c8a0 f   xxhash.obj
 0001:0015b8e0       _XXH64_createState         0055c8e0 f   xxhash.obj
 0001:0015b8f0       _XXH64_freeState           0055c8f0 f   xxhash.obj
 0001:0015b910       _XXH32_reset               0055c910 f   xxhash.obj
 0001:0015b990       _XXH64_reset               0055c990 f   xxhash.obj
 0001:0015ba30       _XXH32_update              0055ca30 f   xxhash.obj
 0001:0015be80       _XXH32_digest              0055ce80 f   xxhash.obj
 0001:0015c030       _XXH64_update              0055d030 f   xxhash.obj
 0001:0015c5e0       _XXH64_digest              0055d5e0 f   xxhash.obj
 0001:0015cba0       ?win_gethwnd@@YAPAUHWND__@@XZ 0055dba0 f   sdlayer.obj
 0001:0015cbf0       ?win_gethinstance@@YAPAUHINSTANCE__@@XZ 0055dbf0 f   sdlayer.obj
 0001:0015cc00       _wm_msgbox                 0055dc00 f   sdlayer.obj
 0001:0015cca0       _wm_ynbox                  0055dca0 f   sdlayer.obj
 0001:0015cd20       _wm_setapptitle            0055dd20 f   sdlayer.obj
 0001:0015cdd0       _WinMain@16                0055ddd0 f   sdlayer.obj
 0001:0015d2b0       _setvsync                  0055e2b0 f   sdlayer.obj
 0001:0015d2f0       ?sdlayer_checkversion@@YAHXZ 0055e2f0 f   sdlayer.obj
 0001:0015d3b0       _initsystem                0055e3b0 f   sdlayer.obj
 0001:0015d480       _uninitsystem              0055e480 f   sdlayer.obj
 0001:0015d4c0       _system_getcvars           0055e4c0 f   sdlayer.obj
 0001:0015d4e0       _initprintf                0055e4e0 f   sdlayer.obj
 0001:0015d540       _initputs                  0055e540 f   sdlayer.obj
 0001:0015d610       _debugprintf               0055e610 f   sdlayer.obj
 0001:0015d640       _initinput                 0055e640 f   sdlayer.obj
 0001:0015da10       _uninitinput               0055ea10 f   sdlayer.obj
 0001:0015da50       _getjoyname                0055ea50 f   sdlayer.obj
 0001:0015db00       _initmouse                 0055eb00 f   sdlayer.obj
 0001:0015db30       _uninitmouse               0055eb30 f   sdlayer.obj
 0001:0015db90       _grabmouse                 0055eb90 f   sdlayer.obj
 0001:0015dc00       _AppGrabMouse              0055ec00 f   sdlayer.obj
 0001:0015dc60       _setjoydeadzone            0055ec60 f   sdlayer.obj
 0001:0015dc90       _getjoydeadzone            0055ec90 f   sdlayer.obj
 0001:0015dcc0       _releaseallbuttons         0055ecc0 f   sdlayer.obj
 0001:0015dcd0       _inittimer                 0055ecd0 f   sdlayer.obj
 0001:0015dd70       _uninittimer               0055ed70 f   sdlayer.obj
 0001:0015ddb0       _sampletimer               0055edb0 f   sdlayer.obj
 0001:0015ded0       _getu64ticks               0055eed0 f   sdlayer.obj
 0001:0015dee0       _getu64tickspersec         0055eee0 f   sdlayer.obj
 0001:0015def0       _gethiticks                0055eef0 f   sdlayer.obj
 0001:0015df30       _gettimerfreq              0055ef30 f   sdlayer.obj
 0001:0015df40       _installusertimercallback  0055ef40 f   sdlayer.obj
 0001:0015df60       _getvalidmodes             0055ef60 f   sdlayer.obj
 0001:0015e4e0       _checkvideomode            0055f4e0 f   sdlayer.obj
 0001:0015e6d0       ?sdlayer_setvideomode_opengl@@YAXXZ 0055f6d0 f   sdlayer.obj
 0001:0015eb90       ?setvideomode_sdlcommon@@YAHPAH0HH0@Z 0055fb90 f   sdlayer.obj
 0001:0015ec80       ?setvideomode_sdlcommonpost@@YAXHHHHH@Z 0055fc80 f   sdlayer.obj
 0001:0015eda0       _setvideomode              0055fda0 f   sdlayer.obj
 0001:0015f400       _resetvideomode            00560400 f   sdlayer.obj
 0001:0015f420       _begindrawing              00560420 f   sdlayer.obj
 0001:0015f500       _enddrawing                00560500 f   sdlayer.obj
 0001:0015f5a0       _showframe                 005605a0 f   sdlayer.obj
 0001:0015f740       _setpalette                00560740 f   sdlayer.obj
 0001:0015f7c0       _setgamma                  005607c0 f   sdlayer.obj
 0001:0015fc90       _handleevents_peekkeys     00560c90 f   sdlayer.obj
 0001:0015fcc0       ?handleevents_updatemousestate@@YAXE@Z 00560cc0 f   sdlayer.obj
 0001:0015fce0       ?handleevents_sdlcommon@@YAHPATSDL_Event@@@Z 00560ce0 f   sdlayer.obj
 0001:00160170       ?handleevents_pollsdl@@YAHXZ 00561170 f   sdlayer.obj
 0001:00160620       _handleevents              00561620 f   sdlayer.obj
 0001:001606a0       ?SoundDriver_IsSupported@@YAHH@Z 005616a0 f   drivers.obj
 0001:001606c0       ?SoundDriver_GetError@@YAHXZ 005616c0 f   drivers.obj
 0001:00160700       ?SoundDriver_ErrorString@@YAPBDH@Z 00561700 f   drivers.obj
 0001:00160750       ?SoundDriver_Init@@YAHPAH0PAX@Z 00561750 f   drivers.obj
 0001:00160780       ?SoundDriver_Shutdown@@YAXXZ 00561780 f   drivers.obj
 0001:001607a0       ?SoundDriver_BeginPlayback@@YAHPADHHP6AXXZ@Z 005617a0 f   drivers.obj
 0001:001607d0       ?SoundDriver_StopPlayback@@YAXXZ 005617d0 f   drivers.obj
 0001:001607f0       ?SoundDriver_Lock@@YAXXZ   005617f0 f   drivers.obj
 0001:00160810       ?SoundDriver_Unlock@@YAXXZ 00561810 f   drivers.obj
 0001:00160830       _FX_ErrorString            00561830 f   fx_man.obj
 0001:001608b0       _FX_Init                   005618b0 f   fx_man.obj
 0001:00160950       _FX_Shutdown               00561950 f   fx_man.obj
 0001:001609a0       _FX_SetCallBack            005619a0 f   fx_man.obj
 0001:001609c0       _FX_SetVolume              005619c0 f   fx_man.obj
 0001:001609e0       _FX_GetVolume              005619e0 f   fx_man.obj
 0001:001609f0       _FX_SetReverseStereo       005619f0 f   fx_man.obj
 0001:00160a10       _FX_GetReverseStereo       00561a10 f   fx_man.obj
 0001:00160a20       _FX_SetReverb              00561a20 f   fx_man.obj
 0001:00160a40       _FX_GetMaxReverbDelay      00561a40 f   fx_man.obj
 0001:00160a50       _FX_GetReverbDelay         00561a50 f   fx_man.obj
 0001:00160a60       _FX_SetReverbDelay         00561a60 f   fx_man.obj
 0001:00160a80       _FX_VoiceAvailable         00561a80 f   fx_man.obj
 0001:00160aa0       _FX_PauseVoice             00561aa0 f   fx_man.obj
 0001:00160ae0       _FX_GetPosition            00561ae0 f   fx_man.obj
 0001:00160b00       _FX_SetPosition            00561b00 f   fx_man.obj
 0001:00160b20       _FX_EndLooping             00561b20 f   fx_man.obj
 0001:00160b40       _FX_SetPan                 00561b40 f   fx_man.obj
 0001:00160b70       _FX_SetPitch               00561b70 f   fx_man.obj
 0001:00160b90       _FX_SetFrequency           00561b90 f   fx_man.obj
 0001:00160bb0       _FX_Pan3D                  00561bb0 f   fx_man.obj
 0001:00160be0       _FX_SoundActive            00561be0 f   fx_man.obj
 0001:00160c00       _FX_SoundsPlaying          00561c00 f   fx_man.obj
 0001:00160c10       _FX_StopSound              00561c10 f   fx_man.obj
 0001:00160c30       _FX_StopAllSounds          00561c30 f   fx_man.obj
 0001:00160c50       _FX_PlayAuto               00561c50 f   fx_man.obj
 0001:00160c90       _FX_PlayLoopedAuto         00561c90 f   fx_man.obj
 0001:00160de0       _FX_PlayAuto3D             00561de0 f   fx_man.obj
 0001:00160e60       _FX_SetVoiceCallback       00561e60 f   fx_man.obj
 0001:00160ea0       _FX_SetPrintf              00561ea0 f   fx_man.obj
 0001:00160ec0       _MV_ErrorString            00561ec0 f   multivoc.obj
 0001:00160f90       ?MV_PlayVoice@@YAXPAUVoiceNode@@@Z 00561f90 f   multivoc.obj
 0001:00161050       ?MV_BeginService@@YAPAUVoiceNode@@H@Z 00562050 f   multivoc.obj
 0001:00161130       _MV_VoicePlaying           00562130 f   multivoc.obj
 0001:00161170       _MV_KillAllVoices          00562170 f   multivoc.obj
 0001:001611f0       _MV_Kill                   005621f0 f   multivoc.obj
 0001:00161310       _MV_VoicesPlaying          00562310 f   multivoc.obj
 0001:00161370       ?MV_AllocVoice@@YAPAUVoiceNode@@H@Z 00562370 f   multivoc.obj
 0001:001614b0       _MV_VoiceAvailable         005624b0 f   multivoc.obj
 0001:00161540       ?MV_SetVoicePitch@@YAXPAUVoiceNode@@IH@Z 00562540 f   multivoc.obj
 0001:00161590       _MV_SetPitch               00562590 f   multivoc.obj
 0001:001615d0       _MV_SetFrequency           005625d0 f   multivoc.obj
 0001:00161610       ?MV_SetVoiceMixMode@@YAXPAUVoiceNode@@@Z 00562610 f   multivoc.obj
 0001:00161790       ?MV_SetVoiceVolume@@YAXPAUVoiceNode@@HHH@Z 00562790 f   multivoc.obj
 0001:001618a0       _MV_PauseVoice             005628a0 f   multivoc.obj
 0001:001618e0       _MV_GetPosition            005628e0 f   multivoc.obj
 0001:00161950       _MV_SetPosition            00562950 f   multivoc.obj
 0001:001619c0       _MV_EndLooping             005629c0 f   multivoc.obj
 0001:00161a10       _MV_SetPan                 00562a10 f   multivoc.obj
 0001:00161a60       _MV_Pan3D                  00562a60 f   multivoc.obj
 0001:00161b30       _MV_SetReverb              00562b30 f   multivoc.obj
 0001:00161bb0       _MV_GetMaxReverbDelay      00562bb0 f   multivoc.obj
 0001:00161bc0       _MV_GetReverbDelay         00562bc0 f   multivoc.obj
 0001:00161be0       _MV_SetReverbDelay         00562be0 f   multivoc.obj
 0001:00161c50       _MV_SetVolume              00562c50 f   multivoc.obj
 0001:00161d30       _MV_GetVolume              00562d30 f   multivoc.obj
 0001:00161d40       _MV_SetCallBack            00562d40 f   multivoc.obj
 0001:00161d50       _MV_SetReverseStereo       00562d50 f   multivoc.obj
 0001:00161d60       _MV_GetReverseStereo       00562d60 f   multivoc.obj
 0001:00161d70       _MV_Init                   00562d70 f   multivoc.obj
 0001:00162680       _MV_Shutdown               00563680 f   multivoc.obj
 0001:001627b0       _MV_SetVoiceCallback       005637b0 f   multivoc.obj
 0001:001627f0       _MV_SetPrintf              005637f0 f   multivoc.obj
 0001:00162800       ?MV_Mix16BitMono@@YAXIIPBDI@Z 00563800 f   mix.obj
 0001:001628b0       ?MV_Mix16BitStereo@@YAXIIPBDI@Z 005638b0 f   mix.obj
 0001:001629d0       ?MV_Mix16BitMono16@@YAXIIPBDI@Z 005639d0 f   mix.obj
 0001:00162ac0       ?MV_Mix16BitStereo16@@YAXIIPBDI@Z 00563ac0 f   mix.obj
 0001:00162c40       ?MV_16BitReverb@@YAXPBDPADPAFH@Z 00563c40 f   mix.obj
 0001:00162ce0       ?MV_Mix16BitMono8Stereo@@YAXIIPBDI@Z 00563ce0 f   mixst.obj
 0001:00162dc0       ?MV_Mix16BitStereo8Stereo@@YAXIIPBDI@Z 00563dc0 f   mixst.obj
 0001:00162ee0       ?MV_Mix16BitMono16Stereo@@YAXIIPBDI@Z 00563ee0 f   mixst.obj
 0001:00163050       ?MV_Mix16BitStereo16Stereo@@YAXIIPBDI@Z 00564050 f   mixst.obj
 0001:001631f0       ?PITCH_Init@@YAXXZ         005641f0 f   pitch.obj
 0001:001632c0       ?PITCH_GetScale@@YAIH@Z    005642c0 f   pitch.obj
 0001:001633b0       _MV_PlayWAV3D              005643b0 f   formats.obj
 0001:001634b0       _MV_PlayWAV                005644b0 f   formats.obj
 0001:001638a0       _MV_PlayVOC3D              005648a0 f   formats.obj
 0001:001639a0       _MV_PlayVOC                005649a0 f   formats.obj
 0001:00164290       ?MV_GetVorbisPosition@@YAHPAUVoiceNode@@@Z 00565290 f   vorbis.obj
 0001:001642b0       ?MV_SetVorbisPosition@@YAXPAUVoiceNode@@H@Z 005652b0 f   vorbis.obj
 0001:001642e0       _MV_PlayVorbis3D           005652e0 f   vorbis.obj
 0001:001643e0       _MV_PlayVorbis             005653e0 f   vorbis.obj
 0001:00164bf0       ?MV_ReleaseVorbisVoice@@YAXPAUVoiceNode@@@Z 00565bf0 f   vorbis.obj
 0001:00164c40       _MV_PlayFLAC               00565c40 f   flac.obj
 0001:00164ca0       _MV_PlayFLAC3D             00565ca0 f   flac.obj
 0001:00164cf0       ?MV_GetXAPosition@@YAHPAUVoiceNode@@@Z 00565cf0 f   xa.obj
 0001:00164d10       ?MV_SetXAPosition@@YAXPAUVoiceNode@@H@Z 00565d10 f   xa.obj
 0001:00164d50       _MV_PlayXA3D               00565d50 f   xa.obj
 0001:00164e70       _MV_PlayXA                 00565e70 f   xa.obj
 0001:00165ac0       ?MV_ReleaseXAVoice@@YAXPAUVoiceNode@@@Z 00566ac0 f   xa.obj
 0001:00165b10       ?NoSoundDrv_GetError@@YAHXZ 00566b10 f   driver_nosound.obj
 0001:00165b20       ?NoSoundDrv_ErrorString@@YAPBDH@Z 00566b20 f   driver_nosound.obj
 0001:00165b30       ?NoSoundDrv_PCM_Init@@YAHPAH0PAX@Z 00566b30 f   driver_nosound.obj
 0001:00165b50       ?NoSoundDrv_PCM_Shutdown@@YAXXZ 00566b50 f   driver_nosound.obj
 0001:00165b60       ?NoSoundDrv_PCM_BeginPlayback@@YAHPADHHP6AXXZ@Z 00566b60 f   driver_nosound.obj
 0001:00165b80       ?NoSoundDrv_PCM_StopPlayback@@YAXXZ 00566b80 f   driver_nosound.obj
 0001:00165b90       ?NoSoundDrv_PCM_Lock@@YAXXZ 00566b90 f   driver_nosound.obj
 0001:00165ba0       ?NoSoundDrv_PCM_Unlock@@YAXXZ 00566ba0 f   driver_nosound.obj
 0001:00165bb0       ?DirectSoundDrv_GetError@@YAHXZ 00566bb0 f   driver_directsound.obj
 0001:00165bc0       ?DirectSoundDrv_ErrorString@@YAPBDH@Z 00566bc0 f   driver_directsound.obj
 0001:00165ce0       ?DirectSoundDrv_PCM_Init@@YAHPAH0PAX@Z 00566ce0 f   driver_directsound.obj
 0001:001661b0       ?DirectSoundDrv_PCM_Shutdown@@YAXXZ 005671b0 f   driver_directsound.obj
 0001:001661e0       ?DirectSoundDrv_PCM_BeginPlayback@@YAHPADHHP6AXXZ@Z 005671e0 f   driver_directsound.obj
 0001:001665d0       ?DirectSoundDrv_PCM_StopPlayback@@YAXXZ 005675d0 f   driver_directsound.obj
 0001:00166620       ?DirectSoundDrv_PCM_Lock@@YAXXZ 00567620 f   driver_directsound.obj
 0001:00166660       ?DirectSoundDrv_PCM_Unlock@@YAXXZ 00567660 f   driver_directsound.obj
 0001:00166680       _enet_initialize_with_callbacks 00567680 f   callbacks.obj
 0001:001666f0       _enet_linked_version       005676f0 f   callbacks.obj
 0001:00166700       _enet_malloc               00567700 f   callbacks.obj
 0001:00166730       _enet_free                 00567730 f   callbacks.obj
 0001:00166750       _enet_host_create          00567750 f   host.obj
 0001:00166b80       _enet_host_destroy         00567b80 f   host.obj
 0001:00166c30       _enet_host_connect         00567c30 f   host.obj
 0001:00166f00       _enet_host_broadcast       00567f00 f   host.obj
 0001:00166f70       _enet_host_compress        00567f70 f   host.obj
 0001:00166fe0       _enet_host_channel_limit   00567fe0 f   host.obj
 0001:00167020       _enet_host_bandwidth_limit 00568020 f   host.obj
 0001:00167050       _enet_host_bandwidth_throttle 00568050 f   host.obj
 0001:001674f0       _enet_list_clear           005684f0 f   list.obj
 0001:00167510       _enet_list_insert          00568510 f   list.obj
 0001:00167550       _enet_list_remove          00568550 f   list.obj
 0001:00167580       _enet_list_move            00568580 f   list.obj
 0001:001675e0       _enet_list_size            005685e0 f   list.obj
 0001:00167620       _enet_packet_create        00568620 f   packet.obj
 0001:001676f0       _enet_packet_destroy       005686f0 f   packet.obj
 0001:00167750       _enet_packet_resize        00568750 f   packet.obj
 0001:001677e0       _enet_crc32                005687e0 f   packet.obj
 0001:00167970       _enet_peer_throttle_configure 00568970 f   peer.obj
 0001:00167a00       _enet_peer_throttle        00568a00 f   peer.obj
 0001:00167ac0       _enet_peer_send            00568ac0 f   peer.obj
 0001:00167df0       _enet_peer_receive         00568df0 f   peer.obj
 0001:00167e90       _enet_peer_reset_queues    00568e90 f   peer.obj
 0001:001680f0       _enet_peer_on_connect      005690f0 f   peer.obj
 0001:00168150       _enet_peer_on_disconnect   00569150 f   peer.obj
 0001:001681b0       _enet_peer_reset           005691b0 f   peer.obj
 0001:001683e0       _enet_peer_ping            005693e0 f   peer.obj
 0001:00168430       _enet_peer_ping_interval   00569430 f   peer.obj
 0001:00168460       _enet_peer_timeout         00569460 f   peer.obj
 0001:001684d0       _enet_peer_disconnect_now  005694d0 f   peer.obj
 0001:00168560       _enet_peer_disconnect      00569560 f   peer.obj
 0001:00168650       _enet_peer_disconnect_later 00569650 f   peer.obj
 0001:001686d0       _enet_peer_queue_acknowledgement 005696d0 f   peer.obj
 0001:001687d0       _enet_peer_setup_outgoing_command 005697d0 f   peer.obj
 0001:001689d0       _enet_peer_queue_outgoing_command 005699d0 f   peer.obj
 0001:00168a50       _enet_peer_dispatch_incoming_unreliable_commands 00569a50 f   peer.obj
 0001:00168c90       _enet_peer_dispatch_incoming_reliable_commands 00569c90 f   peer.obj
 0001:00168da0       _enet_peer_queue_incoming_command 00569da0 f   peer.obj
 0001:00169230       _enet_protocol_command_size 0056a230 f   protocol.obj
 0001:00169250       _enet_host_flush           0056a250 f   protocol.obj
 0001:0016a520       _enet_host_check_events    0056b520 f   protocol.obj
 0001:0016a6f0       _enet_host_service         0056b6f0 f   protocol.obj
 0001:0016cc00       _enet_initialize           0056dc00 f   win32.obj
 0001:0016cc90       _enet_deinitialize         0056dc90 f   win32.obj
 0001:0016ccb0       _enet_host_random_seed     0056dcb0 f   win32.obj
 0001:0016ccc0       _enet_time_get             0056dcc0 f   win32.obj
 0001:0016cce0       _enet_time_set             0056dce0 f   win32.obj
 0001:0016cd00       _enet_address_set_host     0056dd00 f   win32.obj
 0001:0016cd60       _enet_address_get_host_ip  0056dd60 f   win32.obj
 0001:0016cdc0       _enet_address_get_host     0056ddc0 f   win32.obj
 0001:0016ce40       _enet_socket_bind          0056de40 f   win32.obj
 0001:0016ced0       _enet_socket_get_address   0056ded0 f   win32.obj
 0001:0016cf30       _enet_socket_listen        0056df30 f   win32.obj
 0001:0016cf70       _enet_socket_create        0056df70 f   win32.obj
 0001:0016cf90       _enet_socket_set_option    0056df90 f   win32.obj
 0001:0016d0f0       _enet_socket_get_option    0056e0f0 f   win32.obj
 0001:0016d150       _enet_socket_connect       0056e150 f   win32.obj
 0001:0016d1d0       _enet_socket_accept        0056e1d0 f   win32.obj
 0001:0016d250       _enet_socket_shutdown      0056e250 f   win32.obj
 0001:0016d270       _enet_socket_destroy       0056e270 f   win32.obj
 0001:0016d290       _enet_socket_send          0056e290 f   win32.obj
 0001:0016d340       _enet_socket_receive       0056e340 f   win32.obj
 0001:0016d410       _enet_socketset_select     0056e410 f   win32.obj
 0001:0016d460       _enet_socket_wait          0056e460 f   win32.obj
 0001:0016d650       _enet_range_coder_create   0056e650 f   compress.obj
 0001:0016d680       _enet_range_coder_destroy  0056e680 f   compress.obj
 0001:0016d6b0       _enet_range_coder_compress 0056e6b0 f   compress.obj
 0001:0016e250       _enet_range_coder_decompress 0056f250 f   compress.obj
 0001:0016f110       _enet_host_compress_with_range_coder 00570110 f   compress.obj
 0001:0016f1a0       _SDL_DYNAPI_entry          005701a0 f   libSDL2:SDL_dynapi.o
 0001:0017a420       _SDL_CreateThread          0057b420 f   libSDL2:SDL_dynapi.o
 0001:0017a430       _SDL_RWFromFP              0057b430 f   libSDL2:SDL_dynapi.o
 0001:0017a440       _SDL_RegisterApp           0057b440 f   libSDL2:SDL_dynapi.o
 0001:0017a450       _SDL_UnregisterApp         0057b450 f   libSDL2:SDL_dynapi.o
 0001:0017a460       _SDL_Direct3D9GetAdapterIndex 0057b460 f   libSDL2:SDL_dynapi.o
 0001:0017a470       _SDL_RenderGetD3D9Device   0057b470 f   libSDL2:SDL_dynapi.o
 0001:0017a480       _SDL_Init                  0057b480 f   libSDL2:SDL_dynapi.o
 0001:0017a490       _SDL_InitSubSystem         0057b490 f   libSDL2:SDL_dynapi.o
 0001:0017a4a0       _SDL_QuitSubSystem         0057b4a0 f   libSDL2:SDL_dynapi.o
 0001:0017a4b0       _SDL_WasInit               0057b4b0 f   libSDL2:SDL_dynapi.o
 0001:0017a4c0       _SDL_Quit                  0057b4c0 f   libSDL2:SDL_dynapi.o
 0001:0017a4d0       _SDL_ReportAssertion       0057b4d0 f   libSDL2:SDL_dynapi.o
 0001:0017a4e0       _SDL_SetAssertionHandler   0057b4e0 f   libSDL2:SDL_dynapi.o
 0001:0017a4f0       _SDL_GetAssertionReport    0057b4f0 f   libSDL2:SDL_dynapi.o
 0001:0017a500       _SDL_ResetAssertionReport  0057b500 f   libSDL2:SDL_dynapi.o
 0001:0017a510       _SDL_AtomicTryLock         0057b510 f   libSDL2:SDL_dynapi.o
 0001:0017a520       _SDL_AtomicLock            0057b520 f   libSDL2:SDL_dynapi.o
 0001:0017a530       _SDL_AtomicUnlock          0057b530 f   libSDL2:SDL_dynapi.o
 0001:0017a540       _SDL_AtomicCAS             0057b540 f   libSDL2:SDL_dynapi.o
 0001:0017a550       _SDL_AtomicSet             0057b550 f   libSDL2:SDL_dynapi.o
 0001:0017a560       _SDL_AtomicGet             0057b560 f   libSDL2:SDL_dynapi.o
 0001:0017a570       _SDL_AtomicAdd             0057b570 f   libSDL2:SDL_dynapi.o
 0001:0017a580       _SDL_AtomicCASPtr          0057b580 f   libSDL2:SDL_dynapi.o
 0001:0017a590       _SDL_AtomicSetPtr          0057b590 f   libSDL2:SDL_dynapi.o
 0001:0017a5a0       _SDL_AtomicGetPtr          0057b5a0 f   libSDL2:SDL_dynapi.o
 0001:0017a5b0       _SDL_GetNumAudioDrivers    0057b5b0 f   libSDL2:SDL_dynapi.o
 0001:0017a5c0       _SDL_GetAudioDriver        0057b5c0 f   libSDL2:SDL_dynapi.o
 0001:0017a5d0       _SDL_AudioInit             0057b5d0 f   libSDL2:SDL_dynapi.o
 0001:0017a5e0       _SDL_AudioQuit             0057b5e0 f   libSDL2:SDL_dynapi.o
 0001:0017a5f0       _SDL_GetCurrentAudioDriver 0057b5f0 f   libSDL2:SDL_dynapi.o
 0001:0017a600       _SDL_OpenAudio             0057b600 f   libSDL2:SDL_dynapi.o
 0001:0017a610       _SDL_GetNumAudioDevices    0057b610 f   libSDL2:SDL_dynapi.o
 0001:0017a620       _SDL_GetAudioDeviceName    0057b620 f   libSDL2:SDL_dynapi.o
 0001:0017a630       _SDL_OpenAudioDevice       0057b630 f   libSDL2:SDL_dynapi.o
 0001:0017a640       _SDL_GetAudioStatus        0057b640 f   libSDL2:SDL_dynapi.o
 0001:0017a650       _SDL_GetAudioDeviceStatus  0057b650 f   libSDL2:SDL_dynapi.o
 0001:0017a660       _SDL_PauseAudio            0057b660 f   libSDL2:SDL_dynapi.o
 0001:0017a670       _SDL_PauseAudioDevice      0057b670 f   libSDL2:SDL_dynapi.o
 0001:0017a680       _SDL_LoadWAV_RW            0057b680 f   libSDL2:SDL_dynapi.o
 0001:0017a690       _SDL_FreeWAV               0057b690 f   libSDL2:SDL_dynapi.o
 0001:0017a6a0       _SDL_BuildAudioCVT         0057b6a0 f   libSDL2:SDL_dynapi.o
 0001:0017a6d0       _SDL_ConvertAudio          0057b6d0 f   libSDL2:SDL_dynapi.o
 0001:0017a6e0       _SDL_MixAudio              0057b6e0 f   libSDL2:SDL_dynapi.o
 0001:0017a6f0       _SDL_MixAudioFormat        0057b6f0 f   libSDL2:SDL_dynapi.o
 0001:0017a700       _SDL_LockAudio             0057b700 f   libSDL2:SDL_dynapi.o
 0001:0017a710       _SDL_LockAudioDevice       0057b710 f   libSDL2:SDL_dynapi.o
 0001:0017a720       _SDL_UnlockAudio           0057b720 f   libSDL2:SDL_dynapi.o
 0001:0017a730       _SDL_UnlockAudioDevice     0057b730 f   libSDL2:SDL_dynapi.o
 0001:0017a740       _SDL_CloseAudio            0057b740 f   libSDL2:SDL_dynapi.o
 0001:0017a750       _SDL_CloseAudioDevice      0057b750 f   libSDL2:SDL_dynapi.o
 0001:0017a760       _SDL_SetClipboardText      0057b760 f   libSDL2:SDL_dynapi.o
 0001:0017a770       _SDL_GetClipboardText      0057b770 f   libSDL2:SDL_dynapi.o
 0001:0017a780       _SDL_HasClipboardText      0057b780 f   libSDL2:SDL_dynapi.o
 0001:0017a790       _SDL_GetCPUCount           0057b790 f   libSDL2:SDL_dynapi.o
 0001:0017a7a0       _SDL_GetCPUCacheLineSize   0057b7a0 f   libSDL2:SDL_dynapi.o
 0001:0017a7b0       _SDL_HasRDTSC              0057b7b0 f   libSDL2:SDL_dynapi.o
 0001:0017a7c0       _SDL_HasAltiVec            0057b7c0 f   libSDL2:SDL_dynapi.o
 0001:0017a7d0       _SDL_HasMMX                0057b7d0 f   libSDL2:SDL_dynapi.o
 0001:0017a7e0       _SDL_Has3DNow              0057b7e0 f   libSDL2:SDL_dynapi.o
 0001:0017a7f0       _SDL_HasSSE                0057b7f0 f   libSDL2:SDL_dynapi.o
 0001:0017a800       _SDL_HasSSE2               0057b800 f   libSDL2:SDL_dynapi.o
 0001:0017a810       _SDL_HasSSE3               0057b810 f   libSDL2:SDL_dynapi.o
 0001:0017a820       _SDL_HasSSE41              0057b820 f   libSDL2:SDL_dynapi.o
 0001:0017a830       _SDL_HasSSE42              0057b830 f   libSDL2:SDL_dynapi.o
 0001:0017a840       _SDL_GetSystemRAM          0057b840 f   libSDL2:SDL_dynapi.o
 0001:0017a850       _SDL_GetError              0057b850 f   libSDL2:SDL_dynapi.o
 0001:0017a860       _SDL_ClearError            0057b860 f   libSDL2:SDL_dynapi.o
 0001:0017a870       _SDL_Error                 0057b870 f   libSDL2:SDL_dynapi.o
 0001:0017a880       _SDL_PumpEvents            0057b880 f   libSDL2:SDL_dynapi.o
 0001:0017a890       _SDL_PeepEvents            0057b890 f   libSDL2:SDL_dynapi.o
 0001:0017a8a0       _SDL_HasEvent              0057b8a0 f   libSDL2:SDL_dynapi.o
 0001:0017a8b0       _SDL_HasEvents             0057b8b0 f   libSDL2:SDL_dynapi.o
 0001:0017a8c0       _SDL_FlushEvent            0057b8c0 f   libSDL2:SDL_dynapi.o
 0001:0017a8d0       _SDL_FlushEvents           0057b8d0 f   libSDL2:SDL_dynapi.o
 0001:0017a8e0       _SDL_PollEvent             0057b8e0 f   libSDL2:SDL_dynapi.o
 0001:0017a8f0       _SDL_WaitEvent             0057b8f0 f   libSDL2:SDL_dynapi.o
 0001:0017a900       _SDL_WaitEventTimeout      0057b900 f   libSDL2:SDL_dynapi.o
 0001:0017a910       _SDL_PushEvent             0057b910 f   libSDL2:SDL_dynapi.o
 0001:0017a920       _SDL_SetEventFilter        0057b920 f   libSDL2:SDL_dynapi.o
 0001:0017a930       _SDL_GetEventFilter        0057b930 f   libSDL2:SDL_dynapi.o
 0001:0017a940       _SDL_AddEventWatch         0057b940 f   libSDL2:SDL_dynapi.o
 0001:0017a950       _SDL_DelEventWatch         0057b950 f   libSDL2:SDL_dynapi.o
 0001:0017a960       _SDL_FilterEvents          0057b960 f   libSDL2:SDL_dynapi.o
 0001:0017a970       _SDL_EventState            0057b970 f   libSDL2:SDL_dynapi.o
 0001:0017a980       _SDL_RegisterEvents        0057b980 f   libSDL2:SDL_dynapi.o
 0001:0017a990       _SDL_GetBasePath           0057b990 f   libSDL2:SDL_dynapi.o
 0001:0017a9a0       _SDL_GetPrefPath           0057b9a0 f   libSDL2:SDL_dynapi.o
 0001:0017a9b0       _SDL_GameControllerAddMapping 0057b9b0 f   libSDL2:SDL_dynapi.o
 0001:0017a9c0       _SDL_GameControllerMappingForGUID 0057b9c0 f   libSDL2:SDL_dynapi.o
 0001:0017a9d0       _SDL_GameControllerMapping 0057b9d0 f   libSDL2:SDL_dynapi.o
 0001:0017a9e0       _SDL_IsGameController      0057b9e0 f   libSDL2:SDL_dynapi.o
 0001:0017a9f0       _SDL_GameControllerNameForIndex 0057b9f0 f   libSDL2:SDL_dynapi.o
 0001:0017aa00       _SDL_GameControllerOpen    0057ba00 f   libSDL2:SDL_dynapi.o
 0001:0017aa10       _SDL_GameControllerName    0057ba10 f   libSDL2:SDL_dynapi.o
 0001:0017aa20       _SDL_GameControllerGetAttached 0057ba20 f   libSDL2:SDL_dynapi.o
 0001:0017aa30       _SDL_GameControllerGetJoystick 0057ba30 f   libSDL2:SDL_dynapi.o
 0001:0017aa40       _SDL_GameControllerEventState 0057ba40 f   libSDL2:SDL_dynapi.o
 0001:0017aa50       _SDL_GameControllerUpdate  0057ba50 f   libSDL2:SDL_dynapi.o
 0001:0017aa60       _SDL_GameControllerGetAxisFromString 0057ba60 f   libSDL2:SDL_dynapi.o
 0001:0017aa70       _SDL_GameControllerGetStringForAxis 0057ba70 f   libSDL2:SDL_dynapi.o
 0001:0017aa80       _SDL_GameControllerGetBindForAxis 0057ba80 f   libSDL2:SDL_dynapi.o
 0001:0017aab0       _SDL_GameControllerGetAxis 0057bab0 f   libSDL2:SDL_dynapi.o
 0001:0017aac0       _SDL_GameControllerGetButtonFromString 0057bac0 f   libSDL2:SDL_dynapi.o
 0001:0017aad0       _SDL_GameControllerGetStringForButton 0057bad0 f   libSDL2:SDL_dynapi.o
 0001:0017aae0       _SDL_GameControllerGetBindForButton 0057bae0 f   libSDL2:SDL_dynapi.o
 0001:0017ab10       _SDL_GameControllerGetButton 0057bb10 f   libSDL2:SDL_dynapi.o
 0001:0017ab20       _SDL_GameControllerClose   0057bb20 f   libSDL2:SDL_dynapi.o
 0001:0017ab30       _SDL_RecordGesture         0057bb30 f   libSDL2:SDL_dynapi.o
 0001:0017ab40       _SDL_SaveAllDollarTemplates 0057bb40 f   libSDL2:SDL_dynapi.o
 0001:0017ab50       _SDL_SaveDollarTemplate    0057bb50 f   libSDL2:SDL_dynapi.o
 0001:0017ab60       _SDL_LoadDollarTemplates   0057bb60 f   libSDL2:SDL_dynapi.o
 0001:0017ab70       _SDL_NumHaptics            0057bb70 f   libSDL2:SDL_dynapi.o
 0001:0017ab80       _SDL_HapticName            0057bb80 f   libSDL2:SDL_dynapi.o
 0001:0017ab90       _SDL_HapticOpen            0057bb90 f   libSDL2:SDL_dynapi.o
 0001:0017aba0       _SDL_HapticOpened          0057bba0 f   libSDL2:SDL_dynapi.o
 0001:0017abb0       _SDL_HapticIndex           0057bbb0 f   libSDL2:SDL_dynapi.o
 0001:0017abc0       _SDL_MouseIsHaptic         0057bbc0 f   libSDL2:SDL_dynapi.o
 0001:0017abd0       _SDL_HapticOpenFromMouse   0057bbd0 f   libSDL2:SDL_dynapi.o
 0001:0017abe0       _SDL_JoystickIsHaptic      0057bbe0 f   libSDL2:SDL_dynapi.o
 0001:0017abf0       _SDL_HapticOpenFromJoystick 0057bbf0 f   libSDL2:SDL_dynapi.o
 0001:0017ac00       _SDL_HapticClose           0057bc00 f   libSDL2:SDL_dynapi.o
 0001:0017ac10       _SDL_HapticNumEffects      0057bc10 f   libSDL2:SDL_dynapi.o
 0001:0017ac20       _SDL_HapticNumEffectsPlaying 0057bc20 f   libSDL2:SDL_dynapi.o
 0001:0017ac30       _SDL_HapticQuery           0057bc30 f   libSDL2:SDL_dynapi.o
 0001:0017ac40       _SDL_HapticNumAxes         0057bc40 f   libSDL2:SDL_dynapi.o
 0001:0017ac50       _SDL_HapticEffectSupported 0057bc50 f   libSDL2:SDL_dynapi.o
 0001:0017ac60       _SDL_HapticNewEffect       0057bc60 f   libSDL2:SDL_dynapi.o
 0001:0017ac70       _SDL_HapticUpdateEffect    0057bc70 f   libSDL2:SDL_dynapi.o
 0001:0017ac80       _SDL_HapticRunEffect       0057bc80 f   libSDL2:SDL_dynapi.o
 0001:0017ac90       _SDL_HapticStopEffect      0057bc90 f   libSDL2:SDL_dynapi.o
 0001:0017aca0       _SDL_HapticDestroyEffect   0057bca0 f   libSDL2:SDL_dynapi.o
 0001:0017acb0       _SDL_HapticGetEffectStatus 0057bcb0 f   libSDL2:SDL_dynapi.o
 0001:0017acc0       _SDL_HapticSetGain         0057bcc0 f   libSDL2:SDL_dynapi.o
 0001:0017acd0       _SDL_HapticSetAutocenter   0057bcd0 f   libSDL2:SDL_dynapi.o
 0001:0017ace0       _SDL_HapticPause           0057bce0 f   libSDL2:SDL_dynapi.o
 0001:0017acf0       _SDL_HapticUnpause         0057bcf0 f   libSDL2:SDL_dynapi.o
 0001:0017ad00       _SDL_HapticStopAll         0057bd00 f   libSDL2:SDL_dynapi.o
 0001:0017ad10       _SDL_HapticRumbleSupported 0057bd10 f   libSDL2:SDL_dynapi.o
 0001:0017ad20       _SDL_HapticRumbleInit      0057bd20 f   libSDL2:SDL_dynapi.o
 0001:0017ad30       _SDL_HapticRumblePlay      0057bd30 f   libSDL2:SDL_dynapi.o
 0001:0017ad40       _SDL_HapticRumbleStop      0057bd40 f   libSDL2:SDL_dynapi.o
 0001:0017ad50       _SDL_SetHintWithPriority   0057bd50 f   libSDL2:SDL_dynapi.o
 0001:0017ad60       _SDL_SetHint               0057bd60 f   libSDL2:SDL_dynapi.o
 0001:0017ad70       _SDL_GetHint               0057bd70 f   libSDL2:SDL_dynapi.o
 0001:0017ad80       _SDL_AddHintCallback       0057bd80 f   libSDL2:SDL_dynapi.o
 0001:0017ad90       _SDL_DelHintCallback       0057bd90 f   libSDL2:SDL_dynapi.o
 0001:0017ada0       _SDL_ClearHints            0057bda0 f   libSDL2:SDL_dynapi.o
 0001:0017adb0       _SDL_NumJoysticks          0057bdb0 f   libSDL2:SDL_dynapi.o
 0001:0017adc0       _SDL_JoystickNameForIndex  0057bdc0 f   libSDL2:SDL_dynapi.o
 0001:0017add0       _SDL_JoystickOpen          0057bdd0 f   libSDL2:SDL_dynapi.o
 0001:0017ade0       _SDL_JoystickName          0057bde0 f   libSDL2:SDL_dynapi.o
 0001:0017adf0       _SDL_JoystickGetDeviceGUID 0057bdf0 f   libSDL2:SDL_dynapi.o
 0001:0017ae10       _SDL_JoystickGetGUID       0057be10 f   libSDL2:SDL_dynapi.o
 0001:0017ae30       _SDL_JoystickGetGUIDString 0057be30 f   libSDL2:SDL_dynapi.o
 0001:0017ae40       _SDL_JoystickGetGUIDFromString 0057be40 f   libSDL2:SDL_dynapi.o
 0001:0017ae60       _SDL_JoystickGetAttached   0057be60 f   libSDL2:SDL_dynapi.o
 0001:0017ae70       _SDL_JoystickInstanceID    0057be70 f   libSDL2:SDL_dynapi.o
 0001:0017ae80       _SDL_JoystickNumAxes       0057be80 f   libSDL2:SDL_dynapi.o
 0001:0017ae90       _SDL_JoystickNumBalls      0057be90 f   libSDL2:SDL_dynapi.o
 0001:0017aea0       _SDL_JoystickNumHats       0057bea0 f   libSDL2:SDL_dynapi.o
 0001:0017aeb0       _SDL_JoystickNumButtons    0057beb0 f   libSDL2:SDL_dynapi.o
 0001:0017aec0       _SDL_JoystickUpdate        0057bec0 f   libSDL2:SDL_dynapi.o
 0001:0017aed0       _SDL_JoystickEventState    0057bed0 f   libSDL2:SDL_dynapi.o
 0001:0017aee0       _SDL_JoystickGetAxis       0057bee0 f   libSDL2:SDL_dynapi.o
 0001:0017aef0       _SDL_JoystickGetHat        0057bef0 f   libSDL2:SDL_dynapi.o
 0001:0017af00       _SDL_JoystickGetBall       0057bf00 f   libSDL2:SDL_dynapi.o
 0001:0017af10       _SDL_JoystickGetButton     0057bf10 f   libSDL2:SDL_dynapi.o
 0001:0017af20       _SDL_JoystickClose         0057bf20 f   libSDL2:SDL_dynapi.o
 0001:0017af30       _SDL_GetKeyboardFocus      0057bf30 f   libSDL2:SDL_dynapi.o
 0001:0017af40       _SDL_GetKeyboardState      0057bf40 f   libSDL2:SDL_dynapi.o
 0001:0017af50       _SDL_GetModState           0057bf50 f   libSDL2:SDL_dynapi.o
 0001:0017af60       _SDL_SetModState           0057bf60 f   libSDL2:SDL_dynapi.o
 0001:0017af70       _SDL_GetKeyFromScancode    0057bf70 f   libSDL2:SDL_dynapi.o
 0001:0017af80       _SDL_GetScancodeFromKey    0057bf80 f   libSDL2:SDL_dynapi.o
 0001:0017af90       _SDL_GetScancodeName       0057bf90 f   libSDL2:SDL_dynapi.o
 0001:0017afa0       _SDL_GetScancodeFromName   0057bfa0 f   libSDL2:SDL_dynapi.o
 0001:0017afb0       _SDL_GetKeyName            0057bfb0 f   libSDL2:SDL_dynapi.o
 0001:0017afc0       _SDL_GetKeyFromName        0057bfc0 f   libSDL2:SDL_dynapi.o
 0001:0017afd0       _SDL_StartTextInput        0057bfd0 f   libSDL2:SDL_dynapi.o
 0001:0017afe0       _SDL_IsTextInputActive     0057bfe0 f   libSDL2:SDL_dynapi.o
 0001:0017aff0       _SDL_StopTextInput         0057bff0 f   libSDL2:SDL_dynapi.o
 0001:0017b000       _SDL_SetTextInputRect      0057c000 f   libSDL2:SDL_dynapi.o
 0001:0017b010       _SDL_HasScreenKeyboardSupport 0057c010 f   libSDL2:SDL_dynapi.o
 0001:0017b020       _SDL_IsScreenKeyboardShown 0057c020 f   libSDL2:SDL_dynapi.o
 0001:0017b030       _SDL_LoadObject            0057c030 f   libSDL2:SDL_dynapi.o
 0001:0017b040       _SDL_LoadFunction          0057c040 f   libSDL2:SDL_dynapi.o
 0001:0017b050       _SDL_UnloadObject          0057c050 f   libSDL2:SDL_dynapi.o
 0001:0017b060       _SDL_LogSetAllPriority     0057c060 f   libSDL2:SDL_dynapi.o
 0001:0017b070       _SDL_LogSetPriority        0057c070 f   libSDL2:SDL_dynapi.o
 0001:0017b080       _SDL_LogGetPriority        0057c080 f   libSDL2:SDL_dynapi.o
 0001:0017b090       _SDL_LogResetPriorities    0057c090 f   libSDL2:SDL_dynapi.o
 0001:0017b0a0       _SDL_LogMessageV           0057c0a0 f   libSDL2:SDL_dynapi.o
 0001:0017b0b0       _SDL_LogGetOutputFunction  0057c0b0 f   libSDL2:SDL_dynapi.o
 0001:0017b0c0       _SDL_LogSetOutputFunction  0057c0c0 f   libSDL2:SDL_dynapi.o
 0001:0017b0d0       _SDL_SetMainReady          0057c0d0 f   libSDL2:SDL_dynapi.o
 0001:0017b0e0       _SDL_ShowMessageBox        0057c0e0 f   libSDL2:SDL_dynapi.o
 0001:0017b0f0       _SDL_ShowSimpleMessageBox  0057c0f0 f   libSDL2:SDL_dynapi.o
 0001:0017b100       _SDL_GetMouseFocus         0057c100 f   libSDL2:SDL_dynapi.o
 0001:0017b110       _SDL_GetMouseState         0057c110 f   libSDL2:SDL_dynapi.o
 0001:0017b120       _SDL_GetRelativeMouseState 0057c120 f   libSDL2:SDL_dynapi.o
 0001:0017b130       _SDL_WarpMouseInWindow     0057c130 f   libSDL2:SDL_dynapi.o
 0001:0017b140       _SDL_SetRelativeMouseMode  0057c140 f   libSDL2:SDL_dynapi.o
 0001:0017b150       _SDL_GetRelativeMouseMode  0057c150 f   libSDL2:SDL_dynapi.o
 0001:0017b160       _SDL_CreateCursor          0057c160 f   libSDL2:SDL_dynapi.o
 0001:0017b170       _SDL_CreateColorCursor     0057c170 f   libSDL2:SDL_dynapi.o
 0001:0017b180       _SDL_CreateSystemCursor    0057c180 f   libSDL2:SDL_dynapi.o
 0001:0017b190       _SDL_SetCursor             0057c190 f   libSDL2:SDL_dynapi.o
 0001:0017b1a0       _SDL_GetCursor             0057c1a0 f   libSDL2:SDL_dynapi.o
 0001:0017b1b0       _SDL_GetDefaultCursor      0057c1b0 f   libSDL2:SDL_dynapi.o
 0001:0017b1c0       _SDL_FreeCursor            0057c1c0 f   libSDL2:SDL_dynapi.o
 0001:0017b1d0       _SDL_ShowCursor            0057c1d0 f   libSDL2:SDL_dynapi.o
 0001:0017b1e0       _SDL_CreateMutex           0057c1e0 f   libSDL2:SDL_dynapi.o
 0001:0017b1f0       _SDL_LockMutex             0057c1f0 f   libSDL2:SDL_dynapi.o
 0001:0017b200       _SDL_TryLockMutex          0057c200 f   libSDL2:SDL_dynapi.o
 0001:0017b210       _SDL_UnlockMutex           0057c210 f   libSDL2:SDL_dynapi.o
 0001:0017b220       _SDL_DestroyMutex          0057c220 f   libSDL2:SDL_dynapi.o
 0001:0017b230       _SDL_CreateSemaphore       0057c230 f   libSDL2:SDL_dynapi.o
 0001:0017b240       _SDL_DestroySemaphore      0057c240 f   libSDL2:SDL_dynapi.o
 0001:0017b250       _SDL_SemWait               0057c250 f   libSDL2:SDL_dynapi.o
 0001:0017b260       _SDL_SemTryWait            0057c260 f   libSDL2:SDL_dynapi.o
 0001:0017b270       _SDL_SemWaitTimeout        0057c270 f   libSDL2:SDL_dynapi.o
 0001:0017b280       _SDL_SemPost               0057c280 f   libSDL2:SDL_dynapi.o
 0001:0017b290       _SDL_SemValue              0057c290 f   libSDL2:SDL_dynapi.o
 0001:0017b2a0       _SDL_CreateCond            0057c2a0 f   libSDL2:SDL_dynapi.o
 0001:0017b2b0       _SDL_DestroyCond           0057c2b0 f   libSDL2:SDL_dynapi.o
 0001:0017b2c0       _SDL_CondSignal            0057c2c0 f   libSDL2:SDL_dynapi.o
 0001:0017b2d0       _SDL_CondBroadcast         0057c2d0 f   libSDL2:SDL_dynapi.o
 0001:0017b2e0       _SDL_CondWait              0057c2e0 f   libSDL2:SDL_dynapi.o
 0001:0017b2f0       _SDL_CondWaitTimeout       0057c2f0 f   libSDL2:SDL_dynapi.o
 0001:0017b300       _SDL_GetPixelFormatName    0057c300 f   libSDL2:SDL_dynapi.o
 0001:0017b310       _SDL_PixelFormatEnumToMasks 0057c310 f   libSDL2:SDL_dynapi.o
 0001:0017b320       _SDL_MasksToPixelFormatEnum 0057c320 f   libSDL2:SDL_dynapi.o
 0001:0017b330       _SDL_AllocFormat           0057c330 f   libSDL2:SDL_dynapi.o
 0001:0017b340       _SDL_FreeFormat            0057c340 f   libSDL2:SDL_dynapi.o
 0001:0017b350       _SDL_AllocPalette          0057c350 f   libSDL2:SDL_dynapi.o
 0001:0017b360       _SDL_SetPixelFormatPalette 0057c360 f   libSDL2:SDL_dynapi.o
 0001:0017b370       _SDL_SetPaletteColors      0057c370 f   libSDL2:SDL_dynapi.o
 0001:0017b380       _SDL_FreePalette           0057c380 f   libSDL2:SDL_dynapi.o
 0001:0017b390       _SDL_MapRGB                0057c390 f   libSDL2:SDL_dynapi.o
 0001:0017b3c0       _SDL_MapRGBA               0057c3c0 f   libSDL2:SDL_dynapi.o
 0001:0017b3f0       _SDL_GetRGB                0057c3f0 f   libSDL2:SDL_dynapi.o
 0001:0017b400       _SDL_GetRGBA               0057c400 f   libSDL2:SDL_dynapi.o
 0001:0017b410       _SDL_CalculateGammaRamp    0057c410 f   libSDL2:SDL_dynapi.o
 0001:0017b420       _SDL_GetPlatform           0057c420 f   libSDL2:SDL_dynapi.o
 0001:0017b430       _SDL_GetPowerInfo          0057c430 f   libSDL2:SDL_dynapi.o
 0001:0017b440       _SDL_HasIntersection       0057c440 f   libSDL2:SDL_dynapi.o
 0001:0017b450       _SDL_IntersectRect         0057c450 f   libSDL2:SDL_dynapi.o
 0001:0017b460       _SDL_UnionRect             0057c460 f   libSDL2:SDL_dynapi.o
 0001:0017b470       _SDL_EnclosePoints         0057c470 f   libSDL2:SDL_dynapi.o
 0001:0017b480       _SDL_IntersectRectAndLine  0057c480 f   libSDL2:SDL_dynapi.o
 0001:0017b490       _SDL_GetNumRenderDrivers   0057c490 f   libSDL2:SDL_dynapi.o
 0001:0017b4a0       _SDL_GetRenderDriverInfo   0057c4a0 f   libSDL2:SDL_dynapi.o
 0001:0017b4b0       _SDL_CreateWindowAndRenderer 0057c4b0 f   libSDL2:SDL_dynapi.o
 0001:0017b4c0       _SDL_CreateRenderer        0057c4c0 f   libSDL2:SDL_dynapi.o
 0001:0017b4d0       _SDL_CreateSoftwareRenderer 0057c4d0 f   libSDL2:SDL_dynapi.o
 0001:0017b4e0       _SDL_GetRenderer           0057c4e0 f   libSDL2:SDL_dynapi.o
 0001:0017b4f0       _SDL_GetRendererInfo       0057c4f0 f   libSDL2:SDL_dynapi.o
 0001:0017b500       _SDL_GetRendererOutputSize 0057c500 f   libSDL2:SDL_dynapi.o
 0001:0017b510       _SDL_CreateTexture         0057c510 f   libSDL2:SDL_dynapi.o
 0001:0017b520       _SDL_CreateTextureFromSurface 0057c520 f   libSDL2:SDL_dynapi.o
 0001:0017b530       _SDL_QueryTexture          0057c530 f   libSDL2:SDL_dynapi.o
 0001:0017b540       _SDL_SetTextureColorMod    0057c540 f   libSDL2:SDL_dynapi.o
 0001:0017b570       _SDL_GetTextureColorMod    0057c570 f   libSDL2:SDL_dynapi.o
 0001:0017b580       _SDL_SetTextureAlphaMod    0057c580 f   libSDL2:SDL_dynapi.o
 0001:0017b590       _SDL_GetTextureAlphaMod    0057c590 f   libSDL2:SDL_dynapi.o
 0001:0017b5a0       _SDL_SetTextureBlendMode   0057c5a0 f   libSDL2:SDL_dynapi.o
 0001:0017b5b0       _SDL_GetTextureBlendMode   0057c5b0 f   libSDL2:SDL_dynapi.o
 0001:0017b5c0       _SDL_UpdateTexture         0057c5c0 f   libSDL2:SDL_dynapi.o
 0001:0017b5d0       _SDL_UpdateYUVTexture      0057c5d0 f   libSDL2:SDL_dynapi.o
 0001:0017b5e0       _SDL_LockTexture           0057c5e0 f   libSDL2:SDL_dynapi.o
 0001:0017b5f0       _SDL_UnlockTexture         0057c5f0 f   libSDL2:SDL_dynapi.o
 0001:0017b600       _SDL_RenderTargetSupported 0057c600 f   libSDL2:SDL_dynapi.o
 0001:0017b610       _SDL_SetRenderTarget       0057c610 f   libSDL2:SDL_dynapi.o
 0001:0017b620       _SDL_GetRenderTarget       0057c620 f   libSDL2:SDL_dynapi.o
 0001:0017b630       _SDL_RenderSetLogicalSize  0057c630 f   libSDL2:SDL_dynapi.o
 0001:0017b640       _SDL_RenderGetLogicalSize  0057c640 f   libSDL2:SDL_dynapi.o
 0001:0017b650       _SDL_RenderSetViewport     0057c650 f   libSDL2:SDL_dynapi.o
 0001:0017b660       _SDL_RenderGetViewport     0057c660 f   libSDL2:SDL_dynapi.o
 0001:0017b670       _SDL_RenderSetClipRect     0057c670 f   libSDL2:SDL_dynapi.o
 0001:0017b680       _SDL_RenderGetClipRect     0057c680 f   libSDL2:SDL_dynapi.o
 0001:0017b690       _SDL_RenderSetScale        0057c690 f   libSDL2:SDL_dynapi.o
 0001:0017b6a0       _SDL_RenderGetScale        0057c6a0 f   libSDL2:SDL_dynapi.o
 0001:0017b6b0       _SDL_SetRenderDrawColor    0057c6b0 f   libSDL2:SDL_dynapi.o
 0001:0017b6e0       _SDL_GetRenderDrawColor    0057c6e0 f   libSDL2:SDL_dynapi.o
 0001:0017b6f0       _SDL_SetRenderDrawBlendMode 0057c6f0 f   libSDL2:SDL_dynapi.o
 0001:0017b700       _SDL_GetRenderDrawBlendMode 0057c700 f   libSDL2:SDL_dynapi.o
 0001:0017b710       _SDL_RenderClear           0057c710 f   libSDL2:SDL_dynapi.o
 0001:0017b720       _SDL_RenderDrawPoint       0057c720 f   libSDL2:SDL_dynapi.o
 0001:0017b730       _SDL_RenderDrawPoints      0057c730 f   libSDL2:SDL_dynapi.o
 0001:0017b740       _SDL_RenderDrawLine        0057c740 f   libSDL2:SDL_dynapi.o
 0001:0017b750       _SDL_RenderDrawLines       0057c750 f   libSDL2:SDL_dynapi.o
 0001:0017b760       _SDL_RenderDrawRect        0057c760 f   libSDL2:SDL_dynapi.o
 0001:0017b770       _SDL_RenderDrawRects       0057c770 f   libSDL2:SDL_dynapi.o
 0001:0017b780       _SDL_RenderFillRect        0057c780 f   libSDL2:SDL_dynapi.o
 0001:0017b790       _SDL_RenderFillRects       0057c790 f   libSDL2:SDL_dynapi.o
 0001:0017b7a0       _SDL_RenderCopy            0057c7a0 f   libSDL2:SDL_dynapi.o
 0001:0017b7b0       _SDL_RenderCopyEx          0057c7b0 f   libSDL2:SDL_dynapi.o
 0001:0017b7c0       _SDL_RenderReadPixels      0057c7c0 f   libSDL2:SDL_dynapi.o
 0001:0017b7d0       _SDL_RenderPresent         0057c7d0 f   libSDL2:SDL_dynapi.o
 0001:0017b7e0       _SDL_DestroyTexture        0057c7e0 f   libSDL2:SDL_dynapi.o
 0001:0017b7f0       _SDL_DestroyRenderer       0057c7f0 f   libSDL2:SDL_dynapi.o
 0001:0017b800       _SDL_GL_BindTexture        0057c800 f   libSDL2:SDL_dynapi.o
 0001:0017b810       _SDL_GL_UnbindTexture      0057c810 f   libSDL2:SDL_dynapi.o
 0001:0017b820       _SDL_RWFromFile            0057c820 f   libSDL2:SDL_dynapi.o
 0001:0017b830       _SDL_RWFromMem             0057c830 f   libSDL2:SDL_dynapi.o
 0001:0017b840       _SDL_RWFromConstMem        0057c840 f   libSDL2:SDL_dynapi.o
 0001:0017b850       _SDL_AllocRW               0057c850 f   libSDL2:SDL_dynapi.o
 0001:0017b860       _SDL_FreeRW                0057c860 f   libSDL2:SDL_dynapi.o
 0001:0017b870       _SDL_ReadU8                0057c870 f   libSDL2:SDL_dynapi.o
 0001:0017b880       _SDL_ReadLE16              0057c880 f   libSDL2:SDL_dynapi.o
 0001:0017b890       _SDL_ReadBE16              0057c890 f   libSDL2:SDL_dynapi.o
 0001:0017b8a0       _SDL_ReadLE32              0057c8a0 f   libSDL2:SDL_dynapi.o
 0001:0017b8b0       _SDL_ReadBE32              0057c8b0 f   libSDL2:SDL_dynapi.o
 0001:0017b8c0       _SDL_ReadLE64              0057c8c0 f   libSDL2:SDL_dynapi.o
 0001:0017b8d0       _SDL_ReadBE64              0057c8d0 f   libSDL2:SDL_dynapi.o
 0001:0017b8e0       _SDL_WriteU8               0057c8e0 f   libSDL2:SDL_dynapi.o
 0001:0017b8f0       _SDL_WriteLE16             0057c8f0 f   libSDL2:SDL_dynapi.o
 0001:0017b900       _SDL_WriteBE16             0057c900 f   libSDL2:SDL_dynapi.o
 0001:0017b910       _SDL_WriteLE32             0057c910 f   libSDL2:SDL_dynapi.o
 0001:0017b920       _SDL_WriteBE32             0057c920 f   libSDL2:SDL_dynapi.o
 0001:0017b930       _SDL_WriteLE64             0057c930 f   libSDL2:SDL_dynapi.o
 0001:0017b940       _SDL_WriteBE64             0057c940 f   libSDL2:SDL_dynapi.o
 0001:0017b950       _SDL_CreateShapedWindow    0057c950 f   libSDL2:SDL_dynapi.o
 0001:0017b960       _SDL_IsShapedWindow        0057c960 f   libSDL2:SDL_dynapi.o
 0001:0017b970       _SDL_SetWindowShape        0057c970 f   libSDL2:SDL_dynapi.o
 0001:0017b980       _SDL_GetShapedWindowMode   0057c980 f   libSDL2:SDL_dynapi.o
 0001:0017b990       _SDL_malloc                0057c990 f   libSDL2:SDL_dynapi.o
 0001:0017b9a0       _SDL_calloc                0057c9a0 f   libSDL2:SDL_dynapi.o
 0001:0017b9b0       _SDL_realloc               0057c9b0 f   libSDL2:SDL_dynapi.o
 0001:0017b9c0       _SDL_free                  0057c9c0 f   libSDL2:SDL_dynapi.o
 0001:0017b9d0       _SDL_getenv                0057c9d0 f   libSDL2:SDL_dynapi.o
 0001:0017b9e0       _SDL_setenv                0057c9e0 f   libSDL2:SDL_dynapi.o
 0001:0017b9f0       _SDL_qsort                 0057c9f0 f   libSDL2:SDL_dynapi.o
 0001:0017ba00       _SDL_abs                   0057ca00 f   libSDL2:SDL_dynapi.o
 0001:0017ba10       _SDL_isdigit               0057ca10 f   libSDL2:SDL_dynapi.o
 0001:0017ba20       _SDL_isspace               0057ca20 f   libSDL2:SDL_dynapi.o
 0001:0017ba30       _SDL_toupper               0057ca30 f   libSDL2:SDL_dynapi.o
 0001:0017ba40       _SDL_tolower               0057ca40 f   libSDL2:SDL_dynapi.o
 0001:0017ba50       _SDL_memset                0057ca50 f   libSDL2:SDL_dynapi.o
 0001:0017ba60       _SDL_memcpy                0057ca60 f   libSDL2:SDL_dynapi.o
 0001:0017ba70       _SDL_memmove               0057ca70 f   libSDL2:SDL_dynapi.o
 0001:0017ba80       _SDL_memcmp                0057ca80 f   libSDL2:SDL_dynapi.o
 0001:0017ba90       _SDL_wcslen                0057ca90 f   libSDL2:SDL_dynapi.o
 0001:0017baa0       _SDL_wcslcpy               0057caa0 f   libSDL2:SDL_dynapi.o
 0001:0017bab0       _SDL_wcslcat               0057cab0 f   libSDL2:SDL_dynapi.o
 0001:0017bac0       _SDL_strlen                0057cac0 f   libSDL2:SDL_dynapi.o
 0001:0017bad0       _SDL_strlcpy               0057cad0 f   libSDL2:SDL_dynapi.o
 0001:0017bae0       _SDL_utf8strlcpy           0057cae0 f   libSDL2:SDL_dynapi.o
 0001:0017baf0       _SDL_strlcat               0057caf0 f   libSDL2:SDL_dynapi.o
 0001:0017bb00       _SDL_strdup                0057cb00 f   libSDL2:SDL_dynapi.o
 0001:0017bb10       _SDL_strrev                0057cb10 f   libSDL2:SDL_dynapi.o
 0001:0017bb20       _SDL_strupr                0057cb20 f   libSDL2:SDL_dynapi.o
 0001:0017bb30       _SDL_strlwr                0057cb30 f   libSDL2:SDL_dynapi.o
 0001:0017bb40       _SDL_strchr                0057cb40 f   libSDL2:SDL_dynapi.o
 0001:0017bb50       _SDL_strrchr               0057cb50 f   libSDL2:SDL_dynapi.o
 0001:0017bb60       _SDL_strstr                0057cb60 f   libSDL2:SDL_dynapi.o
 0001:0017bb70       _SDL_itoa                  0057cb70 f   libSDL2:SDL_dynapi.o
 0001:0017bb80       _SDL_uitoa                 0057cb80 f   libSDL2:SDL_dynapi.o
 0001:0017bb90       _SDL_ltoa                  0057cb90 f   libSDL2:SDL_dynapi.o
 0001:0017bba0       _SDL_ultoa                 0057cba0 f   libSDL2:SDL_dynapi.o
 0001:0017bbb0       _SDL_lltoa                 0057cbb0 f   libSDL2:SDL_dynapi.o
 0001:0017bbc0       _SDL_ulltoa                0057cbc0 f   libSDL2:SDL_dynapi.o
 0001:0017bbd0       _SDL_atoi                  0057cbd0 f   libSDL2:SDL_dynapi.o
 0001:0017bbe0       _SDL_atof                  0057cbe0 f   libSDL2:SDL_dynapi.o
 0001:0017bbf0       _SDL_strtol                0057cbf0 f   libSDL2:SDL_dynapi.o
 0001:0017bc00       _SDL_strtoul               0057cc00 f   libSDL2:SDL_dynapi.o
 0001:0017bc10       _SDL_strtoll               0057cc10 f   libSDL2:SDL_dynapi.o
 0001:0017bc20       _SDL_strtoull              0057cc20 f   libSDL2:SDL_dynapi.o
 0001:0017bc30       _SDL_strtod                0057cc30 f   libSDL2:SDL_dynapi.o
 0001:0017bc40       _SDL_strcmp                0057cc40 f   libSDL2:SDL_dynapi.o
 0001:0017bc50       _SDL_strncmp               0057cc50 f   libSDL2:SDL_dynapi.o
 0001:0017bc60       _SDL_strcasecmp            0057cc60 f   libSDL2:SDL_dynapi.o
 0001:0017bc70       _SDL_strncasecmp           0057cc70 f   libSDL2:SDL_dynapi.o
 0001:0017bc80       _SDL_vsnprintf             0057cc80 f   libSDL2:SDL_dynapi.o
 0001:0017bc90       _SDL_acos                  0057cc90 f   libSDL2:SDL_dynapi.o
 0001:0017bca0       _SDL_asin                  0057cca0 f   libSDL2:SDL_dynapi.o
 0001:0017bcb0       _SDL_atan                  0057ccb0 f   libSDL2:SDL_dynapi.o
 0001:0017bcc0       _SDL_atan2                 0057ccc0 f   libSDL2:SDL_dynapi.o
 0001:0017bcd0       _SDL_ceil                  0057ccd0 f   libSDL2:SDL_dynapi.o
 0001:0017bce0       _SDL_copysign              0057cce0 f   libSDL2:SDL_dynapi.o
 0001:0017bcf0       _SDL_cos                   0057ccf0 f   libSDL2:SDL_dynapi.o
 0001:0017bd00       _SDL_cosf                  0057cd00 f   libSDL2:SDL_dynapi.o
 0001:0017bd10       _SDL_fabs                  0057cd10 f   libSDL2:SDL_dynapi.o
 0001:0017bd20       _SDL_floor                 0057cd20 f   libSDL2:SDL_dynapi.o
 0001:0017bd30       _SDL_log                   0057cd30 f   libSDL2:SDL_dynapi.o
 0001:0017bd40       _SDL_pow                   0057cd40 f   libSDL2:SDL_dynapi.o
 0001:0017bd50       _SDL_scalbn                0057cd50 f   libSDL2:SDL_dynapi.o
 0001:0017bd60       _SDL_sin                   0057cd60 f   libSDL2:SDL_dynapi.o
 0001:0017bd70       _SDL_sinf                  0057cd70 f   libSDL2:SDL_dynapi.o
 0001:0017bd80       _SDL_sqrt                  0057cd80 f   libSDL2:SDL_dynapi.o
 0001:0017bd90       _SDL_iconv_open            0057cd90 f   libSDL2:SDL_dynapi.o
 0001:0017bda0       _SDL_iconv_close           0057cda0 f   libSDL2:SDL_dynapi.o
 0001:0017bdb0       _SDL_iconv                 0057cdb0 f   libSDL2:SDL_dynapi.o
 0001:0017bdc0       _SDL_iconv_string          0057cdc0 f   libSDL2:SDL_dynapi.o
 0001:0017bdd0       _SDL_CreateRGBSurface      0057cdd0 f   libSDL2:SDL_dynapi.o
 0001:0017bde0       _SDL_CreateRGBSurfaceFrom  0057cde0 f   libSDL2:SDL_dynapi.o
 0001:0017bdf0       _SDL_FreeSurface           0057cdf0 f   libSDL2:SDL_dynapi.o
 0001:0017be00       _SDL_SetSurfacePalette     0057ce00 f   libSDL2:SDL_dynapi.o
 0001:0017be10       _SDL_LockSurface           0057ce10 f   libSDL2:SDL_dynapi.o
 0001:0017be20       _SDL_UnlockSurface         0057ce20 f   libSDL2:SDL_dynapi.o
 0001:0017be30       _SDL_LoadBMP_RW            0057ce30 f   libSDL2:SDL_dynapi.o
 0001:0017be40       _SDL_SaveBMP_RW            0057ce40 f   libSDL2:SDL_dynapi.o
 0001:0017be50       _SDL_SetSurfaceRLE         0057ce50 f   libSDL2:SDL_dynapi.o
 0001:0017be60       _SDL_SetColorKey           0057ce60 f   libSDL2:SDL_dynapi.o
 0001:0017be70       _SDL_GetColorKey           0057ce70 f   libSDL2:SDL_dynapi.o
 0001:0017be80       _SDL_SetSurfaceColorMod    0057ce80 f   libSDL2:SDL_dynapi.o
 0001:0017beb0       _SDL_GetSurfaceColorMod    0057ceb0 f   libSDL2:SDL_dynapi.o
 0001:0017bec0       _SDL_SetSurfaceAlphaMod    0057cec0 f   libSDL2:SDL_dynapi.o
 0001:0017bed0       _SDL_GetSurfaceAlphaMod    0057ced0 f   libSDL2:SDL_dynapi.o
 0001:0017bee0       _SDL_SetSurfaceBlendMode   0057cee0 f   libSDL2:SDL_dynapi.o
 0001:0017bef0       _SDL_GetSurfaceBlendMode   0057cef0 f   libSDL2:SDL_dynapi.o
 0001:0017bf00       _SDL_SetClipRect           0057cf00 f   libSDL2:SDL_dynapi.o
 0001:0017bf10       _SDL_GetClipRect           0057cf10 f   libSDL2:SDL_dynapi.o
 0001:0017bf20       _SDL_ConvertSurface        0057cf20 f   libSDL2:SDL_dynapi.o
 0001:0017bf30       _SDL_ConvertSurfaceFormat  0057cf30 f   libSDL2:SDL_dynapi.o
 0001:0017bf40       _SDL_ConvertPixels         0057cf40 f   libSDL2:SDL_dynapi.o
 0001:0017bf50       _SDL_FillRect              0057cf50 f   libSDL2:SDL_dynapi.o
 0001:0017bf60       _SDL_FillRects             0057cf60 f   libSDL2:SDL_dynapi.o
 0001:0017bf70       _SDL_UpperBlit             0057cf70 f   libSDL2:SDL_dynapi.o
 0001:0017bf80       _SDL_LowerBlit             0057cf80 f   libSDL2:SDL_dynapi.o
 0001:0017bf90       _SDL_SoftStretch           0057cf90 f   libSDL2:SDL_dynapi.o
 0001:0017bfa0       _SDL_UpperBlitScaled       0057cfa0 f   libSDL2:SDL_dynapi.o
 0001:0017bfb0       _SDL_LowerBlitScaled       0057cfb0 f   libSDL2:SDL_dynapi.o
 0001:0017bfc0       _SDL_GetWindowWMInfo       0057cfc0 f   libSDL2:SDL_dynapi.o
 0001:0017bfd0       _SDL_GetThreadName         0057cfd0 f   libSDL2:SDL_dynapi.o
 0001:0017bfe0       _SDL_ThreadID              0057cfe0 f   libSDL2:SDL_dynapi.o
 0001:0017bff0       _SDL_GetThreadID           0057cff0 f   libSDL2:SDL_dynapi.o
 0001:0017c000       _SDL_SetThreadPriority     0057d000 f   libSDL2:SDL_dynapi.o
 0001:0017c010       _SDL_WaitThread            0057d010 f   libSDL2:SDL_dynapi.o
 0001:0017c020       _SDL_DetachThread          0057d020 f   libSDL2:SDL_dynapi.o
 0001:0017c030       _SDL_TLSCreate             0057d030 f   libSDL2:SDL_dynapi.o
 0001:0017c040       _SDL_TLSGet                0057d040 f   libSDL2:SDL_dynapi.o
 0001:0017c050       _SDL_TLSSet                0057d050 f   libSDL2:SDL_dynapi.o
 0001:0017c060       _SDL_GetTicks              0057d060 f   libSDL2:SDL_dynapi.o
 0001:0017c070       _SDL_GetPerformanceCounter 0057d070 f   libSDL2:SDL_dynapi.o
 0001:0017c080       _SDL_GetPerformanceFrequency 0057d080 f   libSDL2:SDL_dynapi.o
 0001:0017c090       _SDL_Delay                 0057d090 f   libSDL2:SDL_dynapi.o
 0001:0017c0a0       _SDL_AddTimer              0057d0a0 f   libSDL2:SDL_dynapi.o
 0001:0017c0b0       _SDL_RemoveTimer           0057d0b0 f   libSDL2:SDL_dynapi.o
 0001:0017c0c0       _SDL_GetNumTouchDevices    0057d0c0 f   libSDL2:SDL_dynapi.o
 0001:0017c0d0       _SDL_GetTouchDevice        0057d0d0 f   libSDL2:SDL_dynapi.o
 0001:0017c0e0       _SDL_GetNumTouchFingers    0057d0e0 f   libSDL2:SDL_dynapi.o
 0001:0017c0f0       _SDL_GetTouchFinger        0057d0f0 f   libSDL2:SDL_dynapi.o
 0001:0017c100       _SDL_GetVersion            0057d100 f   libSDL2:SDL_dynapi.o
 0001:0017c110       _SDL_GetRevision           0057d110 f   libSDL2:SDL_dynapi.o
 0001:0017c120       _SDL_GetRevisionNumber     0057d120 f   libSDL2:SDL_dynapi.o
 0001:0017c130       _SDL_GetNumVideoDrivers    0057d130 f   libSDL2:SDL_dynapi.o
 0001:0017c140       _SDL_GetVideoDriver        0057d140 f   libSDL2:SDL_dynapi.o
 0001:0017c150       _SDL_VideoInit             0057d150 f   libSDL2:SDL_dynapi.o
 0001:0017c160       _SDL_VideoQuit             0057d160 f   libSDL2:SDL_dynapi.o
 0001:0017c170       _SDL_GetCurrentVideoDriver 0057d170 f   libSDL2:SDL_dynapi.o
 0001:0017c180       _SDL_GetNumVideoDisplays   0057d180 f   libSDL2:SDL_dynapi.o
 0001:0017c190       _SDL_GetDisplayName        0057d190 f   libSDL2:SDL_dynapi.o
 0001:0017c1a0       _SDL_GetDisplayBounds      0057d1a0 f   libSDL2:SDL_dynapi.o
 0001:0017c1b0       _SDL_GetNumDisplayModes    0057d1b0 f   libSDL2:SDL_dynapi.o
 0001:0017c1c0       _SDL_GetDisplayMode        0057d1c0 f   libSDL2:SDL_dynapi.o
 0001:0017c1d0       _SDL_GetDesktopDisplayMode 0057d1d0 f   libSDL2:SDL_dynapi.o
 0001:0017c1e0       _SDL_GetCurrentDisplayMode 0057d1e0 f   libSDL2:SDL_dynapi.o
 0001:0017c1f0       _SDL_GetClosestDisplayMode 0057d1f0 f   libSDL2:SDL_dynapi.o
 0001:0017c200       _SDL_GetWindowDisplayIndex 0057d200 f   libSDL2:SDL_dynapi.o
 0001:0017c210       _SDL_SetWindowDisplayMode  0057d210 f   libSDL2:SDL_dynapi.o
 0001:0017c220       _SDL_GetWindowDisplayMode  0057d220 f   libSDL2:SDL_dynapi.o
 0001:0017c230       _SDL_GetWindowPixelFormat  0057d230 f   libSDL2:SDL_dynapi.o
 0001:0017c240       _SDL_CreateWindow          0057d240 f   libSDL2:SDL_dynapi.o
 0001:0017c250       _SDL_CreateWindowFrom      0057d250 f   libSDL2:SDL_dynapi.o
 0001:0017c260       _SDL_GetWindowID           0057d260 f   libSDL2:SDL_dynapi.o
 0001:0017c270       _SDL_GetWindowFromID       0057d270 f   libSDL2:SDL_dynapi.o
 0001:0017c280       _SDL_GetWindowFlags        0057d280 f   libSDL2:SDL_dynapi.o
 0001:0017c290       _SDL_SetWindowTitle        0057d290 f   libSDL2:SDL_dynapi.o
 0001:0017c2a0       _SDL_GetWindowTitle        0057d2a0 f   libSDL2:SDL_dynapi.o
 0001:0017c2b0       _SDL_SetWindowIcon         0057d2b0 f   libSDL2:SDL_dynapi.o
 0001:0017c2c0       _SDL_SetWindowData         0057d2c0 f   libSDL2:SDL_dynapi.o
 0001:0017c2d0       _SDL_GetWindowData         0057d2d0 f   libSDL2:SDL_dynapi.o
 0001:0017c2e0       _SDL_SetWindowPosition     0057d2e0 f   libSDL2:SDL_dynapi.o
 0001:0017c2f0       _SDL_GetWindowPosition     0057d2f0 f   libSDL2:SDL_dynapi.o
 0001:0017c300       _SDL_SetWindowSize         0057d300 f   libSDL2:SDL_dynapi.o
 0001:0017c310       _SDL_GetWindowSize         0057d310 f   libSDL2:SDL_dynapi.o
 0001:0017c320       _SDL_SetWindowMinimumSize  0057d320 f   libSDL2:SDL_dynapi.o
 0001:0017c330       _SDL_GetWindowMinimumSize  0057d330 f   libSDL2:SDL_dynapi.o
 0001:0017c340       _SDL_SetWindowMaximumSize  0057d340 f   libSDL2:SDL_dynapi.o
 0001:0017c350       _SDL_GetWindowMaximumSize  0057d350 f   libSDL2:SDL_dynapi.o
 0001:0017c360       _SDL_SetWindowBordered     0057d360 f   libSDL2:SDL_dynapi.o
 0001:0017c370       _SDL_ShowWindow            0057d370 f   libSDL2:SDL_dynapi.o
 0001:0017c380       _SDL_HideWindow            0057d380 f   libSDL2:SDL_dynapi.o
 0001:0017c390       _SDL_RaiseWindow           0057d390 f   libSDL2:SDL_dynapi.o
 0001:0017c3a0       _SDL_MaximizeWindow        0057d3a0 f   libSDL2:SDL_dynapi.o
 0001:0017c3b0       _SDL_MinimizeWindow        0057d3b0 f   libSDL2:SDL_dynapi.o
 0001:0017c3c0       _SDL_RestoreWindow         0057d3c0 f   libSDL2:SDL_dynapi.o
 0001:0017c3d0       _SDL_SetWindowFullscreen   0057d3d0 f   libSDL2:SDL_dynapi.o
 0001:0017c3e0       _SDL_GetWindowSurface      0057d3e0 f   libSDL2:SDL_dynapi.o
 0001:0017c3f0       _SDL_UpdateWindowSurface   0057d3f0 f   libSDL2:SDL_dynapi.o
 0001:0017c400       _SDL_UpdateWindowSurfaceRects 0057d400 f   libSDL2:SDL_dynapi.o
 0001:0017c410       _SDL_SetWindowGrab         0057d410 f   libSDL2:SDL_dynapi.o
 0001:0017c420       _SDL_GetWindowGrab         0057d420 f   libSDL2:SDL_dynapi.o
 0001:0017c430       _SDL_SetWindowBrightness   0057d430 f   libSDL2:SDL_dynapi.o
 0001:0017c440       _SDL_GetWindowBrightness   0057d440 f   libSDL2:SDL_dynapi.o
 0001:0017c450       _SDL_SetWindowGammaRamp    0057d450 f   libSDL2:SDL_dynapi.o
 0001:0017c460       _SDL_GetWindowGammaRamp    0057d460 f   libSDL2:SDL_dynapi.o
 0001:0017c470       _SDL_DestroyWindow         0057d470 f   libSDL2:SDL_dynapi.o
 0001:0017c480       _SDL_IsScreenSaverEnabled  0057d480 f   libSDL2:SDL_dynapi.o
 0001:0017c490       _SDL_EnableScreenSaver     0057d490 f   libSDL2:SDL_dynapi.o
 0001:0017c4a0       _SDL_DisableScreenSaver    0057d4a0 f   libSDL2:SDL_dynapi.o
 0001:0017c4b0       _SDL_GL_LoadLibrary        0057d4b0 f   libSDL2:SDL_dynapi.o
 0001:0017c4c0       _SDL_GL_GetProcAddress     0057d4c0 f   libSDL2:SDL_dynapi.o
 0001:0017c4d0       _SDL_GL_UnloadLibrary      0057d4d0 f   libSDL2:SDL_dynapi.o
 0001:0017c4e0       _SDL_GL_ExtensionSupported 0057d4e0 f   libSDL2:SDL_dynapi.o
 0001:0017c4f0       _SDL_GL_SetAttribute       0057d4f0 f   libSDL2:SDL_dynapi.o
 0001:0017c500       _SDL_GL_GetAttribute       0057d500 f   libSDL2:SDL_dynapi.o
 0001:0017c510       _SDL_GL_CreateContext      0057d510 f   libSDL2:SDL_dynapi.o
 0001:0017c520       _SDL_GL_MakeCurrent        0057d520 f   libSDL2:SDL_dynapi.o
 0001:0017c530       _SDL_GL_GetCurrentWindow   0057d530 f   libSDL2:SDL_dynapi.o
 0001:0017c540       _SDL_GL_GetCurrentContext  0057d540 f   libSDL2:SDL_dynapi.o
 0001:0017c550       _SDL_GL_GetDrawableSize    0057d550 f   libSDL2:SDL_dynapi.o
 0001:0017c560       _SDL_GL_SetSwapInterval    0057d560 f   libSDL2:SDL_dynapi.o
 0001:0017c570       _SDL_GL_GetSwapInterval    0057d570 f   libSDL2:SDL_dynapi.o
 0001:0017c580       _SDL_GL_SwapWindow         0057d580 f   libSDL2:SDL_dynapi.o
 0001:0017c590       _SDL_GL_DeleteContext      0057d590 f   libSDL2:SDL_dynapi.o
 0001:0017c5a0       _SDL_vsscanf               0057d5a0 f   libSDL2:SDL_dynapi.o
 0001:0017c5b0       _SDL_GameControllerAddMappingsFromRW 0057d5b0 f   libSDL2:SDL_dynapi.o
 0001:0017c5c0       _SDL_GL_ResetAttributes    0057d5c0 f   libSDL2:SDL_dynapi.o
 0001:0017c5d0       _SDL_HasAVX                0057d5d0 f   libSDL2:SDL_dynapi.o
 0001:0017c5e0       _SDL_GetDefaultAssertionHandler 0057d5e0 f   libSDL2:SDL_dynapi.o
 0001:0017c5f0       _SDL_GetAssertionHandler   0057d5f0 f   libSDL2:SDL_dynapi.o
 0001:0017c600       _SDL_DXGIGetOutputInfo     0057d600 f   libSDL2:SDL_dynapi.o
 0001:0017c610       _SDL_RenderIsClipEnabled   0057d610 f   libSDL2:SDL_dynapi.o
 0001:0017c620       _SDL_WarpMouseGlobal       0057d620 f   libSDL2:SDL_dynapi.o
 0001:0017c630       _SDL_sqrtf                 0057d630 f   libSDL2:SDL_dynapi.o
 0001:0017c640       _SDL_tan                   0057d640 f   libSDL2:SDL_dynapi.o
 0001:0017c650       _SDL_tanf                  0057d650 f   libSDL2:SDL_dynapi.o
 0001:0017c660       _SDL_CaptureMouse          0057d660 f   libSDL2:SDL_dynapi.o
 0001:0017c670       _SDL_SetWindowHitTest      0057d670 f   libSDL2:SDL_dynapi.o
 0001:0017c680       _SDL_GetGlobalMouseState   0057d680 f   libSDL2:SDL_dynapi.o
 0001:0017c690       _SDL_HasAVX2               0057d690 f   libSDL2:SDL_dynapi.o
 0001:0017c6a0       _SDL_QueueAudio            0057d6a0 f   libSDL2:SDL_dynapi.o
 0001:0017c6b0       _SDL_GetQueuedAudioSize    0057d6b0 f   libSDL2:SDL_dynapi.o
 0001:0017c6c0       _SDL_ClearQueuedAudio      0057d6c0 f   libSDL2:SDL_dynapi.o
 0001:0017c6d0       _SDL_GetGrabbedWindow      0057d6d0 f   libSDL2:SDL_dynapi.o
 0001:0017c6e0       _SDL_SetWindowsMessageHook 0057d6e0 f   libSDL2:SDL_dynapi.o
 0001:0017c6f0       _SDL_GetDisplayDPI         0057d6f0 f   libSDL2:SDL_dynapi.o
 0001:0017c700       _SDL_JoystickCurrentPowerLevel 0057d700 f   libSDL2:SDL_dynapi.o
 0001:0017c710       _SDL_GameControllerFromInstanceID 0057d710 f   libSDL2:SDL_dynapi.o
 0001:0017c720       _SDL_JoystickFromInstanceID 0057d720 f   libSDL2:SDL_dynapi.o
 0001:0017c730       _SDL_SetError              0057d730 f   libSDL2:SDL_dynapi.o
 0001:0017c780       _SDL_sscanf                0057d780 f   libSDL2:SDL_dynapi.o
 0001:0017c7b0       _SDL_snprintf              0057d7b0 f   libSDL2:SDL_dynapi.o
 0001:0017c7e0       _SDL_Log                   0057d7e0 f   libSDL2:SDL_dynapi.o
 0001:0017c810       _SDL_LogMessage            0057d810 f   libSDL2:SDL_dynapi.o
 0001:0017c840       _SDL_LogVerbose            0057d840 f   libSDL2:SDL_dynapi.o
 0001:0017c870       _SDL_LogDebug              0057d870 f   libSDL2:SDL_dynapi.o
 0001:0017c8a0       _SDL_LogInfo               0057d8a0 f   libSDL2:SDL_dynapi.o
 0001:0017c8d0       _SDL_LogWarn               0057d8d0 f   libSDL2:SDL_dynapi.o
 0001:0017c900       _SDL_LogError              0057d900 f   libSDL2:SDL_dynapi.o
 0001:0017c930       _SDL_LogCritical           0057d930 f   libSDL2:SDL_dynapi.o
 0001:0017ce00       _SDL_SYS_AddJoystickDevice 0057de00 f   libSDL2:SDL_windowsjoystick.o
 0001:0017ce40       _SDL_SYS_NumJoysticks      0057de40 f   libSDL2:SDL_windowsjoystick.o
 0001:0017ce70       _SDL_SYS_JoystickDetect    0057de70 f   libSDL2:SDL_windowsjoystick.o
 0001:0017d080       _SDL_SYS_JoystickInit      0057e080 f   libSDL2:SDL_windowsjoystick.o
 0001:0017d240       _SDL_SYS_JoystickNameForDeviceIndex 0057e240 f   libSDL2:SDL_windowsjoystick.o
 0001:0017d260       _SDL_SYS_GetInstanceIdOfDeviceIndex 0057e260 f   libSDL2:SDL_windowsjoystick.o
 0001:0017d280       _SDL_SYS_JoystickOpen      0057e280 f   libSDL2:SDL_windowsjoystick.o
 0001:0017d320       _SDL_SYS_JoystickAttached  0057e320 f   libSDL2:SDL_windowsjoystick.o
 0001:0017d340       _SDL_SYS_JoystickUpdate    0057e340 f   libSDL2:SDL_windowsjoystick.o
 0001:0017d390       _SDL_SYS_JoystickClose     0057e390 f   libSDL2:SDL_windowsjoystick.o
 0001:0017d3e0       _SDL_SYS_JoystickQuit      0057e3e0 f   libSDL2:SDL_windowsjoystick.o
 0001:0017d4c0       _SDL_SYS_JoystickGetDeviceGUID 0057e4c0 f   libSDL2:SDL_windowsjoystick.o
 0001:0017d500       _SDL_SYS_JoystickGetGUID   0057e500 f   libSDL2:SDL_windowsjoystick.o
 0001:0017d6c0       _SDL_SetError_REAL         0057e6c0 f   libSDL2:SDL_error.o
 0001:0017d870       _SDL_GetError_REAL         0057e870 f   libSDL2:SDL_error.o
 0001:0017d880       _SDL_ClearError_REAL       0057e880 f   libSDL2:SDL_error.o
 0001:0017d890       _SDL_Error_REAL            0057e890 f   libSDL2:SDL_error.o
 0001:0017dae0       _SDL_LogSetAllPriority_REAL 0057eae0 f   libSDL2:SDL_log.o
 0001:0017db10       _SDL_LogSetPriority_REAL   0057eb10 f   libSDL2:SDL_log.o
 0001:0017db70       _SDL_LogGetPriority_REAL   0057eb70 f   libSDL2:SDL_log.o
 0001:0017dbc0       _SDL_LogResetPriorities_REAL 0057ebc0 f   libSDL2:SDL_log.o
 0001:0017dc20       _SDL_Log_REAL              0057ec20 f   libSDL2:SDL_log.o
 0001:0017dcf0       _SDL_LogVerbose_REAL       0057ecf0 f   libSDL2:SDL_log.o
 0001:0017ddf0       _SDL_LogDebug_REAL         0057edf0 f   libSDL2:SDL_log.o
 0001:0017def0       _SDL_LogInfo_REAL          0057eef0 f   libSDL2:SDL_log.o
 0001:0017dff0       _SDL_LogWarn_REAL          0057eff0 f   libSDL2:SDL_log.o
 0001:0017e0f0       _SDL_LogError_REAL         0057f0f0 f   libSDL2:SDL_log.o
 0001:0017e1f0       _SDL_LogCritical_REAL      0057f1f0 f   libSDL2:SDL_log.o
 0001:0017e2f0       _SDL_LogMessage_REAL       0057f2f0 f   libSDL2:SDL_log.o
 0001:0017e3f0       _SDL_LogMessageV_REAL      0057f3f0 f   libSDL2:SDL_log.o
 0001:0017e510       _SDL_LogGetOutputFunction_REAL 0057f510 f   libSDL2:SDL_log.o
 0001:0017e540       _SDL_LogSetOutputFunction_REAL 0057f540 f   libSDL2:SDL_log.o
 0001:0017eb90       _SDL_memset_REAL           0057fb90 f   libSDL2:SDL_string.o
 0001:0017ed90       _SDL_memcpy_REAL           0057fd90 f   libSDL2:SDL_string.o
 0001:0017eda0       _SDL_memmove_REAL          0057fda0 f   libSDL2:SDL_string.o
 0001:0017ef60       _SDL_memcmp_REAL           0057ff60 f   libSDL2:SDL_string.o
 0001:0017efb0       _SDL_strlen_REAL           0057ffb0 f   libSDL2:SDL_string.o
 0001:0017efd0       _SDL_wcslen_REAL           0057ffd0 f   libSDL2:SDL_string.o
 0001:0017eff0       _SDL_wcslcpy_REAL          0057fff0 f   libSDL2:SDL_string.o
 0001:0017f050       _SDL_wcslcat_REAL          00580050 f   libSDL2:SDL_string.o
 0001:0017f0f0       _SDL_strlcpy_REAL          005800f0 f   libSDL2:SDL_string.o
 0001:0017f140       _SDL_utf8strlcpy_REAL      00580140 f   libSDL2:SDL_string.o
 0001:0017f210       _SDL_strlcat_REAL          00580210 f   libSDL2:SDL_string.o
 0001:0017f2b0       _SDL_strdup_REAL           005802b0 f   libSDL2:SDL_string.o
 0001:0017f330       _SDL_strrev_REAL           00580330 f   libSDL2:SDL_string.o
 0001:0017f380       _SDL_strupr_REAL           00580380 f   libSDL2:SDL_string.o
 0001:0017f3b0       _SDL_strlwr_REAL           005803b0 f   libSDL2:SDL_string.o
 0001:0017f3e0       _SDL_strchr_REAL           005803e0 f   libSDL2:SDL_string.o
 0001:0017f410       _SDL_strrchr_REAL          00580410 f   libSDL2:SDL_string.o
 0001:0017f450       _SDL_strstr_REAL           00580450 f   libSDL2:SDL_string.o
 0001:0017f520       _SDL_itoa_REAL             00580520 f   libSDL2:SDL_string.o
 0001:0017f610       _SDL_uitoa_REAL            00580610 f   libSDL2:SDL_string.o
 0001:0017f6a0       _SDL_ltoa_REAL             005806a0 f   libSDL2:SDL_string.o
 0001:0017f790       _SDL_ultoa_REAL            00580790 f   libSDL2:SDL_string.o
 0001:0017f820       _SDL_lltoa_REAL            00580820 f   libSDL2:SDL_string.o
 0001:0017f9e0       _SDL_ulltoa_REAL           005809e0 f   libSDL2:SDL_string.o
 0001:0017fac0       _SDL_atoi_REAL             00580ac0 f   libSDL2:SDL_string.o
 0001:0017fb40       _SDL_atof_REAL             00580b40 f   libSDL2:SDL_string.o
 0001:0017fb60       _SDL_strtol_REAL           00580b60 f   libSDL2:SDL_string.o
 0001:0017fbf0       _SDL_strtoul_REAL          00580bf0 f   libSDL2:SDL_string.o
 0001:0017fda0       _SDL_strtoll_REAL          00580da0 f   libSDL2:SDL_string.o
 0001:0017fe40       _SDL_strtoull_REAL         00580e40 f   libSDL2:SDL_string.o
 0001:00180070       _SDL_strtod_REAL           00581070 f   libSDL2:SDL_string.o
 0001:001800a0       _SDL_strcmp_REAL           005810a0 f   libSDL2:SDL_string.o
 0001:00180100       _SDL_strncmp_REAL          00581100 f   libSDL2:SDL_string.o
 0001:00180180       _SDL_strcasecmp_REAL       00581180 f   libSDL2:SDL_string.o
 0001:00180200       _SDL_strncasecmp_REAL      00581200 f   libSDL2:SDL_string.o
 0001:001802a0       _SDL_vsscanf_REAL          005812a0 f   libSDL2:SDL_string.o
 0001:00180b50       _SDL_sscanf_REAL           00581b50 f   libSDL2:SDL_string.o
 0001:00180b80       _SDL_vsnprintf_REAL        00581b80 f   libSDL2:SDL_string.o
 0001:00181810       _SDL_snprintf_REAL         00582810 f   libSDL2:SDL_string.o
 0001:00181840       _SDL_TLSCreate_REAL        00582840 f   libSDL2:SDL_thread.o
 0001:00181860       _SDL_TLSGet_REAL           00582860 f   libSDL2:SDL_thread.o
 0001:00181890       _SDL_TLSSet_REAL           00582890 f   libSDL2:SDL_thread.o
 0001:00181980       _SDL_Generic_GetTLSData    00582980 f   libSDL2:SDL_thread.o
 0001:00181a20       _SDL_Generic_SetTLSData    00582a20 f   libSDL2:SDL_thread.o
 0001:00181ae0       _SDL_GetErrBuf             00582ae0 f   libSDL2:SDL_thread.o
 0001:00181e60       _SDL_RunThread             00582e60 f   libSDL2:SDL_thread.o
 0001:00181f50       _SDL_CreateThread_REAL     00582f50 f   libSDL2:SDL_thread.o
 0001:001820e0       _SDL_GetThreadID_REAL      005830e0 f   libSDL2:SDL_thread.o
 0001:00182100       _SDL_GetThreadName_REAL    00583100 f   libSDL2:SDL_thread.o
 0001:00182120       _SDL_SetThreadPriority_REAL 00583120 f   libSDL2:SDL_thread.o
 0001:00182130       _SDL_WaitThread_REAL       00583130 f   libSDL2:SDL_thread.o
 0001:00182180       _SDL_DetachThread_REAL     00583180 f   libSDL2:SDL_thread.o
 0001:00182780       _SDL_RWFromFile_REAL       00583780 f   libSDL2:SDL_rwops.o
 0001:00182aa0       _SDL_RWFromFP_REAL         00583aa0 f   libSDL2:SDL_rwops.o
 0001:00182ac0       _SDL_RWFromMem_REAL        00583ac0 f   libSDL2:SDL_rwops.o
 0001:00182b60       _SDL_RWFromConstMem_REAL   00583b60 f   libSDL2:SDL_rwops.o
 0001:00182c00       _SDL_AllocRW_REAL          00583c00 f   libSDL2:SDL_rwops.o
 0001:00182c40       _SDL_FreeRW_REAL           00583c40 f   libSDL2:SDL_rwops.o
 0001:00182c50       _SDL_ReadU8_REAL           00583c50 f   libSDL2:SDL_rwops.o
 0001:00182c90       _SDL_ReadLE16_REAL         00583c90 f   libSDL2:SDL_rwops.o
 0001:00182cd0       _SDL_ReadBE16_REAL         00583cd0 f   libSDL2:SDL_rwops.o
 0001:00182d10       _SDL_ReadLE32_REAL         00583d10 f   libSDL2:SDL_rwops.o
 0001:00182d50       _SDL_ReadBE32_REAL         00583d50 f   libSDL2:SDL_rwops.o
 0001:00182d90       _SDL_ReadLE64_REAL         00583d90 f   libSDL2:SDL_rwops.o
 0001:00182de0       _SDL_ReadBE64_REAL         00583de0 f   libSDL2:SDL_rwops.o
 0001:00182e30       _SDL_WriteU8_REAL          00583e30 f   libSDL2:SDL_rwops.o
 0001:00182e70       _SDL_WriteLE16_REAL        00583e70 f   libSDL2:SDL_rwops.o
 0001:00182eb0       _SDL_WriteBE16_REAL        00583eb0 f   libSDL2:SDL_rwops.o
 0001:00182ef0       _SDL_WriteLE32_REAL        00583ef0 f   libSDL2:SDL_rwops.o
 0001:00182f30       _SDL_WriteBE32_REAL        00583f30 f   libSDL2:SDL_rwops.o
 0001:00182f70       _SDL_WriteLE64_REAL        00583f70 f   libSDL2:SDL_rwops.o
 0001:00182fb0       _SDL_WriteBE64_REAL        00583fb0 f   libSDL2:SDL_rwops.o
 0001:00183110       _WIN_CheckWParamMouseButton 00584110 f   libSDL2:SDL_windowsevents.o
 0001:001831c0       _WIN_CheckWParamMouseButtons 005841c0 f   libSDL2:SDL_windowsevents.o
 0001:00183480       _WIN_CheckRawMouseButtons  00584480 f   libSDL2:SDL_windowsevents.o
 0001:00183740       _WIN_CheckAsyncMouseRelease 00584740 f   libSDL2:SDL_windowsevents.o
 0001:001838f0       _WIN_WindowProc@16         005848f0 f   libSDL2:SDL_windowsevents.o
 0001:00184e10       _WIN_ConvertUTF32toUTF8    00585e10 f   libSDL2:SDL_windowsevents.o
 0001:00184ed0       _SDL_SetWindowsMessageHook_REAL 00585ed0 f   libSDL2:SDL_windowsevents.o
 0001:00184ef0       _WIN_PumpEvents            00585ef0 f   libSDL2:SDL_windowsevents.o
 0001:00185050       _SDL_RegisterApp_REAL      00586050 f   libSDL2:SDL_windowsevents.o
 0001:001851e0       _SDL_UnregisterApp_REAL    005861e0 f   libSDL2:SDL_windowsevents.o
 0001:00185660       _D3D_LoadDLL               00586660 f   libSDL2:SDL_windowsvideo.o
 0001:001856e0       _SDL_Direct3D9GetAdapterIndex_REAL 005866e0 f   libSDL2:SDL_windowsvideo.o
 0001:00185860       _SDL_DXGIGetOutputInfo_REAL 00586860 f   libSDL2:SDL_windowsvideo.o
 0001:00189950       _SDL_RenderGetD3D9Device_REAL 0058a950 f   libSDL2:SDL_render_d3d.o
 0001:001899a0       _SDL_SetMainReady_REAL     0058a9a0 f   libSDL2:SDL.o
 0001:001899b0       _SDL_InitSubSystem_REAL    0058a9b0 f   libSDL2:SDL.o
 0001:00189bb0       _SDL_Init_REAL             0058abb0 f   libSDL2:SDL.o
 0001:00189db0       _SDL_QuitSubSystem_REAL    0058adb0 f   libSDL2:SDL.o
 0001:0018a020       _SDL_WasInit_REAL          0058b020 f   libSDL2:SDL.o
 0001:0018a090       _SDL_Quit_REAL             0058b090 f   libSDL2:SDL.o
 0001:0018a240       _SDL_GetVersion_REAL       0058b240 f   libSDL2:SDL.o
 0001:0018a250       _SDL_GetRevision_REAL      0058b250 f   libSDL2:SDL.o
 0001:0018a260       _SDL_GetRevisionNumber_REAL 0058b260 f   libSDL2:SDL.o
 0001:0018a270       _SDL_GetPlatform_REAL      0058b270 f   libSDL2:SDL.o
 0001:0018a280       __DllMainCRTStartup@12     0058b280 f   libSDL2:SDL.o
 0001:0018a560       _SDL_ReportAssertion_REAL  0058b560 f   libSDL2:SDL_assert.o
 0001:0018a6b0       _SDL_AssertionsQuit        0058b6b0 f   libSDL2:SDL_assert.o
 0001:0018a7b0       _SDL_SetAssertionHandler_REAL 0058b7b0 f   libSDL2:SDL_assert.o
 0001:0018a7e0       _SDL_GetAssertionReport_REAL 0058b7e0 f   libSDL2:SDL_assert.o
 0001:0018a7f0       _SDL_ResetAssertionReport_REAL 0058b7f0 f   libSDL2:SDL_assert.o
 0001:0018a830       _SDL_GetDefaultAssertionHandler_REAL 0058b830 f   libSDL2:SDL_assert.o
 0001:0018a840       _SDL_GetAssertionHandler_REAL 0058b840 f   libSDL2:SDL_assert.o
 0001:0018a860       _SDL_AtomicTryLock_REAL    0058b860 f   libSDL2:SDL_spinlock.o
 0001:0018a880       _SDL_AtomicLock_REAL       0058b880 f   libSDL2:SDL_spinlock.o
 0001:0018a8c0       _SDL_AtomicUnlock_REAL     0058b8c0 f   libSDL2:SDL_spinlock.o
 0001:0018a8d0       _SDL_AtomicCAS_REAL        0058b8d0 f   libSDL2:SDL_atomic.o
 0001:0018a920       _SDL_AtomicCASPtr_REAL     0058b920 f   libSDL2:SDL_atomic.o
 0001:0018a970       _SDL_AtomicSet_REAL        0058b970 f   libSDL2:SDL_atomic.o
 0001:0018a9d0       _SDL_AtomicSetPtr_REAL     0058b9d0 f   libSDL2:SDL_atomic.o
 0001:0018aa30       _SDL_AtomicAdd_REAL        0058ba30 f   libSDL2:SDL_atomic.o
 0001:0018aa90       _SDL_AtomicGet_REAL        0058ba90 f   libSDL2:SDL_atomic.o
 0001:0018aad0       _SDL_AtomicGetPtr_REAL     0058bad0 f   libSDL2:SDL_atomic.o
 0001:0018ad20       _SDL_RunAudio              0058bd20 f   libSDL2:SDL_audio.o
 0001:0018b160       _SDL_AddAudioDevice        0058c160 f   libSDL2:SDL_audio.o
 0001:0018b2c0       _SDL_OpenedAudioDeviceDisconnected 0058c2c0 f   libSDL2:SDL_audio.o
 0001:0018b360       _SDL_RemoveAudioDevice     0058c360 f   libSDL2:SDL_audio.o
 0001:0018b3f0       _SDL_QueueAudio_REAL       0058c3f0 f   libSDL2:SDL_audio.o
 0001:0018b630       _SDL_GetQueuedAudioSize_REAL 0058c630 f   libSDL2:SDL_audio.o
 0001:0018b6b0       _SDL_ClearQueuedAudio_REAL 0058c6b0 f   libSDL2:SDL_audio.o
 0001:0018b740       _SDL_GetNumAudioDrivers_REAL 0058c740 f   libSDL2:SDL_audio.o
 0001:0018b750       _SDL_GetAudioDriver_REAL   0058c750 f   libSDL2:SDL_audio.o
 0001:0018b770       _SDL_GetCurrentAudioDriver_REAL 0058c770 f   libSDL2:SDL_audio.o
 0001:0018b780       _SDL_GetNumAudioDevices_REAL 0058c780 f   libSDL2:SDL_audio.o
 0001:0018b8c0       _SDL_GetAudioDeviceName_REAL 0058c8c0 f   libSDL2:SDL_audio.o
 0001:0018b990       _SDL_GetAudioDeviceStatus_REAL 0058c990 f   libSDL2:SDL_audio.o
 0001:0018b9f0       _SDL_GetAudioStatus_REAL   0058c9f0 f   libSDL2:SDL_audio.o
 0001:0018ba30       _SDL_PauseAudioDevice_REAL 0058ca30 f   libSDL2:SDL_audio.o
 0001:0018ba90       _SDL_PauseAudio_REAL       0058ca90 f   libSDL2:SDL_audio.o
 0001:0018bae0       _SDL_LockAudioDevice_REAL  0058cae0 f   libSDL2:SDL_audio.o
 0001:0018bb10       _SDL_LockAudio_REAL        0058cb10 f   libSDL2:SDL_audio.o
 0001:0018bb40       _SDL_UnlockAudioDevice_REAL 0058cb40 f   libSDL2:SDL_audio.o
 0001:0018bb70       _SDL_UnlockAudio_REAL      0058cb70 f   libSDL2:SDL_audio.o
 0001:0018bba0       _SDL_CloseAudioDevice_REAL 0058cba0 f   libSDL2:SDL_audio.o
 0001:0018ce70       _SDL_OpenAudioDevice_REAL  0058de70 f   libSDL2:SDL_audio.o
 0001:0018cea0       _SDL_OpenAudio_REAL        0058dea0 f   libSDL2:SDL_audio.o
 0001:0018dc80       _SDL_CloseAudio_REAL       0058ec80 f   libSDL2:SDL_audio.o
 0001:0018dd90       _SDL_AudioQuit_REAL        0058ed90 f   libSDL2:SDL_audio.o
 0001:0018df80       _SDL_AudioInit_REAL        0058ef80 f   libSDL2:SDL_audio.o
 0001:0018e480       _SDL_FirstAudioFormat      0058f480 f   libSDL2:SDL_audio.o
 0001:0018e5c0       _SDL_NextAudioFormat       0058f5c0 f   libSDL2:SDL_audio.o
 0001:0018e600       _SDL_CalculateAudioSpec    0058f600 f   libSDL2:SDL_audio.o
 0001:0018e640       _SDL_MixAudio_REAL         0058f640 f   libSDL2:SDL_audio.o
 0001:0018e7a0       _SDL_LoadWAV_RW_REAL       0058f7a0 f   libSDL2:SDL_wave.o
 0001:0018f630       _SDL_FreeWAV_REAL          00590630 f   libSDL2:SDL_wave.o
 0001:00190b50       _SDL_ConvertAudio_REAL     00591b50 f   libSDL2:SDL_audiocvt.o
 0001:00190ba0       _SDL_BuildAudioCVT_REAL    00591ba0 f   libSDL2:SDL_audiocvt.o
 0001:001914d0       _SDL_MixAudioFormat_REAL   005924d0 f   libSDL2:SDL_mixer.o
 0001:00191930       _SDL_SetClipboardText_REAL 00592930 f   libSDL2:SDL_clipboard.o
 0001:001919b0       _SDL_GetClipboardText_REAL 005929b0 f   libSDL2:SDL_clipboard.o
 0001:00191a10       _SDL_HasClipboardText_REAL 00592a10 f   libSDL2:SDL_clipboard.o
 0001:00191a60       _SDL_GetCPUCount_REAL      00592a60 f   libSDL2:SDL_cpuinfo.o
 0001:00191ab0       _SDL_GetCPUCacheLineSize_REAL 00592ab0 f   libSDL2:SDL_cpuinfo.o
 0001:00191bf0       _SDL_HasRDTSC_REAL         00592bf0 f   libSDL2:SDL_cpuinfo.o
 0001:00192020       _SDL_HasAltiVec_REAL       00593020 f   libSDL2:SDL_cpuinfo.o
 0001:00192450       _SDL_HasMMX_REAL           00593450 f   libSDL2:SDL_cpuinfo.o
 0001:00192880       _SDL_Has3DNow_REAL         00593880 f   libSDL2:SDL_cpuinfo.o
 0001:00192cb0       _SDL_HasSSE_REAL           00593cb0 f   libSDL2:SDL_cpuinfo.o
 0001:001930e0       _SDL_HasSSE2_REAL          005940e0 f   libSDL2:SDL_cpuinfo.o
 0001:00193510       _SDL_HasSSE3_REAL          00594510 f   libSDL2:SDL_cpuinfo.o
 0001:00193940       _SDL_HasSSE41_REAL         00594940 f   libSDL2:SDL_cpuinfo.o
 0001:00193d70       _SDL_HasSSE42_REAL         00594d70 f   libSDL2:SDL_cpuinfo.o
 0001:001941a0       _SDL_HasAVX_REAL           005951a0 f   libSDL2:SDL_cpuinfo.o
 0001:001945d0       _SDL_HasAVX2_REAL          005955d0 f   libSDL2:SDL_cpuinfo.o
 0001:00194a00       _SDL_GetSystemRAM_REAL     00595a00 f   libSDL2:SDL_cpuinfo.o
 0001:00194be0       _SDL_StopEventLoop         00595be0 f   libSDL2:SDL_events.o
 0001:00194d90       _SDL_PeepEvents_REAL       00595d90 f   libSDL2:SDL_events.o
 0001:001951a0       _SDL_HasEvent_REAL         005961a0 f   libSDL2:SDL_events.o
 0001:001952e0       _SDL_HasEvents_REAL        005962e0 f   libSDL2:SDL_events.o
 0001:00195440       _SDL_FlushEvent_REAL       00596440 f   libSDL2:SDL_events.o
 0001:00195520       _SDL_FlushEvents_REAL      00596520 f   libSDL2:SDL_events.o
 0001:00195600       _SDL_StartEventLoop        00596600 f   libSDL2:SDL_events.o
 0001:00195740       _SDL_PumpEvents_REAL       00596740 f   libSDL2:SDL_events.o
 0001:00195780       _SDL_PollEvent_REAL        00596780 f   libSDL2:SDL_events.o
 0001:00195a20       _SDL_WaitEvent_REAL        00596a20 f   libSDL2:SDL_events.o
 0001:00195cb0       _SDL_WaitEventTimeout_REAL 00596cb0 f   libSDL2:SDL_events.o
 0001:00195f90       _SDL_PushEvent_REAL        00596f90 f   libSDL2:SDL_events.o
 0001:00196040       _SDL_SetEventFilter_REAL   00597040 f   libSDL2:SDL_events.o
 0001:00196120       _SDL_GetEventFilter_REAL   00597120 f   libSDL2:SDL_events.o
 0001:00196150       _SDL_AddEventWatch_REAL    00597150 f   libSDL2:SDL_events.o
 0001:001961a0       _SDL_DelEventWatch_REAL    005971a0 f   libSDL2:SDL_events.o
 0001:001961f0       _SDL_FilterEvents_REAL     005971f0 f   libSDL2:SDL_events.o
 0001:001962c0       _SDL_EventState_REAL       005972c0 f   libSDL2:SDL_events.o
 0001:001963a0       _SDL_RegisterEvents_REAL   005973a0 f   libSDL2:SDL_events.o
 0001:001963d0       _SDL_SendAppEvent          005973d0 f   libSDL2:SDL_events.o
 0001:00196430       _SDL_SendSysWMEvent        00597430 f   libSDL2:SDL_events.o
 0001:00196490       _SDL_SendKeymapChangedEvent 00597490 f   libSDL2:SDL_events.o
 0001:001964d0       _SDL_GetBasePath_REAL      005974d0 f   libSDL2:SDL_sysfilesystem.o
 0001:00196670       _SDL_GetPrefPath_REAL      00597670 f   libSDL2:SDL_sysfilesystem.o
 0001:001968e0       _SDL_PrivateGetControllerMappingForGUID 005978e0 f   libSDL2:SDL_gamecontroller.o
 0001:00196930       _SDL_GameControllerGetAxisFromString_REAL 00597930 f   libSDL2:SDL_gamecontroller.o
 0001:00196990       _SDL_GameControllerGetStringForAxis_REAL 00597990 f   libSDL2:SDL_gamecontroller.o
 0001:001969b0       _SDL_GameControllerGetButtonFromString_REAL 005979b0 f   libSDL2:SDL_gamecontroller.o
 0001:00196a10       _SDL_GameControllerGetStringForButton_REAL 00597a10 f   libSDL2:SDL_gamecontroller.o
 0001:00196a30       _SDL_PrivateGameControllerParseButton 00597a30 f   libSDL2:SDL_gamecontroller.o
 0001:00196c20       _SDL_PrivateLoadButtonMapping 00597c20 f   libSDL2:SDL_gamecontroller.o
 0001:001971d0       _SDL_PrivateGetControllerGUIDFromMappingString 005981d0 f   libSDL2:SDL_gamecontroller.o
 0001:00197240       _SDL_PrivateGetControllerNameFromMappingString 00598240 f   libSDL2:SDL_gamecontroller.o
 0001:001972c0       _SDL_PrivateGetControllerMappingFromMappingString 005982c0 f   libSDL2:SDL_gamecontroller.o
 0001:00197310       _SDL_PrivateGameControllerRefreshMapping 00598310 f   libSDL2:SDL_gamecontroller.o
 0001:00197950       _SDL_PrivateGetControllerMapping 00598950 f   libSDL2:SDL_gamecontroller.o
 0001:00197a00       _SDL_GameControllerEventWatcher 00598a00 f   libSDL2:SDL_gamecontroller.o
 0001:00198160       _SDL_GameControllerAddMapping_REAL 00599160 f   libSDL2:SDL_gamecontroller.o
 0001:00198440       _SDL_GameControllerAddMappingsFromRW_REAL 00599440 f   libSDL2:SDL_gamecontroller.o
 0001:00198640       _SDL_GameControllerMappingForGUID_REAL 00599640 f   libSDL2:SDL_gamecontroller.o
 0001:00198730       _SDL_GameControllerMapping_REAL 00599730 f   libSDL2:SDL_gamecontroller.o
 0001:00198770       _SDL_GameControllerInit    00599770 f   libSDL2:SDL_gamecontroller.o
 0001:00198890       _SDL_GameControllerNameForIndex_REAL 00599890 f   libSDL2:SDL_gamecontroller.o
 0001:001988c0       _SDL_IsGameController_REAL 005998c0 f   libSDL2:SDL_gamecontroller.o
 0001:001988e0       _SDL_GameControllerOpen_REAL 005998e0 f   libSDL2:SDL_gamecontroller.o
 0001:00198a40       _SDL_GameControllerUpdate_REAL 00599a40 f   libSDL2:SDL_gamecontroller.o
 0001:00198a50       _SDL_GameControllerGetAxis_REAL 00599a50 f   libSDL2:SDL_gamecontroller.o
 0001:00198ad0       _SDL_GameControllerGetButton_REAL 00599ad0 f   libSDL2:SDL_gamecontroller.o
 0001:00198b60       _SDL_GameControllerGetAttached_REAL 00599b60 f   libSDL2:SDL_gamecontroller.o
 0001:00198b80       _SDL_GameControllerName_REAL 00599b80 f   libSDL2:SDL_gamecontroller.o
 0001:00198ba0       _SDL_GameControllerGetJoystick_REAL 00599ba0 f   libSDL2:SDL_gamecontroller.o
 0001:00198bc0       _SDL_GameControllerFromInstanceID_REAL 00599bc0 f   libSDL2:SDL_gamecontroller.o
 0001:00198c00       _SDL_GameControllerGetBindForAxis_REAL 00599c00 f   libSDL2:SDL_gamecontroller.o
 0001:00198c90       _SDL_GameControllerGetBindForButton_REAL 00599c90 f   libSDL2:SDL_gamecontroller.o
 0001:00198d40       _SDL_GameControllerClose_REAL 00599d40 f   libSDL2:SDL_gamecontroller.o
 0001:00198dc0       _SDL_GameControllerQuit    00599dc0 f   libSDL2:SDL_gamecontroller.o
 0001:00198ea0       _SDL_PrivateGameControllerAxis 00599ea0 f   libSDL2:SDL_gamecontroller.o
 0001:00198f10       _SDL_PrivateGameControllerButton 00599f10 f   libSDL2:SDL_gamecontroller.o
 0001:00198fa0       _SDL_GameControllerEventState_REAL 00599fa0 f   libSDL2:SDL_gamecontroller.o
 0001:00199710       _SDL_RecordGesture_REAL    0059a710 f   libSDL2:SDL_gesture.o
 0001:001997a0       _SDL_SaveAllDollarTemplates_REAL 0059a7a0 f   libSDL2:SDL_gesture.o
 0001:00199840       _SDL_SaveDollarTemplate_REAL 0059a840 f   libSDL2:SDL_gesture.o
 0001:00199920       _SDL_LoadDollarTemplates_REAL 0059a920 f   libSDL2:SDL_gesture.o
 0001:00199cb0       _SDL_GestureAddTouch       0059acb0 f   libSDL2:SDL_gesture.o
 0001:00199d50       _SDL_SendGestureMulti      0059ad50 f   libSDL2:SDL_gesture.o
 0001:00199db0       _SDL_GestureProcessEvent   0059adb0 f   libSDL2:SDL_gesture.o
 0001:0019a4c0       _SDL_HapticInit            0059b4c0 f   libSDL2:SDL_haptic.o
 0001:0019a4d0       _SDL_NumHaptics_REAL       0059b4d0 f   libSDL2:SDL_haptic.o
 0001:0019a4e0       _SDL_HapticName_REAL       0059b4e0 f   libSDL2:SDL_haptic.o
 0001:0019a520       _SDL_HapticOpened_REAL     0059b520 f   libSDL2:SDL_haptic.o
 0001:0019a580       _SDL_HapticIndex_REAL      0059b580 f   libSDL2:SDL_haptic.o
 0001:0019a5d0       _SDL_MouseIsHaptic_REAL    0059b5d0 f   libSDL2:SDL_haptic.o
 0001:0019a5e0       _SDL_JoystickIsHaptic_REAL 0059b5e0 f   libSDL2:SDL_haptic.o
 0001:0019a620       _SDL_HapticOpenFromJoystick_REAL 0059b620 f   libSDL2:SDL_haptic.o
 0001:0019a750       _SDL_HapticClose_REAL      0059b750 f   libSDL2:SDL_haptic.o
 0001:0019a860       _SDL_HapticQuit            0059b860 f   libSDL2:SDL_haptic.o
 0001:0019a870       _SDL_HapticNumEffects_REAL 0059b870 f   libSDL2:SDL_haptic.o
 0001:0019a8c0       _SDL_HapticNumEffectsPlaying_REAL 0059b8c0 f   libSDL2:SDL_haptic.o
 0001:0019a910       _SDL_HapticQuery_REAL      0059b910 f   libSDL2:SDL_haptic.o
 0001:0019a960       _SDL_HapticNumAxes_REAL    0059b960 f   libSDL2:SDL_haptic.o
 0001:0019a9b0       _SDL_HapticEffectSupported_REAL 0059b9b0 f   libSDL2:SDL_haptic.o
 0001:0019aa00       _SDL_HapticNewEffect_REAL  0059ba00 f   libSDL2:SDL_haptic.o
 0001:0019ab20       _SDL_HapticUpdateEffect_REAL 0059bb20 f   libSDL2:SDL_haptic.o
 0001:0019abf0       _SDL_HapticRunEffect_REAL  0059bbf0 f   libSDL2:SDL_haptic.o
 0001:0019ac80       _SDL_HapticStopEffect_REAL 0059bc80 f   libSDL2:SDL_haptic.o
 0001:0019ad10       _SDL_HapticDestroyEffect_REAL 0059bd10 f   libSDL2:SDL_haptic.o
 0001:0019ad80       _SDL_HapticGetEffectStatus_REAL 0059bd80 f   libSDL2:SDL_haptic.o
 0001:0019ae20       _SDL_HapticSetGain_REAL    0059be20 f   libSDL2:SDL_haptic.o
 0001:0019af00       _SDL_HapticOpen_REAL       0059bf00 f   libSDL2:SDL_haptic.o
 0001:0019b050       _SDL_HapticOpenFromMouse_REAL 0059c050 f   libSDL2:SDL_haptic.o
 0001:0019b080       _SDL_HapticSetAutocenter_REAL 0059c080 f   libSDL2:SDL_haptic.o
 0001:0019b110       _SDL_HapticPause_REAL      0059c110 f   libSDL2:SDL_haptic.o
 0001:0019b170       _SDL_HapticUnpause_REAL    0059c170 f   libSDL2:SDL_haptic.o
 0001:0019b1d0       _SDL_HapticStopAll_REAL    0059c1d0 f   libSDL2:SDL_haptic.o
 0001:0019b220       _SDL_HapticRumbleSupported_REAL 0059c220 f   libSDL2:SDL_haptic.o
 0001:0019b270       _SDL_HapticRumbleInit_REAL 0059c270 f   libSDL2:SDL_haptic.o
 0001:0019b370       _SDL_HapticRumblePlay_REAL 0059c370 f   libSDL2:SDL_haptic.o
 0001:0019b580       _SDL_HapticRumbleStop_REAL 0059c580 f   libSDL2:SDL_haptic.o
 0001:0019b630       _SDL_SetHintWithPriority_REAL 0059c630 f   libSDL2:SDL_hints.o
 0001:0019b770       _SDL_SetHint_REAL          0059c770 f   libSDL2:SDL_hints.o
 0001:0019b890       _SDL_GetHint_REAL          0059c890 f   libSDL2:SDL_hints.o
 0001:0019b8f0       _SDL_AddHintCallback_REAL  0059c8f0 f   libSDL2:SDL_hints.o
 0001:0019bb00       _SDL_DelHintCallback_REAL  0059cb00 f   libSDL2:SDL_hints.o
 0001:0019bb80       _SDL_ClearHints_REAL       0059cb80 f   libSDL2:SDL_hints.o
 0001:0019bc00       _SDL_JoystickInit          0059cc00 f   libSDL2:SDL_joystick.o
 0001:0019bc50       _SDL_NumJoysticks_REAL     0059cc50 f   libSDL2:SDL_joystick.o
 0001:0019bc60       _SDL_JoystickNameForIndex_REAL 0059cc60 f   libSDL2:SDL_joystick.o
 0001:0019bca0       _SDL_JoystickOpen_REAL     0059cca0 f   libSDL2:SDL_joystick.o
 0001:0019bf80       _SDL_PrivateJoystickValid  0059cf80 f   libSDL2:SDL_joystick.o
 0001:0019bfb0       _SDL_JoystickNumAxes_REAL  0059cfb0 f   libSDL2:SDL_joystick.o
 0001:0019bfe0       _SDL_JoystickNumHats_REAL  0059cfe0 f   libSDL2:SDL_joystick.o
 0001:0019c010       _SDL_JoystickNumBalls_REAL 0059d010 f   libSDL2:SDL_joystick.o
 0001:0019c040       _SDL_JoystickNumButtons_REAL 0059d040 f   libSDL2:SDL_joystick.o
 0001:0019c070       _SDL_JoystickGetAxis_REAL  0059d070 f   libSDL2:SDL_joystick.o
 0001:0019c0c0       _SDL_JoystickGetHat_REAL   0059d0c0 f   libSDL2:SDL_joystick.o
 0001:0019c110       _SDL_JoystickGetBall_REAL  0059d110 f   libSDL2:SDL_joystick.o
 0001:0019c190       _SDL_JoystickGetButton_REAL 0059d190 f   libSDL2:SDL_joystick.o
 0001:0019c1e0       _SDL_JoystickGetAttached_REAL 0059d1e0 f   libSDL2:SDL_joystick.o
 0001:0019c210       _SDL_JoystickInstanceID_REAL 0059d210 f   libSDL2:SDL_joystick.o
 0001:0019c240       _SDL_JoystickFromInstanceID_REAL 0059d240 f   libSDL2:SDL_joystick.o
 0001:0019c280       _SDL_JoystickName_REAL     0059d280 f   libSDL2:SDL_joystick.o
 0001:0019c2b0       _SDL_JoystickClose_REAL    0059d2b0 f   libSDL2:SDL_joystick.o
 0001:0019c370       _SDL_JoystickQuit          0059d370 f   libSDL2:SDL_joystick.o
 0001:0019c440       _SDL_PrivateJoystickAxis   0059d440 f   libSDL2:SDL_joystick.o
 0001:0019c540       _SDL_PrivateJoystickHat    0059d540 f   libSDL2:SDL_joystick.o
 0001:0019c600       _SDL_PrivateJoystickBall   0059d600 f   libSDL2:SDL_joystick.o
 0001:0019c6f0       _SDL_PrivateJoystickButton 0059d6f0 f   libSDL2:SDL_joystick.o
 0001:0019c7d0       _SDL_JoystickUpdate_REAL   0059d7d0 f   libSDL2:SDL_joystick.o
 0001:0019cb10       _SDL_JoystickEventState_REAL 0059db10 f   libSDL2:SDL_joystick.o
 0001:0019cbc0       _SDL_JoystickGetDeviceGUID_REAL 0059dbc0 f   libSDL2:SDL_joystick.o
 0001:0019cc50       _SDL_JoystickGetGUID_REAL  0059dc50 f   libSDL2:SDL_joystick.o
 0001:0019ccc0       _SDL_JoystickGetGUIDString_REAL 0059dcc0 f   libSDL2:SDL_joystick.o
 0001:0019cfe0       _SDL_JoystickGetGUIDFromString_REAL 0059dfe0 f   libSDL2:SDL_joystick.o
 0001:0019d110       _SDL_PrivateJoystickBatteryLevel 0059e110 f   libSDL2:SDL_joystick.o
 0001:0019d120       _SDL_JoystickCurrentPowerLevel_REAL 0059e120 f   libSDL2:SDL_joystick.o
 0001:0019d150       _SDL_UCS4ToUTF8            0059e150 f   libSDL2:SDL_keyboard.o
 0001:0019d2a0       _SDL_KeyboardInit          0059e2a0 f   libSDL2:SDL_keyboard.o
 0001:0019d2d0       _SDL_ResetKeyboard         0059e2d0 f   libSDL2:SDL_keyboard.o
 0001:0019d3b0       _SDL_GetDefaultKeymap      0059e3b0 f   libSDL2:SDL_keyboard.o
 0001:0019d3e0       _SDL_SetKeymap             0059e3e0 f   libSDL2:SDL_keyboard.o
 0001:0019d420       _SDL_SetScancodeName       0059e420 f   libSDL2:SDL_keyboard.o
 0001:0019d430       _SDL_GetKeyboardFocus_REAL 0059e430 f   libSDL2:SDL_keyboard.o
 0001:0019d440       _SDL_SetKeyboardFocus      0059e440 f   libSDL2:SDL_keyboard.o
 0001:0019d560       _SDL_SendKeyboardKey       0059e560 f   libSDL2:SDL_keyboard.o
 0001:0019d6c0       _SDL_SendKeyboardText      0059e6c0 f   libSDL2:SDL_keyboard.o
 0001:0019d750       _SDL_SendEditingText       0059e750 f   libSDL2:SDL_keyboard.o
 0001:0019d7f0       _SDL_KeyboardQuit          0059e7f0 f   libSDL2:SDL_keyboard.o
 0001:0019d800       _SDL_GetKeyboardState_REAL 0059e800 f   libSDL2:SDL_keyboard.o
 0001:0019d820       _SDL_GetModState_REAL      0059e820 f   libSDL2:SDL_keyboard.o
 0001:0019d830       _SDL_SetModState_REAL      0059e830 f   libSDL2:SDL_keyboard.o
 0001:0019d840       _SDL_ToggleModState        0059e840 f   libSDL2:SDL_keyboard.o
 0001:0019d880       _SDL_GetKeyFromScancode_REAL 0059e880 f   libSDL2:SDL_keyboard.o
 0001:0019d8c0       _SDL_GetScancodeFromKey_REAL 0059e8c0 f   libSDL2:SDL_keyboard.o
 0001:0019d8f0       _SDL_GetScancodeName_REAL  0059e8f0 f   libSDL2:SDL_keyboard.o
 0001:0019d930       _SDL_GetScancodeFromName_REAL 0059e930 f   libSDL2:SDL_keyboard.o
 0001:0019d9a0       _SDL_GetKeyName_REAL       0059e9a0 f   libSDL2:SDL_keyboard.o
 0001:0019dae0       _SDL_GetKeyFromName_REAL   0059eae0 f   libSDL2:SDL_keyboard.o
 0001:0019e400       _SDL_GetNumVideoDrivers_REAL 0059f400 f   libSDL2:SDL_video.o
 0001:0019e410       _SDL_GetVideoDriver_REAL   0059f410 f   libSDL2:SDL_video.o
 0001:0019e430       _SDL_GetCurrentVideoDriver_REAL 0059f430 f   libSDL2:SDL_video.o
 0001:0019e460       _SDL_GetVideoDevice        0059f460 f   libSDL2:SDL_video.o
 0001:0019e470       _SDL_AddBasicVideoDisplay  0059f470 f   libSDL2:SDL_video.o
 0001:0019e5b0       _SDL_AddVideoDisplay       0059f5b0 f   libSDL2:SDL_video.o
 0001:0019e680       _SDL_GetNumVideoDisplays_REAL 0059f680 f   libSDL2:SDL_video.o
 0001:0019e6b0       _SDL_GetDisplayDriverData  0059f6b0 f   libSDL2:SDL_video.o
 0001:0019e710       _SDL_GetDisplayName_REAL   0059f710 f   libSDL2:SDL_video.o
 0001:0019e770       _SDL_GetDisplayBounds_REAL 0059f770 f   libSDL2:SDL_video.o
 0001:0019e840       _SDL_GetDisplayDPI_REAL    0059f840 f   libSDL2:SDL_video.o
 0001:0019e8e0       _SDL_AddDisplayMode        0059f8e0 f   libSDL2:SDL_video.o
 0001:0019ea80       _SDL_GetNumDisplayModes_REAL 0059fa80 f   libSDL2:SDL_video.o
 0001:0019eb20       _SDL_GetDisplayMode_REAL   0059fb20 f   libSDL2:SDL_video.o
 0001:0019ec80       _SDL_GetDesktopDisplayMode_REAL 0059fc80 f   libSDL2:SDL_video.o
 0001:0019ed20       _SDL_GetCurrentDisplayMode_REAL 0059fd20 f   libSDL2:SDL_video.o
 0001:0019edc0       _SDL_GetClosestDisplayMode_REAL 0059fdc0 f   libSDL2:SDL_video.o
 0001:0019ee30       _SDL_GetWindowDisplayIndex_REAL 0059fe30 f   libSDL2:SDL_video.o
 0001:0019f5d0       _SDL_GetDisplayForWindow   005a05d0 f   libSDL2:SDL_video.o
 0001:0019f610       _SDL_GetWindowDisplayMode_REAL 005a0610 f   libSDL2:SDL_video.o
 0001:0019f7b0       _SDL_SetWindowDisplayMode_REAL 005a07b0 f   libSDL2:SDL_video.o
 0001:0019f8e0       _SDL_GetWindowPixelFormat_REAL 005a08e0 f   libSDL2:SDL_video.o
 0001:0019f950       _SDL_GetWindowID_REAL      005a0950 f   libSDL2:SDL_video.o
 0001:0019f9a0       _SDL_GetWindowFromID_REAL  005a09a0 f   libSDL2:SDL_video.o
 0001:0019f9e0       _SDL_GetWindowFlags_REAL   005a09e0 f   libSDL2:SDL_video.o
 0001:0019fa30       _SDL_SetWindowTitle_REAL   005a0a30 f   libSDL2:SDL_video.o
 0001:0019fad0       _SDL_GetWindowTitle_REAL   005a0ad0 f   libSDL2:SDL_video.o
 0001:0019fb30       _SDL_SetWindowIcon_REAL    005a0b30 f   libSDL2:SDL_video.o
 0001:0019fbd0       _SDL_SetWindowData_REAL    005a0bd0 f   libSDL2:SDL_video.o
 0001:001a0130       _SDL_GetWindowData_REAL    005a1130 f   libSDL2:SDL_video.o
 0001:001a01e0       _SDL_SetWindowPosition_REAL 005a11e0 f   libSDL2:SDL_video.o
 0001:001a0390       _SDL_GetWindowPosition_REAL 005a1390 f   libSDL2:SDL_video.o
 0001:001a04a0       _SDL_SetWindowBordered_REAL 005a14a0 f   libSDL2:SDL_video.o
 0001:001a0540       _SDL_SetWindowSize_REAL    005a1540 f   libSDL2:SDL_video.o
 0001:001a0680       _SDL_GetWindowSize_REAL    005a1680 f   libSDL2:SDL_video.o
 0001:001a06e0       _SDL_SetWindowMinimumSize_REAL 005a16e0 f   libSDL2:SDL_video.o
 0001:001a07b0       _SDL_GetWindowMinimumSize_REAL 005a17b0 f   libSDL2:SDL_video.o
 0001:001a0810       _SDL_SetWindowMaximumSize_REAL 005a1810 f   libSDL2:SDL_video.o
 0001:001a08e0       _SDL_GetWindowMaximumSize_REAL 005a18e0 f   libSDL2:SDL_video.o
 0001:001a0940       _SDL_ShowWindow_REAL       005a1940 f   libSDL2:SDL_video.o
 0001:001a09d0       _SDL_HideWindow_REAL       005a19d0 f   libSDL2:SDL_video.o
 0001:001a0a80       _SDL_RaiseWindow_REAL      005a1a80 f   libSDL2:SDL_video.o
 0001:001a0ae0       _SDL_MaximizeWindow_REAL   005a1ae0 f   libSDL2:SDL_video.o
 0001:001a0b40       _SDL_MinimizeWindow_REAL   005a1b40 f   libSDL2:SDL_video.o
 0001:001a0bc0       _SDL_RestoreWindow_REAL    005a1bc0 f   libSDL2:SDL_video.o
 0001:001a0c20       _SDL_SetWindowFullscreen_REAL 005a1c20 f   libSDL2:SDL_video.o
 0001:001a0cc0       _SDL_GetWindowSurface_REAL 005a1cc0 f   libSDL2:SDL_video.o
 0001:001a0e30       _SDL_UpdateWindowSurface_REAL 005a1e30 f   libSDL2:SDL_video.o
 0001:001a0ed0       _SDL_UpdateWindowSurfaceRects_REAL 005a1ed0 f   libSDL2:SDL_video.o
 0001:001a0f60       _SDL_GetWindowBrightness_REAL 005a1f60 f   libSDL2:SDL_video.o
 0001:001a0fb0       _SDL_GetWindowGammaRamp_REAL 005a1fb0 f   libSDL2:SDL_video.o
 0001:001a1150       _SDL_SetWindowGammaRamp_REAL 005a2150 f   libSDL2:SDL_video.o
 0001:001a12b0       _SDL_SetWindowBrightness_REAL 005a22b0 f   libSDL2:SDL_video.o
 0001:001a1450       _SDL_UpdateWindowGrab      005a2450 f   libSDL2:SDL_video.o
 0001:001a1790       _SDL_RecreateWindow        005a2790 f   libSDL2:SDL_video.o
 0001:001a1b20       _SDL_SetWindowGrab_REAL    005a2b20 f   libSDL2:SDL_video.o
 0001:001a1ba0       _SDL_GetWindowGrab_REAL    005a2ba0 f   libSDL2:SDL_video.o
 0001:001a1bf0       _SDL_GetGrabbedWindow_REAL 005a2bf0 f   libSDL2:SDL_video.o
 0001:001a1c00       _SDL_OnWindowShown         005a2c00 f   libSDL2:SDL_video.o
 0001:001a1c20       _SDL_OnWindowHidden        005a2c20 f   libSDL2:SDL_video.o
 0001:001a1c30       _SDL_OnWindowResized       005a2c30 f   libSDL2:SDL_video.o
 0001:001a1c60       _SDL_OnWindowMinimized     005a2c60 f   libSDL2:SDL_video.o
 0001:001a1c70       _SDL_OnWindowRestored      005a2c70 f   libSDL2:SDL_video.o
 0001:001a1c90       _SDL_OnWindowEnter         005a2c90 f   libSDL2:SDL_video.o
 0001:001a1cc0       _SDL_OnWindowLeave         005a2cc0 f   libSDL2:SDL_video.o
 0001:001a1cd0       _SDL_OnWindowFocusGained   005a2cd0 f   libSDL2:SDL_video.o
 0001:001a1de0       _SDL_OnWindowFocusLost     005a2de0 f   libSDL2:SDL_video.o
 0001:001a1f40       _SDL_GetFocusWindow        005a2f40 f   libSDL2:SDL_video.o
 0001:001a1f80       _SDL_IsScreenSaverEnabled_REAL 005a2f80 f   libSDL2:SDL_video.o
 0001:001a1fa0       _SDL_EnableScreenSaver_REAL 005a2fa0 f   libSDL2:SDL_video.o
 0001:001a1fe0       _SDL_DisableScreenSaver_REAL 005a2fe0 f   libSDL2:SDL_video.o
 0001:001a2020       _SDL_GL_LoadLibrary_REAL   005a3020 f   libSDL2:SDL_video.o
 0001:001a20e0       _SDL_GL_GetProcAddress_REAL 005a30e0 f   libSDL2:SDL_video.o
 0001:001a2150       _SDL_GL_UnloadLibrary_REAL 005a3150 f   libSDL2:SDL_video.o
 0001:001a21a0       _SDL_GL_ExtensionSupported_REAL 005a31a0 f   libSDL2:SDL_video.o
 0001:001a23f0       _SDL_GL_ResetAttributes_REAL 005a33f0 f   libSDL2:SDL_video.o
 0001:001a24b0       _SDL_GL_SetAttribute_REAL  005a34b0 f   libSDL2:SDL_video.o
 0001:001a26f0       _SDL_GL_GetAttribute_REAL  005a36f0 f   libSDL2:SDL_video.o
 0001:001a2cb0       _SDL_GL_CreateContext_REAL 005a3cb0 f   libSDL2:SDL_video.o
 0001:001a2d80       _SDL_GL_MakeCurrent_REAL   005a3d80 f   libSDL2:SDL_video.o
 0001:001a2f00       _SDL_DestroyWindow_REAL    005a3f00 f   libSDL2:SDL_video.o
 0001:001a31a0       _SDL_CreateWindowFrom_REAL 005a41a0 f   libSDL2:SDL_video.o
 0001:001a3290       _SDL_VideoQuit_REAL        005a4290 f   libSDL2:SDL_video.o
 0001:001a3490       _SDL_VideoInit_REAL        005a4490 f   libSDL2:SDL_video.o
 0001:001a38c0       _SDL_CreateWindow_REAL     005a48c0 f   libSDL2:SDL_video.o
 0001:001a3ce0       _SDL_GL_GetCurrentWindow_REAL 005a4ce0 f   libSDL2:SDL_video.o
 0001:001a3d10       _SDL_GL_GetCurrentContext_REAL 005a4d10 f   libSDL2:SDL_video.o
 0001:001a3d40       _SDL_GL_GetDrawableSize_REAL 005a4d40 f   libSDL2:SDL_video.o
 0001:001a3dd0       _SDL_GL_SetSwapInterval_REAL 005a4dd0 f   libSDL2:SDL_video.o
 0001:001a3e50       _SDL_GL_GetSwapInterval_REAL 005a4e50 f   libSDL2:SDL_video.o
 0001:001a3ea0       _SDL_GL_SwapWindow_REAL    005a4ea0 f   libSDL2:SDL_video.o
 0001:001a3f40       _SDL_GL_DeleteContext_REAL 005a4f40 f   libSDL2:SDL_video.o
 0001:001a3fa0       _SDL_GetWindowWMInfo_REAL  005a4fa0 f   libSDL2:SDL_video.o
 0001:001a4040       _SDL_StartTextInput_REAL   005a5040 f   libSDL2:SDL_video.o
 0001:001a40d0       _SDL_IsTextInputActive_REAL 005a50d0 f   libSDL2:SDL_video.o
 0001:001a4100       _SDL_StopTextInput_REAL    005a5100 f   libSDL2:SDL_video.o
 0001:001a4190       _SDL_SetTextInputRect_REAL 005a5190 f   libSDL2:SDL_video.o
 0001:001a41c0       _SDL_HasScreenKeyboardSupport_REAL 005a51c0 f   libSDL2:SDL_video.o
 0001:001a41f0       _SDL_IsScreenKeyboardShown_REAL 005a51f0 f   libSDL2:SDL_video.o
 0001:001a4230       _SDL_ShowMessageBox_REAL   005a5230 f   libSDL2:SDL_video.o
 0001:001a44c0       _SDL_ShowSimpleMessageBox_REAL 005a54c0 f   libSDL2:SDL_video.o
 0001:001a4550       _SDL_ShouldAllowTopmost    005a5550 f   libSDL2:SDL_video.o
 0001:001a4580       _SDL_SetWindowHitTest_REAL 005a5580 f   libSDL2:SDL_video.o
 0001:001a4620       _SDL_ComputeDiagonalDPI    005a5620 f   libSDL2:SDL_video.o
 0001:001a4680       _SDL_LoadObject_REAL       005a5680 f   libSDL2:SDL_sysloadso.o
 0001:001a4730       _SDL_LoadFunction_REAL     005a5730 f   libSDL2:SDL_sysloadso.o
 0001:001a47b0       _SDL_UnloadObject_REAL     005a57b0 f   libSDL2:SDL_sysloadso.o
 0001:001a47d0       _SDL_MouseInit             005a57d0 f   libSDL2:SDL_mouse.o
 0001:001a47e0       _SDL_GetMouse              005a57e0 f   libSDL2:SDL_mouse.o
 0001:001a47f0       _SDL_SetDoubleClickTime    005a57f0 f   libSDL2:SDL_mouse.o
 0001:001a4800       _SDL_GetMouseFocus_REAL    005a5800 f   libSDL2:SDL_mouse.o
 0001:001a4810       _SDL_SetMouseFocus         005a5810 f   libSDL2:SDL_mouse.o
 0001:001a4d00       _SDL_ResetMouse            005a5d00 f   libSDL2:SDL_mouse.o
 0001:001a5220       _SDL_SendMouseMotion       005a6220 f   libSDL2:SDL_mouse.o
 0001:001a56d0       _SDL_SendMouseButton       005a66d0 f   libSDL2:SDL_mouse.o
 0001:001a59a0       _SDL_SendMouseWheel        005a69a0 f   libSDL2:SDL_mouse.o
 0001:001a5af0       _SDL_GetMouseState_REAL    005a6af0 f   libSDL2:SDL_mouse.o
 0001:001a5b20       _SDL_GetRelativeMouseState_REAL 005a6b20 f   libSDL2:SDL_mouse.o
 0001:001a5b60       _SDL_GetGlobalMouseState_REAL 005a6b60 f   libSDL2:SDL_mouse.o
 0001:001a5bb0       _SDL_WarpMouseInWindow_REAL 005a6bb0 f   libSDL2:SDL_mouse.o
 0001:001a5c20       _SDL_WarpMouseGlobal_REAL  005a6c20 f   libSDL2:SDL_mouse.o
 0001:001a5c40       _SDL_SetRelativeMouseMode_REAL 005a6c40 f   libSDL2:SDL_mouse.o
 0001:001a5e60       _SDL_GetRelativeMouseMode_REAL 005a6e60 f   libSDL2:SDL_mouse.o
 0001:001a5e70       _SDL_CaptureMouse_REAL     005a6e70 f   libSDL2:SDL_mouse.o
 0001:001a5f20       _SDL_CreateColorCursor_REAL 005a6f20 f   libSDL2:SDL_mouse.o
 0001:001a6010       _SDL_CreateCursor_REAL     005a7010 f   libSDL2:SDL_mouse.o
 0001:001a6160       _SDL_CreateSystemCursor_REAL 005a7160 f   libSDL2:SDL_mouse.o
 0001:001a61b0       _SDL_SetCursor_REAL        005a71b0 f   libSDL2:SDL_mouse.o
 0001:001a6250       _SDL_SetDefaultCursor      005a7250 f   libSDL2:SDL_mouse.o
 0001:001a6270       _SDL_MouseQuit             005a7270 f   libSDL2:SDL_mouse.o
 0001:001a6400       _SDL_GetCursor_REAL        005a7400 f   libSDL2:SDL_mouse.o
 0001:001a6410       _SDL_GetDefaultCursor_REAL 005a7410 f   libSDL2:SDL_mouse.o
 0001:001a6420       _SDL_FreeCursor_REAL       005a7420 f   libSDL2:SDL_mouse.o
 0001:001a6490       _SDL_ShowCursor_REAL       005a7490 f   libSDL2:SDL_mouse.o
 0001:001a6510       _SDL_CreateMutex_REAL      005a7510 f   libSDL2:SDL_sysmutex.o
 0001:001a6560       _SDL_DestroyMutex_REAL     005a7560 f   libSDL2:SDL_sysmutex.o
 0001:001a6590       _SDL_LockMutex_REAL        005a7590 f   libSDL2:SDL_sysmutex.o
 0001:001a65c0       _SDL_TryLockMutex_REAL     005a75c0 f   libSDL2:SDL_sysmutex.o
 0001:001a65f0       _SDL_UnlockMutex_REAL      005a75f0 f   libSDL2:SDL_sysmutex.o
 0001:001a6620       _SDL_CreateSemaphore_REAL  005a7620 f   libSDL2:SDL_syssem.o
 0001:001a66a0       _SDL_DestroySemaphore_REAL 005a76a0 f   libSDL2:SDL_syssem.o
 0001:001a66e0       _SDL_SemWaitTimeout_REAL   005a76e0 f   libSDL2:SDL_syssem.o
 0001:001a6750       _SDL_SemTryWait_REAL       005a7750 f   libSDL2:SDL_syssem.o
 0001:001a67d0       _SDL_SemWait_REAL          005a77d0 f   libSDL2:SDL_syssem.o
 0001:001a6850       _SDL_SemValue_REAL         005a7850 f   libSDL2:SDL_syssem.o
 0001:001a6880       _SDL_SemPost_REAL          005a7880 f   libSDL2:SDL_syssem.o
 0001:001a68f0       _SDL_CreateCond_REAL       005a78f0 f   libSDL2:SDL_syscond.o
 0001:001a69a0       _SDL_DestroyCond_REAL      005a79a0 f   libSDL2:SDL_syscond.o
 0001:001a69f0       _SDL_CondSignal_REAL       005a79f0 f   libSDL2:SDL_syscond.o
 0001:001a6a70       _SDL_CondBroadcast_REAL    005a7a70 f   libSDL2:SDL_syscond.o
 0001:001a6b10       _SDL_CondWaitTimeout_REAL  005a7b10 f   libSDL2:SDL_syscond.o
 0001:001a6be0       _SDL_CondWait_REAL         005a7be0 f   libSDL2:SDL_syscond.o
 0001:001a6ed0       _SDL_GetPixelFormatName_REAL 005a7ed0 f   libSDL2:SDL_pixels.o
 0001:001a71c0       _SDL_PixelFormatEnumToMasks_REAL 005a81c0 f   libSDL2:SDL_pixels.o
 0001:001a7460       _SDL_MasksToPixelFormatEnum_REAL 005a8460 f   libSDL2:SDL_pixels.o
 0001:001a7930       _SDL_AllocFormat_REAL      005a8930 f   libSDL2:SDL_pixels.o
 0001:001a7b80       _SDL_InitFormat            005a8b80 f   libSDL2:SDL_pixels.o
 0001:001a7d30       _SDL_FreeFormat_REAL       005a8d30 f   libSDL2:SDL_pixels.o
 0001:001a7dd0       _SDL_AllocPalette_REAL     005a8dd0 f   libSDL2:SDL_pixels.o
 0001:001a7e70       _SDL_SetPixelFormatPalette_REAL 005a8e70 f   libSDL2:SDL_pixels.o
 0001:001a7f00       _SDL_SetPaletteColors_REAL 005a8f00 f   libSDL2:SDL_pixels.o
 0001:001a7f80       _SDL_FreePalette_REAL      005a8f80 f   libSDL2:SDL_pixels.o
 0001:001a7fd0       _SDL_DitherColors          005a8fd0 f   libSDL2:SDL_pixels.o
 0001:001a8050       _SDL_CalculatePitch        005a9050 f   libSDL2:SDL_pixels.o
 0001:001a80a0       _SDL_FindColor             005a90a0 f   libSDL2:SDL_pixels.o
 0001:001a8160       _SDL_MapRGB_REAL           005a9160 f   libSDL2:SDL_pixels.o
 0001:001a8250       _SDL_MapRGBA_REAL          005a9250 f   libSDL2:SDL_pixels.o
 0001:001a8360       _SDL_GetRGB_REAL           005a9360 f   libSDL2:SDL_pixels.o
 0001:001a8440       _SDL_GetRGBA_REAL          005a9440 f   libSDL2:SDL_pixels.o
 0001:001a8550       _SDL_AllocBlitMap          005a9550 f   libSDL2:SDL_pixels.o
 0001:001a8590       _SDL_InvalidateMap         005a9590 f   libSDL2:SDL_pixels.o
 0001:001a85f0       _SDL_MapSurface            005a95f0 f   libSDL2:SDL_pixels.o
 0001:001a8a90       _SDL_FreeBlitMap           005a9a90 f   libSDL2:SDL_pixels.o
 0001:001a8b00       _SDL_CalculateGammaRamp_REAL 005a9b00 f   libSDL2:SDL_pixels.o
 0001:001a8c40       _SDL_GetPowerInfo_REAL     005a9c40 f   libSDL2:SDL_power.o
 0001:001a8ca0       _SDL_HasIntersection_REAL  005a9ca0 f   libSDL2:SDL_rect.o
 0001:001a8d50       _SDL_IntersectRect_REAL    005a9d50 f   libSDL2:SDL_rect.o
 0001:001a8e50       _SDL_UnionRect_REAL        005a9e50 f   libSDL2:SDL_rect.o
 0001:001a8f60       _SDL_EnclosePoints_REAL    005a9f60 f   libSDL2:SDL_rect.o
 0001:001a9240       _SDL_IntersectRectAndLine_REAL 005aa240 f   libSDL2:SDL_rect.o
 0001:001a9810       _SDL_GetSpanEnclosingRect  005aa810 f   libSDL2:SDL_rect.o
 0001:001a9940       _SDL_GetNumRenderDrivers_REAL 005aa940 f   libSDL2:SDL_render.o
 0001:001a9950       _SDL_GetRenderDriverInfo_REAL 005aa950 f   libSDL2:SDL_render.o
 0001:001a9990       _SDL_CreateWindowAndRenderer_REAL 005aa990 f   libSDL2:SDL_render.o
 0001:001a9cd0       _SDL_CreateRenderer_REAL   005aacd0 f   libSDL2:SDL_render.o
 0001:001aa010       _SDL_CreateSoftwareRenderer_REAL 005ab010 f   libSDL2:SDL_render.o
 0001:001aa0f0       _SDL_GetRenderer_REAL      005ab0f0 f   libSDL2:SDL_render.o
 0001:001aa110       _SDL_GetRendererInfo_REAL  005ab110 f   libSDL2:SDL_render.o
 0001:001aa160       _SDL_GetRendererOutputSize_REAL 005ab160 f   libSDL2:SDL_render.o
 0001:001aa230       _SDL_QueryTexture_REAL     005ab230 f   libSDL2:SDL_render.o
 0001:001aa2b0       _SDL_SetTextureColorMod_REAL 005ab2b0 f   libSDL2:SDL_render.o
 0001:001aa4d0       _SDL_GetTextureColorMod_REAL 005ab4d0 f   libSDL2:SDL_render.o
 0001:001aa540       _SDL_SetTextureAlphaMod_REAL 005ab540 f   libSDL2:SDL_render.o
 0001:001aa690       _SDL_GetTextureAlphaMod_REAL 005ab690 f   libSDL2:SDL_render.o
 0001:001aa6e0       _SDL_SetTextureBlendMode_REAL 005ab6e0 f   libSDL2:SDL_render.o
 0001:001aa750       _SDL_GetTextureBlendMode_REAL 005ab750 f   libSDL2:SDL_render.o
 0001:001aa7a0       _SDL_LockTexture_REAL      005ab7a0 f   libSDL2:SDL_render.o
 0001:001aa910       _SDL_UnlockTexture_REAL    005ab910 f   libSDL2:SDL_render.o
 0001:001aac10       _SDL_UpdateTexture_REAL    005abc10 f   libSDL2:SDL_render.o
 0001:001ab050       _SDL_UpdateYUVTexture_REAL 005ac050 f   libSDL2:SDL_render.o
 0001:001ab430       _SDL_RenderTargetSupported_REAL 005ac430 f   libSDL2:SDL_render.o
 0001:001ab460       _SDL_SetRenderTarget_REAL  005ac460 f   libSDL2:SDL_render.o
 0001:001ab6f0       _SDL_GetRenderTarget_REAL  005ac6f0 f   libSDL2:SDL_render.o
 0001:001ab700       _SDL_RenderGetLogicalSize_REAL 005ac700 f   libSDL2:SDL_render.o
 0001:001ab750       _SDL_RenderSetViewport_REAL 005ac750 f   libSDL2:SDL_render.o
 0001:001ac0d0       _SDL_RenderSetLogicalSize_REAL 005ad0d0 f   libSDL2:SDL_render.o
 0001:001ac220       _SDL_RenderGetViewport_REAL 005ad220 f   libSDL2:SDL_render.o
 0001:001ac2b0       _SDL_RenderSetClipRect_REAL 005ad2b0 f   libSDL2:SDL_render.o
 0001:001ac400       _SDL_RenderGetClipRect_REAL 005ad400 f   libSDL2:SDL_render.o
 0001:001ac490       _SDL_RenderIsClipEnabled_REAL 005ad490 f   libSDL2:SDL_render.o
 0001:001ac4c0       _SDL_RenderSetScale_REAL   005ad4c0 f   libSDL2:SDL_render.o
 0001:001ac510       _SDL_RenderGetScale_REAL   005ad510 f   libSDL2:SDL_render.o
 0001:001ac550       _SDL_SetRenderDrawColor_REAL 005ad550 f   libSDL2:SDL_render.o
 0001:001ac5d0       _SDL_GetRenderDrawColor_REAL 005ad5d0 f   libSDL2:SDL_render.o
 0001:001ac660       _SDL_SetRenderDrawBlendMode_REAL 005ad660 f   libSDL2:SDL_render.o
 0001:001ac6a0       _SDL_GetRenderDrawBlendMode_REAL 005ad6a0 f   libSDL2:SDL_render.o
 0001:001ac6e0       _SDL_RenderClear_REAL      005ad6e0 f   libSDL2:SDL_render.o
 0001:001ac730       _SDL_RenderDrawPoint_REAL  005ad730 f   libSDL2:SDL_render.o
 0001:001ac8b0       _SDL_RenderDrawPoints_REAL 005ad8b0 f   libSDL2:SDL_render.o
 0001:001aca60       _SDL_RenderDrawLine_REAL   005ada60 f   libSDL2:SDL_render.o
 0001:001acce0       _SDL_RenderDrawLines_REAL  005adce0 f   libSDL2:SDL_render.o
 0001:001acff0       _SDL_RenderDrawRect_REAL   005adff0 f   libSDL2:SDL_render.o
 0001:001ad3b0       _SDL_RenderDrawRects_REAL  005ae3b0 f   libSDL2:SDL_render.o
 0001:001ad7f0       _SDL_RenderFillRect_REAL   005ae7f0 f   libSDL2:SDL_render.o
 0001:001ad920       _SDL_RenderFillRects_REAL  005ae920 f   libSDL2:SDL_render.o
 0001:001ada30       _SDL_RenderCopy_REAL       005aea30 f   libSDL2:SDL_render.o
 0001:001adc10       _SDL_RenderCopyEx_REAL     005aec10 f   libSDL2:SDL_render.o
 0001:001adef0       _SDL_RenderReadPixels_REAL 005aeef0 f   libSDL2:SDL_render.o
 0001:001ae050       _SDL_RenderPresent_REAL    005af050 f   libSDL2:SDL_render.o
 0001:001ae090       _SDL_DestroyTexture_REAL   005af090 f   libSDL2:SDL_render.o
 0001:001ae140       _SDL_CreateTexture_REAL    005af140 f   libSDL2:SDL_render.o
 0001:001ae810       _SDL_CreateTextureFromSurface_REAL 005af810 f   libSDL2:SDL_render.o
 0001:001aeba0       _SDL_DestroyRenderer_REAL  005afba0 f   libSDL2:SDL_render.o
 0001:001aecd0       _SDL_GL_BindTexture_REAL   005afcd0 f   libSDL2:SDL_render.o
 0001:001aed70       _SDL_GL_UnbindTexture_REAL 005afd70 f   libSDL2:SDL_render.o
 0001:001af1b0       _SDL_CreateShapedWindow_REAL 005b01b0 f   libSDL2:SDL_shape.o
 0001:001af240       _SDL_IsShapedWindow_REAL   005b0240 f   libSDL2:SDL_shape.o
 0001:001af260       _SDL_CalculateShapeBitmap  005b0260 f   libSDL2:SDL_shape.o
 0001:001af490       _SDL_CalculateShapeTree    005b0490 f   libSDL2:SDL_shape.o
 0001:001af510       _SDL_TraverseShapeTree     005b0510 f   libSDL2:SDL_shape.o
 0001:001afc00       _SDL_FreeShapeTree         005b0c00 f   libSDL2:SDL_shape.o
 0001:001b01f0       _SDL_SetWindowShape_REAL   005b11f0 f   libSDL2:SDL_shape.o
 0001:001b02a0       _SDL_GetShapedWindowMode_REAL 005b12a0 f   libSDL2:SDL_shape.o
 0001:001b0850       _SDL_malloc_REAL           005b1850 f   libSDL2:SDL_malloc.o
 0001:001b1dc0       _SDL_free_REAL             005b2dc0 f   libSDL2:SDL_malloc.o
 0001:001b2860       _SDL_calloc_REAL           005b3860 f   libSDL2:SDL_malloc.o
 0001:001b28d0       _SDL_realloc_REAL          005b38d0 f   libSDL2:SDL_malloc.o
 0001:001b2be0       _memalign                  005b3be0 f   libSDL2:SDL_malloc.o
 0001:001b2bf0       _independent_calloc        005b3bf0 f   libSDL2:SDL_malloc.o
 0001:001b2f10       _independent_comalloc      005b3f10 f   libSDL2:SDL_malloc.o
 0001:001b31b0       _valloc                    005b41b0 f   libSDL2:SDL_malloc.o
 0001:001b3290       _pvalloc                   005b4290 f   libSDL2:SDL_malloc.o
 0001:001b3370       _malloc_trim               005b4370 f   libSDL2:SDL_malloc.o
 0001:001b3490       _malloc_footprint          005b4490 f   libSDL2:SDL_malloc.o
 0001:001b34a0       _malloc_max_footprint      005b44a0 f   libSDL2:SDL_malloc.o
 0001:001b34b0       _mallinfo                  005b44b0 f   libSDL2:SDL_malloc.o
 0001:001b36f0       _malloc_stats              005b46f0 f   libSDL2:SDL_malloc.o
 0001:001b3870       _malloc_usable_size        005b4870 f   libSDL2:SDL_malloc.o
 0001:001b38b0       _mallopt                   005b48b0 f   libSDL2:SDL_malloc.o
 0001:001b3a00       _SDL_setenv_REAL           005b4a00 f   libSDL2:SDL_getenv.o
 0001:001b3aa0       _SDL_getenv_REAL           005b4aa0 f   libSDL2:SDL_getenv.o
 0001:001b3d30       _SDL_qsort_REAL            005b4d30 f   libSDL2:SDL_qsort.o
 0001:001b5620       _SDL_atan_REAL             005b6620 f   libSDL2:SDL_stdlib.o
 0001:001b5630       _SDL_atan2_REAL            005b6630 f   libSDL2:SDL_stdlib.o
 0001:001b5640       _SDL_acos_REAL             005b6640 f   libSDL2:SDL_stdlib.o
 0001:001b56a0       _SDL_asin_REAL             005b66a0 f   libSDL2:SDL_stdlib.o
 0001:001b5700       _SDL_ceil_REAL             005b6700 f   libSDL2:SDL_stdlib.o
 0001:001b5730       _SDL_copysign_REAL         005b6730 f   libSDL2:SDL_stdlib.o
 0001:001b5740       _SDL_cos_REAL              005b6740 f   libSDL2:SDL_stdlib.o
 0001:001b5750       _SDL_cosf_REAL             005b6750 f   libSDL2:SDL_stdlib.o
 0001:001b5770       _SDL_fabs_REAL             005b6770 f   libSDL2:SDL_stdlib.o
 0001:001b5780       _SDL_floor_REAL            005b6780 f   libSDL2:SDL_stdlib.o
 0001:001b5790       _SDL_log_REAL              005b6790 f   libSDL2:SDL_stdlib.o
 0001:001b57a0       _SDL_pow_REAL              005b67a0 f   libSDL2:SDL_stdlib.o
 0001:001b57b0       _SDL_scalbn_REAL           005b67b0 f   libSDL2:SDL_stdlib.o
 0001:001b57c0       _SDL_sin_REAL              005b67c0 f   libSDL2:SDL_stdlib.o
 0001:001b57d0       _SDL_sinf_REAL             005b67d0 f   libSDL2:SDL_stdlib.o
 0001:001b57f0       _SDL_sqrt_REAL             005b67f0 f   libSDL2:SDL_stdlib.o
 0001:001b5800       _SDL_sqrtf_REAL            005b6800 f   libSDL2:SDL_stdlib.o
 0001:001b5820       _SDL_tan_REAL              005b6820 f   libSDL2:SDL_stdlib.o
 0001:001b5830       _SDL_tanf_REAL             005b6830 f   libSDL2:SDL_stdlib.o
 0001:001b5850       _SDL_abs_REAL              005b6850 f   libSDL2:SDL_stdlib.o
 0001:001b5860       _SDL_isdigit_REAL          005b6860 f   libSDL2:SDL_stdlib.o
 0001:001b5880       _SDL_isspace_REAL          005b6880 f   libSDL2:SDL_stdlib.o
 0001:001b58a0       _SDL_toupper_REAL          005b68a0 f   libSDL2:SDL_stdlib.o
 0001:001b58c0       _SDL_tolower_REAL          005b68c0 f   libSDL2:SDL_stdlib.o
 0001:001b59c0       _SDL_iconv_open_REAL       005b69c0 f   libSDL2:SDL_iconv.o
 0001:001b5ad0       _SDL_iconv_REAL            005b6ad0 f   libSDL2:SDL_iconv.o
 0001:001b6480       _SDL_iconv_close_REAL      005b7480 f   libSDL2:SDL_iconv.o
 0001:001b64a0       _SDL_iconv_string_REAL     005b74a0 f   libSDL2:SDL_iconv.o
 0001:001b6fc0       _SDL_SetSurfacePalette_REAL 005b7fc0 f   libSDL2:SDL_surface.o
 0001:001b7010       _SDL_SetSurfaceRLE_REAL    005b8010 f   libSDL2:SDL_surface.o
 0001:001b7060       _SDL_SetColorKey_REAL      005b8060 f   libSDL2:SDL_surface.o
 0001:001b71a0       _SDL_GetColorKey_REAL      005b81a0 f   libSDL2:SDL_surface.o
 0001:001b71d0       _SDL_SetSurfaceColorMod_REAL 005b81d0 f   libSDL2:SDL_surface.o
 0001:001b7260       _SDL_GetSurfaceColorMod_REAL 005b8260 f   libSDL2:SDL_surface.o
 0001:001b72c0       _SDL_SetSurfaceAlphaMod_REAL 005b82c0 f   libSDL2:SDL_surface.o
 0001:001b7320       _SDL_GetSurfaceAlphaMod_REAL 005b8320 f   libSDL2:SDL_surface.o
 0001:001b7350       _SDL_SetSurfaceBlendMode_REAL 005b8350 f   libSDL2:SDL_surface.o
 0001:001b73e0       _SDL_GetSurfaceBlendMode_REAL 005b83e0 f   libSDL2:SDL_surface.o
 0001:001b7450       _SDL_SetClipRect_REAL      005b8450 f   libSDL2:SDL_surface.o
 0001:001b74d0       _SDL_GetClipRect_REAL      005b84d0 f   libSDL2:SDL_surface.o
 0001:001b7500       _SDL_LowerBlit_REAL        005b8500 f   libSDL2:SDL_surface.o
 0001:001b7590       _SDL_UpperBlit_REAL        005b8590 f   libSDL2:SDL_surface.o
 0001:001b7890       _SDL_LowerBlitScaled_REAL  005b8890 f   libSDL2:SDL_surface.o
 0001:001b79a0       _SDL_UpperBlitScaled_REAL  005b89a0 f   libSDL2:SDL_surface.o
 0001:001b7f60       _SDL_LockSurface_REAL      005b8f60 f   libSDL2:SDL_surface.o
 0001:001b7fb0       _SDL_UnlockSurface_REAL    005b8fb0 f   libSDL2:SDL_surface.o
 0001:001b7fe0       _SDL_ConvertPixels_REAL    005b8fe0 f   libSDL2:SDL_surface.o
 0001:001b85d0       _SDL_FreeSurface_REAL      005b95d0 f   libSDL2:SDL_surface.o
 0001:001b86b0       _SDL_CreateRGBSurface_REAL 005b96b0 f   libSDL2:SDL_surface.o
 0001:001b88d0       _SDL_ConvertSurface_REAL   005b98d0 f   libSDL2:SDL_surface.o
 0001:001b8f50       _SDL_ConvertSurfaceFormat_REAL 005b9f50 f   libSDL2:SDL_surface.o
 0001:001b8fa0       _SDL_CreateRGBSurfaceFrom_REAL 005b9fa0 f   libSDL2:SDL_surface.o
 0001:001b9200       _SDL_LoadBMP_RW_REAL       005ba200 f   libSDL2:SDL_bmp.o
 0001:001b9b70       _SDL_SaveBMP_RW_REAL       005bab70 f   libSDL2:SDL_bmp.o
 0001:001ba160       _SDL_FillRect_REAL         005bb160 f   libSDL2:SDL_fillrect.o
 0001:001bb0c0       _SDL_FillRects_REAL        005bc0c0 f   libSDL2:SDL_fillrect.o
 0001:001bb140       _SDL_SoftStretch_REAL      005bc140 f   libSDL2:SDL_stretch.o
 0001:001bb6f0       _SDL_SYS_CreateThread      005bc6f0 f   libSDL2:SDL_systhread.o
 0001:001bb7b0       _SDL_SYS_SetupThread       005bc7b0 f   libSDL2:SDL_systhread.o
 0001:001bb7c0       _SDL_ThreadID_REAL         005bc7c0 f   libSDL2:SDL_systhread.o
 0001:001bb7d0       _SDL_SYS_SetThreadPriority 005bc7d0 f   libSDL2:SDL_systhread.o
 0001:001bb820       _SDL_SYS_WaitThread        005bc820 f   libSDL2:SDL_systhread.o
 0001:001bb860       _SDL_SYS_DetachThread      005bc860 f   libSDL2:SDL_systhread.o
 0001:001bb900       _SDL_TicksInit             005bc900 f   libSDL2:SDL_systimer.o
 0001:001bb990       _SDL_TicksQuit             005bc990 f   libSDL2:SDL_systimer.o
 0001:001bba00       _SDL_GetTicks_REAL         005bca00 f   libSDL2:SDL_systimer.o
 0001:001bbb00       _SDL_GetPerformanceCounter_REAL 005bcb00 f   libSDL2:SDL_systimer.o
 0001:001bbb30       _SDL_GetPerformanceFrequency_REAL 005bcb30 f   libSDL2:SDL_systimer.o
 0001:001bbb60       _SDL_Delay_REAL            005bcb60 f   libSDL2:SDL_systimer.o
 0001:001bbd70       _SDL_TimerQuit             005bcd70 f   libSDL2:SDL_timer.o
 0001:001bbe70       _SDL_TimerInit             005bce70 f   libSDL2:SDL_timer.o
 0001:001bbf40       _SDL_AddTimer_REAL         005bcf40 f   libSDL2:SDL_timer.o
 0001:001bc200       _SDL_RemoveTimer_REAL      005bd200 f   libSDL2:SDL_timer.o
 0001:001bc2a0       _SDL_TouchInit             005bd2a0 f   libSDL2:SDL_touch.o
 0001:001bc2b0       _SDL_GetNumTouchDevices_REAL 005bd2b0 f   libSDL2:SDL_touch.o
 0001:001bc2c0       _SDL_GetTouchDevice_REAL   005bd2c0 f   libSDL2:SDL_touch.o
 0001:001bc300       _SDL_GetTouch              005bd300 f   libSDL2:SDL_touch.o
 0001:001bc390       _SDL_GetFinger             005bd390 f   libSDL2:SDL_touch.o
 0001:001bc3f0       _SDL_GetNumTouchFingers_REAL 005bd3f0 f   libSDL2:SDL_touch.o
 0001:001bc490       _SDL_GetTouchFinger_REAL   005bd490 f   libSDL2:SDL_touch.o
 0001:001bc570       _SDL_AddTouch              005bd570 f   libSDL2:SDL_touch.o
 0001:001bc680       _SDL_SendTouch             005bd680 f   libSDL2:SDL_touch.o
 0001:001bca10       _SDL_SendTouchMotion       005bda10 f   libSDL2:SDL_touch.o
 0001:001bcc80       _SDL_DelTouch              005bdc80 f   libSDL2:SDL_touch.o
 0001:001bcdc0       _SDL_TouchQuit             005bddc0 f   libSDL2:SDL_touch.o
 0001:001bce20       _WIN_UnloadXInputDLL       005bde20 f   libSDL2:SDL_xinput.o
 0001:001bce60       _WIN_LoadXInputDLL         005bde60 f   libSDL2:SDL_xinput.o
 0001:001bd0b0       _WIN_SetErrorFromHRESULT   005be0b0 f   libSDL2:SDL_windows.o
 0001:001bd170       _WIN_SetError              005be170 f   libSDL2:SDL_windows.o
 0001:001bd190       _WIN_CoInitialize          005be190 f   libSDL2:SDL_windows.o
 0001:001bd1f0       _WIN_CoUninitialize        005be1f0 f   libSDL2:SDL_windows.o
 0001:001bd200       _WIN_IsWindowsVistaOrGreater 005be200 f   libSDL2:SDL_windows.o
 0001:001bd210       _SDL_XINPUT_Enabled        005be210 f   libSDL2:SDL_xinputjoystick.o
 0001:001bd220       _SDL_XINPUT_JoystickInit   005be220 f   libSDL2:SDL_xinputjoystick.o
 0001:001bd270       _SDL_XINPUT_JoystickDetect 005be270 f   libSDL2:SDL_xinputjoystick.o
 0001:001bd590       _SDL_XINPUT_JoystickOpen   005be590 f   libSDL2:SDL_xinputjoystick.o
 0001:001bd6d0       _SDL_XINPUT_JoystickUpdate 005be6d0 f   libSDL2:SDL_xinputjoystick.o
 0001:001bda40       _SDL_XINPUT_JoystickClose  005bea40 f   libSDL2:SDL_xinputjoystick.o
 0001:001bda50       _SDL_XINPUT_JoystickQuit   005bea50 f   libSDL2:SDL_xinputjoystick.o
 0001:001bda70       _SDL_SYS_IsXInputGamepad_DeviceIndex 005bea70 f   libSDL2:SDL_xinputjoystick.o
 0001:001be620       _SDL_DINPUT_JoystickInit   005bf620 f   libSDL2:SDL_dinputjoystick.o
 0001:001be730       _SDL_DINPUT_JoystickDetect 005bf730 f   libSDL2:SDL_dinputjoystick.o
 0001:001be790       _SDL_DINPUT_JoystickOpen   005bf790 f   libSDL2:SDL_dinputjoystick.o
 0001:001beb90       _SDL_DINPUT_JoystickUpdate 005bfb90 f   libSDL2:SDL_dinputjoystick.o
 0001:001bec10       _SDL_DINPUT_JoystickClose  005bfc10 f   libSDL2:SDL_dinputjoystick.o
 0001:001bec50       _SDL_DINPUT_JoystickQuit   005bfc50 f   libSDL2:SDL_dinputjoystick.o
 0001:001bed40       _SDL_XINPUT_MaybeAddDevice 005bfd40 f   libSDL2:SDL_xinputhaptic.o
 0001:001bee60       _SDL_XINPUT_HapticInit     005bfe60 f   libSDL2:SDL_xinputhaptic.o
 0001:001beee0       _SDL_XINPUT_MaybeRemoveDevice 005bfee0 f   libSDL2:SDL_xinputhaptic.o
 0001:001bef50       _SDL_XINPUT_HapticOpen     005bff50 f   libSDL2:SDL_xinputhaptic.o
 0001:001bf140       _SDL_XINPUT_JoystickSameHaptic 005c0140 f   libSDL2:SDL_xinputhaptic.o
 0001:001bf160       _SDL_XINPUT_HapticOpenFromJoystick 005c0160 f   libSDL2:SDL_xinputhaptic.o
 0001:001bf380       _SDL_XINPUT_HapticClose    005c0380 f   libSDL2:SDL_xinputhaptic.o
 0001:001bf3c0       _SDL_XINPUT_HapticQuit     005c03c0 f   libSDL2:SDL_xinputhaptic.o
 0001:001bf3e0       _SDL_XINPUT_HapticNewEffect 005c03e0 f   libSDL2:SDL_xinputhaptic.o
 0001:001bf450       _SDL_XINPUT_HapticUpdateEffect 005c0450 f   libSDL2:SDL_xinputhaptic.o
 0001:001bf4c0       _SDL_XINPUT_HapticRunEffect 005c04c0 f   libSDL2:SDL_xinputhaptic.o
 0001:001bf580       _SDL_XINPUT_HapticStopEffect 005c0580 f   libSDL2:SDL_xinputhaptic.o
 0001:001bf600       _SDL_XINPUT_HapticDestroyEffect 005c0600 f   libSDL2:SDL_xinputhaptic.o
 0001:001bf670       _SDL_XINPUT_HapticGetEffectStatus 005c0670 f   libSDL2:SDL_xinputhaptic.o
 0001:001bf680       _SDL_XINPUT_HapticSetGain  005c0680 f   libSDL2:SDL_xinputhaptic.o
 0001:001bf690       _SDL_XINPUT_HapticSetAutocenter 005c0690 f   libSDL2:SDL_xinputhaptic.o
 0001:001bf6a0       _SDL_XINPUT_HapticPause    005c06a0 f   libSDL2:SDL_xinputhaptic.o
 0001:001bf6b0       _SDL_XINPUT_HapticUnpause  005c06b0 f   libSDL2:SDL_xinputhaptic.o
 0001:001bf6c0       _SDL_XINPUT_HapticStopAll  005c06c0 f   libSDL2:SDL_xinputhaptic.o
 0001:001bfe20       _SDL_DINPUT_HapticInit     005c0e20 f   libSDL2:SDL_dinputhaptic.o
 0001:001bffa0       _SDL_DINPUT_MaybeAddDevice 005c0fa0 f   libSDL2:SDL_dinputhaptic.o
 0001:001c0160       _SDL_DINPUT_MaybeRemoveDevice 005c1160 f   libSDL2:SDL_dinputhaptic.o
 0001:001c01e0       _SDL_DINPUT_HapticOpen     005c11e0 f   libSDL2:SDL_dinputhaptic.o
 0001:001c02b0       _SDL_DINPUT_JoystickSameHaptic 005c12b0 f   libSDL2:SDL_dinputhaptic.o
 0001:001c0350       _SDL_DINPUT_HapticOpenFromJoystick 005c1350 f   libSDL2:SDL_dinputhaptic.o
 0001:001c0430       _SDL_DINPUT_HapticClose    005c1430 f   libSDL2:SDL_dinputhaptic.o
 0001:001c0470       _SDL_DINPUT_HapticQuit     005c1470 f   libSDL2:SDL_dinputhaptic.o
 0001:001c04c0       _SDL_DINPUT_HapticNewEffect 005c14c0 f   libSDL2:SDL_dinputhaptic.o
 0001:001c10e0       _SDL_DINPUT_HapticUpdateEffect 005c20e0 f   libSDL2:SDL_dinputhaptic.o
 0001:001c1c50       _SDL_DINPUT_HapticRunEffect 005c2c50 f   libSDL2:SDL_dinputhaptic.o
 0001:001c1ca0       _SDL_DINPUT_HapticStopEffect 005c2ca0 f   libSDL2:SDL_dinputhaptic.o
 0001:001c1ce0       _SDL_DINPUT_HapticDestroyEffect 005c2ce0 f   libSDL2:SDL_dinputhaptic.o
 0001:001c1da0       _SDL_DINPUT_HapticGetEffectStatus 005c2da0 f   libSDL2:SDL_dinputhaptic.o
 0001:001c1df0       _SDL_DINPUT_HapticSetGain  005c2df0 f   libSDL2:SDL_dinputhaptic.o
 0001:001c1e60       _SDL_DINPUT_HapticSetAutocenter 005c2e60 f   libSDL2:SDL_dinputhaptic.o
 0001:001c1ee0       _SDL_DINPUT_HapticPause    005c2ee0 f   libSDL2:SDL_dinputhaptic.o
 0001:001c1f30       _SDL_DINPUT_HapticUnpause  005c2f30 f   libSDL2:SDL_dinputhaptic.o
 0001:001c1f80       _SDL_DINPUT_HapticStopAll  005c2f80 f   libSDL2:SDL_dinputhaptic.o
 0001:001c1fd0       _SDL_SYS_GetTLSData        005c2fd0 f   libSDL2:SDL_systls.o
 0001:001c2060       _SDL_SYS_SetTLSData        005c3060 f   libSDL2:SDL_systls.o
 0001:001c2750       _WIN_InitMouse             005c3750 f   libSDL2:SDL_windowsmouse.o
 0001:001c2800       _WIN_QuitMouse             005c3800 f   libSDL2:SDL_windowsmouse.o
 0001:001c2c70       _WIN_CreateWindowFrom      005c3c70 f   libSDL2:SDL_windowswindow.o
 0001:001c2d90       _WIN_SetWindowTitle        005c3d90 f   libSDL2:SDL_windowswindow.o
 0001:001c2e00       _WIN_SetWindowIcon         005c3e00 f   libSDL2:SDL_windowswindow.o
 0001:001c2fd0       _WIN_SetWindowPosition     005c3fd0 f   libSDL2:SDL_windowswindow.o
 0001:001c30e0       _WIN_SetWindowSize         005c40e0 f   libSDL2:SDL_windowswindow.o
 0001:001c31f0       _WIN_ShowWindow            005c41f0 f   libSDL2:SDL_windowswindow.o
 0001:001c3220       _WIN_HideWindow            005c4220 f   libSDL2:SDL_windowswindow.o
 0001:001c3250       _WIN_RaiseWindow           005c4250 f   libSDL2:SDL_windowswindow.o
 0001:001c3360       _WIN_MaximizeWindow        005c4360 f   libSDL2:SDL_windowswindow.o
 0001:001c33a0       _WIN_MinimizeWindow        005c43a0 f   libSDL2:SDL_windowswindow.o
 0001:001c33d0       _WIN_SetWindowBordered     005c43d0 f   libSDL2:SDL_windowswindow.o
 0001:001c3550       _WIN_RestoreWindow         005c4550 f   libSDL2:SDL_windowswindow.o
 0001:001c3590       _WIN_SetWindowFullscreen   005c4590 f   libSDL2:SDL_windowswindow.o
 0001:001c37a0       _WIN_SetWindowGammaRamp    005c47a0 f   libSDL2:SDL_windowswindow.o
 0001:001c3830       _WIN_GetWindowGammaRamp    005c4830 f   libSDL2:SDL_windowswindow.o
 0001:001c38c0       _WIN_SetWindowGrab         005c48c0 f   libSDL2:SDL_windowswindow.o
 0001:001c3b20       _WIN_DestroyWindow         005c4b20 f   libSDL2:SDL_windowswindow.o
 0001:001c3bc0       _WIN_CreateWindow          005c4bc0 f   libSDL2:SDL_windowswindow.o
 0001:001c3e20       _WIN_GetWindowWMInfo       005c4e20 f   libSDL2:SDL_windowswindow.o
 0001:001c3e80       _SDL_HelperWindowCreate    005c4e80 f   libSDL2:SDL_windowswindow.o
 0001:001c3fc0       _SDL_HelperWindowDestroy   005c4fc0 f   libSDL2:SDL_windowswindow.o
 0001:001c4060       _WIN_OnWindowEnter         005c5060 f   libSDL2:SDL_windowswindow.o
 0001:001c40b0       _WIN_UpdateClipCursor      005c50b0 f   libSDL2:SDL_windowswindow.o
 0001:001c41e0       _WIN_SetWindowHitTest      005c51e0 f   libSDL2:SDL_windowswindow.o
 0001:001c41f0       _TSFSink_AddRef@4          005c51f0 f   libSDL2:SDL_windowskeyboard.o
 0001:001c42e0       _TSFSink_Release@4         005c52e0 f   libSDL2:SDL_windowskeyboard.o
 0001:001c4830       _UIElementSink_QueryInterface@12 005c5830 f   libSDL2:SDL_windowskeyboard.o
 0001:001c48b0       _IPPASink_QueryInterface@12 005c58b0 f   libSDL2:SDL_windowskeyboard.o
 0001:001c4d60       _IPPASink_OnActivated@32   005c5d60 f   libSDL2:SDL_windowskeyboard.o
 0001:001c4fa0       _UIElementSink_BeginUIElement@12 005c5fa0 f   libSDL2:SDL_windowskeyboard.o
 0001:001c50f0       _UIElementSink_UpdateUIElement@8 005c60f0 f   libSDL2:SDL_windowskeyboard.o
 0001:001c5250       _UIElementSink_EndUIElement@8 005c6250 f   libSDL2:SDL_windowskeyboard.o
 0001:001c5f00       _WIN_UpdateKeymap          005c6f00 f   libSDL2:SDL_windowskeyboard.o
 0001:001c5fd0       _WIN_InitKeyboard          005c6fd0 f   libSDL2:SDL_windowskeyboard.o
 0001:001c6220       _WIN_QuitKeyboard          005c7220 f   libSDL2:SDL_windowskeyboard.o
 0001:001c63d0       _WIN_StartTextInput        005c73d0 f   libSDL2:SDL_windowskeyboard.o
 0001:001c6580       _WIN_StopTextInput         005c7580 f   libSDL2:SDL_windowskeyboard.o
 0001:001c6740       _WIN_SetTextInputRect      005c7740 f   libSDL2:SDL_windowskeyboard.o
 0001:001c6800       _IME_HandleMessage         005c7800 f   libSDL2:SDL_windowskeyboard.o
 0001:001c70b0       _UILess_GetUIElement       005c80b0 f   libSDL2:SDL_windowskeyboard.o
 0001:001c7120       _IME_Present               005c8120 f   libSDL2:SDL_windowskeyboard.o
 0001:001c7bf0       _SDL_SendWindowEvent       005c8bf0 f   libSDL2:SDL_windowevents.o
 0001:001c7ed0       _SDL_SendDropFile          005c8ed0 f   libSDL2:SDL_dropevents.o
 0001:001c7f30       _CombineRectRegions        005c8f30 f   libSDL2:SDL_windowsshape.o
 0001:001c7fc0       _Win32_CreateShaper        005c8fc0 f   libSDL2:SDL_windowsshape.o
 0001:001c8050       _Win32_SetWindowShape      005c9050 f   libSDL2:SDL_windowsshape.o
 0001:001c8130       _Win32_ResizeWindowShape   005c9130 f   libSDL2:SDL_windowsshape.o
 0001:001c81a0       _WIN_SetClipboardText      005c91a0 f   libSDL2:SDL_windowsclipboard.o
 0001:001c8370       _WIN_GetClipboardText      005c9370 f   libSDL2:SDL_windowsclipboard.o
 0001:001c8460       _WIN_HasClipboardText      005c9460 f   libSDL2:SDL_windowsclipboard.o
 0001:001c8570       _WIN_CheckClipboardUpdate  005c9570 f   libSDL2:SDL_windowsclipboard.o
 0001:001c9230       _WIN_InitModes             005ca230 f   libSDL2:SDL_windowsmodes.o
 0001:001c9400       _WIN_GetDisplayBounds      005ca400 f   libSDL2:SDL_windowsmodes.o
 0001:001c94f0       _WIN_GetDisplayDPI         005ca4f0 f   libSDL2:SDL_windowsmodes.o
 0001:001c9550       _WIN_GetDisplayModes       005ca550 f   libSDL2:SDL_windowsmodes.o
 0001:001c95e0       _WIN_SetDisplayMode        005ca5e0 f   libSDL2:SDL_windowsmodes.o
 0001:001c96a0       _WIN_QuitModes             005ca6a0 f   libSDL2:SDL_windowsmodes.o
 0001:001c96b0       _WIN_CreateWindowFramebuffer 005ca6b0 f   libSDL2:SDL_windowsframebuffer.o
 0001:001c9980       _WIN_UpdateWindowFramebuffer 005ca980 f   libSDL2:SDL_windowsframebuffer.o
 0001:001c99e0       _WIN_DestroyWindowFramebuffer 005ca9e0 f   libSDL2:SDL_windowsframebuffer.o
 0001:001ca3b0       _WIN_GL_LoadLibrary        005cb3b0 f   libSDL2:SDL_windowsopengl.o
 0001:001ca510       _WIN_GL_GetProcAddress     005cb510 f   libSDL2:SDL_windowsopengl.o
 0001:001ca560       _WIN_GL_UnloadLibrary      005cb560 f   libSDL2:SDL_windowsopengl.o
 0001:001ca5a0       _WIN_GL_InitExtensions     005cb5a0 f   libSDL2:SDL_windowsopengl.o
 0001:001cada0       _WIN_GL_SetupWindow        005cbda0 f   libSDL2:SDL_windowsopengl.o
 0001:001cae40       _WIN_GL_CreateContext      005cbe40 f   libSDL2:SDL_windowsopengl.o
 0001:001cb230       _WIN_GL_MakeCurrent        005cc230 f   libSDL2:SDL_windowsopengl.o
 0001:001cb2b0       _WIN_GL_SetSwapInterval    005cc2b0 f   libSDL2:SDL_windowsopengl.o
 0001:001cb320       _WIN_GL_GetSwapInterval    005cc320 f   libSDL2:SDL_windowsopengl.o
 0001:001cb340       _WIN_GL_SwapWindow         005cc340 f   libSDL2:SDL_windowsopengl.o
 0001:001cb360       _WIN_GL_DeleteContext      005cc360 f   libSDL2:SDL_windowsopengl.o
 0001:001cb390       _WIN_GL_SetPixelFormatFrom 005cc390 f   libSDL2:SDL_windowsopengl.o
 0001:001cb420       _MatrixIdentity            005cc420 f   libSDL2:SDL_d3dmath.o
 0001:001cb4c0       _MatrixMultiply            005cc4c0 f   libSDL2:SDL_d3dmath.o
 0001:001cb760       _MatrixScaling             005cc760 f   libSDL2:SDL_d3dmath.o
 0001:001cb820       _MatrixTranslation         005cc820 f   libSDL2:SDL_d3dmath.o
 0001:001cb8e0       _MatrixRotationX           005cc8e0 f   libSDL2:SDL_d3dmath.o
 0001:001cb9c0       _MatrixRotationY           005cc9c0 f   libSDL2:SDL_d3dmath.o
 0001:001cbaa0       _MatrixRotationZ           005ccaa0 f   libSDL2:SDL_d3dmath.o
 0001:001cbb80       _SDL_QuitInit              005ccb80 f   libSDL2:SDL_quit.o
 0001:001cbbc0       _SDL_QuitQuit              005ccbc0 f   libSDL2:SDL_quit.o
 0001:001cbbd0       _SDL_SendQuit              005ccbd0 f   libSDL2:SDL_quit.o
 0001:001cbbf0       _SDL_SendPendingQuit       005ccbf0 f   libSDL2:SDL_quit.o
 0001:001cc580       _GetXmaPacketFrameCount    005cd580 f   libSDL2:SDL_xaudio2.o
 0001:001cc590       _GetXmaPacketFirstFrameOffsetInBits 005cd590 f   libSDL2:SDL_xaudio2.o
 0001:001cc5c0       _GetXmaPacketMetadata      005cd5c0 f   libSDL2:SDL_xaudio2.o
 0001:001cc5d0       _GetXmaPacketSkipCount     005cd5d0 f   libSDL2:SDL_xaudio2.o
 0001:001cc5e0       _GetXmaBlockContainingSample 005cd5e0 f   libSDL2:SDL_xaudio2.o
 0001:001cc640       _GetXmaFrameLengthInBits   005cd640 f   libSDL2:SDL_xaudio2.o
 0001:001cc6b0       _GetXmaFrameBitPosition    005cd6b0 f   libSDL2:SDL_xaudio2.o
 0001:001cc7d0       _GetLastXmaFrameBitPosition 005cd7d0 f   libSDL2:SDL_xaudio2.o
 0001:001cc8d0       _GetXmaDecodePositionForSample 005cd8d0 f   libSDL2:SDL_xaudio2.o
 0001:001cca20       _GetXmaSampleRate          005cda20 f   libSDL2:SDL_xaudio2.o
 0001:001cca60       _GetStandardChannelMaskFromXmaMask 005cda60 f   libSDL2:SDL_xaudio2.o
 0001:001ccac0       _GetXmaChannelMaskFromStandardMask 005cdac0 f   libSDL2:SDL_xaudio2.o
 0001:001ccb20       _LocalizeXma2Format        005cdb20 f   libSDL2:SDL_xaudio2.o
 0001:001ccbc0       _XAudio2Create             005cdbc0 f   libSDL2:SDL_xaudio2.o
 0001:001ece00       _SDL_SYS_HapticInit        005ede00 f   libSDL2:SDL_windowshaptic.o
 0001:001ece20       _SDL_SYS_AddHapticDevice   005ede20 f   libSDL2:SDL_windowshaptic.o
 0001:001ece50       _SDL_SYS_RemoveHapticDevice 005ede50 f   libSDL2:SDL_windowshaptic.o
 0001:001eceb0       _SDL_SYS_NumHaptics        005edeb0 f   libSDL2:SDL_windowshaptic.o
 0001:001ecec0       _SDL_SYS_HapticName        005edec0 f   libSDL2:SDL_windowshaptic.o
 0001:001ecef0       _SDL_SYS_HapticOpen        005edef0 f   libSDL2:SDL_windowshaptic.o
 0001:001ecf50       _SDL_SYS_HapticMouse       005edf50 f   libSDL2:SDL_windowshaptic.o
 0001:001ecf90       _SDL_SYS_JoystickIsHaptic  005edf90 f   libSDL2:SDL_windowshaptic.o
 0001:001ecfc0       _SDL_SYS_JoystickSameHaptic 005edfc0 f   libSDL2:SDL_windowshaptic.o
 0001:001ed000       _SDL_SYS_HapticOpenFromJoystick 005ee000 f   libSDL2:SDL_windowshaptic.o
 0001:001ed030       _SDL_SYS_HapticClose       005ee030 f   libSDL2:SDL_windowshaptic.o
 0001:001ed090       _SDL_SYS_HapticQuit        005ee090 f   libSDL2:SDL_windowshaptic.o
 0001:001ed130       _SDL_SYS_HapticNewEffect   005ee130 f   libSDL2:SDL_windowshaptic.o
 0001:001ed1d0       _SDL_SYS_HapticUpdateEffect 005ee1d0 f   libSDL2:SDL_windowshaptic.o
 0001:001ed200       _SDL_SYS_HapticRunEffect   005ee200 f   libSDL2:SDL_windowshaptic.o
 0001:001ed230       _SDL_SYS_HapticStopEffect  005ee230 f   libSDL2:SDL_windowshaptic.o
 0001:001ed260       _SDL_SYS_HapticDestroyEffect 005ee260 f   libSDL2:SDL_windowshaptic.o
 0001:001ed2a0       _SDL_SYS_HapticGetEffectStatus 005ee2a0 f   libSDL2:SDL_windowshaptic.o
 0001:001ed2d0       _SDL_SYS_HapticSetGain     005ee2d0 f   libSDL2:SDL_windowshaptic.o
 0001:001ed300       _SDL_SYS_HapticSetAutocenter 005ee300 f   libSDL2:SDL_windowshaptic.o
 0001:001ed330       _SDL_SYS_HapticPause       005ee330 f   libSDL2:SDL_windowshaptic.o
 0001:001ed350       _SDL_SYS_HapticUnpause     005ee350 f   libSDL2:SDL_windowshaptic.o
 0001:001ed370       _SDL_SYS_HapticStopAll     005ee370 f   libSDL2:SDL_windowshaptic.o
 0001:001ed9c0       _WIN_ShowMessageBox        005ee9c0 f   libSDL2:SDL_windowsmessagebox.o
 0001:001ee370       _SDL_CalculateBlit         005ef370 f   libSDL2:SDL_blit.o
 0001:001eecf0       _SDL_RLEBlit               005efcf0 f   libSDL2:SDL_RLEaccel.o
 0001:001f1460       _SDL_RLEAlphaBlit          005f2460 f   libSDL2:SDL_RLEaccel.o
 0001:001f1ed0       _SDL_UnRLESurface          005f2ed0 f   libSDL2:SDL_RLEaccel.o
 0001:001f2150       _SDL_RLESurface            005f3150 f   libSDL2:SDL_RLEaccel.o
 0001:001f2e00       _SDL_GetPowerInfo_Windows  005f3e00 f   libSDL2:SDL_syspower.o
 0001:001fd930       _GLES2_GetFBO              005fe930 f   libSDL2:SDL_render_gles2.o
 0001:001ff600       _SW_CreateRendererForSurface 00600600 f   libSDL2:SDL_render_sw.o
 0001:00200ec0       _SDL_SW_CreateYUVTexture   00601ec0 f   libSDL2:SDL_yuv_sw.o
 0001:00201110       _SDL_SW_QueryYUVTexturePixels 00602110 f   libSDL2:SDL_yuv_sw.o
 0001:00201130       _SDL_SW_UpdateYUVTexture   00602130 f   libSDL2:SDL_yuv_sw.o
 0001:00201490       _SDL_SW_UpdateYUVTexturePlanar 00602490 f   libSDL2:SDL_yuv_sw.o
 0001:002016e0       _SDL_SW_LockYUVTexture     006026e0 f   libSDL2:SDL_yuv_sw.o
 0001:00201780       _SDL_SW_UnlockYUVTexture   00602780 f   libSDL2:SDL_yuv_sw.o
 0001:00201790       _SDL_SW_CopyYUVToRGB       00602790 f   libSDL2:SDL_yuv_sw.o
 0001:00202120       _SDL_SW_DestroyYUVTexture  00603120 f   libSDL2:SDL_yuv_sw.o
 0001:00202180       _SDL_uclibc_atan           00603180 f   libSDL2:s_atan.o
 0001:00202350       _SDL_uclibc_atan2          00603350 f   libSDL2:e_atan2.o
 0001:00202600       _SDL_uclibc_sqrt           00603600 f   libSDL2:e_sqrt.o
 0001:00202840       _SDL_uclibc_floor          00603840 f   libSDL2:s_floor.o
 0001:002029b0       _SDL_uclibc_copysign       006039b0 f   libSDL2:s_copysign.o
 0001:002029e0       _SDL_uclibc_cos            006039e0 f   libSDL2:s_cos.o
 0001:00202ab0       _SDL_uclibc_fabs           00603ab0 f   libSDL2:s_fabs.o
 0001:00202ad0       _SDL_uclibc_log            00603ad0 f   libSDL2:e_log.o
 0001:00202d20       _SDL_uclibc_pow            00603d20 f   libSDL2:e_pow.o
 0001:002034f0       _SDL_uclibc_scalbn         006044f0 f   libSDL2:s_scalbn.o
 0001:00203620       _SDL_uclibc_sin            00604620 f   libSDL2:s_sin.o
 0001:00203700       _SDL_uclibc_tan            00604700 f   libSDL2:s_tan.o
 0001:00203780       _WIN_GLES_LoadLibrary      00604780 f   libSDL2:SDL_windowsopengles.o
 0001:00203840       _WIN_GLES_CreateContext    00604840 f   libSDL2:SDL_windowsopengles.o
 0001:00203910       _WIN_GLES_DeleteContext    00604910 f   libSDL2:SDL_windowsopengles.o
 0001:00203940       _WIN_GLES_SwapWindow       00604940 f   libSDL2:SDL_windowsopengles.o
 0001:00203960       _WIN_GLES_MakeCurrent      00604960 f   libSDL2:SDL_windowsopengles.o
 0001:002039b0       _WIN_GLES_SetupWindow      006049b0 f   libSDL2:SDL_windowsopengles.o
 0001:00203a90       _WIN_GLES_SetSwapInterval  00604a90 f   libSDL2:SDL_windowsopengles.o
 0001:00203ab0       _SDL_SendClipboardUpdate   00604ab0 f   libSDL2:SDL_clipboardevents.o
 0001:00203b00       _SDL_EGL_GetProcAddress    00604b00 f   libSDL2:SDL_egl.o
 0001:00203ba0       _SDL_EGL_UnloadLibrary     00604ba0 f   libSDL2:SDL_egl.o
 0001:00203c20       _SDL_EGL_LoadLibrary       00604c20 f   libSDL2:SDL_egl.o
 0001:00204240       _SDL_EGL_ChooseConfig      00605240 f   libSDL2:SDL_egl.o
 0001:00204600       _SDL_EGL_CreateContext     00605600 f   libSDL2:SDL_egl.o
 0001:00204850       _SDL_EGL_MakeCurrent       00605850 f   libSDL2:SDL_egl.o
 0001:002048e0       _SDL_EGL_SetSwapInterval   006058e0 f   libSDL2:SDL_egl.o
 0001:00204950       _SDL_EGL_GetSwapInterval   00605950 f   libSDL2:SDL_egl.o
 0001:00204970       _SDL_EGL_SwapBuffers       00605970 f   libSDL2:SDL_egl.o
 0001:002049a0       _SDL_EGL_DeleteContext     006059a0 f   libSDL2:SDL_egl.o
 0001:00204a00       _SDL_EGL_CreateSurface     00605a00 f   libSDL2:SDL_egl.o
 0001:00204a50       _SDL_EGL_DestroySurface    00605a50 f   libSDL2:SDL_egl.o
 0001:00204a80       _DUMMY_PumpEvents          00605a80 f   libSDL2:SDL_nullevents.o
 0001:00204a90       _SDL_DUMMY_CreateWindowFramebuffer 00605a90 f   libSDL2:SDL_nullframebuffer.o
 0001:00204b90       _SDL_DUMMY_UpdateWindowFramebuffer 00605b90 f   libSDL2:SDL_nullframebuffer.o
 0001:00204c50       _SDL_DUMMY_DestroyWindowFramebuffer 00605c50 f   libSDL2:SDL_nullframebuffer.o
 0001:00216ee0       _SDL_BlitCopy              00617ee0 f   libSDL2:SDL_blit_copy.o
 0001:00221500       _SDL_CalculateBlitN        00622500 f   libSDL2:SDL_blit_N.o
 0001:00229600       _SDL_CalculateBlitA        0062a600 f   libSDL2:SDL_blit_A.o
 0001:0022cc70       _SDL_CalculateBlit1        0062dc70 f   libSDL2:SDL_blit_1.o
 0001:0022dc20       _SDL_CalculateBlit0        0062ec20 f   libSDL2:SDL_blit_0.o
 0001:0022dca0       _SDL_Blit_Slow             0062eca0 f   libSDL2:SDL_blit_slow.o
 0001:0022e840       _GL_CreateShaderContext    0062f840 f   libSDL2:SDL_shaders_gl.o
 0001:0022ec00       _GL_SelectShader           0062fc00 f   libSDL2:SDL_shaders_gl.o
 0001:0022ec20       _GL_DestroyShaderContext   0062fc20 f   libSDL2:SDL_shaders_gl.o
 0001:0022ec70       _GLES2_GetShader           0062fc70 f   libSDL2:SDL_shaders_gles2.o
 0001:00234400       _SDL_BlendFillRect         00635400 f   libSDL2:SDL_blendfillrect.o
 0001:002346b0       _SDL_BlendFillRects        006356b0 f   libSDL2:SDL_blendfillrect.o
 0001:0023f380       _SDL_BlendLine             00640380 f   libSDL2:SDL_blendline.o
 0001:0023f4f0       _SDL_BlendLines            006404f0 f   libSDL2:SDL_blendline.o
 0001:00240990       _SDL_DrawLine              00641990 f   libSDL2:SDL_drawline.o
 0001:00240a90       _SDL_DrawLines             00641a90 f   libSDL2:SDL_drawline.o
 0001:00242060       _SDL_BlendPoint            00643060 f   libSDL2:SDL_blendpoint.o
 0001:002422f0       _SDL_BlendPoints           006432f0 f   libSDL2:SDL_blendpoint.o
 0001:00242560       _SDL_DrawPoint             00643560 f   libSDL2:SDL_drawpoint.o
 0001:00242630       _SDL_DrawPoints            00643630 f   libSDL2:SDL_drawpoint.o
 0001:00242760       _SDLgfx_rotozoomSurfaceSizeTrig 00643760 f   libSDL2:SDL_rotate.o
 0001:00242fa0       _SDLgfx_rotateSurface      00643fa0 f   libSDL2:SDL_rotate.o
 0001:00243de0       _ColorRGBDitherYV12MMX1X   00644de0 f   libSDL2:SDL_yuv_mmx.o
 0001:00243f90       _Color565DitherYV12MMX1X   00644f90 f   libSDL2:SDL_yuv_mmx.o
 0001:00244210       ___ieee754_rem_pio2        00645210 f   libSDL2:e_rem_pio2.o
 0001:00244560       ___kernel_sin              00645560 f   libSDL2:k_sin.o
 0001:00244620       ___kernel_cos              00645620 f   libSDL2:k_cos.o
 0001:00244760       ___kernel_tan              00645760 f   libSDL2:k_tan.o
 0001:00244960       ___kernel_rem_pio2         00645960 f   libSDL2:k_rem_pio2.o
 0001:00245370       ___WSAFDIsSet@8            00646370 f   ws2_32:WS2_32.dll
 0001:00245376       _ImmGetIMEFileNameA@12     00646376 f   imm32:IMM32.dll
 0001:0024537c       _ImmGetContext@4           0064637c f   imm32:IMM32.dll
 0001:00245382       _ImmReleaseContext@8       00646382 f   imm32:IMM32.dll
 0001:00245388       _ImmNotifyIME@16           00646388 f   imm32:IMM32.dll
 0001:0024538e       _ImmAssociateContext@8     0064638e f   imm32:IMM32.dll
 0001:00245394       _ImmSetCompositionStringW@24 00646394 f   imm32:IMM32.dll
 0001:0024539a       _ImmSetCompositionWindow@8 0064639a f   imm32:IMM32.dll
 0001:002453a0       _ImmGetCompositionStringW@16 006463a0 f   imm32:IMM32.dll
 0001:002453a6       _ImmGetCandidateListW@16   006463a6 f   imm32:IMM32.dll
 0001:002453ac       _GetFileVersionInfoSizeA@8 006463ac f   version:VERSION.dll
 0001:002453b2       _GetFileVersionInfoA@16    006463b2 f   version:VERSION.dll
 0001:002453b8       _VerQueryValueA@16         006463b8 f   version:VERSION.dll
 0001:00247510       _ov_raw_seek               00648510 f   libvorbisfile:vorbisfile.o
 0001:002485d0       _ov_pcm_seek_page          006495d0 f   libvorbisfile:vorbisfile.o
 0001:00249610       _ov_pcm_seek               0064a610 f   libvorbisfile:vorbisfile.o
 0001:00249b30       _ov_clear                  0064ab30 f   libvorbisfile:vorbisfile.o
 0001:00249c60       _ov_open_callbacks         0064ac60 f   libvorbisfile:vorbisfile.o
 0001:00249f10       _ov_open                   0064af10 f   libvorbisfile:vorbisfile.o
 0001:0024a1a0       _ov_fopen                  0064b1a0 f   libvorbisfile:vorbisfile.o
 0001:0024a400       _ov_halfrate               0064b400 f   libvorbisfile:vorbisfile.o
 0001:0024a560       _ov_halfrate_p             0064b560 f   libvorbisfile:vorbisfile.o
 0001:0024a580       _ov_test_callbacks         0064b580 f   libvorbisfile:vorbisfile.o
 0001:0024a7d0       _ov_test                   0064b7d0 f   libvorbisfile:vorbisfile.o
 0001:0024aa00       _ov_test_open              0064ba00 f   libvorbisfile:vorbisfile.o
 0001:0024aa60       _ov_streams                0064ba60 f   libvorbisfile:vorbisfile.o
 0001:0024aa70       _ov_seekable               0064ba70 f   libvorbisfile:vorbisfile.o
 0001:0024aa80       _ov_bitrate_instant        0064ba80 f   libvorbisfile:vorbisfile.o
 0001:0024ab10       _ov_serialnumber           0064bb10 f   libvorbisfile:vorbisfile.o
 0001:0024ab60       _ov_raw_total              0064bb60 f   libvorbisfile:vorbisfile.o
 0001:0024acb0       _ov_pcm_total              0064bcb0 f   libvorbisfile:vorbisfile.o
 0001:0024acf0       _ov_time_total             0064bcf0 f   libvorbisfile:vorbisfile.o
 0001:0024ada0       _ov_time_seek_page         0064bda0 f   libvorbisfile:vorbisfile.o
 0001:0024af40       _ov_time_seek              0064bf40 f   libvorbisfile:vorbisfile.o
 0001:0024b0e0       _ov_bitrate                0064c0e0 f   libvorbisfile:vorbisfile.o
 0001:0024b2a0       _ov_raw_tell               0064c2a0 f   libvorbisfile:vorbisfile.o
 0001:0024b2c0       _ov_pcm_tell               0064c2c0 f   libvorbisfile:vorbisfile.o
 0001:0024b2e0       _ov_time_tell              0064c2e0 f   libvorbisfile:vorbisfile.o
 0001:0024b4b0       _ov_info                   0064c4b0 f   libvorbisfile:vorbisfile.o
 0001:0024b4f0       _ov_comment                0064c4f0 f   libvorbisfile:vorbisfile.o
 0001:0024b530       _ov_read_filter            0064c530 f   libvorbisfile:vorbisfile.o
 0001:0024b5b0       _ov_read                   0064c5b0 f   libvorbisfile:vorbisfile.o
 0001:0024b610       _ov_read_float             0064c610 f   libvorbisfile:vorbisfile.o
 0001:0024b6e0       _ov_crosslap               0064c6e0 f   libvorbisfile:vorbisfile.o
 0001:0024ba00       _ov_raw_seek_lap           0064ca00 f   libvorbisfile:vorbisfile.o
 0001:0024ba20       _ov_pcm_seek_lap           0064ca20 f   libvorbisfile:vorbisfile.o
 0001:0024ba40       _ov_pcm_seek_page_lap      0064ca40 f   libvorbisfile:vorbisfile.o
 0001:0024ba60       _ov_time_seek_lap          0064ca60 f   libvorbisfile:vorbisfile.o
 0001:0024ba80       _ov_time_seek_page_lap     0064ca80 f   libvorbisfile:vorbisfile.o
 0001:0024baa0       _vpx_codec_dec_init_ver    0064caa0 f   libvpx:vpx_decoder.c.o
 0001:0024bc10       _vpx_codec_peek_stream_info 0064cc10 f   libvpx:vpx_decoder.c.o
 0001:0024bc70       _vpx_codec_get_stream_info 0064cc70 f   libvpx:vpx_decoder.c.o
 0001:0024bce0       _vpx_codec_decode          0064cce0 f   libvpx:vpx_decoder.c.o
 0001:0024bd60       _vpx_codec_get_frame       0064cd60 f   libvpx:vpx_decoder.c.o
 0001:0024bda0       _vpx_codec_register_put_frame_cb 0064cda0 f   libvpx:vpx_decoder.c.o
 0001:0024be00       _vpx_codec_register_put_slice_cb 0064ce00 f   libvpx:vpx_decoder.c.o
 0001:0024be60       _vpx_codec_get_mem_map     0064ce60 f   libvpx:vpx_decoder.c.o
 0001:0024bec0       _vpx_codec_set_mem_map     0064cec0 f   libvpx:vpx_decoder.c.o
 0001:0024cfc0       _vpx_codec_vp8_dx          0064dfc0 f   libvpx:vp8_dx_iface.c.o
 0001:0024cfd0       _vpx_mmap_dtor             0064dfd0 f   libvpx:vpx_codec.c.o
 0001:0024cfe0       _vpx_codec_version         0064dfe0 f   libvpx:vpx_codec.c.o
 0001:0024cff0       _vpx_codec_version_str     0064dff0 f   libvpx:vpx_codec.c.o
 0001:0024d000       _vpx_codec_version_extra_str 0064e000 f   libvpx:vpx_codec.c.o
 0001:0024d010       _vpx_codec_iface_name      0064e010 f   libvpx:vpx_codec.c.o
 0001:0024d030       _vpx_codec_err_to_string   0064e030 f   libvpx:vpx_codec.c.o
 0001:0024d050       _vpx_codec_error           0064e050 f   libvpx:vpx_codec.c.o
 0001:0024d080       _vpx_codec_error_detail    0064e080 f   libvpx:vpx_codec.c.o
 0001:0024d0b0       _vpx_codec_destroy         0064e0b0 f   libvpx:vpx_codec.c.o
 0001:0024d110       _vpx_codec_get_caps        0064e110 f   libvpx:vpx_codec.c.o
 0001:0024d130       _vpx_codec_control_        0064e130 f   libvpx:vpx_codec.c.o
 0001:0024d1b0       _vpx_mmap_alloc            0064e1b0 f   libvpx:vpx_codec.c.o
 0001:0024d220       _vpx_validate_mmaps        0064e220 f   libvpx:vpx_codec.c.o
 0001:0024d440       _vp8dx_get_reference       0064e440 f   libvpx:onyxd_if.c.o
 0001:0024d520       _vp8dx_set_reference       0064e520 f   libvpx:onyxd_if.c.o
 0001:0024d6c0       _check_fragments_for_errors 0064e6c0 f   libvpx:onyxd_if.c.o
 0001:0024d7f0       _vp8dx_receive_compressed_data 0064e7f0 f   libvpx:onyxd_if.c.o
 0001:0024dd60       _vp8dx_get_raw_frame       0064ed60 f   libvpx:onyxd_if.c.o
 0001:0024ddf0       _vp8dx_references_buffer   0064edf0 f   libvpx:onyxd_if.c.o
 0001:0024de50       _vp8_create_decoder_instances 0064ee50 f   libvpx:onyxd_if.c.o
 0001:0024de80       _vp8_remove_decoder_instances 0064ee80 f   libvpx:onyxd_if.c.o
 0001:0024ded0       _vp8_rtcd                  0064eed0 f   libvpx:rtcd.c.o
 0001:0024e870       _vp8_de_alloc_frame_buffers 0064f870 f   libvpx:alloccommon.c.o
 0001:0024e940       _vp8_alloc_frame_buffers   0064f940 f   libvpx:alloccommon.c.o
 0001:0024ed30       _vp8_setup_version         0064fd30 f   libvpx:alloccommon.c.o
 0001:0024ee10       _vp8_create_common         0064fe10 f   libvpx:alloccommon.c.o
 0001:0024eec0       _vp8_remove_common         0064fec0 f   libvpx:alloccommon.c.o
 0001:0024ef90       _vp8_setup_block_dptrs     0064ff90 f   libvpx:mbpitch.c.o
 0001:0024f0e0       _vp8_build_block_doffsets  006500e0 f   libvpx:mbpitch.c.o
 0001:0024f1e0       _vpx_mem_get_version       006501e0 f   libvpx:vpx_mem.c.o
 0001:0024f1f0       _vpx_mem_set_heap_size     006501f0 f   libvpx:vpx_mem.c.o
 0001:0024f200       _vpx_memalign              00650200 f   libvpx:vpx_mem.c.o
 0001:0024f240       _vpx_malloc                00650240 f   libvpx:vpx_mem.c.o
 0001:0024f270       _vpx_calloc                00650270 f   libvpx:vpx_mem.c.o
 0001:0024f2c0       _vpx_realloc               006502c0 f   libvpx:vpx_mem.c.o
 0001:0024f330       _vpx_free                  00650330 f   libvpx:vpx_mem.c.o
 0001:0024f350       _vpx_memcpy                00650350 f   libvpx:vpx_mem.c.o
 0001:0024f360       _vpx_memset                00650360 f   libvpx:vpx_mem.c.o
 0001:0024f370       _vpx_memmove               00650370 f   libvpx:vpx_mem.c.o
 0001:0024f380       _vpx_mem_set_functions     00650380 f   libvpx:vpx_mem.c.o
 0001:0024f390       _vpx_mem_unset_functions   00650390 f   libvpx:vpx_mem.c.o
 0001:0024f800       _vp8cx_init_de_quantizer   00650800 f   libvpx:decodeframe.c.o
 0001:0024f8c0       _vp8_mb_init_dequantizer   006508c0 f   libvpx:decodeframe.c.o
 0001:0024fb20       _vp8_decode_frame          00650b20 f   libvpx:decodeframe.c.o
 0001:00253890       _vp8_loop_filter_update_sharpness 00654890 f   libvpx:loopfilter.c.o
 0001:00253a00       _vp8_loop_filter_init      00654a00 f   libvpx:loopfilter.c.o
 0001:00253c50       _vp8_loop_filter_frame_init 00654c50 f   libvpx:loopfilter.c.o
 0001:00253fe0       _vp8_loop_filter_row_normal 00654fe0 f   libvpx:loopfilter.c.o
 0001:002541e0       _vp8_loop_filter_row_simple 006551e0 f   libvpx:loopfilter.c.o
 0001:00254340       _vp8_loop_filter_frame     00655340 f   libvpx:loopfilter.c.o
 0001:00254820       _vp8_loop_filter_frame_yonly 00655820 f   libvpx:loopfilter.c.o
 0001:00254bc0       _vp8_loop_filter_partial_frame 00655bc0 f   libvpx:loopfilter.c.o
 0001:002550e0       _vp8_yv12_extend_frame_borders_c 006560e0 f   libvpx:yv12extend.c.o
 0001:002552f0       _vp9_extend_frame_borders_c 006562f0 f   libvpx:yv12extend.c.o
 0001:002554b0       _vp9_extend_frame_inner_borders_c 006564b0 f   libvpx:yv12extend.c.o
 0001:00255670       _vp8_yv12_copy_frame_c     00656670 f   libvpx:yv12extend.c.o
 0001:00255740       _vpx_yv12_copy_y_c         00656740 f   libvpx:yv12extend.c.o
 0001:002559a0       _vp8_post_proc_down_and_across_mb_row_c 006569a0 f   libvpx:postproc.c.o
 0001:00255cb0       _vp8_mbpost_proc_across_ip_c 00656cb0 f   libvpx:postproc.c.o
 0001:00255fd0       _vp8_mbpost_proc_down_c    00656fd0 f   libvpx:postproc.c.o
 0001:002564e0       _vp8_deblock               006574e0 f   libvpx:postproc.c.o
 0001:00256720       _vp8_gaussian              00657720 f   libvpx:postproc.c.o
 0001:00256770       _vp8_plane_add_noise_c     00657770 f   libvpx:postproc.c.o
 0001:00256830       _vp8_blend_mb_inner_c      00657830 f   libvpx:postproc.c.o
 0001:00256a30       _vp8_blend_mb_outer_c      00657a30 f   libvpx:postproc.c.o
 0001:002570a0       _vp8_blend_b_c             006580a0 f   libvpx:postproc.c.o
 0001:00257270       _vp8_post_proc_frame       00658270 f   libvpx:postproc.c.o
 0001:00257870       _vpx_scale_rtcd            00658870 f   libvpx:vpx_scale_rtcd.c.o
 0001:00257920       _vpx_reset_mmx_state       00658920     libvpx:emms.asm.o
 0001:00257930       _vp8_dequantize_b_mmx      00658930 f   libvpx:idct_blk_mmx.c.o
 0001:00257960       _vp8_dequant_idct_add_y_block_mmx 00658960 f   libvpx:idct_blk_mmx.c.o
 0001:00257b30       _vp8_dequant_idct_add_uv_block_mmx 00658b30 f   libvpx:idct_blk_mmx.c.o
 0001:00257d40       _vp8_dequantize_b_impl_mmx 00658d40     libvpx:dequantize_mmx.asm.o
 0001:00257d7f       _vp8_dequant_idct_add_mmx  00658d7f     libvpx:dequantize_mmx.asm.o
 0001:00257f20       _vp8_dequant_idct_add_y_block_sse2 00658f20 f   libvpx:idct_blk_sse2.c.o
 0001:00257fe0       _vp8_dequant_idct_add_uv_block_sse2 00658fe0 f   libvpx:idct_blk_sse2.c.o
 0001:00258130       _vp8_dequant_idct_add_y_block_c 00659130 f   libvpx:idct_blk.c.o
 0001:002581e0       _vp8_dequant_idct_add_uv_block_c 006591e0 f   libvpx:idct_blk.c.o
 0001:002595f0       _vp8_loop_filter_horizontal_edge_c 0065a5f0 f   libvpx:loopfilter_filters.c.o
 0001:00259940       _vp8_loop_filter_vertical_edge_c 0065a940 f   libvpx:loopfilter_filters.c.o
 0001:00259bf0       _vp8_mbloop_filter_horizontal_edge_c 0065abf0 f   libvpx:loopfilter_filters.c.o
 0001:0025a010       _vp8_mbloop_filter_vertical_edge_c 0065b010 f   libvpx:loopfilter_filters.c.o
 0001:0025a360       _vp8_loop_filter_simple_horizontal_edge_c 0065b360 f   libvpx:loopfilter_filters.c.o
 0001:0025a4b0       _vp8_loop_filter_simple_vertical_edge_c 0065b4b0 f   libvpx:loopfilter_filters.c.o
 0001:0025a610       _vp8_loop_filter_mbh_c     0065b610 f   libvpx:loopfilter_filters.c.o
 0001:0025aa90       _vp8_loop_filter_mbv_c     0065ba90 f   libvpx:loopfilter_filters.c.o
 0001:0025ae60       _vp8_loop_filter_bh_c      0065be60 f   libvpx:loopfilter_filters.c.o
 0001:0025af40       _vp8_loop_filter_bhs_c     0065bf40 f   libvpx:loopfilter_filters.c.o
 0001:0025afa0       _vp8_loop_filter_bv_c      0065bfa0 f   libvpx:loopfilter_filters.c.o
 0001:0025b070       _vp8_loop_filter_bvs_c     0065c070 f   libvpx:loopfilter_filters.c.o
 0001:0025b0d0       _vp8_loop_filter_mbh_mmx   0065c0d0 f   libvpx:loopfilter_x86.c.o
 0001:0025b180       _vp8_loop_filter_mbv_mmx   0065c180 f   libvpx:loopfilter_x86.c.o
 0001:0025b230       _vp8_loop_filter_bh_mmx    0065c230 f   libvpx:loopfilter_x86.c.o
 0001:0025b370       _vp8_loop_filter_bhs_mmx   0065c370 f   libvpx:loopfilter_x86.c.o
 0001:0025b3d0       _vp8_loop_filter_bv_mmx    0065c3d0 f   libvpx:loopfilter_x86.c.o
 0001:0025b500       _vp8_loop_filter_bvs_mmx   0065c500 f   libvpx:loopfilter_x86.c.o
 0001:0025b560       _vp8_loop_filter_mbh_sse2  0065c560 f   libvpx:loopfilter_x86.c.o
 0001:0025b5e0       _vp8_loop_filter_mbv_sse2  0065c5e0 f   libvpx:loopfilter_x86.c.o
 0001:0025b660       _vp8_loop_filter_bh_sse2   0065c660 f   libvpx:loopfilter_x86.c.o
 0001:0025b750       _vp8_loop_filter_bhs_sse2  0065c750 f   libvpx:loopfilter_x86.c.o
 0001:0025b7b0       _vp8_loop_filter_bv_sse2   0065c7b0 f   libvpx:loopfilter_x86.c.o
 0001:0025b890       _vp8_loop_filter_bvs_sse2  0065c890 f   libvpx:loopfilter_x86.c.o
 0001:0025b900       _vp8_loop_filter_horizontal_edge_mmx 0065c900     libvpx:loopfilter_mmx.asm.o
 0001:0025bb11       _vp8_loop_filter_vertical_edge_mmx 0065cb11     libvpx:loopfilter_mmx.asm.o
 0001:0025be01       _vp8_mbloop_filter_horizontal_edge_mmx 0065ce01     libvpx:loopfilter_mmx.asm.o
 0001:0025c0d8       _vp8_mbloop_filter_vertical_edge_mmx 0065d0d8     libvpx:loopfilter_mmx.asm.o
 0001:0025c4ec       _vp8_loop_filter_simple_horizontal_edge_mmx 0065d4ec     libvpx:loopfilter_mmx.asm.o
 0001:0025c5f2       _vp8_loop_filter_simple_vertical_edge_mmx 0065d5f2     libvpx:loopfilter_mmx.asm.o
 0001:0025c7b0       _vp8_loop_filter_horizontal_edge_sse2 0065d7b0     libvpx:loopfilter_sse2.asm.o
 0001:0025c9f8       _vp8_loop_filter_horizontal_edge_uv_sse2 0065d9f8     libvpx:loopfilter_sse2.asm.o
 0001:0025cc9a       _vp8_mbloop_filter_horizontal_edge_sse2 0065dc9a     libvpx:loopfilter_sse2.asm.o
 0001:0025cf86       _vp8_mbloop_filter_horizontal_edge_uv_sse2 0065df86     libvpx:loopfilter_sse2.asm.o
 0001:0025d2da       _vp8_loop_filter_vertical_edge_sse2 0065e2da     libvpx:loopfilter_sse2.asm.o
 0001:0025d6e7       _vp8_loop_filter_vertical_edge_uv_sse2 0065e6e7     libvpx:loopfilter_sse2.asm.o
 0001:0025dafa       _vp8_mbloop_filter_vertical_edge_sse2 0065eafa     libvpx:loopfilter_sse2.asm.o
 0001:0025e012       _vp8_mbloop_filter_vertical_edge_uv_sse2 0065f012     libvpx:loopfilter_sse2.asm.o
 0001:0025e530       _vp8_loop_filter_simple_horizontal_edge_sse2 0065f530     libvpx:loopfilter_sse2.asm.o
 0001:0025e645       _vp8_loop_filter_simple_vertical_edge_sse2 0065f645     libvpx:loopfilter_sse2.asm.o
 0001:0025e900       _vp8_short_idct4x4llm_c    0065f900 f   libvpx:idctllm.c.o
 0001:0025ef30       _vp8_dc_only_idct_add_c    0065ff30 f   libvpx:idctllm.c.o
 0001:0025f1e0       _vp8_short_inv_walsh4x4_c  006601e0 f   libvpx:idctllm.c.o
 0001:0025f4c0       _vp8_short_inv_walsh4x4_1_c 006604c0 f   libvpx:idctllm.c.o
 0001:0025f540       _vp8_short_idct4x4llm_mmx  00660540     libvpx:idctllm_mmx.asm.o
 0001:0025f6c3       _vp8_dc_only_idct_add_mmx  006606c3     libvpx:idctllm_mmx.asm.o
 0001:0025f740       _vp8_short_inv_walsh4x4_mmx 00660740     libvpx:iwalsh_mmx.asm.o
 0001:0025f890       _vp8_short_inv_walsh4x4_sse2 00660890     libvpx:iwalsh_sse2.asm.o
 0001:0025f9f0       _vp8_copy_mem8x8_mmx       006609f0     libvpx:recon_mmx.asm.o
 0001:0025fa51       _vp8_copy_mem8x4_mmx       00660a51     libvpx:recon_mmx.asm.o
 0001:0025fa8a       _vp8_copy_mem16x16_mmx     00660a8a     libvpx:recon_mmx.asm.o
 0001:0025fbe0       _vp8_copy_mem16x16_sse2    00660be0     libvpx:recon_sse2.asm.o
 0001:0025fcb9       _vp8_intra_pred_uv_dc_mmx2 00660cb9     libvpx:recon_sse2.asm.o
 0001:0025fd45       _vp8_intra_pred_uv_dctop_mmx2 00660d45     libvpx:recon_sse2.asm.o
 0001:0025fd96       _vp8_intra_pred_uv_dcleft_mmx2 00660d96     libvpx:recon_sse2.asm.o
 0001:0025fe10       _vp8_intra_pred_uv_dc128_mmx 00660e10     libvpx:recon_sse2.asm.o
 0001:0025fe46       _vp8_intra_pred_uv_tm_sse2 00660e46     libvpx:recon_sse2.asm.o
 0001:0025fec5       _vp8_intra_pred_uv_tm_ssse3 00660ec5     libvpx:recon_sse2.asm.o
 0001:0025ff34       _vp8_intra_pred_uv_ve_mmx  00660f34     libvpx:recon_sse2.asm.o
 0001:0025ff69       _vp8_intra_pred_uv_ho_mmx2 00660f69     libvpx:recon_sse2.asm.o
 0001:0025ffa8       _vp8_intra_pred_uv_ho_ssse3 00660fa8     libvpx:recon_sse2.asm.o
 0001:0026003f       _vp8_intra_pred_y_dc_sse2  0066103f     libvpx:recon_sse2.asm.o
 0001:00260129       _vp8_intra_pred_y_dctop_sse2 00661129     libvpx:recon_sse2.asm.o
 0001:002601a2       _vp8_intra_pred_y_dcleft_sse2 006611a2     libvpx:recon_sse2.asm.o
 0001:0026026a       _vp8_intra_pred_y_dc128_sse2 0066126a     libvpx:recon_sse2.asm.o
 0001:002602b6       _vp8_intra_pred_y_tm_sse2  006612b6     libvpx:recon_sse2.asm.o
 0001:00260356       _vp8_intra_pred_y_tm_ssse3 00661356     libvpx:recon_sse2.asm.o
 0001:002603e6       _vp8_intra_pred_y_ve_sse2  006613e6     libvpx:recon_sse2.asm.o
 0001:00260431       _vp8_intra_pred_y_ho_sse2  00661431     libvpx:recon_sse2.asm.o
 0001:00260480       _vp8_copy_mem16x16_c       00661480 f   libvpx:reconinter.c.o
 0001:002604c0       _vp8_copy_mem8x8_c         006614c0 f   libvpx:reconinter.c.o
 0001:00260550       _vp8_copy_mem8x4_c         00661550 f   libvpx:reconinter.c.o
 0001:002605a0       _vp8_build_inter_predictors_b 006615a0 f   libvpx:reconinter.c.o
 0001:002606a0       _vp8_build_inter16x16_predictors_mbuv 006616a0 f   libvpx:reconinter.c.o
 0001:002607f0       _vp8_build_inter4x4_predictors_mbuv 006617f0 f   libvpx:reconinter.c.o
 0001:00260f90       _vp8_build_inter16x16_predictors_mby 00661f90 f   libvpx:reconinter.c.o
 0001:00261030       _vp8_build_inter16x16_predictors_mb 00662030 f   libvpx:reconinter.c.o
 0001:002612d0       _vp8_build_inter_predictors_mb 006622d0 f   libvpx:reconinter.c.o
 0001:00262350       _vp8_build_intra_predictors_mbuv_s_sse2 00663350 f   libvpx:recon_wrapper_sse2.c.o
 0001:00262450       _vp8_build_intra_predictors_mbuv_s_ssse3 00663450 f   libvpx:recon_wrapper_sse2.c.o
 0001:00262550       _vp8_build_intra_predictors_mby_s_sse2 00663550 f   libvpx:recon_wrapper_sse2.c.o
 0001:00262600       _vp8_build_intra_predictors_mby_s_ssse3 00663600 f   libvpx:recon_wrapper_sse2.c.o
 0001:002626b0       _vp8_build_intra_predictors_mby_s_c 006636b0 f   libvpx:reconintra.c.o
 0001:00262b00       _vp8_build_intra_predictors_mbuv_s_c 00663b00 f   libvpx:reconintra.c.o
 0001:00262ee0       _vp8_mbpost_proc_down_mmx  00663ee0     libvpx:postproc_mmx.asm.o
 0001:00263074       _vp8_plane_add_noise_mmx   00664074     libvpx:postproc_mmx.asm.o
 0001:002630d0       _vp8_post_proc_down_and_across_mb_row_sse2 006640d0     libvpx:postproc_sse2.asm.o
 0001:0026335f       _vp8_mbpost_proc_down_xmm  0066435f     libvpx:postproc_sse2.asm.o
 0001:00263545       _vp8_mbpost_proc_across_ip_xmm 00664545     libvpx:postproc_sse2.asm.o
 0001:002636e5       _vp8_plane_add_noise_wmt   006646e5     libvpx:postproc_sse2.asm.o
 0001:00263740       _vp8_filter_by_weight16x16_sse2 00664740     libvpx:mfqe_sse2.asm.o
 0001:002637d9       _vp8_filter_by_weight8x8_sse2 006647d9     libvpx:mfqe_sse2.asm.o
 0001:00263849       _vp8_variance_and_sad_16x16_sse2 00664849     libvpx:mfqe_sse2.asm.o
 0001:00263930       _vp8_sixtap_predict4x4_mmx 00664930 f   libvpx:vp8_asm_stubs.c.o
 0001:002639f0       _vp8_sixtap_predict16x16_mmx 006649f0 f   libvpx:vp8_asm_stubs.c.o
 0001:00263c50       _vp8_sixtap_predict8x8_mmx 00664c50 f   libvpx:vp8_asm_stubs.c.o
 0001:00263da0       _vp8_sixtap_predict8x4_mmx 00664da0 f   libvpx:vp8_asm_stubs.c.o
 0001:00263ef0       _vp8_bilinear_predict16x16_mmx 00664ef0 f   libvpx:vp8_asm_stubs.c.o
 0001:00263fe0       _vp8_sixtap_predict16x16_sse2 00664fe0 f   libvpx:vp8_asm_stubs.c.o
 0001:00264120       _vp8_sixtap_predict8x8_sse2 00665120 f   libvpx:vp8_asm_stubs.c.o
 0001:00264280       _vp8_sixtap_predict8x4_sse2 00665280 f   libvpx:vp8_asm_stubs.c.o
 0001:002643e0       _vp8_sixtap_predict16x16_ssse3 006653e0 f   libvpx:vp8_asm_stubs.c.o
 0001:00264540       _vp8_sixtap_predict8x8_ssse3 00665540 f   libvpx:vp8_asm_stubs.c.o
 0001:002646a0       _vp8_sixtap_predict8x4_ssse3 006656a0 f   libvpx:vp8_asm_stubs.c.o
 0001:00264800       _vp8_sixtap_predict4x4_ssse3 00665800 f   libvpx:vp8_asm_stubs.c.o
 0001:00264b00       _vp8_sixtap_predict4x4_c   00665b00 f   libvpx:filter.c.o
 0001:00264fe0       _vp8_sixtap_predict8x8_c   00665fe0 f   libvpx:filter.c.o
 0001:00265430       _vp8_sixtap_predict8x4_c   00666430 f   libvpx:filter.c.o
 0001:00265880       _vp8_sixtap_predict16x16_c 00666880 f   libvpx:filter.c.o
 0001:00265be0       _vp8_bilinear_predict4x4_c 00666be0 f   libvpx:filter.c.o
 0001:00265c30       _vp8_bilinear_predict8x8_c 00666c30 f   libvpx:filter.c.o
 0001:00265c80       _vp8_bilinear_predict8x4_c 00666c80 f   libvpx:filter.c.o
 0001:00265cd0       _vp8_bilinear_predict16x16_c 00666cd0 f   libvpx:filter.c.o
 0001:00265d20       _vp8_filter_block1d8_h6_sse2 00666d20     libvpx:subpixel_sse2.asm.o
 0001:00265dec       _vp8_filter_block1d16_h6_sse2 00666dec     libvpx:subpixel_sse2.asm.o
 0001:00265f56       _vp8_filter_block1d8_v6_sse2 00666f56     libvpx:subpixel_sse2.asm.o
 0001:00265fe5       _vp8_filter_block1d16_v6_sse2 00666fe5     libvpx:subpixel_sse2.asm.o
 0001:002660d5       _vp8_filter_block1d8_h6_only_sse2 006670d5     libvpx:subpixel_sse2.asm.o
 0001:0026619d       _vp8_filter_block1d16_h6_only_sse2 0066719d     libvpx:subpixel_sse2.asm.o
 0001:002662ff       _vp8_filter_block1d8_v6_only_sse2 006672ff     libvpx:subpixel_sse2.asm.o
 0001:002663a2       _vp8_unpack_block1d16_h6_sse2 006673a2     libvpx:subpixel_sse2.asm.o
 0001:002663de       _vp8_bilinear_predict16x16_sse2 006673de     libvpx:subpixel_sse2.asm.o
 0001:00266649       _vp8_bilinear_predict8x8_sse2 00667649     libvpx:subpixel_sse2.asm.o
 0001:002667a0       _vp8_filter_block1d8_h6_ssse3 006677a0     libvpx:subpixel_ssse3.asm.o
 0001:002668b9       _vp8_filter_block1d16_h6_ssse3 006678b9     libvpx:subpixel_ssse3.asm.o
 0001:002669aa       _vp8_filter_block1d4_h6_ssse3 006679aa     libvpx:subpixel_ssse3.asm.o
 0001:00266abf       _vp8_filter_block1d16_v6_ssse3 00667abf     libvpx:subpixel_ssse3.asm.o
 0001:00266c7b       _vp8_filter_block1d8_v6_ssse3 00667c7b     libvpx:subpixel_ssse3.asm.o
 0001:00266d8b       _vp8_filter_block1d4_v6_ssse3 00667d8b     libvpx:subpixel_ssse3.asm.o
 0001:00266e71       _vp8_bilinear_predict16x16_ssse3 00667e71     libvpx:subpixel_ssse3.asm.o
 0001:00267108       _vp8_bilinear_predict8x8_ssse3 00668108     libvpx:subpixel_ssse3.asm.o
 0001:00267480       _vp8_filter_block1d_h6_mmx 00668480     libvpx:subpixel_mmx.asm.o
 0001:0026751b       _vp8_filter_block1dc_v6_mmx 0066851b     libvpx:subpixel_mmx.asm.o
 0001:002675a4       _vp8_bilinear_predict8x8_mmx 006685a4     libvpx:subpixel_mmx.asm.o
 0001:002676b5       _vp8_bilinear_predict8x4_mmx 006686b5     libvpx:subpixel_mmx.asm.o
 0001:002677c6       _vp8_bilinear_predict4x4_mmx 006687c6     libvpx:subpixel_mmx.asm.o
 0001:00267880       _vp8_variance4x4_mmx       00668880 f   libvpx:variance_mmx.c.o
 0001:002678e0       _vp8_variance8x8_mmx       006688e0 f   libvpx:variance_mmx.c.o
 0001:00267940       _vp8_mse16x16_mmx          00668940 f   libvpx:variance_mmx.c.o
 0001:00267a40       _vp8_variance16x16_mmx     00668a40 f   libvpx:variance_mmx.c.o
 0001:00267b50       _vp8_variance16x8_mmx      00668b50 f   libvpx:variance_mmx.c.o
 0001:00267be0       _vp8_variance8x16_mmx      00668be0 f   libvpx:variance_mmx.c.o
 0001:00267c70       _vp8_sub_pixel_variance4x4_mmx 00668c70 f   libvpx:variance_mmx.c.o
 0001:00267cf0       _vp8_sub_pixel_variance8x8_mmx 00668cf0 f   libvpx:variance_mmx.c.o
 0001:00267d70       _vp8_sub_pixel_variance16x16_mmx 00668d70 f   libvpx:variance_mmx.c.o
 0001:00267e40       _vp8_sub_pixel_mse16x16_mmx 00668e40 f   libvpx:variance_mmx.c.o
 0001:00267f00       _vp8_sub_pixel_variance16x8_mmx 00668f00 f   libvpx:variance_mmx.c.o
 0001:00267fd0       _vp8_sub_pixel_variance8x16_mmx 00668fd0 f   libvpx:variance_mmx.c.o
 0001:00268050       _vp8_variance_halfpixvar16x16_h_mmx 00669050 f   libvpx:variance_mmx.c.o
 0001:00268110       _vp8_variance_halfpixvar16x16_v_mmx 00669110 f   libvpx:variance_mmx.c.o
 0001:002681d0       _vp8_variance_halfpixvar16x16_hv_mmx 006691d0 f   libvpx:variance_mmx.c.o
 0001:00268290       _vp8_variance4x4_wmt       00669290 f   libvpx:variance_sse2.c.o
 0001:002682f0       _vp8_variance8x8_wmt       006692f0 f   libvpx:variance_sse2.c.o
 0001:00268350       _vp8_variance16x16_wmt     00669350 f   libvpx:variance_sse2.c.o
 0001:002683b0       _vp8_mse16x16_wmt          006693b0 f   libvpx:variance_sse2.c.o
 0001:00268400       _vp8_variance16x8_wmt      00669400 f   libvpx:variance_sse2.c.o
 0001:00268490       _vp8_variance8x16_wmt      00669490 f   libvpx:variance_sse2.c.o
 0001:00268520       _vp8_sub_pixel_variance4x4_wmt 00669520 f   libvpx:variance_sse2.c.o
 0001:002685a0       _vp8_sub_pixel_variance8x8_wmt 006695a0 f   libvpx:variance_sse2.c.o
 0001:00268710       _vp8_sub_pixel_variance16x16_wmt 00669710 f   libvpx:variance_sse2.c.o
 0001:00268900       _vp8_sub_pixel_mse16x16_wmt 00669900 f   libvpx:variance_sse2.c.o
 0001:00268ad0       _vp8_sub_pixel_variance16x8_wmt 00669ad0 f   libvpx:variance_sse2.c.o
 0001:00268cc0       _vp8_sub_pixel_variance8x16_wmt 00669cc0 f   libvpx:variance_sse2.c.o
 0001:00268e30       _vp8_variance_halfpixvar16x16_h_wmt 00669e30 f   libvpx:variance_sse2.c.o
 0001:00268e90       _vp8_variance_halfpixvar16x16_v_wmt 00669e90 f   libvpx:variance_sse2.c.o
 0001:00268ef0       _vp8_variance_halfpixvar16x16_hv_wmt 00669ef0 f   libvpx:variance_sse2.c.o
 0001:00268f50       _vp8_get_mb_ss_c           00669f50 f   libvpx:variance_c.c.o
 0001:00268f80       _vp8_variance16x16_c       00669f80 f   libvpx:variance_c.c.o
 0001:00269190       _vp8_variance8x16_c        0066a190 f   libvpx:variance_c.c.o
 0001:002692c0       _vp8_variance16x8_c        0066a2c0 f   libvpx:variance_c.c.o
 0001:002694d0       _vp8_variance8x8_c         0066a4d0 f   libvpx:variance_c.c.o
 0001:00269600       _vp8_variance4x4_c         0066a600 f   libvpx:variance_c.c.o
 0001:002697d0       _vp8_mse16x16_c            0066a7d0 f   libvpx:variance_c.c.o
 0001:002699a0       _vp8_sub_pixel_variance4x4_c 0066a9a0 f   libvpx:variance_c.c.o
 0001:00269e30       _vp8_sub_pixel_variance8x8_c 0066ae30 f   libvpx:variance_c.c.o
 0001:0026a210       _vp8_sub_pixel_variance16x16_c 0066b210 f   libvpx:variance_c.c.o
 0001:0026a660       _vp8_variance_halfpixvar16x16_h_c 0066b660 f   libvpx:variance_c.c.o
 0001:0026a6b0       _vp8_variance_halfpixvar16x16_v_c 0066b6b0 f   libvpx:variance_c.c.o
 0001:0026a700       _vp8_variance_halfpixvar16x16_hv_c 0066b700 f   libvpx:variance_c.c.o
 0001:0026a750       _vp8_sub_pixel_mse16x16_c  0066b750 f   libvpx:variance_c.c.o
 0001:0026a7a0       _vp8_sub_pixel_variance16x8_c 0066b7a0 f   libvpx:variance_c.c.o
 0001:0026abf0       _vp8_sub_pixel_variance8x16_c 0066bbf0 f   libvpx:variance_c.c.o
 0001:0026afd0       _vp8_sub_pixel_variance16x16_ssse3 0066bfd0 f   libvpx:variance_ssse3.c.o
 0001:0026b140       _vp8_sub_pixel_variance16x8_ssse3 0066c140 f   libvpx:variance_ssse3.c.o
 0001:0026b2b0       _vp8_sad16x16_c            0066c2b0 f   libvpx:sad_c.c.o
 0001:0026b430       _vp8_sad8x8_c              0066c430 f   libvpx:sad_c.c.o
 0001:0026b510       _vp8_sad16x8_c             0066c510 f   libvpx:sad_c.c.o
 0001:0026b690       _vp8_sad8x16_c             0066c690 f   libvpx:sad_c.c.o
 0001:0026b770       _vp8_sad4x4_c              0066c770 f   libvpx:sad_c.c.o
 0001:0026b900       _vp8_sad16x16x3_c          0066c900 f   libvpx:sad_c.c.o
 0001:0026bd80       _vp8_sad16x16x8_c          0066cd80 f   libvpx:sad_c.c.o
 0001:0026c980       _vp8_sad16x8x3_c           0066d980 f   libvpx:sad_c.c.o
 0001:0026ce00       _vp8_sad16x8x8_c           0066de00 f   libvpx:sad_c.c.o
 0001:0026da00       _vp8_sad8x8x3_c            0066ea00 f   libvpx:sad_c.c.o
 0001:0026dc80       _vp8_sad8x8x8_c            0066ec80 f   libvpx:sad_c.c.o
 0001:0026e320       _vp8_sad8x16x3_c           0066f320 f   libvpx:sad_c.c.o
 0001:0026e5a0       _vp8_sad8x16x8_c           0066f5a0 f   libvpx:sad_c.c.o
 0001:0026ec40       _vp8_sad4x4x3_c            0066fc40 f   libvpx:sad_c.c.o
 0001:0026f100       _vp8_sad4x4x8_c            00670100 f   libvpx:sad_c.c.o
 0001:0026fd80       _vp8_sad16x16x4d_c         00670d80 f   libvpx:sad_c.c.o
 0001:00270380       _vp8_sad16x8x4d_c          00671380 f   libvpx:sad_c.c.o
 0001:00270980       _vp8_sad8x8x4d_c           00671980 f   libvpx:sad_c.c.o
 0001:00270ce0       _vp8_sad8x16x4d_c          00671ce0 f   libvpx:sad_c.c.o
 0001:00271040       _vp8_sad4x4x4d_c           00672040 f   libvpx:sad_c.c.o
 0001:00271660       _vp8_copy32xn_c            00672660 f   libvpx:sad_c.c.o
 0001:002716c0       _vp8_sad16x16_mmx          006726c0     libvpx:sad_mmx.asm.o
 0001:00271749       _vp8_sad8x16_mmx           00672749     libvpx:sad_mmx.asm.o
 0001:002717af       _vp8_sad8x8_mmx            006727af     libvpx:sad_mmx.asm.o
 0001:00271812       _vp8_sad4x4_mmx            00672812     libvpx:sad_mmx.asm.o
 0001:002718a6       _vp8_sad16x8_mmx           006728a6     libvpx:sad_mmx.asm.o
 0001:00271930       _vp8_sad16x16_wmt          00672930     libvpx:sad_sse2.asm.o
 0001:002719b2       _vp8_sad8x16_wmt           006729b2     libvpx:sad_sse2.asm.o
 0001:00271a01       _vp8_sad8x8_wmt            00672a01     libvpx:sad_sse2.asm.o
 0001:00271a3e       _vp8_sad4x4_wmt            00672a3e     libvpx:sad_sse2.asm.o
 0001:00271a8d       _vp8_sad16x8_wmt           00672a8d     libvpx:sad_sse2.asm.o
 0001:00271af7       _vp8_copy32xn_sse2         00672af7     libvpx:sad_sse2.asm.o
 0001:00271ba0       _vp8_sad16x16x3_sse3       00672ba0     libvpx:sad_sse3.asm.o
 0001:00271ecd       _vp8_sad16x8x3_sse3        00672ecd     libvpx:sad_sse3.asm.o
 0001:00272082       _vp8_sad8x16x3_sse3        00673082     libvpx:sad_sse3.asm.o
 0001:002722e7       _vp8_sad8x8x3_sse3         006732e7     libvpx:sad_sse3.asm.o
 0001:00272424       _vp8_sad4x4x3_sse3         00673424     libvpx:sad_sse3.asm.o
 0001:002724c1       _vp8_sad16x16_sse3         006734c1     libvpx:sad_sse3.asm.o
 0001:00272547       _vp8_copy32xn_sse3         00673547     libvpx:sad_sse3.asm.o
 0001:002725e8       _vp8_sad16x16x4d_sse3      006735e8     libvpx:sad_sse3.asm.o
 0001:00272a18       _vp8_sad16x8x4d_sse3       00673a18     libvpx:sad_sse3.asm.o
 0001:00272c58       _vp8_sad8x16x4d_sse3       00673c58     libvpx:sad_sse3.asm.o
 0001:00272f82       _vp8_sad8x8x4d_sse3        00673f82     libvpx:sad_sse3.asm.o
 0001:00273124       _vp8_sad4x4x4d_sse3        00674124     libvpx:sad_sse3.asm.o
 0001:00273200       _vp8_sad16x16x3_ssse3      00674200     libvpx:sad_ssse3.asm.o
 0001:0027749c       _vp8_sad16x8x3_ssse3       0067849c     libvpx:sad_ssse3.asm.o
 0001:00279620       _vp8_sad16x16x8_sse4       0067a620     libvpx:sad_sse4.asm.o
 0001:00279b78       _vp8_sad16x8x8_sse4        0067ab78     libvpx:sad_sse4.asm.o
 0001:00279e30       _vp8_sad8x8x8_sse4         0067ae30     libvpx:sad_sse4.asm.o
 0001:00279fb4       _vp8_sad8x16x8_sse4        0067afb4     libvpx:sad_sse4.asm.o
 0001:0027a2a4       _vp8_sad4x4x8_sse4         0067b2a4     libvpx:sad_sse4.asm.o
 0001:0027a340       _vp8_clear_system_state_c  0067b340 f   libvpx:systemdependent.c.o
 0001:0027a350       _vp8_machine_specific_config 0067b350 f   libvpx:systemdependent.c.o
 0001:0027a470       _vp8_dequantize_b_c        0067b470 f   libvpx:dequantize.c.o
 0001:0027a550       _vp8_dequant_idct_add_c    0067b550 f   libvpx:dequantize.c.o
 0001:0027a870       _vp8_filter_by_weight16x16_c 0067b870 f   libvpx:mfqe.c.o
 0001:0027a8d0       _vp8_filter_by_weight8x8_c 0067b8d0 f   libvpx:mfqe.c.o
 0001:0027a9e0       _vp8_filter_by_weight4x4_c 0067b9e0 f   libvpx:mfqe.c.o
 0001:0027abd0       _vp8_multiframe_quality_enhance 0067bbd0 f   libvpx:mfqe.c.o
 0001:0027baf0       _vp8_yv12_de_alloc_frame_buffer 0067caf0 f   libvpx:yv12config.c.o
 0001:0027bb80       _vp8_yv12_realloc_frame_buffer 0067cb80 f   libvpx:yv12config.c.o
 0001:0027bd00       _vp8_yv12_alloc_frame_buffer 0067cd00 f   libvpx:yv12config.c.o
 0001:0027bef0       _vp9_free_frame_buffer     0067cef0 f   libvpx:yv12config.c.o
 0001:0027bf80       _vp9_realloc_frame_buffer  0067cf80 f   libvpx:yv12config.c.o
 0001:0027c150       _vp9_alloc_frame_buffer    0067d150 f   libvpx:yv12config.c.o
 0001:0027c3a0       _vp8_mv_cont               0067d3a0 f   libvpx:entropymode.c.o
 0001:0027c3d0       _vp8_init_mbmode_probs     0067d3d0 f   libvpx:entropymode.c.o
 0001:0027c420       _vp8_default_bmode_probs   0067d420 f   libvpx:entropymode.c.o
 0001:0027c440       _vp8_default_coef_probs    0067d440 f   libvpx:entropy.c.o
 0001:0027c4d0       _vp8dx_start_decode        0067d4d0 f   libvpx:dboolhuff.c.o
 0001:0027c5d0       _vp8dx_bool_decoder_fill   0067d5d0 f   libvpx:dboolhuff.c.o
 0001:0027c6b0       _vp8_dc_quant              0067d6b0 f   libvpx:quant_common.c.o
 0001:0027c6d0       _vp8_dc2quant              0067d6d0 f   libvpx:quant_common.c.o
 0001:0027c700       _vp8_dc_uv_quant           0067d700 f   libvpx:quant_common.c.o
 0001:0027c730       _vp8_ac_yquant             0067d730 f   libvpx:quant_common.c.o
 0001:0027c750       _vp8_ac2quant              0067d750 f   libvpx:quant_common.c.o
 0001:0027c790       _vp8_ac_uv_quant           0067d790 f   libvpx:quant_common.c.o
 0001:0027cbe0       _vp8_decode_mode_mvs       0067dbe0 f   libvpx:decodemv.c.o
 0001:0027ecc0       _vp8_setup_intra_recon     0067fcc0 f   libvpx:setupintrarecon.c.o
 0001:0027ed90       _vp8_setup_intra_recon_top_line 0067fd90 f   libvpx:setupintrarecon.c.o
 0001:0027f610       _vp8_reset_mb_tokens_context 00680610 f   libvpx:detokenize.c.o
 0001:0027f650       _vp8_decode_mb_tokens      00680650 f   libvpx:detokenize.c.o
 0001:00280190       _vp8_copy_and_extend_frame 00681190 f   libvpx:extend.c.o
 0001:00280280       _vp8_copy_and_extend_frame_with_rect 00681280 f   libvpx:extend.c.o
 0001:002804d0       _vp8_extend_mb_row         006814d0 f   libvpx:extend.c.o
 0001:002805a0       _vp8_intra4x4_predict_c    006815a0 f   libvpx:reconintra4x4.c.o
 0001:00280fa0       _vp8_idct_dequant_0_2x_sse2 00681fa0     libvpx:idctllm_sse2.asm.o
 0001:00281047       _vp8_idct_dequant_full_2x_sse2 00682047     libvpx:idctllm_sse2.asm.o
 0001:002812d5       _vp8_idct_dequant_dc_0_2x_sse2 006822d5     libvpx:idctllm_sse2.asm.o
 0001:0028135e       _vp8_idct_dequant_dc_full_2x_sse2 0068235e     libvpx:idctllm_sse2.asm.o
 0001:00281600       _vp8_get_mb_ss_mmx         00682600     libvpx:variance_impl_mmx.asm.o
 0001:00281654       _vp8_get8x8var_mmx         00682654     libvpx:variance_impl_mmx.asm.o
 0001:00281852       _vp8_get4x4var_mmx         00682852     libvpx:variance_impl_mmx.asm.o
 0001:0028191c       _vp8_get4x4sse_cs_mmx      0068291c     libvpx:variance_impl_mmx.asm.o
 0001:002819a6       _vp8_filter_block2d_bil4x4_var_mmx 006829a6     libvpx:variance_impl_mmx.asm.o
 0001:00281a84       _vp8_filter_block2d_bil_var_mmx 00682a84     libvpx:variance_impl_mmx.asm.o
 0001:00281be0       _vp8_get_mb_ss_sse2        00682be0     libvpx:variance_impl_sse2.asm.o
 0001:00281c52       _vp8_get16x16var_sse2      00682c52     libvpx:variance_impl_sse2.asm.o
 0001:00281d7d       _vp8_get8x8var_sse2        00682d7d     libvpx:variance_impl_sse2.asm.o
 0001:00281f19       _vp8_filter_block2d_bil_var_sse2 00682f19     libvpx:variance_impl_sse2.asm.o
 0001:00282177       _vp8_half_horiz_vert_variance8x_h_sse2 00683177     libvpx:variance_impl_sse2.asm.o
 0001:00282237       _vp8_half_horiz_vert_variance16x_h_sse2 00683237     libvpx:variance_impl_sse2.asm.o
 0001:0028232e       _vp8_half_vert_variance8x_h_sse2 0068332e     libvpx:variance_impl_sse2.asm.o
 0001:002823d6       _vp8_half_vert_variance16x_h_sse2 006833d6     libvpx:variance_impl_sse2.asm.o
 0001:002824bb       _vp8_half_horiz_variance8x_h_sse2 006834bb     libvpx:variance_impl_sse2.asm.o
 0001:00282560       _vp8_half_horiz_variance16x_h_sse2 00683560     libvpx:variance_impl_sse2.asm.o
 0001:00282640       _vp8_filter_block2d_bil_var_ssse3 00683640     libvpx:variance_impl_ssse3.asm.o
 0001:00282990       _vp8_find_near_mvs         00683990 f   libvpx:findnearmv.c.o
 0001:00282bd0       _vp8_find_near_mvs_bias    00683bd0 f   libvpx:findnearmv.c.o
 0001:00283210       _vp8_mv_ref_probs          00684210 f   libvpx:findnearmv.c.o
 0001:00283260       _png_write_info_before_PLTE 00684260 f   libpng_mini:pngwrite.o
 0001:002832e0       _png_write_info            006842e0 f   libpng_mini:pngwrite.o
 0001:00283370       _png_write_end             00684370 f   libpng_mini:pngwrite.o
 0001:002833f0       _png_create_write_struct_2 006843f0 f   libpng_mini:pngwrite.o
 0001:002834a0       _png_create_write_struct   006844a0 f   libpng_mini:pngwrite.o
 0001:002834f0       _png_write_row             006844f0 f   libpng_mini:pngwrite.o
 0001:002835f0       _png_write_rows            006845f0 f   libpng_mini:pngwrite.o
 0001:00283630       _png_write_image           00684630 f   libpng_mini:pngwrite.o
 0001:00283680       _png_destroy_write_struct  00684680 f   libpng_mini:pngwrite.o
 0001:00283700       _png_set_filter            00684700 f   libpng_mini:pngwrite.o
 0001:00283730       _png_set_compression_level 00684730 f   libpng_mini:pngwrite.o
 0001:00283750       _png_set_compression_mem_level 00684750 f   libpng_mini:pngwrite.o
 0001:00283770       _png_set_compression_strategy 00684770 f   libpng_mini:pngwrite.o
 0001:00283790       _png_set_compression_window_bits 00684790 f   libpng_mini:pngwrite.o
 0001:002837c0       _png_set_compression_method 006847c0 f   libpng_mini:pngwrite.o
 0001:002837e0       _png_set_write_status_fn   006847e0 f   libpng_mini:pngwrite.o
 0001:00283800       _png_write_png             00684800 f   libpng_mini:pngwrite.o
 0001:00283890       _png_set_IHDR              00684890 f   libpng_mini:pngset.o
 0001:00283990       _png_set_PLTE              00684990 f   libpng_mini:pngset.o
 0001:00283a50       _png_set_text_2            00684a50 f   libpng_mini:pngset.o
 0001:00283d40       _png_set_text              00684d40 f   libpng_mini:pngset.o
 0001:00283d80       _png_set_rows              00684d80 f   libpng_mini:pngset.o
 0001:00283de0       _png_set_compression_buffer_size 00684de0 f   libpng_mini:pngset.o
 0001:00283e40       _png_set_invalid           00684e40 f   libpng_mini:pngset.o
 0001:00283e60       _png_malloc_base           00684e60 f   libpng_mini:pngmem.o
 0001:00283ea0       _png_malloc_array          00684ea0 f   libpng_mini:pngmem.o
 0001:00283ef0       _png_realloc_array         00684ef0 f   libpng_mini:pngmem.o
 0001:00283fd0       _png_malloc                00684fd0 f   libpng_mini:pngmem.o
 0001:00284010       _png_calloc                00685010 f   libpng_mini:pngmem.o
 0001:00284050       _png_malloc_default        00685050 f   libpng_mini:pngmem.o
 0001:00284090       _png_malloc_warn           00685090 f   libpng_mini:pngmem.o
 0001:002840b0       _png_free                  006850b0 f   libpng_mini:pngmem.o
 0001:002840e0       _png_destroy_png_struct    006850e0 f   libpng_mini:pngmem.o
 0001:00284180       _png_free_default          00685180 f   libpng_mini:pngmem.o
 0001:002841a0       _png_set_mem_fn            006851a0 f   libpng_mini:pngmem.o
 0001:002841d0       _png_get_mem_ptr           006851d0 f   libpng_mini:pngmem.o
 0001:002841f0       _png_zalloc                006851f0 f   libpng_mini:png.o
 0001:00284230       _png_zfree                 00685230 f   libpng_mini:png.o
 0001:00284240       _png_reset_crc             00685240 f   libpng_mini:png.o
 0001:00284270       _png_calculate_crc         00685270 f   libpng_mini:png.o
 0001:002842d0       _png_user_version_check    006852d0 f   libpng_mini:png.o
 0001:00284340       _png_create_png_struct     00685340 f   libpng_mini:png.o
 0001:00284460       _png_create_info_struct    00685460 f   libpng_mini:png.o
 0001:00284500       _png_info_init_3           00685500 f   libpng_mini:png.o
 0001:002845a0       _png_data_freer            006855a0 f   libpng_mini:png.o
 0001:002845f0       _png_free_data             006855f0 f   libpng_mini:png.o
 0001:00284770       _png_destroy_info_struct   00685770 f   libpng_mini:png.o
 0001:00284820       _png_get_io_ptr            00685820 f   libpng_mini:png.o
 0001:00284840       _png_init_io               00685840 f   libpng_mini:png.o
 0001:00284860       _png_get_copyright         00685860 f   libpng_mini:png.o
 0001:00284870       _png_get_libpng_ver        00685870 f   libpng_mini:png.o
 0001:00284880       _png_get_header_ver        00685880 f   libpng_mini:png.o
 0001:00284890       _png_get_header_version    00685890 f   libpng_mini:png.o
 0001:002848a0       _png_access_version_number 006858a0 f   libpng_mini:png.o
 0001:002848b0       _png_zstream_error         006858b0 f   libpng_mini:png.o
 0001:00284970       _png_check_IHDR            00685970 f   libpng_mini:png.o
 0001:00284a50       _png_safecat               00685a50 f   libpng_mini:pngerror.o
 0001:00284aa0       _png_free_jmpbuf           00685aa0 f   libpng_mini:pngerror.o
 0001:00284b30       _png_longjmp               00685b30 f   libpng_mini:pngerror.o
 0001:00284b70       _png_err                   00685b70 f   libpng_mini:pngerror.o
 0001:00284ba0       _png_chunk_report          00685ba0 f   libpng_mini:pngerror.o
 0001:00284bc0       _png_set_longjmp_fn        00685bc0 f   libpng_mini:pngerror.o
 0001:00284c50       _png_set_error_fn          00685c50 f   libpng_mini:pngerror.o
 0001:00284c70       _png_get_error_ptr         00685c70 f   libpng_mini:pngerror.o
 0001:00284d70       _png_save_uint_32          00685d70 f   libpng_mini:pngwutil.o
 0001:00284da0       _png_save_uint_16          00685da0 f   libpng_mini:pngwutil.o
 0001:00284dc0       _png_write_sig             00685dc0 f   libpng_mini:pngwutil.o
 0001:00284e30       _png_write_chunk_start     00685e30 f   libpng_mini:pngwutil.o
 0001:00284e70       _png_write_chunk_data      00685e70 f   libpng_mini:pngwutil.o
 0001:00284f10       _png_write_chunk_end       00685f10 f   libpng_mini:pngwutil.o
 0001:00284f30       _png_write_chunk           00685f30 f   libpng_mini:pngwutil.o
 0001:00284f70       _png_free_buffer_list      00685f70 f   libpng_mini:pngwutil.o
 0001:00284fb0       _png_write_IHDR            00685fb0 f   libpng_mini:pngwutil.o
 0001:002851d0       _png_write_PLTE            006861d0 f   libpng_mini:pngwutil.o
 0001:00285280       _png_compress_IDAT         00686280 f   libpng_mini:pngwutil.o
 0001:00285830       _png_write_IEND            00686830 f   libpng_mini:pngwutil.o
 0001:00285860       _png_write_start_row       00686860 f   libpng_mini:pngwutil.o
 0001:002858f0       _png_write_finish_row      006868f0 f   libpng_mini:pngwutil.o
 0001:00285940       _png_write_find_filter     00686940 f   libpng_mini:pngwutil.o
 0001:002859a0       _png_default_write_data    006869a0 f   libpng_mini:pngwio.o
 0001:002859f0       _png_write_data            006869f0 f   libpng_mini:pngwio.o
 0001:00285a10       _png_set_write_fn          00686a10 f   libpng_mini:pngwio.o
 0001:00286a40       _deflateSetDictionary      00687a40 f   libz_mini:deflate.o
 0001:00286c70       _deflateResetKeep          00687c70 f   libz_mini:deflate.o
 0001:00286d50       _deflateReset              00687d50 f   libz_mini:deflate.o
 0001:00286e20       _deflateSetHeader          00687e20 f   libz_mini:deflate.o
 0001:00286e50       _deflatePending            00687e50 f   libz_mini:deflate.o
 0001:00286e90       _deflatePrime              00687e90 f   libz_mini:deflate.o
 0001:00286f20       _deflateTune               00687f20 f   libz_mini:deflate.o
 0001:00286f60       _deflateBound              00687f60 f   libz_mini:deflate.o
 0001:00287070       _deflate                   00688070 f   libz_mini:deflate.o
 0001:002880f0       _deflateParams             006890f0 f   libz_mini:deflate.o
 0001:00288200       _deflateEnd                00689200 f   libz_mini:deflate.o
 0001:00288300       _deflateInit2_             00689300 f   libz_mini:deflate.o
 0001:002885d0       _deflateInit_              006895d0 f   libz_mini:deflate.o
 0001:00288620       _deflateCopy               00689620 f   libz_mini:deflate.o
 0001:00288a10       _get_crc_table             00689a10 f   libz_mini:crc32.o
 0001:00288a20       _crc32                     00689a20 f   libz_mini:crc32.o
 0001:00288cd0       _crc32_combine             00689cd0 f   libz_mini:crc32.o
 0001:00288cf0       _crc32_combine64           00689cf0 f   libz_mini:crc32.o
 0001:00289f10       __tr_init                  0068af10 f   libz_mini:trees.o
 0001:00289ff0       __tr_stored_block          0068aff0 f   libz_mini:trees.o
 0001:0028a110       __tr_flush_bits            0068b110 f   libz_mini:trees.o
 0001:0028a120       __tr_align                 0068b120 f   libz_mini:trees.o
 0001:0028a210       __tr_flush_block           0068b210 f   libz_mini:trees.o
 0001:0028a840       __tr_tally                 0068b840 f   libz_mini:trees.o
 0001:0028a8e0       _zlibVersion               0068b8e0 f   libz_mini:zutil.o
 0001:0028a8f0       _zlibCompileFlags          0068b8f0 f   libz_mini:zutil.o
 0001:0028a900       _zError                    0068b900 f   libz_mini:zutil.o
 0001:0028a920       _zcalloc                   0068b920 f   libz_mini:zutil.o
 0001:0028a940       _zcfree                    0068b940 f   libz_mini:zutil.o
 0001:0028a9f0       _adler32                   0068b9f0 f   libz_mini:adler32.o
 0001:0028adb0       _adler32_combine           0068bdb0 f   libz_mini:adler32.o
 0001:0028add0       _adler32_combine64         0068bdd0 f   libz_mini:adler32.o
 0001:0028adf0       _DirectSoundCreate@12      0068bdf0 f   dsound:DSOUND.dll
 0001:0028b3b0       ___ashldi3                 0068c3b0 f   libcompat-to-msvc:dll_math.o
 0001:0028b410       ___ashrdi3                 0068c410 f   libcompat-to-msvc:dll_math.o
 0001:0028b460       ___cmpdi2                  0068c460 f   libcompat-to-msvc:dll_math.o
 0001:0028b4a0       ___divdi3                  0068c4a0 f   libcompat-to-msvc:dll_math.o
 0001:0028bab0       ___lshrdi3                 0068cab0 f   libcompat-to-msvc:dll_math.o
 0001:0028bb00       ___moddi3                  0068cb00 f   libcompat-to-msvc:dll_math.o
 0001:0028bb90       ___qdivrem                 0068cb90 f   libcompat-to-msvc:dll_math.o
 0001:0028bc20       ___ucmpdi2                 0068cc20 f   libcompat-to-msvc:dll_math.o
 0001:0028bc60       ___udivdi3                 0068cc60 f   libcompat-to-msvc:dll_math.o
 0001:0028c200       ___umoddi3                 0068d200 f   libcompat-to-msvc:dll_math.o
 0001:0028c270       ___chkstk_ms               0068d270     libcompat-to-msvc:dll_dependency.o
 0001:0028c29a       __alloca                   0068d29a     libcompat-to-msvc:dll_dependency.o
 0001:0028c29a       ___chkstk                  0068d29a     libcompat-to-msvc:dll_dependency.o
 0001:0028c2d0       ___ms_vsnprintf            0068d2d0 f   libcompat-to-msvc:vsnprintf.o
 0001:0028c2e0       ___mingw_vsnprintf         0068d2e0 f   libcompat-to-msvc:vsnprintf.o
 0001:0028c2f0       _sprintf                   0068d2f0 f   msvcrtd:MSVCR100D.dll
 0001:0028c300       @__security_check_cookie@4 0068d300 f   msvcrtd:secchk.obj
 0001:0028c310       _exit                      0068d310 f   msvcrtd:MSVCR100D.dll
 0001:0028c316       _fflush                    0068d316 f   msvcrtd:MSVCR100D.dll
 0001:0028c31c       _fclose                    0068d31c f   msvcrtd:MSVCR100D.dll
 0001:0028c322       __wassert                  0068d322 f   msvcrtd:MSVCR100D.dll
 0001:0028c328       _memcpy                    0068d328 f   msvcrtd:MSVCR100D.dll
 0001:0028c330       __aullshr                  0068d330 f   msvcrtd:ullshr.obj
 0001:0028c350       __allmul                   0068d350 f   msvcrtd:llmul.obj
 0001:0028c390       __allshl                   0068d390 f   msvcrtd:llshl.obj
 0001:0028c3b0       __ftol2_sse                0068d3b0 f   msvcrtd:ftol2.obj
 0001:0028c3b9       __ftol2_pentium4           0068d3b9 f   msvcrtd:ftol2.obj
 0001:0028c3cc       __ftol2_sse_excpt          0068d3cc f   msvcrtd:ftol2.obj
 0001:0028c3e6       __ftol2                    0068d3e6 f   msvcrtd:ftol2.obj
 0001:0028c460       __alloca_probe             0068d460     msvcrtd:chkstk.obj
 0001:0028c460       __chkstk                   0068d460 f   msvcrtd:chkstk.obj
 0001:0028c48c       _free                      0068d48c f   msvcrtd:MSVCR100D.dll
 0001:0028c492       _memset                    0068d492 f   msvcrtd:MSVCR100D.dll
 0001:0028c498       _calloc                    0068d498 f   msvcrtd:MSVCR100D.dll
 0001:0028c49e       _labs                      0068d49e f   msvcrtd:MSVCR100D.dll
 0001:0028c4a4       _rand                      0068d4a4 f   msvcrtd:MSVCR100D.dll
 0001:0028c4aa       __snprintf                 0068d4aa f   msvcrtd:MSVCR100D.dll
 0001:0028c4b0       _strncpy                   0068d4b0 f   msvcrtd:MSVCR100D.dll
 0001:0028c4b6       _strlen                    0068d4b6 f   msvcrtd:MSVCR100D.dll
 0001:0028c4bc       _strcat                    0068d4bc f   msvcrtd:MSVCR100D.dll
 0001:0028c4c2       __stricmp                  0068d4c2 f   msvcrtd:MSVCR100D.dll
 0001:0028c4c8       _realloc                   0068d4c8 f   msvcrtd:MSVCR100D.dll
 0001:0028c4ce       _strrchr                   0068d4ce f   msvcrtd:MSVCR100D.dll
 0001:0028c4d4       _strcmp                    0068d4d4 f   msvcrtd:MSVCR100D.dll
 0001:0028c4da       _toupper                   0068d4da f   msvcrtd:MSVCR100D.dll
 0001:0028c4e0       _sscanf                    0068d4e0 f   msvcrtd:MSVCR100D.dll
 0001:0028c4e6       _strtok                    0068d4e6 f   msvcrtd:MSVCR100D.dll
 0001:0028c4ec       _strcpy                    0068d4ec f   msvcrtd:MSVCR100D.dll
 0001:0028c4f2       _fprintf                   0068d4f2 f   msvcrtd:MSVCR100D.dll
 0001:0028c4f8       ___iob_func                0068d4f8 f   msvcrtd:MSVCR100D.dll
 0001:0028c4fe       _atoi                      0068d4fe f   msvcrtd:MSVCR100D.dll
 0001:0028c504       _strtol                    0068d504 f   msvcrtd:MSVCR100D.dll
 0001:0028c510       __onexit                   0068d510 f   msvcrtd:atonexit.obj
 0001:0028c610       _atexit                    0068d610 f   msvcrtd:atonexit.obj
 0001:0028c62c       __time64                   0068d62c f   msvcrtd:MSVCR100D.dll
 0001:0028c632       __strdup                   0068d632 f   msvcrtd:MSVCR100D.dll
 0001:0028c638       _isdigit                   0068d638 f   msvcrtd:MSVCR100D.dll
 0001:0028c63e       _tolower                   0068d63e f   msvcrtd:MSVCR100D.dll
 0001:0028c644       _malloc                    0068d644 f   msvcrtd:MSVCR100D.dll
 0001:0028c64a       _strchr                    0068d64a f   msvcrtd:MSVCR100D.dll
 0001:0028c650       __chdir                    0068d650 f   msvcrtd:MSVCR100D.dll
 0001:0028c656       _memcmp                    0068d656 f   msvcrtd:MSVCR100D.dll
 0001:0028c660       __aulldiv                  0068d660 f   msvcrtd:ulldiv.obj
 0001:0028c6c8       _islower                   0068d6c8 f   msvcrtd:MSVCR100D.dll
 0001:0028c6ce       _isupper                   0068d6ce f   msvcrtd:MSVCR100D.dll
 0001:0028c6d4       _getenv                    0068d6d4 f   msvcrtd:MSVCR100D.dll
 0001:0028c6da       _fopen                     0068d6da f   msvcrtd:MSVCR100D.dll
 0001:0028c6e0       _fwrite                    0068d6e0 f   msvcrtd:MSVCR100D.dll
 0001:0028c6e6       _perror                    0068d6e6 f   msvcrtd:MSVCR100D.dll
 0001:0028c6ec       _fseek                     0068d6ec f   msvcrtd:MSVCR100D.dll
 0001:0028c6f2       _strstr                    0068d6f2 f   msvcrtd:MSVCR100D.dll
 0001:0028c6f8       _strncmp                   0068d6f8 f   msvcrtd:MSVCR100D.dll
 0001:0028c6fe       _isalnum                   0068d6fe f   msvcrtd:MSVCR100D.dll
 0001:0028c704       __strtoi64                 0068d704 f   msvcrtd:MSVCR100D.dll
 0001:0028c70a       __errno                    0068d70a f   msvcrtd:MSVCR100D.dll
 0001:0028c710       __stat64i32                0068d710 f   msvcrtd:MSVCR100D.dll
 0001:0028c716       __localtime64              0068d716 f   msvcrtd:MSVCR100D.dll
 0001:0028c71c       __aligned_free             0068d71c f   msvcrtd:MSVCR100D.dll
 0001:0028c722       _sqrt                      0068d722 f   msvcrtd:MSVCR100D.dll
 0001:0028c728       _strncat                   0068d728 f   msvcrtd:MSVCR100D.dll
 0001:0028c72e       __aligned_malloc           0068d72e f   msvcrtd:MSVCR100D.dll
 0001:0028c734       _qsort                     0068d734 f   msvcrtd:MSVCR100D.dll
 0001:0028c73a       _bsearch                   0068d73a f   msvcrtd:MSVCR100D.dll
 0001:0028c740       _strerror                  0068d740 f   msvcrtd:MSVCR100D.dll
 0001:0028c746       _ftell                     0068d746 f   msvcrtd:MSVCR100D.dll
 0001:0028c74c       _atof                      0068d74c f   msvcrtd:MSVCR100D.dll
 0001:0028c752       _memmove                   0068d752 f   msvcrtd:MSVCR100D.dll
 0001:0028c758       __fstat64i32               0068d758 f   msvcrtd:MSVCR100D.dll
 0001:0028c75e       _isalpha                   0068d75e f   msvcrtd:MSVCR100D.dll
 0001:0028c764       _printf                    0068d764 f   msvcrtd:MSVCR100D.dll
 0001:0028c76a       __strnicmp                 0068d76a f   msvcrtd:MSVCR100D.dll
 0001:0028c770       _setvbuf                   0068d770 f   msvcrtd:MSVCR100D.dll
 0001:0028c776       _freopen                   0068d776 f   msvcrtd:MSVCR100D.dll
 0001:0028c77c       __getdcwd                  0068d77c f   msvcrtd:MSVCR100D.dll
 0001:0028c782       __findfirst64i32           0068d782 f   msvcrtd:MSVCR100D.dll
 0001:0028c788       __findnext64i32            0068d788 f   msvcrtd:MSVCR100D.dll
 0001:0028c78e       __findclose                0068d78e f   msvcrtd:MSVCR100D.dll
 0001:0028c7a0       __allshr                   0068d7a0 f   msvcrtd:llshr.obj
 0001:0028c7d0       __alldiv                   0068d7d0 f   msvcrtd:lldiv.obj
 0001:0028c87a       _atan                      0068d87a f   msvcrtd:MSVCR100D.dll
 0001:0028c880       _sin                       0068d880 f   msvcrtd:MSVCR100D.dll
 0001:0028c886       _pow                       0068d886 f   msvcrtd:MSVCR100D.dll
 0001:0028c88c       _longjmp                   0068d88c f   msvcrtd:MSVCR100D.dll
 0001:0028c892       __setjmp3                  0068d892 f   msvcrtd:MSVCR100D.dll
 0001:0028c898       _rewind                    0068d898 f   msvcrtd:MSVCR100D.dll
 0001:0028c89e       _fread                     0068d89e f   msvcrtd:MSVCR100D.dll
 0001:0028c8a4       __lrotl                    0068d8a4 f   msvcrtd:MSVCR100D.dll
 0001:0028c8aa       __fileno                   0068d8aa f   msvcrtd:MSVCR100D.dll
 0001:0028c8b0       _fabs                      0068d8b0 f   msvcrtd:MSVCR100D.dll
 0001:0028c8b6       _cos                       0068d8b6 f   msvcrtd:MSVCR100D.dll
 0001:0028c8bc       _floor                     0068d8bc f   msvcrtd:MSVCR100D.dll
 0001:0028c8c2       _tan                       0068d8c2 f   msvcrtd:MSVCR100D.dll
 0001:0028c8c8       _strtoul                   0068d8c8 f   msvcrtd:MSVCR100D.dll
 0001:0028c8ce       _vsnprintf                 0068d8ce f   msvcrtd:MSVCR100D.dll
 0001:0028c8ce       __vsnprintf                0068d8ce f   msvcrtd:MSVCR100D.dll
 0001:0028c8d4       _fputs                     0068d8d4 f   msvcrtd:MSVCR100D.dll
 0001:0028c8da       __rotl                     0068d8da f   msvcrtd:MSVCR100D.dll
 0001:0028c8e0       __byteswap_ulong           0068d8e0 f   msvcrtd:MSVCR100D.dll
 0001:0028c8e6       __rotl64                   0068d8e6 f   msvcrtd:MSVCR100D.dll
 0001:0028c8ec       __byteswap_uint64          0068d8ec f   msvcrtd:MSVCR100D.dll
 0001:0028c8f2       _getchar                   0068d8f2 f   msvcrtd:MSVCR100D.dll
 0001:0028c8f8       _puts                      0068d8f8 f   msvcrtd:MSVCR100D.dll
 0001:0028c8fe       _vsprintf                  0068d8fe f   msvcrtd:MSVCR100D.dll
 0001:0028c904       _signal                    0068d904 f   msvcrtd:MSVCR100D.dll
 0001:0028c90a       _vfprintf                  0068d90a f   msvcrtd:MSVCR100D.dll
 0001:0028c910       _atol                      0068d910 f   msvcrtd:MSVCR100D.dll
 0001:0028c916       _abort                     0068d916 f   msvcrtd:MSVCR100D.dll
 0001:0028ca10       _WinMainCRTStartup         0068da10 f   msvcrtd:crtexew.obj
 0001:0028cd30       _NtCurrentTeb              0068dd30 f i msvcrtd:crtexew.obj
 0001:0028cdae       __assert                   0068ddae f   msvcrtd:MSVCR100D.dll
 0001:0028cdb4       _exp                       0068ddb4 f   msvcrtd:MSVCR100D.dll
 0001:0028cdc0       ___report_gsfailure        0068ddc0 f   msvcrtd:gs_report.obj
 0001:0028ced0       ___sse2_available_init     0068ded0 f   msvcrtd:cpu_disp.obj
 0001:0028cee6       __unlock                   0068dee6 f   msvcrtd:MSVCR100D.dll
 0001:0028ceec       ___dllonexit               0068deec f   msvcrtd:MSVCR100D.dll
 0001:0028cef2       __lock                     0068def2 f   msvcrtd:MSVCR100D.dll
 0001:0028cf00       __except_handler4          0068df00 f   msvcrtd:chandler4gs.obj
 0001:0028cf30       ?__CxxUnhandledExceptionFilter@@YGJPAU_EXCEPTION_POINTERS@@@Z 0068df30 f   msvcrtd:unhandld.obj
 0001:0028cfa0       ___CxxSetUnhandledExceptionFilter 0068dfa0 f   msvcrtd:unhandld.obj
 0001:0028cfc0       __setdefaultprecision      0068dfc0 f   msvcrtd:fp8.obj
 0001:0028d000       __invoke_watson_if_error   0068e000 f i msvcrtd:fp8.obj
 0001:0028d030       __setargv                  0068e030 f   msvcrtd:dllargv.obj
 0001:0028d030       __matherr                  0068e030 f   msvcrtd:merr.obj
 0001:0028d040       __RTC_Initialize           0068e040 f   msvcrtd:_initsect_.obj
 0001:0028d070       __RTC_Terminate            0068e070 f   msvcrtd:_initsect_.obj
 0001:0028d096       __amsg_exit                0068e096 f   msvcrtd:MSVCR100D.dll
 0001:0028d0a0       ___security_init_cookie    0068e0a0 f   msvcrtd:gs_support.obj
 0001:0028d180       __XcptFilter               0068e180 f   msvcrtd:MSVCR100D.dll
 0001:0028d190       __ValidateImageBase        0068e190 f   msvcrtd:pesect.obj
 0001:0028d1f0       __FindPESection            0068e1f0 f   msvcrtd:pesect.obj
 0001:0028d270       __IsNonwritableInCurrentImage 0068e270 f   msvcrtd:pesect.obj
 0001:0028d382       __initterm                 0068e382 f   msvcrtd:MSVCR100D.dll
 0001:0028d388       __initterm_e               0068e388 f   msvcrtd:MSVCR100D.dll
 0001:0028d38e       __crt_debugger_hook        0068e38e f   msvcrtd:MSVCR100D.dll
 0001:0028d394       __except_handler4_common   0068e394 f   msvcrtd:MSVCR100D.dll
 0001:0028d39a       ?terminate@@YAXXZ          0068e39a f   msvcrtd:MSVCR100D.dll
 0001:0028d3a0       __controlfp_s              0068e3a0 f   msvcrtd:MSVCR100D.dll
 0001:0028d3a6       __invoke_watson            0068e3a6 f   msvcrtd:MSVCR100D.dll
 0001:0028d3ac       _InterlockedCompareExchange@12 0068e3ac f   kernel32:KERNEL32.dll
 0001:0028d3b2       _GetSystemPowerStatus@4    0068e3b2 f   kernel32:KERNEL32.dll
 0001:0028d580       _ogg_page_version          0068e580 f   libogg:framing.o
 0001:0028d590       _ogg_page_continued        0068e590 f   libogg:framing.o
 0001:0028d5a0       _ogg_page_bos              0068e5a0 f   libogg:framing.o
 0001:0028d5c0       _ogg_page_eos              0068e5c0 f   libogg:framing.o
 0001:0028d5e0       _ogg_page_granulepos       0068e5e0 f   libogg:framing.o
 0001:0028d630       _ogg_page_serialno         0068e630 f   libogg:framing.o
 0001:0028d640       _ogg_page_pageno           0068e640 f   libogg:framing.o
 0001:0028d650       _ogg_page_packets          0068e650 f   libogg:framing.o
 0001:0028d680       _ogg_stream_check          0068e680 f   libogg:framing.o
 0001:0028d6a0       _ogg_stream_clear          0068e6a0 f   libogg:framing.o
 0001:0028d710       _ogg_stream_init           0068e710 f   libogg:framing.o
 0001:0028d8d0       _ogg_stream_destroy        0068e8d0 f   libogg:framing.o
 0001:0028d900       _ogg_page_checksum_set     0068e900 f   libogg:framing.o
 0001:0028dcc0       _ogg_stream_iovecin        0068ecc0 f   libogg:framing.o
 0001:0028df70       _ogg_stream_packetin       0068ef70 f   libogg:framing.o
 0001:0028dfc0       _ogg_stream_flush          0068efc0 f   libogg:framing.o
 0001:0028dfe0       _ogg_stream_flush_fill     0068efe0 f   libogg:framing.o
 0001:0028e000       _ogg_stream_pageout        0068f000 f   libogg:framing.o
 0001:0028e070       _ogg_stream_pageout_fill   0068f070 f   libogg:framing.o
 0001:0028e0d0       _ogg_stream_eos            0068f0d0 f   libogg:framing.o
 0001:0028e0f0       _ogg_sync_init             0068f0f0 f   libogg:framing.o
 0001:0028e130       _ogg_sync_clear            0068f130 f   libogg:framing.o
 0001:0028e180       _ogg_sync_destroy          0068f180 f   libogg:framing.o
 0001:0028e1b0       _ogg_sync_check            0068f1b0 f   libogg:framing.o
 0001:0028e1c0       _ogg_sync_buffer           0068f1c0 f   libogg:framing.o
 0001:0028e260       _ogg_sync_wrote            0068f260 f   libogg:framing.o
 0001:0028e290       _ogg_sync_pageseek         0068f290 f   libogg:framing.o
 0001:0028e440       _ogg_sync_pageout          0068f440 f   libogg:framing.o
 0001:0028e4b0       _ogg_stream_pagein         0068f4b0 f   libogg:framing.o
 0001:0028e880       _ogg_sync_reset            0068f880 f   libogg:framing.o
 0001:0028e8c0       _ogg_stream_reset          0068f8c0 f   libogg:framing.o
 0001:0028e950       _ogg_stream_reset_serialno 0068f950 f   libogg:framing.o
 0001:0028ea00       _ogg_stream_packetout      0068fa00 f   libogg:framing.o
 0001:0028ea30       _ogg_stream_packetpeek     0068fa30 f   libogg:framing.o
 0001:0028ea60       _ogg_packet_clear          0068fa60 f   libogg:framing.o
 0001:0028eab0       _vorbis_synthesis          0068fab0 f   libvorbis:synthesis.o
 0001:0028ecb0       _vorbis_synthesis_trackonly 0068fcb0 f   libvorbis:synthesis.o
 0001:0028edd0       _vorbis_packet_blocksize   0068fdd0 f   libvorbis:synthesis.o
 0001:0028ee80       _vorbis_synthesis_halfrate 0068fe80 f   libvorbis:synthesis.o
 0001:0028eeb0       _vorbis_synthesis_halfrate_p 0068feb0 f   libvorbis:synthesis.o
 0001:0028f040       _vorbis_comment_init       00690040 f   libvorbis:info.o
 0001:0028f060       _vorbis_comment_add        00690060 f   libvorbis:info.o
 0001:0028f100       _vorbis_comment_add_tag    00690100 f   libvorbis:info.o
 0001:0028f230       _vorbis_comment_query      00690230 f   libvorbis:info.o
 0001:0028f340       _vorbis_comment_query_count 00690340 f   libvorbis:info.o
 0001:0028f430       _vorbis_comment_clear      00690430 f   libvorbis:info.o
 0001:0028f4c0       _vorbis_info_blocksize     006904c0 f   libvorbis:info.o
 0001:0028f4e0       _vorbis_info_init          006904e0 f   libvorbis:info.o
 0001:0028f540       _vorbis_info_clear         00690540 f   libvorbis:info.o
 0001:0028f6d0       _vorbis_synthesis_idheader 006906d0 f   libvorbis:info.o
 0001:0028f780       _vorbis_synthesis_headerin 00690780 f   libvorbis:info.o
 0001:0028ff10       _vorbis_commentheader_out  00690f10 f   libvorbis:info.o
 0001:0028ffc0       _vorbis_analysis_headerout 00690fc0 f   libvorbis:info.o
 0001:002908c0       _vorbis_granule_time       006918c0 f   libvorbis:info.o
 0001:00290910       _vorbis_version_string     00691910 f   libvorbis:info.o
 0001:00290a70       _vorbis_block_init         00691a70 f   libvorbis:block.o
 0001:00290b30       __vorbis_block_alloc       00691b30 f   libvorbis:block.o
 0001:00290bb0       __vorbis_block_ripcord     00691bb0 f   libvorbis:block.o
 0001:00290c20       _vorbis_block_clear        00691c20 f   libvorbis:block.o
 0001:00290d00       _vorbis_dsp_clear          00691d00 f   libvorbis:block.o
 0001:00291460       _vorbis_analysis_init      00692460 f   libvorbis:block.o
 0001:002914e0       _vorbis_analysis_buffer    006924e0 f   libvorbis:block.o
 0001:002915b0       _vorbis_analysis_wrote     006925b0 f   libvorbis:block.o
 0001:00291740       _vorbis_analysis_blockout  00692740 f   libvorbis:block.o
 0001:00291c80       _vorbis_synthesis_restart  00692c80 f   libvorbis:block.o
 0001:00291d10       _vorbis_synthesis_init     00692d10 f   libvorbis:block.o
 0001:00291dc0       _vorbis_synthesis_blockin  00692dc0 f   libvorbis:block.o
 0001:002925e0       _vorbis_synthesis_pcmout   006935e0 f   libvorbis:block.o
 0001:00292660       _vorbis_synthesis_read     00693660 f   libvorbis:block.o
 0001:00292690       _vorbis_synthesis_lapout   00693690 f   libvorbis:block.o
 0001:002928d0       _vorbis_window             006938d0 f   libvorbis:block.o
 0001:00292e60       _ov_ilog                   00693e60 f   libvorbis:sharedbook.o
 0001:00292e80       __float32_pack             00693e80 f   libvorbis:sharedbook.o
 0001:00292f30       __float32_unpack           00693f30 f   libvorbis:sharedbook.o
 0001:00292f80       __make_words               00693f80 f   libvorbis:sharedbook.o
 0001:002931c0       __book_maptype1_quantvals  006941c0 f   libvorbis:sharedbook.o
 0001:00293260       __book_unquantize          00694260 f   libvorbis:sharedbook.o
 0001:00293290       _vorbis_staticbook_destroy 00694290 f   libvorbis:sharedbook.o
 0001:002932e0       _vorbis_book_clear         006942e0 f   libvorbis:sharedbook.o
 0001:00293360       _vorbis_book_init_encode   00694360 f   libvorbis:sharedbook.o
 0001:00293560       _vorbis_book_init_decode   00694560 f   libvorbis:sharedbook.o
 0001:00293c50       _vorbis_book_codeword      00694c50 f   libvorbis:sharedbook.o
 0001:00293c70       _vorbis_book_codelen       00694c70 f   libvorbis:sharedbook.o
 0001:00295d60       __vp_global_look           00696d60 f   libvorbis:psy.o
 0001:00295da0       __vp_global_free           00696da0 f   libvorbis:psy.o
 0001:00295dc0       __vi_gpsy_free             00696dc0 f   libvorbis:psy.o
 0001:00295de0       __vi_psy_free              00696de0 f   libvorbis:psy.o
 0001:00295e00       __vp_psy_init              00696e00 f   libvorbis:psy.o
 0001:00296650       __vp_psy_clear             00697650 f   libvorbis:psy.o
 0001:00296740       __vp_noisemask             00697740 f   libvorbis:psy.o
 0001:002968a0       __vp_tonemask              006978a0 f   libvorbis:psy.o
 0001:00296cb0       __vp_offset_and_mix        00697cb0 f   libvorbis:psy.o
 0001:00296de0       __vp_ampmax_decay          00697de0 f   libvorbis:psy.o
 0001:00296e30       __vp_couple_quantize_normalize 00697e30 f   libvorbis:psy.o
 0001:002976e0       _vorbis_staticbook_pack    006986e0 f   libvorbis:codebook.o
 0001:00297ad0       _vorbis_staticbook_unpack  00698ad0 f   libvorbis:codebook.o
 0001:00297ed0       _vorbis_book_encode        00698ed0 f   libvorbis:codebook.o
 0001:00297f30       _vorbis_book_decode        00698f30 f   libvorbis:codebook.o
 0001:00298100       _vorbis_book_decodevs_add  00699100 f   libvorbis:codebook.o
 0001:002983c0       _vorbis_book_decodev_add   006993c0 f   libvorbis:codebook.o
 0001:002989a0       _vorbis_book_decodev_set   006999a0 f   libvorbis:codebook.o
 0001:00298c30       _vorbis_book_decodevv_add  00699c30 f   libvorbis:codebook.o
 0001:00298ed0       _vorbis_lpc_from_data      00699ed0 f   libvorbis:lpc.o
 0001:00299110       _vorbis_lpc_predict        0069a110 f   libvorbis:lpc.o
 0001:00299560       __ve_envelope_init         0069a560 f   libvorbis:envelope.o
 0001:00299790       __ve_envelope_clear        0069a790 f   libvorbis:envelope.o
 0001:00299820       __ve_envelope_search       0069a820 f   libvorbis:envelope.o
 0001:00299ab0       __ve_envelope_mark         0069aab0 f   libvorbis:envelope.o
 0001:00299bc0       __ve_envelope_shift        0069abc0 f   libvorbis:envelope.o
 0001:0029a4e0       _mdct_init                 0069b4e0 f   libvorbis:mdct.o
 0001:0029a740       _mdct_clear                0069b740 f   libvorbis:mdct.o
 0001:0029a7a0       _mdct_backward             0069b7a0 f   libvorbis:mdct.o
 0001:0029ab40       _mdct_forward              0069bb40 f   libvorbis:mdct.o
 0001:0029aed0       _vorbis_bitrate_init       0069bed0 f   libvorbis:bitrate.o
 0001:0029b040       _vorbis_bitrate_clear      0069c040 f   libvorbis:bitrate.o
 0001:0029b070       _vorbis_bitrate_managed    0069c070 f   libvorbis:bitrate.o
 0001:0029b0a0       _vorbis_bitrate_addblock   0069c0a0 f   libvorbis:bitrate.o
 0001:0029b600       _vorbis_bitrate_flushpacket 0069c600 f   libvorbis:bitrate.o
 0001:0029de90       _drft_forward              0069ee90 f   libvorbis:smallft.o
 0001:0029e0c0       _drft_backward             0069f0c0 f   libvorbis:smallft.o
 0001:0029e390       _drft_init                 0069f390 f   libvorbis:smallft.o
 0001:0029e620       _drft_clear                0069f620 f   libvorbis:smallft.o
 0001:0029e670       __vorbis_window_get        0069f670 f   libvorbis:window.o
 0001:0029e680       __vorbis_apply_window      0069f680 f   libvorbis:window.o
 0001:0029fa00       _res0_free_info            006a0a00 f   libvorbis:res0.o
 0001:0029fa20       _res0_pack                 006a0a20 f   libvorbis:res0.o
 0001:0029fbb0       _res0_look                 006a0bb0 f   libvorbis:res0.o
 0001:0029fe20       _res1_class                006a0e20 f   libvorbis:res0.o
 0001:002a0090       _res2_class                006a1090 f   libvorbis:res0.o
 0001:002a04f0       _res0_inverse              006a14f0 f   libvorbis:res0.o
 0001:002a0570       _res1_inverse              006a1570 f   libvorbis:res0.o
 0001:002a10b0       _res2_inverse              006a20b0 f   libvorbis:res0.o
 0001:002a12d0       _res0_free_look            006a22d0 f   libvorbis:res0.o
 0001:002a1690       _res2_forward              006a2690 f   libvorbis:res0.o
 0001:002a1760       _res1_forward              006a2760 f   libvorbis:res0.o
 0001:002a17e0       _res0_unpack               006a27e0 f   libvorbis:res0.o
 0001:002a32b0       _floor1_fit                006a42b0 f   libvorbis:floor1.o
 0001:002a3c20       _floor1_interpolate_fit    006a4c20 f   libvorbis:floor1.o
 0001:002a3cd0       _floor1_encode             006a4cd0 f   libvorbis:floor1.o
 0001:002a4db0       _vorbis_lsp_to_curve       006a5db0 f   libvorbis:lsp.o
 0001:002a4fc0       _vorbis_lpc_to_lsp         006a5fc0 f   libvorbis:lsp.o
 0001:002a54a0       __getcwd                   006a64a0 f   msvcrtd:MSVCR100D.dll
 0001:002a54a0       _getcwd                    006a64a0 f   msvcrtd:MSVCR100D.dll
 0001:002a54a6       __mkdir                    006a64a6 f   msvcrtd:MSVCR100D.dll
 0001:002a54a6       _mkdir                     006a64a6 f   msvcrtd:MSVCR100D.dll
 0001:002a54ac       _access                    006a64ac f   msvcrtd:MSVCR100D.dll
 0001:002a54ac       __access                   006a64ac f   msvcrtd:MSVCR100D.dll
 0001:002a54b2       _strupr                    006a64b2 f   msvcrtd:MSVCR100D.dll
 0001:002a54b2       __strupr                   006a64b2 f   msvcrtd:MSVCR100D.dll
 0001:002a54b8       _close                     006a64b8 f   msvcrtd:MSVCR100D.dll
 0001:002a54b8       __close                    006a64b8 f   msvcrtd:MSVCR100D.dll
 0001:002a54be       __read                     006a64be f   msvcrtd:MSVCR100D.dll
 0001:002a54be       _read                      006a64be f   msvcrtd:MSVCR100D.dll
 0001:002a54c4       _open                      006a64c4 f   msvcrtd:MSVCR100D.dll
 0001:002a54c4       __open                     006a64c4 f   msvcrtd:MSVCR100D.dll
 0001:002a54ca       _fdopen                    006a64ca f   msvcrtd:MSVCR100D.dll
 0001:002a54ca       __fdopen                   006a64ca f   msvcrtd:MSVCR100D.dll
 0001:002a54d0       __lseek                    006a64d0 f   msvcrtd:MSVCR100D.dll
 0001:002a54d0       _lseek                     006a64d0 f   msvcrtd:MSVCR100D.dll
 0001:002a54d6       __write                    006a64d6 f   msvcrtd:MSVCR100D.dll
 0001:002a54d6       _write                     006a64d6 f   msvcrtd:MSVCR100D.dll
 0001:002a54dc       __unlink                   006a64dc f   msvcrtd:MSVCR100D.dll
 0001:002a54dc       _unlink                    006a64dc f   msvcrtd:MSVCR100D.dll
 0001:002a54e2       __filelength               006a64e2 f   msvcrtd:MSVCR100D.dll
 0001:002a54e2       _filelength                006a64e2 f   msvcrtd:MSVCR100D.dll
 0001:002a54e8       _memchr                    006a64e8 f   msvcrtd:MSVCR100D.dll
 0001:002a54ee       _ldexp                     006a64ee f   msvcrtd:MSVCR100D.dll
 0001:002a54f4       _log                       006a64f4 f   msvcrtd:MSVCR100D.dll
 0001:002a54fa       _ceil                      006a64fa f   msvcrtd:MSVCR100D.dll
 0001:002a5500       _acos                      006a6500 f   msvcrtd:MSVCR100D.dll
 0001:002a5510       _oggpack_writeinit         006a6510 f   libogg:bitwise.o
 0001:002a5560       _oggpackB_writeinit        006a6560 f   libogg:bitwise.o
 0001:002a5570       _oggpack_writecheck        006a6570 f   libogg:bitwise.o
 0001:002a5590       _oggpackB_writecheck       006a6590 f   libogg:bitwise.o
 0001:002a55b0       _oggpack_writetrunc        006a65b0 f   libogg:bitwise.o
 0001:002a55f0       _oggpackB_writetrunc       006a65f0 f   libogg:bitwise.o
 0001:002a5630       _oggpack_reset             006a6630 f   libogg:bitwise.o
 0001:002a5660       _oggpackB_reset            006a6660 f   libogg:bitwise.o
 0001:002a5690       _oggpack_writeclear        006a6690 f   libogg:bitwise.o
 0001:002a56d0       _oggpack_write             006a66d0 f   libogg:bitwise.o
 0001:002a5800       _oggpack_writealign        006a6800 f   libogg:bitwise.o
 0001:002a5830       _oggpackB_write            006a6830 f   libogg:bitwise.o
 0001:002a5960       _oggpackB_writealign       006a6960 f   libogg:bitwise.o
 0001:002a5ae0       _oggpack_writecopy         006a6ae0 f   libogg:bitwise.o
 0001:002a5b10       _oggpackB_writecopy        006a6b10 f   libogg:bitwise.o
 0001:002a5b40       _oggpackB_writeclear       006a6b40 f   libogg:bitwise.o
 0001:002a5b50       _oggpackB_readinit         006a6b50 f   libogg:bitwise.o
 0001:002a5b80       _oggpack_readinit          006a6b80 f   libogg:bitwise.o
 0001:002a5b90       _oggpack_look              006a6b90 f   libogg:bitwise.o
 0001:002a5c50       _oggpackB_look             006a6c50 f   libogg:bitwise.o
 0001:002a5d10       _oggpack_look1             006a6d10 f   libogg:bitwise.o
 0001:002a5d40       _oggpackB_look1            006a6d40 f   libogg:bitwise.o
 0001:002a5d70       _oggpack_adv               006a6d70 f   libogg:bitwise.o
 0001:002a5dd0       _oggpackB_adv              006a6dd0 f   libogg:bitwise.o
 0001:002a5e30       _oggpack_adv1              006a6e30 f   libogg:bitwise.o
 0001:002a5e60       _oggpackB_adv1             006a6e60 f   libogg:bitwise.o
 0001:002a5e90       _oggpack_read              006a6e90 f   libogg:bitwise.o
 0001:002a5fb0       _oggpackB_read             006a6fb0 f   libogg:bitwise.o
 0001:002a60e0       _oggpack_read1             006a70e0 f   libogg:bitwise.o
 0001:002a6140       _oggpackB_read1            006a7140 f   libogg:bitwise.o
 0001:002a61b0       _oggpack_bits              006a71b0 f   libogg:bitwise.o
 0001:002a61c0       _oggpackB_bytes            006a71c0 f   libogg:bitwise.o
 0001:002a61e0       _oggpack_bytes             006a71e0 f   libogg:bitwise.o
 0001:002a61f0       _oggpackB_bits             006a71f0 f   libogg:bitwise.o
 0001:002a6200       _oggpack_get_buffer        006a7200 f   libogg:bitwise.o
 0001:002a6210       _oggpackB_get_buffer       006a7210 f   libogg:bitwise.o
 0002:00000000       _sethlinesizes             006af000     a.obj
 0002:00000000       _dep_begin                 006af000     a.obj
 0002:000000c0       _prosethlinesizes          006af0c0     a.obj
 0002:00000100       _setvlinebpl               006af100     a.obj
 0002:00000170       _setpalookupaddress        006af170     a.obj
 0002:000001a0       _prosetpalookupaddress     006af1a0     a.obj
 0002:000001b0       _setuphlineasm4            006af1b0     a.obj
 0002:000001f0       _hlineasm4                 006af1f0     a.obj
 0002:000003f0       _prohlineasm4              006af3f0     a.obj
 0002:00000450       _setupvlineasm             006af450     a.obj
 0002:000004b0       _prosetupvlineasm          006af4b0     a.obj
 0002:00000510       _setupmvlineasm            006af510     a.obj
 0002:00000530       _setuptvlineasm            006af530     a.obj
 0002:00000540       _prevlineasm1              006af540     a.obj
 0002:00000580       _vlineasm1                 006af580     a.obj
 0002:000005d0       _vlineasm1nonpow2          006af5d0     a.obj
 0002:00000640       _mvlineasm1                006af640     a.obj
 0002:00000690       _mvlineasm1nonpow2         006af690     a.obj
 0002:00000700       _fixtransluscence          006af700     a.obj
 0002:00000740       _settransnormal            006af740     a.obj
 0002:000007e0       _settransreverse           006af7e0     a.obj
 0002:00000880       _tvlineasm1                006af880     a.obj
 0002:000008f0       _tvlineasm1nonpow2         006af8f0     a.obj
 0002:00000960       _vlineasm4                 006af960     a.obj
 0002:00000b50       _provlineasm4              006afb50     a.obj
 0002:00000d70       _mvlineasm4                006afd70     a.obj
 0002:00001000       _setupspritevline          006b0000     a.obj
 0002:00001050       _spritevline               006b0050     a.obj
 0002:000010b0       _msetupspritevline         006b00b0     a.obj
 0002:00001100       _mspritevline              006b0100     a.obj
 0002:00001160       _tsetupspritevline         006b0160     a.obj
 0002:000011b0       _tspritevline              006b01b0     a.obj
 0002:00001230       _msethlineshift            006b0230     a.obj
 0002:00001260       _mhline                    006b0260     a.obj
 0002:000012d0       _mhlineskipmodify          006b02d0     a.obj
 0002:000013d0       _tsethlineshift            006b03d0     a.obj
 0002:00001400       _thline                    006b0400     a.obj
 0002:00001460       _thlineskipmodify          006b0460     a.obj
 0002:00001560       _setuptvlineasm2           006b0560     a.obj
 0002:000015a0       _tvlineasm2                006b05a0     a.obj
 0002:000016e0       _setupslopevlin2           006b06e0     a.obj
 0002:00001750       _slopevlin2                006b0750     a.obj
 0002:000017d0       _setupslopevlin            006b07d0     a.obj
 0002:00001830       _slopevlin                 006b0830     a.obj
 0002:00001960       _setuprhlineasm4           006b0960     a.obj
 0002:00001a20       _rhlineasm4                006b0a20     a.obj
 0002:00001b60       _setuprmhlineasm4          006b0b60     a.obj
 0002:00001ba0       _rmhlineasm4               006b0ba0     a.obj
 0002:00001c20       _setupqrhlineasm4          006b0c20     a.obj
 0002:00001ca0       _qrhlineasm4               006b0ca0     a.obj
 0002:00001d64       _setupdrawslab             006b0d64     a.obj
 0002:00001dd0       _drawslab                  006b0dd0     a.obj
 0002:00001f8a       _stretchhline              006b0f8a     a.obj
 0002:00002025       _mmxoverlay                006b1025     a.obj
 0002:0000212d       _dep_end                   006b112d     a.obj
 0003:00000000       __imp__RegOpenKeyExA@20    006b2000     advapi32:ADVAPI32.dll
 0003:00000004       __imp__RegCloseKey@4       006b2004     advapi32:ADVAPI32.dll
 0003:00000008       \177ADVAPI32_NULL_THUNK_DATA 006b2008     advapi32:ADVAPI32.dll
 0003:0000000c       __imp__InitCommonControlsEx@4 006b200c     comctl32:COMCTL32.dll
 0003:00000010       \177COMCTL32_NULL_THUNK_DATA 006b2010     comctl32:COMCTL32.dll
 0003:00000014       __imp__DirectSoundCreate@12 006b2014     dsound:DSOUND.dll
 0003:00000018       \177DSOUND_NULL_THUNK_DATA 006b2018     dsound:DSOUND.dll
 0003:0000001c       __imp__GetTextMetricsW@8   006b201c     gdi32:GDI32.dll
 0003:00000020       __imp__CreateFontIndirectW@4 006b2020     gdi32:GDI32.dll
 0003:00000024       __imp__GetPixelFormat@4    006b2024     gdi32:GDI32.dll
 0003:00000028       __imp__SwapBuffers@4       006b2028     gdi32:GDI32.dll
 0003:0000002c       __imp__DescribePixelFormat@16 006b202c     gdi32:GDI32.dll
 0003:00000030       __imp__SetPixelFormat@12   006b2030     gdi32:GDI32.dll
 0003:00000034       __imp__ChoosePixelFormat@8 006b2034     gdi32:GDI32.dll
 0003:00000038       __imp__BitBlt@36           006b2038     gdi32:GDI32.dll
 0003:0000003c       __imp__GetDIBits@28        006b203c     gdi32:GDI32.dll
 0003:00000040       __imp__CreateCompatibleBitmap@12 006b2040     gdi32:GDI32.dll
 0003:00000044       __imp__CombineRgn@16       006b2044     gdi32:GDI32.dll
 0003:00000048       __imp__CreateRectRgn@16    006b2048     gdi32:GDI32.dll
 0003:0000004c       __imp__ExtTextOutW@32      006b204c     gdi32:GDI32.dll
 0003:00000050       __imp__SetTextColor@8      006b2050     gdi32:GDI32.dll
 0003:00000054       __imp__Rectangle@20        006b2054     gdi32:GDI32.dll
 0003:00000058       __imp__GetTextExtentPoint32W@16 006b2058     gdi32:GDI32.dll
 0003:0000005c       __imp__SelectObject@8      006b205c     gdi32:GDI32.dll
 0003:00000060       __imp__SetBkMode@8         006b2060     gdi32:GDI32.dll
 0003:00000064       __imp__CreateFontW@56      006b2064     gdi32:GDI32.dll
 0003:00000068       __imp__CreateSolidBrush@4  006b2068     gdi32:GDI32.dll
 0003:0000006c       __imp__CreatePen@12        006b206c     gdi32:GDI32.dll
 0003:00000070       __imp__CreateCompatibleDC@4 006b2070     gdi32:GDI32.dll
 0003:00000074       __imp__GetDeviceGammaRamp@8 006b2074     gdi32:GDI32.dll
 0003:00000078       __imp__DeleteDC@4          006b2078     gdi32:GDI32.dll
 0003:0000007c       __imp__SetDeviceGammaRamp@8 006b207c     gdi32:GDI32.dll
 0003:00000080       __imp__CreateDCW@16        006b2080     gdi32:GDI32.dll
 0003:00000084       __imp__CreateBitmap@20     006b2084     gdi32:GDI32.dll
 0003:00000088       __imp__CreateDIBSection@24 006b2088     gdi32:GDI32.dll
 0003:0000008c       __imp__GetDeviceCaps@8     006b208c     gdi32:GDI32.dll
 0003:00000090       __imp__DeleteObject@4      006b2090     gdi32:GDI32.dll
 0003:00000094       \177GDI32_NULL_THUNK_DATA  006b2094     gdi32:GDI32.dll
 0003:00000098       __imp__ImmGetContext@4     006b2098     imm32:IMM32.dll
 0003:0000009c       __imp__ImmReleaseContext@8 006b209c     imm32:IMM32.dll
 0003:000000a0       __imp__ImmNotifyIME@16     006b20a0     imm32:IMM32.dll
 0003:000000a4       __imp__ImmAssociateContext@8 006b20a4     imm32:IMM32.dll
 0003:000000a8       __imp__ImmSetCompositionStringW@24 006b20a8     imm32:IMM32.dll
 0003:000000ac       __imp__ImmSetCompositionWindow@8 006b20ac     imm32:IMM32.dll
 0003:000000b0       __imp__ImmGetCompositionStringW@16 006b20b0     imm32:IMM32.dll
 0003:000000b4       __imp__ImmGetCandidateListW@16 006b20b4     imm32:IMM32.dll
 0003:000000b8       __imp__ImmGetIMEFileNameA@12 006b20b8     imm32:IMM32.dll
 0003:000000bc       \177IMM32_NULL_THUNK_DATA  006b20bc     imm32:IMM32.dll
 0003:000000c0       __imp__ReleaseSemaphore@12 006b20c0     kernel32:KERNEL32.dll
 0003:000000c4       __imp__CreateSemaphoreW@16 006b20c4     kernel32:KERNEL32.dll
 0003:000000c8       __imp__LeaveCriticalSection@4 006b20c8     kernel32:KERNEL32.dll
 0003:000000cc       __imp__TryEnterCriticalSection@4 006b20cc     kernel32:KERNEL32.dll
 0003:000000d0       __imp__EnterCriticalSection@4 006b20d0     kernel32:KERNEL32.dll
 0003:000000d4       __imp__DeleteCriticalSection@4 006b20d4     kernel32:KERNEL32.dll
 0003:000000d8       __imp__InitializeCriticalSectionAndSpinCount@8 006b20d8     kernel32:KERNEL32.dll
 0003:000000dc       __imp__CreateDirectoryW@8  006b20dc     kernel32:KERNEL32.dll
 0003:000000e0       __imp__lstrcatW@8          006b20e0     kernel32:KERNEL32.dll
 0003:000000e4       __imp__LoadLibraryW@4      006b20e4     kernel32:KERNEL32.dll
 0003:000000e8       __imp__GlobalMemoryStatusEx@4 006b20e8     kernel32:KERNEL32.dll
 0003:000000ec       __imp__GetSystemInfo@4     006b20ec     kernel32:KERNEL32.dll
 0003:000000f0       __imp__ExitProcess@4       006b20f0     kernel32:KERNEL32.dll
 0003:000000f4       __imp__GetTickCount@0      006b20f4     kernel32:KERNEL32.dll
 0003:000000f8       __imp__CreateFileW@28      006b20f8     kernel32:KERNEL32.dll
 0003:000000fc       __imp__SetErrorMode@4      006b20fc     kernel32:KERNEL32.dll
 0003:00000100       __imp__GetFileSizeEx@8     006b2100     kernel32:KERNEL32.dll
 0003:00000104       __imp__SetFilePointerEx@20 006b2104     kernel32:KERNEL32.dll
 0003:00000108       __imp__ReadFile@20         006b2108     kernel32:KERNEL32.dll
 0003:0000010c       __imp__WriteFile@20        006b210c     kernel32:KERNEL32.dll
 0003:00000110       __imp__SetFilePointer@16   006b2110     kernel32:KERNEL32.dll
 0003:00000114       __imp__WriteConsoleW@20    006b2114     kernel32:KERNEL32.dll
 0003:00000118       __imp__lstrlenW@4          006b2118     kernel32:KERNEL32.dll
 0003:0000011c       __imp__GetStdHandle@4      006b211c     kernel32:KERNEL32.dll
 0003:00000120       __imp__AttachConsole@4     006b2120     kernel32:KERNEL32.dll
 0003:00000124       __imp__OutputDebugStringW@4 006b2124     kernel32:KERNEL32.dll
 0003:00000128       __imp__GetModuleHandleW@4  006b2128     kernel32:KERNEL32.dll
 0003:0000012c       __imp__WaitForMultipleObjects@16 006b212c     kernel32:KERNEL32.dll
 0003:00000130       __imp__ReleaseMutex@4      006b2130     kernel32:KERNEL32.dll
 0003:00000134       __imp__ExitThread@4        006b2134     kernel32:KERNEL32.dll
 0003:00000138       __imp__CreateThread@24     006b2138     kernel32:KERNEL32.dll
 0003:0000013c       __imp__SetThreadPriority@8 006b213c     kernel32:KERNEL32.dll
 0003:00000140       __imp__CreateEventA@16     006b2140     kernel32:KERNEL32.dll
 0003:00000144       __imp__CreateMutexA@12     006b2144     kernel32:KERNEL32.dll
 0003:00000148       __imp__SetPriorityClass@8  006b2148     kernel32:KERNEL32.dll
 0003:0000014c       __imp__GetCommandLineA@0   006b214c     kernel32:KERNEL32.dll
 0003:00000150       __imp__FormatMessageA@28   006b2150     kernel32:KERNEL32.dll
 0003:00000154       __imp__VirtualFree@12      006b2154     kernel32:KERNEL32.dll
 0003:00000158       __imp__QueryPerformanceCounter@4 006b2158     kernel32:KERNEL32.dll
 0003:0000015c       __imp__QueryPerformanceFrequency@4 006b215c     kernel32:KERNEL32.dll
 0003:00000160       __imp__WaitForSingleObject@8 006b2160     kernel32:KERNEL32.dll
 0003:00000164       __imp__GetVersionExA@4     006b2164     kernel32:KERNEL32.dll
 0003:00000168       __imp__FindFirstFileA@8    006b2168     kernel32:KERNEL32.dll
 0003:0000016c       __imp__FindNextFileA@8     006b216c     kernel32:KERNEL32.dll
 0003:00000170       __imp__FindClose@4         006b2170     kernel32:KERNEL32.dll
 0003:00000174       __imp__GetLogicalDrives@0  006b2174     kernel32:KERNEL32.dll
 0003:00000178       __imp__GetModuleHandleA@4  006b2178     kernel32:KERNEL32.dll
 0003:0000017c       __imp__FreeLibrary@4       006b217c     kernel32:KERNEL32.dll
 0003:00000180       __imp__GetShortPathNameA@12 006b2180     kernel32:KERNEL32.dll
 0003:00000184       __imp__GetLongPathNameA@12 006b2184     kernel32:KERNEL32.dll
 0003:00000188       __imp__VirtualProtect@16   006b2188     kernel32:KERNEL32.dll
 0003:0000018c       __imp__LoadLibraryA@4      006b218c     kernel32:KERNEL32.dll
 0003:00000190       __imp__GetProcAddress@8    006b2190     kernel32:KERNEL32.dll
 0003:00000194       __imp__TlsGetValue@4       006b2194     kernel32:KERNEL32.dll
 0003:00000198       __imp__TlsAlloc@0          006b2198     kernel32:KERNEL32.dll
 0003:0000019c       __imp__TlsSetValue@8       006b219c     kernel32:KERNEL32.dll
 0003:000001a0       __imp__CompareStringA@24   006b21a0     kernel32:KERNEL32.dll
 0003:000001a4       __imp__GlobalAlloc@8       006b21a4     kernel32:KERNEL32.dll
 0003:000001a8       __imp__GlobalLock@4        006b21a8     kernel32:KERNEL32.dll
 0003:000001ac       __imp__GlobalUnlock@4      006b21ac     kernel32:KERNEL32.dll
 0003:000001b0       __imp__WideCharToMultiByte@32 006b21b0     kernel32:KERNEL32.dll
 0003:000001b4       __imp__MulDiv@12           006b21b4     kernel32:KERNEL32.dll
 0003:000001b8       __imp__GetSystemPowerStatus@4 006b21b8     kernel32:KERNEL32.dll
 0003:000001bc       __imp__EncodePointer@4     006b21bc     kernel32:KERNEL32.dll
 0003:000001c0       __imp__DecodePointer@4     006b21c0     kernel32:KERNEL32.dll
 0003:000001c4       __imp__InterlockedExchange@8 006b21c4     kernel32:KERNEL32.dll
 0003:000001c8       __imp__HeapSetInformation@16 006b21c8     kernel32:KERNEL32.dll
 0003:000001cc       __imp__GetStartupInfoW@4   006b21cc     kernel32:KERNEL32.dll
 0003:000001d0       __imp__TerminateProcess@8  006b21d0     kernel32:KERNEL32.dll
 0003:000001d4       __imp__UnhandledExceptionFilter@4 006b21d4     kernel32:KERNEL32.dll
 0003:000001d8       __imp__IsDebuggerPresent@0 006b21d8     kernel32:KERNEL32.dll
 0003:000001dc       __imp__IsProcessorFeaturePresent@4 006b21dc     kernel32:KERNEL32.dll
 0003:000001e0       __imp__GetSystemTimeAsFileTime@4 006b21e0     kernel32:KERNEL32.dll
 0003:000001e4       __imp__VirtualQuery@12     006b21e4     kernel32:KERNEL32.dll
 0003:000001e8       __imp__VirtualAlloc@16     006b21e8     kernel32:KERNEL32.dll
 0003:000001ec       __imp__InterlockedCompareExchange@12 006b21ec     kernel32:KERNEL32.dll
 0003:000001f0       __imp__FormatMessageW@28   006b21f0     kernel32:KERNEL32.dll
 0003:000001f4       __imp__SetEnvironmentVariableA@8 006b21f4     kernel32:KERNEL32.dll
 0003:000001f8       __imp__GetEnvironmentVariableA@12 006b21f8     kernel32:KERNEL32.dll
 0003:000001fc       __imp__GetCurrentThread@0  006b21fc     kernel32:KERNEL32.dll
 0003:00000200       __imp__VerSetConditionMask@16 006b2200     kernel32:KERNEL32.dll
 0003:00000204       __imp__VerifyVersionInfoW@16 006b2204     kernel32:KERNEL32.dll
 0003:00000208       __imp__CreateSemaphoreA@16 006b2208     kernel32:KERNEL32.dll
 0003:0000020c       __imp__CreateFileA@28      006b220c     kernel32:KERNEL32.dll
 0003:00000210       __imp__GetCurrentThreadId@0 006b2210     kernel32:KERNEL32.dll
 0003:00000214       __imp__GetCurrentProcessId@0 006b2214     kernel32:KERNEL32.dll
 0003:00000218       __imp__GetCurrentProcess@0 006b2218     kernel32:KERNEL32.dll
 0003:0000021c       __imp__GetLastError@0      006b221c     kernel32:KERNEL32.dll
 0003:00000220       __imp__CloseHandle@4       006b2220     kernel32:KERNEL32.dll
 0003:00000224       __imp__SetUnhandledExceptionFilter@4 006b2224     kernel32:KERNEL32.dll
 0003:00000228       __imp__GetModuleFileNameA@12 006b2228     kernel32:KERNEL32.dll
 0003:0000022c       __imp__Sleep@4             006b222c     kernel32:KERNEL32.dll
 0003:00000230       \177KERNEL32_NULL_THUNK_DATA 006b2230     kernel32:KERNEL32.dll
 0003:00000234       __imp___invoke_watson      006b2234     msvcrtd:MSVCR100D.dll
 0003:00000238       __imp___controlfp_s        006b2238     msvcrtd:MSVCR100D.dll
 0003:0000023c       __imp_?terminate@@YAXXZ    006b223c     msvcrtd:MSVCR100D.dll
 0003:00000240       __imp___except_handler4_common 006b2240     msvcrtd:MSVCR100D.dll
 0003:00000244       __imp___crt_debugger_hook  006b2244     msvcrtd:MSVCR100D.dll
 0003:00000248       __imp___initterm_e         006b2248     msvcrtd:MSVCR100D.dll
 0003:0000024c       __imp___initterm           006b224c     msvcrtd:MSVCR100D.dll
 0003:00000250       __imp___CrtDbgReportW      006b2250     msvcrtd:MSVCR100D.dll
 0003:00000254       __imp___CrtSetCheckCount   006b2254     msvcrtd:MSVCR100D.dll
 0003:00000258       __imp___acmdln             006b2258     msvcrtd:MSVCR100D.dll
 0003:0000025c       __imp___ismbblead          006b225c     msvcrtd:MSVCR100D.dll
 0003:00000260       __imp___cexit              006b2260     msvcrtd:MSVCR100D.dll
 0003:00000264       __imp___XcptFilter         006b2264     msvcrtd:MSVCR100D.dll
 0003:00000268       __imp___exit               006b2268     msvcrtd:MSVCR100D.dll
 0003:0000026c       __imp____getmainargs       006b226c     msvcrtd:MSVCR100D.dll
 0003:00000270       __imp___amsg_exit          006b2270     msvcrtd:MSVCR100D.dll
 0003:00000274       __imp____set_app_type      006b2274     msvcrtd:MSVCR100D.dll
 0003:00000278       __imp___fmode              006b2278     msvcrtd:MSVCR100D.dll
 0003:0000027c       __imp___commode            006b227c     msvcrtd:MSVCR100D.dll
 0003:00000280       __imp____setusermatherr    006b2280     msvcrtd:MSVCR100D.dll
 0003:00000284       __imp___configthreadlocale 006b2284     msvcrtd:MSVCR100D.dll
 0003:00000288       __imp___onexit             006b2288     msvcrtd:MSVCR100D.dll
 0003:0000028c       __imp___lock               006b228c     msvcrtd:MSVCR100D.dll
 0003:00000290       __imp____dllonexit         006b2290     msvcrtd:MSVCR100D.dll
 0003:00000294       __imp___unlock             006b2294     msvcrtd:MSVCR100D.dll
 0003:00000298       __imp__exp                 006b2298     msvcrtd:MSVCR100D.dll
 0003:0000029c       __imp___assert             006b229c     msvcrtd:MSVCR100D.dll
 0003:000002a0       __imp__abort               006b22a0     msvcrtd:MSVCR100D.dll
 0003:000002a4       __imp__atol                006b22a4     msvcrtd:MSVCR100D.dll
 0003:000002a8       __imp__vfprintf            006b22a8     msvcrtd:MSVCR100D.dll
 0003:000002ac       __imp__signal              006b22ac     msvcrtd:MSVCR100D.dll
 0003:000002b0       __imp__vsprintf            006b22b0     msvcrtd:MSVCR100D.dll
 0003:000002b4       __imp__puts                006b22b4     msvcrtd:MSVCR100D.dll
 0003:000002b8       __imp__getchar             006b22b8     msvcrtd:MSVCR100D.dll
 0003:000002bc       __imp___byteswap_uint64    006b22bc     msvcrtd:MSVCR100D.dll
 0003:000002c0       __imp___rotl64             006b22c0     msvcrtd:MSVCR100D.dll
 0003:000002c4       __imp___byteswap_ulong     006b22c4     msvcrtd:MSVCR100D.dll
 0003:000002c8       __imp___rotl               006b22c8     msvcrtd:MSVCR100D.dll
 0003:000002cc       __imp__fputs               006b22cc     msvcrtd:MSVCR100D.dll
 0003:000002d0       __imp___vsnprintf          006b22d0     msvcrtd:MSVCR100D.dll
 0003:000002d4       __imp__strtoul             006b22d4     msvcrtd:MSVCR100D.dll
 0003:000002d8       __imp__tan                 006b22d8     msvcrtd:MSVCR100D.dll
 0003:000002dc       __imp__floor               006b22dc     msvcrtd:MSVCR100D.dll
 0003:000002e0       __imp__cos                 006b22e0     msvcrtd:MSVCR100D.dll
 0003:000002e4       __imp__fabs                006b22e4     msvcrtd:MSVCR100D.dll
 0003:000002e8       __imp___fileno             006b22e8     msvcrtd:MSVCR100D.dll
 0003:000002ec       __imp___lrotl              006b22ec     msvcrtd:MSVCR100D.dll
 0003:000002f0       __imp__fread               006b22f0     msvcrtd:MSVCR100D.dll
 0003:000002f4       __imp__rewind              006b22f4     msvcrtd:MSVCR100D.dll
 0003:000002f8       __imp___setjmp3            006b22f8     msvcrtd:MSVCR100D.dll
 0003:000002fc       __imp__longjmp             006b22fc     msvcrtd:MSVCR100D.dll
 0003:00000300       __imp___unlink             006b2300     msvcrtd:MSVCR100D.dll
 0003:00000304       __imp___filelength         006b2304     msvcrtd:MSVCR100D.dll
 0003:00000308       __imp__pow                 006b2308     msvcrtd:MSVCR100D.dll
 0003:0000030c       __imp__sin                 006b230c     msvcrtd:MSVCR100D.dll
 0003:00000310       __imp__atan                006b2310     msvcrtd:MSVCR100D.dll
 0003:00000314       __imp___findclose          006b2314     msvcrtd:MSVCR100D.dll
 0003:00000318       __imp___findnext64i32      006b2318     msvcrtd:MSVCR100D.dll
 0003:0000031c       __imp___findfirst64i32     006b231c     msvcrtd:MSVCR100D.dll
 0003:00000320       __imp___getdcwd            006b2320     msvcrtd:MSVCR100D.dll
 0003:00000324       __imp__freopen             006b2324     msvcrtd:MSVCR100D.dll
 0003:00000328       __imp___write              006b2328     msvcrtd:MSVCR100D.dll
 0003:0000032c       __imp___lseek              006b232c     msvcrtd:MSVCR100D.dll
 0003:00000330       __imp___fdopen             006b2330     msvcrtd:MSVCR100D.dll
 0003:00000334       __imp___open               006b2334     msvcrtd:MSVCR100D.dll
 0003:00000338       __imp___read               006b2338     msvcrtd:MSVCR100D.dll
 0003:0000033c       __imp___close              006b233c     msvcrtd:MSVCR100D.dll
 0003:00000340       __imp___access             006b2340     msvcrtd:MSVCR100D.dll
 0003:00000344       __imp___mkdir              006b2344     msvcrtd:MSVCR100D.dll
 0003:00000348       __imp___getcwd             006b2348     msvcrtd:MSVCR100D.dll
 0003:0000034c       __imp___strupr             006b234c     msvcrtd:MSVCR100D.dll
 0003:00000350       __imp__setvbuf             006b2350     msvcrtd:MSVCR100D.dll
 0003:00000354       __imp___strnicmp           006b2354     msvcrtd:MSVCR100D.dll
 0003:00000358       __imp__printf              006b2358     msvcrtd:MSVCR100D.dll
 0003:0000035c       __imp__isalpha             006b235c     msvcrtd:MSVCR100D.dll
 0003:00000360       __imp__memchr              006b2360     msvcrtd:MSVCR100D.dll
 0003:00000364       __imp__ldexp               006b2364     msvcrtd:MSVCR100D.dll
 0003:00000368       __imp__log                 006b2368     msvcrtd:MSVCR100D.dll
 0003:0000036c       __imp__ceil                006b236c     msvcrtd:MSVCR100D.dll
 0003:00000370       __imp__free                006b2370     msvcrtd:MSVCR100D.dll
 0003:00000374       __imp__sprintf             006b2374     msvcrtd:MSVCR100D.dll
 0003:00000378       __imp__exit                006b2378     msvcrtd:MSVCR100D.dll
 0003:0000037c       __imp__fflush              006b237c     msvcrtd:MSVCR100D.dll
 0003:00000380       __imp__fclose              006b2380     msvcrtd:MSVCR100D.dll
 0003:00000384       __imp___wassert            006b2384     msvcrtd:MSVCR100D.dll
 0003:00000388       __imp__memcpy              006b2388     msvcrtd:MSVCR100D.dll
 0003:0000038c       __imp__acos                006b238c     msvcrtd:MSVCR100D.dll
 0003:00000390       __imp__memset              006b2390     msvcrtd:MSVCR100D.dll
 0003:00000394       __imp__calloc              006b2394     msvcrtd:MSVCR100D.dll
 0003:00000398       __imp__labs                006b2398     msvcrtd:MSVCR100D.dll
 0003:0000039c       __imp__rand                006b239c     msvcrtd:MSVCR100D.dll
 0003:000003a0       __imp___snprintf           006b23a0     msvcrtd:MSVCR100D.dll
 0003:000003a4       __imp__strncpy             006b23a4     msvcrtd:MSVCR100D.dll
 0003:000003a8       __imp__strlen              006b23a8     msvcrtd:MSVCR100D.dll
 0003:000003ac       __imp__strcat              006b23ac     msvcrtd:MSVCR100D.dll
 0003:000003b0       __imp___stricmp            006b23b0     msvcrtd:MSVCR100D.dll
 0003:000003b4       __imp__realloc             006b23b4     msvcrtd:MSVCR100D.dll
 0003:000003b8       __imp__strrchr             006b23b8     msvcrtd:MSVCR100D.dll
 0003:000003bc       __imp__strcmp              006b23bc     msvcrtd:MSVCR100D.dll
 0003:000003c0       __imp__toupper             006b23c0     msvcrtd:MSVCR100D.dll
 0003:000003c4       __imp__sscanf              006b23c4     msvcrtd:MSVCR100D.dll
 0003:000003c8       __imp__strtok              006b23c8     msvcrtd:MSVCR100D.dll
 0003:000003cc       __imp__strcpy              006b23cc     msvcrtd:MSVCR100D.dll
 0003:000003d0       __imp__fprintf             006b23d0     msvcrtd:MSVCR100D.dll
 0003:000003d4       __imp____iob_func          006b23d4     msvcrtd:MSVCR100D.dll
 0003:000003d8       __imp__atoi                006b23d8     msvcrtd:MSVCR100D.dll
 0003:000003dc       __imp__strtol              006b23dc     msvcrtd:MSVCR100D.dll
 0003:000003e0       __imp___time64             006b23e0     msvcrtd:MSVCR100D.dll
 0003:000003e4       __imp___strdup             006b23e4     msvcrtd:MSVCR100D.dll
 0003:000003e8       __imp__isdigit             006b23e8     msvcrtd:MSVCR100D.dll
 0003:000003ec       __imp__tolower             006b23ec     msvcrtd:MSVCR100D.dll
 0003:000003f0       __imp__malloc              006b23f0     msvcrtd:MSVCR100D.dll
 0003:000003f4       __imp__strchr              006b23f4     msvcrtd:MSVCR100D.dll
 0003:000003f8       __imp___chdir              006b23f8     msvcrtd:MSVCR100D.dll
 0003:000003fc       __imp__memcmp              006b23fc     msvcrtd:MSVCR100D.dll
 0003:00000400       __imp__islower             006b2400     msvcrtd:MSVCR100D.dll
 0003:00000404       __imp__isupper             006b2404     msvcrtd:MSVCR100D.dll
 0003:00000408       __imp__getenv              006b2408     msvcrtd:MSVCR100D.dll
 0003:0000040c       __imp__fopen               006b240c     msvcrtd:MSVCR100D.dll
 0003:00000410       __imp__fwrite              006b2410     msvcrtd:MSVCR100D.dll
 0003:00000414       __imp__perror              006b2414     msvcrtd:MSVCR100D.dll
 0003:00000418       __imp__fseek               006b2418     msvcrtd:MSVCR100D.dll
 0003:0000041c       __imp__strstr              006b241c     msvcrtd:MSVCR100D.dll
 0003:00000420       __imp__strncmp             006b2420     msvcrtd:MSVCR100D.dll
 0003:00000424       __imp__isalnum             006b2424     msvcrtd:MSVCR100D.dll
 0003:00000428       __imp___strtoi64           006b2428     msvcrtd:MSVCR100D.dll
 0003:0000042c       __imp___errno              006b242c     msvcrtd:MSVCR100D.dll
 0003:00000430       __imp___stat64i32          006b2430     msvcrtd:MSVCR100D.dll
 0003:00000434       __imp___localtime64        006b2434     msvcrtd:MSVCR100D.dll
 0003:00000438       __imp___aligned_free       006b2438     msvcrtd:MSVCR100D.dll
 0003:0000043c       __imp__sqrt                006b243c     msvcrtd:MSVCR100D.dll
 0003:00000440       __imp__strncat             006b2440     msvcrtd:MSVCR100D.dll
 0003:00000444       __imp___aligned_malloc     006b2444     msvcrtd:MSVCR100D.dll
 0003:00000448       __imp__qsort               006b2448     msvcrtd:MSVCR100D.dll
 0003:0000044c       __imp__bsearch             006b244c     msvcrtd:MSVCR100D.dll
 0003:00000450       __imp__strerror            006b2450     msvcrtd:MSVCR100D.dll
 0003:00000454       __imp__ftell               006b2454     msvcrtd:MSVCR100D.dll
 0003:00000458       __imp__atof                006b2458     msvcrtd:MSVCR100D.dll
 0003:0000045c       __imp__memmove             006b245c     msvcrtd:MSVCR100D.dll
 0003:00000460       __imp___fstat64i32         006b2460     msvcrtd:MSVCR100D.dll
 0003:00000464       \177MSVCR100D_NULL_THUNK_DATA 006b2464     msvcrtd:MSVCR100D.dll
 0003:00000468       __imp__SysFreeString@4     006b2468     oleaut32:OLEAUT32.dll
 0003:0000046c       \177OLEAUT32_NULL_THUNK_DATA 006b246c     oleaut32:OLEAUT32.dll
 0003:00000470       __imp__DragAcceptFiles@8   006b2470     shell32:SHELL32.dll
 0003:00000474       __imp__DragQueryFileW@16   006b2474     shell32:SHELL32.dll
 0003:00000478       __imp__SHGetFolderPathW@20 006b2478     shell32:SHELL32.dll
 0003:0000047c       __imp__DragFinish@4        006b247c     shell32:SHELL32.dll
 0003:00000480       __imp__ShellExecuteExA@4   006b2480     shell32:SHELL32.dll
 0003:00000484       \177SHELL32_NULL_THUNK_DATA 006b2484     shell32:SHELL32.dll
 0003:00000488       __imp__SHGetValueA@24      006b2488     shlwapi:SHLWAPI.dll
 0003:0000048c       \177SHLWAPI_NULL_THUNK_DATA 006b248c     shlwapi:SHLWAPI.dll
 0003:00000490       __imp__GetSysColorBrush@4  006b2490     user32:USER32.dll
 0003:00000494       __imp__DestroyWindow@4     006b2494     user32:USER32.dll
 0003:00000498       __imp__SetWindowTextA@8    006b2498     user32:USER32.dll
 0003:0000049c       __imp__GetSystemMetrics@4  006b249c     user32:USER32.dll
 0003:000004a0       __imp__SetWindowPos@28     006b24a0     user32:USER32.dll
 0003:000004a4       __imp__ReleaseDC@8         006b24a4     user32:USER32.dll
 0003:000004a8       __imp__GetDC@4             006b24a8     user32:USER32.dll
 0003:000004ac       __imp__MoveWindow@24       006b24ac     user32:USER32.dll
 0003:000004b0       __imp__GetClientRect@8     006b24b0     user32:USER32.dll
 0003:000004b4       __imp__LoadBitmapA@8       006b24b4     user32:USER32.dll
 0003:000004b8       __imp__GetWindowRect@8     006b24b8     user32:USER32.dll
 0003:000004bc       __imp__AdjustWindowRect@12 006b24bc     user32:USER32.dll
 0003:000004c0       __imp__GetWindowLongA@8    006b24c0     user32:USER32.dll
 0003:000004c4       __imp__IsDlgButtonChecked@8 006b24c4     user32:USER32.dll
 0003:000004c8       __imp__IsDialogMessageA@8  006b24c8     user32:USER32.dll
 0003:000004cc       __imp__IsWindow@4          006b24cc     user32:USER32.dll
 0003:000004d0       __imp__DispatchMessageA@4  006b24d0     user32:USER32.dll
 0003:000004d4       __imp__TranslateMessage@4  006b24d4     user32:USER32.dll
 0003:000004d8       __imp__GetMessageA@16      006b24d8     user32:USER32.dll
 0003:000004dc       __imp__MessageBoxA@16      006b24dc     user32:USER32.dll
 0003:000004e0       __imp__RegisterHotKey@16   006b24e0     user32:USER32.dll
 0003:000004e4       __imp__UnregisterHotKey@8  006b24e4     user32:USER32.dll
 0003:000004e8       __imp__wsprintfA           006b24e8     user32:USER32.dll
 0003:000004ec       __imp__GetKeyboardLayoutNameA@4 006b24ec     user32:USER32.dll
 0003:000004f0       __imp__LoadKeyboardLayoutA@8 006b24f0     user32:USER32.dll
 0003:000004f4       __imp__DefWindowProcW@16   006b24f4     user32:USER32.dll
 0003:000004f8       __imp__EnableWindow@8      006b24f8     user32:USER32.dll
 0003:000004fc       __imp__CreateWindowExW@48  006b24fc     user32:USER32.dll
 0003:00000500       __imp__RegisterDeviceNotificationW@12 006b2500     user32:USER32.dll
 0003:00000504       __imp__PeekMessageW@20     006b2504     user32:USER32.dll
 0003:00000508       __imp__GetMessageW@16      006b2508     user32:USER32.dll
 0003:0000050c       __imp__UnregisterDeviceNotification@4 006b250c     user32:USER32.dll
 0003:00000510       __imp__UnregisterClassW@8  006b2510     user32:USER32.dll
 0003:00000514       __imp__DispatchMessageW@4  006b2514     user32:USER32.dll
 0003:00000518       __imp__GetAsyncKeyState@4  006b2518     user32:USER32.dll
 0003:0000051c       __imp__GetPropW@8          006b251c     user32:USER32.dll
 0003:00000520       __imp__IsRectEmpty@4       006b2520     user32:USER32.dll
 0003:00000524       __imp__ClientToScreen@8    006b2524     user32:USER32.dll
 0003:00000528       __imp__CallWindowProcW@20  006b2528     user32:USER32.dll
 0003:0000052c       __imp__GetMessageExtraInfo@0 006b252c     user32:USER32.dll
 0003:00000530       __imp__ClipCursor@4        006b2530     user32:USER32.dll
 0003:00000534       __imp__GetRawInputData@20  006b2534     user32:USER32.dll
 0003:00000538       __imp__GetCursorPos@4      006b2538     user32:USER32.dll
 0003:0000053c       __imp__WindowFromPoint@8   006b253c     user32:USER32.dll
 0003:00000540       __imp__ScreenToClient@8    006b2540     user32:USER32.dll
 0003:00000544       __imp__GetUpdateRect@12    006b2544     user32:USER32.dll
 0003:00000548       __imp__ValidateRect@8      006b2548     user32:USER32.dll
 0003:0000054c       __imp__GetWindowLongW@8    006b254c     user32:USER32.dll
 0003:00000550       __imp__AdjustWindowRectEx@16 006b2550     user32:USER32.dll
 0003:00000554       __imp__IsIconic@4          006b2554     user32:USER32.dll
 0003:00000558       __imp__SetCursor@4         006b2558     user32:USER32.dll
 0003:0000055c       __imp__GetKeyState@4       006b255c     user32:USER32.dll
 0003:00000560       __imp__GetMenu@4           006b2560     user32:USER32.dll
 0003:00000564       __imp__LoadImageW@24       006b2564     user32:USER32.dll
 0003:00000568       __imp__RegisterClassW@4    006b2568     user32:USER32.dll
 0003:0000056c       __imp__GetClassInfoW@12    006b256c     user32:USER32.dll
 0003:00000570       __imp__GetRawInputDeviceInfoA@16 006b2570     user32:USER32.dll
 0003:00000574       __imp__GetDlgItem@8        006b2574     user32:USER32.dll
 0003:00000578       __imp__SendMessageA@16     006b2578     user32:USER32.dll
 0003:0000057c       __imp__ShowWindow@8        006b257c     user32:USER32.dll
 0003:00000580       __imp__SetFocus@4          006b2580     user32:USER32.dll
 0003:00000584       __imp__RegisterClassExW@4  006b2584     user32:USER32.dll
 0003:00000588       __imp__GetClipboardSequenceNumber@0 006b2588     user32:USER32.dll
 0003:0000058c       __imp__DialogBoxIndirectParamW@20 006b258c     user32:USER32.dll
 0003:00000590       __imp__SystemParametersInfoA@16 006b2590     user32:USER32.dll
 0003:00000594       __imp__DrawTextW@20        006b2594     user32:USER32.dll
 0003:00000598       __imp__SystemParametersInfoW@16 006b2598     user32:USER32.dll
 0003:0000059c       __imp__EndDialog@8         006b259c     user32:USER32.dll
 0003:000005a0       __imp__GetDesktopWindow@0  006b25a0     user32:USER32.dll
 0003:000005a4       __imp__ChangeDisplaySettingsExW@20 006b25a4     user32:USER32.dll
 0003:000005a8       __imp__EnumDisplayDevicesW@16 006b25a8     user32:USER32.dll
 0003:000005ac       __imp__EnumDisplayMonitors@16 006b25ac     user32:USER32.dll
 0003:000005b0       __imp__EnumDisplaySettingsW@12 006b25b0     user32:USER32.dll
 0003:000005b4       __imp__GetClipboardData@4  006b25b4     user32:USER32.dll
 0003:000005b8       __imp__IsClipboardFormatAvailable@4 006b25b8     user32:USER32.dll
 0003:000005bc       __imp__CloseClipboard@0    006b25bc     user32:USER32.dll
 0003:000005c0       __imp__CreateDialogParamA@20 006b25c0     user32:USER32.dll
 0003:000005c4       __imp__SetClipboardData@8  006b25c4     user32:USER32.dll
 0003:000005c8       __imp__EmptyClipboard@0    006b25c8     user32:USER32.dll
 0003:000005cc       __imp__OpenClipboard@4     006b25cc     user32:USER32.dll
 0003:000005d0       __imp__SetWindowRgn@12     006b25d0     user32:USER32.dll
 0003:000005d4       __imp__MapVirtualKeyW@8    006b25d4     user32:USER32.dll
 0003:000005d8       __imp__GetKeyboardLayout@4 006b25d8     user32:USER32.dll
 0003:000005dc       __imp__TrackMouseEvent@4   006b25dc     user32:USER32.dll
 0003:000005e0       __imp__RemovePropW@8       006b25e0     user32:USER32.dll
 0003:000005e4       __imp__SendMessageW@16     006b25e4     user32:USER32.dll
 0003:000005e8       __imp__CreateIconFromResource@16 006b25e8     user32:USER32.dll
 0003:000005ec       __imp__SetWindowTextW@8    006b25ec     user32:USER32.dll
 0003:000005f0       __imp__GetWindowTextW@12   006b25f0     user32:USER32.dll
 0003:000005f4       __imp__GetWindowTextLengthW@4 006b25f4     user32:USER32.dll
 0003:000005f8       __imp__GetFocus@0          006b25f8     user32:USER32.dll
 0003:000005fc       __imp__SetWindowLongW@12   006b25fc     user32:USER32.dll
 0003:00000600       __imp__SetPropW@12         006b2600     user32:USER32.dll
 0003:00000604       __imp__GetDoubleClickTime@0 006b2604     user32:USER32.dll
 0003:00000608       __imp__RegisterRawInputDevices@12 006b2608     user32:USER32.dll
 0003:0000060c       __imp__CreateIconIndirect@4 006b260c     user32:USER32.dll
 0003:00000610       __imp__LoadCursorW@8       006b2610     user32:USER32.dll
 0003:00000614       __imp__DestroyIcon@4       006b2614     user32:USER32.dll
 0003:00000618       __imp__SetCursorPos@8      006b2618     user32:USER32.dll
 0003:0000061c       __imp__GetRawInputDeviceList@12 006b261c     user32:USER32.dll
 0003:00000620       \177USER32_NULL_THUNK_DATA 006b2620     user32:USER32.dll
 0003:00000624       __imp__GetFileVersionInfoA@16 006b2624     version:VERSION.dll
 0003:00000628       __imp__VerQueryValueA@16   006b2628     version:VERSION.dll
 0003:0000062c       __imp__GetFileVersionInfoSizeA@8 006b262c     version:VERSION.dll
 0003:00000630       \177VERSION_NULL_THUNK_DATA 006b2630     version:VERSION.dll
 0003:00000634       __imp__midiStreamPause@4   006b2634     winmm:WINMM.dll
 0003:00000638       __imp__midiOutUnprepareHeader@12 006b2638     winmm:WINMM.dll
 0003:0000063c       __imp__midiStreamClose@4   006b263c     winmm:WINMM.dll
 0003:00000640       __imp__midiStreamStop@4    006b2640     winmm:WINMM.dll
 0003:00000644       __imp__midiStreamOpen@24   006b2644     winmm:WINMM.dll
 0003:00000648       __imp__midiOutGetDevCapsA@12 006b2648     winmm:WINMM.dll
 0003:0000064c       __imp__midiStreamProperty@12 006b264c     winmm:WINMM.dll
 0003:00000650       __imp__timeBeginPeriod@4   006b2650     winmm:WINMM.dll
 0003:00000654       __imp__timeEndPeriod@4     006b2654     winmm:WINMM.dll
 0003:00000658       __imp__waveOutUnprepareHeader@12 006b2658     winmm:WINMM.dll
 0003:0000065c       __imp__midiStreamRestart@4 006b265c     winmm:WINMM.dll
 0003:00000660       __imp__waveOutClose@4      006b2660     winmm:WINMM.dll
 0003:00000664       __imp__waveOutWrite@12     006b2664     winmm:WINMM.dll
 0003:00000668       __imp__waveOutGetErrorTextW@12 006b2668     winmm:WINMM.dll
 0003:0000066c       __imp__waveOutOpen@24      006b266c     winmm:WINMM.dll
 0003:00000670       __imp__waveOutPrepareHeader@12 006b2670     winmm:WINMM.dll
 0003:00000674       __imp__waveInOpen@24       006b2674     winmm:WINMM.dll
 0003:00000678       __imp__waveInGetNumDevs@0  006b2678     winmm:WINMM.dll
 0003:0000067c       __imp__waveInGetDevCapsW@12 006b267c     winmm:WINMM.dll
 0003:00000680       __imp__waveOutGetNumDevs@0 006b2680     winmm:WINMM.dll
 0003:00000684       __imp__waveOutGetDevCapsW@12 006b2684     winmm:WINMM.dll
 0003:00000688       __imp__midiOutPrepareHeader@12 006b2688     winmm:WINMM.dll
 0003:0000068c       __imp__midiStreamOut@12    006b268c     winmm:WINMM.dll
 0003:00000690       __imp__waveInClose@4       006b2690     winmm:WINMM.dll
 0003:00000694       __imp__timeGetTime@0       006b2694     winmm:WINMM.dll
 0003:00000698       \177WINMM_NULL_THUNK_DATA  006b2698     winmm:WINMM.dll
 0003:0000069c       __imp__socket@12           006b269c     ws2_32:WS2_32.dll
 0003:000006a0       __imp__connect@12          006b26a0     ws2_32:WS2_32.dll
 0003:000006a4       __imp__gethostbyname@4     006b26a4     ws2_32:WS2_32.dll
 0003:000006a8       __imp__WSAStartup@8        006b26a8     ws2_32:WS2_32.dll
 0003:000006ac       __imp__htonl@4             006b26ac     ws2_32:WS2_32.dll
 0003:000006b0       __imp__ntohl@4             006b26b0     ws2_32:WS2_32.dll
 0003:000006b4       __imp__ntohs@4             006b26b4     ws2_32:WS2_32.dll
 0003:000006b8       __imp__WSACleanup@0        006b26b8     ws2_32:WS2_32.dll
 0003:000006bc       __imp__inet_addr@4         006b26bc     ws2_32:WS2_32.dll
 0003:000006c0       __imp__inet_ntoa@4         006b26c0     ws2_32:WS2_32.dll
 0003:000006c4       __imp__gethostbyaddr@12    006b26c4     ws2_32:WS2_32.dll
 0003:000006c8       __imp__bind@12             006b26c8     ws2_32:WS2_32.dll
 0003:000006cc       __imp__getsockname@12      006b26cc     ws2_32:WS2_32.dll
 0003:000006d0       __imp__listen@8            006b26d0     ws2_32:WS2_32.dll
 0003:000006d4       __imp__setsockopt@20       006b26d4     ws2_32:WS2_32.dll
 0003:000006d8       __imp__ioctlsocket@12      006b26d8     ws2_32:WS2_32.dll
 0003:000006dc       __imp__getsockopt@20       006b26dc     ws2_32:WS2_32.dll
 0003:000006e0       __imp__WSAGetLastError@0   006b26e0     ws2_32:WS2_32.dll
 0003:000006e4       __imp__accept@12           006b26e4     ws2_32:WS2_32.dll
 0003:000006e8       __imp__shutdown@8          006b26e8     ws2_32:WS2_32.dll
 0003:000006ec       __imp__WSASendTo@36        006b26ec     ws2_32:WS2_32.dll
 0003:000006f0       __imp__WSARecvFrom@36      006b26f0     ws2_32:WS2_32.dll
 0003:000006f4       __imp__select@20           006b26f4     ws2_32:WS2_32.dll
 0003:000006f8       __imp____WSAFDIsSet@8      006b26f8     ws2_32:WS2_32.dll
 0003:000006fc       __imp__closesocket@4       006b26fc     ws2_32:WS2_32.dll
 0003:00000700       __imp__recv@16             006b2700     ws2_32:WS2_32.dll
 0003:00000704       __imp__send@16             006b2704     ws2_32:WS2_32.dll
 0003:00000708       __imp__htons@4             006b2708     ws2_32:WS2_32.dll
 0003:0000070c       \177WS2_32_NULL_THUNK_DATA 006b270c     ws2_32:WS2_32.dll
 0003:00000710       __imp__CoUninitialize@0    006b2710     ole32:ole32.dll
 0003:00000714       __imp__CoInitializeEx@8    006b2714     ole32:ole32.dll
 0003:00000718       __imp__CoCreateInstance@20 006b2718     ole32:ole32.dll
 0003:0000071c       \177ole32_NULL_THUNK_DATA  006b271c     ole32:ole32.dll
 0003:00000720       ___xc_a                    006b2720     msvcrtd:cinitexe.obj
 0003:00000748       ___xc_z                    006b2748     msvcrtd:cinitexe.obj
 0003:0000074c       ___xi_a                    006b274c     msvcrtd:cinitexe.obj
 0003:0000075c       ___xi_z                    006b275c     msvcrtd:cinitexe.obj
 0003:000036c0       __real@40f0000000000000    006b56c0     game.obj
 0003:00003d50       __real@3fa0e5604189374c    006b5d50     actors.obj
 0003:00003d58       __real@3feef1a9fbe76c8b    006b5d58     actors.obj
 0003:00003d68       __real@3fe8000000000000    006b5d68     actors.obj
 0003:000050b8       __real@0000000000000000    006b70b8     animvpx.obj
 0003:000050c0       __real@bf800000            006b70c0     animvpx.obj
 0003:00005508       _CheatFunctionFlags        006b7508     cheats.obj
 0003:00005574       _CheatFunctionIDs          006b7574     cheats.obj
 0003:0000558c       ?g_NAMMattCheatQuote@@3QBDB 006b758c     cheats.obj
 0003:00005d58       __real@3ff5555560000000    006b7d58     sbar.obj
 0003:000076c8       __real@4059000000000000    006b96c8     demo.obj
 0003:000076d0       __real@408f400000000000    006b96d0     demo.obj
 0003:00009b90       _SectorLabels              006bbb90     gamedef.obj
 0003:00009e40       _WallLabels                006bbe40     gamedef.obj
 0003:0000a180       _ActorLabels               006bc180     gamedef.obj
 0003:0000a638       _TsprLabels                006bc638     gamedef.obj
 0003:0000af38       _PlayerLabels              006bcf38     gamedef.obj
 0003:0000b9b8       _ProjectileLabels          006bd9b8     gamedef.obj
 0003:0000c0f8       _UserdefsLabels            006be0f8     gamedef.obj
 0003:0000c818       _InputLabels               006be818     gamedef.obj
 0003:0000c8d8       _TileDataLabels            006be8d8     gamedef.obj
 0003:0000c974       _PalDataLabels             006be974     gamedef.obj
 0003:0000ca48       _iter_tokens               006bea48     gamedef.obj
 0003:00012f10       __real@3f70101020000000    006c4f10     gamevars.obj
 0003:00012f18       __real@406fe00000000000    006c4f18     gamevars.obj
 0003:000132c4       _g_player                  006c52c4     global.obj
 0003:00015a68       __real@3ff0000000000000    006c7a68     menus.obj
 0003:00015a70       __real@41700000            006c7a70     menus.obj
 0003:00015a78       __real@402e000000000000    006c7a78     menus.obj
 0003:00015a80       __real@4024000000000000    006c7a80     menus.obj
 0003:0001ae58       _oldkeydefaults            006cce58     config.obj
 0003:0001d17c       __real@40e00000            006cf17c     config.obj
 0003:0001d620       __real@47800000            006cf620     osdfuncs.obj
 0003:0001d624       __real@3f2b851f            006cf624     osdfuncs.obj
 0003:0001e098       _ConsoleKeys               006d0098     osdcmds.obj
 0003:0001e420       _ConsoleButtons            006d0420     osdcmds.obj
 0003:000200c8       __real@43800000            006d20c8     osdcmds.obj
 0003:00021b10       __real@4010000000000000    006d3b10     control.obj
 0003:00021b18       __real@4000000000000000    006d3b18     control.obj
 0003:000246c0       __real@40200000            006d66c0     baselayer.obj
 0003:000246c4       __real@c0200000            006d66c4     baselayer.obj
 0003:00024e28       __real@4090000000000000    006d6e28     cache1d.obj
 0003:00027f28       __real@bff0000000000000    006d9f28     defs.obj
 0003:00028210       __real@3fb99999a0000000    006da210     defs.obj
 0003:00028280       __real@4050624dd2f1a9fc    006da280     defs.obj
 0003:000288f4       _pow2char                  006da8f4     engine.obj
 0003:00028a68       _pow2long                  006daa68     engine.obj
 0003:0002a8d8       __real@c0d45f3060000000    006dc8d8     engine.obj
 0003:0002a8e0       __real@3f799999a0000000    006dc8e0     engine.obj
 0003:0002a8e8       __real@3fe0000000000000    006dc8e8     engine.obj
 0003:0002a8f0       __real@40d0000000000000    006dc8f0     engine.obj
 0003:0002a8f8       __real@3f6921fb60000000    006dc8f8     engine.obj
 0003:0002a900       __real@437f0000            006dc900     engine.obj
 0003:0002a908       __real@4020000000000000    006dc908     engine.obj
 0003:0002a918       __real@4008000000000000    006dc918     engine.obj
 0003:0002a920       __real@4350000000000000    006dc920     engine.obj
 0003:0002a928       __real@3f699999a0000000    006dc928     engine.obj
 0003:0002a930       __real@4120000000000000    006dc930     engine.obj
 0003:0002a938       __real@3fe51eb860000000    006dc938     engine.obj
 0003:0002a940       __real@3fd51eb860000000    006dc940     engine.obj
 0003:0002a948       __real@3f28f5c3            006dc948     engine.obj
 0003:0002a94c       __real@3ea8f5c3            006dc94c     engine.obj
 0003:0002a950       __real@3f30000000000000    006dc950     engine.obj
 0003:0002ea6c       __real@3d800000            006e0a6c     polymost.obj
 0003:0002ea70       __real@72177617            006e0a70     polymost.obj
 0003:0002ea74       __real@7212699f            006e0a74     polymost.obj
 0003:0002ea78       __real@46424d33e0000000    006e0a78     polymost.obj
 0003:0002ea80       __real@f212699f            006e0a80     polymost.obj
 0003:0002ea84       __real@42c80000            006e0a84     polymost.obj
 0003:0002ea88       __real@3a83126f            006e0a88     polymost.obj
 0003:0002ea90       __real@3f50624de0000000    006e0a90     polymost.obj
 0003:0002ea98       __real@400c000000000000    006e0a98     polymost.obj
 0003:0002eaa0       __real@3fecccccc0000000    006e0aa0     polymost.obj
 0003:0002eaa8       __real@3fbc28f5c28f5c29    006e0aa8     polymost.obj
 0003:0002eab0       __real@3fe2e147ae147ae1    006e0ab0     polymost.obj
 0003:0002eab8       __real@3fd3333333333333    006e0ab8     polymost.obj
 0003:0002eac0       __real@3f90000000000000    006e0ac0     polymost.obj
 0003:0002eac8       __real@40000000            006e0ac8     polymost.obj
 0003:0002eacc       __real@44408000            006e0acc     polymost.obj
 0003:0002ead0       __real@45f00800            006e0ad0     polymost.obj
 0003:0002ead4       __real@45b81000            006e0ad4     polymost.obj
 0003:0002ead8       __real@44400000            006e0ad8     polymost.obj
 0003:0002eadc       __real@47057800            006e0adc     polymost.obj
 0003:0002eae0       __real@46040000            006e0ae0     polymost.obj
 0003:0002eae4       __real@47057000            006e0ae4     polymost.obj
 0003:0002eae8       __real@4440c000            006e0ae8     polymost.obj
 0003:0002eaec       __real@47057500            006e0aec     polymost.obj
 0003:0002eaf0       __real@40a9000000000000    006e0af0     polymost.obj
 0003:0002eaf8       __real@4030000000000000    006e0af8     polymost.obj
 0003:0002eb00       __real@3ff0ccccc0000000    006e0b00     polymost.obj
 0003:0002eb08       __real@749dc5ae            006e0b08     polymost.obj
 0003:0002eb0c       __real@f49dc5ae            006e0b0c     polymost.obj
 0003:0002eb10       __real@4070400000000000    006e0b10     polymost.obj
 0003:0002eb18       __real@3f1421f600000000    006e0b18     polymost.obj
 0003:0002eb20       __real@3ef0000000000000    006e0b20     polymost.obj
 0003:0002eb28       __real@3ed0000000000000    006e0b28     polymost.obj
 0003:0002eb30       __real@3e60000000000000    006e0b30     polymost.obj
 0003:0002eb38       __real@3df4000000000000    006e0b38     polymost.obj
 0003:0002eb40       __real@3ee0000000000000    006e0b40     polymost.obj
 0003:0002eb48       __real@bed0000000000000    006e0b48     polymost.obj
 0003:0002eb50       __real@be90000000000000    006e0b50     polymost.obj
 0003:0002eb58       __real@40a0000000000000    006e0b58     polymost.obj
 0003:0002eb60       __real@3fc0000000000000    006e0b60     polymost.obj
 0003:0002eb68       __real@3f60000000000000    006e0b68     polymost.obj
 0003:0002eb70       __real@bef0000000000000    006e0b70     polymost.obj
 0003:0002eb78       __real@3e90000000000000    006e0b78     polymost.obj
 0003:0002eb80       __real@3e00000000000000    006e0b80     polymost.obj
 0003:0002eb88       __real@c2000000            006e0b88     polymost.obj
 0003:0002eb8c       __real@42000000            006e0b8c     polymost.obj
 0003:0002eb90       __real@40c0000000000000    006e0b90     polymost.obj
 0003:0002eb98       __real@c0c0000000000000    006e0b98     polymost.obj
 0003:0002ebc0       __real@3f40000000000000    006e0bc0     polymost.obj
 0003:0002ebc8       __real@4070000000000000    006e0bc8     polymost.obj
 0003:0002ebd0       __real@3f70000000000000    006e0bd0     polymost.obj
 0003:0002ebd8       __real@3c499999a0000000    006e0bd8     polymost.obj
 0003:0002ebe0       __real@3df0000000000000    006e0be0     polymost.obj
 0003:0002ebe8       __real@3e7ad7f2a0000000    006e0be8     polymost.obj
 0003:0002ebf0       __real@3ba3d70a            006e0bf0     polymost.obj
 0003:0002ebf8       __real@3f847ae140000000    006e0bf8     polymost.obj
 0003:0002ec00       __real@3f50000000000000    006e0c00     polymost.obj
 0003:0002ec08       __real@bfb0000000000000    006e0c08     polymost.obj
 0003:0002ec10       __real@3fb0000000000000    006e0c10     polymost.obj
 0003:0002ec18       __real@3ea0000000000000    006e0c18     polymost.obj
 0003:0002ec20       __real@bfc0000000000000    006e0c20     polymost.obj
 0003:0002ec28       __real@3ff8000000000000    006e0c28     polymost.obj
 0003:0002ec30       __real@c010000000000000    006e0c30     polymost.obj
 0003:0002ec38       __real@bdd0000000000000    006e0c38     polymost.obj
 0003:0002ec40       __real@3f60624de0000000    006e0c40     polymost.obj
 0003:0002ec48       __real@3f2a36e2e0000000    006e0c48     polymost.obj
 0003:0002ec50       __real@3f800347            006e0c50     polymost.obj
 0003:0002ec58       __real@3f4921fb60000000    006e0c58     polymost.obj
 0003:0002ec60       __real@40047ae140000000    006e0c60     polymost.obj
 0003:0002ec68       __real@40c99999a0000000    006e0c68     polymost.obj
 0003:0002ec70       __real@40a4000000000000    006e0c70     polymost.obj
 0003:0002ec78       __real@3e10000000000000    006e0c78     polymost.obj
 0003:0002ec80       __real@3f1a36e2e0000000    006e0c80     polymost.obj
 0003:0002ec88       __real@bfe0000000000000    006e0c88     polymost.obj
 0003:0002ec90       __real@bdf0000000000000    006e0c90     polymost.obj
 0003:0002ec98       __real@3fa0000000000000    006e0c98     polymost.obj
 0003:0002eca0       __real@3d400000            006e0ca0     polymost.obj
 0003:0002eca4       __real@3d000000            006e0ca4     polymost.obj
 0003:0002eca8       __real@3c800000            006e0ca8     polymost.obj
 0003:00032050       __real@4016c16c20000000    006e4050     polymer.obj
 0003:00032058       __real@3fe921fb54442d18    006e4058     polymer.obj
 0003:00032060       __real@4110000000000000    006e4060     polymer.obj
 0003:00032068       __real@4076800000000000    006e4068     polymer.obj
 0003:00032070       __real@c066800000000000    006e4070     polymer.obj
 0003:00032078       __real@4056800000000000    006e4078     polymer.obj
 0003:00032080       __real@7f7fc99e            006e4080     polymer.obj
 0003:000320a0       __real@c000000000000000    006e40a0     polymer.obj
 0003:000320a8       __real@41800000            006e40a8     polymer.obj
 0003:000320ac       __real@41000000            006e40ac     polymer.obj
 0003:000320b0       __real@40cfff8000000000    006e40b0     polymer.obj
 0003:000320b8       __real@40f8724000000000    006e40b8     polymer.obj
 0003:000320c0       __real@40cd4c0000000000    006e40c0     polymer.obj
 0003:000320c8       __real@3fd0000000000000    006e40c8     polymer.obj
 0003:000320d0       __real@3fc99999a0000000    006e40d0     polymer.obj
 0003:000320d8       __real@3e6dfd77            006e40d8     polymer.obj
 0003:000320dc       __real@447a0000            006e40dc     polymer.obj
 0003:000320e0       __real@3f3504f3            006e40e0     polymer.obj
 0003:000320e4       __real@3f9ccccd            006e40e4     polymer.obj
 0003:000320e8       __real@4050000000000000    006e40e8     polymer.obj
 0003:000320f0       __real@c2b40000            006e40f0     polymer.obj
 0003:000320f4       __real@42b40000            006e40f4     polymer.obj
 0003:000320f8       __real@400921fb54442d18    006e40f8     polymer.obj
 0003:00032100       __real@3e800000            006e4100     polymer.obj
 0003:00032104       __real@40a00000            006e4104     polymer.obj
 0003:00032108       __real@41f00000            006e4108     polymer.obj
 0003:00032ce0       __real@40efffe000000000    006e4ce0     mdsprite.obj
 0003:00032ce8       __real@4050800000000000    006e4ce8     mdsprite.obj
 0003:00032cf0       __real@3ef0001000000000    006e4cf0     mdsprite.obj
 0003:00032d00       __real@3f10000000000000    006e4d00     mdsprite.obj
 0003:00032d08       __real@3c23d70a            006e4d08     mdsprite.obj
 0003:00032d10       __real@3f499999a0000000    006e4d10     mdsprite.obj
 0003:00032d18       __real@4124000000000000    006e4d18     mdsprite.obj
 0003:00032d20       __real@3f00000000000000    006e4d20     mdsprite.obj
 0003:00032d28       __real@3eb0000000000000    006e4d28     mdsprite.obj
 0003:00032d30       __real@bf10000000000000    006e4d30     mdsprite.obj
 0003:00032d38       __real@bf50000000000000    006e4d38     mdsprite.obj
 0003:00032d40       __real@4040000000000000    006e4d40     mdsprite.obj
 0003:00032d48       __real@4180000000000000    006e4d48     mdsprite.obj
 0003:00033328       __real@3b800000            006e5328     voxmodel.obj
 0003:00033330       __real@3ff4000000000000    006e5330     voxmodel.obj
 0003:00033338       __real@3fe99999a0000000    006e5338     voxmodel.obj
 0003:00034e68       __real@3fb999999999999a    006e6e68     scriptfile.obj
 0003:00036098       __real@3f000000            006e8098     sdlayer.obj
 0003:000360a0       __real@4060000000000000    006e80a0     sdlayer.obj
 0003:000360a8       __real@405fc00000000000    006e80a8     sdlayer.obj
 0003:000360b0       __real@bf4ccccd            006e80b0     sdlayer.obj
 0003:000360b8       __real@bfe99999a0000000    006e80b8     sdlayer.obj
 0003:000360c0       __real@3f4ccccd            006e80c0     sdlayer.obj
 0003:000360c4       __real@40400000            006e80c4     sdlayer.obj
 0003:000360c8       __real@3dcccccd            006e80c8     sdlayer.obj
 0003:000360cc       __real@40800000            006e80cc     sdlayer.obj
 0003:000364d0       __real@4082c00000000000    006e84d0     pitch.obj
 0003:0003cdf0       _c_dfDIJoystick2           006eedf0     libSDL2:SDL_dinputjoystick.o
 0003:0003e3a0       _sdl_audio_rate_filters    006f03a0     libSDL2:SDL_audiotypecvt.o
 0003:0003fb40       _sdl_audio_type_filters    006f1b40     libSDL2:SDL_audiotypecvt.o
 0003:00046560       _vpx_codec_vp8_dx_algo     006f8560     libvpx:vp8_dx_iface.c.o
 0003:000465c0       _vp8_ctf_maps              006f85c0     libvpx:vp8_dx_iface.c.o
 0003:00046b20       _vp8_rv                    006f8b20     libvpx:postproc.c.o
 0003:00046f10       _vp8_sub_pel_filters       006f8f10     libvpx:filter.c.o
 0003:00046f70       _vp8_bilinear_filters      006f8f70     libvpx:filter.c.o
 0003:00047020       _vp8_small_mvtree          006f9020     libvpx:entropymode.c.o
 0003:0004702e       _vp8_sub_mv_ref_tree       006f902e     libvpx:entropymode.c.o
 0003:00047034       _vp8_mv_ref_tree           006f9034     libvpx:entropymode.c.o
 0003:0004703c       _vp8_mbsplit_tree          006f903c     libvpx:entropymode.c.o
 0003:00047042       _vp8_uv_mode_tree          006f9042     libvpx:entropymode.c.o
 0003:00047048       _vp8_kf_ymode_tree         006f9048     libvpx:entropymode.c.o
 0003:00047050       _vp8_ymode_tree            006f9050     libvpx:entropymode.c.o
 0003:00047058       _vp8_bmode_tree            006f9058     libvpx:entropymode.c.o
 0003:0004706a       _vp8_mbsplit_probs         006f906a     libvpx:entropymode.c.o
 0003:00047070       _vp8_mbsplit_count         006f9070     libvpx:entropymode.c.o
 0003:00047080       _vp8_mbsplits              006f9080     libvpx:entropymode.c.o
 0003:00047180       _vp8_sub_mv_ref_prob2      006f9180     libvpx:entropymode.c.o
 0003:000471a0       _vp8_kf_bmode_prob         006f91a0     libvpx:entropymode.c.o
 0003:00047524       _vp8_bmode_prob            006f9524     libvpx:entropymode.c.o
 0003:0004752d       _vp8_kf_uv_mode_prob       006f952d     libvpx:entropymode.c.o
 0003:00047530       _vp8_uv_mode_prob          006f9530     libvpx:entropymode.c.o
 0003:00047533       _vp8_kf_ymode_prob         006f9533     libvpx:entropymode.c.o
 0003:00047537       _vp8_ymode_prob            006f9537     libvpx:entropymode.c.o
 0003:00047540       _vp8_small_mvencodings     006f9540     libvpx:entropymode.c.o
 0003:00047580       _vp8_sub_mv_ref_encoding_array 006f9580     libvpx:entropymode.c.o
 0003:000475a0       _vp8_mv_ref_encoding_array 006f95a0     libvpx:entropymode.c.o
 0003:000475e0       _vp8_mbsplit_encodings     006f95e0     libvpx:entropymode.c.o
 0003:00047600       _vp8_uv_mode_encodings     006f9600     libvpx:entropymode.c.o
 0003:00047620       _vp8_kf_ymode_encodings    006f9620     libvpx:entropymode.c.o
 0003:00047660       _vp8_ymode_encodings       006f9660     libvpx:entropymode.c.o
 0003:000476a0       _vp8_bmode_encodings       006f96a0     libvpx:entropymode.c.o
 0003:00047b20       _vp8_extra_bits            006f9b20     libvpx:entropy.c.o
 0003:00047c40       _vp8_coef_encodings        006f9c40     libvpx:entropy.c.o
 0003:00047ca0       _vp8_coef_tree             006f9ca0     libvpx:entropy.c.o
 0003:00047cb8       _vp8_mb_feature_data_bits  006f9cb8     libvpx:entropy.c.o
 0003:00047cc0       _vp8_default_zig_zag_mask  006f9cc0     libvpx:entropy.c.o
 0003:00047ce0       _vp8_default_inv_zig_zag   006f9ce0     libvpx:entropy.c.o
 0003:00047d00       _vp8_default_zig_zag1d     006f9d00     libvpx:entropy.c.o
 0003:00047d40       _vp8_prev_token_class      006f9d40     libvpx:entropy.c.o
 0003:00047d50       _vp8_coef_bands            006f9d50     libvpx:entropy.c.o
 0003:00047d60       _vp8_norm                  006f9d60     libvpx:entropy.c.o
 0003:00047e60       _vp8_coef_update_probs     006f9e60     libvpx:entropy.c.o
 0003:00048280       _vp8_default_mv_context    006fa280     libvpx:entropymv.c.o
 0003:000482c0       _vp8_mv_update_probs       006fa2c0     libvpx:entropymv.c.o
 0003:00048700       _vp8_sub_mv_ref_prob3      006fa700     libvpx:decodemv.c.o
 0003:00048800       _vp8_bilinear_filters_x86_8 006fa800     libvpx:filter_x86.c.o
 0003:00048900       _vp8_bilinear_filters_x86_4 006fa900     libvpx:filter_x86.c.o
 0003:00048980       _vp8_mode_contexts         006fa980     libvpx:modecont.c.o
 0003:000489e0       _vp8_mbsplit_offset        006fa9e0     libvpx:findnearmv.c.o
 0003:00048d60       _deflate_copyright         006fad60     libz_mini:deflate.o
 0003:0004aec0       __length_code              006fcec0     libz_mini:trees.o
 0003:0004afc0       __dist_code                006fcfc0     libz_mini:trees.o
 0003:0004b8c0       _z_errmsg                  006fd8c0     libz_mini:zutil.o
 0003:0004b900       ??_C@_1GA@EHAKPACL@?$AAf?$AA?3?$AA?2?$AAd?$AAd?$AA?2?$AAv?$AAc?$AAt?$AAo?$AAo?$AAl?$AAs?$AA?2?$AAc?$AAr?$AAt?$AA_?$AAb?$AAl?$AAd?$AA?2?$AAs?$AAe?$AAl?$AAf?$AA_?$AAx?$AA8?$AA6?$AA?2?$AAc@ 006fd900     msvcrtd:crtexew.obj
 0003:0004b960       ??_C@_1FA@DALEHHGL@?$AA_?$AA_?$AAn?$AAa?$AAt?$AAi?$AAv?$AAe?$AA_?$AAs?$AAt?$AAa?$AAr?$AAt?$AAu?$AAp?$AA_?$AAs?$AAt?$AAa?$AAt?$AAe?$AA?5?$AA?$DN?$AA?$DN?$AA?5?$AA_?$AA_?$AAi?$AAn?$AAi?$AAt@ 006fd960     msvcrtd:crtexew.obj
 0003:0004b9b8       ??_C@_1GE@KOCFNGPB@?$AA_?$AAc?$AAo?$AAn?$AAt?$AAr?$AAo?$AAl?$AAf?$AAp?$AA_?$AAs?$AA?$CI?$AA?$CI?$AA?$CI?$AAv?$AAo?$AAi?$AAd?$AA?5?$AA?$CK?$AA?$CJ?$AA0?$AA?$CJ?$AA?0?$AA?5?$AA0?$AAx?$AA0?$AA0?$AA0?$AA1@ 006fd9b8     msvcrtd:fp8.obj
 0003:0004ba1c       ??_C@_1CK@JMKHCBEI@?$AA_?$AAs?$AAe?$AAt?$AAd?$AAe?$AAf?$AAa?$AAu?$AAl?$AAt?$AAp?$AAr?$AAe?$AAc?$AAi?$AAs?$AAi?$AAo?$AAn?$AA?$AA@ 006fda1c     msvcrtd:fp8.obj
 0003:0004ba48       ??_C@_1GG@PHGJJHBC@?$AAf?$AA?3?$AA?2?$AAd?$AAd?$AA?2?$AAv?$AAc?$AAt?$AAo?$AAo?$AAl?$AAs?$AA?2?$AAc?$AAr?$AAt?$AA_?$AAb?$AAl?$AAd?$AA?2?$AAs?$AAe?$AAl?$AAf?$AA_?$AAx?$AA8?$AA6?$AA?2?$AAc@ 006fda48     msvcrtd:fp8.obj
 0003:0004bf38       __mapping_P                006fdf38     libvorbis:registry.o
 0003:0004bf3c       __residue_P                006fdf3c     libvorbis:registry.o
 0003:0004bf48       __floor_P                  006fdf48     libvorbis:registry.o
 0003:0005a080       _mapping0_exportbundle     0070c080     libvorbis:mapping0.o
 0003:0005a0c0       _residue2_exportbundle     0070c0c0     libvorbis:res0.o
 0003:0005a0e0       _residue1_exportbundle     0070c0e0     libvorbis:res0.o
 0003:0005a100       _residue0_exportbundle     0070c100     libvorbis:res0.o
 0003:0005a140       _floor0_exportbundle       0070c140     libvorbis:floor0.o
 0003:0005a180       _floor1_exportbundle       0070c180     libvorbis:floor1.o
 0003:0005a6e0       _CLSID_DirectDraw          0070c6e0     libSDL2:SDL_windowsjoystick.o
 0003:0005a6f0       _CLSID_DirectDraw7         0070c6f0     libSDL2:SDL_windowsjoystick.o
 0003:0005a700       _CLSID_DirectDrawClipper   0070c700     libSDL2:SDL_windowsjoystick.o
 0003:0005a710       _CLSID_DirectInput         0070c710     libSDL2:SDL_windowsjoystick.o
 0003:0005a720       _CLSID_DirectInput8        0070c720     libSDL2:SDL_windowsjoystick.o
 0003:0005a730       _CLSID_DirectInputDevice   0070c730     libSDL2:SDL_windowsjoystick.o
 0003:0005a740       _CLSID_DirectInputDevice8  0070c740     libSDL2:SDL_windowsjoystick.o
 0003:0005a750       _CLSID_DirectSound         0070c750     libSDL2:SDL_windowsjoystick.o
 0003:0005a760       _CLSID_DirectSound8        0070c760     libSDL2:SDL_windowsjoystick.o
 0003:0005a770       _CLSID_DirectSoundCapture  0070c770     libSDL2:SDL_windowsjoystick.o
 0003:0005a780       _CLSID_DirectSoundCapture8 0070c780     libSDL2:SDL_windowsjoystick.o
 0003:0005a790       _CLSID_DirectSoundFullDuplex 0070c790     libSDL2:SDL_windowsjoystick.o
 0003:0005a7a0       _CLSID_XAudio2             0070c7a0     libSDL2:SDL_xaudio2.o
 0003:0005a7b0       _CLSID_XAudio2_Debug       0070c7b0     libSDL2:SDL_xaudio2.o
 0003:0005a7c0       _DSDEVID_DefaultCapture    0070c7c0     libSDL2:SDL_windowsjoystick.o
 0003:0005a7d0       _DSDEVID_DefaultPlayback   0070c7d0     libSDL2:SDL_windowsjoystick.o
 0003:0005a7e0       _DSDEVID_DefaultVoiceCapture 0070c7e0     libSDL2:SDL_windowsjoystick.o
 0003:0005a7f0       _DSDEVID_DefaultVoicePlayback 0070c7f0     libSDL2:SDL_windowsjoystick.o
 0003:0005a800       _DSDEVID_WinePlayback      0070c800     libSDL2:SDL_windowsjoystick.o
 0003:0005a810       _GUID_Button               0070c810     libSDL2:SDL_windowsjoystick.o
 0003:0005a820       _GUID_ConstantForce        0070c820     libSDL2:SDL_windowsjoystick.o
 0003:0005a830       _GUID_CustomForce          0070c830     libSDL2:SDL_windowsjoystick.o
 0003:0005a840       _GUID_Damper               0070c840     libSDL2:SDL_windowsjoystick.o
 0003:0005a850       _GUID_Friction             0070c850     libSDL2:SDL_windowsjoystick.o
 0003:0005a860       _GUID_Inertia              0070c860     libSDL2:SDL_windowsjoystick.o
 0003:0005a870       _GUID_Joystick             0070c870     libSDL2:SDL_windowsjoystick.o
 0003:0005a880       _GUID_Key                  0070c880     libSDL2:SDL_windowsjoystick.o
 0003:0005a890       _GUID_POV                  0070c890     libSDL2:SDL_windowsjoystick.o
 0003:0005a8a0       _GUID_RampForce            0070c8a0     libSDL2:SDL_windowsjoystick.o
 0003:0005a8b0       _GUID_RxAxis               0070c8b0     libSDL2:SDL_windowsjoystick.o
 0003:0005a8c0       _GUID_RyAxis               0070c8c0     libSDL2:SDL_windowsjoystick.o
 0003:0005a8d0       _GUID_RzAxis               0070c8d0     libSDL2:SDL_windowsjoystick.o
 0003:0005a8e0       _GUID_SawtoothDown         0070c8e0     libSDL2:SDL_windowsjoystick.o
 0003:0005a8f0       _GUID_SawtoothUp           0070c8f0     libSDL2:SDL_windowsjoystick.o
 0003:0005a900       _GUID_Sine                 0070c900     libSDL2:SDL_windowsjoystick.o
 0003:0005a910       _GUID_Slider               0070c910     libSDL2:SDL_windowsjoystick.o
 0003:0005a920       _GUID_Spring               0070c920     libSDL2:SDL_windowsjoystick.o
 0003:0005a930       _GUID_Square               0070c930     libSDL2:SDL_windowsjoystick.o
 0003:0005a940       _GUID_SysKeyboard          0070c940     libSDL2:SDL_windowsjoystick.o
 0003:0005a950       _GUID_SysKeyboardEm        0070c950     libSDL2:SDL_windowsjoystick.o
 0003:0005a960       _GUID_SysKeyboardEm2       0070c960     libSDL2:SDL_windowsjoystick.o
 0003:0005a970       _GUID_SysMouse             0070c970     libSDL2:SDL_windowsjoystick.o
 0003:0005a980       _GUID_SysMouseEm           0070c980     libSDL2:SDL_windowsjoystick.o
 0003:0005a990       _GUID_SysMouseEm2          0070c990     libSDL2:SDL_windowsjoystick.o
 0003:0005a9a0       _GUID_Triangle             0070c9a0     libSDL2:SDL_windowsjoystick.o
 0003:0005a9b0       _GUID_Unknown              0070c9b0     libSDL2:SDL_windowsjoystick.o
 0003:0005a9c0       _GUID_XAxis                0070c9c0     libSDL2:SDL_windowsjoystick.o
 0003:0005a9d0       _GUID_YAxis                0070c9d0     libSDL2:SDL_windowsjoystick.o
 0003:0005a9e0       _GUID_ZAxis                0070c9e0     libSDL2:SDL_windowsjoystick.o
 0003:0005a9f0       _IID_AsyncIUnknown         0070c9f0     libSDL2:SDL_windowsjoystick.o
 0003:0005aa00       _IID_IAdviseSink           0070ca00     libSDL2:SDL_windowsjoystick.o
 0003:0005aa10       _IID_IBindCtx              0070ca10     libSDL2:SDL_windowsjoystick.o
 0003:0005aa20       _IID_IBindStatusCallback   0070ca20     libSDL2:SDL_windowsjoystick.o
 0003:0005aa30       _IID_IBinding              0070ca30     libSDL2:SDL_windowsjoystick.o
 0003:0005aa40       _IID_IClassFactory         0070ca40     libSDL2:SDL_windowsjoystick.o
 0003:0005aa50       _IID_ICreateTypeInfo       0070ca50     libSDL2:SDL_windowsjoystick.o
 0003:0005aa60       _IID_IDataObject           0070ca60     libSDL2:SDL_windowsjoystick.o
 0003:0005aa70       _IID_IDirectDraw           0070ca70     libSDL2:SDL_windowsjoystick.o
 0003:0005aa80       _IID_IDirectDraw2          0070ca80     libSDL2:SDL_windowsjoystick.o
 0003:0005aa90       _IID_IDirectDraw3          0070ca90     libSDL2:SDL_windowsjoystick.o
 0003:0005aaa0       _IID_IDirectDraw4          0070caa0     libSDL2:SDL_windowsjoystick.o
 0003:0005aab0       _IID_IDirectDraw7          0070cab0     libSDL2:SDL_windowsjoystick.o
 0003:0005aac0       _IID_IDirectDrawClipper    0070cac0     libSDL2:SDL_windowsjoystick.o
 0003:0005aad0       _IID_IDirectDrawColorControl 0070cad0     libSDL2:SDL_windowsjoystick.o
 0003:0005aae0       _IID_IDirectDrawGammaControl 0070cae0     libSDL2:SDL_windowsjoystick.o
 0003:0005aaf0       _IID_IDirectDrawPalette    0070caf0     libSDL2:SDL_windowsjoystick.o
 0003:0005ab00       _IID_IDirectDrawSurface    0070cb00     libSDL2:SDL_windowsjoystick.o
 0003:0005ab10       _IID_IDirectDrawSurface2   0070cb10     libSDL2:SDL_windowsjoystick.o
 0003:0005ab20       _IID_IDirectDrawSurface3   0070cb20     libSDL2:SDL_windowsjoystick.o
 0003:0005ab30       _IID_IDirectDrawSurface4   0070cb30     libSDL2:SDL_windowsjoystick.o
 0003:0005ab40       _IID_IDirectDrawSurface7   0070cb40     libSDL2:SDL_windowsjoystick.o
 0003:0005ab50       _IID_IDirectInput2A        0070cb50     libSDL2:SDL_windowsjoystick.o
 0003:0005ab60       _IID_IDirectInput2W        0070cb60     libSDL2:SDL_windowsjoystick.o
 0003:0005ab70       _IID_IDirectInput7A        0070cb70     libSDL2:SDL_windowsjoystick.o
 0003:0005ab80       _IID_IDirectInput7W        0070cb80     libSDL2:SDL_windowsjoystick.o
 0003:0005ab90       _IID_IDirectInput8A        0070cb90     libSDL2:SDL_windowsjoystick.o
 0003:0005aba0       _IID_IDirectInput8W        0070cba0     libSDL2:SDL_windowsjoystick.o
 0003:0005abb0       _IID_IDirectInputA         0070cbb0     libSDL2:SDL_windowsjoystick.o
 0003:0005abc0       _IID_IDirectInputDevice2A  0070cbc0     libSDL2:SDL_windowsjoystick.o
 0003:0005abd0       _IID_IDirectInputDevice2W  0070cbd0     libSDL2:SDL_windowsjoystick.o
 0003:0005abe0       _IID_IDirectInputDevice7A  0070cbe0     libSDL2:SDL_windowsjoystick.o
 0003:0005abf0       _IID_IDirectInputDevice7W  0070cbf0     libSDL2:SDL_windowsjoystick.o
 0003:0005ac00       _IID_IDirectInputDevice8A  0070cc00     libSDL2:SDL_windowsjoystick.o
 0003:0005ac10       _IID_IDirectInputDevice8W  0070cc10     libSDL2:SDL_windowsjoystick.o
 0003:0005ac20       _IID_IDirectInputDeviceA   0070cc20     libSDL2:SDL_windowsjoystick.o
 0003:0005ac30       _IID_IDirectInputDeviceW   0070cc30     libSDL2:SDL_windowsjoystick.o
 0003:0005ac40       _IID_IDirectInputEffect    0070cc40     libSDL2:SDL_windowsjoystick.o
 0003:0005ac50       _IID_IDirectInputW         0070cc50     libSDL2:SDL_windowsjoystick.o
 0003:0005ac60       _IID_IDirectSound          0070cc60     libSDL2:SDL_windowsjoystick.o
 0003:0005ac70       _IID_IDirectSound3DBuffer  0070cc70     libSDL2:SDL_windowsjoystick.o
 0003:0005ac80       _IID_IDirectSound3DListener 0070cc80     libSDL2:SDL_windowsjoystick.o
 0003:0005ac90       _IID_IDirectSound8         0070cc90     libSDL2:SDL_windowsjoystick.o
 0003:0005aca0       _IID_IDirectSoundBuffer    0070cca0     libSDL2:SDL_windowsjoystick.o
 0003:0005acb0       _IID_IDirectSoundBuffer8   0070ccb0     libSDL2:SDL_windowsjoystick.o
 0003:0005acc0       _IID_IDirectSoundCapture   0070ccc0     libSDL2:SDL_windowsjoystick.o
 0003:0005acd0       _IID_IDirectSoundCaptureBuffer 0070ccd0     libSDL2:SDL_windowsjoystick.o
 0003:0005ace0       _IID_IDirectSoundCaptureBuffer8 0070cce0     libSDL2:SDL_windowsjoystick.o
 0003:0005acf0       _IID_IDirectSoundFullDuplex 0070ccf0     libSDL2:SDL_windowsjoystick.o
 0003:0005ad00       _IID_IDirectSoundNotify    0070cd00     libSDL2:SDL_windowsjoystick.o
 0003:0005ad10       _IID_IDispatch             0070cd10     libSDL2:SDL_windowsjoystick.o
 0003:0005ad20       _IID_IEnumFORMATETC        0070cd20     libSDL2:SDL_windowsjoystick.o
 0003:0005ad30       _IID_IEnumMoniker          0070cd30     libSDL2:SDL_windowsjoystick.o
 0003:0005ad40       _IID_IEnumSTATDATA         0070cd40     libSDL2:SDL_windowsjoystick.o
 0003:0005ad50       _IID_IEnumSTATSTG          0070cd50     libSDL2:SDL_windowsjoystick.o
 0003:0005ad60       _IID_IEnumString           0070cd60     libSDL2:SDL_windowsjoystick.o
 0003:0005ad70       _IID_IEnumUnknown          0070cd70     libSDL2:SDL_windowsjoystick.o
 0003:0005ad80       _IID_IEnumVARIANT          0070cd80     libSDL2:SDL_windowsjoystick.o
 0003:0005ad90       _IID_IErrorLog             0070cd90     libSDL2:SDL_windowsjoystick.o
 0003:0005ada0       _IID_IKsPropertySet        0070cda0     libSDL2:SDL_windowsjoystick.o
 0003:0005adb0       _IID_IMoniker              0070cdb0     libSDL2:SDL_windowsjoystick.o
 0003:0005adc0       _IID_IPersist              0070cdc0     libSDL2:SDL_windowsjoystick.o
 0003:0005add0       _IID_IPersistStream        0070cdd0     libSDL2:SDL_windowsjoystick.o
 0003:0005ade0       _IID_IPropertyBag          0070cde0     libSDL2:SDL_windowsjoystick.o
 0003:0005adf0       _IID_IRecordInfo           0070cdf0     libSDL2:SDL_windowsjoystick.o
 0003:0005ae00       _IID_IRunningObjectTable   0070ce00     libSDL2:SDL_windowsjoystick.o
 0003:0005ae10       _IID_ISequentialStream     0070ce10     libSDL2:SDL_windowsjoystick.o
 0003:0005ae20       _IID_IStorage              0070ce20     libSDL2:SDL_windowsjoystick.o
 0003:0005ae30       _IID_IStream               0070ce30     libSDL2:SDL_windowsjoystick.o
 0003:0005ae40       _IID_ITypeComp             0070ce40     libSDL2:SDL_windowsjoystick.o
 0003:0005ae50       _IID_ITypeInfo             0070ce50     libSDL2:SDL_windowsjoystick.o
 0003:0005ae60       _IID_ITypeLib              0070ce60     libSDL2:SDL_windowsjoystick.o
 0003:0005ae70       _IID_IUnknown              0070ce70     libSDL2:SDL_windowsjoystick.o
 0003:0005ae80       _IID_IXAudio2              0070ce80     libSDL2:SDL_xaudio2.o
 0003:0005d064       ___rtc_iaa                 0070f064     msvcrtd:_initsect_.obj
 0003:0005d068       ___rtc_izz                 0070f068     msvcrtd:_initsect_.obj
 0003:0005d06c       ___rtc_taa                 0070f06c     msvcrtd:_initsect_.obj
 0003:0005d070       ___rtc_tzz                 0070f070     msvcrtd:_initsect_.obj
 0003:0005d0d4       __IMPORT_DESCRIPTOR_USER32 0070f0d4     user32:USER32.dll
 0003:0005d0e8       __IMPORT_DESCRIPTOR_GDI32  0070f0e8     gdi32:GDI32.dll
 0003:0005d0fc       __IMPORT_DESCRIPTOR_SHELL32 0070f0fc     shell32:SHELL32.dll
 0003:0005d110       __IMPORT_DESCRIPTOR_WINMM  0070f110     winmm:WINMM.dll
 0003:0005d124       __IMPORT_DESCRIPTOR_WS2_32 0070f124     ws2_32:WS2_32.dll
 0003:0005d138       __IMPORT_DESCRIPTOR_COMCTL32 0070f138     comctl32:COMCTL32.dll
 0003:0005d14c       __IMPORT_DESCRIPTOR_SHLWAPI 0070f14c     shlwapi:SHLWAPI.dll
 0003:0005d160       __IMPORT_DESCRIPTOR_OLEAUT32 0070f160     oleaut32:OLEAUT32.dll
 0003:0005d174       __IMPORT_DESCRIPTOR_ole32  0070f174     ole32:ole32.dll
 0003:0005d188       __IMPORT_DESCRIPTOR_IMM32  0070f188     imm32:IMM32.dll
 0003:0005d19c       __IMPORT_DESCRIPTOR_VERSION 0070f19c     version:VERSION.dll
 0003:0005d1b0       __IMPORT_DESCRIPTOR_DSOUND 0070f1b0     dsound:DSOUND.dll
 0003:0005d1c4       __IMPORT_DESCRIPTOR_ADVAPI32 0070f1c4     advapi32:ADVAPI32.dll
 0003:0005d1d8       __IMPORT_DESCRIPTOR_MSVCR100D 0070f1d8     msvcrtd:MSVCR100D.dll
 0003:0005d1ec       __IMPORT_DESCRIPTOR_KERNEL32 0070f1ec     kernel32:KERNEL32.dll
 0003:0005d200       __NULL_IMPORT_DESCRIPTOR   0070f200     user32:USER32.dll
 0004:00000000       _AppProperName             00712000     game.obj
 0004:00000004       _AppTechnicalName          00712004     game.obj
 0004:00000008       _voting                    00712008     game.obj
 0004:0000000c       _vote_map                  0071200c     game.obj
 0004:00000010       _vote_episode              00712010     game.obj
 0004:00000014       _defaultrtsfilename        00712014     game.obj
 0004:00000028       _hud_showmapname           00712028     game.obj
 0004:0000002c       _CrosshairColors           0071202c     game.obj
 0004:00000038       ?h_dukeanim@@3Uhashtable_t@@A 00712038     anim.obj
 0004:00000040       ?animvpx_read_ivf_header_errmsg@@3PAPBDA 00712040     animvpx.obj
 0004:0000005c       ?animvpx_nextpic_errmsg@@3PAPBDA 0071205c     animvpx.obj
 0004:00000080       _CheatStrings              00712080     cheats.obj
 0004:0000029c       ?althud_flashing@@3HA      0071229c     sbar.obj
 0004:000002a0       ?althud_numbertile@@3HA    007122a0     sbar.obj
 0004:000002a4       ?althud_shadows@@3HA       007122a4     sbar.obj
 0004:000002a8       _hud_glowingquotes         007122a8     screentext.obj
 0004:000002b0       _g_gameType                007122b0     common.obj
 0004:000002e8       _g_modDir                  007122e8     common.obj
 0004:000003f8       ?g_demo_recFilePtr@@3HA    007123f8     demo.obj
 0004:000003fc       ?g_demo_showStats@@3HA     007123fc     demo.obj
 0004:00000408       ?demoplay_diffs@@3HA       00712408     demo.obj
 0004:0000040c       ?demorec_diffs_cvar@@3HA   0071240c     demo.obj
 0004:00000410       ?demorec_difftics_cvar@@3HA 00712410     demo.obj
 0004:00000414       ?demorec_diffcompress_cvar@@3HA 00712414     demo.obj
 0004:00000418       ?demorec_synccompress_cvar@@3HA 00712418     demo.obj
 0004:0000041c       ?demorec_seeds_cvar@@3HA   0071241c     demo.obj
 0004:00000420       ?demoplay_showsync@@3HA    00712420     demo.obj
 0004:00000438       _g_scriptVersion           00712438     gamedef.obj
 0004:00000440       _g_szScriptFileName        00712440     gamedef.obj
 0004:00000748       _keyw                      00712748     gamedef.obj
 0004:00000d88       _EventNames                00712d88     gamedef.obj
 0004:00000f5c       _h_gamevars                00712f5c     gamedef.obj
 0004:00000f64       _h_arrays                  00712f64     gamedef.obj
 0004:00000f6c       _h_labels                  00712f6c     gamedef.obj
 0004:00000fd4       _g_currentEventExec        00712fd4     gameexec.obj
 0004:00000fd8       _g_iReturnVarID            00712fd8     gameexec.obj
 0004:00000fdc       _g_iWeaponVarID            00712fdc     gameexec.obj
 0004:00000fe0       _g_iWorksLikeVarID         00712fe0     gameexec.obj
 0004:00000fe4       _g_iZRangeVarID            00712fe4     gameexec.obj
 0004:00000fe8       _g_iAngRangeVarID          00712fe8     gameexec.obj
 0004:00000fec       _g_iAimAngleVarID          00712fec     gameexec.obj
 0004:00000ff0       _g_iLoTagID                00712ff0     gameexec.obj
 0004:00000ff4       _g_iHiTagID                00712ff4     gameexec.obj
 0004:00000ff8       _g_iTextureID              00712ff8     gameexec.obj
 0004:00000ffc       _g_iThisActorID            00712ffc     gameexec.obj
 0004:00001000       _g_iStructVarIDs           00713000     gameexec.obj
 0004:000013b8       _s_buildDate               007133b8     global.obj
 0004:000013bc       _g_spriteGravity           007133bc     global.obj
 0004:000013c0       _g_spriteDeleteQueueSize   007133c0     global.obj
 0004:000013c2       _g_numGametypes            007133c2     global.obj
 0004:000013c3       _g_numVolumes              007133c3     global.obj
 0004:000013c4       _g_timerTicsPerSecond      007133c4     global.obj
 0004:000013c8       _EpisodeNames              007133c8     global.obj
 0004:000014b0       _SkillNames                007134b0     global.obj
 0004:00001598       _GametypeNames             00713598     global.obj
 0004:000017a8       _GametypeFlags             007137a8     global.obj
 0004:000017e8       _g_actorRespawnTime        007137e8     global.obj
 0004:000017ec       _g_itemRespawnTime         007137ec     global.obj
 0004:000017f0       _g_rpgBlastRadius          007137f0     global.obj
 0004:000017f4       _g_pipebombBlastRadius     007137f4     global.obj
 0004:000017f8       _g_shrinkerBlastRadius     007137f8     global.obj
 0004:000017fc       _g_tripbombBlastRadius     007137fc     global.obj
 0004:00001800       _g_morterBlastRadius       00713800     global.obj
 0004:00001804       _g_bouncemineBlastRadius   00713804     global.obj
 0004:00001808       _g_seenineBlastRadius      00713808     global.obj
 0004:0000180c       _g_scriptSize              0071380c     global.obj
 0004:00001810       _BlimpSpawnSprites         00713810     global.obj
 0004:00001830       _g_playerFriction          00713830     global.obj
 0004:00001834       _g_numFreezeBounces        00713834     global.obj
 0004:00001838       _g_lastSaveSlot            00713838     global.obj
 0004:0000183c       _CheatKeys                 0071383c     global.obj
 0004:00001840       _setupfilename             00713840     global.obj
 0004:00001940       _g_skillSoundVoice         00713940     menus.obj
 0004:000046bc       _m_currentMenu             007166bc     menus.obj
 0004:00004ba8       ?SECTOREFFECTOR@@3HA       00716ba8     namesdyn.obj
 0004:00004bac       ?ACTIVATOR@@3HA            00716bac     namesdyn.obj
 0004:00004bb0       ?TOUCHPLATE@@3HA           00716bb0     namesdyn.obj
 0004:00004bb4       ?ACTIVATORLOCKED@@3HA      00716bb4     namesdyn.obj
 0004:00004bb8       ?MUSICANDSFX@@3HA          00716bb8     namesdyn.obj
 0004:00004bbc       ?LOCATORS@@3HA             00716bbc     namesdyn.obj
 0004:00004bc0       ?CYCLER@@3HA               00716bc0     namesdyn.obj
 0004:00004bc4       ?MASTERSWITCH@@3HA         00716bc4     namesdyn.obj
 0004:00004bc8       ?RESPAWN@@3HA              00716bc8     namesdyn.obj
 0004:00004bcc       ?GPSPEED@@3HA              00716bcc     namesdyn.obj
 0004:00004bd0       ?FOF@@3HA                  00716bd0     namesdyn.obj
 0004:00004bd4       ?ARROW@@3HA                00716bd4     namesdyn.obj
 0004:00004bd8       ?FIRSTGUNSPRITE@@3HA       00716bd8     namesdyn.obj
 0004:00004bdc       ?CHAINGUNSPRITE@@3HA       00716bdc     namesdyn.obj
 0004:00004be0       ?RPGSPRITE@@3HA            00716be0     namesdyn.obj
 0004:00004be4       ?FREEZESPRITE@@3HA         00716be4     namesdyn.obj
 0004:00004be8       ?SHRINKERSPRITE@@3HA       00716be8     namesdyn.obj
 0004:00004bec       ?HEAVYHBOMB@@3HA           00716bec     namesdyn.obj
 0004:00004bf0       ?TRIPBOMBSPRITE@@3HA       00716bf0     namesdyn.obj
 0004:00004bf4       ?SHOTGUNSPRITE@@3HA        00716bf4     namesdyn.obj
 0004:00004bf8       ?DEVISTATORSPRITE@@3HA     00716bf8     namesdyn.obj
 0004:00004bfc       ?HEALTHBOX@@3HA            00716bfc     namesdyn.obj
 0004:00004c00       ?AMMOBOX@@3HA              00716c00     namesdyn.obj
 0004:00004c04       ?GROWSPRITEICON@@3HA       00716c04     namesdyn.obj
 0004:00004c08       ?INVENTORYBOX@@3HA         00716c08     namesdyn.obj
 0004:00004c0c       ?FREEZEAMMO@@3HA           00716c0c     namesdyn.obj
 0004:00004c10       ?AMMO@@3HA                 00716c10     namesdyn.obj
 0004:00004c14       ?BATTERYAMMO@@3HA          00716c14     namesdyn.obj
 0004:00004c18       ?DEVISTATORAMMO@@3HA       00716c18     namesdyn.obj
 0004:00004c1c       ?RPGAMMO@@3HA              00716c1c     namesdyn.obj
 0004:00004c20       ?GROWAMMO@@3HA             00716c20     namesdyn.obj
 0004:00004c24       ?CRYSTALAMMO@@3HA          00716c24     namesdyn.obj
 0004:00004c28       ?HBOMBAMMO@@3HA            00716c28     namesdyn.obj
 0004:00004c2c       ?AMMOLOTS@@3HA             00716c2c     namesdyn.obj
 0004:00004c30       ?SHOTGUNAMMO@@3HA          00716c30     namesdyn.obj
 0004:00004c34       ?COLA@@3HA                 00716c34     namesdyn.obj
 0004:00004c38       ?SIXPAK@@3HA               00716c38     namesdyn.obj
 0004:00004c3c       ?FIRSTAID@@3HA             00716c3c     namesdyn.obj
 0004:00004c40       ?SHIELD@@3HA               00716c40     namesdyn.obj
 0004:00004c44       ?STEROIDS@@3HA             00716c44     namesdyn.obj
 0004:00004c48       ?AIRTANK@@3HA              00716c48     namesdyn.obj
 0004:00004c4c       ?JETPACK@@3HA              00716c4c     namesdyn.obj
 0004:00004c50       ?HEATSENSOR@@3HA           00716c50     namesdyn.obj
 0004:00004c54       ?ACCESSCARD@@3HA           00716c54     namesdyn.obj
 0004:00004c58       ?BOOTS@@3HA                00716c58     namesdyn.obj
 0004:00004c5c       ?MIRRORBROKE@@3HA          00716c5c     namesdyn.obj
 0004:00004c60       ?CLOUDYOCEAN@@3HA          00716c60     namesdyn.obj
 0004:00004c64       ?CLOUDYSKIES@@3HA          00716c64     namesdyn.obj
 0004:00004c68       ?MOONSKY1@@3HA             00716c68     namesdyn.obj
 0004:00004c6c       ?BIGORBIT1@@3HA            00716c6c     namesdyn.obj
 0004:00004c70       ?LA@@3HA                   00716c70     namesdyn.obj
 0004:00004c74       ?ATOMICHEALTH@@3HA         00716c74     namesdyn.obj
 0004:00004c78       ?TECHLIGHT2@@3HA           00716c78     namesdyn.obj
 0004:00004c7c       ?TECHLIGHTBUST2@@3HA       00716c7c     namesdyn.obj
 0004:00004c80       ?TECHLIGHT4@@3HA           00716c80     namesdyn.obj
 0004:00004c84       ?TECHLIGHTBUST4@@3HA       00716c84     namesdyn.obj
 0004:00004c88       ?WALLLIGHT4@@3HA           00716c88     namesdyn.obj
 0004:00004c8c       ?WALLLIGHTBUST4@@3HA       00716c8c     namesdyn.obj
 0004:00004c90       ?ACCESSSWITCH@@3HA         00716c90     namesdyn.obj
 0004:00004c94       ?SLOTDOOR@@3HA             00716c94     namesdyn.obj
 0004:00004c98       ?LIGHTSWITCH@@3HA          00716c98     namesdyn.obj
 0004:00004c9c       ?SPACEDOORSWITCH@@3HA      00716c9c     namesdyn.obj
 0004:00004ca0       ?SPACELIGHTSWITCH@@3HA     00716ca0     namesdyn.obj
 0004:00004ca4       ?FRANKENSTINESWITCH@@3HA   00716ca4     namesdyn.obj
 0004:00004ca8       ?NUKEBUTTON@@3HA           00716ca8     namesdyn.obj
 0004:00004cac       ?MULTISWITCH@@3HA          00716cac     namesdyn.obj
 0004:00004cb0       ?DOORTILE5@@3HA            00716cb0     namesdyn.obj
 0004:00004cb4       ?DOORTILE6@@3HA            00716cb4     namesdyn.obj
 0004:00004cb8       ?DOORTILE1@@3HA            00716cb8     namesdyn.obj
 0004:00004cbc       ?DOORTILE2@@3HA            00716cbc     namesdyn.obj
 0004:00004cc0       ?DOORTILE3@@3HA            00716cc0     namesdyn.obj
 0004:00004cc4       ?DOORTILE4@@3HA            00716cc4     namesdyn.obj
 0004:00004cc8       ?DOORTILE7@@3HA            00716cc8     namesdyn.obj
 0004:00004ccc       ?DOORTILE8@@3HA            00716ccc     namesdyn.obj
 0004:00004cd0       ?DOORTILE9@@3HA            00716cd0     namesdyn.obj
 0004:00004cd4       ?DOORTILE10@@3HA           00716cd4     namesdyn.obj
 0004:00004cd8       ?DOORSHOCK@@3HA            00716cd8     namesdyn.obj
 0004:00004cdc       ?DIPSWITCH@@3HA            00716cdc     namesdyn.obj
 0004:00004ce0       ?DIPSWITCH2@@3HA           00716ce0     namesdyn.obj
 0004:00004ce4       ?TECHSWITCH@@3HA           00716ce4     namesdyn.obj
 0004:00004ce8       ?DIPSWITCH3@@3HA           00716ce8     namesdyn.obj
 0004:00004cec       ?ACCESSSWITCH2@@3HA        00716cec     namesdyn.obj
 0004:00004cf0       ?FLOORSLIME@@3HA           00716cf0     namesdyn.obj
 0004:00004cf4       ?BIGFORCE@@3HA             00716cf4     namesdyn.obj
 0004:00004cf8       ?MASKWALL9@@3HA            00716cf8     namesdyn.obj
 0004:00004cfc       ?SCREENBREAK1@@3HA         00716cfc     namesdyn.obj
 0004:00004d00       ?SCREENBREAK2@@3HA         00716d00     namesdyn.obj
 0004:00004d04       ?SCREENBREAK3@@3HA         00716d04     namesdyn.obj
 0004:00004d08       ?SCREENBREAK4@@3HA         00716d08     namesdyn.obj
 0004:00004d0c       ?SCREENBREAK5@@3HA         00716d0c     namesdyn.obj
 0004:00004d10       ?SCREENBREAK6@@3HA         00716d10     namesdyn.obj
 0004:00004d14       ?SCREENBREAK7@@3HA         00716d14     namesdyn.obj
 0004:00004d18       ?SCREENBREAK8@@3HA         00716d18     namesdyn.obj
 0004:00004d1c       ?SCREENBREAK9@@3HA         00716d1c     namesdyn.obj
 0004:00004d20       ?SCREENBREAK10@@3HA        00716d20     namesdyn.obj
 0004:00004d24       ?SCREENBREAK11@@3HA        00716d24     namesdyn.obj
 0004:00004d28       ?SCREENBREAK12@@3HA        00716d28     namesdyn.obj
 0004:00004d2c       ?SCREENBREAK13@@3HA        00716d2c     namesdyn.obj
 0004:00004d30       ?MASKWALL1@@3HA            00716d30     namesdyn.obj
 0004:00004d34       ?W_TECHWALL1@@3HA          00716d34     namesdyn.obj
 0004:00004d38       ?W_TECHWALL2@@3HA          00716d38     namesdyn.obj
 0004:00004d3c       ?W_TECHWALL15@@3HA         00716d3c     namesdyn.obj
 0004:00004d40       ?W_TECHWALL3@@3HA          00716d40     namesdyn.obj
 0004:00004d44       ?W_TECHWALL4@@3HA          00716d44     namesdyn.obj
 0004:00004d48       ?W_TECHWALL10@@3HA         00716d48     namesdyn.obj
 0004:00004d4c       ?W_TECHWALL16@@3HA         00716d4c     namesdyn.obj
 0004:00004d50       ?WATERTILE2@@3HA           00716d50     namesdyn.obj
 0004:00004d54       ?BPANNEL1@@3HA             00716d54     namesdyn.obj
 0004:00004d58       ?PANNEL1@@3HA              00716d58     namesdyn.obj
 0004:00004d5c       ?PANNEL2@@3HA              00716d5c     namesdyn.obj
 0004:00004d60       ?STATIC@@3HA               00716d60     namesdyn.obj
 0004:00004d64       ?W_SCREENBREAK@@3HA        00716d64     namesdyn.obj
 0004:00004d68       ?W_HITTECHWALL3@@3HA       00716d68     namesdyn.obj
 0004:00004d6c       ?W_HITTECHWALL4@@3HA       00716d6c     namesdyn.obj
 0004:00004d70       ?W_HITTECHWALL2@@3HA       00716d70     namesdyn.obj
 0004:00004d74       ?W_HITTECHWALL1@@3HA       00716d74     namesdyn.obj
 0004:00004d78       ?MASKWALL10@@3HA           00716d78     namesdyn.obj
 0004:00004d7c       ?MASKWALL11@@3HA           00716d7c     namesdyn.obj
 0004:00004d80       ?DOORTILE22@@3HA           00716d80     namesdyn.obj
 0004:00004d84       ?FANSPRITE@@3HA            00716d84     namesdyn.obj
 0004:00004d88       ?FANSPRITEBROKE@@3HA       00716d88     namesdyn.obj
 0004:00004d8c       ?FANSHADOW@@3HA            00716d8c     namesdyn.obj
 0004:00004d90       ?FANSHADOWBROKE@@3HA       00716d90     namesdyn.obj
 0004:00004d94       ?DOORTILE18@@3HA           00716d94     namesdyn.obj
 0004:00004d98       ?DOORTILE19@@3HA           00716d98     namesdyn.obj
 0004:00004d9c       ?DOORTILE20@@3HA           00716d9c     namesdyn.obj
 0004:00004da0       ?VIEWSCREEN2@@3HA          00716da0     namesdyn.obj
 0004:00004da4       ?VIEWSCREEN@@3HA           00716da4     namesdyn.obj
 0004:00004da8       ?GLASS@@3HA                00716da8     namesdyn.obj
 0004:00004dac       ?GLASS2@@3HA               00716dac     namesdyn.obj
 0004:00004db0       ?STAINGLASS1@@3HA          00716db0     namesdyn.obj
 0004:00004db4       ?MASKWALL5@@3HA            00716db4     namesdyn.obj
 0004:00004db8       ?SATELITE@@3HA             00716db8     namesdyn.obj
 0004:00004dbc       ?FUELPOD@@3HA              00716dbc     namesdyn.obj
 0004:00004dc0       ?CRACK1@@3HA               00716dc0     namesdyn.obj
 0004:00004dc4       ?CRACK2@@3HA               00716dc4     namesdyn.obj
 0004:00004dc8       ?CRACK3@@3HA               00716dc8     namesdyn.obj
 0004:00004dcc       ?CRACK4@@3HA               00716dcc     namesdyn.obj
 0004:00004dd0       ?FOOTPRINTS@@3HA           00716dd0     namesdyn.obj
 0004:00004dd4       ?DOMELITE@@3HA             00716dd4     namesdyn.obj
 0004:00004dd8       ?CAMERAPOLE@@3HA           00716dd8     namesdyn.obj
 0004:00004ddc       ?CHAIR1@@3HA               00716ddc     namesdyn.obj
 0004:00004de0       ?CHAIR2@@3HA               00716de0     namesdyn.obj
 0004:00004de4       ?BROKENCHAIR@@3HA          00716de4     namesdyn.obj
 0004:00004de8       ?MIRROR@@3HA               00716de8     namesdyn.obj
 0004:00004dec       ?WATERFOUNTAIN@@3HA        00716dec     namesdyn.obj
 0004:00004df0       ?WATERFOUNTAINBROKE@@3HA   00716df0     namesdyn.obj
 0004:00004df4       ?FEMMAG1@@3HA              00716df4     namesdyn.obj
 0004:00004df8       ?TOILET@@3HA               00716df8     namesdyn.obj
 0004:00004dfc       ?STALL@@3HA                00716dfc     namesdyn.obj
 0004:00004e00       ?STALLBROKE@@3HA           00716e00     namesdyn.obj
 0004:00004e04       ?FEMMAG2@@3HA              00716e04     namesdyn.obj
 0004:00004e08       ?REACTOR2@@3HA             00716e08     namesdyn.obj
 0004:00004e0c       ?REACTOR2BURNT@@3HA        00716e0c     namesdyn.obj
 0004:00004e10       ?REACTOR2SPARK@@3HA        00716e10     namesdyn.obj
 0004:00004e14       ?GRATE1@@3HA               00716e14     namesdyn.obj
 0004:00004e18       ?BGRATE1@@3HA              00716e18     namesdyn.obj
 0004:00004e1c       ?SOLARPANNEL@@3HA          00716e1c     namesdyn.obj
 0004:00004e20       ?NAKED1@@3HA               00716e20     namesdyn.obj
 0004:00004e24       ?ANTENNA@@3HA              00716e24     namesdyn.obj
 0004:00004e28       ?MASKWALL12@@3HA           00716e28     namesdyn.obj
 0004:00004e2c       ?TOILETBROKE@@3HA          00716e2c     namesdyn.obj
 0004:00004e30       ?PIPE2@@3HA                00716e30     namesdyn.obj
 0004:00004e34       ?PIPE1B@@3HA               00716e34     namesdyn.obj
 0004:00004e38       ?PIPE3@@3HA                00716e38     namesdyn.obj
 0004:00004e3c       ?PIPE1@@3HA                00716e3c     namesdyn.obj
 0004:00004e40       ?CAMERA1@@3HA              00716e40     namesdyn.obj
 0004:00004e44       ?PIPE2B@@3HA               00716e44     namesdyn.obj
 0004:00004e48       ?BOLT1@@3HA                00716e48     namesdyn.obj
 0004:00004e4c       ?W_NUMBERS@@3HA            00716e4c     namesdyn.obj
 0004:00004e50       ?WATERDRIP@@3HA            00716e50     namesdyn.obj
 0004:00004e54       ?WATERBUBBLE@@3HA          00716e54     namesdyn.obj
 0004:00004e58       ?WATERBUBBLEMAKER@@3HA     00716e58     namesdyn.obj
 0004:00004e5c       ?W_FORCEFIELD@@3HA         00716e5c     namesdyn.obj
 0004:00004e60       ?VACUUM@@3HA               00716e60     namesdyn.obj
 0004:00004e64       ?FOOTPRINTS2@@3HA          00716e64     namesdyn.obj
 0004:00004e68       ?FOOTPRINTS3@@3HA          00716e68     namesdyn.obj
 0004:00004e6c       ?FOOTPRINTS4@@3HA          00716e6c     namesdyn.obj
 0004:00004e70       ?EGG@@3HA                  00716e70     namesdyn.obj
 0004:00004e74       ?SCALE@@3HA                00716e74     namesdyn.obj
 0004:00004e78       ?CHAIR3@@3HA               00716e78     namesdyn.obj
 0004:00004e7c       ?CAMERALIGHT@@3HA          00716e7c     namesdyn.obj
 0004:00004e80       ?MOVIECAMERA@@3HA          00716e80     namesdyn.obj
 0004:00004e84       ?IVUNIT@@3HA               00716e84     namesdyn.obj
 0004:00004e88       ?POT1@@3HA                 00716e88     namesdyn.obj
 0004:00004e8c       ?POT2@@3HA                 00716e8c     namesdyn.obj
 0004:00004e90       ?POT3@@3HA                 00716e90     namesdyn.obj
 0004:00004e94       ?PIPE3B@@3HA               00716e94     namesdyn.obj
 0004:00004e98       ?WALLLIGHT3@@3HA           00716e98     namesdyn.obj
 0004:00004e9c       ?WALLLIGHTBUST3@@3HA       00716e9c     namesdyn.obj
 0004:00004ea0       ?WALLLIGHT1@@3HA           00716ea0     namesdyn.obj
 0004:00004ea4       ?WALLLIGHTBUST1@@3HA       00716ea4     namesdyn.obj
 0004:00004ea8       ?WALLLIGHT2@@3HA           00716ea8     namesdyn.obj
 0004:00004eac       ?WALLLIGHTBUST2@@3HA       00716eac     namesdyn.obj
 0004:00004eb0       ?LIGHTSWITCH2@@3HA         00716eb0     namesdyn.obj
 0004:00004eb4       ?WAITTOBESEATED@@3HA       00716eb4     namesdyn.obj
 0004:00004eb8       ?DOORTILE14@@3HA           00716eb8     namesdyn.obj
 0004:00004ebc       ?STATUE@@3HA               00716ebc     namesdyn.obj
 0004:00004ec0       ?MIKE@@3HA                 00716ec0     namesdyn.obj
 0004:00004ec4       ?VASE@@3HA                 00716ec4     namesdyn.obj
 0004:00004ec8       ?SUSHIPLATE1@@3HA          00716ec8     namesdyn.obj
 0004:00004ecc       ?SUSHIPLATE2@@3HA          00716ecc     namesdyn.obj
 0004:00004ed0       ?SUSHIPLATE3@@3HA          00716ed0     namesdyn.obj
 0004:00004ed4       ?SUSHIPLATE4@@3HA          00716ed4     namesdyn.obj
 0004:00004ed8       ?DOORTILE16@@3HA           00716ed8     namesdyn.obj
 0004:00004edc       ?SUSHIPLATE5@@3HA          00716edc     namesdyn.obj
 0004:00004ee0       ?OJ@@3HA                   00716ee0     namesdyn.obj
 0004:00004ee4       ?MASKWALL13@@3HA           00716ee4     namesdyn.obj
 0004:00004ee8       ?HURTRAIL@@3HA             00716ee8     namesdyn.obj
 0004:00004eec       ?POWERSWITCH1@@3HA         00716eec     namesdyn.obj
 0004:00004ef0       ?LOCKSWITCH1@@3HA          00716ef0     namesdyn.obj
 0004:00004ef4       ?POWERSWITCH2@@3HA         00716ef4     namesdyn.obj
 0004:00004ef8       ?ATM@@3HA                  00716ef8     namesdyn.obj
 0004:00004efc       ?STATUEFLASH@@3HA          00716efc     namesdyn.obj
 0004:00004f00       ?ATMBROKE@@3HA             00716f00     namesdyn.obj
 0004:00004f04       ?STRIPEBALL@@3HA           00716f04     namesdyn.obj
 0004:00004f08       ?QUEBALL@@3HA              00716f08     namesdyn.obj
 0004:00004f0c       ?POCKET@@3HA               00716f0c     namesdyn.obj
 0004:00004f10       ?WOODENHORSE@@3HA          00716f10     namesdyn.obj
 0004:00004f14       ?TREE1@@3HA                00716f14     namesdyn.obj
 0004:00004f18       ?TREE2@@3HA                00716f18     namesdyn.obj
 0004:00004f1c       ?CACTUS@@3HA               00716f1c     namesdyn.obj
 0004:00004f20       ?MASKWALL2@@3HA            00716f20     namesdyn.obj
 0004:00004f24       ?MASKWALL3@@3HA            00716f24     namesdyn.obj
 0004:00004f28       ?MASKWALL4@@3HA            00716f28     namesdyn.obj
 0004:00004f2c       ?FIREEXT@@3HA              00716f2c     namesdyn.obj
 0004:00004f30       ?TOILETWATER@@3HA          00716f30     namesdyn.obj
 0004:00004f34       ?NEON1@@3HA                00716f34     namesdyn.obj
 0004:00004f38       ?NEON2@@3HA                00716f38     namesdyn.obj
 0004:00004f3c       ?CACTUSBROKE@@3HA          00716f3c     namesdyn.obj
 0004:00004f40       ?BOUNCEMINE@@3HA           00716f40     namesdyn.obj
 0004:00004f44       ?BROKEFIREHYDRENT@@3HA     00716f44     namesdyn.obj
 0004:00004f48       ?BOX@@3HA                  00716f48     namesdyn.obj
 0004:00004f4c       ?BULLETHOLE@@3HA           00716f4c     namesdyn.obj
 0004:00004f50       ?BOTTLE1@@3HA              00716f50     namesdyn.obj
 0004:00004f54       ?BOTTLE2@@3HA              00716f54     namesdyn.obj
 0004:00004f58       ?BOTTLE3@@3HA              00716f58     namesdyn.obj
 0004:00004f5c       ?BOTTLE4@@3HA              00716f5c     namesdyn.obj
 0004:00004f60       ?FEMPIC5@@3HA              00716f60     namesdyn.obj
 0004:00004f64       ?FEMPIC6@@3HA              00716f64     namesdyn.obj
 0004:00004f68       ?FEMPIC7@@3HA              00716f68     namesdyn.obj
 0004:00004f6c       ?HYDROPLANT@@3HA           00716f6c     namesdyn.obj
 0004:00004f70       ?OCEANSPRITE1@@3HA         00716f70     namesdyn.obj
 0004:00004f74       ?OCEANSPRITE2@@3HA         00716f74     namesdyn.obj
 0004:00004f78       ?OCEANSPRITE3@@3HA         00716f78     namesdyn.obj
 0004:00004f7c       ?OCEANSPRITE4@@3HA         00716f7c     namesdyn.obj
 0004:00004f80       ?OCEANSPRITE5@@3HA         00716f80     namesdyn.obj
 0004:00004f84       ?GENERICPOLE@@3HA          00716f84     namesdyn.obj
 0004:00004f88       ?CONE@@3HA                 00716f88     namesdyn.obj
 0004:00004f8c       ?HANGLIGHT@@3HA            00716f8c     namesdyn.obj
 0004:00004f90       ?HYDRENT@@3HA              00716f90     namesdyn.obj
 0004:00004f94       ?MASKWALL14@@3HA           00716f94     namesdyn.obj
 0004:00004f98       ?TIRE@@3HA                 00716f98     namesdyn.obj
 0004:00004f9c       ?PIPE5@@3HA                00716f9c     namesdyn.obj
 0004:00004fa0       ?PIPE6@@3HA                00716fa0     namesdyn.obj
 0004:00004fa4       ?PIPE4@@3HA                00716fa4     namesdyn.obj
 0004:00004fa8       ?PIPE4B@@3HA               00716fa8     namesdyn.obj
 0004:00004fac       ?BROKEHYDROPLANT@@3HA      00716fac     namesdyn.obj
 0004:00004fb0       ?PIPE5B@@3HA               00716fb0     namesdyn.obj
 0004:00004fb4       ?NEON3@@3HA                00716fb4     namesdyn.obj
 0004:00004fb8       ?NEON4@@3HA                00716fb8     namesdyn.obj
 0004:00004fbc       ?NEON5@@3HA                00716fbc     namesdyn.obj
 0004:00004fc0       ?BOTTLE5@@3HA              00716fc0     namesdyn.obj
 0004:00004fc4       ?BOTTLE6@@3HA              00716fc4     namesdyn.obj
 0004:00004fc8       ?BOTTLE8@@3HA              00716fc8     namesdyn.obj
 0004:00004fcc       ?SPOTLITE@@3HA             00716fcc     namesdyn.obj
 0004:00004fd0       ?MASKWALL15@@3HA           00716fd0     namesdyn.obj
 0004:00004fd4       ?BOTTLE7@@3HA              00716fd4     namesdyn.obj
 0004:00004fd8       ?HORSEONSIDE@@3HA          00716fd8     namesdyn.obj
 0004:00004fdc       ?GLASSPIECES@@3HA          00716fdc     namesdyn.obj
 0004:00004fe0       ?NEON6@@3HA                00716fe0     namesdyn.obj
 0004:00004fe4       ?MASKWALL6@@3HA            00716fe4     namesdyn.obj
 0004:00004fe8       ?RUBBERCAN@@3HA            00716fe8     namesdyn.obj
 0004:00004fec       ?PLUG@@3HA                 00716fec     namesdyn.obj
 0004:00004ff0       ?OOZFILTER@@3HA            00716ff0     namesdyn.obj
 0004:00004ff4       ?FLOORPLASMA@@3HA          00716ff4     namesdyn.obj
 0004:00004ff8       ?REACTOR@@3HA              00716ff8     namesdyn.obj
 0004:00004ffc       ?REACTORSPARK@@3HA         00716ffc     namesdyn.obj
 0004:00005000       ?REACTORBURNT@@3HA         00717000     namesdyn.obj
 0004:00005004       ?DOORTILE15@@3HA           00717004     namesdyn.obj
 0004:00005008       ?HANDSWITCH@@3HA           00717008     namesdyn.obj
 0004:0000500c       ?CIRCLEPANNEL@@3HA         0071700c     namesdyn.obj
 0004:00005010       ?CIRCLEPANNELBROKE@@3HA    00717010     namesdyn.obj
 0004:00005014       ?PULLSWITCH@@3HA           00717014     namesdyn.obj
 0004:00005018       ?MASKWALL8@@3HA            00717018     namesdyn.obj
 0004:0000501c       ?BIGHOLE@@3HA              0071701c     namesdyn.obj
 0004:00005020       ?ALIENSWITCH@@3HA          00717020     namesdyn.obj
 0004:00005024       ?DOORTILE21@@3HA           00717024     namesdyn.obj
 0004:00005028       ?HANDPRINTSWITCH@@3HA      00717028     namesdyn.obj
 0004:0000502c       ?BOTTLE10@@3HA             0071702c     namesdyn.obj
 0004:00005030       ?BOTTLE11@@3HA             00717030     namesdyn.obj
 0004:00005034       ?BOTTLE12@@3HA             00717034     namesdyn.obj
 0004:00005038       ?BOTTLE13@@3HA             00717038     namesdyn.obj
 0004:0000503c       ?BOTTLE14@@3HA             0071703c     namesdyn.obj
 0004:00005040       ?BOTTLE15@@3HA             00717040     namesdyn.obj
 0004:00005044       ?BOTTLE16@@3HA             00717044     namesdyn.obj
 0004:00005048       ?BOTTLE17@@3HA             00717048     namesdyn.obj
 0004:0000504c       ?BOTTLE18@@3HA             0071704c     namesdyn.obj
 0004:00005050       ?BOTTLE19@@3HA             00717050     namesdyn.obj
 0004:00005054       ?DOORTILE17@@3HA           00717054     namesdyn.obj
 0004:00005058       ?MASKWALL7@@3HA            00717058     namesdyn.obj
 0004:0000505c       ?DOORTILE11@@3HA           0071705c     namesdyn.obj
 0004:00005060       ?DOORTILE12@@3HA           00717060     namesdyn.obj
 0004:00005064       ?VENDMACHINE@@3HA          00717064     namesdyn.obj
 0004:00005068       ?COLAMACHINE@@3HA          00717068     namesdyn.obj
 0004:0000506c       ?CRANEPOLE@@3HA            0071706c     namesdyn.obj
 0004:00005070       ?CRANE@@3HA                00717070     namesdyn.obj
 0004:00005074       ?BARBROKE@@3HA             00717074     namesdyn.obj
 0004:00005078       ?BLOODPOOL@@3HA            00717078     namesdyn.obj
 0004:0000507c       ?NUKEBARREL@@3HA           0071707c     namesdyn.obj
 0004:00005080       ?NUKEBARRELDENTED@@3HA     00717080     namesdyn.obj
 0004:00005084       ?NUKEBARRELLEAKED@@3HA     00717084     namesdyn.obj
 0004:00005088       ?CANWITHSOMETHING@@3HA     00717088     namesdyn.obj
 0004:0000508c       ?MONEY@@3HA                0071708c     namesdyn.obj
 0004:00005090       ?BANNER@@3HA               00717090     namesdyn.obj
 0004:00005094       ?EXPLODINGBARREL@@3HA      00717094     namesdyn.obj
 0004:00005098       ?EXPLODINGBARREL2@@3HA     00717098     namesdyn.obj
 0004:0000509c       ?FIREBARREL@@3HA           0071709c     namesdyn.obj
 0004:000050a0       ?SEENINE@@3HA              007170a0     namesdyn.obj
 0004:000050a4       ?SEENINEDEAD@@3HA          007170a4     namesdyn.obj
 0004:000050a8       ?STEAM@@3HA                007170a8     namesdyn.obj
 0004:000050ac       ?CEILINGSTEAM@@3HA         007170ac     namesdyn.obj
 0004:000050b0       ?PIPE6B@@3HA               007170b0     namesdyn.obj
 0004:000050b4       ?TRANSPORTERBEAM@@3HA      007170b4     namesdyn.obj
 0004:000050b8       ?RAT@@3HA                  007170b8     namesdyn.obj
 0004:000050bc       ?TRASH@@3HA                007170bc     namesdyn.obj
 0004:000050c0       ?FEMPIC1@@3HA              007170c0     namesdyn.obj
 0004:000050c4       ?FEMPIC2@@3HA              007170c4     namesdyn.obj
 0004:000050c8       ?BLANKSCREEN@@3HA          007170c8     namesdyn.obj
 0004:000050cc       ?PODFEM1@@3HA              007170cc     namesdyn.obj
 0004:000050d0       ?FEMPIC3@@3HA              007170d0     namesdyn.obj
 0004:000050d4       ?FEMPIC4@@3HA              007170d4     namesdyn.obj
 0004:000050d8       ?FEM1@@3HA                 007170d8     namesdyn.obj
 0004:000050dc       ?FEM2@@3HA                 007170dc     namesdyn.obj
 0004:000050e0       ?FEM3@@3HA                 007170e0     namesdyn.obj
 0004:000050e4       ?FEM5@@3HA                 007170e4     namesdyn.obj
 0004:000050e8       ?BLOODYPOLE@@3HA           007170e8     namesdyn.obj
 0004:000050ec       ?FEM4@@3HA                 007170ec     namesdyn.obj
 0004:000050f0       ?FEM6@@3HA                 007170f0     namesdyn.obj
 0004:000050f4       ?FEM6PAD@@3HA              007170f4     namesdyn.obj
 0004:000050f8       ?FEM8@@3HA                 007170f8     namesdyn.obj
 0004:000050fc       ?HELECOPT@@3HA             007170fc     namesdyn.obj
 0004:00005100       ?FETUSJIB@@3HA             00717100     namesdyn.obj
 0004:00005104       ?HOLODUKE@@3HA             00717104     namesdyn.obj
 0004:00005108       ?SPACEMARINE@@3HA          00717108     namesdyn.obj
 0004:0000510c       ?INDY@@3HA                 0071710c     namesdyn.obj
 0004:00005110       ?FETUS@@3HA                00717110     namesdyn.obj
 0004:00005114       ?FETUSBROKE@@3HA           00717114     namesdyn.obj
 0004:00005118       ?MONK@@3HA                 00717118     namesdyn.obj
 0004:0000511c       ?LUKE@@3HA                 0071711c     namesdyn.obj
 0004:00005120       ?COOLEXPLOSION1@@3HA       00717120     namesdyn.obj
 0004:00005124       ?WATERSPLASH2@@3HA         00717124     namesdyn.obj
 0004:00005128       ?FIREVASE@@3HA             00717128     namesdyn.obj
 0004:0000512c       ?FEM7@@3HA                 0071712c     namesdyn.obj
 0004:00005130       ?APLAYERTOP@@3HA           00717130     namesdyn.obj
 0004:00005134       ?APLAYER@@3HA              00717134     namesdyn.obj
 0004:00005138       ?PLAYERONWATER@@3HA        00717138     namesdyn.obj
 0004:0000513c       ?DUKELYINGDEAD@@3HA        0071713c     namesdyn.obj
 0004:00005140       ?DUKETORSO@@3HA            00717140     namesdyn.obj
 0004:00005144       ?DUKEGUN@@3HA              00717144     namesdyn.obj
 0004:00005148       ?DUKELEG@@3HA              00717148     namesdyn.obj
 0004:0000514c       ?SHARK@@3HA                0071714c     namesdyn.obj
 0004:00005150       ?BLOOD@@3HA                00717150     namesdyn.obj
 0004:00005154       ?FIRELASER@@3HA            00717154     namesdyn.obj
 0004:00005158       ?TRANSPORTERSTAR@@3HA      00717158     namesdyn.obj
 0004:0000515c       ?SPIT@@3HA                 0071715c     namesdyn.obj
 0004:00005160       ?LOOGIE@@3HA               00717160     namesdyn.obj
 0004:00005164       ?FIST@@3HA                 00717164     namesdyn.obj
 0004:00005168       ?FREEZEBLAST@@3HA          00717168     namesdyn.obj
 0004:0000516c       ?SHRINKSPARK@@3HA          0071716c     namesdyn.obj
 0004:00005170       ?TONGUE@@3HA               00717170     namesdyn.obj
 0004:00005174       ?MORTER@@3HA               00717174     namesdyn.obj
 0004:00005178       ?SHRINKEREXPLOSION@@3HA    00717178     namesdyn.obj
 0004:0000517c       ?RADIUSEXPLOSION@@3HA      0071717c     namesdyn.obj
 0004:00005180       ?FORCERIPPLE@@3HA          00717180     namesdyn.obj
 0004:00005184       ?LIZTROOP@@3HA             00717184     namesdyn.obj
 0004:00005188       ?LIZTROOPRUNNING@@3HA      00717188     namesdyn.obj
 0004:0000518c       ?LIZTROOPSTAYPUT@@3HA      0071718c     namesdyn.obj
 0004:00005190       ?LIZTROOPSHOOT@@3HA        00717190     namesdyn.obj
 0004:00005194       ?LIZTROOPJETPACK@@3HA      00717194     namesdyn.obj
 0004:00005198       ?LIZTROOPONTOILET@@3HA     00717198     namesdyn.obj
 0004:0000519c       ?LIZTROOPJUSTSIT@@3HA      0071719c     namesdyn.obj
 0004:000051a0       ?LIZTROOPDUCKING@@3HA      007171a0     namesdyn.obj
 0004:000051a4       ?HEADJIB1@@3HA             007171a4     namesdyn.obj
 0004:000051a8       ?ARMJIB1@@3HA              007171a8     namesdyn.obj
 0004:000051ac       ?LEGJIB1@@3HA              007171ac     namesdyn.obj
 0004:000051b0       ?OCTABRAIN@@3HA            007171b0     namesdyn.obj
 0004:000051b4       ?OCTABRAINSTAYPUT@@3HA     007171b4     namesdyn.obj
 0004:000051b8       ?INNERJAW@@3HA             007171b8     namesdyn.obj
 0004:000051bc       ?DRONE@@3HA                007171bc     namesdyn.obj
 0004:000051c0       ?EXPLOSION2@@3HA           007171c0     namesdyn.obj
 0004:000051c4       ?COMMANDER@@3HA            007171c4     namesdyn.obj
 0004:000051c8       ?COMMANDERSTAYPUT@@3HA     007171c8     namesdyn.obj
 0004:000051cc       ?RECON@@3HA                007171cc     namesdyn.obj
 0004:000051d0       ?TANK@@3HA                 007171d0     namesdyn.obj
 0004:000051d4       ?PIGCOP@@3HA               007171d4     namesdyn.obj
 0004:000051d8       ?PIGCOPSTAYPUT@@3HA        007171d8     namesdyn.obj
 0004:000051dc       ?PIGCOPDIVE@@3HA           007171dc     namesdyn.obj
 0004:000051e0       ?LIZMAN@@3HA               007171e0     namesdyn.obj
 0004:000051e4       ?LIZMANSTAYPUT@@3HA        007171e4     namesdyn.obj
 0004:000051e8       ?LIZMANSPITTING@@3HA       007171e8     namesdyn.obj
 0004:000051ec       ?LIZMANFEEDING@@3HA        007171ec     namesdyn.obj
 0004:000051f0       ?LIZMANJUMP@@3HA           007171f0     namesdyn.obj
 0004:000051f4       ?FECES@@3HA                007171f4     namesdyn.obj
 0004:000051f8       ?LIZMANHEAD1@@3HA          007171f8     namesdyn.obj
 0004:000051fc       ?LIZMANARM1@@3HA           007171fc     namesdyn.obj
 0004:00005200       ?LIZMANLEG1@@3HA           00717200     namesdyn.obj
 0004:00005204       ?EXPLOSION2BOT@@3HA        00717204     namesdyn.obj
 0004:00005208       ?JIBS1@@3HA                00717208     namesdyn.obj
 0004:0000520c       ?JIBS2@@3HA                0071720c     namesdyn.obj
 0004:00005210       ?JIBS3@@3HA                00717210     namesdyn.obj
 0004:00005214       ?JIBS4@@3HA                00717214     namesdyn.obj
 0004:00005218       ?JIBS5@@3HA                00717218     namesdyn.obj
 0004:0000521c       ?BURNING@@3HA              0071721c     namesdyn.obj
 0004:00005220       ?FIRE@@3HA                 00717220     namesdyn.obj
 0004:00005224       ?JIBS6@@3HA                00717224     namesdyn.obj
 0004:00005228       ?BLOODSPLAT1@@3HA          00717228     namesdyn.obj
 0004:0000522c       ?BLOODSPLAT3@@3HA          0071722c     namesdyn.obj
 0004:00005230       ?BLOODSPLAT2@@3HA          00717230     namesdyn.obj
 0004:00005234       ?BLOODSPLAT4@@3HA          00717234     namesdyn.obj
 0004:00005238       ?OOZ@@3HA                  00717238     namesdyn.obj
 0004:0000523c       ?OOZ2@@3HA                 0071723c     namesdyn.obj
 0004:00005240       ?WALLBLOOD1@@3HA           00717240     namesdyn.obj
 0004:00005244       ?WALLBLOOD2@@3HA           00717244     namesdyn.obj
 0004:00005248       ?WALLBLOOD3@@3HA           00717248     namesdyn.obj
 0004:0000524c       ?WALLBLOOD4@@3HA           0071724c     namesdyn.obj
 0004:00005250       ?WALLBLOOD5@@3HA           00717250     namesdyn.obj
 0004:00005254       ?WALLBLOOD7@@3HA           00717254     namesdyn.obj
 0004:00005258       ?WALLBLOOD8@@3HA           00717258     namesdyn.obj
 0004:0000525c       ?BURNING2@@3HA             0071725c     namesdyn.obj
 0004:00005260       ?FIRE2@@3HA                00717260     namesdyn.obj
 0004:00005264       ?CRACKKNUCKLES@@3HA        00717264     namesdyn.obj
 0004:00005268       ?SMALLSMOKE@@3HA           00717268     namesdyn.obj
 0004:0000526c       ?FLOORFLAME@@3HA           0071726c     namesdyn.obj
 0004:00005270       ?ROTATEGUN@@3HA            00717270     namesdyn.obj
 0004:00005274       ?GREENSLIME@@3HA           00717274     namesdyn.obj
 0004:00005278       ?WATERDRIPSPLASH@@3HA      00717278     namesdyn.obj
 0004:0000527c       ?SCRAP6@@3HA               0071727c     namesdyn.obj
 0004:00005280       ?SCRAP1@@3HA               00717280     namesdyn.obj
 0004:00005284       ?SCRAP2@@3HA               00717284     namesdyn.obj
 0004:00005288       ?SCRAP3@@3HA               00717288     namesdyn.obj
 0004:0000528c       ?SCRAP4@@3HA               0071728c     namesdyn.obj
 0004:00005290       ?SCRAP5@@3HA               00717290     namesdyn.obj
 0004:00005294       ?ORGANTIC@@3HA             00717294     namesdyn.obj
 0004:00005298       ?BETAVERSION@@3HA          00717298     namesdyn.obj
 0004:0000529c       ?SELECTDIR@@3HA            0071729c     namesdyn.obj
 0004:000052a0       ?F1HELP@@3HA               007172a0     namesdyn.obj
 0004:000052a4       ?GROWSPARK@@3HA            007172a4     namesdyn.obj
 0004:000052a8       ?MENUSCREEN@@3HA           007172a8     namesdyn.obj
 0004:000052ac       ?MENUBAR@@3HA              007172ac     namesdyn.obj
 0004:000052b0       ?KILLSICON@@3HA            007172b0     namesdyn.obj
 0004:000052b4       ?FIRSTAID_ICON@@3HA        007172b4     namesdyn.obj
 0004:000052b8       ?HEAT_ICON@@3HA            007172b8     namesdyn.obj
 0004:000052bc       ?BOTTOMSTATUSBAR@@3HA      007172bc     namesdyn.obj
 0004:000052c0       ?BOOT_ICON@@3HA            007172c0     namesdyn.obj
 0004:000052c4       ?FRAGBAR@@3HA              007172c4     namesdyn.obj
 0004:000052c8       ?JETPACK_ICON@@3HA         007172c8     namesdyn.obj
 0004:000052cc       ?AIRTANK_ICON@@3HA         007172cc     namesdyn.obj
 0004:000052d0       ?STEROIDS_ICON@@3HA        007172d0     namesdyn.obj
 0004:000052d4       ?HOLODUKE_ICON@@3HA        007172d4     namesdyn.obj
 0004:000052d8       ?ACCESS_ICON@@3HA          007172d8     namesdyn.obj
 0004:000052dc       ?DIGITALNUM@@3HA           007172dc     namesdyn.obj
 0004:000052e0       ?DUKECAR@@3HA              007172e0     namesdyn.obj
 0004:000052e4       ?CAMCORNER@@3HA            007172e4     namesdyn.obj
 0004:000052e8       ?CAMLIGHT@@3HA             007172e8     namesdyn.obj
 0004:000052ec       ?SLIDEBAR@@3HA             007172ec     namesdyn.obj
 0004:000052f0       ?DREALMS@@3HA              007172f0     namesdyn.obj
 0004:000052f4       ?BETASCREEN@@3HA           007172f4     namesdyn.obj
 0004:000052f8       ?WINDOWBORDER1@@3HA        007172f8     namesdyn.obj
 0004:000052fc       ?TEXTBOX@@3HA              007172fc     namesdyn.obj
 0004:00005300       ?WINDOWBORDER2@@3HA        00717300     namesdyn.obj
 0004:00005304       ?DUKENUKEM@@3HA            00717304     namesdyn.obj
 0004:00005308       ?THREEDEE@@3HA             00717308     namesdyn.obj
 0004:0000530c       ?INGAMEDUKETHREEDEE@@3HA   0071730c     namesdyn.obj
 0004:00005310       ?TENSCREEN@@3HA            00717310     namesdyn.obj
 0004:00005314       ?PLUTOPAKSPRITE@@3HA       00717314     namesdyn.obj
 0004:00005318       ?DEVISTATOR@@3HA           00717318     namesdyn.obj
 0004:0000531c       ?KNEE@@3HA                 0071731c     namesdyn.obj
 0004:00005320       ?CROSSHAIR@@3HA            00717320     namesdyn.obj
 0004:00005324       ?FIRSTGUN@@3HA             00717324     namesdyn.obj
 0004:00005328       ?FIRSTGUNRELOAD@@3HA       00717328     namesdyn.obj
 0004:0000532c       ?SHELL@@3HA                0071732c     namesdyn.obj
 0004:00005330       ?SHOTGUNSHELL@@3HA         00717330     namesdyn.obj
 0004:00005334       ?CHAINGUN@@3HA             00717334     namesdyn.obj
 0004:00005338       ?RPGGUN@@3HA               00717338     namesdyn.obj
 0004:0000533c       ?FREEZE@@3HA               0071733c     namesdyn.obj
 0004:00005340       ?SHRINKER@@3HA             00717340     namesdyn.obj
 0004:00005344       ?HANDHOLDINGLASER@@3HA     00717344     namesdyn.obj
 0004:00005348       ?TRIPBOMB@@3HA             00717348     namesdyn.obj
 0004:0000534c       ?LASERLINE@@3HA            0071734c     namesdyn.obj
 0004:00005350       ?HANDHOLDINGACCESS@@3HA    00717350     namesdyn.obj
 0004:00005354       ?HANDREMOTE@@3HA           00717354     namesdyn.obj
 0004:00005358       ?HANDTHROW@@3HA            00717358     namesdyn.obj
 0004:0000535c       ?TIP@@3HA                  0071735c     namesdyn.obj
 0004:00005360       ?SCUBAMASK@@3HA            00717360     namesdyn.obj
 0004:00005364       ?FORCESPHERE@@3HA          00717364     namesdyn.obj
 0004:00005368       ?SHOTSPARK1@@3HA           00717368     namesdyn.obj
 0004:0000536c       ?RPG@@3HA                  0071736c     namesdyn.obj
 0004:00005370       ?LASERSITE@@3HA            00717370     namesdyn.obj
 0004:00005374       ?SHOTGUN@@3HA              00717374     namesdyn.obj
 0004:00005378       ?BOSS1@@3HA                00717378     namesdyn.obj
 0004:0000537c       ?BOSS1STAYPUT@@3HA         0071737c     namesdyn.obj
 0004:00005380       ?BOSS1SHOOT@@3HA           00717380     namesdyn.obj
 0004:00005384       ?BOSS1LOB@@3HA             00717384     namesdyn.obj
 0004:00005388       ?BOSSTOP@@3HA              00717388     namesdyn.obj
 0004:0000538c       ?BOSS2@@3HA                0071738c     namesdyn.obj
 0004:00005390       ?BOSS3@@3HA                00717390     namesdyn.obj
 0004:00005394       ?SPINNINGNUKEICON@@3HA     00717394     namesdyn.obj
 0004:00005398       ?SMALLFNTCURSOR@@3HA       00717398     namesdyn.obj
 0004:0000539c       ?STARTALPHANUM@@3HA        0071739c     namesdyn.obj
 0004:000053a0       ?ENDALPHANUM@@3HA          007173a0     namesdyn.obj
 0004:000053a4       ?BIGALPHANUM@@3HA          007173a4     namesdyn.obj
 0004:000053a8       ?BIGPERIOD@@3HA            007173a8     namesdyn.obj
 0004:000053ac       ?BIGCOMMA@@3HA             007173ac     namesdyn.obj
 0004:000053b0       ?BIGX_@@3HA                007173b0     namesdyn.obj
 0004:000053b4       ?BIGQ@@3HA                 007173b4     namesdyn.obj
 0004:000053b8       ?BIGSEMI@@3HA              007173b8     namesdyn.obj
 0004:000053bc       ?BIGCOLIN@@3HA             007173bc     namesdyn.obj
 0004:000053c0       ?THREEBYFIVE@@3HA          007173c0     namesdyn.obj
 0004:000053c4       ?BIGAPPOS@@3HA             007173c4     namesdyn.obj
 0004:000053c8       ?MINIFONT@@3HA             007173c8     namesdyn.obj
 0004:000053cc       ?RESPAWNMARKERRED@@3HA     007173cc     namesdyn.obj
 0004:000053d0       ?RESPAWNMARKERYELLOW@@3HA  007173d0     namesdyn.obj
 0004:000053d4       ?RESPAWNMARKERGREEN@@3HA   007173d4     namesdyn.obj
 0004:000053d8       ?BONUSSCREEN@@3HA          007173d8     namesdyn.obj
 0004:000053dc       ?VIEWBORDER@@3HA           007173dc     namesdyn.obj
 0004:000053e0       ?VICTORY1@@3HA             007173e0     namesdyn.obj
 0004:000053e4       ?ORDERING@@3HA             007173e4     namesdyn.obj
 0004:000053e8       ?TEXTSTORY@@3HA            007173e8     namesdyn.obj
 0004:000053ec       ?LOADSCREEN@@3HA           007173ec     namesdyn.obj
 0004:000053f0       ?BORNTOBEWILDSCREEN@@3HA   007173f0     namesdyn.obj
 0004:000053f4       ?BLIMP@@3HA                007173f4     namesdyn.obj
 0004:000053f8       ?FEM9@@3HA                 007173f8     namesdyn.obj
 0004:000053fc       ?FRAMEEFFECT1_13@@3HA      007173fc     namesdyn.obj
 0004:00005400       ?FRAMEEFFECT1@@3HA         00717400     namesdyn.obj
 0004:00005404       ?PANNEL3@@3HA              00717404     namesdyn.obj
 0004:00005408       ?SCREENBREAK14@@3HA        00717408     namesdyn.obj
 0004:0000540c       ?SCREENBREAK15@@3HA        0071740c     namesdyn.obj
 0004:00005410       ?SCREENBREAK19@@3HA        00717410     namesdyn.obj
 0004:00005414       ?SCREENBREAK16@@3HA        00717414     namesdyn.obj
 0004:00005418       ?SCREENBREAK17@@3HA        00717418     namesdyn.obj
 0004:0000541c       ?SCREENBREAK18@@3HA        0071741c     namesdyn.obj
 0004:00005420       ?W_TECHWALL11@@3HA         00717420     namesdyn.obj
 0004:00005424       ?W_TECHWALL12@@3HA         00717424     namesdyn.obj
 0004:00005428       ?W_TECHWALL13@@3HA         00717428     namesdyn.obj
 0004:0000542c       ?W_TECHWALL14@@3HA         0071742c     namesdyn.obj
 0004:00005430       ?W_TECHWALL5@@3HA          00717430     namesdyn.obj
 0004:00005434       ?W_TECHWALL6@@3HA          00717434     namesdyn.obj
 0004:00005438       ?W_TECHWALL7@@3HA          00717438     namesdyn.obj
 0004:0000543c       ?W_TECHWALL8@@3HA          0071743c     namesdyn.obj
 0004:00005440       ?W_TECHWALL9@@3HA          00717440     namesdyn.obj
 0004:00005444       ?BPANNEL3@@3HA             00717444     namesdyn.obj
 0004:00005448       ?W_HITTECHWALL16@@3HA      00717448     namesdyn.obj
 0004:0000544c       ?W_HITTECHWALL10@@3HA      0071744c     namesdyn.obj
 0004:00005450       ?W_HITTECHWALL15@@3HA      00717450     namesdyn.obj
 0004:00005454       ?W_MILKSHELF@@3HA          00717454     namesdyn.obj
 0004:00005458       ?W_MILKSHELFBROKE@@3HA     00717458     namesdyn.obj
 0004:0000545c       ?PURPLELAVA@@3HA           0071745c     namesdyn.obj
 0004:00005460       ?TARGET@@3HA               00717460     namesdyn.obj
 0004:00005464       ?DUCK@@3HA                 00717464     namesdyn.obj
 0004:00005468       ?PUKE@@3HA                 00717468     namesdyn.obj
 0004:0000546c       ?DOORTILE23@@3HA           0071746c     namesdyn.obj
 0004:00005470       ?SPEAKER@@3HA              00717470     namesdyn.obj
 0004:00005474       ?MAIL@@3HA                 00717474     namesdyn.obj
 0004:00005478       ?HOTMEAT@@3HA              00717478     namesdyn.obj
 0004:0000547c       ?TRIPODCAMERA@@3HA         0071747c     namesdyn.obj
 0004:00005480       ?PAPER@@3HA                00717480     namesdyn.obj
 0004:00005484       ?GENERICPOLE2@@3HA         00717484     namesdyn.obj
 0004:00005488       ?XXXSTACY@@3HA             00717488     namesdyn.obj
 0004:0000548c       ?LETTER@@3HA               0071748c     namesdyn.obj
 0004:00005490       ?SIDEBOLT1@@3HA            00717490     namesdyn.obj
 0004:00005494       ?FOODOBJECT16@@3HA         00717494     namesdyn.obj
 0004:00005498       ?TAMPON@@3HA               00717498     namesdyn.obj
 0004:0000549c       ?CANWITHSOMETHING2@@3HA    0071749c     namesdyn.obj
 0004:000054a0       ?CANWITHSOMETHING3@@3HA    007174a0     namesdyn.obj
 0004:000054a4       ?CANWITHSOMETHING4@@3HA    007174a4     namesdyn.obj
 0004:000054a8       ?DOLPHIN1@@3HA             007174a8     namesdyn.obj
 0004:000054ac       ?DOLPHIN2@@3HA             007174ac     namesdyn.obj
 0004:000054b0       ?NEWBEAST@@3HA             007174b0     namesdyn.obj
 0004:000054b4       ?NEWBEASTSTAYPUT@@3HA      007174b4     namesdyn.obj
 0004:000054b8       ?BOSS4@@3HA                007174b8     namesdyn.obj
 0004:000054bc       ?BOSS4STAYPUT@@3HA         007174bc     namesdyn.obj
 0004:000054c0       ?FEM10@@3HA                007174c0     namesdyn.obj
 0004:000054c4       ?TOUGHGAL@@3HA             007174c4     namesdyn.obj
 0004:000054c8       ?MAN@@3HA                  007174c8     namesdyn.obj
 0004:000054cc       ?MAN2@@3HA                 007174cc     namesdyn.obj
 0004:000054d0       ?WOMAN@@3HA                007174d0     namesdyn.obj
 0004:000054d4       ?NATURALLIGHTNING@@3HA     007174d4     namesdyn.obj
 0004:000054d8       ?WEATHERWARN@@3HA          007174d8     namesdyn.obj
 0004:000054dc       ?DUKETAG@@3HA              007174dc     namesdyn.obj
 0004:000054e0       ?SIGN1@@3HA                007174e0     namesdyn.obj
 0004:000054e4       ?SIGN2@@3HA                007174e4     namesdyn.obj
 0004:000054e8       ?JURYGUY@@3HA              007174e8     namesdyn.obj
 0004:000054f4       ?g_netPort@@3GA            007174f4     net.obj
 0004:000054f8       ?g_netIndex@@3HA           007174f8     net.obj
 0004:00005500       ?g_netStatnums@@3PAFA      00717500     net.obj
 0004:00005510       _mouseyaxismode            00717510     player.obj
 0004:00005514       _WeaponPickupSprites       00717514     player.obj
 0004:000055b0       _s_buildRev                007175b0     rev.obj
 0004:000055b4       _s_buildTimestamp          007175b4     rev.obj
 0004:000055b8       _gamefunctions             007175b8     config.obj
 0004:00005cb8       _keydefaults               00717cb8     config.obj
 0004:00007378       _h_gamefuncs               00719378     config.obj
 0004:00007380       ?osdhightile@@3HA          00719380     osdfuncs.obj
 0004:00007384       ?osdscale@@3MA             00719384     osdfuncs.obj
 0004:00007388       ?osdrscale@@3MA            00719388     osdfuncs.obj
 0004:0000738c       _r_ambientlight            0071938c     osdcmds.obj
 0004:00007390       _r_ambientlightrecip       00719390     osdcmds.obj
 0004:00007398       ?controlstrings@@3PAPBDA   00719398     startwin.game.obj
 0004:000073bc       _CONTROL_MouseSensitivity  007193bc     control.obj
 0004:000076ec       ?PISTOL_RICOCHET@@3HA      007196ec     soundsdyn.obj
 0004:000076f0       ?PISTOL_BODYHIT@@3HA       007196f0     soundsdyn.obj
 0004:000076f4       ?PISTOL_FIRE@@3HA          007196f4     soundsdyn.obj
 0004:000076f8       ?EJECT_CLIP@@3HA           007196f8     soundsdyn.obj
 0004:000076fc       ?INSERT_CLIP@@3HA          007196fc     soundsdyn.obj
 0004:00007700       ?CHAINGUN_FIRE@@3HA        00719700     soundsdyn.obj
 0004:00007704       ?RPG_SHOOT@@3HA            00719704     soundsdyn.obj
 0004:00007708       ?POOLBALLHIT@@3HA          00719708     soundsdyn.obj
 0004:0000770c       ?RPG_EXPLODE@@3HA          0071970c     soundsdyn.obj
 0004:00007710       ?CAT_FIRE@@3HA             00719710     soundsdyn.obj
 0004:00007714       ?SHRINKER_FIRE@@3HA        00719714     soundsdyn.obj
 0004:00007718       ?PIPEBOMB_BOUNCE@@3HA      00719718     soundsdyn.obj
 0004:0000771c       ?PIPEBOMB_EXPLODE@@3HA     0071971c     soundsdyn.obj
 0004:00007720       ?LASERTRIP_ONWALL@@3HA     00719720     soundsdyn.obj
 0004:00007724       ?LASERTRIP_ARMING@@3HA     00719724     soundsdyn.obj
 0004:00007728       ?LASERTRIP_EXPLODE@@3HA    00719728     soundsdyn.obj
 0004:0000772c       ?VENT_BUST@@3HA            0071972c     soundsdyn.obj
 0004:00007730       ?GLASS_BREAKING@@3HA       00719730     soundsdyn.obj
 0004:00007734       ?GLASS_HEAVYBREAK@@3HA     00719734     soundsdyn.obj
 0004:00007738       ?SHORT_CIRCUIT@@3HA        00719738     soundsdyn.obj
 0004:0000773c       ?ITEM_SPLASH@@3HA          0071973c     soundsdyn.obj
 0004:00007740       ?DUKE_GASP@@3HA            00719740     soundsdyn.obj
 0004:00007744       ?SLIM_RECOG@@3HA           00719744     soundsdyn.obj
 0004:00007748       ?DUKE_URINATE@@3HA         00719748     soundsdyn.obj
 0004:0000774c       ?ENDSEQVOL3SND2@@3HA       0071974c     soundsdyn.obj
 0004:00007750       ?ENDSEQVOL3SND3@@3HA       00719750     soundsdyn.obj
 0004:00007754       ?DUKE_CRACK@@3HA           00719754     soundsdyn.obj
 0004:00007758       ?SLIM_ATTACK@@3HA          00719758     soundsdyn.obj
 0004:0000775c       ?SOMETHINGHITFORCE@@3HA    0071975c     soundsdyn.obj
 0004:00007760       ?DUKE_DRINKING@@3HA        00719760     soundsdyn.obj
 0004:00007764       ?DUKE_GRUNT@@3HA           00719764     soundsdyn.obj
 0004:00007768       ?DUKE_HARTBEAT@@3HA        00719768     soundsdyn.obj
 0004:0000776c       ?DUKE_ONWATER@@3HA         0071976c     soundsdyn.obj
 0004:00007770       ?DUKE_LAND@@3HA            00719770     soundsdyn.obj
 0004:00007774       ?DUKE_WALKINDUCTS@@3HA     00719774     soundsdyn.obj
 0004:00007778       ?DUKE_UNDERWATER@@3HA      00719778     soundsdyn.obj
 0004:0000777c       ?DUKE_JETPACK_ON@@3HA      0071977c     soundsdyn.obj
 0004:00007780       ?DUKE_JETPACK_IDLE@@3HA    00719780     soundsdyn.obj
 0004:00007784       ?DUKE_JETPACK_OFF@@3HA     00719784     soundsdyn.obj
 0004:00007788       ?DUKETALKTOBOSS@@3HA       00719788     soundsdyn.obj
 0004:0000778c       ?SQUISHED@@3HA             0071978c     soundsdyn.obj
 0004:00007790       ?TELEPORTER@@3HA           00719790     soundsdyn.obj
 0004:00007794       ?ELEVATOR_ON@@3HA          00719794     soundsdyn.obj
 0004:00007798       ?ELEVATOR_OFF@@3HA         00719798     soundsdyn.obj
 0004:0000779c       ?SUBWAY@@3HA               0071979c     soundsdyn.obj
 0004:000077a0       ?SWITCH_ON@@3HA            007197a0     soundsdyn.obj
 0004:000077a4       ?FLUSH_TOILET@@3HA         007197a4     soundsdyn.obj
 0004:000077a8       ?EARTHQUAKE@@3HA           007197a8     soundsdyn.obj
 0004:000077ac       ?END_OF_LEVEL_WARN@@3HA    007197ac     soundsdyn.obj
 0004:000077b0       ?WIND_AMBIENCE@@3HA        007197b0     soundsdyn.obj
 0004:000077b4       ?SOMETHING_DRIPPING@@3HA   007197b4     soundsdyn.obj
 0004:000077b8       ?BOS1_RECOG@@3HA           007197b8     soundsdyn.obj
 0004:000077bc       ?BOS2_RECOG@@3HA           007197bc     soundsdyn.obj
 0004:000077c0       ?DUKE_GETWEAPON2@@3HA      007197c0     soundsdyn.obj
 0004:000077c4       ?SHOTGUN_FIRE@@3HA         007197c4     soundsdyn.obj
 0004:000077c8       ?PRED_RECOG@@3HA           007197c8     soundsdyn.obj
 0004:000077cc       ?CAPT_RECOG@@3HA           007197cc     soundsdyn.obj
 0004:000077d0       ?PIG_RECOG@@3HA            007197d0     soundsdyn.obj
 0004:000077d4       ?RECO_ROAM@@3HA            007197d4     soundsdyn.obj
 0004:000077d8       ?RECO_RECOG@@3HA           007197d8     soundsdyn.obj
 0004:000077dc       ?RECO_ATTACK@@3HA          007197dc     soundsdyn.obj
 0004:000077e0       ?RECO_PAIN@@3HA            007197e0     soundsdyn.obj
 0004:000077e4       ?DRON_RECOG@@3HA           007197e4     soundsdyn.obj
 0004:000077e8       ?COMM_RECOG@@3HA           007197e8     soundsdyn.obj
 0004:000077ec       ?OCTA_RECOG@@3HA           007197ec     soundsdyn.obj
 0004:000077f0       ?TURR_RECOG@@3HA           007197f0     soundsdyn.obj
 0004:000077f4       ?SLIM_DYING@@3HA           007197f4     soundsdyn.obj
 0004:000077f8       ?BOS3_RECOG@@3HA           007197f8     soundsdyn.obj
 0004:000077fc       ?BOS1_WALK@@3HA            007197fc     soundsdyn.obj
 0004:00007800       ?THUD@@3HA                 00719800     soundsdyn.obj
 0004:00007804       ?WIERDSHOT_FLY@@3HA        00719804     soundsdyn.obj
 0004:00007808       ?SLIM_ROAM@@3HA            00719808     soundsdyn.obj
 0004:0000780c       ?SHOTGUN_COCK@@3HA         0071980c     soundsdyn.obj
 0004:00007810       ?GENERIC_AMBIENCE17@@3HA   00719810     soundsdyn.obj
 0004:00007814       ?BONUS_SPEECH1@@3HA        00719814     soundsdyn.obj
 0004:00007818       ?BONUS_SPEECH2@@3HA        00719818     soundsdyn.obj
 0004:0000781c       ?BONUS_SPEECH3@@3HA        0071981c     soundsdyn.obj
 0004:00007820       ?BONUS_SPEECH4@@3HA        00719820     soundsdyn.obj
 0004:00007824       ?DUKE_LAND_HURT@@3HA       00719824     soundsdyn.obj
 0004:00007828       ?DUKE_SEARCH2@@3HA         00719828     soundsdyn.obj
 0004:0000782c       ?DUKE_CRACK2@@3HA          0071982c     soundsdyn.obj
 0004:00007830       ?DUKE_SEARCH@@3HA          00719830     soundsdyn.obj
 0004:00007834       ?DUKE_GET@@3HA             00719834     soundsdyn.obj
 0004:00007838       ?DUKE_LONGTERM_PAIN@@3HA   00719838     soundsdyn.obj
 0004:0000783c       ?MONITOR_ACTIVE@@3HA       0071983c     soundsdyn.obj
 0004:00007840       ?NITEVISION_ONOFF@@3HA     00719840     soundsdyn.obj
 0004:00007844       ?DUKE_CRACK_FIRST@@3HA     00719844     soundsdyn.obj
 0004:00007848       ?DUKE_USEMEDKIT@@3HA       00719848     soundsdyn.obj
 0004:0000784c       ?DUKE_TAKEPILLS@@3HA       0071984c     soundsdyn.obj
 0004:00007850       ?DUKE_PISSRELIEF@@3HA      00719850     soundsdyn.obj
 0004:00007854       ?SELECT_WEAPON@@3HA        00719854     soundsdyn.obj
 0004:00007858       ?JIBBED_ACTOR5@@3HA        00719858     soundsdyn.obj
 0004:0000785c       ?JIBBED_ACTOR6@@3HA        0071985c     soundsdyn.obj
 0004:00007860       ?DUKE_GOTHEALTHATLOW@@3HA  00719860     soundsdyn.obj
 0004:00007864       ?BOSSTALKTODUKE@@3HA       00719864     soundsdyn.obj
 0004:00007868       ?WAR_AMBIENCE2@@3HA        00719868     soundsdyn.obj
 0004:0000786c       ?EXITMENUSOUND@@3HA        0071986c     soundsdyn.obj
 0004:00007870       ?FLY_BY@@3HA               00719870     soundsdyn.obj
 0004:00007874       ?DUKE_SCREAM@@3HA          00719874     soundsdyn.obj
 0004:00007878       ?SHRINKER_HIT@@3HA         00719878     soundsdyn.obj
 0004:0000787c       ?RATTY@@3HA                0071987c     soundsdyn.obj
 0004:00007880       ?BONUSMUSIC@@3HA           00719880     soundsdyn.obj
 0004:00007884       ?ALIEN_SWITCH1@@3HA        00719884     soundsdyn.obj
 0004:00007888       ?RIPHEADNECK@@3HA          00719888     soundsdyn.obj
 0004:0000788c       ?ENDSEQVOL3SND4@@3HA       0071988c     soundsdyn.obj
 0004:00007890       ?ENDSEQVOL3SND5@@3HA       00719890     soundsdyn.obj
 0004:00007894       ?ENDSEQVOL3SND6@@3HA       00719894     soundsdyn.obj
 0004:00007898       ?ENDSEQVOL3SND7@@3HA       00719898     soundsdyn.obj
 0004:0000789c       ?ENDSEQVOL3SND8@@3HA       0071989c     soundsdyn.obj
 0004:000078a0       ?ENDSEQVOL3SND9@@3HA       007198a0     soundsdyn.obj
 0004:000078a4       ?WHIPYOURASS@@3HA          007198a4     soundsdyn.obj
 0004:000078a8       ?ENDSEQVOL2SND1@@3HA       007198a8     soundsdyn.obj
 0004:000078ac       ?ENDSEQVOL2SND2@@3HA       007198ac     soundsdyn.obj
 0004:000078b0       ?ENDSEQVOL2SND3@@3HA       007198b0     soundsdyn.obj
 0004:000078b4       ?ENDSEQVOL2SND4@@3HA       007198b4     soundsdyn.obj
 0004:000078b8       ?ENDSEQVOL2SND5@@3HA       007198b8     soundsdyn.obj
 0004:000078bc       ?ENDSEQVOL2SND6@@3HA       007198bc     soundsdyn.obj
 0004:000078c0       ?ENDSEQVOL2SND7@@3HA       007198c0     soundsdyn.obj
 0004:000078c4       ?SOMETHINGFROZE@@3HA       007198c4     soundsdyn.obj
 0004:000078c8       ?WIND_REPEAT@@3HA          007198c8     soundsdyn.obj
 0004:000078cc       ?BOS4_RECOG@@3HA           007198cc     soundsdyn.obj
 0004:000078d0       ?LIGHTNING_SLAP@@3HA       007198d0     soundsdyn.obj
 0004:000078d4       ?THUNDER@@3HA              007198d4     soundsdyn.obj
 0004:000078d8       ?INTRO4_1@@3HA             007198d8     soundsdyn.obj
 0004:000078dc       ?INTRO4_2@@3HA             007198dc     soundsdyn.obj
 0004:000078e0       ?INTRO4_3@@3HA             007198e0     soundsdyn.obj
 0004:000078e4       ?INTRO4_4@@3HA             007198e4     soundsdyn.obj
 0004:000078e8       ?INTRO4_5@@3HA             007198e8     soundsdyn.obj
 0004:000078ec       ?INTRO4_6@@3HA             007198ec     soundsdyn.obj
 0004:000078f0       ?BOSS4_DEADSPEECH@@3HA     007198f0     soundsdyn.obj
 0004:000078f4       ?BOSS4_FIRSTSEE@@3HA       007198f4     soundsdyn.obj
 0004:000078f8       ?VOL4ENDSND1@@3HA          007198f8     soundsdyn.obj
 0004:000078fc       ?VOL4ENDSND2@@3HA          007198fc     soundsdyn.obj
 0004:00007900       ?EXPANDERSHOOT@@3HA        00719900     soundsdyn.obj
 0004:00007904       ?INTRO4_B@@3HA             00719904     soundsdyn.obj
 0004:00007908       ?BIGBANG@@3HA              00719908     soundsdyn.obj
 0004:00009d1c       ?sdlappicon@@3U0@A         0071bd1c     game_icon.obj
 0004:00009d34       ?MIDI_Tempo@@3HA           0071bd34     midi.obj
 0004:00009d38       ?MUSIC_SoundDevice@@3HA    0071bd38     music.obj
 0004:00009d48       _mouseinwindow             0071bd48     baselayer.obj
 0004:00009d49       _AppMouseGrab              0071bd49     baselayer.obj
 0004:00009d50       _scantoasc                 0071bd50     baselayer.obj
 0004:00009dd0       _defaultres                0071bdd0     baselayer.obj
 0004:00009e78       _glinfo                    0071be78     baselayer.obj
 0004:00009ea4       _flushlogwindow            0071bea4     baselayer.obj
 0004:00009ea8       _toupperlookup             0071bea8     cache1d.obj
 0004:0000a0d4       _s_buildInfo               0071c0d4     common.obj
 0004:0000a108       ?mapversion@@3HA           0071c108     engine.obj
 0004:0000a10c       _g_loadedMapVersion        0071c10c     engine.obj
 0004:0000a110       _pskybits_override         0071c110     engine.obj
 0004:0000a114       _usevoxels                 0071c114     engine.obj
 0004:0000a118       _novoxmips                 0071c118     engine.obj
 0004:0000a11c       _editorgridextent          0071c11c     engine.obj
 0004:0000a134       _r_usenewaspect            0071c134     engine.obj
 0004:0000a138       _vid_gamma                 0071c138     engine.obj
 0004:0000a13c       _vid_contrast              0071c13c     engine.obj
 0004:0000a140       _engineerrstr              0071c140     engine.obj
 0004:0000a144       _showheightindicators      0071c144     engine.obj
 0004:0000a148       _circlewall                0071c148     engine.obj
 0004:0000a14c       _showinnergray             0071c14c     engine.obj
 0004:0000a154       _yax_globalcf              0071c154     engine.obj
 0004:0000a158       _r_tror_nomaskpass         0071c158     engine.obj
 0004:0000a15c       _yax_globallev             0071c15c     engine.obj
 0004:0000a160       _yax_globalbunch           0071c160     engine.obj
 0004:0000a164       _m32_sideelev              0071c164     engine.obj
 0004:0000a168       _m32_sideang               0071c168     engine.obj
 0004:0000a170       _xdimen                    0071c170     engine.obj
 0004:0000a174       _fxdimen                   0071c174     engine.obj
 0004:0000a17c       _pointhighlight            0071c17c     engine.obj
 0004:0000a180       _linehighlight             0071c180     engine.obj
 0004:0000a184       _searchx                   0071c184     engine.obj
 0004:0000a188       _vgapal16                  0071c188     engine.obj
 0004:0000a590       _apptitle                  0071c590     engine.obj
 0004:0000a690       _basepaltable              0071c690     engine.obj
 0004:0000aa90       _clipmoveboxtracenum       0071ca90     engine.obj
 0004:0000aa94       _drawlinepat               0071ca94     engine.obj
 0004:0000ac38       _TEXCACHEFILE              0071cc38     texcache.obj
 0004:0000ad7c       ?kplib_yrbrend_func@@3P6AXHHPAH@ZA 0071cd7c     kplib.obj
 0004:0000ae08       _usemodels                 0071ce08     polymost.obj
 0004:0000ae0c       _usehightile               0071ce0c     polymost.obj
 0004:0000ae10       _shadescale                0071ce10     polymost.obj
 0004:0000ae14       _r_usenewshading           0071ce14     polymost.obj
 0004:0000ae18       _r_usetileshades           0071ce18     polymost.obj
 0004:0000ae20       _glfiltermodes             0071ce20     polymost.obj
 0004:0000ae68       _glanisotropy              0071ce68     polymost.obj
 0004:0000ae6c       _gltexfiltermode           0071ce6c     polymost.obj
 0004:0000ae70       _glusetexcompr             0071ce70     polymost.obj
 0004:0000ae74       _glusetexcache             0071ce74     polymost.obj
 0004:0000ae78       _glusememcache             0071ce78     polymost.obj
 0004:0000ae7c       _r_detailmapping           0071ce7c     polymost.obj
 0004:0000ae80       _r_glowmapping             0071ce80     polymost.obj
 0004:0000ae84       _glprojectionhacks         0071ce84     polymost.obj
 0004:0000ae88       _glrendmode                0071ce88     polymost.obj
 0004:0000ae8c       _r_fullbrights             0071ce8c     polymost.obj
 0004:0000ae90       _r_vertexarrays            0071ce90     polymost.obj
 0004:0000ae94       _r_vbos                    0071ce94     polymost.obj
 0004:0000ae98       _r_vbocount                0071ce98     polymost.obj
 0004:0000ae9c       _r_animsmoothing           0071ce9c     polymost.obj
 0004:0000aea0       _r_downsizevar             0071cea0     polymost.obj
 0004:0000aea4       _r_parallaxskyclamping     0071cea4     polymost.obj
 0004:0000aeb4       _pr_lighting               0071ceb4     polymer.obj
 0004:0000aeb8       _pr_normalmapping          0071ceb8     polymer.obj
 0004:0000aebc       _pr_specularmapping        0071cebc     polymer.obj
 0004:0000aec0       _pr_shadows                0071cec0     polymer.obj
 0004:0000aec4       _pr_shadowcount            0071cec4     polymer.obj
 0004:0000aec8       _pr_shadowdetail           0071cec8     polymer.obj
 0004:0000aecc       _pr_shadowfiltering        0071cecc     polymer.obj
 0004:0000aed0       _pr_maxlightpasses         0071ced0     polymer.obj
 0004:0000aed4       _pr_maxlightpriority       0071ced4     polymer.obj
 0004:0000aed8       _pr_fov                    0071ced8     polymer.obj
 0004:0000aedc       _pr_billboardingmode       0071cedc     polymer.obj
 0004:0000aee0       _pr_verbosity              0071cee0     polymer.obj
 0004:0000aee4       _pr_vbos                   0071cee4     polymer.obj
 0004:0000aee8       _pr_gpusmoothing           0071cee8     polymer.obj
 0004:0000aeec       _pr_parallaxscale          0071ceec     polymer.obj
 0004:0000aef0       _pr_specularpower          0071cef0     polymer.obj
 0004:0000aef4       _pr_specularfactor         0071cef4     polymer.obj
 0004:0000aef8       _pr_highpalookups          0071cef8     polymer.obj
 0004:0000aefc       _pr_artmapping             0071cefc     polymer.obj
 0004:0000af00       _pr_hudfov                 0071cf00     polymer.obj
 0004:0000af04       _r_pr_maxlightpasses       0071cf04     polymer.obj
 0004:0000af08       ?mapvbousage@@3IA          0071cf08     polymer.obj
 0004:0000af0c       ?modelvbousage@@3IA        0071cf0c     polymer.obj
 0004:0000af20       ?textfont@@3PADA           0071cf20     textfont.obj
 0004:0000b720       ?smalltextfont@@3PADA      0071d720     smalltextfont.obj
 0004:0000bf60       ?connectpoint2@@3PAHA      0071df60     mmulti_null.obj
 0004:0000bff0       ?backgroundidle@@3HA       0071dff0     winbits.obj
 0004:0000bffc       _appactive                 0071dffc     sdlayer.obj
 0004:0000bffd       ?modechange@@3DA           0071dffd     sdlayer.obj
 0004:0000c000       _xres                      0071e000     sdlayer.obj
 0004:0000c004       _yres                      0071e004     sdlayer.obj
 0004:0000c008       ?ASS_SoundDriver@@3HA      0071e008     drivers.obj
 0004:0000c064       ?MV_SampleSize@@3HA        0071e064     multivoc.obj
 0004:0000c068       _MV_ErrorCode              0071e068     multivoc.obj
 0004:0000c06c       ?loopStartTags@@3PAPBDA    0071e06c     multivoc.obj
 0004:0000c074       ?loopEndTags@@3PAPBDA      0071e074     multivoc.obj
 0004:0000c07c       ?loopLengthTags@@3PAPBDA   0071e07c     multivoc.obj
 0004:0000c9d8       _WINDOWS_bootstrap         0071e9d8     libSDL2:SDL_windowsvideo.o
 0004:0000c9e8       _g_WindowFrameUsableWhileCursorHidden 0071e9e8     libSDL2:SDL_windowsvideo.o
 0004:0000c9ec       _g_WindowsEnableMessageLoop 0071e9ec     libSDL2:SDL_windowsvideo.o
 0004:0000cb60       _D3D_RenderDriver          0071eb60     libSDL2:SDL_render_d3d.o
 0004:0000d5e0       _SDL_expand_byte           0071f5e0     libSDL2:SDL_pixels.o
 0004:0000e30c       _XAUDIO2_bootstrap         0072030c     libSDL2:SDL_xaudio2.o
 0004:0000e31c       _DSOUND_bootstrap          0072031c     libSDL2:SDL_directsound.o
 0004:0000e32c       _WINMM_bootstrap           0072032c     libSDL2:SDL_winmm.o
 0004:0000e33c       _DISKAUD_bootstrap         0072033c     libSDL2:SDL_diskaudio.o
 0004:0000e34c       _DUMMYAUD_bootstrap        0072034c     libSDL2:SDL_dummyaudio.o
 0004:0000e35c       _DUMMY_bootstrap           0072035c     libSDL2:SDL_nullvideo.o
 0004:0000e380       _GL_RenderDriver           00720380     libSDL2:SDL_render_gl.o
 0004:0000e3e0       _GLES2_RenderDriver        007203e0     libSDL2:SDL_render_gles2.o
 0004:0000e440       _SW_RenderDriver           00720440     libSDL2:SDL_render_sw.o
 0004:0000e4a0       _SDL_GeneratedBlitFuncTable 007204a0     libSDL2:SDL_blit_auto.o
 0004:0000f130       ___security_cookie         00721130     msvcrtd:gs_cookie.obj
 0004:0000f134       ___security_cookie_complement 00721134     msvcrtd:gs_cookie.obj
 0004:0000f140       ___globallocalestatus      00721140     msvcrtd:xthdloc.obj
 0004:0000f144       ___defaultmatherr          00721144     msvcrtd:merr.obj
 0004:0000f148       ___native_dllmain_reason   00721148     msvcrtd:natstart.obj
 0004:0000f14c       ___native_vcclrit_reason   0072114c     msvcrtd:natstart.obj
 0004:0000f230       _ror_protectedsectors      00721230     game.obj
 0004:00010230       _tempwallptr               00722230     game.obj
 0004:0001023c       _ticrandomseed             0072223c     game.obj
 0004:00010244       _g_quitDeadline            00722244     game.obj
 0004:00010248       _g_cameraDistance          00722248     game.obj
 0004:0001024c       _g_cameraClock             0072224c     game.obj
 0004:00010254       _g_noSetup                 00722254     game.obj
 0004:0001026c       _g_forceWeaponChoice       0072226c     game.obj
 0004:00010270       _g_fakeMultiMode           00722270     game.obj
 0004:00010274       _g_Debug                   00722274     game.obj
 0004:00010278       ?g_moveActorsTime@@3NA     00722278     game.obj
 0004:00010280       _boardfilename             00722280     game.obj
 0004:00010380       _currentboardfilename      00722380     game.obj
 0004:00010488       _g_rtsNamePtr              00722488     game.obj
 0004:0001048c       _g_Shareware               0072248c     game.obj
 0004:00010490       _g_levelTextTime           00722490     game.obj
 0004:00010494       _r_maxfps                  00722494     game.obj
 0004:00010498       _g_frameDelay              00722498     game.obj
 0004:0001049c       _DefaultCrosshairColors    0072249c     game.obj
 0004:000104a0       _g_crosshairSum            007224a0     game.obj
 0004:00010570       _otherp                    00722570     actors.obj
 0004:00010578       _block_deletesprite        00722578     actors.obj
 0004:00010798       ?g_animPtr@@3PAUdukeanim_t@@A 00722798     anim.obj
 0004:000109c4       ?althud_numberpal@@3HA     007229c4     sbar.obj
 0004:00010e5c       ?user_quote_time@@3PAHA    00722e5c     screentext.obj
 0004:00010e74       _quotebotgoal              00722e74     screentext.obj
 0004:00010e78       _quotebot                  00722e78     screentext.obj
 0004:00010e7c       ?minitext_yofs@@3HA        00722e7c     screentext.obj
 0004:00010e80       ?minitext_lowercase@@3HA   00722e80     screentext.obj
 0004:00010e98       _CommandPaths              00722e98     common.obj
 0004:00010e9c       _g_groupFileHandle         00722e9c     common.obj
 0004:00010ea0       _g_selectedGrp             00722ea0     common.obj
 0004:00010ea4       _CommandGrps               00722ea4     common.obj
 0004:00010ea8       _usecwd                    00722ea8     common.obj
 0004:00010fb0       _g_usingAddon              00722fb0     common.obj
 0004:00010fb4       _g_gameNamePtr             00722fb4     common.obj
 0004:00010fb8       _g_grpNamePtr              00722fb8     common.obj
 0004:00010fbc       _g_scriptNamePtr           00722fbc     common.obj
 0004:00010fc0       _g_scriptModules           00722fc0     common.obj
 0004:00010fc4       _g_scriptModulesNum        00722fc4     common.obj
 0004:000110c8       ?g_demo_totalCnt@@3HA      007230c8     demo.obj
 0004:00011ab8       ?g_demo_cnt@@3HA           00723ab8     demo.obj
 0004:00011af0       ?g_firstDemoFile@@3PADA    00723af0     demo.obj
 0004:00011bf0       ?g_demo_filePtr@@3PAU_iobuf@@A 00723bf0     demo.obj
 0004:00011bf4       ?g_demo_goalCnt@@3HA       00723bf4     demo.obj
 0004:00011bf8       ?g_demo_paused@@3HA        00723bf8     demo.obj
 0004:00011bfc       ?g_demo_rewind@@3HA        00723bfc     demo.obj
 0004:00011c00       ?demorec_force_cvar@@3HA   00723c00     demo.obj
 0004:00011c18       _DefaultProjectile         00723c18     gamedef.obj
 0004:00011c5c       _g_numCompilerWarnings     00723c5c     gamedef.obj
 0004:00011c64       _g_numCompilerErrors       00723c64     gamedef.obj
 0004:00011c68       _g_szBuf                   00723c68     gamedef.obj
 0004:00012278       _bitptr                    00724278     gamedef.obj
 0004:0001227c       _g_totalLines              0072427c     gamedef.obj
 0004:00012284       _g_lineNumber              00724284     gamedef.obj
 0004:000122a8       _g_numQuoteRedefinitions   007242a8     gamedef.obj
 0004:000122ac       _g_numProjectiles          007242ac     gamedef.obj
 0004:000122b0       _g_errorLineNum            007242b0     gameexec.obj
 0004:000122b4       _insptr                    007242b4     gameexec.obj
 0004:000122b8       _vm                        007242b8     gameexec.obj
 0004:000122d4       _g_tw                      007242d4     gameexec.obj
 0004:000122d8       _apScriptGameEvent         007242d8     gameexec.obj
 0004:00012550       _aplWeaponFlags            00724550     gamevars.obj
 0004:00012580       _aplWeaponTotalTime        00724580     gamevars.obj
 0004:000125b0       _aplWeaponShotsPerBurst    007245b0     gamevars.obj
 0004:000125e0       _aplWeaponSelectSound      007245e0     gamevars.obj
 0004:00012610       _aplWeaponFlashColor       00724610     gamevars.obj
 0004:00012640       _aplWeaponSound2Sound      00724640     gamevars.obj
 0004:00012670       _aplWeaponHoldDelay        00724670     gamevars.obj
 0004:000126a0       _aplWeaponReloadSound1     007246a0     gamevars.obj
 0004:000126d0       ?aGameArrays@@3PAUgamearray_t@@A 007246d0     gamevars.obj
 0004:000146d0       ?aGameVars@@3PAUgamevar_t@@A 007266d0     gamevars.obj
 0004:0001c6d4       _aplWeaponReload           0072e6d4     gamevars.obj
 0004:0001c704       _aplWeaponSpawn            0072e704     gamevars.obj
 0004:0001c734       _aplWeaponFireDelay        0072e734     gamevars.obj
 0004:0001c768       ?g_weaponOverridden@@3PAUweapondata_t@@A 0072e768     gamevars.obj
 0004:0001caf8       _aplWeaponShoots           0072eaf8     gamevars.obj
 0004:0001cb28       _aplWeaponSound2Time       0072eb28     gamevars.obj
 0004:0001cb58       _aplWeaponClip             0072eb58     gamevars.obj
 0004:0001cb88       _aplWeaponInitialSound     0072eb88     gamevars.obj
 0004:0001cbb8       _aplWeaponSpawnTime        0072ebb8     gamevars.obj
 0004:0001cbe8       _aplWeaponWorksLike        0072ebe8     gamevars.obj
 0004:0001cc18       _aplWeaponFireSound        0072ec18     gamevars.obj
 0004:0001cc48       _aplWeaponReloadSound2     0072ec48     gamevars.obj
 0004:0001cc78       ?g_gameVarCount@@3HA       0072ec78     gamevars.obj
 0004:0001cc7c       ?g_gameArrayCount@@3HA     0072ec7c     gamevars.obj
 0004:0001cc80       _g_numDefaultLabels        0072ec80     global.obj
 0004:0001cc84       _g_numClouds               0072ec84     global.obj
 0004:0001cc86       _g_numSkills               0072ec86     global.obj
 0004:0001cc87       _g_loadFromGroupOnly       0072ec87     global.obj
 0004:0001cc88       _inputfifo                 0072ec88     global.obj
 0004:0001ce08       _g_playerSpawnPoints       0072ee08     global.obj
 0004:0001cf08       _g_musicIndex              0072ef08     global.obj
 0004:0001cf0c       _g_freezerSelfDamage       0072ef0c     global.obj
 0004:0001cf10       _SpriteProjectile          0072ef10     global.obj
 0004:0011cf10       _MapInfo                   0082ef10     global.obj
 0004:0011ff10       _omyhoriz                  00831f10     global.obj
 0004:0011ff12       _pus                       00831f12     global.obj
 0004:0011ff13       _myhardlanding             00831f13     global.obj
 0004:0011ff14       _g_screenCapture           00831f14     global.obj
 0004:0011ff18       _g_scriptPtr               00831f18     global.obj
 0004:0011ff1c       _myhoriz                   00831f1c     global.obj
 0004:0011ff1e       _myreturntocenter          00831f1e     global.obj
 0004:0011ff1f       _g_numPlayerSprites        00831f1f     global.obj
 0004:0011ff20       _animategoal               00831f20     global.obj
 0004:00120f20       _neartaghitdist            00832f20     global.obj
 0004:00120f24       _g_curViewscreen           00832f24     global.obj
 0004:00120f26       _ready2send                00832f26     global.obj
 0004:00120f27       _pub                       00832f27     global.obj
 0004:00120f28       _recsync                   00832f28     global.obj
 0004:00128548       _animwall                  0083a548     global.obj
 0004:00128d48       _g_globalRandom            0083ad48     global.obj
 0004:00128d4a       _myonground                0083ad4a     global.obj
 0004:00128d4b       _myjumpingtoggle           0083ad4b     global.obj
 0004:00128d4c       _everyothertime            0083ad4c     global.obj
 0004:00128d50       _animatesect               0083ad50     global.obj
 0004:00129550       _avg                       0083b550     global.obj
 0004:0012955c       _script                    0083b55c     global.obj
 0004:00129560       _g_moveThingsCount         0083b560     global.obj
 0004:00129564       _myang                     0083b564     global.obj
 0004:00129568       _sbar                      0083b568     global.obj
 0004:001295cc       _g_numCyclers              0083b5cc     global.obj
 0004:001295d0       _lockclock                 0083b5d0     global.obj
 0004:001295d4       _startofdynamicinterpolations 0083b5d4     global.obj
 0004:001295d8       _playerswhenstarted        0083b5d8     global.obj
 0004:001295dc       _g_currentFrameRate        0083b5dc     global.obj
 0004:001295e0       _g_tile                    0083b5e0     global.obj
 0004:001dd5e0       _screenpeek                008ef5e0     global.obj
 0004:001dd5e4       _g_earthquakeTime          008ef5e4     global.obj
 0004:001dd5e8       _g_mirrorSector            008ef5e8     global.obj
 0004:001dd668       _cyclers                   008ef668     global.obj
 0004:001e0668       _g_musicSize               008f2668     global.obj
 0004:001e066c       _g_numLabels               008f266c     global.obj
 0004:001e0670       _g_mirrorWall              008f2670     global.obj
 0004:001e06f0       ?bakipos@@3PAHA            008f26f0     global.obj
 0004:001f06f0       _ScriptQuotes              009026f0     global.obj
 0004:002006f0       _myvel                     009126f0     global.obj
 0004:002006fc       _g_impactDamage            009126fc     global.obj
 0004:00200700       ?curipos@@3PAPAHA          00912700     global.obj
 0004:00210700       _omy                       00922700     global.obj
 0004:0021070c       _g_animateCount            0092270c     global.obj
 0004:00210710       _g_restorePalette          00922710     global.obj
 0004:00210714       _g_maxPlayerHealth         00922714     global.obj
 0004:00210718       _actor                     00922718     global.obj
 0004:00410718       _g_sounds                  00b22718     global.obj
 0004:0048c718       _clouds                    00b9e718     global.obj
 0004:0048c918       _g_scriptDebug             00b9e918     global.obj
 0004:0048c91c       _myhorizoff                00b9e91c     global.obj
 0004:0048c920       _ScriptQuoteRedefinitions  00b9e920     global.obj
 0004:0049c920       _packbuf                   00bae920     global.obj
 0004:004a4920       _menutextbuf               00bb6920     global.obj
 0004:004a49a0       _g_showShareware           00bb69a0     global.obj
 0004:004a49a4       _EpisodeFlags              00bb69a4     global.obj
 0004:004a49c0       _myjumpingcounter          00bb69c0     global.obj
 0004:004a49c4       _my                        00bb69c4     global.obj
 0004:004a49d0       _g_origins                 00bb69d0     global.obj
 0004:004a89d0       _loc                       00bba9d0     global.obj
 0004:004a89dc       _g_tripbombLaserMode       00bba9dc     global.obj
 0004:004a89e0       _szPlayerName              00bba9e0     global.obj
 0004:004a8a00       _cloudx                    00bbaa00     global.obj
 0004:004a8a04       _cloudtotalclock           00bbaa04     global.obj
 0004:004a9038       _tempbuf                   00bbb038     global.obj
 0004:004ab038       _g_spriteDeleteQueuePos    00bbd038     global.obj
 0004:004ab03c       _label                     00bbd03c     global.obj
 0004:004ab040       _typebuf                   00bbd040     global.obj
 0004:004ab0d0       _g_mirrorCount             00bbd0d0     global.obj
 0004:004ab0d4       _labeltype                 00bbd0d4     global.obj
 0004:004ab0d8       ?oldipos@@3PAHA            00bbd0d8     global.obj
 0004:004bb0d8       _cloudy                    00bcd0d8     global.obj
 0004:004bb0dc       _mycursectnum              00bcd0dc     global.obj
 0004:004bb0e0       _SpriteDeletionQueue       00bcd0e0     global.obj
 0004:004bb8e0       _g_damageCameras           00bcd8e0     global.obj
 0004:004bb8e4       _g_startArmorAmount        00bcd8e4     global.obj
 0004:004bb8e8       _buf                       00bcd8e8     global.obj
 0004:004bbce8       _animateptr                00bcdce8     global.obj
 0004:004bcce8       _g_gameQuit                00bcece8     global.obj
 0004:004bccec       ?g_interpolationLock@@3HA  00bcecec     global.obj
 0004:004bccf0       _ototalclock               00bcecf0     global.obj
 0004:004bccf4       _omyang                    00bcecf4     global.obj
 0004:004bccf8       _ud                        00bcecf8     global.obj
 0004:004bd51c       ?g_numInterpolations@@3HA  00bcf51c     global.obj
 0004:004bd520       _animatevel                00bcf520     global.obj
 0004:004be520       _g_numAnimWalls            00bd0520     global.obj
 0004:004be524       _g_noEnemies               00bd0524     global.obj
 0004:004be528       _labelcode                 00bd0528     global.obj
 0004:004be52c       _duke3d_globalflags        00bd052c     global.obj
 0004:004be530       _g_soundlocks              00bd0530     global.obj
 0004:004bf530       _omyhorizoff               00bd1530     global.obj
 0004:004bf534       _g_doQuickSave             00bd1534     global.obj
 0004:004bfa60       _m_menuchange_watchpoint   00bd1a60     menus.obj
 0004:004c0218       _g_currentMenu             00bd2218     menus.obj
 0004:004c128c       ?menufiltermode@@3HA       00bd328c     menus.obj
 0004:004c1c90       _m_mousewake_watchpoint    00bd3c90     menus.obj
 0004:004c1d80       _m_mouselastactivity       00bd3d80     menus.obj
 0004:004c33a4       ?m_mousecaught@@3HA        00bd53a4     menus.obj
 0004:004c33a8       _droidinput                00bd53a8     menus.obj
 0004:004c40c8       ?resolution@@3PAUresolution_t@@A 00bd60c8     menus.obj
 0004:004c6228       ?DynamicTileMap@@3PAFA     00bd8228     namesdyn.obj
 0004:004d6e00       ?g_netPassword@@3PADA      00be8e00     net.obj
 0004:004d6e20       ?tempMapDiff@@3Unetmapdiff_t@@A 00be8e20     net.obj
 0004:00716e30       ?pendingnewgame@@3Unewgame_t@@A 00e28e30     net.obj
 0004:00716e40       ?g_mapStateHistory@@3PAPAUnetmapstate_t@@A 00e28e40     net.obj
 0004:00716ff8       ?g_mapStartState@@3Unetmapstate_t@@A 00e28ff8     net.obj
 0004:00957000       ?tempnetbuf@@3PAEA         01069000     net.obj
 0004:00b97194       ?g_netServer@@3PAU_ENetHost@@A 012a9194     net.obj
 0004:00b97198       ?g_netClient@@3PAU_ENetHost@@A 012a9198     net.obj
 0004:00b9719c       ?g_netClientPeer@@3PAU_ENetPeer@@A 012a919c     net.obj
 0004:00b971a0       ?g_netDisconnect@@3HA      012a91a0     net.obj
 0004:00b971a4       ?g_netPlayersWaiting@@3HA  012a91a4     net.obj
 0004:00b971a8       ?g_networkMode@@3HA        012a91a8     net.obj
 0004:00b971ac       ?NET_75_CHECK@@3HA         012a91ac     net.obj
 0004:00b971b0       ?g_netMapRevision@@3IA     012a91b0     net.obj
 0004:00b971d4       ?lastvisinc@@3HA           012a91d4     player.obj
 0004:00b971d8       _hudweap                   012a91d8     player.obj
 0004:00b971f8       _g_numObituaries           012a91f8     player.obj
 0004:00b971fc       _g_numSelfObituaries       012a91fc     player.obj
 0004:00b97204       _g_myAimMode               012a9204     player.obj
 0004:00b97208       ?g_myAimStat@@3HA          012a9208     player.obj
 0004:00b9720c       ?g_oldAimStat@@3HA         012a920c     player.obj
 0004:00b97210       _g_emuJumpTics             012a9210     player.obj
 0004:00b97284       _g_halfScreen              012a9284     premap.obj
 0004:00b99098       _g_halveScreenArea         012ab098     premap.obj
 0004:00b998dc       _g_oldverSavegame          012ab8dc     savegame.obj
 0004:00b9cb1c       ?rts_lumplockbyte@@3PADA   012aeb1c     rts.obj
 0004:00b9cb68       ?osdshown@@3HA             012aeb68     osdfuncs.obj
 0004:00b9cb6c       _osdcmd_cheatsinfo_stat    012aeb6c     osdcmds.obj
 0004:00b9cb78       _cl_cheatmask              012aeb78     osdcmds.obj
 0004:00b9cb80       _foundgrps                 012aeb80     grpscan.obj
 0004:00b9cb84       _listgrps                  012aeb84     grpscan.obj
 0004:00b9d400       _CONTROL_OSDInput          012af400     control.obj
 0004:00b9d7b8       _CONTROL_KeyBinds          012af7b8     control.obj
 0004:00b9e3b8       _CONTROL_MouseBinds        012b03b8     control.obj
 0004:00b9e6e8       _CONTROL_JoyPresent        012b06e8     control.obj
 0004:00b9e6ec       _CONTROL_JoystickEnabled   012b06ec     control.obj
 0004:00b9e6f0       _CONTROL_MousePresent      012b06f0     control.obj
 0004:00b9e6f4       _CONTROL_MouseEnabled      012b06f4     control.obj
 0004:00b9e6f8       _CONTROL_ButtonState       012b06f8     control.obj
 0004:00b9e700       _CONTROL_ButtonHeldState   012b0700     control.obj
 0004:00b9e718       _CONTROL_Started           012b0718     control.obj
 0004:00b9e71c       _CONTROL_BindsEnabled      012b071c     control.obj
 0004:00b9e720       _CONTROL_SmoothMouse       012b0720     control.obj
 0004:00b9e730       _KB_LastScan               012b0730     keyboard.obj
 0004:00b9e78c       _g_numEnvSoundsPlaying     012b078c     sounds.obj
 0004:00b9e990       _g_maxSoundPos             012b0990     sounds.obj
 0004:00b9ebc8       ?DynamicSoundMap@@3PAFA    012b0bc8     soundsdyn.obj
 0004:00ba0bc8       ?KICK_HIT@@3HA             012b2bc8     soundsdyn.obj
 0004:00ba1248       ?m_szAppName@MiniDumper@@0PBDB 012b3248     mdump.obj
 0004:00ba124c       ?g_dumper@@3VMiniDumper@@A 012b324c     mdump.obj
 0004:00ba1298       ?MIDI_PatchMap@@3PADA      012b3298     midi.obj
 0004:00ba1328       ?_MIDI_GlobalPositionInTicks@@3IA 012b3328     midi.obj
 0004:00ba1334       ?_MIDI_PositionInTicks@@3IA 012b3334     midi.obj
 0004:00ba1388       ?MUSIC_ErrorCode@@3HA      012b3388     music.obj
 0004:00ba2164       ?_MPU_BuffersWaiting@@3HA  012b4164     mpu401.obj
 0004:00ba2170       _keyasciififoend           012b4170     baselayer.obj
 0004:00ba2171       _keyfifoplc                012b4171     baselayer.obj
 0004:00ba2172       _keyasciififoplc           012b4172     baselayer.obj
 0004:00ba2173       _mousepressstate           012b4173     baselayer.obj
 0004:00ba2174       _baselayer_osdcmd_vidmode_func 012b4174     baselayer.obj
 0004:00ba2178       _keyasciififo              012b4178     baselayer.obj
 0004:00ba21b8       _keyremap                  012b41b8     baselayer.obj
 0004:00ba22b8       _key_names                 012b42b8     baselayer.obj
 0004:00ba3ab8       _keystatus                 012b5ab8     baselayer.obj
 0004:00ba3bb8       _mouseabs                  012b5bb8     baselayer.obj
 0004:00ba3bc0       _keyfifo                   012b5bc0     baselayer.obj
 0004:00ba3c00       _keyfifoend                012b5c00     baselayer.obj
 0004:00ba3c01       _inputdevices              012b5c01     baselayer.obj
 0004:00ba3c02       _moustat                   012b5c02     baselayer.obj
 0004:00ba3c03       _mousegrab                 012b5c03     baselayer.obj
 0004:00ba3c04       _keyremapinit              012b5c04     baselayer.obj
 0004:00ba3c08       _mousex                    012b5c08     baselayer.obj
 0004:00ba3c0c       _mousey                    012b5c0c     baselayer.obj
 0004:00ba3c10       _mouseb                    012b5c10     baselayer.obj
 0004:00ba3c14       _joyaxis                   012b5c14     baselayer.obj
 0004:00ba3c18       _joyb                      012b5c18     baselayer.obj
 0004:00ba3c1c       _joyhat                    012b5c1c     baselayer.obj
 0004:00ba3c20       _joyisgamepad              012b5c20     baselayer.obj
 0004:00ba3c21       _joynumaxes                012b5c21     baselayer.obj
 0004:00ba3c22       _joynumbuttons             012b5c22     baselayer.obj
 0004:00ba3c23       _joynumhats                012b5c23     baselayer.obj
 0004:00ba3c24       _joyaxespresent            012b5c24     baselayer.obj
 0004:00ba3c28       _keypresscallback          012b5c28     baselayer.obj
 0004:00ba3c2c       _mousepresscallback        012b5c2c     baselayer.obj
 0004:00ba3c30       _joypresscallback          012b5c30     baselayer.obj
 0004:00bb4a90       _kpzbufsiz                 012c6a90     cache1d.obj
 0004:00bb4a94       ?fnofs@@3HA                012c6a94     cache1d.obj
 0004:00bb4a98       ?cac@@3PAUcactype@@A       012c6a98     cache1d.obj
 0004:00be0f80       _kpzbuf                    012f2f80     cache1d.obj
 0004:00be0f94       ?cacnum@@3HA               012f2f94     cache1d.obj
 0004:00be0fa0       _pathsearchmode            012f2fa0     cache1d.obj
 0004:00be0fa4       _numgroupfiles             012f2fa4     cache1d.obj
 0004:00be0fa8       ?check_filename_casing_fn@@3P6AHXZA 012f2fa8     cache1d.obj
 0004:00be0fb0       _g_defNamePtr              012f2fb0     common.obj
 0004:00be0fb4       _g_defModules              012f2fb4     common.obj
 0004:00be0fb8       _g_defModulesNum           012f2fb8     common.obj
 0004:00be0fbc       _g_clipMapFiles            012f2fbc     common.obj
 0004:00be0fc0       _g_clipMapFilesNum         012f2fc0     common.obj
 0004:00be0fd0       _crc32table                012f2fd0     crc32.obj
 0004:00bf2938       _globalshade               01304938     engine.obj
 0004:00bf293c       _totalclock                0130493c     engine.obj
 0004:00cb7140       _faketiledata              013c9140     engine.obj
 0004:00cd5140       _tilesiz                   013e7140     engine.obj
 0004:00d11148       _globalflags               01423148     engine.obj
 0004:00d1114c       _globaly2                  0142314c     engine.obj
 0004:00d11154       _mdinited                  01423154     engine.obj
 0004:00d1115c       _asm3                      0142315c     engine.obj
 0004:00d11160       _globalorientation         01423160     engine.obj
 0004:00d11164       _numsectors                01423164     engine.obj
 0004:00d11167       _redcol                    01423167     engine.obj
 0004:00d11188       _headspritestat            01423188     engine.obj
 0004:00d1198a       _paletteloaded             0142398a     engine.obj
 0004:00d11998       _gotsector                 01423998     engine.obj
 0004:00d11b98       _windowx2                  01423b98     engine.obj
 0004:00d11b9c       _sinviewingrangeglobalang  01423b9c     engine.obj
 0004:00d11ba0       _globalx1                  01423ba0     engine.obj
 0004:00d11ba4       _yxaspect                  01423ba4     engine.obj
 0004:00d427e8       _globalposz                014547e8     engine.obj
 0004:00d427ec       _singlobalang              014547ec     engine.obj
 0004:00d427f0       _g_loadedMapHack           014547f0     engine.obj
 0004:00d42c14       _fglobalposx               01454c14     engine.obj
 0004:00d42c18       _windowy1                  01454c18     engine.obj
 0004:00d42c20       _xdimenscale               01454c20     engine.obj
 0004:00d42c24       _randomseed                01454c24     engine.obj
 0004:00d42c28       _mdpause                   01454c28     engine.obj
 0004:00d42c30       _g_noFloorPal              01454c30     engine.obj
 0004:00d46d50       _vplce                     01458d50     engine.obj
 0004:00d46d60       _windowy2                  01458d60     engine.obj
 0004:00d46d64       _frameoffset               01458d64     engine.obj
 0004:00d66d68       ?sloptable@@3PAHA          01478d68     engine.obj
 0004:00d76d68       _h_ysize                   01488d68     engine.obj
 0004:00d85d6c       _windowy                   01497d6c     engine.obj
 0004:00d85d70       _numframes                 01497d70     engine.obj
 0004:00d85d74       _Numsprites                01497d74     engine.obj
 0004:00d8697c       _sector                    0149897c     engine.obj
 0004:00da4b80       _parallaxvisibility        014b6b80     engine.obj
 0004:00da4b88       _bunchlast                 014b6b88     engine.obj
 0004:00da7b90       _reciptable                014b9b90     engine.obj
 0004:00da9b90       _xyaspect                  014bbb90     engine.obj
 0004:00da9b94       _ydimen                    014bbb94     engine.obj
 0004:00da9b98       _palookup                  014bbb98     engine.obj
 0004:00da9f98       _thesector                 014bbf98     engine.obj
 0004:00dacf98       _picsiz                    014bef98     engine.obj
 0004:00db4798       _spritesmooth              014c6798     engine.obj
 0004:00db47a0       _ylookup                   014c67a0     engine.obj
 0004:00db47a8       _yax_gotsector             014c67a8     engine.obj
 0004:00db49a8       _parallaxyoffs_override    014c69a8     engine.obj
 0004:00db49b0       _totalclocklock            014c69b0     engine.obj
 0004:00db49c4       _cosglobalang              014c69c4     engine.obj
 0004:00db49ce       _numalphatabs              014c69ce     engine.obj
 0004:00db49cf       _whitecol                  014c69cf     engine.obj
 0004:00db49d0       _nextsectbunch             014c69d0     engine.obj
 0004:00db91d0       _show2dsector              014cb1d0     engine.obj
 0004:00db97d8       _spritesortcnt             014cb7d8     engine.obj
 0004:00db97de       _curbasepal                014cb7de     engine.obj
 0004:00db97e0       _searchit                  014cb7e0     engine.obj
 0004:00db97e2       _showinvisibility          014cb7e2     engine.obj
 0004:00db97e3       _parallaxtype              014cb7e3     engine.obj
 0004:00dbf7e8       _globalhoriz               014d17e8     engine.obj
 0004:00dbf7ec       _ydim16                    014d17ec     engine.obj
 0004:00e75bf0       _editorcolors              01587bf0     engine.obj
 0004:00ea7d18       _voxmodels                 015b9d18     engine.obj
 0004:00eabd18       _wall                      015bdd18     engine.obj
 0004:00eabd1c       _m32_sidecos               015bdd1c     engine.obj
 0004:00eb1d5c       _asm2                      015c3d5c     engine.obj
 0004:00eb1d60       _gotpic                    015c3d60     engine.obj
 0004:00eb2c60       ?voxoff@@3PAY04HA          015c4c60     engine.obj
 0004:00ec6c60       _xdimscale                 015d8c60     engine.obj
 0004:00ec6c64       _ydim                      015d8c64     engine.obj
 0004:00ec6c68       _headspritesect            015d8c68     engine.obj
 0004:00ec8c6a       _blackcol                  015dac6a     engine.obj
 0004:00ec8c6b       _display_mirror            015dac6b     engine.obj
 0004:00ec8c70       _headsectbunch             015dac70     engine.obj
 0004:00ef10cc       _globalposy                016030cc     engine.obj
 0004:00ef10d0       _maskwall                  016030d0     engine.obj
 0004:00ef40dc       _globalpisibility          016060dc     engine.obj
 0004:00ef58e0       _tspriteptr                016078e0     engine.obj
 0004:00ef98e4       _searchbottomwall          0160b8e4     engine.obj
 0004:00ef98e8       _nextmodelid               0160b8e8     engine.obj
 0004:00ef98ec       _espbak                    0160b8ec     engine.obj
 0004:00ef98f0       _halfxdim16                0160b8f0     engine.obj
 0004:00ef98f4       _yax_nomaskdidit           0160b8f4     engine.obj
 0004:00ef98f8       _waloff                    0160b8f8     engine.obj
 0004:00f178f8       _wallchanged               016298f8     engine.obj
 0004:00f280f8       _pskynummultis             0163a0f8     engine.obj
 0004:00f280fc       _m32_sidesin               0163a0fc     engine.obj
 0004:00f28104       _midydim16                 0163a104     engine.obj
 0004:00f28108       _thewall                   0163a108     engine.obj
 0004:00f2b108       _xb1                       0163d108     engine.obj
 0004:00f31108       _cosviewingrangeglobalang  01643108     engine.obj
 0004:00f31130       _prevspritesect            01643130     engine.obj
 0004:00f39130       _palookupfog               0164b130     engine.obj
 0004:00f39530       _globalcisibility          0164b530     engine.obj
 0004:00f39534       _globaly3                  0164b534     engine.obj
 0004:00f39538       _tiletovox                 0164b538     engine.obj
 0004:00f48538       _blendtable                0165a538     engine.obj
 0004:00f4897c       _debug1                    0165a97c     engine.obj
 0004:00f48980       _show2dwall                0165a980     engine.obj
 0004:00f491a4       _haveymost                 0165b1a4     engine.obj
 0004:00f491c4       _numyaxbunches             0165b1c4     engine.obj
 0004:00f491c8       _curpalettefaded           0165b1c8     engine.obj
 0004:00f495c8       ?sqrtable@@3PAGA           0165b5c8     engine.obj
 0004:00f4b5cc       _spriteext                 0165d5cc     engine.obj
 0004:00f4b5d0       _rx1                       0165d5d0     engine.obj
 0004:00f515d0       _numpages                  016635d0     engine.obj
 0004:00f515d8       _tile2model                016635d8     engine.obj
 0004:00ffa1d8       _show2dsprite              0170c1d8     engine.obj
 0004:00ffa9d8       _globalvisibility          0170c9d8     engine.obj
 0004:00ffa9dc       _numbunches                0170c9dc     engine.obj
 0004:00ffa9e0       _g_visibility              0170c9e0     engine.obj
 0004:00ffaa04       _editorzrange              0170ca04     engine.obj
 0004:00ffaa20       _windowx1                  0170ca20     engine.obj
 0004:00ffaa28       _spritecol2d               0170ca28     engine.obj
 0004:01009a28       _walock                    0171ba28     engine.obj
 0004:01011228       _numwalls                  01723228     engine.obj
 0004:01011230       _h_xoffs                   01723230     engine.obj
 0004:01018a30       _models                    0172aa30     engine.obj
 0004:01018a34       _globalang                 0172aa34     engine.obj
 0004:01018a38       _sprite                    0172aa38     engine.obj
 0004:01018a3c       _searchsector              0172aa3c     engine.obj
 0004:01018c50       _guniqhudid                0172ac50     engine.obj
 0004:01018c54       _globaltilesizy            0172ac54     engine.obj
 0004:01018c58       _bunchp2                   0172ac58     engine.obj
 0004:0101bc58       _graysectbitmap            0172dc58     engine.obj
 0004:0101be58       _debug2                    0172de58     engine.obj
 0004:0101be68       _h_xsize                   0172de68     engine.obj
 0004:0102ae6c       _searchwall                0173ce6c     engine.obj
 0004:0102ae70       _globalcursectnum          0173ce70     engine.obj
 0004:0102b678       _globalpal                 0173d678     engine.obj
 0004:0102b680       _curpalette                0173d680     engine.obj
 0004:0102ba80       _parallaxyscale_override   0173da80     engine.obj
 0004:0102ba88       _sintable                  0173da88     engine.obj
 0004:0102ca88       _tilecols                  0173ea88     engine.obj
 0004:01034288       _fglobalposz               01746288     engine.obj
 0004:010342cc       _validmodecnt              017462cc     engine.obj
 0004:0103a2d0       _validmode                 0174c2d0     engine.obj
 0004:0103b2d4       _usermaphacks              0174d2d4     engine.obj
 0004:0103b2d8       _palette                   0174d2d8     engine.obj
 0004:0103b5d8       _fglobalposy               0174d5d8     engine.obj
 0004:0103b5dc       _multipsky                 0174d5dc     engine.obj
 0004:0103b5e0       _numshades                 0174d5e0     engine.obj
 0004:0103b5e4       _xdim                      0174d5e4     engine.obj
 0004:0103b5e8       _spritechanged             0174d5e8     engine.obj
 0004:0104b628       _PaletteIndexFullbrights   0175d628     engine.obj
 0004:0105ce4c       _globalx3                  0176ee4c     engine.obj
 0004:01060e50       _bunchfirst                01772e50     engine.obj
 0004:01063e50       _num_usermaphacks          01775e50     engine.obj
 0004:01063e58       _nextspritestat            01775e58     engine.obj
 0004:0106be58       _h_yoffs                   0177de58     engine.obj
 0004:01073658       _yax_nextwall              01785658     engine.obj
 0004:01083658       _ebpbak                    01795658     engine.obj
 0004:0108365c       _startumost                0179565c     engine.obj
 0004:01083660       _palookupoffse             01795660     engine.obj
 0004:01083670       _faketile                  01795670     engine.obj
 0004:01089570       _picanm                    0179b570     engine.obj
 0004:010a7574       _searchy                   017b9574     engine.obj
 0004:010a7578       _globvis                   017b9578     engine.obj
 0004:010a757c       _globalpicnum              017b957c     engine.obj
 0004:010a7580       _m32_wallsprite            017b9580     engine.obj
 0004:010b7584       _bufplce                   017c9584     engine.obj
 0004:010b7594       _g_rotatespriteNoWidescreen 017c9594     engine.obj
 0004:010b7598       _tsprite                   017c9598     engine.obj
 0004:010b759c       _startdmost                017c959c     engine.obj
 0004:010bcea0       ?shlookup@@3PAGA           017ceea0     engine.obj
 0004:010bf0a0       _halfxdimen                017d10a0     engine.obj
 0004:010bf0a8       _g_pskyidx                 017d10a8     engine.obj
 0004:010bf0ac       _searchisbottom            017d10ac     engine.obj
 0004:010bf0b0       _globalhisibility          017d10b0     engine.obj
 0004:010bf0b4       _windowpos                 017d10b4     engine.obj
 0004:0114b0bc       _numscans                  0185d0bc     engine.obj
 0004:011518c0       _voxscale                  018638c0     engine.obj
 0004:011558c0       _multipskytile             018678c0     engine.obj
 0004:011558c4       _m32_swcnt                 018678c4     engine.obj
 0004:011558c8       _tailspritefree            018678c8     engine.obj
 0004:011558cc       _globalposx                018678cc     engine.obj
 0004:011558d0       _yax_bunchnum              018678d0     engine.obj
 0004:011598d0       _britable                  0186b8d0     engine.obj
 0004:0116b2e0       _ry1                       0187d2e0     engine.obj
 0004:0117e2fc       _vince                     018902fc     engine.obj
 0004:0117e310       _fpuasm                    01890310     engine.obj
 0004:0117e318       _sectorborder              01890318     engine.obj
 0004:0117e51c       _searchstat                0189051c     engine.obj
 0004:0118d540       _graywallbitmap            0189f540     engine.obj
 0004:0118dd40       _prevspritestat            0189fd40     engine.obj
 0004:01195d40       _nextspritesect            018a7d40     engine.obj
 0004:0119dd44       _maskwallcnt               018afd44     engine.obj
 0004:0119dd48       _asm4                      018afd48     engine.obj
 0004:0119dd4c       _windowx                   018afd4c     engine.obj
 0004:0119dd50       _asm1                      018afd50     engine.obj
 0004:0119dd58       _m32_wallscreenxy          018afd58     engine.obj
 0004:011c7df8       _sectorchanged             018d9df8     engine.obj
 0004:011cbe04       _viewingrange              018dde04     engine.obj
 0004:011cbe08       _xdimenrecip               018dde08     engine.obj
 0004:011cbe0d       _inpreparemirror           018dde0d     engine.obj
 0004:011cbe0e       _palfadedelta              018dde0e     engine.obj
 0004:011cbe14       _newaspect_enable          018dde14     engine.obj
 0004:011cbe18       _r_screenxy                018dde18     engine.obj
 0004:011cbe1c       _curbrightness             018dde1c     engine.obj
 0004:011cbe20       _gammabrightness           018dde20     engine.obj
 0004:011cbe24       _vid_brightness            018dde24     engine.obj
 0004:011cbe34       _showfirstwall             018dde34     engine.obj
 0004:011cbe3c       _editstatus                018dde3c     engine.obj
 0004:011cbe40       _numgraysects              018dde40     engine.obj
 0004:011cbe44       _autogray                  018dde44     engine.obj
 0004:011cbe48       _g_nodraw                  018dde48     engine.obj
 0004:011cbe4c       _scansector_retfast        018dde4c     engine.obj
 0004:011cbe50       _yax_nomaskpass            018dde50     engine.obj
 0004:011cbe60       _m32_sideview              018dde60     engine.obj
 0004:011cbe68       _chsecptr_onextwall        018dde68     engine.obj
 0004:011cbe74       _qsetmode                  018dde74     engine.obj
 0004:011cbe78       _highlightcnt              018dde78     engine.obj
 0004:011cbe7c       _hitallsprites             018dde7c     engine.obj
 0004:011cbe88       ?capturecount@@3FA         018dde88     engine.obj
 0004:011cbe94       _palfadergb                018dde94     engine.obj
 0004:011cbea0       _g_maskDrawMode            018ddea0     engine.obj
 0004:011cbea8       _setaspect_new_use_dimen   018ddea8     engine.obj
 0004:011e4a14       ?bglGetFloatv@@3P6GXIPAM@ZA 018f6a14     glbuild.obj
 0004:011e4a18       ?bglDebugMessageControlARB@@3P6GXIIIHPBIE@ZA 018f6a18     glbuild.obj
 0004:011e4a1c       ?bglDeleteTextures@@3P6GXHPBI@ZA 018f6a1c     glbuild.obj
 0004:011e4a20       ?bglReadBuffer@@3P6GXI@ZA  018f6a20     glbuild.obj
 0004:011e4a24       ?bglPushAttrib@@3P6GXI@ZA  018f6a24     glbuild.obj
 0004:011e4a28       ?bglLinkProgramARB@@3P6GXI@ZA 018f6a28     glbuild.obj
 0004:011e4a2c       ?bglVertexAttrib4NubARB@@3P6GXIEEEE@ZA 018f6a2c     glbuild.obj
 0004:011e4a30       ?bglGetAttachedObjectsARB@@3P6GXIHPAHPAI@ZA 018f6a30     glbuild.obj
 0004:011e4a34       ?bglGenFramebuffersEXT@@3P6GXHPAI@ZA 018f6a34     glbuild.obj
 0004:011e4a38       ?bgluTessBeginPolygon@@3P6GXPAVGLUtesselator@@PAX@ZA 018f6a38     glbuild.obj
 0004:011e4a3c       ?bglUniform4ivARB@@3P6GXHHPBH@ZA 018f6a3c     glbuild.obj
 0004:011e4a40       ?bglUniform2fvARB@@3P6GXHHPBM@ZA 018f6a40     glbuild.obj
 0004:011e4a44       ?bglPushMatrix@@3P6GXXZA   018f6a44     glbuild.obj
 0004:011e4a48       ?bglEndList@@3P6GXXZA      018f6a48     glbuild.obj
 0004:011e4a4c       ?bglUniform1iARB@@3P6GXHH@ZA 018f6a4c     glbuild.obj
 0004:011e4a50       ?bglShaderSourceARB@@3P6GXIHPAPBDPBH@ZA 018f6a50     glbuild.obj
 0004:011e4a54       ?bglVertexAttrib3dARB@@3P6GXINNN@ZA 018f6a54     glbuild.obj
 0004:011e4a58       ?bglGetUniformfvARB@@3P6GXIHPAM@ZA 018f6a58     glbuild.obj
 0004:011e4a5c       ?bglGetQueryObjectivARB@@3P6GXIIPAH@ZA 018f6a5c     glbuild.obj
 0004:011e4a60       ?bglBindAttribLocationARB@@3P6GXIIPBD@ZA 018f6a60     glbuild.obj
 0004:011e4a64       ?bgluDeleteTess@@3P6GXPAVGLUtesselator@@@ZA 018f6a64     glbuild.obj
 0004:011e4a68       ?bglVertex3dv@@3P6GXPBN@ZA 018f6a68     glbuild.obj
 0004:011e4a6c       ?bglVertexAttrib3fvARB@@3P6GXIPBM@ZA 018f6a6c     glbuild.obj
 0004:011e4a70       ?bglColor4ub@@3P6GXEEEE@ZA 018f6a70     glbuild.obj
 0004:011e4a74       ?bglLoadIdentity@@3P6GXXZA 018f6a74     glbuild.obj
 0004:011e4a78       ?bglGetString@@3P6GPBEI@ZA 018f6a78     glbuild.obj
 0004:011e4a7c       ?bwglSwapIntervalEXT@@3P6GHH@ZA 018f6a7c     glbuild.obj
 0004:011e4a80       ?bglDeleteProgramsARB@@3P6GXHPBI@ZA 018f6a80     glbuild.obj
 0004:011e4a84       ?bglEnableClientState@@3P6GXI@ZA 018f6a84     glbuild.obj
 0004:011e4a88       ?bglColor3f@@3P6GXMMM@ZA   018f6a88     glbuild.obj
 0004:011e4a8c       ?bglDrawElements@@3P6GXIHIPBX@ZA 018f6a8c     glbuild.obj
 0004:011e4a90       ?bglGetAttribLocationARB@@3P6GHIPBD@ZA 018f6a90     glbuild.obj
 0004:011e4a94       ?bglVertexAttrib1dARB@@3P6GXIN@ZA 018f6a94     glbuild.obj
 0004:011e4a98       ?bglUniform4iARB@@3P6GXHHHHH@ZA 018f6a98     glbuild.obj
 0004:011e4a9c       ?bglBindFramebufferEXT@@3P6GXII@ZA 018f6a9c     glbuild.obj
 0004:011e4aa0       ?bglUniform2iARB@@3P6GXHHH@ZA 018f6aa0     glbuild.obj
 0004:011e4aa4       ?bglVertexAttrib4ubvARB@@3P6GXIPBE@ZA 018f6aa4     glbuild.obj
 0004:011e4aa8       ?bglMultiTexCoord2dARB@@3P6GXINN@ZA 018f6aa8     glbuild.obj
 0004:011e4aac       ?bglDrawBuffer@@3P6GXI@ZA  018f6aac     glbuild.obj
 0004:011e4ab0       ?bglPopMatrix@@3P6GXXZA    018f6ab0     glbuild.obj
 0004:011e4ab4       ?bgluTessEndContour@@3P6GXPAVGLUtesselator@@@ZA 018f6ab4     glbuild.obj
 0004:011e4ab8       ?bglGetObjectParameterfvARB@@3P6GXIIPAM@ZA 018f6ab8     glbuild.obj
 0004:011e4abc       ?bgluTessEndPolygon@@3P6GXPAVGLUtesselator@@@ZA 018f6abc     glbuild.obj
 0004:011e4ac0       ?bglFrustum@@3P6GXNNNNNN@ZA 018f6ac0     glbuild.obj
 0004:011e4ac4       ?bglVertexAttrib4ivARB@@3P6GXIPBH@ZA 018f6ac4     glbuild.obj
 0004:011e4ac8       ?bglEnable@@3P6GXI@ZA      018f6ac8     glbuild.obj
 0004:011e4acc       ?bglVertexAttrib4uivARB@@3P6GXIPBI@ZA 018f6acc     glbuild.obj
 0004:011e4ad0       ?bwglDeleteContext@@3P6GHPAUHGLRC__@@@ZA 018f6ad0     glbuild.obj
 0004:011e4ad4       ?bglEnableVertexAttribArrayARB@@3P6GXI@ZA 018f6ad4     glbuild.obj
 0004:011e4ad8       ?bglPolygonOffset@@3P6GXMM@ZA 018f6ad8     glbuild.obj
 0004:011e4adc       ?bglEnd@@3P6GXXZA          018f6adc     glbuild.obj
 0004:011e4ae0       ?bglGetUniformivARB@@3P6GXIHPAH@ZA 018f6ae0     glbuild.obj
 0004:011e4ae4       ?bglBufferDataARB@@3P6GXIHPBXI@ZA 018f6ae4     glbuild.obj
 0004:011e4ae8       ?bglNormalPointer@@3P6GXIHPBX@ZA 018f6ae8     glbuild.obj
 0004:011e4aec       ?bglVertexAttrib4fvARB@@3P6GXIPBM@ZA 018f6aec     glbuild.obj
 0004:011e4af0       ?bglDeleteQueriesARB@@3P6GXHPBI@ZA 018f6af0     glbuild.obj
 0004:011e4af4       ?bglFramebufferTexture2DEXT@@3P6GXIIIIH@ZA 018f6af4     glbuild.obj
 0004:011e4af8       ?bgluProject@@3P6GHNNNPBN0PBHPAN22@ZA 018f6af8     glbuild.obj
 0004:011e4afc       ?bglVertexAttrib4NbvARB@@3P6GXIPBC@ZA 018f6afc     glbuild.obj
 0004:011e4b00       ?bglDeleteObjectARB@@3P6GXI@ZA 018f6b00     glbuild.obj
 0004:011e4b04       ?bglGenProgramsARB@@3P6GXHPAI@ZA 018f6b04     glbuild.obj
 0004:011e4b08       ?bglGetCompressedTexImageARB@@3P6GXIHPAX@ZA 018f6b08     glbuild.obj
 0004:011e4b0c       ?bglRotatef@@3P6GXMMMM@ZA  018f6b0c     glbuild.obj
 0004:011e4b10       ?bglUniform2ivARB@@3P6GXHHPBH@ZA 018f6b10     glbuild.obj
 0004:011e4b14       ?bglUseProgramObjectARB@@3P6GXI@ZA 018f6b14     glbuild.obj
 0004:011e4b18       ?bglBindTexture@@3P6GXII@ZA 018f6b18     glbuild.obj
 0004:011e4b1c       ?bglTexCoordPointer@@3P6GXHIHPBX@ZA 018f6b1c     glbuild.obj
 0004:011e4b20       ?bglFogi@@3P6GXIH@ZA       018f6b20     glbuild.obj
 0004:011e4b24       ?bglEndQueryARB@@3P6GXI@ZA 018f6b24     glbuild.obj
 0004:011e4b28       ?bglScalef@@3P6GXMMM@ZA    018f6b28     glbuild.obj
 0004:011e4b2c       ?bglFrontFace@@3P6GXI@ZA   018f6b2c     glbuild.obj
 0004:011e4b30       ?bglClipPlane@@3P6GXIPBN@ZA 018f6b30     glbuild.obj
 0004:011e4b34       ?bglGetError@@3P6GIXZA     018f6b34     glbuild.obj
 0004:011e4b38       ?bgluTessBeginContour@@3P6GXPAVGLUtesselator@@@ZA 018f6b38     glbuild.obj
 0004:011e4b3c       ?bglVertexAttrib3fARB@@3P6GXIMMM@ZA 018f6b3c     glbuild.obj
 0004:011e4b40       ?bglGetVertexAttribivARB@@3P6GXIIPAH@ZA 018f6b40     glbuild.obj
 0004:011e4b44       ?bglGetActiveUniformARB@@3P6GXIIHPAH0PAIPAD@ZA 018f6b44     glbuild.obj
 0004:011e4b48       ?bglVertexAttrib4NuivARB@@3P6GXIPBI@ZA 018f6b48     glbuild.obj
 0004:011e4b4c       ?bglShadeModel@@3P6GXI@ZA  018f6b4c     glbuild.obj
 0004:011e4b50       ?bglDrawPixels@@3P6GXHHIIPBX@ZA 018f6b50     glbuild.obj
 0004:011e4b54       ?bglUniform4fvARB@@3P6GXHHPBM@ZA 018f6b54     glbuild.obj
 0004:011e4b58       ?bglGetVertexAttribfvARB@@3P6GXIIPAM@ZA 018f6b58     glbuild.obj
 0004:011e4b5c       ?bglCompressedTexImage2DARB@@3P6GXIHIHHHHPBX@ZA 018f6b5c     glbuild.obj
 0004:011e4b60       ?bglVertex2i@@3P6GXHH@ZA   018f6b60     glbuild.obj
 0004:011e4b64       ?bglCopyTexSubImage2D@@3P6GXIHHHHHHH@ZA 018f6b64     glbuild.obj
 0004:011e4b68       ?bglVertexAttrib3sARB@@3P6GXIFFF@ZA 018f6b68     glbuild.obj
 0004:011e4b6c       ?bglPixelStorei@@3P6GXIH@ZA 018f6b6c     glbuild.obj
 0004:011e4b70       ?bgluUnProject@@3P6GHNNNPBN0PBHPAN22@ZA 018f6b70     glbuild.obj
 0004:011e4b74       ?bgluTessProperty@@3P6GXPAVGLUtesselator@@IN@ZA 018f6b74     glbuild.obj
 0004:011e4b78       ?bglBegin@@3P6GXI@ZA       018f6b78     glbuild.obj
 0004:011e4b7c       ?bglUniform3iARB@@3P6GXHHHH@ZA 018f6b7c     glbuild.obj
 0004:011e4b80       ?bglDeleteLists@@3P6GXIH@ZA 018f6b80     glbuild.obj
 0004:011e4b84       ?bglBlendFunc@@3P6GXII@ZA  018f6b84     glbuild.obj
 0004:011e4b88       ?bglBlendEquation@@3P6GXI@ZA 018f6b88     glbuild.obj
 0004:011e4b8c       ?bgluTessCallback@@3P6GXPAVGLUtesselator@@IP6GXXZ@ZA 018f6b8c     glbuild.obj
 0004:011e4b90       ?bglDetachObjectARB@@3P6GXII@ZA 018f6b90     glbuild.obj
 0004:011e4b94       ?bglBeginQueryARB@@3P6GXII@ZA 018f6b94     glbuild.obj
 0004:011e4b98       ?bglColorMask@@3P6GXEEEE@ZA 018f6b98     glbuild.obj
 0004:011e4b9c       ?bglMultMatrixd@@3P6GXPBN@ZA 018f6b9c     glbuild.obj
 0004:011e4ba0       ?bglProgramStringARB@@3P6GXIIHPBX@ZA 018f6ba0     glbuild.obj
 0004:011e4ba4       ?bglVertexAttrib2dARB@@3P6GXINN@ZA 018f6ba4     glbuild.obj
 0004:011e4ba8       ?bglCallList@@3P6GXI@ZA    018f6ba8     glbuild.obj
 0004:011e4bac       ?bglUniformMatrix2fvARB@@3P6GXHHEPBM@ZA 018f6bac     glbuild.obj
 0004:011e4bb0       ?bglIsQueryARB@@3P6GEI@ZA  018f6bb0     glbuild.obj
 0004:011e4bb4       ?bglBufferSubDataARB@@3P6GXIHHPBX@ZA 018f6bb4     glbuild.obj
 0004:011e4bb8       ?bglVertex3f@@3P6GXMMM@ZA  018f6bb8     glbuild.obj
 0004:011e4bbc       ?bglTexCoord2d@@3P6GXNN@ZA 018f6bbc     glbuild.obj
 0004:011e4bc0       ?bglVertexAttrib2sARB@@3P6GXIFF@ZA 018f6bc0     glbuild.obj
 0004:011e4bc4       ?bglVertexAttrib2svARB@@3P6GXIPBF@ZA 018f6bc4     glbuild.obj
 0004:011e4bc8       ?bglGetShaderSourceARB@@3P6GXIHPAHPAD@ZA 018f6bc8     glbuild.obj
 0004:011e4bcc       ?bglBufferStorage@@3P6GXIHPBXI@ZA 018f6bcc     glbuild.obj
 0004:011e4bd0       ?bglLoadMatrixf@@3P6GXPBM@ZA 018f6bd0     glbuild.obj
 0004:011e4bd4       ?bglDisableClientState@@3P6GXI@ZA 018f6bd4     glbuild.obj
 0004:011e4bd8       ?bgluErrorString@@3P6GPBEI@ZA 018f6bd8     glbuild.obj
 0004:011e4bdc       ?bglClear@@3P6GXI@ZA       018f6bdc     glbuild.obj
 0004:011e4be0       ?bglVertexPointer@@3P6GXHIHPBX@ZA 018f6be0     glbuild.obj
 0004:011e4be4       ?bglFogf@@3P6GXIM@ZA       018f6be4     glbuild.obj
 0004:011e4be8       ?bglVertexAttrib4NsvARB@@3P6GXIPBF@ZA 018f6be8     glbuild.obj
 0004:011e4bec       ?bglPopAttrib@@3P6GXXZA    018f6bec     glbuild.obj
 0004:011e4bf0       ?bwglSetPixelFormat@@3P6GHPAUHDC__@@HPBUtagPIXELFORMATDESCRIPTOR@@@ZA 018f6bf0     glbuild.obj
 0004:011e4bf4       ?bwglDescribePixelFormat@@3P6GHPAUHDC__@@HIPAUtagPIXELFORMATDESCRIPTOR@@@ZA 018f6bf4     glbuild.obj
 0004:011e4bf8       ?bglVertexAttrib2fARB@@3P6GXIMM@ZA 018f6bf8     glbuild.obj
 0004:011e4bfc       ?bglLoadMatrixd@@3P6GXPBN@ZA 018f6bfc     glbuild.obj
 0004:011e4c00       ?bglViewport@@3P6GXHHHH@ZA 018f6c00     glbuild.obj
 0004:011e4c04       ?bglDeleteFramebuffersEXT@@3P6GXHPBI@ZA 018f6c04     glbuild.obj
 0004:011e4c08       ?bglUniformMatrix3fvARB@@3P6GXHHEPBM@ZA 018f6c08     glbuild.obj
 0004:011e4c0c       ?bglReadPixels@@3P6GXHHHHIIPAX@ZA 018f6c0c     glbuild.obj
 0004:011e4c10       ?bglGetActiveAttribARB@@3P6GXIIHPAH0PAIPAD@ZA 018f6c10     glbuild.obj
 0004:011e4c14       ?bglUniform1fARB@@3P6GXHM@ZA 018f6c14     glbuild.obj
 0004:011e4c18       ?bwglGetProcAddress@@3P6GP6GHXZPBD@ZA 018f6c18     glbuild.obj
 0004:011e4c1c       ?bglTexParameterf@@3P6GXIIM@ZA 018f6c1c     glbuild.obj
 0004:011e4c20       ?bglMatrixMode@@3P6GXI@ZA  018f6c20     glbuild.obj
 0004:011e4c24       ?bglStencilOp@@3P6GXIII@ZA 018f6c24     glbuild.obj
 0004:011e4c28       ?bglTranslatef@@3P6GXMMM@ZA 018f6c28     glbuild.obj
 0004:011e4c2c       ?bglDisable@@3P6GXI@ZA     018f6c2c     glbuild.obj
 0004:011e4c30       ?bglGetIntegerv@@3P6GXIPAH@ZA 018f6c30     glbuild.obj
 0004:011e4c34       ?bglVertexAttrib4NusvARB@@3P6GXIPBG@ZA 018f6c34     glbuild.obj
 0004:011e4c38       ?bwglSwapBuffers@@3P6GHPAUHDC__@@@ZA 018f6c38     glbuild.obj
 0004:011e4c3c       ?bglLightfv@@3P6GXIIPBM@ZA 018f6c3c     glbuild.obj
 0004:011e4c40       ?bglVertex3d@@3P6GXNNN@ZA  018f6c40     glbuild.obj
 0004:011e4c44       ?bglGetQueryObjectuivARB@@3P6GXIIPAI@ZA 018f6c44     glbuild.obj
 0004:011e4c48       ?bglColor4f@@3P6GXMMMM@ZA  018f6c48     glbuild.obj
 0004:011e4c4c       ?bglCopyTexImage2D@@3P6GXIHIHHHHH@ZA 018f6c4c     glbuild.obj
 0004:011e4c50       ?bglVertexAttrib2fvARB@@3P6GXIPBM@ZA 018f6c50     glbuild.obj
 0004:011e4c54       ?bwglCreateContextAttribsARB@@3P6GPAUHGLRC__@@PAUHDC__@@PAU1@PBH@ZA 018f6c54     glbuild.obj
 0004:011e4c58       ?bglClearColor@@3P6GXMMMM@ZA 018f6c58     glbuild.obj
 0004:011e4c5c       ?bglAttachObjectARB@@3P6GXII@ZA 018f6c5c     glbuild.obj
 0004:011e4c60       ?bglRecti@@3P6GXHHHH@ZA    018f6c60     glbuild.obj
 0004:011e4c64       ?bglNormal3f@@3P6GXMMM@ZA  018f6c64     glbuild.obj
 0004:011e4c68       ?bglScissor@@3P6GXHHHH@ZA  018f6c68     glbuild.obj
 0004:011e4c6c       ?bglVertexAttrib3dvARB@@3P6GXIPBN@ZA 018f6c6c     glbuild.obj
 0004:011e4c70       ?bglMapBufferARB@@3P6GPAXII@ZA 018f6c70     glbuild.obj
 0004:011e4c74       ?bgluNewTess@@3P6GPAVGLUtesselator@@XZA 018f6c74     glbuild.obj
 0004:011e4c78       ?bglVertexAttrib1dvARB@@3P6GXIPBN@ZA 018f6c78     glbuild.obj
 0004:011e4c7c       ?bglGetVertexAttribdvARB@@3P6GXIIPAN@ZA 018f6c7c     glbuild.obj
 0004:011e4c80       ?bglMultiTexCoord2fARB@@3P6GXIMM@ZA 018f6c80     glbuild.obj
 0004:011e4c84       ?bglUnmapBufferARB@@3P6GEI@ZA 018f6c84     glbuild.obj
 0004:011e4c88       ?bglHint@@3P6GXII@ZA       018f6c88     glbuild.obj
 0004:011e4c8c       ?bglTexImage2D@@3P6GXIHHHHHIIPBX@ZA 018f6c8c     glbuild.obj
 0004:011e4c90       ?bglTexCoord2i@@3P6GXHH@ZA 018f6c90     glbuild.obj
 0004:011e4c94       ?bglDepthFunc@@3P6GXI@ZA   018f6c94     glbuild.obj
 0004:011e4c98       ?bwglGetPixelFormat@@3P6GHPAUHDC__@@@ZA 018f6c98     glbuild.obj
 0004:011e4c9c       ?bglVertex2f@@3P6GXMM@ZA   018f6c9c     glbuild.obj
 0004:011e4ca0       ?bglGetVertexAttribPointervARB@@3P6GXIIPAPAX@ZA 018f6ca0     glbuild.obj
 0004:011e4ca4       ?bglVertexAttrib4bvARB@@3P6GXIPBC@ZA 018f6ca4     glbuild.obj
 0004:011e4ca8       ?bglVertex3fv@@3P6GXPBM@ZA 018f6ca8     glbuild.obj
 0004:011e4cac       ?bglVertexAttrib1fARB@@3P6GXIM@ZA 018f6cac     glbuild.obj
 0004:011e4cb0       ?bglMapBufferRange@@3P6GPAXIHHI@ZA 018f6cb0     glbuild.obj
 0004:011e4cb4       ?bglUniform3ivARB@@3P6GXHHPBH@ZA 018f6cb4     glbuild.obj
 0004:011e4cb8       ?bglVertexAttrib4svARB@@3P6GXIPBF@ZA 018f6cb8     glbuild.obj
 0004:011e4cbc       ?bglVertexAttrib4sARB@@3P6GXIFFFF@ZA 018f6cbc     glbuild.obj
 0004:011e4cc0       ?bglGetQueryivARB@@3P6GXIIPAH@ZA 018f6cc0     glbuild.obj
 0004:011e4cc4       ?bglCreateProgramObjectARB@@3P6GIXZA 018f6cc4     glbuild.obj
 0004:011e4cc8       ?bglVertexAttrib4usvARB@@3P6GXIPBG@ZA 018f6cc8     glbuild.obj
 0004:011e4ccc       ?bglPolygonMode@@3P6GXII@ZA 018f6ccc     glbuild.obj
 0004:011e4cd0       ?bglVertexAttrib1svARB@@3P6GXIPBF@ZA 018f6cd0     glbuild.obj
 0004:011e4cd4       ?bglUniform3fvARB@@3P6GXHHPBM@ZA 018f6cd4     glbuild.obj
 0004:011e4cd8       ?bglFogfv@@3P6GXIPBM@ZA    018f6cd8     glbuild.obj
 0004:011e4cdc       ?bgluTessNormal@@3P6GXPAVGLUtesselator@@NNN@ZA 018f6cdc     glbuild.obj
 0004:011e4ce0       ?bglDeleteBuffersARB@@3P6GXHPBI@ZA 018f6ce0     glbuild.obj
 0004:011e4ce4       ?bglVertexAttrib4NivARB@@3P6GXIPBH@ZA 018f6ce4     glbuild.obj
 0004:011e4cec       ?bglVertexAttrib4NubvARB@@3P6GXIPBE@ZA 018f6cec     glbuild.obj
 0004:011e4cf0       ?bglOrtho@@3P6GXNNNNNN@ZA  018f6cf0     glbuild.obj
 0004:011e4cf4       ?bglVertexAttrib3svARB@@3P6GXIPBF@ZA 018f6cf4     glbuild.obj
 0004:011e4cf8       ?bglUniformMatrix4fvARB@@3P6GXHHEPBM@ZA 018f6cf8     glbuild.obj
 0004:011e4cfc       ?bglTexCoord2f@@3P6GXMM@ZA 018f6cfc     glbuild.obj
 0004:011e4d00       ?bglBindProgramARB@@3P6GXII@ZA 018f6d00     glbuild.obj
 0004:011e4d04       ?bglUniform4fARB@@3P6GXHMMMM@ZA 018f6d04     glbuild.obj
 0004:011e4d08       ?bwglCreateContext@@3P6GPAUHGLRC__@@PAUHDC__@@@ZA 018f6d08     glbuild.obj
 0004:011e4d0c       ?bglDepthMask@@3P6GXE@ZA   018f6d0c     glbuild.obj
 0004:011e4d10       ?bglCheckFramebufferStatusEXT@@3P6GII@ZA 018f6d10     glbuild.obj
 0004:011e4d14       ?bglGetObjectParameterivARB@@3P6GXIIPAH@ZA 018f6d14     glbuild.obj
 0004:011e4d18       ?bwglMakeCurrent@@3P6GHPAUHDC__@@PAUHGLRC__@@@ZA 018f6d18     glbuild.obj
 0004:011e4d1c       ?bglCreateShaderObjectARB@@3P6GII@ZA 018f6d1c     glbuild.obj
 0004:011e4d20       ?bgluTessVertex@@3P6GXPAVGLUtesselator@@PANPAX@ZA 018f6d20     glbuild.obj
 0004:011e4d24       ?bglValidateProgramARB@@3P6GXI@ZA 018f6d24     glbuild.obj
 0004:011e4d28       ?bglTexEnvf@@3P6GXIIM@ZA   018f6d28     glbuild.obj
 0004:011e4d2c       ?bglClientActiveTextureARB@@3P6GXI@ZA 018f6d2c     glbuild.obj
 0004:011e4d30       ?bglAlphaFunc@@3P6GXIM@ZA  018f6d30     glbuild.obj
 0004:011e4d34       ?bglUniform1ivARB@@3P6GXHHPBH@ZA 018f6d34     glbuild.obj
 0004:011e4d38       ?bglUniform1fvARB@@3P6GXHHPBM@ZA 018f6d38     glbuild.obj
 0004:011e4d3c       ?bglVertexAttrib4dvARB@@3P6GXIPBN@ZA 018f6d3c     glbuild.obj
 0004:011e4d40       ?bglVertexAttrib4fARB@@3P6GXIMMMM@ZA 018f6d40     glbuild.obj
 0004:011e4d44       ?bglGenBuffersARB@@3P6GXHPAI@ZA 018f6d44     glbuild.obj
 0004:011e4d48       ?bgluPerspective@@3P6GXNNNN@ZA 018f6d48     glbuild.obj
 0004:011e4d4c       ?bglVertexAttrib1sARB@@3P6GXIF@ZA 018f6d4c     glbuild.obj
 0004:011e4d50       ?bglTexImage3D@@3P6GXIHHHHHHIIPBX@ZA 018f6d50     glbuild.obj
 0004:011e4d54       ?bglUniform2fARB@@3P6GXHMM@ZA 018f6d54     glbuild.obj
 0004:011e4d58       ?bwglChoosePixelFormat@@3P6GHPAUHDC__@@PBUtagPIXELFORMATDESCRIPTOR@@@ZA 018f6d58     glbuild.obj
 0004:011e4d5c       ?bglStencilFunc@@3P6GXIHI@ZA 018f6d5c     glbuild.obj
 0004:011e4d60       ?bglGetUniformLocationARB@@3P6GHIPBD@ZA 018f6d60     glbuild.obj
 0004:011e4d64       ?bglRasterPos4i@@3P6GXHHHH@ZA 018f6d64     glbuild.obj
 0004:011e4d68       ?bglCullFace@@3P6GXI@ZA    018f6d68     glbuild.obj
 0004:011e4d6c       ?bglNewList@@3P6GXII@ZA    018f6d6c     glbuild.obj
 0004:011e4d70       ?bglVertexAttrib2dvARB@@3P6GXIPBN@ZA 018f6d70     glbuild.obj
 0004:011e4d74       ?bglVertexAttrib4dARB@@3P6GXINNNN@ZA 018f6d74     glbuild.obj
 0004:011e4d78       ?bglClearStencil@@3P6GXH@ZA 018f6d78     glbuild.obj
 0004:011e4d7c       ?bglActiveTextureARB@@3P6GXI@ZA 018f6d7c     glbuild.obj
 0004:011e4d80       ?bglTexGenfv@@3P6GXIIPBM@ZA 018f6d80     glbuild.obj
 0004:011e4d84       ?bglGetTexParameteriv@@3P6GXIIPAH@ZA 018f6d84     glbuild.obj
 0004:011e4d88       ?bglDisableVertexAttribArrayARB@@3P6GXI@ZA 018f6d88     glbuild.obj
 0004:011e4d8c       ?bglCompileShaderARB@@3P6GXI@ZA 018f6d8c     glbuild.obj
 0004:011e4d90       ?bglMultMatrixf@@3P6GXPBM@ZA 018f6d90     glbuild.obj
 0004:011e4d94       ?bglDebugMessageCallbackARB@@3P6GXP6GXIIIIHPBDPBX@Z1@ZA 018f6d94     glbuild.obj
 0004:011e4d98       ?bglDrawArrays@@3P6GXIHH@ZA 018f6d98     glbuild.obj
 0004:011e4d9c       ?bglGetInfoLogARB@@3P6GXIHPAHPAD@ZA 018f6d9c     glbuild.obj
 0004:011e4da0       ?bglGetTexLevelParameteriv@@3P6GXIHIPAH@ZA 018f6da0     glbuild.obj
 0004:011e4da4       ?bglBindBufferARB@@3P6GXII@ZA 018f6da4     glbuild.obj
 0004:011e4da8       ?bglGenQueriesARB@@3P6GXHPAI@ZA 018f6da8     glbuild.obj
 0004:011e4dac       ?bglGetHandleARB@@3P6GII@ZA 018f6dac     glbuild.obj
 0004:011e4db0       ?bglGetDoublev@@3P6GXIPAN@ZA 018f6db0     glbuild.obj
 0004:011e4db4       ?bglUniform3fARB@@3P6GXHMMM@ZA 018f6db4     glbuild.obj
 0004:011e4db8       ?bglVertexAttrib1fvARB@@3P6GXIPBM@ZA 018f6db8     glbuild.obj
 0004:011e4dbc       ?bglTexSubImage2D@@3P6GXIHHHHHIIPBX@ZA 018f6dbc     glbuild.obj
 0004:011e4dc0       ?bglVertexAttribPointerARB@@3P6GXIHIEHPBX@ZA 018f6dc0     glbuild.obj
 0004:011e4dc4       ?bglGenTextures@@3P6GXHPAI@ZA 018f6dc4     glbuild.obj
 0004:011e4dc8       ?bglTexParameteri@@3P6GXIIH@ZA 018f6dc8     glbuild.obj
 0004:011e4dcc       ?gldriver@@3PADA           018f6dcc     glbuild.obj
 0004:011e4dd0       ?glulibrary@@3PADA         018f6dd0     glbuild.obj
 0004:011e4dd8       _texcache                  018f6dd8     texcache.obj
 0004:011ece14       ?iystp@@3HA                018fee14     kplib.obj
 0004:011f50a4       ?nbpl@@3HA                 019070a4     kplib.obj
 0004:011f70ac       ?ixoff@@3HA                019090ac     kplib.obj
 0004:011f7d1c       ?ixsiz@@3HA                01909d1c     kplib.obj
 0004:011ffd30       ?intlac@@3HA               01911d30     kplib.obj
 0004:0122a33c       ?xsizbpl@@3HA              0193c33c     kplib.obj
 0004:012376e0       _kzfs                      019496e0     kplib.obj
 0004:01238b10       ?iyoff@@3HA                0194ab10     kplib.obj
 0004:0123b4a8       ?ixstp@@3HA                0194d4a8     kplib.obj
 0004:0123b6e8       _hicreplc                  0194d6e8     hightile.obj
 0004:012596e8       _hictinting                0196b6e8     hightile.obj
 0004:01259ae8       _hicinitcounter            0196bae8     hightile.obj
 0004:01259af0       _glox1                     0196baf0     polymost.obj
 0004:01259af4       _gcosang2                  0196baf4     polymost.obj
 0004:01259b00       _gchang                    0196bb00     polymost.obj
 0004:01259b04       _gshang                    0196bb04     polymost.obj
 0004:01259b08       _gvisibility               0196bb08     polymost.obj
 0004:01259b0c       _gyxscale                  0196bb0c     polymost.obj
 0004:0127fb10       _gctang                    01991b10     polymost.obj
 0004:0127fb14       ?glox2@@3MA                01991b14     polymost.obj
 0004:0127fb18       _alphahackarray            01991b18     polymost.obj
 0004:0128731c       _grhalfxdown10             0199931c     polymost.obj
 0004:01287320       _fxdim                     01999320     polymost.obj
 0004:01287324       _fydimen                   01999324     polymost.obj
 0004:01287328       _mdtims                    01999328     polymost.obj
 0004:01287330       _gloy1                     01999330     polymost.obj
 0004:01287334       _gsinang                   01999334     polymost.obj
 0004:0128d350       _fsinglobalang             0199f350     polymost.obj
 0004:0128d358       _ptempbuf                  0199f358     polymost.obj
 0004:01290358       _fydim                     019a2358     polymost.obj
 0004:0129035c       ?fogcol@@3Ucoltypef@@A     019a235c     polymost.obj
 0004:0129036c       _polymost_hitdata          019a236c     polymost.obj
 0004:01290384       _grhalfxdown10x            019a2384     polymost.obj
 0004:0129038c       _gstang                    019a238c     polymost.obj
 0004:01290390       ?fogtable@@3PAUcoltypef@@A 019a2390     polymost.obj
 0004:01291390       ?wsprinfo@@3PAUwallspriteinfo_t@@A 019a3390     polymost.obj
 0004:012c1390       _ghalfx                    019d3390     polymost.obj
 0004:012c1398       _fcosglobalang             019d3398     polymost.obj
 0004:012c13b8       _gxyaspect                 019d33b8     polymost.obj
 0004:012c13bc       _gsinang2                  019d33bc     polymost.obj
 0004:012c13c4       _omdtims                   019d33c4     polymost.obj
 0004:012c13d0       _fviewingrange             019d33d0     polymost.obj
 0004:012c13d8       _gcosang                   019d33d8     polymost.obj
 0004:012c13e4       ?gloy2@@3MA                019d33e4     polymost.obj
 0004:012c1400       _rendmode                  019d3400     polymost.obj
 0004:012c1404       _vsync                     019d3404     polymost.obj
 0004:012c1408       _shadescale_unbounded      019d3408     polymost.obj
 0004:012c140c       _r_npotwallmode            019d340c     polymost.obj
 0004:012c1410       _gtang                     019d3410     polymost.obj
 0004:012c141c       ?r_polygonmode@@3HA        019d341c     polymost.obj
 0004:012c1424       _glmultisample             019d3424     polymost.obj
 0004:012c1428       _glnvmultisamplehint       019d3428     polymost.obj
 0004:012c142c       _gltexmaxsize              019d342c     polymost.obj
 0004:012c1430       ?gltexmiplevel@@3HA        019d3430     polymost.obj
 0004:012c1438       _r_downsize                019d3438     polymost.obj
 0004:012c143c       _r_parallaxskypanning      019d343c     polymost.obj
 0004:012c1440       _drawingskybox             019d3440     polymost.obj
 0004:012c1444       _hicprecaching             019d3444     polymost.obj
 0004:012c14a4       ?curmodelviewmatrix@@3PAMA 019d34a4     polymer.obj
 0004:012c14a8       ?asi@@3Us_pranimatespritesinfo@@A 019d34a8     polymer.obj
 0004:012c14bc       ?overridematerial@@3HA     019d34bc     polymer.obj
 0004:012c14c0       ?prwalls@@3PAPAUs_prwall@@A 019d34c0     polymer.obj
 0004:012d34c0       ?prindexringvbo@@3IA       019e54c0     polymer.obj
 0004:012d34c4       ?horizang@@3MA             019e54c4     polymer.obj
 0004:012d34c8       _prsprites                 019e54c8     polymer.obj
 0004:012e34c8       ?prwalldataoffset@@3HA     019f54c8     polymer.obj
 0004:012e34cc       ?culledface@@3HA           019f54cc     polymer.obj
 0004:012e34d0       ?skyboxdatavbo@@3IA        019f54d0     polymer.obj
 0004:012e34d4       ?prindexring@@3PAIA        019f54d4     polymer.obj
 0004:012e34d8       ?globaloldoverridematerial@@3HA 019f54d8     polymer.obj
 0004:012e34e0       ?cursectormasks@@3PAFA     019f54e0     polymer.obj
 0004:012e34e4       ?prcanbucket@@3HA          019f54e4     polymer.obj
 0004:012e34e8       _prartmaps                 019f54e8     polymer.obj
 0004:013014e8       ?prhighpalookups@@3PAY0BAA@Us_prhighpalookup@@A 01a134e8     polymer.obj
 0004:013814e8       ?mirrors@@3PAUs_prmirror@@A 01a934e8     polymer.obj
 0004:01381538       ?prtess@@3PAVGLUtesselator@@A 01a93538     polymer.obj
 0004:0138153c       _lightcount                01a9353c     polymer.obj
 0004:01381540       ?mdspritespace@@3PAY03MA   01a93540     polymer.obj
 0004:01381580       _prlights                  01a93580     polymer.obj
 0004:013c4580       ?cursectormaskcount@@3PAFA 01ad6580     polymer.obj
 0004:013c4584       ?rotatespritematerialbits@@3HA 01ad6584     polymer.obj
 0004:013c4588       ?mdspritematerial@@3Us_prmaterial@@A 01ad6588     polymer.obj
 0004:013c45ec       ?depth@@3HA                01ad65ec     polymer.obj
 0004:013c45f0       ?artskydata@@3PAMA         01ad65f0     polymer.obj
 0004:013c4630       ?prbasepalmaps@@3PAIA      01ad6630     polymer.obj
 0004:013c4a30       ?rootmodelviewmatrix@@3PAMA 01ad6a30     polymer.obj
 0004:013d4a70       ?curlight@@3HA             01ae6a70     polymer.obj
 0004:013d4a78       ?prprograms@@3PAUs_prrograminfo@@A 01ae6a78     polymer.obj
 0004:103d4a78       ?polymersearching@@3HA     10ae6a78     polymer.obj
 0004:103d4a7c       ?prindexringoffset@@3HA    10ae6a7c     polymer.obj
 0004:103d6a80       ?prrts@@3PAUs_prrt@@A      10ae8a80     polymer.obj
 0004:103d6a84       ?viewangle@@3FA            10ae8a84     polymer.obj
 0004:103d6a88       ?prsectors@@3PAPAUs_prsector@@A 10ae8a88     polymer.obj
 0004:103dca88       ?curskymodelviewmatrix@@3PAMA 10aeea88     polymer.obj
 0004:103dca8c       ?prbuckethead@@3PAUs_prbucket@@A 10aeea8c     polymer.obj
 0004:103dca90       ?prlookups@@3PAIA          10aeea90     polymer.obj
 0004:103dce90       ?spritemodelview@@3PAMA    10aeee90     polymer.obj
 0004:103dced0       ?rootskymodelviewmatrix@@3PAMA 10aeeed0     polymer.obj
 0004:103dcf10       ?prmapvbo@@3IA             10aeef10     polymer.obj
 0004:103dcf14       _pr_wireframe              10aeef14     polymer.obj
 0004:103dcf18       _pr_customaspect           10aeef18     polymer.obj
 0004:103dcf20       _pr_buckets                10aeef20     polymer.obj
 0004:103dcf24       _pr_overrideparallax       10aeef24     polymer.obj
 0004:103dcf28       _pr_parallaxbias           10aeef28     polymer.obj
 0004:103dcf2c       _pr_overridespecular       10aeef2c     polymer.obj
 0004:103dcf30       _pr_overridehud            10aeef30     polymer.obj
 0004:103dcf34       _pr_hudxadd                10aeef34     polymer.obj
 0004:103dcf38       _pr_hudyadd                10aeef38     polymer.obj
 0004:103dcf3c       _pr_hudzadd                10aeef3c     polymer.obj
 0004:103dcf40       _pr_hudangadd              10aeef40     polymer.obj
 0004:103dcf44       _pr_overridemodelscale     10aeef44     polymer.obj
 0004:103dcf48       _pr_ati_fboworkaround      10aeef48     polymer.obj
 0004:103dcf4c       _pr_ati_nodepthoffset      10aeef4c     polymer.obj
 0004:103dcf50       _pr_nullrender             10aeef50     polymer.obj
 0004:103dd788       _globalnoeffect            10aef788     mdsprite.obj
 0004:103dd864       ?vnum@@3HA                 10aef864     voxmodel.obj
 0004:103dd868       ?vmax@@3HA                 10aef868     voxmodel.obj
 0004:103dd87c       ?myconnectindex@@3HA       10aef87c     mmulti_null.obj
 0004:103dd880       ?numplayers@@3HA           10aef880     mmulti_null.obj
 0004:103dd884       ?connecthead@@3HA          10aef884     mmulti_null.obj
 0004:103dd888       ?syncstate@@3EA            10aef888     mmulti_null.obj
 0004:103dd88c       _osdlog                    10aef88c     osd.obj
 0004:103dd890       _osdlogfn                  10aef890     osd.obj
 0004:103dd898       _osd                       10aef898     osd.obj
 0004:103dd8a8       _m32_osd_tryscript         10aef8a8     osd.obj
 0004:103df8b0       _divtable64                10af18b0     pragmas.obj
 0004:1041f8b0       _dmval                     10b318b0     pragmas.obj
 0004:1041f8b8       _divtable32                10b318b8     pragmas.obj
 0004:1043f8f8       ?pwinever@@3P6GHXZA        10b518f8     winbits.obj
 0004:1043f99c       ?silentvideomodeswitch@@3DA 10b5199c     winbits.obj
 0004:1043f9a0       ?win_timerfreq@@3_JA       10b519a0     winbits.obj
 0004:1043fdb8       _bytesperline              10b51db8     sdlayer.obj
 0004:1043fdc8       ?joydead@@3PAGA            10b51dc8     sdlayer.obj
 0004:104409dc       ?joysatur@@3PAGA           10b529dc     sdlayer.obj
 0004:104409e4       _inputchecked              10b529e4     sdlayer.obj
 0004:104409e8       _quitevent                 10b529e8     sdlayer.obj
 0004:104409e9       ?novideo@@3DA              10b529e9     sdlayer.obj
 0004:104409ea       _offscreenrendering        10b529ea     sdlayer.obj
 0004:104409eb       ?videomodereset@@3DA       10b529eb     sdlayer.obj
 0004:10440a04       _bpp                       10b52a04     sdlayer.obj
 0004:10440a08       _fullscreen                10b52a08     sdlayer.obj
 0004:10440a0c       _frameplace                10b52a0c     sdlayer.obj
 0004:10440a10       ?lockcount@@3HA            10b52a10     sdlayer.obj
 0004:10440a14       _nofog                     10b52a14     sdlayer.obj
 0004:10440a18       ?nogl@@3DA                 10b52a18     sdlayer.obj
 0004:10440a28       ?timerticspersec@@3HA      10b52a28     sdlayer.obj
 0004:10441298       ?FX_ErrorCode@@3HA         10b53298     fx_man.obj
 0004:1044129c       ?FX_Installed@@3HA         10b5329c     fx_man.obj
 0004:104412a0       ?MV_LeftVolume@@3PBFB      10b532a0     multivoc.obj
 0004:104412a4       ?MV_MixPosition@@3IA       10b532a4     multivoc.obj
 0004:104612b4       ?MV_RightChannelOffset@@3HA 10b732b4     multivoc.obj
 0004:10461328       ?MV_MixBuffer@@3PAPADA     10b73328     multivoc.obj
 0004:1046136c       ?MV_MixRate@@3HA           10b7336c     multivoc.obj
 0004:104613e0       ?MV_MixDestination@@3PADA  10b733e0     multivoc.obj
 0004:104613e4       ?MV_RightVolume@@3PBFB     10b733e4     multivoc.obj
 0004:10461428       ?MV_PanTable@@3PAY0BAA@UPan@@A 10b73428     multivoc.obj
 0004:1047142c       ?MV_Installed@@3HA         10b8342c     multivoc.obj
 0004:1047143c       _MV_Printf                 10b8343c     multivoc.obj
 0004:104729e0       _SDL_Instance              10b849e0     libSDL2:SDL_windowsevents.o
 0004:104729e4       _SDL_Appstyle              10b849e4     libSDL2:SDL_windowsevents.o
 0004:104729e8       _SDL_Appname               10b849e8     libSDL2:SDL_windowsevents.o
 0004:10472c80       _SDL_EventOK               10b84c80     libSDL2:SDL_events.o
 0004:104730d0       _SDL_numGestureTouches     10b850d0     libSDL2:SDL_gesture.o
 0004:104730d4       _SDL_haptics               10b850d4     libSDL2:SDL_haptic.o
 0004:10473f08       _SDL_XInputVersion         10b85f08     libSDL2:SDL_xinput.o
 0004:10473f0c       _SDL_XInputGetBatteryInformation 10b85f0c     libSDL2:SDL_xinput.o
 0004:10473f10       _SDL_XInputGetCapabilities 10b85f10     libSDL2:SDL_xinput.o
 0004:10473f14       _SDL_XInputSetState        10b85f14     libSDL2:SDL_xinput.o
 0004:10473f18       _SDL_XInputGetState        10b85f18     libSDL2:SDL_xinput.o
 0004:10473f48       _SDL_cursor                10b85f48     libSDL2:SDL_windowsmouse.o
 0004:10473f50       _SDL_HelperWindow          10b85f50     libSDL2:SDL_windowswindow.o
 0004:10474480       _SDL_hapticlist            10b86480     libSDL2:SDL_windowshaptic.o
 0004:104748a4       _vp8_sad16x16x4d           10b868a4     libvpx:rtcd.c.o
 0004:104748a8       _vp8_sad16x8x4d            10b868a8     libvpx:rtcd.c.o
 0004:104748ac       _vp8_sad8x16x4d            10b868ac     libvpx:rtcd.c.o
 0004:104748b0       _vp8_sad8x8x4d             10b868b0     libvpx:rtcd.c.o
 0004:104748b4       _vp8_sad4x4x4d             10b868b4     libvpx:rtcd.c.o
 0004:104748b8       _vp8_sad16x16x8            10b868b8     libvpx:rtcd.c.o
 0004:104748bc       _vp8_sad16x8x8             10b868bc     libvpx:rtcd.c.o
 0004:104748c0       _vp8_sad8x16x8             10b868c0     libvpx:rtcd.c.o
 0004:104748c4       _vp8_sad8x8x8              10b868c4     libvpx:rtcd.c.o
 0004:104748c8       _vp8_sad4x4x8              10b868c8     libvpx:rtcd.c.o
 0004:104748cc       _vp8_sad16x16x3            10b868cc     libvpx:rtcd.c.o
 0004:104748d0       _vp8_sad16x8x3             10b868d0     libvpx:rtcd.c.o
 0004:104748d4       _vp8_sad8x16x3             10b868d4     libvpx:rtcd.c.o
 0004:104748d8       _vp8_sad8x8x3              10b868d8     libvpx:rtcd.c.o
 0004:104748dc       _vp8_sad4x4x3              10b868dc     libvpx:rtcd.c.o
 0004:104748e0       _vp8_sad16x16              10b868e0     libvpx:rtcd.c.o
 0004:104748e4       _vp8_sad16x8               10b868e4     libvpx:rtcd.c.o
 0004:104748e8       _vp8_sad8x16               10b868e8     libvpx:rtcd.c.o
 0004:104748ec       _vp8_sad8x8                10b868ec     libvpx:rtcd.c.o
 0004:104748f0       _vp8_sad4x4                10b868f0     libvpx:rtcd.c.o
 0004:104748f4       _vp8_variance_halfpixvar16x16_hv 10b868f4     libvpx:rtcd.c.o
 0004:104748f8       _vp8_variance_halfpixvar16x16_v 10b868f8     libvpx:rtcd.c.o
 0004:104748fc       _vp8_variance_halfpixvar16x16_h 10b868fc     libvpx:rtcd.c.o
 0004:10474900       _vp8_sub_pixel_variance16x16 10b86900     libvpx:rtcd.c.o
 0004:10474904       _vp8_sub_pixel_variance16x8 10b86904     libvpx:rtcd.c.o
 0004:10474908       _vp8_sub_pixel_variance8x16 10b86908     libvpx:rtcd.c.o
 0004:1047490c       _vp8_sub_pixel_variance8x8 10b8690c     libvpx:rtcd.c.o
 0004:10474910       _vp8_sub_pixel_variance4x4 10b86910     libvpx:rtcd.c.o
 0004:10474914       _vp8_variance16x16         10b86914     libvpx:rtcd.c.o
 0004:10474918       _vp8_variance16x8          10b86918     libvpx:rtcd.c.o
 0004:1047491c       _vp8_variance8x16          10b8691c     libvpx:rtcd.c.o
 0004:10474920       _vp8_variance8x8           10b86920     libvpx:rtcd.c.o
 0004:10474924       _vp8_variance4x4           10b86924     libvpx:rtcd.c.o
 0004:10474928       _vp8_bilinear_predict4x4   10b86928     libvpx:rtcd.c.o
 0004:1047492c       _vp8_bilinear_predict8x4   10b8692c     libvpx:rtcd.c.o
 0004:10474930       _vp8_bilinear_predict8x8   10b86930     libvpx:rtcd.c.o
 0004:10474934       _vp8_bilinear_predict16x16 10b86934     libvpx:rtcd.c.o
 0004:10474938       _vp8_sixtap_predict4x4     10b86938     libvpx:rtcd.c.o
 0004:1047493c       _vp8_sixtap_predict8x4     10b8693c     libvpx:rtcd.c.o
 0004:10474940       _vp8_sixtap_predict8x8     10b86940     libvpx:rtcd.c.o
 0004:10474944       _vp8_sixtap_predict16x16   10b86944     libvpx:rtcd.c.o
 0004:10474948       _vp8_filter_by_weight8x8   10b86948     libvpx:rtcd.c.o
 0004:1047494c       _vp8_filter_by_weight16x16 10b8694c     libvpx:rtcd.c.o
 0004:10474950       _vp8_plane_add_noise       10b86950     libvpx:rtcd.c.o
 0004:10474954       _vp8_post_proc_down_and_across_mb_row 10b86954     libvpx:rtcd.c.o
 0004:10474958       _vp8_mbpost_proc_across_ip 10b86958     libvpx:rtcd.c.o
 0004:1047495c       _vp8_mbpost_proc_down      10b8695c     libvpx:rtcd.c.o
 0004:10474960       _vp8_build_intra_predictors_mbuv_s 10b86960     libvpx:rtcd.c.o
 0004:10474964       _vp8_build_intra_predictors_mby_s 10b86964     libvpx:rtcd.c.o
 0004:10474968       _vp8_copy_mem8x4           10b86968     libvpx:rtcd.c.o
 0004:1047496c       _vp8_copy_mem8x8           10b8696c     libvpx:rtcd.c.o
 0004:10474970       _vp8_copy_mem16x16         10b86970     libvpx:rtcd.c.o
 0004:10474974       _vp8_dc_only_idct_add      10b86974     libvpx:rtcd.c.o
 0004:10474978       _vp8_short_inv_walsh4x4    10b86978     libvpx:rtcd.c.o
 0004:1047497c       _vp8_short_idct4x4llm      10b8697c     libvpx:rtcd.c.o
 0004:10474980       _vp8_loop_filter_simple_bh 10b86980     libvpx:rtcd.c.o
 0004:10474984       _vp8_loop_filter_simple_bv 10b86984     libvpx:rtcd.c.o
 0004:10474988       _vp8_loop_filter_simple_mbh 10b86988     libvpx:rtcd.c.o
 0004:1047498c       _vp8_loop_filter_simple_mbv 10b8698c     libvpx:rtcd.c.o
 0004:10474990       _vp8_loop_filter_bh        10b86990     libvpx:rtcd.c.o
 0004:10474994       _vp8_loop_filter_mbh       10b86994     libvpx:rtcd.c.o
 0004:10474998       _vp8_loop_filter_bv        10b86998     libvpx:rtcd.c.o
 0004:1047499c       _vp8_loop_filter_mbv       10b8699c     libvpx:rtcd.c.o
 0004:104749a0       _vp8_dequant_idct_add_uv_block 10b869a0     libvpx:rtcd.c.o
 0004:104749a4       _vp8_dequant_idct_add_y_block 10b869a4     libvpx:rtcd.c.o
 0004:104749a8       _vp8_dequant_idct_add      10b869a8     libvpx:rtcd.c.o
 0004:104749ac       _vp8_dequantize_b          10b869ac     libvpx:rtcd.c.o
 0004:104749b0       _vp8_clear_system_state    10b869b0     libvpx:rtcd.c.o
 0004:10474d04       __commode                  10b86d04     msvcrtd:xncommod.obj
 0004:10474d08       __fmode                    10b86d08     msvcrtd:xtxtmode.obj
 0004:10474d0c       __dowildcard               10b86d0c     msvcrtd:wildcard.obj
 0004:10474d10       __newmode                  10b86d10     msvcrtd:_newmode.obj
 0004:10474d14       _recordAll                 10b86d14     <common>
 0004:10474d18       _SDL_gestureTouch          10b86d18     <common>
 0004:10474d1c       _SDL_EventOKParam          10b86d1c     <common>
 0004:10474d20       _SYS_Joystick              10b86d20     <common>
 0004:10474d24       ___native_startup_state    10b86d24     <common>
 0004:10474d28       ___native_startup_lock     10b86d28     <common>
 0004:10474d2c       ___sse2_available          10b86d2c     <common>
 0004:10474d30       __NoHeapEnableTerminationOnCorruption 10b86d30     <common>
 0004:10474d34       ___dyn_tls_init_callback   10b86d34     <common>
 0004:10474d38       ___onexitend               10b86d38     <common>
 0004:10474d3c       ___onexitbegin             10b86d3c     <common>
 0007:00000520       _vp8_six_tap_mmx           10b95520     libvpx:subpixel_mmx.asm.o

 entry point at        0001:0028ca10

 Static symbols

 0001:000004e0       ?G_DrawTileGeneric@@YAXHHHHHHH@Z 004014e0 f   game.obj
 0001:00000560       _rotatesprite_win          00401560 f   game.obj
 0001:000006f0       _G_HandleAsync             004016f0 f   game.obj
 0001:00000790       _getrendermode             00401790 f   game.obj
 0001:00000960       ?G_DisplayExtraScreens@@YAXXZ 00401960 f   game.obj
 0001:00000c00       _rotatesprite_fs           00401c00 f   game.obj
 0001:00000c50       _G_GetLogoFlags            00401c50 f   game.obj
 0001:00000c70       ?fadepaltile@@YAXHHHHHHH@Z 00401c70 f   game.obj
 0001:00000d50       _klabs                     00401d50 f   game.obj
 0001:00001040       _getclosestcol             00402040 f   game.obj
 0001:000022c0       _scale                     004032c0 f   game.obj
 0001:00002300       _tabledivide64             00403300 f   game.obj
 0001:000023d0       _mulscale16                004033d0 f   game.obj
 0001:000023e0       _G_RestoreInterpolations   004033e0 f   game.obj
 0001:00002430       _calc_smoothratio          00403430 f   game.obj
 0001:00002450       _clamp                     00403450 f   game.obj
 0001:00002490       _VM_HaveEvent              00403490 f   game.obj
 0001:000024c0       _VM_OnEvent                004034c0 f   game.obj
 0001:00002500       ?G_ShowCacheLocks@@YAXXZ   00403500 f   game.obj
 0001:000027e0       ?G_PrintFPS@@YAXXZ         004037e0 f   game.obj
 0001:00002c00       _getticks                  00403c00 f   game.obj
 0001:00002c10       ?G_PrintCoords@@YAXH@Z     00403c10 f   game.obj
 0001:00003270       ?G_MoveClouds@@YAXXZ       00404270 f   game.obj
 0001:00003390       ?G_DrawOverheadMap@@YAXHHHF@Z 00404390 f   game.obj
 0001:000047e0       _divscale16                004057e0 f   game.obj
 0001:00004800       _divscale                  00405800 f   game.obj
 0001:00004840       _mulscale                  00405840 f   game.obj
 0001:00004860       _dmulscale16               00405860 f   game.obj
 0001:00004890       _push_nofog                00405890 f   game.obj
 0001:000048b0       _pop_nofog                 004058b0 f   game.obj
 0001:000048e0       ?G_ShowScores@@YAXXZ       004058e0 f   game.obj
 0001:00004b90       ?G_LastMapInfoIndex@@YAHXZ 00405b90 f   game.obj
 0001:00004bd0       ?palaccum_add@@YAXPAUpalaccum_t@@PBUpalette_t@@H@Z 00405bd0 f   game.obj
 0001:00004ca0       ?G_FadePalaccum@@YAXPBUpalaccum_t@@@Z 00405ca0 f   game.obj
 0001:00004d10       ?gtextsc@@YAHH@Z           00405d10 f   game.obj
 0001:000063d0       _B_BUF32                   004073d0 f   game.obj
 0001:000063e0       _divscale22                004073e0 f   game.obj
 0001:00006400       _swapchar                  00407400 f   game.obj
 0001:00006420       _swapbufreverse            00407420 f   game.obj
 0001:00006510       _getzsofslope              00407510 f   game.obj
 0001:00006540       _G_GetCameraPosition       00407540 f   game.obj
 0001:00006610       ?G_DoThirdPerson@@YAHPBUDukePlayer_t@@PAUvec3_t@@PAFHH@Z 00407610 f   game.obj
 0001:00006a00       _mulscale28                00407a00 f   game.obj
 0001:00006a10       ?G_OROR_DupeSprites@@YAXPBUspritetype@@@Z 00407a10 f   game.obj
 0001:00006c30       ?G_SE40@@YAXH@Z            00407c30 f   game.obj
 0001:00007380       ?G_ReadGLFrame@@YAXXZ      00408380 f   game.obj
 0001:00007510       _xcalloc                   00408510 f   game.obj
 0001:00007d90       ?A_ResetVars@@YAXH@Z       00408d90 f   game.obj
 0001:00007df0       ?G_InitActor@@YAHHHH@Z     00408df0 f   game.obj
 0001:0000ea50       _krand                     0040fa50 f   game.obj
 0001:0000ea80       _getceilzofslope           0040fa80 f   game.obj
 0001:0000eab0       _getflorzofslope           0040fab0 f   game.obj
 0001:0000eae0       _P_Get                     0040fae0 f   game.obj
 0001:0000eb00       _P_GetP                    0040fb00 f   game.obj
 0001:0000eb30       _Sect_SetInterpolation     0040fb30 f   game.obj
 0001:0000eb50       _A_SetSprite               0040fb50 f   game.obj
 0001:0000ec40       _A_MoveSprite              0040fc40 f   game.obj
 0001:0000ec60       _A_CheckEnemySprite        0040fc60 f   game.obj
 0001:0000ec80       _A_CheckEnemyTile          0040fc80 f   game.obj
 0001:0000eca0       ?G_HaveActor@@YAHH@Z       0040fca0 f   game.obj
 0001:0000ecc0       ?Yax_SetBunchInterpolation@@YAXHH@Z 0040fcc0 f   game.obj
 0001:00011b30       _md_tilehasmodel           00412b30 f   game.obj
 0001:00011b70       _G_GetViewscreenSizeShift  00412b70 f   game.obj
 0001:00011bd0       ?G_MaybeTakeOnFloorPal@@YAHPAUtspritetype@@H@Z 00412bd0 f   game.obj
 0001:00011c60       ?getofs_viewtype5@@YAHPBUtspritetype@@PAU1@HE@Z 00412c60 f   game.obj
 0001:00011cf0       ?getofs_viewtype7@@YAHPBUtspritetype@@PAU1@HE@Z 00412cf0 f   game.obj
 0001:00011d80       ?G_CheckAdultTile@@YAHH@Z  00412d80 f   game.obj
 0001:000121d0       ?G_DoEventAnimSprites@@YAXH@Z 004131d0 f   game.obj
 0001:00013a30       _mulscale6                 00414a30 f   game.obj
 0001:00013a40       _G_SetStatusBarScale       00414a40 f   game.obj
 0001:00013af0       ?parsedefinitions_game_include@@YAXPBDPAUscriptfile@@0H@Z 00414af0 f   game.obj
 0001:00013b40       ?parsedefinitions_game@@YAHPAUscriptfile@@H@Z 00414b40 f   game.obj
 0001:000143e0       _xrealloc                  004153e0 f   game.obj
 0001:00014410       ?S_DefineSound@@YAHHPBD@Z  00415410 f   game.obj
 0001:00014440       ?S_DefineAudioIfSupported@@YAHPAPADPBD@Z 00415440 f   game.obj
 0001:00014490       _realloc_copy              00415490 f   game.obj
 0001:000144f0       ?S_DefineMusic@@YAHPBD0@Z  004154f0 f   game.obj
 0001:000145b0       _G_GetMusicIdx             004155b0 f   game.obj
 0001:000146e0       ?G_Cleanup@@YAXXZ          004156e0 f   game.obj
 0001:000148b0       ?G_FreeHashAnim@@YAXPBDH@Z 004158b0 f   game.obj
 0001:000148e0       ?A_InitEnemyFlags@@YAXXZ   004158e0 f   game.obj
 0001:00014e20       ?P_SetupMiscInputSettings@@YAXXZ 00415e20 f   game.obj
 0001:00016580       _time                      00417580 f   game.obj
 0001:000165a0       _xstrdup                   004175a0 f   game.obj
 0001:000165d0       _BGetTime                  004175d0 f   game.obj
 0001:000165e0       _G_GetTeamPalette          004175e0 f   game.obj
 0001:00016610       _G_NewGame_EnterLevel      00417610 f   game.obj
 0001:00016650       ?idle@@YAXXZ               00417650 f   game.obj
 0001:00016660       ?G_CheckCommandLine@@YAXHPBQBD@Z 00417660 f   game.obj
 0001:00017d60       _Bstrncpyz                 00418d60 f   game.obj
 0001:00017d90       _dup_filename              00418d90 f   game.obj
 0001:00017de0       _xmalloc                   00418de0 f   game.obj
 0001:00017e10       ?G_ShowParameterHelp@@YAXXZ 00418e10 f   game.obj
 0001:00017e60       ?G_ShowDebugHelp@@YAXXZ    00418e60 f   game.obj
 0001:00017eb0       ?G_AddDemo@@YAXPBD@Z       00418eb0 f   game.obj
 0001:00017fa0       ?G_DisplayLogo@@YAXXZ      00418fa0 f   game.obj
 0001:00018750       ?G_PostLoadPalette@@YAXXZ  00419750 f   game.obj
 0001:000187f0       ?G_FatalEngineError@@YAXXZ 004197f0 f   game.obj
 0001:00018840       ?G_Startup@@YAXXZ          00419840 f   game.obj
 0001:00018cc0       ?G_CompileScripts@@YAXXZ   00419cc0 f   game.obj
 0001:00018e50       ?G_CheckGametype@@YAXXZ    00419e50 f   game.obj
 0001:00018ec0       ?G_HandleMemErr@@YAXHPBD0@Z 00419ec0 f   game.obj
 0001:00018f10       ?G_EndOfLevel@@YAHXZ       00419f10 f   game.obj
 0001:000190b0       ?check_filename_casing@@YAHXZ 0041a0b0 f   game.obj
 0001:000190e0       ?G_MoveLoop@@YAHXZ         0041a0e0 f   game.obj
 0001:000197e0       _G_UpdateInterpolations    0041a7e0 f   game.obj
 0001:00019820       ?G_DoOrderScreen@@YAXXZ    0041a820 f   game.obj
 0001:00019940       ?G_PrintTime3@@YAPBDH@Z    0041a940 f   game.obj
 0001:000199a0       ?G_PrintTime_ClockPad@@YAHXZ 0041a9a0 f   game.obj
 0001:00019bb0       ?G_PrintTime2@@YAPBDH@Z    0041abb0 f   game.obj
 0001:0001ae60       ?G_BonusCutscenes@@YAXXZ   0041be60 f   game.obj
 0001:0001bc80       ?G_HandleEventsWhileNoInput@@YAXXZ 0041cc80 f   game.obj
 0001:0001bca0       ?G_PlaySoundWhileNoInput@@YAHH@Z 0041cca0 f   game.obj
 0001:0001bcf0       ?G_DisplayMPResultsScreen@@YAXXZ 0041ccf0 f   game.obj
 0001:0001c1c0       ?G_DrawCameraText@@YAXF@Z  0041d1c0 f   game.obj
 0001:0001c6d0       _ksgn                      0041d6d0 f   game.obj
 0001:0001cd20       ?G_SetupGameButtons@@YAXXZ 0041dd20 f   game.obj
 0001:0001cfa0       _sector_tracker_hook       0041dfa0 f   game.obj
 0001:0001d000       _wall_tracker_hook         0041e000 f   game.obj
 0001:0001d060       _sprite_tracker_hook       0041e060 f   game.obj
 0001:0001e1c0       _mulscale16                0041f1c0 f   actors.obj
 0001:0001ef20       _krand                     0041ff20 f   actors.obj
 0001:0001ef50       _P_GetP                    0041ff50 f   actors.obj
 0001:0001ef80       _A_CheckEnemySprite        0041ff80 f   actors.obj
 0001:0001efa0       _A_CheckEnemyTile          0041ffa0 f   actors.obj
 0001:0001efc0       ?G_WallSpriteDist@@YAHPBUtwalltype@@PBUspritetype@@@Z 0041ffc0 f   actors.obj
 0001:0001f000       _klabs                     00420000 f   actors.obj
 0001:0001f700       _yax_waltosecmask          00420700 f   actors.obj
 0001:0001f720       ?Proj_MaybeDoTransport@@YAHHQBUtspritetype@@HH@Z 00420720 f   actors.obj
 0001:0001f880       ?A_CheckNeedZUpdate@@YAHHHPAH@Z 00420880 f   actors.obj
 0001:0001f9a0       ?A_CheckNoSE7Water@@YAHPBUspritetype@@HHPAH@Z 004209a0 f   actors.obj
 0001:0001fa70       ?A_DeleteLight@@YAXH@Z     00420a70 f   actors.obj
 0001:0001fbd0       _getrendermode             00420bd0 f   actors.obj
 0001:0001fbe0       _VM_HaveEvent              00420be0 f   actors.obj
 0001:0001ff70       _getflorzofslope           00420f70 f   actors.obj
 0001:00020200       ?G_ToggleWallInterpolation@@YAHHH@Z 00421200 f   actors.obj
 0001:00020470       _VM_OnEventWithBoth        00421470 f   actors.obj
 0001:00020c90       _P_Get                     00421c90 f   actors.obj
 0001:00020cb0       ?P_Nudge@@YAXHHH@Z         00421cb0 f   actors.obj
 0001:00021950       ?A_DoLight@@YAXHH@Z        00422950 f   actors.obj
 0001:00023230       _VM_OnEvent                00424230 f   actors.obj
 0001:00023270       ?G_MoveZombieActors@@YAXXZ 00424270 f   actors.obj
 0001:000238c0       ?G_MovePlayers@@YAXXZ      004248c0 f   actors.obj
 0001:000240a0       _logapproach               004250a0 f   actors.obj
 0001:000240d0       _A_SetSprite               004250d0 f   actors.obj
 0001:000241c0       _A_MoveSprite              004251c0 f   actors.obj
 0001:000241e0       _G_CheckForSpaceCeiling    004251e0 f   actors.obj
 0001:00024280       _G_CheckForSpaceFloor      00425280 f   actors.obj
 0001:00024320       ?G_HaveActor@@YAHH@Z       00425320 f   actors.obj
 0001:00024340       ?G_MoveFX@@YAXXZ           00425340 f   actors.obj
 0001:00024950       _S_IsAmbientSFX            00425950 f   actors.obj
 0001:000249b0       ?G_MoveFallers@@YAXXZ      004259b0 f   actors.obj
 0001:00024ec0       ?G_MoveStandables@@YAXXZ   00425ec0 f   actors.obj
 0001:00028230       _G_CheckPlayerInSector     00429230 f   actors.obj
 0001:000282b0       ?G_MoveWeapons@@YAXXZ      004292b0 f   actors.obj
 0001:000293b0       _ksgn                      0042a3b0 f   actors.obj
 0001:000293d0       ?A_DoProjectileBounce@@YAXH@Z 0042a3d0 f   actors.obj
 0001:000296c0       _divscale17                0042a6c0 f   actors.obj
 0001:000296e0       _divscale                  0042a6e0 f   actors.obj
 0001:00029720       _tabledivide64             0042a720 f   actors.obj
 0001:000297f0       _dmulscale8                0042a7f0 f   actors.obj
 0001:00029820       _mulscale10                0042a820 f   actors.obj
 0001:00029830       _mulscale14                0042a830 f   actors.obj
 0001:00029840       ?P_HandleBeingSpitOn@@YAXPAUDukePlayer_t@@@Z 0042a840 f   actors.obj
 0001:00029930       ?G_WeaponHitCeilingOrFloor@@YAXHPAUspritetype@@PAH@Z 0042a930 f   actors.obj
 0001:00029a50       ?Proj_BounceOffWall@@YAXPAUspritetype@@H@Z 0042aa50 f   actors.obj
 0001:00029b10       ?Proj_MaybeDamageCF@@YAHPBUspritetype@@@Z 0042ab10 f   actors.obj
 0001:00029c20       ?Proj_MoveCustom@@YAXH@Z   0042ac20 f   actors.obj
 0001:0002a720       ?A_DoProjectileEffects@@YAXHPBUvec3_t@@H@Z 0042b720 f   actors.obj
 0001:0002a880       ?P_Submerge@@YAHHHPAUDukePlayer_t@@HH@Z 0042b880 f   actors.obj
 0001:0002a990       ?P_Emerge@@YAHHHPAUDukePlayer_t@@HH@Z 0042b990 f   actors.obj
 0001:0002aa50       ?P_FinishWaterChange@@YAXHPAUDukePlayer_t@@HHH@Z 0042ba50 f   actors.obj
 0001:0002abd0       ?G_MoveTransports@@YAXXZ   0042bbd0 f   actors.obj
 0001:0002c000       ?A_CheckNonTeleporting@@YAHH@Z 0042d000 f   actors.obj
 0001:0002c0b0       ?G_MoveActors@@YAXXZ       0042d0b0 f   actors.obj
 0001:000306f0       _A_Shoot                   004316f0 f   actors.obj
 0001:00030710       _P_PalFrom                 00431710 f   actors.obj
 0001:00030750       ?A_FindLocator@@YAFHH@Z    00431750 f   actors.obj
 0001:000307d0       ?G_MoveMisc@@YAXXZ         004317d0 f   actors.obj
 0001:00032670       _getzsofslope              00433670 f   actors.obj
 0001:000326a0       ?G_MoveEffectors@@YAXXZ    004336a0 f   actors.obj
 0001:0003a260       _mulscale12                0043b260 f   actors.obj
 0001:0003a270       ?move_rotfixed_sprite@@YAHHHH@Z 0043b270 f   actors.obj
 0001:0003a450       ?G_FindExplosionInSector@@YAHH@Z 0043b450 f   actors.obj
 0001:0003a4c0       ?HandleSE31@@YAXHHHHH@Z    0043b4c0 f   actors.obj
 0001:0003a730       ?MaybeTrainKillPlayer@@YAXPBUspritetype@@H@Z 0043b730 f   actors.obj
 0001:0003a890       ?MaybeTrainKillEnemies@@YAXHH@Z 0043b890 f   actors.obj
 0001:0003aa00       ?G_DoEffectorLights@@YAXXZ 0043ba00 f   actors.obj
 0001:0003b8c0       _sector_tracker_hook       0043c8c0 f   actors.obj
 0001:0003b920       _wall_tracker_hook         0043c920 f   actors.obj
 0001:0003b980       _sprite_tracker_hook       0043c980 f   actors.obj
 0001:0003c940       _xcalloc                   0043d940 f   anim.obj
 0001:0003d100       _Bstrncpyz                 0043e100 f   anim.obj
 0001:0003d130       _getticks                  0043e130 f   anim.obj
 0001:0003d140       _getrendermode             0043e140 f   anim.obj
 0001:0003d150       _rotatesprite_fs           0043e150 f   anim.obj
 0001:0003d1a0       _G_HandleAsync             0043e1a0 f   anim.obj
 0001:0003d1b0       _VM_OnEventWithReturn      0043e1b0 f   anim.obj
 0001:0003d1f0       _VM_HaveEvent              0043e1f0 f   anim.obj
 0001:0003d9f0       _B_PASS16                  0043e9f0 f   animvpx.obj
 0001:0003da00       _B_PASS32                  0043ea00 f   animvpx.obj
 0001:0003da10       ?animvpx_check_header@@YAHPBUanimvpx_ivf_header_t@@@Z 0043ea10 f   animvpx.obj
 0001:0003dbd0       ?get_codec_error@@YAXPAUanimvpx_codec_ctx@@@Z 0043ebd0 f   animvpx.obj
 0001:0003e230       _clamp                     0043f230 f   animvpx.obj
 0001:0003e270       _getticks                  0043f270 f   animvpx.obj
 0001:0003e280       _vpx_codec_control_VP8D_GET_FRAME_CORRUPTED 0043f280 f   animvpx.obj
 0001:0003e2a0       ?animvpx_read_frame@@YAHHPAPAEPAI1@Z 0043f2a0 f   animvpx.obj
 0001:00040040       _VM_OnEventWithReturn      00441040 f   cheats.obj
 0001:00040080       _VM_HaveEvent              00441080 f   cheats.obj
 0001:000400b0       ?G_CheatGetInv@@YAXXZ      004410b0 f   cheats.obj
 0001:00040150       ?doinvcheat@@YAXHHH@Z      00441150 f   cheats.obj
 0001:000401b0       ?end_cheat@@YAXXZ          004411b0 f   cheats.obj
 0001:000401e0       _sector_tracker_hook       004411e0 f   cheats.obj
 0001:00040240       _sprite_tracker_hook       00441240 f   cheats.obj
 0001:00040360       _scale                     00441360 f   sbar.obj
 0001:000403a0       _tabledivide64             004413a0 f   sbar.obj
 0001:00040a30       _rotatesprite_win          00441a30 f   sbar.obj
 0001:00040a80       ?invensc@@YAHH@Z           00441a80 f   sbar.obj
 0001:00040c00       _rotatesprite_fs           00441c00 f   sbar.obj
 0001:00042330       _getrendermode             00443330 f   sbar.obj
 0001:00042340       ?sbarx@@YAHH@Z             00443340 f   sbar.obj
 0001:00042390       ?sbary@@YAHH@Z             00443390 f   sbar.obj
 0001:000423f0       ?G_PatchStatusBar@@YAXHHHH@Z 004433f0 f   sbar.obj
 0001:00042560       _rotatesprite              00443560 f   sbar.obj
 0001:000425b0       ?G_DrawInvNum@@YAXHHHDDH@Z 004435b0 f   sbar.obj
 0001:000428d0       ?G_DrawWeapAmounts@@YAXPBUDukePlayer_t@@HHH@Z 004438d0 f   sbar.obj
 0001:00042dd0       ?G_DrawWeapNum@@YAXFHHHHH@Z 00443dd0 f   sbar.obj
 0001:000430a0       ?G_DrawWeapNum2@@YAXDHHHHD@Z 004440a0 f   sbar.obj
 0001:00043490       ?G_DrawDigiNum_@@YAXHHHHDH@Z 00444490 f   sbar.obj
 0001:00043520       ?G_DrawDigiNum@@YAXHHHDH@Z 00444520 f   sbar.obj
 0001:00043550       ?G_DrawAltDigiNum@@YAXHHHDH@Z 00444550 f   sbar.obj
 0001:00043810       ?sbarxr@@YAHH@Z            00444810 f   sbar.obj
 0001:00043870       ?G_GetInvAmount@@YAHPBUDukePlayer_t@@@Z 00444870 f   sbar.obj
 0001:00043940       ?G_GetInvOn@@YAHPBUDukePlayer_t@@@Z 00444940 f   sbar.obj
 0001:000439a0       ?G_GetMorale@@YAHHH@Z      004449a0 f   sbar.obj
 0001:000439c0       ?rotatesprite_althud@@YAXHHHFFCDH@Z 004449c0 f   sbar.obj
 0001:00043a90       ?rotatesprite_althudr@@YAXHHHFFCDH@Z 00444a90 f   sbar.obj
 0001:00044540       _VM_OnEventWithReturn      00445540 f   sbar.obj
 0001:00044580       _VM_HaveEvent              00445580 f   sbar.obj
 0001:000446b0       _scale                     004456b0 f   screentext.obj
 0001:000446f0       _tabledivide64             004456f0 f   screentext.obj
 0001:000448c0       _xmalloc                   004458c0 f   screentext.obj
 0001:00045430       _SetIfGreater              00446430 f   screentext.obj
 0001:00046c30       _klabs                     00447c30 f   screentext.obj
 0001:00046c40       _ksgn                      00447c40 f   screentext.obj
 0001:00046c60       _getrendermode             00447c60 f   screentext.obj
 0001:00046c70       ?texto@@YAHH@Z             00447c70 f   screentext.obj
 0001:00046ca0       ?texta@@YAHH@Z             00447ca0 f   screentext.obj
 0001:00046d00       _clamp                     00447d00 f   screentext.obj
 0001:00046d40       ?calc_ybase@@YAHH@Z        00447d40 f   screentext.obj
 0001:000473e0       _getpskyidx                004483e0 f   common.obj
 0001:00047720       _dup_filename              00448720 f   common.obj
 0001:00047770       _Bstrncpyz                 00448770 f   common.obj
 0001:000477a0       _xmalloc                   004487a0 f   common.obj
 0001:00047ba0       ?G_TryLoadingGrp@@YAHQBD@Z 00448ba0 f   common.obj
 0001:00047bf0       ?G_LoadGrpDependencyChain@@YAHQBUgrpfile_t@@@Z 00448bf0 f   common.obj
 0001:00047c80       ?G_LoadAddon@@YAXXZ        00448c80 f   common.obj
 0001:000480a0       ?G_ReadRegistryValue@@YAHQBD0QADPAK@Z 004490a0 f   common.obj
 0001:00048250       _xstrdup                   00449250 f   common.obj
 0001:00048280       _xcalloc                   00449280 f   common.obj
 0001:00048400       _xrealloc                  00449400 f   common.obj
 0001:00048910       ?S_TryExtensionReplacements@@YAHQADDE@Z 00449910 f   common.obj
 0001:000489b0       ?S_TryFormats@@YAHQAD0D@Z  004499b0 f   common.obj
 0001:00049030       ?Demo_WriteSync@@YAXXZ     0044a030 f   demo.obj
 0001:0004a3e0       _rotatesprite              0044b3e0 f   demo.obj
 0001:0004a430       _rotatesprite_fs           0044b430 f   demo.obj
 0001:0004a480       _getticks                  0044b480 f   demo.obj
 0001:0004a490       _G_HandleAsync             0044b490 f   demo.obj
 0001:0004a4a0       _calc_smoothratio          0044b4a0 f   demo.obj
 0001:0004a4c0       _clamp                     0044b4c0 f   demo.obj
 0001:0004a500       ?Demo_RestoreModes@@YAXH@Z 0044b500 f   demo.obj
 0001:0004a590       ?G_OpenDemoRead@@YAHH@Z    0044b590 f   demo.obj
 0001:0004a780       ?Demo_UpdateState@@YAHH@Z  0044b780 f   demo.obj
 0001:0004a7e0       ?Demo_ReadSync@@YAHH@Z     0044b7e0 f   demo.obj
 0001:0004a8b0       ?Demo_StopProfiling@@YAXXZ 0044b8b0 f   demo.obj
 0001:0004a8c0       ?Demo_GToc@@YAXN@Z         0044b8c0 f   demo.obj
 0001:0004a8f0       ?Demo_RToc@@YAXNN@Z        0044b8f0 f   demo.obj
 0001:0004a930       ?Demo_DisplayProfStatus@@YAXXZ 0044b930 f   demo.obj
 0001:0004a9f0       ?Demo_SetupProfile@@YAXXZ  0044b9f0 f   demo.obj
 0001:0004aa40       ?Demo_FinishProfile@@YAXXZ 0044ba40 f   demo.obj
 0001:0004b380       _clamp                     0044c380 f   gamedef.obj
 0001:0004b450       _dup_filename              0044c450 f   gamedef.obj
 0001:0004b4a0       _Bstrncpyz                 0044c4a0 f   gamedef.obj
 0001:0004b4d0       _xmalloc                   0044c4d0 f   gamedef.obj
 0001:0004b500       ?check_filename_case@@YAXPBD@Z 0044c500 f   gamedef.obj
 0001:0004b840       _xcalloc                   0044c840 f   gamedef.obj
 0001:0004bbb0       ?C_ReplaceQuoteSubstring@@YAXIQBD0@Z 0044cbb0 f   gamedef.obj
 0001:0004c490       _getticks                  0044d490 f   gamedef.obj
 0001:0004c4a0       ?C_SetScriptSize@@YAHH@Z   0044d4a0 f   gamedef.obj
 0001:0004c800       _xrealloc                  0044d800 f   gamedef.obj
 0001:0004c830       ?C_Include@@YAXPBD@Z       0044d830 f   gamedef.obj
 0001:0004ca10       ?C_SkipComments@@YAHXZ     0044da10 f   gamedef.obj
 0001:0004cd20       ?ispecial@@YAHD@Z          0044dd20 f   gamedef.obj
 0001:0004cd80       ?C_NextLine@@YAXXZ         0044dd80 f   gamedef.obj
 0001:0004cdc0       ?C_ParseCommand@@YAHH@Z    0044ddc0 f   gamedef.obj
 0001:00053d00       _xstrdup                   00454d00 f   gamedef.obj
 0001:00053d30       _klabs                     00454d30 f   gamedef.obj
 0001:00053d40       ?C_GetLabelType@@YAPADH@Z  00454d40 f   gamedef.obj
 0001:00053e10       ?C_SkipSpace@@YAXXZ        00454e10 f   gamedef.obj
 0001:00053e50       ?isaltok@@YAHD@Z           00454e50 f   gamedef.obj
 0001:00053ed0       ?C_GetLabelNameID@@YAHPBUmemberlabel_t@@QBUhashtable_t@@PBD@Z 00454ed0 f   gamedef.obj
 0001:00053f10       ?C_GetNextLabelName@@YAXXZ 00454f10 f   gamedef.obj
 0001:00053fd0       ?C_IsLabelChar@@YAHDH@Z    00454fd0 f   gamedef.obj
 0001:00054040       ?C_GetKeyword@@YAHXZ       00455040 f   gamedef.obj
 0001:000540f0       ?C_GetNextKeyword@@YAHXZ   004550f0 f   gamedef.obj
 0001:000542f0       ?C_GetNextVarType@@YAXH@Z  004552f0 f   gamedef.obj
 0001:00055130       ?C_GetLabelNameOffset@@YAHQBUhashtable_t@@PBD@Z 00456130 f   gamedef.obj
 0001:00055150       ?parse_decimal_number@@YAHXZ 00456150 f   gamedef.obj
 0001:000551f0       ?parse_hex_constant@@YAHPBD@Z 004561f0 f   gamedef.obj
 0001:00055250       ?C_GetManyVarsType@@YAXHH@Z 00456250 f   gamedef.obj
 0001:00055280       ?C_GetNextValue@@YAHH@Z    00456280 f   gamedef.obj
 0001:000557f0       ?C_GetStructureIndexes@@YAHHQBUhashtable_t@@@Z 004567f0 f   gamedef.obj
 0001:00055990       ?C_IntPow2@@YAHH@Z         00456990 f   gamedef.obj
 0001:000559c0       ?C_Pow2IntLogBase2@@YAIH@Z 004569c0 f   gamedef.obj
 0001:00055a20       ?C_CheckMalformedBranch@@YAHH@Z 00456a20 f   gamedef.obj
 0001:00055b40       ?C_CheckEmptyBranch@@YAHHH@Z 00456b40 f   gamedef.obj
 0001:00055c50       ?C_CountCaseStatements@@YAHXZ 00456c50 f   gamedef.obj
 0001:00055d10       ?C_SetDefName@@YAHPBD@Z    00456d10 f   gamedef.obj
 0001:00055d60       ?C_DefineProjectile@@YAXHHH@Z 00456d60 f   gamedef.obj
 0001:00056020       ?C_SetCfgName@@YAXPBD@Z    00457020 f   gamedef.obj
 0001:00056200       _stat                      00457200 f   gamedef.obj
 0001:00056220       ?C_BitOrNextValue@@YAXPAH@Z 00457220 f   gamedef.obj
 0001:00056250       ?C_FinishBitOr@@YAXH@Z     00457250 f   gamedef.obj
 0001:000562d0       ?C_FillEventBreakStackWithJump@@YAXPAHH@Z 004572d0 f   gamedef.obj
 0001:00056350       ?C_AddDefaultDefinitions@@YAXXZ 00457350 f   gamedef.obj
 0001:00056960       ?C_AddDefinition@@YAXPBDHH@Z 00457960 f   gamedef.obj
 0001:000569f0       ?C_ScriptVersionString@@YAPBDH@Z 004579f0 f   gamedef.obj
 0001:00057240       ?VM_EventCommon_@@YAHHHHHH@Z 00458240 f   gameexec.obj
 0001:000573d0       ?VM_DeleteSprite@@YAXHH@Z  004583d0 f   gameexec.obj
 0001:00057660       _klabs                     00458660 f   gameexec.obj
 0001:00057670       _krand                     00458670 f   gameexec.obj
 0001:000576a0       _A_CheckEnemySprite        004586a0 f   gameexec.obj
 0001:000576c0       _A_CheckEnemyTile          004586c0 f   gameexec.obj
 0001:00057ca0       _A_SetSprite               00458ca0 f   gameexec.obj
 0001:00057d90       _A_MoveSprite              00458d90 f   gameexec.obj
 0001:00057db0       ?VM_GetZRange@@YAXHPAH0H@Z 00458db0 f   gameexec.obj
 0001:00058140       _G_CheckForSpaceCeiling    00459140 f   gameexec.obj
 0001:000581e0       _G_CheckForSpaceFloor      004591e0 f   gameexec.obj
 0001:00058380       _localtime                 00459380 f   gameexec.obj
 0001:000583a0       _time                      004593a0 f   gameexec.obj
 0001:00058420       ?VM_Execute@@YAXH@Z        00459420 f   gameexec.obj
 0001:00068410       _system_15bit_rand         00469410 f   gameexec.obj
 0001:00068420       _Bstrncpyz                 00469420 f   gameexec.obj
 0001:00068450       _xmalloc                   00469450 f   gameexec.obj
 0001:00068480       _xaligned_malloc           00469480 f   gameexec.obj
 0001:000684b0       _mulscale                  004694b0 f   gameexec.obj
 0001:000684d0       _mulscale15                004694d0 f   gameexec.obj
 0001:000684e0       _mulscale16                004694e0 f   gameexec.obj
 0001:000684f0       _ksgn                      004694f0 f   gameexec.obj
 0001:00068510       _getceilzofslope           00469510 f   gameexec.obj
 0001:00068540       _getflorzofslope           00469540 f   gameexec.obj
 0001:00068570       _getticks                  00469570 f   gameexec.obj
 0001:00068580       _A_Shoot                   00469580 f   gameexec.obj
 0001:000685a0       _P_PalFrom                 004695a0 f   gameexec.obj
 0001:000685e0       _P_GetP                    004695e0 f   gameexec.obj
 0001:00068610       _Sect_ClearInterpolation   00469610 f   gameexec.obj
 0001:00068630       _Sect_SetInterpolation     00469630 f   gameexec.obj
 0001:00068650       ?Gv_DivVar@@YIXHH@Z        00469650 f   gameexec.obj
 0001:00068830       ?Gv_AddVar@@YIXHH@Z        00469830 f   gameexec.obj
 0001:000689a0       ?Gv_SubVar@@YIXHH@Z        004699a0 f   gameexec.obj
 0001:00068b10       ?Gv_MulVar@@YIXHH@Z        00469b10 f   gameexec.obj
 0001:00068c90       ?Gv_ModVar@@YIXHH@Z        00469c90 f   gameexec.obj
 0001:00068e10       ?Gv_AndVar@@YIXHH@Z        00469e10 f   gameexec.obj
 0001:00068f80       ?Gv_XorVar@@YIXHH@Z        00469f80 f   gameexec.obj
 0001:000690f0       ?Gv_OrVar@@YIXHH@Z         0046a0f0 f   gameexec.obj
 0001:00069260       ?G_HaveActor@@YAHH@Z       0046a260 f   gameexec.obj
 0001:00069280       ?VM_CheckSquished@@YAHXZ   0046a280 f   gameexec.obj
 0001:00069460       _yax_getbunches            0046a460 f   gameexec.obj
 0001:00069490       ?P_ForceAngle@@YAXPAUDukePlayer_t@@@Z 0046a490 f   gameexec.obj
 0001:00069500       ?P_AddWeaponAmmoCommon@@YAXPAUDukePlayer_t@@HH@Z 0046a500 f   gameexec.obj
 0001:00069560       ?P_AddWeaponMaybeSwitch@@YAXPAUDukePlayer_t@@H@Z 0046a560 f   gameexec.obj
 0001:00069660       _P_Get                     0046a660 f   gameexec.obj
 0001:00069680       ?VM_AddWeapon@@YAHHHPAUDukePlayer_t@@@Z 0046a680 f   gameexec.obj
 0001:00069730       ?VM_Fall@@YAXHPAUspritetype@@@Z 0046a730 f   gameexec.obj
 0001:00069bc0       ?A_GetWaterZOffset@@YAHH@Z 0046abc0 f   gameexec.obj
 0001:00069ca0       ?A_GetVerticalVel@@YAHPBUactor_t@@@Z 0046aca0 f   gameexec.obj
 0001:00069ce0       ?VM_ResetPlayer@@YAHHHH@Z  0046ace0 f   gameexec.obj
 0001:00069dd0       ?G_ShowView@@YAXUvec3_t@@HHHHHHHH@Z 0046add0 f   gameexec.obj
 0001:0006a080       _clamp                     0046b080 f   gameexec.obj
 0001:0006a0c0       _scale                     0046b0c0 f   gameexec.obj
 0001:0006a100       _tabledivide64             0046b100 f   gameexec.obj
 0001:0006a1d0       _swaplong                  0046b1d0 f   gameexec.obj
 0001:0006a1f0       _getrendermode             0046b1f0 f   gameexec.obj
 0001:0006a200       _G_RestoreInterpolations   0046b200 f   gameexec.obj
 0001:0006a250       _calc_smoothratio          0046b250 f   gameexec.obj
 0001:0006a8a0       ?VM_Move@@YAXXZ            0046b8a0 f   gameexec.obj
 0001:0006b380       ?VM_AlterAng@@YAXH@Z       0046c380 f   gameexec.obj
 0001:0006b840       ?VM_AddAngle@@YAXHH@Z      0046c840 f   gameexec.obj
 0001:0006b8b0       ?VM_FacePlayer@@YAXH@Z     0046c8b0 f   gameexec.obj
 0001:0006b950       ?VM_GetCeilZOfSlope@@YAHXZ 0046c950 f   gameexec.obj
 0001:0006ba00       ?VM_GetFlorZOfSlope@@YAHXZ 0046ca00 f   gameexec.obj
 0001:0006ca10       _sprite_tracker_hook       0046da10 f   gameexec.obj
 0001:0006ca70       _wall_tracker_hook         0046da70 f   gameexec.obj
 0001:00072ce0       _xmalloc                   00473ce0 f   gamevars.obj
 0001:00072d10       _xaligned_malloc           00473d10 f   gamevars.obj
 0001:00072d40       ?Gv_Free@@YAHXZ            00473d40 f   gamevars.obj
 0001:00073870       _xcalloc                   00474870 f   gamevars.obj
 0001:00075900       ?Gv_GetVarIndex@@YAHPBD@Z  00476900 f   gamevars.obj
 0001:00075b30       ?G_StaticToDynamicTile@@YAHH@Z 00476b30 f   gamevars.obj
 0001:00075c70       ?G_StaticToDynamicSound@@YAHH@Z 00476c70 f   gamevars.obj
 0001:00075d60       ?Gv_Clear@@YAXXZ           00476d60 f   gamevars.obj
 0001:00075e10       ?Gv_AddSystemVars@@YAXXZ   00476e10 f   gamevars.obj
 0001:00077060       ?Gv_GetVarDataPtr@@YAPAHPBD@Z 00478060 f   gamevars.obj
 0001:00077840       _sector_tracker_hook       00478840 f   gamevars.obj
 0001:000778a0       _wall_tracker_hook         004788a0 f   gamevars.obj
 0001:00077900       _sprite_tracker_hook       00478900 f   gamevars.obj
 0001:00079080       ?MenuEntry_DisableOnCondition@@YAXQAUMenuEntry_t@@H@Z 0047a080 f   menus.obj
 0001:00079180       _scale                     0047a180 f   menus.obj
 0001:000791c0       _tabledivide64             0047a1c0 f   menus.obj
 0001:000797c0       _getrendermode             0047a7c0 f   menus.obj
 0001:000797d0       _VM_OnEventWithReturn      0047a7d0 f   menus.obj
 0001:00079810       _VM_HaveEvent              0047a810 f   menus.obj
 0001:00079840       ?WithSDL2_StartTextInput@@YAXXZ 0047a840 f   menus.obj
 0001:00079850       ?M_MenuEntryFocus@@YAXXZ   0047a850 f   menus.obj
 0001:000798a0       ?M_MenuFileSelectInit@@YAXPAUMenuFileSelect_t@@@Z 0047a8a0 f   menus.obj
 0001:00079980       ?M_FindMenu@@YAPAUMenu_t@@H@Z 0047a980 f   menus.obj
 0001:000799b0       ?M_FindMenuBinarySearch@@YAPAUMenu_t@@HII@Z 0047a9b0 f   menus.obj
 0001:0007a240       _clamp                     0047b240 f   menus.obj
 0001:0007a280       _rotatesprite_fs_alpha     0047b280 f   menus.obj
 0001:0007a2d0       ?M_BlackTranslucentBackgroundOK@@YAHH@Z 0047b2d0 f   menus.obj
 0001:0007a310       ?M_UpdateScreenOK@@YAHH@Z  0047b310 f   menus.obj
 0001:0007a370       ?M_RunMenu@@YAXPAUMenu_t@@Uvec2_t@@@Z 0047b370 f   menus.obj
 0001:0007ada0       _klabs                     0047bda0 f   menus.obj
 0001:0007adb0       _rotatesprite_fs           0047bdb0 f   menus.obj
 0001:0007ae00       ?M_DrawTopBar@@YAXUvec2_t@@@Z 0047be00 f   menus.obj
 0001:0007ae40       ?M_DrawTopBarCaption@@YAXPBDUvec2_t@@@Z 0047be40 f   menus.obj
 0001:0007af10       ?M_PreMenu@@YAXH@Z         0047bf10 f   menus.obj
 0001:0007b8c0       ?M_PreMenuDrawBackground@@YAXHUvec2_t@@@Z 0047c8c0 f   menus.obj
 0001:0007ba10       ?M_DrawBackground@@YAXUvec2_t@@@Z 0047ca10 f   menus.obj
 0001:0007ba50       ?M_PreMenuDraw@@YAXHPAUMenuEntry_t@@Uvec2_t@@@Z 0047ca50 f   menus.obj
 0001:0007f0c0       _G_GetTeamPalette          004800c0 f   menus.obj
 0001:0007f0f0       ?shadowminitext@@YAXHHPBDH@Z 004800f0 f   menus.obj
 0001:0007f180       ?creditsminitext@@YAXHHPBDH@Z 00480180 f   menus.obj
 0001:0007f210       ?M_PreMenuOptionListDraw@@YAXPAUMenuEntry_t@@Uvec2_t@@@Z 00480210 f   menus.obj
 0001:0007f3d0       ?M_PreMenuCustom2ColScreenDraw@@YAXPAUMenuEntry_t@@Uvec2_t@@@Z 004803d0 f   menus.obj
 0001:0007f570       ?M_BlackRectangle@@YAXHHHHH@Z 00480570 f   menus.obj
 0001:0007f640       ?xdim_from_320_16@@YAHH@Z  00480640 f   menus.obj
 0001:0007f690       ?ydim_from_200_16@@YAHH@Z  00480690 f   menus.obj
 0001:0007f6b0       ?M_MenuText@@YA?AUvec2_t@@HHPBUMenuFont_t@@PBDEHH@Z 004806b0 f   menus.obj
 0001:0007f7c0       ?M_ShadePal@@YAXPBUMenuFont_t@@EPAH1@Z 004807c0 f   menus.obj
 0001:0007f830       ?M_MouseWithinBounds@@YAHQBUvec2_t@@HHHH@Z 00480830 f   menus.obj
 0001:0007f880       ?M_MouseOutsideBounds@@YAHQBUvec2_t@@HHHH@Z 00480880 f   menus.obj
 0001:0007f8d0       ?M_RunMenu_Scrollbar@@YAXPAUMenu_t@@QBUMenuMenuFormat_t@@HQAHHUvec2_t@@@Z 004808d0 f   menus.obj
 0001:0007fad0       ?M_RunMenu_MenuMenu@@YAHPAUMenu_t@@PAUMenuMenu_t@@PAUMenuEntry_t@@HUvec2_t@@@Z 00480ad0 f   menus.obj
 0001:00081f70       _Blrintf                   00482f70 f   menus.obj
 0001:00081f90       ?M_MenuEntryOptionSource@@YAHPAUMenuEntry_t@@H@Z 00482f90 f   menus.obj
 0001:00082050       ?rotatesprite_ybounds@@YAXHHHFFCDHHH@Z 00483050 f   menus.obj
 0001:000820b0       ?M_FindOptionBinarySearch@@YAHPAUMenuOption_t@@HII@Z 004830b0 f   menus.obj
 0001:00082190       ?M_RunMenu_MenuOptionList@@YAXPAUMenu_t@@PAUMenuEntry_t@@PAUMenuOption_t@@Uvec2_t@@@Z 00483190 f   menus.obj
 0001:000826d0       ?M_RunMenu_MouseReturn@@YAXPAUMenu_t@@Uvec2_t@@@Z 004836d0 f   menus.obj
 0001:00082800       ?x_widescreen_left@@YAHXZ  00483800 f   menus.obj
 0001:00082830       ?M_RunMenu_AbbreviateNameIntoBuffer@@YAXPBDH@Z 00483830 f   menus.obj
 0001:000828a0       ?M_RunMenuRecurse@@YAXHUvec2_t@@@Z 004838a0 f   menus.obj
 0001:00082900       ?M_RunMenuInput_MenuMenu_MovementVerify@@YAPAUMenuEntry_t@@PAUMenuMenu_t@@@Z 00483900 f   menus.obj
 0001:000829a0       ?M_RunMenuInput_MenuEntryLink_Activate@@YAXPAUMenuEntry_t@@@Z 004839a0 f   menus.obj
 0001:000829e0       ?M_MenuEntryLinkActivate@@YAXPAUMenuEntry_t@@@Z 004839e0 f   menus.obj
 0001:00082f10       _G_NewGame_EnterLevel      00483f10 f   menus.obj
 0001:00082f50       ?M_StartGameWithoutSkill@@YAXXZ 00483f50 f   menus.obj
 0001:00082fc0       ?M_Cheat@@YAXH@Z           00483fc0 f   menus.obj
 0001:00083000       ?M_RunMenuInput_MenuEntryOption_Activate@@YAHPAUMenuEntry_t@@PAUMenuOption_t@@@Z 00484000 f   menus.obj
 0001:00083070       ?M_RunMenuInput_MenuEntryOptionList_MovementVerify@@YAXPAUMenuOption_t@@@Z 00484070 f   menus.obj
 0001:00083160       ?M_RunMenuInput_MenuEntryOption_Movement@@YAHPAUMenuEntry_t@@PAUMenuOption_t@@W4MenuMovement_t@@@Z 00484160 f   menus.obj
 0001:000832c0       ?M_RunMenuInput_MenuEntryOption_Modify@@YAHPAUMenuEntry_t@@PAUMenuOption_t@@H@Z 004842c0 f   menus.obj
 0001:00083340       ?M_MenuEntryOptionModify@@YAHPAUMenuEntry_t@@H@Z 00484340 f   menus.obj
 0001:000837a0       ?M_MenuEntryOptionDidModify@@YAXPAUMenuEntry_t@@@Z 004847a0 f   menus.obj
 0001:000838a0       ?M_RunMenuInput_MenuEntryOptionList_Activate@@YAHPAUMenuEntry_t@@PAUMenuOption_t@@@Z 004848a0 f   menus.obj
 0001:000838e0       ?M_RunMenuInput_MenuEntryCustom2Col_Activate@@YAXPAUMenuEntry_t@@@Z 004848e0 f   menus.obj
 0001:00083900       ?M_MenuCustom2ColScreen@@YAXXZ 00484900 f   menus.obj
 0001:00083920       ?M_RunMenuInput_MenuEntryRangeInt32_MovementVerify@@YAXPAUMenuEntry_t@@PAUMenuRangeInt32_t@@H@Z 00484920 f   menus.obj
 0001:00083950       ?M_MenuEntryRangeInt32Modify@@YAHPAUMenuEntry_t@@H@Z 00484950 f   menus.obj
 0001:00083ab0       _G_SetStatusBarScale       00484ab0 f   menus.obj
 0001:00083ad0       ?M_RunMenuInput_MenuEntryRangeInt32_MovementArbitrary@@YAXPAUMenuEntry_t@@PAUMenuRangeInt32_t@@H@Z 00484ad0 f   menus.obj
 0001:00083b70       ?M_RunMenuInput_MenuEntryRangeFloat_MovementVerify@@YAXPAUMenuEntry_t@@PAUMenuRangeFloat_t@@M@Z 00484b70 f   menus.obj
 0001:00083bb0       ?M_MenuEntryRangeFloatModify@@YAHPAUMenuEntry_t@@M@Z 00484bb0 f   menus.obj
 0001:00083bd0       ?M_MenuEntryRangeFloatDidModify@@YAHPAUMenuEntry_t@@@Z 00484bd0 f   menus.obj
 0001:00083d20       ?M_RunMenuInput_MenuEntryRangeFloat_MovementArbitrary@@YAXPAUMenuEntry_t@@PAUMenuRangeFloat_t@@M@Z 00484d20 f   menus.obj
 0001:00083da0       ?M_RunMenuInput_MenuEntryRangeDouble_MovementVerify@@YAXPAUMenuRangeDouble_t@@N@Z 00484da0 f   menus.obj
 0001:00083dc0       ?M_MenuEntryRangeDoubleModify@@YAHXZ 00484dc0 f   menus.obj
 0001:00083dd0       ?M_RunMenuInput_MenuEntryRangeDouble_MovementArbitrary@@YAXPAUMenuRangeDouble_t@@N@Z 00484dd0 f   menus.obj
 0001:00083e60       ?M_RunMenuInput_MenuEntryString_Activate@@YAXPAUMenuEntry_t@@@Z 00484e60 f   menus.obj
 0001:00083ec0       ?M_MenuEntryStringActivate@@YAXXZ 00484ec0 f   menus.obj
 0001:00083f30       ?M_RunMenuInput_MenuEntryString_Submit@@YAXPAUMenuEntry_t@@PAUMenuString_t@@@Z 00484f30 f   menus.obj
 0001:00083f80       ?WithSDL2_StopTextInput@@YAXXZ 00484f80 f   menus.obj
 0001:00083f90       ?M_MenuEntryStringSubmit@@YAHPAUMenuEntry_t@@PAD@Z 00484f90 f   menus.obj
 0001:000840f0       ?M_RunMenuInput_FileSelect_MovementVerify@@YAXPAUMenuFileSelect_t@@@Z 004850f0 f   menus.obj
 0001:000841d0       ?M_RunMenuInput_FileSelect_Select@@YAXPAUMenuFileSelect_t@@@Z 004851d0 f   menus.obj
 0001:00084250       ?M_MenuFileSelect@@YAXH@Z  00485250 f   menus.obj
 0001:000842c0       ?M_RunMenuInput@@YAXPAUMenu_t@@@Z 004852c0 f   menus.obj
 0001:000850f0       ?M_PreMenuInput@@YAXPAUMenuEntry_t@@@Z 004860f0 f   menus.obj
 0001:000851a0       ?M_PreMenuCustom2ColScreen@@YAHPAUMenuEntry_t@@@Z 004861a0 f   menus.obj
 0001:00085260       ?M_MenuVerify@@YAXH@Z      00486260 f   menus.obj
 0001:00085420       ?M_MenuTextFormSubmit@@YAXPAD@Z 00486420 f   menus.obj
 0001:000857b0       ?M_Cheat_Warp@@YAHQBD@Z    004867b0 f   menus.obj
 0001:000858f0       ?M_Cheat_Skill@@YAHQBD@Z   004868f0 f   menus.obj
 0001:00085960       ?M_CheatStringMatch@@YAHPBD0@Z 00486960 f   menus.obj
 0001:000859d0       ?M_RunMenuInput_MouseAdvance@@YAHXZ 004869d0 f   menus.obj
 0001:00085a20       ?M_RunMenuInput_MouseReturn@@YAHXZ 00486a20 f   menus.obj
 0001:00085b20       ?M_RunMenuInput_MenuMenu_Movement@@YAPAUMenuEntry_t@@PAUMenuMenu_t@@W4MenuMovement_t@@@Z 00486b20 f   menus.obj
 0001:00085ca0       ?M_RunMenuInput_MenuEntryOptionList_Movement@@YAXPAUMenuOption_t@@W4MenuMovement_t@@@Z 00486ca0 f   menus.obj
 0001:00085d70       ?M_RunMenuInput_MenuEntryRangeInt32_Movement@@YAXPAUMenuEntry_t@@PAUMenuRangeInt32_t@@W4MenuMovement_t@@@Z 00486d70 f   menus.obj
 0001:00085f80       ?M_RunMenuInput_MenuEntryRangeFloat_Movement@@YAXPAUMenuEntry_t@@PAUMenuRangeFloat_t@@W4MenuMovement_t@@@Z 00486f80 f   menus.obj
 0001:00086180       ?M_RunMenuInput_MenuEntryRangeDouble_Movement@@YAXPAUMenuRangeDouble_t@@W4MenuMovement_t@@@Z 00487180 f   menus.obj
 0001:00086380       ?M_RunMenuInput_MenuEntryString_Cancel@@YAXPAUMenuString_t@@@Z 00487380 f   menus.obj
 0001:000863a0       ?M_MenuEntryStringCancel@@YAXXZ 004873a0 f   menus.obj
 0001:000863d0       ?M_RunMenuInput_FileSelect_Movement@@YAXPAUMenuFileSelect_t@@W4MenuMovement_t@@@Z 004873d0 f   menus.obj
 0001:00086560       _wall_tracker_hook         00487560 f   menus.obj
 0001:00086ca0       _G_HandleAsync             00487ca0 f   net.obj
 0001:00086cb0       ?display_betascreen@@YAXXZ 00487cb0 f   net.obj
 0001:00086d70       _rotatesprite_fs           00487d70 f   net.obj
 0001:00087120       _xstrdup                   00488120 f   net.obj
 0001:000876d0       ?P_RemovePlayer@@YAXH@Z    004886d0 f   net.obj
 0001:00087e60       _B_UNBUF32                 00488e60 f   net.obj
 0001:00088050       _B_BUF16                   00489050 f   net.obj
 0001:00088060       _B_BUF32                   00489060 f   net.obj
 0001:00088170       _B_UNBUF16                 00489170 f   net.obj
 0001:00088360       _xcalloc                   00489360 f   net.obj
 0001:00088d90       ?Net_CompareActors@@YAHPBX0@Z 00489d90 f   net.obj
 0001:0008add0       _scale                     0048bdd0 f   net.obj
 0001:0008ae10       _tabledivide64             0048be10 f   net.obj
 0001:0008b9c0       _sprite_tracker_hook       0048c9c0 f   net.obj
 0001:0008bbc0       _P_PalFrom                 0048cbc0 f   player.obj
 0001:0008bfe0       _P_GetP                    0048cfe0 f   player.obj
 0001:0008c010       _A_CheckEnemySprite        0048d010 f   player.obj
 0001:0008c030       _A_CheckEnemyTile          0048d030 f   player.obj
 0001:0008c050       ?A_ShootCustom@@YAHHHFQAUvec3_t@@@Z 0048d050 f   player.obj
 0001:0008ce10       _mulscale3                 0048de10 f   player.obj
 0001:0008ce20       _klabs                     0048de20 f   player.obj
 0001:0008ce30       _krand                     0048de30 f   player.obj
 0001:0008ce60       _A_SetSprite               0048de60 f   player.obj
 0001:0008cf50       _A_MoveSprite              0048df50 f   player.obj
 0001:0008cf70       ?A_DoWaterTracers@@YAXHHHHHHH@Z 0048df70 f   player.obj
 0001:0008d120       ?Proj_GetProjectile@@YAPAUprojectile_t@@H@Z 0048e120 f   player.obj
 0001:0008d160       ?A_HitscanProjTrail@@YAXPBUvec3_t@@0HH@Z 0048e160 f   player.obj
 0001:0008d3a0       _getzsofslope              0048e3a0 f   player.obj
 0001:0008d3d0       ?A_SetHitData@@YAXHPBUhitdata_t@@@Z 0048e3d0 f   player.obj
 0001:0008d410       ?safeldist@@YAHHPBUspritetype@@@Z 0048e410 f   player.obj
 0001:0008d450       ?GetAutoAimAngle@@YAHHHHHHPBUvec3_t@@HPAHPAF@Z 0048e450 f   player.obj
 0001:0008d650       _VM_OnEvent                0048e650 f   player.obj
 0001:0008d690       _VM_HaveEvent              0048e690 f   player.obj
 0001:0008d6c0       ?A_FindTargetSprite@@YAHPBUspritetype@@HH@Z 0048e6c0 f   player.obj
 0001:0008df10       _scale                     0048ef10 f   player.obj
 0001:0008df50       _tabledivide64             0048ef50 f   player.obj
 0001:0008e020       _mulscale                  0048f020 f   player.obj
 0001:0008e040       _P_Get                     0048f040 f   player.obj
 0001:0008e060       ?Proj_InsertShotspark@@YAHPBUhitdata_t@@HHHHH@Z 0048f060 f   player.obj
 0001:0008e100       ?Proj_GetExtra@@YAHH@Z     0048f100 f   player.obj
 0001:0008e150       ?A_GetShootZvel@@YAHH@Z    0048f150 f   player.obj
 0001:0008e180       ?P_PreFireHitscan@@YAXHHHPAUvec3_t@@PAHPAFHH@Z 0048f180 f   player.obj
 0001:0008e400       ?Proj_MaybeAddSpread@@YAXHPAHPAFHH@Z 0048f400 f   player.obj
 0001:0008e460       ?A_PreFireHitscan@@YAXPBUspritetype@@PAUvec3_t@@PAHPAFH@Z 0048f460 f   player.obj
 0001:0008e550       ?Proj_DoHitscan@@YAHHHPBUvec3_t@@HFPAUhitdata_t@@@Z 0048f550 f   player.obj
 0001:0008e600       ?Proj_DoRandDecalSize@@YAXHH@Z 0048f600 f   player.obj
 0001:0008e6c0       ?SectorContainsSE13@@YAHH@Z 0048f6c0 f   player.obj
 0001:0008e740       ?P_PostFireHitscan@@YAHHHPAUhitdata_t@@HHHHHHH@Z 0048f740 f   player.obj
 0001:0008edc0       ?CheckShootSwitchTile@@YAHH@Z 0048fdc0 f   player.obj
 0001:0008ee40       ?Proj_MaybeSpawn@@YAXHHPBUhitdata_t@@@Z 0048fe40 f   player.obj
 0001:0008ef00       ?HandleHitWall@@YAXPAUhitdata_t@@@Z 0048ff00 f   player.obj
 0001:0008ef80       _redwallp                  0048ff80 f   player.obj
 0001:0008efc0       ?Proj_MaybeDamageCF2@@YAHHH@Z 0048ffc0 f   player.obj
 0001:0008f070       ?A_PostFireHitscan@@YAHPBUhitdata_t@@HHHHHH@Z 00490070 f   player.obj
 0001:0008f150       ?Proj_CheckBlood@@YAHPBUvec3_t@@PBUhitdata_t@@HH@Z 00490150 f   player.obj
 0001:0008f2b0       ?Proj_HandleKnee@@YAXPAUhitdata_t@@HHHHPBUprojectile_t@@HHHH@Z 004902b0 f   player.obj
 0001:0008f560       ?A_ShootHardcoded@@YAHHHFUvec3_t@@PAUspritetype@@HPAUDukePlayer_t@@@Z 00490560 f   player.obj
 0001:00091220       ?G_InitialActorStrength@@YAHH@Z 00492220 f   player.obj
 0001:00091260       ?G_HaveActor@@YAHH@Z       00492260 f   player.obj
 0001:00091490       _getrendermode             00492490 f   player.obj
 0001:000914a0       ?G_DrawTileScaled@@YAXHHHHHH@Z 004924a0 f   player.obj
 0001:00091650       _rotatesprite              00492650 f   player.obj
 0001:000916a0       _md_tilehasmodel           004926a0 f   player.obj
 0001:00094070       _ksgn                      00495070 f   player.obj
 0001:00094090       _rotatesprite_win          00495090 f   player.obj
 0001:000940e0       ?P_DisplaySpit@@YAXXZ      004950e0 f   player.obj
 0001:00094240       _rotatesprite_fs           00495240 f   player.obj
 0001:00094290       ?P_DisplayFist@@YAHH@Z     00495290 f   player.obj
 0001:00094430       _clamp                     00495430 f   player.obj
 0001:00094470       ?G_DrawWeaponTileWithID@@YAXHHHHHHHE@Z 00495470 f   player.obj
 0001:000944c0       ?G_DrawWeaponTile@@YAXHHHHHHE@Z 004954c0 f   player.obj
 0001:00094630       _logapproach               00495630 f   player.obj
 0001:00094660       ?P_DisplayKnee@@YAHH@Z     00495660 f   player.obj
 0001:00094800       ?P_DisplayKnuckles@@YAHH@Z 00495800 f   player.obj
 0001:00094990       ?P_DisplayTip@@YAHH@Z      00495990 f   player.obj
 0001:00094b20       ?P_DisplayAccess@@YAHH@Z   00495b20 f   player.obj
 0001:00096380       _mulscale9                 00497380 f   player.obj
 0001:000964d0       ?P_AddWeaponNoSwitch@@YAXPAUDukePlayer_t@@H@Z 004974d0 f   player.obj
 0001:000965c0       ?P_ChangeWeapon@@YAXPAUDukePlayer_t@@H@Z 004975c0 f   player.obj
 0001:00096740       _VM_OnEventWithReturn      00497740 f   player.obj
 0001:00097120       _B_BUF32                   00498120 f   player.obj
 0001:0009ac30       _mulscale16                0049bc30 f   player.obj
 0001:0009ac40       _yax_getbunches            0049bc40 f   player.obj
 0001:0009ac70       _uhypsq                    0049bc70 f   player.obj
 0001:0009ac90       _getflorzofslope           0049bc90 f   player.obj
 0001:0009acc0       ?P_IncurDamage@@YAXPAUDukePlayer_t@@@Z 0049bcc0 f   player.obj
 0001:0009ae10       ?P_DoCounters@@YAHH@Z      0049be10 f   player.obj
 0001:0009b6e0       _A_Shoot                   0049c6e0 f   player.obj
 0001:0009b700       ?P_CheckTouchDamage@@YAXPAUDukePlayer_t@@H@Z 0049c700 f   player.obj
 0001:0009b960       _G_GetForcefieldPicnum     0049c960 f   player.obj
 0001:0009b9a0       ?DoWallTouchDamage@@YAXPBUDukePlayer_t@@H@Z 0049c9a0 f   player.obj
 0001:0009ba40       ?P_CheckFloorDamage@@YAHPAUDukePlayer_t@@H@Z 0049ca40 f   player.obj
 0001:0009bce0       ?P_ProcessWeapon@@YAXH@Z   0049cce0 f   player.obj
 0001:0009d640       ?P_FireWeapon@@YAXH@Z      0049e640 f   player.obj
 0001:0009d8b0       ?P_DoWeaponSpawn@@YAXH@Z   0049e8b0 f   player.obj
 0001:0009d9b0       ?P_DoFist@@YAHPAUDukePlayer_t@@@Z 0049e9b0 f   player.obj
 0001:0009dae0       ?getzsofslope_player@@YAXFHHPAH0@Z 0049eae0 f   player.obj
 0001:0009dc00       _getceilzofslope           0049ec00 f   player.obj
 0001:0009dc30       _sprite_tracker_hook       0049ec30 f   player.obj
 0001:0009e280       _getrendermode             0049f280 f   premap.obj
 0001:0009e290       _getticks                  0049f290 f   premap.obj
 0001:0009e2a0       _G_HandleAsync             0049f2a0 f   premap.obj
 0001:0009e2b0       ?tloadtile@@YAXHH@Z        0049f2b0 f   premap.obj
 0001:0009e330       ?flag_precache@@YAXHH@Z    0049f330 f   premap.obj
 0001:0009e3d0       ?G_CacheSpriteNum@@YAXH@Z  0049f3d0 f   premap.obj
 0001:0009ecc0       _A_CheckEnemySprite        0049fcc0 f   premap.obj
 0001:0009ece0       _A_CheckEnemyTile          0049fce0 f   premap.obj
 0001:0009ed00       ?G_PrecacheSprites@@YAXXZ  0049fd00 f   premap.obj
 0001:0009f370       ?G_PrecacheSounds@@YAXXZ   004a0370 f   premap.obj
 0001:0009f3d0       ?G_CacheSound@@YAHI@Z      004a03d0 f   premap.obj
 0001:0009f510       ?G_DoLoadScreen@@YAXPBDH@Z 004a0510 f   premap.obj
 0001:0009fa10       _scale                     004a0a10 f   premap.obj
 0001:0009fa50       _tabledivide64             004a0a50 f   premap.obj
 0001:0009fb20       _rotatesprite              004a0b20 f   premap.obj
 0001:0009fb70       _rotatesprite_fs           004a0b70 f   premap.obj
 0001:0009fbc0       _VM_OnEventWithReturn      004a0bc0 f   premap.obj
 0001:0009fc00       _VM_HaveEvent              004a0c00 f   premap.obj
 0001:0009fea0       _clamp                     004a0ea0 f   premap.obj
 0001:000a0130       _krand                     004a1130 f   premap.obj
 0001:000a0590       _VM_OnEvent                004a1590 f   premap.obj
 0001:000a05d0       ?P_ResetTintFade@@YAXPAUDukePlayer_t@@@Z 004a15d0 f   premap.obj
 0001:000a0fb0       _G_GetLogoFlags            004a1fb0 f   premap.obj
 0001:000a1110       _clearbufbyte              004a2110 f   premap.obj
 0001:000a1300       _realloc_copy              004a2300 f   premap.obj
 0001:000a1360       _xrealloc                  004a2360 f   premap.obj
 0001:000a1d00       _xstrdup                   004a2d00 f   premap.obj
 0001:000a1d30       _xcalloc                   004a2d30 f   premap.obj
 0001:000a1d60       ?prelevel@@YAXD@Z          004a2d60 f   premap.obj
 0001:000a2ea0       ?A_ResetVars@@YAXH@Z       004a3ea0 f   premap.obj
 0001:000a2f00       _G_GetForcefieldPicnum     004a3f00 f   premap.obj
 0001:000a2f40       ?resetprestat@@YAXHH@Z     004a3f40 f   premap.obj
 0001:000a31f0       ?G_SetupRotfixedSprites@@YAXXZ 004a41f0 f   premap.obj
 0001:000a34e0       ?G_CheckExitSprite@@YAHH@Z 004a44e0 f   premap.obj
 0001:000a3540       ?resetpspritevars@@YAXD@Z  004a4540 f   premap.obj
 0001:000a4180       _G_GetTeamPalette          004a5180 f   premap.obj
 0001:000a41b0       ?clearfrags@@YAXXZ         004a51b0 f   premap.obj
 0001:000a4220       ?G_FadeLoad@@YAXHHHHHHHH@Z 004a5220 f   premap.obj
 0001:000a42d0       ?G_LoadMapHack@@YAXPADPBD@Z 004a52d0 f   premap.obj
 0001:000a4350       _append_ext_UNSAFE         004a5350 f   premap.obj
 0001:000a43a0       ?G_TryMapHack@@YAHPBD@Z    004a53a0 f   premap.obj
 0001:000a43e0       ?G_HaveUserMap@@YAHXZ      004a53e0 f   premap.obj
 0001:000a44c0       _sector_tracker_hook       004a54c0 f   premap.obj
 0001:000a4520       _wall_tracker_hook         004a5520 f   premap.obj
 0001:000a4580       _sprite_tracker_hook       004a5580 f   premap.obj
 0001:000a4950       _Sect_SetInterpolation     004a5950 f   savegame.obj
 0001:000a4fc0       _append_ext_UNSAFE         004a5fc0 f   savegame.obj
 0001:000a5010       _G_NewGame_EnterLevel      004a6010 f   savegame.obj
 0001:000a5050       _VM_OnEvent                004a6050 f   savegame.obj
 0001:000a5090       _VM_HaveEvent              004a6090 f   savegame.obj
 0001:000a52c0       _getrendermode             004a62c0 f   savegame.obj
 0001:000a52d0       ?G_SaveTimers@@YAXXZ       004a62d0 f   savegame.obj
 0001:000a5310       ?G_RestoreTimers@@YAXXZ    004a6310 f   savegame.obj
 0001:000a58b0       _localtime                 004a68b0 f   savegame.obj
 0001:000a58d0       _time                      004a68d0 f   savegame.obj
 0001:000a58f0       _Bstrncpyz                 004a68f0 f   savegame.obj
 0001:000a5920       ?calcsz@@YAIPBUdataspec_@@@Z 004a6920 f   savegame.obj
 0001:000a5990       ?ds_getcnt@@YAHPBUdataspec_@@@Z 004a6990 f   savegame.obj
 0001:000a59f0       ?sv_makevarspec@@YAXXZ     004a69f0 f   savegame.obj
 0001:000a5ce0       _xmalloc                   004a6ce0 f   savegame.obj
 0001:000a5d10       ?SV_AllocSnap@@YAXH@Z      004a6d10 f   savegame.obj
 0001:000a62b0       ?cmpspecdata@@YAXPBUdataspec_@@PAPAE1@Z 004a72b0 f   savegame.obj
 0001:000a6460       ?ds_get@@YAXPBUdataspec_@@PAPAXPAH@Z 004a7460 f   savegame.obj
 0001:000a64b0       ?docmpsd@@YAXPBXPAXIIPAPAE@Z 004a74b0 f   savegame.obj
 0001:000a6e20       ?getnumvar@@YAHPBUdataspec_@@@Z 004a7e20 f   savegame.obj
 0001:000a7020       ?applydiff@@YAHPBUdataspec_@@PAPAE1@Z 004a8020 f   savegame.obj
 0001:000a7620       ?sv_postudload@@YAXXZ      004a8620 f   savegame.obj
 0001:000a76d0       ?dosaveplayer2@@YAPAEPAU_iobuf@@PAE@Z 004a86d0 f   savegame.obj
 0001:000a78c0       _getticks                  004a88c0 f   savegame.obj
 0001:000a78d0       ?writespecdata@@YAPAEPBUdataspec_@@PAU_iobuf@@PAE@Z 004a88d0 f   savegame.obj
 0001:000a7a60       ?doloadplayer2@@YAHHPAPAE@Z 004a8a60 f   savegame.obj
 0001:000a7d40       ?readspecdata@@YAHPBUdataspec_@@HPAPAE@Z 004a8d40 f   savegame.obj
 0001:000a8190       ?postloadplayer@@YAXH@Z    004a9190 f   savegame.obj
 0001:000a85b0       _sector_tracker_hook       004a95b0 f   savegame.obj
 0001:000a8610       _wall_tracker_hook         004a9610 f   savegame.obj
 0001:000a8670       ?sv_prespriteextsave@@YAXXZ 004a9670 f   savegame.obj
 0001:000a8700       ?sv_postspriteext@@YAXXZ   004a9700 f   savegame.obj
 0001:000a8760       ?sv_calcbitptrsize@@YAXXZ  004a9760 f   savegame.obj
 0001:000a8780       ?sv_prescriptsave_once@@YAXXZ 004a9780 f   savegame.obj
 0001:000a8830       ?sv_prescriptload_once@@YAXXZ 004a9830 f   savegame.obj
 0001:000a8880       ?sv_postscript_once@@YAXXZ 004a9880 f   savegame.obj
 0001:000a8920       ?sv_preactordatasave@@YAXXZ 004a9920 f   savegame.obj
 0001:000a8970       ?sv_postactordata@@YAXXZ   004a9970 f   savegame.obj
 0001:000a89c0       ?sv_preprojectilesave@@YAXXZ 004a99c0 f   savegame.obj
 0001:000a8ae0       _xrealloc                  004a9ae0 f   savegame.obj
 0001:000a8b10       ?sv_postprojectilesave@@YAXXZ 004a9b10 f   savegame.obj
 0001:000a8b20       ?sv_preprojectileload@@YAXXZ 004a9b20 f   savegame.obj
 0001:000a8ba0       ?sv_postprojectileload@@YAXXZ 004a9ba0 f   savegame.obj
 0001:000a8c80       ?sv_preanimateptrsave@@YAXXZ 004a9c80 f   savegame.obj
 0001:000a8cb0       ?sv_postanimateptr@@YAXXZ  004a9cb0 f   savegame.obj
 0001:000a8ce0       ?sv_prequote@@YAXXZ        004a9ce0 f   savegame.obj
 0001:000a8d30       _xcalloc                   004a9d30 f   savegame.obj
 0001:000a8d60       ?sv_quotesave@@YAXXZ       004a9d60 f   savegame.obj
 0001:000a8e00       ?sv_quoteload@@YAXXZ       004a9e00 f   savegame.obj
 0001:000a8e80       ?sv_prequoteredef@@YAXXZ   004a9e80 f   savegame.obj
 0001:000a8ed0       ?sv_quoteredefsave@@YAXXZ  004a9ed0 f   savegame.obj
 0001:000a8f30       ?sv_quoteredefload@@YAXXZ  004a9f30 f   savegame.obj
 0001:000a8fc0       ?sv_postquoteredef@@YAXXZ  004a9fc0 f   savegame.obj
 0001:000a8fe0       ?sv_restsave@@YAXXZ        004a9fe0 f   savegame.obj
 0001:000a91a0       ?sv_restload@@YAXXZ        004aa1a0 f   savegame.obj
 0001:000a9a30       ?A_FP_ManhattanDist@@YAHPBUDukePlayer_t@@PBUspritetype@@@Z 004aaa30 f   sector.obj
 0001:000a9aa0       _klabs                     004aaaa0 f   sector.obj
 0001:000aa200       _getrendermode             004ab200 f   sector.obj
 0001:000aa210       _polymer_invalidatesprite  004ab210 f   sector.obj
 0001:000aa240       _G_GetViewscreenSizeShift  004ab240 f   sector.obj
 0001:000aa2a0       ?G_SetupCamTile@@YAXHHH@Z  004ab2a0 f   sector.obj
 0001:000aa420       _G_GetCameraPosition       004ab420 f   sector.obj
 0001:000aa4f0       _mulscale16                004ab4f0 f   sector.obj
 0001:000aa8b0       _krand                     004ab8b0 f   sector.obj
 0001:000aa8e0       _G_GetForcefieldPicnum     004ab8e0 f   sector.obj
 0001:000ac430       _E_SpriteIsValid           004ad430 f   sector.obj
 0001:000ac570       _A_CheckEnemyTile          004ad570 f   sector.obj
 0001:000adc60       ?G_IsLikeDipswitch@@YAHH@Z 004aec60 f   sector.obj
 0001:000adcc0       ?G_GetBaseSwitch@@YAHH@Z   004aecc0 f   sector.obj
 0001:000aed50       ?BreakWall@@YAXHHH@Z       004afd50 f   sector.obj
 0001:000af200       _VM_OnEventWithBoth        004b0200 f   sector.obj
 0001:000af250       _VM_HaveEvent              004b0250 f   sector.obj
 0001:000b15a0       _A_Shoot                   004b25a0 f   sector.obj
 0001:000b15c0       _P_Get                     004b25c0 f   sector.obj
 0001:000b15e0       _P_GetP                    004b25e0 f   sector.obj
 0001:000b1610       _A_CheckEnemySprite        004b2610 f   sector.obj
 0001:000b1630       ?G_InitialActorStrength@@YAHH@Z 004b2630 f   sector.obj
 0001:000b1670       ?G_HaveActor@@YAHH@Z       004b2670 f   sector.obj
 0001:000b2af0       _VM_OnEventWithReturn      004b3af0 f   sector.obj
 0001:000b2b30       _VM_OnEvent                004b3b30 f   sector.obj
 0001:000b2b70       ?P_CheckDetonatorSpecialCase@@YAHQAUDukePlayer_t@@H@Z 004b3b70 f   sector.obj
 0001:000b40f0       _P_PalFrom                 004b50f0 f   sector.obj
 0001:000b4130       ?P_FindWall@@YAHPAUDukePlayer_t@@PAF@Z 004b5130 f   sector.obj
 0001:000b41e0       ?our_neartag_blacklist@@YAHH@Z 004b51e0 f   sector.obj
 0001:000b4240       ?G_ClearCameras@@YAXPAUDukePlayer_t@@@Z 004b5240 f   sector.obj
 0001:000b4260       _sector_tracker_hook       004b5260 f   sector.obj
 0001:000b42c0       _wall_tracker_hook         004b52c0 f   sector.obj
 0001:000b4320       _sprite_tracker_hook       004b5320 f   sector.obj
 0001:000b44d0       _xcalloc                   004b54d0 f   rts.obj
 0001:000b4500       ?RTS_AddFile@@YAHPBD@Z     004b5500 f   rts.obj
 0001:000b4700       _B_PASS32                  004b5700 f   rts.obj
 0001:000b4710       _xmalloc                   004b5710 f   rts.obj
 0001:000b4740       _xrealloc                  004b5740 f   rts.obj
 0001:000b4890       ?RTS_ReadLump@@YAXHPAX@Z   004b5890 f   rts.obj
 0001:000b4970       _xstrdup                   004b5970 f   config.obj
 0001:000b6240       _stat                      004b7240 f   config.obj
 0001:000b6260       _Bstrncpyz                 004b7260 f   config.obj
 0001:000b6290       _dup_filename              004b7290 f   config.obj
 0001:000b62e0       _xmalloc                   004b72e0 f   config.obj
 0001:000b6640       _CONTROL_KeyIsBound        004b7640 f   config.obj
 0001:000b6680       _CONTROL_MouseIsBound      004b7680 f   config.obj
 0001:000b7100       ?CONFIG_GetMapEntryName@@YAPBDQADQBD@Z 004b8100 f   config.obj
 0001:000b71c0       ?CONFIG_GetMD4EntryName@@YAXQADQBE@Z 004b81c0 f   config.obj
 0001:000b7240       _B_SWAP32                  004b8240 f   config.obj
 0001:000b7270       _B_UNBUF32                 004b8270 f   config.obj
 0001:000b7670       _B_PASS16                  004b8670 f   animlib.obj
 0001:000b7680       _B_PASS32                  004b8680 f   animlib.obj
 0001:000b7690       _xrealloc                  004b8690 f   animlib.obj
 0001:000b7770       ?drawframe@@YAXG@Z         004b8770 f   animlib.obj
 0001:000b77b0       ?findpage@@YAGG@Z          004b87b0 f   animlib.obj
 0001:000b78b0       ?loadpage@@YAXGPAPAG@Z     004b88b0 f   animlib.obj
 0001:000b7910       ?renderframe@@YAXGPAG@Z    004b8910 f   animlib.obj
 0001:000b79e0       ?decodeframe@@YAXPAE0@Z    004b89e0 f   animlib.obj
 0001:000b7b80       _B_UNBUF16                 004b8b80 f   animlib.obj
 0001:000b7d20       _Blrintf                   004b8d20 f   osdfuncs.obj
 0001:000b7d40       _rotatesprite_fs           004b8d40 f   osdfuncs.obj
 0001:000b7d90       ?GAME_isspace@@YAHH@Z      004b8d90 f   osdfuncs.obj
 0001:000b7dc0       ?GAME_getchartile@@YAHH@Z  004b8dc0 f   osdfuncs.obj
 0001:000b8120       _BGetTime                  004b9120 f   osdfuncs.obj
 0001:000b83d0       _clearbuf                  004b93d0 f   osdfuncs.obj
 0001:000b83f0       _getrendermode             004b93f0 f   osdfuncs.obj
 0001:000b85a0       _getrendermode             004b95a0 f   osdcmds.obj
 0001:000b9cc0       _xstrdup                   004bacc0 f   osdcmds.obj
 0001:000b9cf0       ?osdcmd_quit@@YAHPBUosdfuncparm_t@@@Z 004bacf0 f   osdcmds.obj
 0001:000b9d10       ?osdcmd_changelevel@@YAHPBUosdfuncparm_t@@@Z 004bad10 f   osdcmds.obj
 0001:000b9f10       _G_NewGame_EnterLevel      004baf10 f   osdcmds.obj
 0001:000b9f50       ?osdcmd_map@@YAHPBUosdfuncparm_t@@@Z 004baf50 f   osdcmds.obj
 0001:000ba2c0       ?osdcmd_demo@@YAHPBUosdfuncparm_t@@@Z 004bb2c0 f   osdcmds.obj
 0001:000ba390       _clamp                     004bb390 f   osdcmds.obj
 0001:000ba3d0       ?osdcmd_god@@YAHPBUosdfuncparm_t@@@Z 004bb3d0 f   osdcmds.obj
 0001:000ba420       ?osdcmd_noclip@@YAHPBUosdfuncparm_t@@@Z 004bb420 f   osdcmds.obj
 0001:000ba470       ?osdcmd_restartsound@@YAHPBUosdfuncparm_t@@@Z 004bb470 f   osdcmds.obj
 0001:000ba4b0       ?osdcmd_music@@YAHPBUosdfuncparm_t@@@Z 004bb4b0 f   osdcmds.obj
 0001:000ba540       _G_GetMusicIdx             004bb540 f   osdcmds.obj
 0001:000ba5d0       ?osdcmd_vidmode@@YAHPBUosdfuncparm_t@@@Z 004bb5d0 f   osdcmds.obj
 0001:000ba7f0       ?osdcmd_spawn@@YAHPBUosdfuncparm_t@@@Z 004bb7f0 f   osdcmds.obj
 0001:000bab70       ?osdcmd_setvar@@YAHPBUosdfuncparm_t@@@Z 004bbb70 f   osdcmds.obj
 0001:000bacc0       ?osdcmd_addlogvar@@YAHPBUosdfuncparm_t@@@Z 004bbcc0 f   osdcmds.obj
 0001:000bad90       ?osdcmd_setactorvar@@YAHPBUosdfuncparm_t@@@Z 004bbd90 f   osdcmds.obj
 0001:000baf20       ?osdcmd_addpath@@YAHPBUosdfuncparm_t@@@Z 004bbf20 f   osdcmds.obj
 0001:000baf80       ?osdcmd_initgroupfile@@YAHPBUosdfuncparm_t@@@Z 004bbf80 f   osdcmds.obj
 0001:000bafe0       ?osdcmd_cmenu@@YAHPBUosdfuncparm_t@@@Z 004bbfe0 f   osdcmds.obj
 0001:000bb030       ?osdcmd_crosshaircolor@@YAHPBUosdfuncparm_t@@@Z 004bc030 f   osdcmds.obj
 0001:000bb0f0       ?osdcmd_give@@YAHPBUosdfuncparm_t@@@Z 004bc0f0 f   osdcmds.obj
 0001:000bb350       ?osdcmd_name@@YAHPBUosdfuncparm_t@@@Z 004bc350 f   osdcmds.obj
 0001:000bb410       ?osdcmd_button@@YAHPBUosdfuncparm_t@@@Z 004bc410 f   osdcmds.obj
 0001:000bb440       ?osdcmd_bind@@YAHPBUosdfuncparm_t@@@Z 004bc440 f   osdcmds.obj
 0001:000bba90       _CONTROL_KeyIsBound        004bca90 f   osdcmds.obj
 0001:000bbad0       _CONTROL_MouseIsBound      004bcad0 f   osdcmds.obj
 0001:000bbb10       ?osdcmd_unbindall@@YAHPBUosdfuncparm_t@@@Z 004bcb10 f   osdcmds.obj
 0001:000bbbb0       ?osdcmd_unbind@@YAHPBUosdfuncparm_t@@@Z 004bcbb0 f   osdcmds.obj
 0001:000bbcc0       ?osdcmd_quicksave@@YAHPBUosdfuncparm_t@@@Z 004bccc0 f   osdcmds.obj
 0001:000bbd00       ?osdcmd_quickload@@YAHPBUosdfuncparm_t@@@Z 004bcd00 f   osdcmds.obj
 0001:000bbd40       ?osdcmd_screenshot@@YAHPBUosdfuncparm_t@@@Z 004bcd40 f   osdcmds.obj
 0001:000bbd60       ?osdcmd_inittimer@@YAHPBUosdfuncparm_t@@@Z 004bcd60 f   osdcmds.obj
 0001:000bbdc0       ?osdcmd_disconnect@@YAHPBUosdfuncparm_t@@@Z 004bcdc0 f   osdcmds.obj
 0001:000bbde0       ?osdcmd_connect@@YAHPBUosdfuncparm_t@@@Z 004bcde0 f   osdcmds.obj
 0001:000bbe10       ?osdcmd_password@@YAHPBUosdfuncparm_t@@@Z 004bce10 f   osdcmds.obj
 0001:000bbe50       ?osdcmd_listplayers@@YAHPBUosdfuncparm_t@@@Z 004bce50 f   osdcmds.obj
 0001:000bbf40       ?osdcmd_kick@@YAHPBUosdfuncparm_t@@@Z 004bcf40 f   osdcmds.obj
 0001:000bc040       ?osdcmd_kickban@@YAHPBUosdfuncparm_t@@@Z 004bd040 f   osdcmds.obj
 0001:000bc180       ?osdcmd_cvar_set_game@@YAHPBUosdfuncparm_t@@@Z 004bd180 f   osdcmds.obj
 0001:000bc6f0       _Blrintf                   004bd6f0 f   osdcmds.obj
 0001:000bc710       ?osdcmd_cvar_set_multi@@YAHPBUosdfuncparm_t@@@Z 004bd710 f   osdcmds.obj
 0001:000bc740       _sprite_tracker_hook       004bd740 f   osdcmds.obj
 0001:000bc970       ?LoadGameList@@YAXXZ       004bd970 f   grpscan.obj
 0001:000bcae0       _xstrdup                   004bdae0 f   grpscan.obj
 0001:000bcb10       _xcalloc                   004bdb10 f   grpscan.obj
 0001:000bcb40       _dup_filename              004bdb40 f   grpscan.obj
 0001:000bcb90       _Bstrncpyz                 004bdb90 f   grpscan.obj
 0001:000bcbc0       _xmalloc                   004bdbc0 f   grpscan.obj
 0001:000bcbf0       ?LoadList@@YAXPBD@Z        004bdbf0 f   grpscan.obj
 0001:000bcfd0       ?LoadGroupsCache@@YAHXZ    004bdfd0 f   grpscan.obj
 0001:000bd0f0       ?FreeGroupsCache@@YAXXZ    004be0f0 f   grpscan.obj
 0001:000bd130       ?RemoveGroup@@YAXPAUgrpfile_t@@@Z 004be130 f   grpscan.obj
 0001:000bd1b0       ?ProcessGroups@@YAXPAU_CACHE1D_FIND_REC@@@Z 004be1b0 f   grpscan.obj
 0001:000bd580       _fstat                     004be580 f   grpscan.obj
 0001:000bd5a0       _stat                      004be5a0 f   grpscan.obj
 0001:000bd5c0       ?FindGrpInfo@@YAPBUgrpinfo_t@@HH@Z 004be5c0 f   grpscan.obj
 0001:000bd650       ?FreeGameList@@YAXXZ       004be650 f   grpscan.obj
 0001:000bd6c0       ?process_vaca13@@YAXH@Z    004be6c0 f   grpscan.obj
 0001:000be030       ?process_vacapp15@@YAXH@Z  004bf030 f   grpscan.obj
 0001:000be410       ?SetPage@@YAXH@Z           004bf410 f   startwin.game.obj
 0001:000be4a0       ?EnableConfig@@YAXH@Z      004bf4a0 f   startwin.game.obj
 0001:000be560       ?startup_dlgproc@@YGHPAUHWND__@@IIJ@Z 004bf560 f   startwin.game.obj
 0001:000becb0       ?ConfigPageProc@@YGHPAUHWND__@@IIJ@Z 004bfcb0 f   startwin.game.obj
 0001:000bf090       ?PopulateForm@@YAXH@Z      004c0090 f   startwin.game.obj
 0001:000bf7a0       ?getfilenames@@YAHPBD@Z    004c07a0 f   startwin.game.obj
 0001:000bf7d0       ?clearfilenames@@YAXXZ     004c07d0 f   startwin.game.obj
 0001:000bfe60       _xmalloc                   004c0e60 f   file_lib.obj
 0001:000c0640       ?CONTROL_PollDevices@@YAXPAUControlInfo@@@Z 004c1640 f   control.obj
 0001:000c0800       ?CONTROL_GetMouseDelta@@YAXXZ 004c1800 f   control.obj
 0001:000c08d0       ?CONTROL_GetDeviceButtons@@YAXXZ 004c18d0 f   control.obj
 0001:000c09b0       ?DoGetDeviceButtons@@YAXHHHPAH000PAE@Z 004c19b0 f   control.obj
 0001:000c0ae0       ?CONTROL_DigitizeAxis@@YAXHW4controldevice@@@Z 004c1ae0 f   control.obj
 0001:000c0ba0       ?CONTROL_ScaleAxis@@YAXHW4controldevice@@@Z 004c1ba0 f   control.obj
 0001:000c0c10       _mulscale16                004c1c10 f   control.obj
 0001:000c0c20       ?CONTROL_ApplyAxis@@YAXHPAUControlInfo@@W4controldevice@@@Z 004c1c20 f   control.obj
 0001:000c0d30       ?CONTROL_GetFunctionInput@@YAXXZ 004c1d30 f   control.obj
 0001:000c0e60       ?CONTROL_SetFlag@@YAXHH@Z  004c1e60 f   control.obj
 0001:000c0ee0       ?CONTROL_AxisFunctionState@@YAXPAH@Z 004c1ee0 f   control.obj
 0001:000c0fd0       ?CONTROL_ButtonFunctionState@@YAXPAH@Z 004c1fd0 f   control.obj
 0001:000c1350       ?CONTROL_GetTime@@YAHXZ    004c2350 f   control.obj
 0001:000c1480       ?KB_KeyEvent@@YAXHH@Z      004c2480 f   keyboard.obj
 0001:000c1760       _xmalloc                   004c2760 f   scriplib.obj
 0001:000c28d0       ?SCRIPT_ParseString@@YAPADPAPADPAD@Z 004c38d0 f   scriplib.obj
 0001:000c2bd0       _xcalloc                   004c3bd0 f   scriplib.obj
 0001:000c3850       _scale                     004c4850 f   sounds.obj
 0001:000c3890       _tabledivide64             004c4890 f   sounds.obj
 0001:000c3c10       _G_GetLogoFlags            004c4c10 f   sounds.obj
 0001:000c3ef0       _xaligned_malloc           004c4ef0 f   sounds.obj
 0001:000c4240       _S_IsAmbientSFX            004c5240 f   sounds.obj
 0001:000c4a80       _P_Get                     004c5a80 f   sounds.obj
 0001:000c4aa0       _P_GetP                    004c5aa0 f   sounds.obj
 0001:000c4ad0       _VM_OnEventWithReturn      004c5ad0 f   sounds.obj
 0001:000c4b10       _VM_HaveEvent              004c5b10 f   sounds.obj
 0001:000c4b40       ?S_GetPitch@@YAHH@Z        004c5b40 f   sounds.obj
 0001:000c4bf0       _klabs                     004c5bf0 f   sounds.obj
 0001:000c4c00       ?S_GetSlot@@YAHH@Z         004c5c00 f   sounds.obj
 0001:000c4c60       ?S_TakeSlot@@YAHH@Z        004c5c60 f   sounds.obj
 0001:000c4dd0       ?S_CalcDistAndAng@@YAHHHHHPBUvec3_t@@0PAH1@Z 004c5dd0 f   sounds.obj
 0001:000c5050       _divscale14                004c6050 f   sounds.obj
 0001:000c5070       _divscale                  004c6070 f   sounds.obj
 0001:000c50b0       ?S_GetAngle@@YAHHPBUvec3_t@@0@Z 004c60b0 f   sounds.obj
 0001:000c5fe0       ?_MIDI_SendControlChange@@YAHHHH@Z 004c6fe0 f   midi.obj
 0001:000c60c0       ?_MIDI_SendChannelVolumes@@YAXXZ 004c70c0 f   midi.obj
 0001:000c6100       ?_MIDI_SetChannelVolume@@YAXHH@Z 004c7100 f   midi.obj
 0001:000c6190       _clamp                     004c7190 f   midi.obj
 0001:000c62c0       ?_MIDI_ResetTracks@@YAXXZ  004c72c0 f   midi.obj
 0001:000c63e0       ?_MIDI_ReadDelta@@YAHPAUtrack@@@Z 004c73e0 f   midi.obj
 0001:000c66a0       _B_UNBUF32                 004c76a0 f   midi.obj
 0001:000c66b0       _xmalloc                   004c76b0 f   midi.obj
 0001:000c66e0       ?_MIDI_ReadNumber@@YAHPAXI@Z 004c76e0 f   midi.obj
 0001:000c6740       ?_MIDI_ServiceRoutine@@YAHXZ 004c7740 f   midi.obj
 0001:000c6ac0       ?_MIDI_AdvanceTick@@YAXXZ  004c7ac0 f   midi.obj
 0001:000c6b60       ?_MIDI_SysEx@@YAXPAUtrack@@@Z 004c7b60 f   midi.obj
 0001:000c6b90       ?_MIDI_MetaEvent@@YAXPAUtrack@@@Z 004c7b90 f   midi.obj
 0001:000c6ce0       ?_MIDI_InterpretControllerInfo@@YAHPAUtrack@@HHHH@Z 004c7ce0 f   midi.obj
 0001:000c72c0       ?_MIDI_InitEMIDI@@YAXXZ    004c82c0 f   midi.obj
 0001:000c7a20       _clamp                     004c8a20 f   music.obj
 0001:000c8500       _scale                     004c9500 f   baselayer.obj
 0001:000c8540       _tabledivide64             004c9540 f   baselayer.obj
 0001:000c8840       _xaligned_malloc           004c9840 f   baselayer.obj
 0001:000c90c0       ?osdfunc_setrendermode@@YAHPBUosdfuncparm_t@@@Z 004ca0c0 f   baselayer.obj
 0001:000c91f0       _getrendermode             004ca1f0 f   baselayer.obj
 0001:000c9200       ?osdcmd_hicsetpalettetint@@YAHPBUosdfuncparm_t@@@Z 004ca200 f   baselayer.obj
 0001:000c92d0       ?osdcmd_cvar_set_baselayer@@YAHPBUosdfuncparm_t@@@Z 004ca2d0 f   baselayer.obj
 0001:000c9560       _xrealloc                  004ca560 f   cache1d.obj
 0001:000c9a20       _mulscale32                004caa20 f   cache1d.obj
 0001:000c9a30       ?inc_and_check_cacnum@@YAXXZ 004caa30 f   cache1d.obj
 0001:000c9b40       ?reportandexit@@YAXPBD@Z   004cab40 f   cache1d.obj
 0001:000c9f10       _stat                      004caf10 f   cache1d.obj
 0001:000c9f30       _xstrdup                   004caf30 f   cache1d.obj
 0001:000c9f60       _xmalloc                   004caf60 f   cache1d.obj
 0001:000ca430       ?openfrompath_internal@@YAHPBDPAPADHH@Z 004cb430 f   cache1d.obj
 0001:000cae10       _B_PASS32                  004cbe10 f   cache1d.obj
 0001:000cae20       ?initgroupfile_crc32@@YAXH@Z 004cbe20 f   cache1d.obj
 0001:000caff0       ?kopen_internal@@YAHPBDPAPADDDDHPAEPAH3@Z 004cbff0 f   cache1d.obj
 0001:000cb320       _kztell                    004cc320 f   cache1d.obj
 0001:000cb350       _kzclose                   004cc350 f   cache1d.obj
 0001:000cb380       ?kzipopen@@YAHPBD@Z        004cc380 f   cache1d.obj
 0001:000cb400       ?check_filename_mismatch@@YAHQBDH@Z 004cc400 f   cache1d.obj
 0001:000cbb40       _kzfilelength              004ccb40 f   cache1d.obj
 0001:000cbd50       ?kread_grp@@YAHHPAXH@Z     004ccd50 f   cache1d.obj
 0001:000cbd80       ?klseek_grp@@YAHHHH@Z      004ccd80 f   cache1d.obj
 0001:000cbdb0       ?kclose_grp@@YAXH@Z        004ccdb0 f   cache1d.obj
 0001:000cc660       ?klistaddentry@@YAHPAPAU_CACHE1D_FIND_REC@@PBDHH@Z 004cd660 f   cache1d.obj
 0001:000cc840       ?kdfread_func@@YAHHPAXH@Z  004cd840 f   cache1d.obj
 0001:000cc860       ?dfwrite_func@@YAXHPBXH@Z  004cd860 f   cache1d.obj
 0001:000cc8a0       ?c1d_read_compressed@@YAHPAXIIH@Z 004cd8a0 f   cache1d.obj
 0001:000cca90       ?decompress_part@@YAIHPAI@Z 004cda90 f   cache1d.obj
 0001:000ccb10       _B_PASS16                  004cdb10 f   cache1d.obj
 0001:000ccb40       ?c1d_write_compressed@@YAXPBXIIH@Z 004cdb40 f   cache1d.obj
 0001:000ccd40       ?compress_part@@YAIIH@Z    004cdd40 f   cache1d.obj
 0001:000ccdb0       ?lzwcompress@@YAHPBDHPAD@Z 004cddb0 f   cache1d.obj
 0001:000cd1e0       ?lzwuncompress@@YAHPBDHPAD@Z 004ce1e0 f   cache1d.obj
 0001:000cd5f0       _dup_filename              004ce5f0 f   common.obj
 0001:000cd640       _Bstrncpyz                 004ce640 f   common.obj
 0001:000cd670       _xmalloc                   004ce670 f   common.obj
 0001:000cd720       _xstrdup                   004ce720 f   common.obj
 0001:000cd750       _xrealloc                  004ce750 f   common.obj
 0001:000cdbe0       _sepldist                  004cebe0 f   common.obj
 0001:000cdc50       _klabs                     004cec50 f   common.obj
 0001:000cdc60       _swaplong                  004cec60 f   common.obj
 0001:000cdcd0       _sepdist                   004cecd0 f   common.obj
 0001:000cdef0       _clearbuf                  004ceef0 f   common.obj
 0001:000cdf10       _getrendermode             004cef10 f   common.obj
 0001:000ce730       _fstat                     004cf730 f   compat.obj
 0001:000cea30       _stat                      004cfa30 f   compat.obj
 0001:000ced70       ?libdivide__count_trailing_zeros32@@YAHI@Z 004cfd70 f   compat.obj
 0001:000ceda0       ?libdivide__count_leading_zeros32@@YAHI@Z 004cfda0 f   compat.obj
 0001:000cedd0       ?libdivide_64_div_32_to_32@@YAIIIIPAI@Z 004cfdd0 f   compat.obj
 0001:000ceeb0       ?libdivide__mullhi_u32@@YAIII@Z 004cfeb0 f   compat.obj
 0001:000cf160       ?libdivide__count_trailing_zeros64@@YAH_K@Z 004d0160 f   compat.obj
 0001:000cf1b0       ?libdivide__count_leading_zeros64@@YAH_K@Z 004d01b0 f   compat.obj
 0001:000cf200       ?libdivide_128_div_64_to_64@@YA_K_K00PA_K@Z 004d0200 f   compat.obj
 0001:000cf630       ?libdivide__mullhi_u64@@YA_K_K0@Z 004d0630 f   compat.obj
 0001:000cfa20       ?libdivide__mullhi_s32@@YAHHH@Z 004d0a20 f   compat.obj
 0001:000d0000       ?libdivide__mullhi_s64@@YA_J_J0@Z 004d1000 f   compat.obj
 0001:000d0700       ?defsparser_include@@YAXPBDPBUscriptfile@@0@Z 004d1700 f   defs.obj
 0001:000d07b0       ?defsparser@@YAHPAUscriptfile@@@Z 004d17b0 f   defs.obj
 0001:000d7870       _Blrintf                   004d8870 f   defs.obj
 0001:000d7890       _clamp                     004d8890 f   defs.obj
 0001:000d78d0       _xmalloc                   004d88d0 f   defs.obj
 0001:000d7900       _xrealloc                  004d8900 f   defs.obj
 0001:000d7930       _md_tilehasmodel           004d8930 f   defs.obj
 0001:000d7970       ?check_tile_range@@YAHPBDPAH1PBUscriptfile@@0@Z 004d8970 f   defs.obj
 0001:000d7a10       _swaplong                  004d8a10 f   defs.obj
 0001:000d7a30       ?check_tile@@YAHPBDHPBUscriptfile@@0@Z 004d8a30 f   defs.obj
 0001:000d7a70       ?Defs_LoadTileIntoBuffer@@YAHH@Z 004d8a70 f   defs.obj
 0001:000d7af0       ?maybe_grow_buffer@@YAXQAPADQAHH@Z 004d8af0 f   defs.obj
 0001:000d7b40       ?Defs_ApplyPaletteToTileBuffer@@YAXHH@Z 004d8b40 f   defs.obj
 0001:000d7b90       ?Defs_ImportTileFromTexture@@YAHQBDHHH@Z 004d8b90 f   defs.obj
 0001:000d7e20       _B_PASS16                  004d8e20 f   defs.obj
 0001:000d7e30       _B_UNBUF16                 004d8e30 f   defs.obj
 0001:000d7e40       ?tile_from_truecolpic@@YAXHPBUpalette_t@@H@Z 004d8e40 f   defs.obj
 0001:000d8b50       _yax_getbunches            004d9b50 f   engine.obj
 0001:000d8e10       ?yax_islockededge@@YAHHH@Z 004d9e10 f   engine.obj
 0001:000d9920       _getrendermode             004da920 f   engine.obj
 0001:000d9a20       _xrealloc                  004daa20 f   engine.obj
 0001:000da310       ?yax_scanbunches@@YAXHHPBE@Z 004db310 f   engine.obj
 0001:000da500       ?yax_walldist@@YAHH@Z      004db500 f   engine.obj
 0001:000da550       _klabs                     004db550 f   engine.obj
 0001:000da560       ?yax_getclosestpointonwall@@YAXHPAH0@Z 004db560 f   engine.obj
 0001:000da760       ?yax_cmpbunches@@YAHPBX0@Z 004db760 f   engine.obj
 0001:000da7a0       _B_UNBUF16                 004db7a0 f   engine.obj
 0001:000da7b0       ?yax_copytsprites@@YAXXZ   004db7b0 f   engine.obj
 0001:000da990       ?draw_rainbow_background@@YAXXZ 004db990 f   engine.obj
 0001:000dc400       _xmalloc                   004dd400 f   engine.obj
 0001:000dc430       _xcalloc                   004dd430 f   engine.obj
 0001:000dc460       _swapshort                 004dd460 f   engine.obj
 0001:000dc480       _uhypsq                    004dd480 f   engine.obj
 0001:000dc4a0       ?clipmapinfo_init@@YAXXZ   004dd4a0 f   engine.obj
 0001:000dcd90       _getzsofslope              004ddd90 f   engine.obj
 0001:000dcdc0       ?getscore@@YAHHHHH@Z       004dddc0 f   engine.obj
 0001:000dce40       _swaplong                  004dde40 f   engine.obj
 0001:000dd290       _spriteheightofs           004de290 f   engine.obj
 0001:000dd2c0       ?scansector@@YAXF@Z        004de2c0 f   engine.obj
 0001:000dda90       _mulscale5                 004dea90 f   engine.obj
 0001:000ddaa0       _dmulscale6                004deaa0 f   engine.obj
 0001:000ddad0       _dmulscale32               004dead0 f   engine.obj
 0001:000ddaf0       _yax_isislandwall          004deaf0 f   engine.obj
 0001:000ddb20       ?get_rel_coords@@YA?AUvec2_t@@HH@Z 004deb20 f   engine.obj
 0001:000ddb80       ?get_screen_coords@@YAHUvec2_t@@0PAH111@Z 004deb80 f   engine.obj
 0001:000ddd50       _scale                     004ded50 f   engine.obj
 0001:000ddd90       _tabledivide64             004ded90 f   engine.obj
 0001:000de090       _dmulscale2                004df090 f   engine.obj
 0001:000de4b0       _mulscale16                004df4b0 f   engine.obj
 0001:000dec40       ?do_deletespritestat@@YAXF@Z 004dfc40 f   engine.obj
 0001:000def60       _divscale24                004dff60 f   engine.obj
 0001:000def80       _divscale                  004dff80 f   engine.obj
 0001:000defc0       _mulscale24                004dffc0 f   engine.obj
 0001:000df020       ?rintersect@@YAHHHHHHHHHHHPAH00@Z 004e0020 f   engine.obj
 0001:000df6a0       _clearbuf                  004e06a0 f   engine.obj
 0001:000df6c0       ?loadtables@@YAHXZ         004e06c0 f   engine.obj
 0001:000df950       _divscale30                004e0950 f   engine.obj
 0001:000df970       _krecipasm                 004e0970 f   engine.obj
 0001:000df9c0       ?initksqrt@@YAXXZ          004e09c0 f   engine.obj
 0001:000dfa80       ?msqrtasm@@YAHH@Z          004e0a80 f   engine.obj
 0001:000dfab0       ?calcbritable@@YAXXZ       004e0ab0 f   engine.obj
 0001:000dfb70       ?loadpalette@@YAXXZ        004e0b70 f   engine.obj
 0001:000e00d0       _B_PASS16                  004e10d0 f   engine.obj
 0001:000e0140       ?E_PostLoadPalette@@YAXXZ  004e1140 f   engine.obj
 0001:000e0340       _getclosestcol             004e1340 f   engine.obj
 0001:000e0360       ?E_FatalError@@YAHQBD@Z    004e1360 f   engine.obj
 0001:000e1110       _divscale16                004e2110 f   engine.obj
 0001:000e1130       _mulscale8                 004e2130 f   engine.obj
 0001:000e1140       _set_globalpos             004e2140 f   engine.obj
 0001:000e1180       ?bunchfront@@YAHHH@Z       004e2180 f   engine.obj
 0001:000e1280       ?drawalls@@YAXH@Z          004e2280 f   engine.obj
 0001:000e2ee0       _copybufbyte               004e3ee0 f   engine.obj
 0001:000e2f40       _getceilzofslope           004e3f40 f   engine.obj
 0001:000e2f70       _getflorzofslope           004e3f70 f   engine.obj
 0001:000e2fa0       ?prepwall@@YAXHPBUwalltypev7@@@Z 004e3fa0 f   engine.obj
 0001:000e3470       _divscale12                004e4470 f   engine.obj
 0001:000e3490       _mulscale2                 004e4490 f   engine.obj
 0001:000e34a0       _mulscale11                004e44a0 f   engine.obj
 0001:000e34b0       _mulscale18                004e44b0 f   engine.obj
 0001:000e34c0       _mulscale19                004e44c0 f   engine.obj
 0001:000e34d0       _mulscale21                004e44d0 f   engine.obj
 0001:000e34e0       ?wallmost@@YAHPAFHHD@Z     004e44e0 f   engine.obj
 0001:000e3ec0       _mulscale15                004e4ec0 f   engine.obj
 0001:000e3ed0       _mulscale20                004e4ed0 f   engine.obj
 0001:000e3ee0       _mulscale30                004e4ee0 f   engine.obj
 0001:000e3ef0       ?nsqrtasm@@YAHH@Z          004e4ef0 f   engine.obj
 0001:000e3f30       ?wallmosts_finish@@YAXPAFHHHHHH@Z 004e4f30 f   engine.obj
 0001:000e4020       _clamp                     004e5020 f   engine.obj
 0001:000e4060       _tabledivide32             004e5060 f   engine.obj
 0001:000e40f0       _qinterpolatedown16short   004e50f0 f   engine.obj
 0001:000e4150       ?owallmost@@YAHPAFH_J@Z    004e5150 f   engine.obj
 0001:000e4600       ?mulscale20z@@YA_JHH@Z     004e5600 f   engine.obj
 0001:000e4630       ?wallmost_getz@@YA_JHH_JHHHHHHHH@Z 004e5630 f   engine.obj
 0001:000e4760       _divscale28                004e5760 f   engine.obj
 0001:000e4780       ?dmulscale24z@@YA_JHHHH@Z  004e5780 f   engine.obj
 0001:000e47d0       ?ceilscan@@YAXHHH@Z        004e57d0 f   engine.obj
 0001:000e4da0       ?hline@@YAXHH@Z            004e5da0 f   engine.obj
 0001:000e4e90       _getpalookupsh             004e5e90 f   engine.obj
 0001:000e4eb0       _getpalookup               004e5eb0 f   engine.obj
 0001:000e4f30       ?slowhline@@YAXHH@Z        004e5f30 f   engine.obj
 0001:000e50d0       ?setup_globals_cf1@@YAHPBUsectortypev7@@HHHHHHHH@Z 004e60d0 f   engine.obj
 0001:000e5800       _mulscale4                 004e6800 f   engine.obj
 0001:000e5810       _mulscale10                004e6810 f   engine.obj
 0001:000e5820       _dmulscale10               004e6820 f   engine.obj
 0001:000e5850       _dmulscale14               004e6850 f   engine.obj
 0001:000e5880       _setgotpic                 004e6880 f   engine.obj
 0001:000e58c0       ?calc_globalshifts@@YAXXZ  004e68c0 f   engine.obj
 0001:000e5950       ?setup_blend@@YAXHH@Z      004e6950 f   engine.obj
 0001:000e59b0       ?florscan@@YAXHHH@Z        004e69b0 f   engine.obj
 0001:000e6070       ?wallscan@@YAXHHPBF0PBH1@Z 004e7070 f   engine.obj
 0001:000e6c10       ?tweak_tsizes@@YAXPAUvec2_t@@@Z 004e7c10 f   engine.obj
 0001:000e6ca0       ?calc_bufplc@@YAXPAHHUvec2_t@@@Z 004e7ca0 f   engine.obj
 0001:000e6d10       ?calc_vplcinc@@YAXPAIPAHPBHHH@Z 004e7d10 f   engine.obj
 0001:000e6d60       ?calc_vplcinc_wall@@YAXPAIPAH_JH@Z 004e7d60 f   engine.obj
 0001:000e6db0       ?calc_vplcinc_sprite@@YAXPAIPAHHH@Z 004e7db0 f   engine.obj
 0001:000e6ea0       _Blrintf                   004e7ea0 f   engine.obj
 0001:000e6ec0       ?grouscan@@YAXHHHD@Z       004e7ec0 f   engine.obj
 0001:000e7c00       _dmulscale9                004e8c00 f   engine.obj
 0001:000e7c30       _mulscale12                004e8c30 f   engine.obj
 0001:000e7c40       _mulscale14                004e8c40 f   engine.obj
 0001:000e7c50       _dmulscale16               004e8c50 f   engine.obj
 0001:000e7c80       _dmulscale17               004e8c80 f   engine.obj
 0001:000e7cb0       _dmulscale25               004e8cb0 f   engine.obj
 0001:000e7ce0       _mulscale27                004e8ce0 f   engine.obj
 0001:000e7cf0       _mulscale28                004e8cf0 f   engine.obj
 0001:000e7d00       ?setupslopevlin_alsotrans@@YAXHHH@Z 004e8d00 f   engine.obj
 0001:000e7d60       ?tslopevlin@@YAXPAEHPBHHHH@Z 004e8d60 f   engine.obj
 0001:000e7eb0       ?parascan@@YAXHHHDH@Z      004e8eb0 f   engine.obj
 0001:000e8750       _mulscale23                004e9750 f   engine.obj
 0001:000e8760       _getpsky                   004e9760 f   engine.obj
 0001:000e87f0       _getpskyidx                004e97f0 f   engine.obj
 0001:000e8830       ?oldnonpow2@@YAHXZ         004e9830 f   engine.obj
 0001:000e8840       ?setup_globals_wall1@@YAXPBUwalltypev7@@H@Z 004e9840 f   engine.obj
 0001:000e8920       ?setup_globals_wall2@@YAXPBUwalltypev7@@EHH@Z 004e9920 f   engine.obj
 0001:000e8ac0       ?should_clip_cwall@@YAHHH@Z 004e9ac0 f   engine.obj
 0001:000e8b40       ?should_clip_fwall@@YAHHH@Z 004e9b40 f   engine.obj
 0001:000e8bc0       ?dosetaspect@@YAXXZ        004e9bc0 f   engine.obj
 0001:000e8f40       _xaligned_malloc           004e9f40 f   engine.obj
 0001:000e8f70       _divscale14                004e9f70 f   engine.obj
 0001:000e8f90       _divscale26                004e9f90 f   engine.obj
 0001:000e8fb0       _mulscale1                 004e9fb0 f   engine.obj
 0001:000e8fc0       _mulscale32                004e9fc0 f   engine.obj
 0001:000ea230       _swapptr                   004eb230 f   engine.obj
 0001:000ea260       ?drawsprite@@YAXH@Z        004eb260 f   engine.obj
 0001:000ea300       ?drawsprite_classic@@YAXH@Z 004eb300 f   engine.obj
 0001:000eed50       _B_PASS32                  004efd50 f   engine.obj
 0001:000eed60       _divscale18                004efd60 f   engine.obj
 0001:000eed80       _divscale19                004efd80 f   engine.obj
 0001:000eeda0       _dmulscale8                004efda0 f   engine.obj
 0001:000eedd0       _mulscale9                 004efdd0 f   engine.obj
 0001:000eede0       _dmulscale12               004efde0 f   engine.obj
 0001:000eee10       _mulscale22                004efe10 f   engine.obj
 0001:000eee20       _mulscale31                004efe20 f   engine.obj
 0001:000eee30       _qinterpolatedown16        004efe30 f   engine.obj
 0001:000eee80       _bad_tspr                  004efe80 f   engine.obj
 0001:000eeec0       ?maskwallscan@@YAXHHH@Z    004efec0 f   engine.obj
 0001:000efb10       ?spritewallfront@@YAHPBUtspritetype@@H@Z 004f0b10 f   engine.obj
 0001:000efb90       ?transmaskwallscan@@YAXHHH@Z 004f0b90 f   engine.obj
 0001:000efd20       ?transmaskvline@@YAXH@Z    004f0d20 f   engine.obj
 0001:000eff20       ?transmaskvline2@@YAXH@Z   004f0f20 f   engine.obj
 0001:000f0440       ?ceilspritescan@@YAXHH@Z   004f1440 f   engine.obj
 0001:000f0600       ?ceilspritehline@@YAXHH@Z  004f1600 f   engine.obj
 0001:000f0810       ?nonpow2_mhline@@YAXHIHHIPAD@Z 004f1810 f   engine.obj
 0001:000f0920       _divideu32                 004f1920 f   engine.obj
 0001:000f0980       _divscale32                004f1980 f   engine.obj
 0001:000f09a0       ?nonpow2_thline@@YAXHIHHIPAD@Z 004f19a0 f   engine.obj
 0001:000f0b80       ?drawvox@@YAXHHHHHHDCDPBH0@Z 004f1b80 f   engine.obj
 0001:000f1e70       _divscale21                004f2e70 f   engine.obj
 0001:000f1e90       _dmulscale18               004f2e90 f   engine.obj
 0001:000f1ec0       _ksgn                      004f2ec0 f   engine.obj
 0001:000f1ee0       ?mulscale16z@@YA_JHH@Z     004f2ee0 f   engine.obj
 0001:000f1f10       ?setup_globals_sprite1@@YAXPBUtspritetype@@PBUsectortypev7@@HHHHPAH2@Z 004f2f10 f   engine.obj
 0001:000f2170       ?falpha_to_blend@@YAEMPAHHH@Z 004f3170 f   engine.obj
 0001:000f2240       ?mulscale_triple30@@YAHHHH@Z 004f3240 f   engine.obj
 0001:000f2280       ?drawmaskwall@@YAXF@Z      004f3280 f   engine.obj
 0001:000f28c0       ?equation@@YA?AUs_equation@@MMMM@Z 004f38c0 f   engine.obj
 0001:000f2960       ?sameside@@YAHPBUs_equation@@PBUvec2f_t@@1@Z 004f3960 f   engine.obj
 0001:000f4060       _mulscale                  004f5060 f   engine.obj
 0001:000f4080       _dmulscale1                004f5080 f   engine.obj
 0001:000f40b0       _dmulscale28               004f50b0 f   engine.obj
 0001:000f40e0       ?getclipmask@@YAHHHHH@Z    004f50e0 f   engine.obj
 0001:000f4110       ?fillpolygon@@YAXH@Z       004f5110 f   engine.obj
 0001:000f4820       ?clippoly@@YAHHH@Z         004f5820 f   engine.obj
 0001:000f5770       ?addscaleclamp@@YAHHHHH@Z  004f6770 f   engine.obj
 0001:000f5990       ?clearmapartfilename@@YAXXZ 004f6990 f   engine.obj
 0001:000f59c0       ?E_RecalcPicSiz@@YAXXZ     004f69c0 f   engine.obj
 0001:000f5b50       _append_ext_UNSAFE         004f6b50 f   engine.obj
 0001:000f6880       ?have_maptext@@YAHXZ       004f7880 f   engine.obj
 0001:000f68a0       ?prepare_loadboard@@YAXHPAUvec3_t@@PAF1@Z 004f78a0 f   engine.obj
 0001:000f6a00       ?finish_loadboard@@YAHPBUvec3_t@@PAFFD@Z 004f7a00 f   engine.obj
 0001:000f6c50       ?check_sprite@@YAXH@Z      004f7c50 f   engine.obj
 0001:000f6eb0       ?remove_sprite@@YAXH@Z     004f7eb0 f   engine.obj
 0001:000f7950       ?convertv5sectv6@@YAXPAUsectortypev5@@PAUsectortypev6@@@Z 004f8950 f   engine.obj
 0001:000f7a70       ?convertv5wallv6@@YAXPAUwalltypev5@@PAUwalltypev6@@H@Z 004f8a70 f   engine.obj
 0001:000f7b70       ?sectorofwallv5@@YAFF@Z    004f8b70 f   engine.obj
 0001:000f7c10       ?convertv5sprv6@@YAXPAUspritetypev5@@PAUspritetypev6@@@Z 004f8c10 f   engine.obj
 0001:000f7d80       ?convertv6sectv7@@YAXPAUsectortypev6@@PAUsectortypev7@@@Z 004f8d80 f   engine.obj
 0001:000f8040       ?convertv6wallv7@@YAXPAUwalltypev6@@PAUwalltypev7@@@Z 004f9040 f   engine.obj
 0001:000f8190       ?convertv6sprv7@@YAXPAUspritetypev6@@PAUspritetype@@@Z 004f9190 f   engine.obj
 0001:000f9790       ?get_mapversion@@YAHXZ     004fa790 f   engine.obj
 0001:000f9ac0       ?initsmost@@YAXXZ          004faac0 f   engine.obj
 0001:000f9d20       ?PolymostProcessVoxels@@YAXXZ 004fad20 f   engine.obj
 0001:000fa0c0       _getticks                  004fb0c0 f   engine.obj
 0001:000fa0d0       ?dorotatesprite@@YAXHHHFFCDHEEHHHHH@Z 004fb0d0 f   engine.obj
 0001:000fc270       ?clippoly4@@YAHHHHH@Z      004fd270 f   engine.obj
 0001:000fc7b0       ?set_picsiz@@YAXH@Z        004fd7b0 f   engine.obj
 0001:000fcaf0       _B_UNBUF32                 004fdaf0 f   engine.obj
 0001:000fcdf0       ?maybe_grow_buffer@@YAXQAPADQAHH@Z 004fddf0 f   engine.obj
 0001:000fce40       ?E_GetArtFileName@@YAPBDH@Z 004fde40 f   engine.obj
 0001:000fcf00       ?E_ReadArtFileOfID@@YAHH@Z 004fdf00 f   engine.obj
 0001:000fd260       _Bstrncpyz                 004fe260 f   engine.obj
 0001:000fd4b0       ?postloadtile@@YAXF@Z      004fe4b0 f   engine.obj
 0001:000fea50       ?get_wallspr_points@@YAXPBUspritetype@@PAH111@Z 004ffa50 f   engine.obj
 0001:000feb80       ?get_floorspr_points@@YAXPBUtspritetype@@HHPAH1111111@Z 004ffb80 f   engine.obj
 0001:000ffcb0       _yax_waltosecmask          00500cb0 f   engine.obj
 0001:000ffcd0       ?mapinfo_set@@YAXPAUmapinfo_t@@0@Z 00500cd0 f   engine.obj
 0001:000ffd50       ?hit_set@@YAXPAUhitdata_t@@HHHHHH@Z 00500d50 f   engine.obj
 0001:000ffd90       ?hitscan_trysector@@YAHPBUvec3_t@@PBUsectortypev7@@PAUhitdata_t@@HHHGFHHPBH@Z 00500d90 f   engine.obj
 0001:001001f0       _divscale15                005011f0 f   engine.obj
 0001:00100210       _dmulscale15               00501210 f   engine.obj
 0001:00100240       ?get_floorspr_clipyou@@YAHHHHHHHHH@Z 00501240 f   engine.obj
 0001:00100380       ?try_facespr_intersect@@YAHPBUspritetype@@PBUvec3_t@@HHHPAU2@H@Z 00501380 f   engine.obj
 0001:001005a0       _mulscale7                 005015a0 f   engine.obj
 0001:00100f00       ?clipsprite_initindex@@YAHHPAUspritetype@@PAHPBUvec3_t@@@Z 00501f00 f   engine.obj
 0001:001013d0       _divscale22                005023d0 f   engine.obj
 0001:00102dc0       _divscale20                00503dc0 f   engine.obj
 0001:00102de0       ?keepaway@@YAXPAH0H@Z      00503de0 f   engine.obj
 0001:00102ed0       ?raytrace@@YAHHHPAH0@Z     00503ed0 f   engine.obj
 0001:001030f0       ?clipsprite_try@@YAHPBUspritetype@@HHHH@Z 005040f0 f   engine.obj
 0001:00103360       ?addclipline@@YAXHHHHH@Z   00504360 f   engine.obj
 0001:00103410       ?clipmove_tweak_pos@@YAXPBUvec3_t@@HHHHHHPAH1@Z 00504410 f   engine.obj
 0001:00103470       ?check_floor_curb@@YAHHHHHHH@Z 00504470 f   engine.obj
 0001:00103c70       ?inside_p@@YAHHHF@Z        00504c70 f   engine.obj
 0001:00103f50       ?inside_exclude_p@@YAHHHFPBE@Z 00504f50 f   engine.obj
 0001:001041f0       ?inside_z_p@@YAHHHHF@Z     005051f0 f   engine.obj
 0001:00105e90       ?maybe_alloc_palookup@@YAXH@Z 00506e90 f   engine.obj
 0001:00105ef0       ?alloc_palookup@@YAXH@Z    00506ef0 f   engine.obj
 0001:00105f30       ?palookup_isdefault@@YAHH@Z 00506f30 f   engine.obj
 0001:00106720       ?setpalettefade_calc@@YAXE@Z 00507720 f   engine.obj
 0001:001067f0       ?getpal@@YA?AUpalette_t@@H@Z 005077f0 f   engine.obj
 0001:00106be0       ?drawpixel_safe@@YAXPAXD@Z 00507be0 f   engine.obj
 0001:00106d20       _drawpixel                 00507d20 f   engine.obj
 0001:00106e90       _readpixel                 00507e90 f   engine.obj
 0001:00107420       _swapchar                  00508420 f   engine.obj
 0001:00107440       _swapchar2                 00508440 f   engine.obj
 0001:001076e0       _copybufreverse            005086e0 f   engine.obj
 0001:001077b0       ?sectorofwall_internal@@YAHF@Z 005087b0 f   engine.obj
 0001:001079e0       _dmulscale3                005089e0 f   engine.obj
 0001:00109000       _clearbufbyte              0050a000 f   engine.obj
 0001:0010a310       ?drawline16mid@@YAXHHHHD@Z 0050b310 f   engine.obj
 0001:0010ad20       ?sideview_getdist@@YAXFF@Z 0050bd20 f   engine.obj
 0001:0010ae50       ?sideview_cmppoints@@YAHPBX0@Z 0050be50 f   engine.obj
 0001:0010aeb0       ?drawscreen_drawwall@@YAXHHHHHH@Z 0050beb0 f   engine.obj
 0001:0010bb10       ?drawscreen_drawsprite@@YAXHHHHH@Z 0050cb10 f   engine.obj
 0001:0010c810       _mulscale6                 0050d810 f   engine.obj
 0001:0010c820       _mulscale13                0050d820 f   engine.obj
 0001:0010cd40       ?printext_checkypos@@YAHHPAH0@Z 0050dd40 f   engine.obj
 0001:0010cff0       ?screencapture_png@@YAHPBDD0@Z 0050dff0 f   engine.obj
 0001:0010d620       ?screencapture_common1@@YAHPADPBDPAPAU_iobuf@@@Z 0050e620 f   engine.obj
 0001:0010d820       ?PolymerProcessModels@@YAXXZ 0050e820 f   engine.obj
 0001:0010d9e0       _polymer_invalidateartmap  0050e9e0 f   engine.obj
 0001:0010ddd0       _xstrdup                   0050edd0 f   engine.obj
 0001:0010de00       ?hash_getcode@@YAIPBD@Z    0050ee00 f   engine.obj
 0001:0010e240       ?inthash_getcode@@YAIH@Z   0050f240 f   engine.obj
 0001:0010e3e0       _sector_tracker_hook       0050f3e0 f   engine.obj
 0001:0010e440       _wall_tracker_hook         0050f440 f   engine.obj
 0001:0010e4a0       _sprite_tracker_hook       0050f4a0 f   engine.obj
 0001:0010e500       ??$ALLOC_MAPART_ARRAY@$$BY0HIAA@EPAE@@YAXAAY0HIAA@EAAPAE@Z 0050f500 f   engine.obj
 0001:0010e550       ??$ALLOC_MAPART_ARRAY@$$BY0HIAA@HPAH@@YAXAAY0HIAA@HAAPAH@Z 0050f550 f   engine.obj
 0001:0010e5a0       ??$ALLOC_MAPART_ARRAY@$$BY0HIAA@Uvec2_t@@PAU1@@@YAXAAY0HIAA@Uvec2_t@@AAPAU0@@Z 0050f5a0 f   engine.obj
 0001:0010e5f0       ??$ALLOC_MAPART_ARRAY@$$BY0HIAA@Upicanm_t@@PAU1@@@YAXAAY0HIAA@Upicanm_t@@AAPAU0@@Z 0050f5f0 f   engine.obj
 0001:0010f4a0       ?getproc_@@YAPAXPBDPAHHH@Z 005104a0 f   glbuild.obj
 0001:00110c30       ?glugetproc_@@YAPAXPBDPAHH@Z 00511c30 f   glbuild.obj
 0001:00110eb0       _filnamcmp                 00511eb0 f   texcache.obj
 0001:00111380       _xcalloc                   00512380 f   texcache.obj
 0001:001113b0       _getrendermode             005123b0 f   texcache.obj
 0001:001113c0       ?texcache_tryart@@YAPAUpthtyp_t@@HHHH@Z 005123c0 f   texcache.obj
 0001:00111590       _polymost_want_npotytex    00512590 f   texcache.obj
 0001:001115e0       _check_nonpow2             005125e0 f   texcache.obj
 0001:00111610       _polymost_is_npotmode      00512610 f   texcache.obj
 0001:00111840       ?texcache_clearmemcache@@YAXXZ 00512840 f   texcache.obj
 0001:001118f0       ?texcache_closefiles@@YAXXZ 005128f0 f   texcache.obj
 0001:00111af0       ?texcache_enabled@@YAHXZ   00512af0 f   texcache.obj
 0001:00111ba0       ?texcache_deletefiles@@YAXXZ 00512ba0 f   texcache.obj
 0001:00111e00       _Bstrncpyz                 00512e00 f   texcache.obj
 0001:00111e30       _xrealloc                  00512e30 f   texcache.obj
 0001:00112190       _B_PASS32                  00513190 f   texcache.obj
 0001:001121a0       ?texcache_calcid@@YAPBDPADPBDHHD@Z 005131a0 f   texcache.obj
 0001:00112a90       ?texcache_setuptexture@@YAXPAHPAI@Z 00513a90 f   texcache.obj
 0001:00112ad0       ?texcache_loadmips@@YAHPBUtexcachehead_t@@PAIPAH2@Z 00513ad0 f   texcache.obj
 0001:00112f90       ?yrbrend@@YAXHHPAH@Z       00513f90 f   kplib.obj
 0001:00113960       _B_SWAP16                  00514960 f   kplib.obj
 0001:00113980       _B_SWAP32                  00514980 f   kplib.obj
 0001:001139b0       _B_PASS16                  005149b0 f   kplib.obj
 0001:001139c0       _B_PASS32                  005149c0 f   kplib.obj
 0001:001139d0       _B_UNBUF16                 005149d0 f   kplib.obj
 0001:001139e0       _B_UNBUF32                 005149e0 f   kplib.obj
 0001:001139f0       ?istarga@@YAHPBEH@Z        005149f0 f   kplib.obj
 0001:00113c70       ?kpngrend@@YAHPBDHHHHH@Z   00514c70 f   kplib.obj
 0001:00114b80       _tabledivide32             00515b80 f   kplib.obj
 0001:00114c10       ?peekbits@@YAHH@Z          00515c10 f   kplib.obj
 0001:00114c50       ?suckbits@@YAXH@Z          00515c50 f   kplib.obj
 0001:00114c70       ?suckbitsnextblock@@YAXXZ  00515c70 f   kplib.obj
 0001:00114e00       _B_BUF32                   00515e00 f   kplib.obj
 0001:00114e10       ?getbits@@YAHH@Z           00515e10 f   kplib.obj
 0001:00114e40       ?hufgetsym@@YAHPAH0@Z      00515e40 f   kplib.obj
 0001:00114ea0       ?qhufgencode@@YAXPAH00PAEH@Z 00515ea0 f   kplib.obj
 0001:00114fa0       ?bitrev@@YAHHH@Z           00515fa0 f   kplib.obj
 0001:00114fc0       ?hufgencode@@YAXPAHH00@Z   00515fc0 f   kplib.obj
 0001:00115190       ?initpass@@YAHXZ           00516190 f   kplib.obj
 0001:001155f0       ?putbuf@@YAXPBEH@Z         005165f0 f   kplib.obj
 0001:00115c50       ?Paeth686@@YAHHHH@Z        00516c50 f   kplib.obj
 0001:00115c90       ?rgbhlineasm@@YAXHHHH@Z    00516c90 f   kplib.obj
 0001:00115cf0       ?pal8hlineasm@@YAXHHHH@Z   00516cf0 f   kplib.obj
 0001:00115d30       ?initpngtables@@YAXXZ      00516d30 f   kplib.obj
 0001:00115e90       ?kpegrend@@YAHPBDHHHHH@Z   00516e90 f   kplib.obj
 0001:00117f20       ?mulshr24@@YAHHH@Z         00518f20 f   kplib.obj
 0001:00117f30       ?initkpeg@@YAXXZ           00518f30 f   kplib.obj
 0001:001181f0       ?huffgetval@@YAXHHHPAH0@Z  005191f0 f   kplib.obj
 0001:001182c0       ?invdct8x8@@YAXPAHE@Z      005192c0 f   kplib.obj
 0001:00118650       ?mulshr32@@YAHHH@Z         00519650 f   kplib.obj
 0001:00118660       ?kgifrend@@YAHPBDHHHHH@Z   00519660 f   kplib.obj
 0001:00118d60       _B_BUF16                   00519d60 f   kplib.obj
 0001:00118d70       ?ktgarend@@YAHPBDHHHHH@Z   00519d70 f   kplib.obj
 0001:00119230       ?kbmprend@@YAHPBDHHHHH@Z   0051a230 f   kplib.obj
 0001:00119a80       ?kpcxrend@@YAHPBDHHHHH@Z   0051aa80 f   kplib.obj
 0001:0011a8d0       ?kzcheckhashsiz@@YAHH@Z    0051b8d0 f   kplib.obj
 0001:0011a9a0       ?kzcalchash@@YAHPBD@Z      0051b9a0 f   kplib.obj
 0001:0011aeb0       ?kzcheckhash@@YAHPBDPAPADPAH2PAD@Z 0051beb0 f   kplib.obj
 0001:0011afb0       _filnamcmp                 0051bfb0 f   kplib.obj
 0001:0011bee0       ?putbuf4zip@@YAXPBEHH@Z    0051cee0 f   kplib.obj
 0001:0011c0b0       _xmalloc                   0051d0b0 f   kplib.obj
 0001:0011c550       _xstrdup                   0051d550 f   hightile.obj
 0001:0011c580       _xcalloc                   0051d580 f   hightile.obj
 0001:0011cc00       _clamp                     0051dc00 f   polymost.obj
 0001:0011cc40       _getrendermode             0051dc40 f   polymost.obj
 0001:0011cc50       ?bind_2d_texture@@YAXIH@Z  0051dc50 f   polymost.obj
 0001:0011d0b0       ?fogcalc@@YAXHHHH@Z        0051e0b0 f   polymost.obj
 0001:0011d280       _md_tilehasmodel           0051e280 f   polymost.obj
 0001:0011d2c0       ?fogcalc_old@@YAXHH@Z      0051e2c0 f   polymost.obj
 0001:0011d3f0       _klabs                     0051e3f0 f   polymost.obj
 0001:0011dae0       ?fixtransparency@@YAXPAUcoltype@@Uvec2_t@@1H@Z 0051eae0 f   polymost.obj
 0001:0011e810       _xmalloc                   0051f810 f   polymost.obj
 0001:0011e840       _xcalloc                   0051f840 f   polymost.obj
 0001:0011e870       _xrealloc                  0051f870 f   polymost.obj
 0001:0011e8a0       _polymost_want_npotytex    0051f8a0 f   polymost.obj
 0001:0011e8f0       _check_nonpow2             0051f8f0 f   polymost.obj
 0001:0011e920       _polymost_is_npotmode      0051f920 f   polymost.obj
 0001:0011e960       _bricolor                  0051f960 f   polymost.obj
 0001:0011ea00       ?polymost_setuptexture@@YAXHH@Z 0051fa00 f   polymost.obj
 0001:0011eb50       _Blrintf                   0051fb50 f   polymost.obj
 0001:0011fae0       _B_PASS16                  00520ae0 f   polymost.obj
 0001:0011faf0       _B_UNBUF16                 00520af0 f   polymost.obj
 0001:0011fb00       _swapchar                  00520b00 f   polymost.obj
 0001:0011fb20       _getticks                  00520b20 f   polymost.obj
 0001:00120b60       _getzsofslope              00521b60 f   polymost.obj
 0001:00120b90       ?get_projhack_ratio@@YAMXZ 00521b90 f   polymost.obj
 0001:001212e0       _dmulscale6                005222e0 f   polymost.obj
 0001:00121310       _yax_isislandwall          00522310 f   polymost.obj
 0001:00121d70       ?resizeglcheck@@YAXXZ      00522d70 f   polymost.obj
 0001:00121fb0       ?polymost_drawalls@@YAXH@Z 00522fb0 f   polymost.obj
 0001:00126020       _mulscale4                 00527020 f   polymost.obj
 0001:00126030       _getceilzofslope           00527030 f   polymost.obj
 0001:00126060       _getflorzofslope           00527060 f   polymost.obj
 0001:00126090       _get_floor_fogpal          00527090 f   polymost.obj
 0001:001260c0       _fogpal_shade              005270c0 f   polymost.obj
 0001:001260e0       _getpsky                   005270e0 f   polymost.obj
 0001:00126170       _getpskyidx                00527170 f   polymost.obj
 0001:001261b0       ?polymost_domost@@YAXMMMM@Z 005271b0 f   polymost.obj
 0001:00127050       _swaplong                  00528050 f   polymost.obj
 0001:00127070       ?polymost_drawpoly@@YAXQBUvec2f_t@@HH@Z 00528070 f   polymost.obj
 0001:00128f50       _have_basepal_tint         00529f50 f   polymost.obj
 0001:00128fa0       _hictinting_apply          00529fa0 f   polymost.obj
 0001:00129020       _getshadefactor            0052a020 f   polymost.obj
 0001:00129130       _eligible_for_tileshades   0052a130 f   polymost.obj
 0001:00129170       _polymer_eligible_for_artmap 0052a170 f   polymost.obj
 0001:001291b0       _setgotpic                 0052a1b0 f   polymost.obj
 0001:001291f0       ?our_texcache_fetch@@YAPAUpthtyp_t@@H@Z 0052a1f0 f   polymost.obj
 0001:00129250       _getpalookup               0052a250 f   polymost.obj
 0001:001292d0       ?vsdel@@YAXH@Z             0052a2d0 f   polymost.obj
 0001:00129370       ?vsinsaft@@YAHH@Z          0052a370 f   polymost.obj
 0001:00129430       ?polymost_internal_nonparallaxed@@YAXUvec2f_t@@0MMMMMMH@Z 0052a430 f   polymost.obj
 0001:0012a010       _swap64bit                 0052b010 f   polymost.obj
 0001:0012a040       _polymost_invsqrt_approximation 0052b040 f   polymost.obj
 0001:0012a090       ?calc_ypanning@@YAXHMMMMEEH@Z 0052b090 f   polymost.obj
 0001:0012a250       ?testvisiblemost@@YAHMM@Z  0052b250 f   polymost.obj
 0001:0012a2d0       ?polymost_getclosestpointonwall@@YAHQBUvec2_t@@HQAU1@@Z 0052b2d0 f   polymost.obj
 0001:0012a450       _tabledivide64             0052b450 f   polymost.obj
 0001:0012a520       ?polymost_bunchfront@@YAHHH@Z 0052b520 f   polymost.obj
 0001:0012a640       ?polymost_initmosts@@YAXPBM0H@Z 0052b640 f   polymost.obj
 0001:0012aa90       ?vsp_finalize_init@@YAXH@Z 0052ba90 f   polymost.obj
 0001:0012e110       _bad_tspr                  0052f110 f   polymost.obj
 0001:0012e150       ?polymost_findwall@@YAHQBUtspritetype@@PAH@Z 0052f150 f   polymost.obj
 0001:0012fb00       _mulscale16                00530b00 f   polymost.obj
 0001:0012fb10       ?tessectrap@@YAXPBM0PBHH@Z 00530b10 f   polymost.obj
 0001:001308b0       ?drawtrap@@YAXMMMMMM@Z     005318b0 f   polymost.obj
 0001:00131420       ?gen_font_glyph_tex@@YAHXZ 00532420 f   polymost.obj
 0001:001325e0       ?osdcmd_cvar_set_polymost@@YAHPBUosdfuncparm_t@@@Z 005335e0 f   polymost.obj
 0001:001327d0       ?gltexturemode@@YAHPBUosdfuncparm_t@@@Z 005337d0 f   polymost.obj
 0001:00132a30       _sprite_tracker_hook       00533a30 f   polymost.obj
 0001:00132ee0       _getticks                  00533ee0 f   polymer.obj
 0001:00133b60       _getrendermode             00534b60 f   polymer.obj
 0001:00133b70       _getzsofslope              00534b70 f   polymer.obj
 0001:00134370       _B_UNBUF16                 00535370 f   polymer.obj
 0001:00134380       _dot2f                     00535380 f   polymer.obj
 0001:001343b0       _dot3f                     005353b0 f   polymer.obj
 0001:001343f0       _relvec2f                  005353f0 f   polymer.obj
 0001:001345b0       _get_floor_fogpal          005355b0 f   polymer.obj
 0001:001345e0       _fogpal_shade              005355e0 f   polymer.obj
 0001:00134600       ?polymer_drawsearchplane@@YAXPAUs_prplane@@PAEE1@Z 00535600 f   polymer.obj
 0001:00134d20       _bad_tspr                  00535d20 f   polymer.obj
 0001:00135160       _polymer_invalidatesprite  00536160 f   polymer.obj
 0001:001351f0       _xmalloc                   005361f0 f   polymer.obj
 0001:00135260       _polymer_displayrooms      00536260 f   polymer.obj
 0001:001364d0       _xcalloc                   005374d0 f   polymer.obj
 0001:00136500       _set_globalpos             00537500 f   polymer.obj
 0001:00136540       _polymer_emptybuckets      00537540 f   polymer.obj
 0001:00136720       _polymer_drawplane         00537720 f   polymer.obj
 0001:00136a40       _polymer_bucketplane       00537a40 f   polymer.obj
 0001:00136b80       _xrealloc                  00537b80 f   polymer.obj
 0001:00136bb0       _polymer_inb4mirror        00537bb0 f   polymer.obj
 0001:00136d50       _polymer_animatesprites    00537d50 f   polymer.obj
 0001:00136d90       _polymer_freeboard         00537d90 f   polymer.obj
 0001:001371c0       _polymer_invalidateartmap  005381c0 f   polymer.obj
 0001:00137200       _polymer_initsector        00538200 f   polymer.obj
 0001:00137410       _polymer_updatesector      00538410 f   polymer.obj
 0001:001381a0       _swaplong                  005391a0 f   polymer.obj
 0001:00138320       _polymer_buildfloor        00539320 f   polymer.obj
 0001:001385e0       _polymer_drawsector        005395e0 f   polymer.obj
 0001:00138890       _get_ceiling_fogpal        00539890 f   polymer.obj
 0001:001388c0       _polymer_initwall          005398c0 f   polymer.obj
 0001:00138ad0       _polymer_updatewall        00539ad0 f   polymer.obj
 0001:0013a700       ?calc_ypancoef@@YAMDFH@Z   0053b700 f   polymer.obj
 0001:0013a7c0       _Blrintf                   0053b7c0 f   polymer.obj
 0001:0013a7e0       _polymer_drawwall          0053b7e0 f   polymer.obj
 0001:0013aa60       _polymer_computeplane      0053ba60 f   polymer.obj
 0001:0013b430       _polymer_crossproduct      0053c430 f   polymer.obj
 0001:0013b490       _polymer_normalize         0053c490 f   polymer.obj
 0001:0013b510       _polymer_pokesector        0053c510 f   polymer.obj
 0001:0013b640       _polymer_extractfrustum    0053c640 f   polymer.obj
 0001:0013b760       _polymer_planeinfrustum    0053c760 f   polymer.obj
 0001:0013b850       _polymer_scansprites       0053c850 f   polymer.obj
 0001:0013b930       _polymer_updatesprite      0053c930 f   polymer.obj
 0001:0013c410       _polymer_transformpoint    0053d410 f   polymer.obj
 0001:0013c4b0       _polymer_getsky            0053d4b0 f   polymer.obj
 0001:0013c5a0       _getpsky                   0053d5a0 f   polymer.obj
 0001:0013c630       _getpskyidx                0053d630 f   polymer.obj
 0001:0013c670       _polymer_drawsky           0053d670 f   polymer.obj
 0001:0013c780       _polymer_initartsky        0053d780 f   polymer.obj
 0001:0013c830       _polymer_drawartsky        0053d830 f   polymer.obj
 0001:0013cb50       _have_basepal_tint         0053db50 f   polymer.obj
 0001:0013cba0       _hictinting_apply          0053dba0 f   polymer.obj
 0001:0013cc20       _getshadefactor            0053dc20 f   polymer.obj
 0001:0013cd30       _eligible_for_tileshades   0053dd30 f   polymer.obj
 0001:0013cd70       _polymer_drawartskyquad    0053dd70 f   polymer.obj
 0001:0013ce90       _polymer_drawskybox        0053de90 f   polymer.obj
 0001:0013d160       _polymer_drawmdsprite      0053e160 f   polymer.obj
 0001:0013fa40       _hictinting_apply_ub       00540a40 f   polymer.obj
 0001:0013fb20       _polymer_loadmodelvbos     00540b20 f   polymer.obj
 0001:0013fd30       _polymer_getscratchmaterial 00540d30 f   polymer.obj
 0001:0013fe20       _polymer_getbuildmaterial  00540e20 f   polymer.obj
 0001:00140380       _polymer_eligible_for_artmap 00541380 f   polymer.obj
 0001:001403c0       _polymer_findbucket        005413c0 f   polymer.obj
 0001:00140500       ?polymer_setupartmap@@YAXFD@Z 00541500 f   polymer.obj
 0001:001408b0       _polymer_bindmaterial      005418b0 f   polymer.obj
 0001:001418e0       _polymer_unbindmaterial    005428e0 f   polymer.obj
 0001:00141990       _polymer_compileprogram    00542990 f   polymer.obj
 0001:00142020       _polymer_removelight       00543020 f   polymer.obj
 0001:001420e0       _polymer_updatelights      005430e0 f   polymer.obj
 0001:00142250       _polymer_resetplanelights  00543250 f   polymer.obj
 0001:00142290       _polymer_addplanelight     00543290 f   polymer.obj
 0001:001424c0       _polymer_deleteplanelight  005434c0 f   polymer.obj
 0001:00142550       _polymer_planeinlight      00543550 f   polymer.obj
 0001:00142690       _polymer_invalidatesectorlights 00543690 f   polymer.obj
 0001:00142760       _polymer_invalidateplanelights 00543760 f   polymer.obj
 0001:00142800       _polymer_processspotlight  00543800 f   polymer.obj
 0001:00142a20       _polymer_culllight         00543a20 f   polymer.obj
 0001:00143090       _polymer_prepareshadows    00544090 f   polymer.obj
 0001:00143420       _polymer_initrendertargets 00544420 f   polymer.obj
 0001:00143b70       _wall_tracker_hook         00544b70 f   polymer.obj
 0001:001440d0       ?nullskintexids@@YAXI@Z    005450d0 f   mdsprite.obj
 0001:001442b0       _xrealloc                  005452b0 f   mdsprite.obj
 0001:00144490       _Blrintf                   00545490 f   mdsprite.obj
 0001:001444b0       ?addtileP@@YAHHHH@Z        005454b0 f   mdsprite.obj
 0001:001445a0       ?framename2index@@YAHPAUmdmodel_t@@PBD@Z 005455a0 f   mdsprite.obj
 0001:00144780       _xmalloc                   00545780 f   mdsprite.obj
 0001:00144950       _xstrdup                   00545950 f   mdsprite.obj
 0001:00144980       _xcalloc                   00545980 f   mdsprite.obj
 0001:001457e0       _Bstrncpyz                 005467e0 f   mdsprite.obj
 0001:00145810       _getticks                  00546810 f   mdsprite.obj
 0001:00145820       _check_nonpow2             00546820 f   mdsprite.obj
 0001:00145850       ?QuitOnFatalError@@YAXPBD@Z 00546850 f   mdsprite.obj
 0001:001458a0       ?daskinloader@@YAHHPAH00000PADHD@Z 005468a0 f   mdsprite.obj
 0001:00146030       _B_PASS16                  00547030 f   mdsprite.obj
 0001:00146040       _B_UNBUF16                 00547040 f   mdsprite.obj
 0001:00146050       _swapchar                  00547050 f   mdsprite.obj
 0001:00146070       ?hicfxmask@@YAHH@Z         00547070 f   mdsprite.obj
 0001:001467a0       _swapshort                 005477a0 f   mdsprite.obj
 0001:001467c0       _swaplong                  005477c0 f   mdsprite.obj
 0001:00147050       ?invertmatrix@@YAXPAM0@Z   00548050 f   mdsprite.obj
 0001:00147240       ?normalize@@YAXPAM@Z       00548240 f   mdsprite.obj
 0001:001472c0       _polymost_invsqrt_approximation 005482c0 f   mdsprite.obj
 0001:00147310       ?init_mdtrig_arrays@@YAXXZ 00548310 f   mdsprite.obj
 0001:001476a0       ?mdload@@YAPAUmdmodel_t@@PBD@Z 005486a0 f   mdsprite.obj
 0001:001477c0       _B_PASS32                  005487c0 f   mdsprite.obj
 0001:001477d0       ?md2load@@YAPAUmd2model_t@@HPBD@Z 005487d0 f   mdsprite.obj
 0001:001486f0       ?md3load@@YAPAUmd3model_t@@H@Z 005496f0 f   mdsprite.obj
 0001:00148c30       ?md3postload_common@@YAXPAUmd3model_t@@@Z 00549c30 f   mdsprite.obj
 0001:00149040       ?md3postload_polymer_check@@YAHPAUmd3model_t@@@Z 0054a040 f   mdsprite.obj
 0001:00149390       ?polymost_md3draw@@YAHPAUmd3model_t@@PBUtspritetype@@@Z 0054a390 f   mdsprite.obj
 0001:0014aed0       _clamp                     0054bed0 f   mdsprite.obj
 0001:0014af10       _fclamp                    0054bf10 f   mdsprite.obj
 0001:0014af60       _have_basepal_tint         0054bf60 f   mdsprite.obj
 0001:0014afb0       _hictinting_apply          0054bfb0 f   mdsprite.obj
 0001:0014b030       _sepldist                  0054c030 f   mdsprite.obj
 0001:0014b0a0       _klabs                     0054c0a0 f   mdsprite.obj
 0001:0014b0b0       ?mdloadvbos@@YAXPAUmd3model_t@@@Z 0054c0b0 f   mdsprite.obj
 0001:0014b190       ?quicksort@@YAXPAGPAMHH@Z  0054c190 f   mdsprite.obj
 0001:0014b210       ?md3draw_handle_triangles@@YAXPBUmd3surf_t@@PAGHPBUmd3model_t@@@Z 0054c210 f   mdsprite.obj
 0001:0014b480       ?mdfree@@YAXPAUmdmodel_t@@@Z 0054c480 f   mdsprite.obj
 0001:0014b4c0       ?md3free@@YAXPAUmd3model_t@@@Z 0054c4c0 f   mdsprite.obj
 0001:0014b8b0       _xmalloc                   0054c8b0 f   voxmodel.obj
 0001:0014bb60       _xcalloc                   0054cb60 f   voxmodel.obj
 0001:0014bb90       ?vox2poly@@YAPAUvoxmodel_t@@XZ 0054cb90 f   voxmodel.obj
 0001:0014c840       ?isrectfree@@YAHHHHH@Z     0054d840 f   voxmodel.obj
 0001:0014c970       ?setrect@@YAXHHHH@Z        0054d970 f   voxmodel.obj
 0001:0014cab0       ?cntquad@@YAXHHHHHHHHHH@Z  0054dab0 f   voxmodel.obj
 0001:0014cbb0       ?addquad@@YAXHHHHHHHHHH@Z  0054dbb0 f   voxmodel.obj
 0001:0014d370       ?getvox@@YAHHHH@Z          0054e370 f   voxmodel.obj
 0001:0014d3f0       ?isolid@@YAHHHH@Z          0054e3f0 f   voxmodel.obj
 0001:0014d460       ?loadvox@@YAHPBD@Z         0054e460 f   voxmodel.obj
 0001:0014d8e0       ?putvox@@YAXHHHH@Z         0054e8e0 f   voxmodel.obj
 0001:0014d9f0       _xrealloc                  0054e9f0 f   voxmodel.obj
 0001:0014da20       ?isair@@YAHH@Z             0054ea20 f   voxmodel.obj
 0001:0014da50       ?alloc_vcolhashead@@YAXXZ  0054ea50 f   voxmodel.obj
 0001:0014dab0       ?alloc_vbit@@YAXXZ         0054eab0 f   voxmodel.obj
 0001:0014db20       ?read_pal@@YAXHQAH@Z       0054eb20 f   voxmodel.obj
 0001:0014dba0       _B_PASS32                  0054eba0 f   voxmodel.obj
 0001:0014dbb0       ?loadkvx@@YAHPBD@Z         0054ebb0 f   voxmodel.obj
 0001:0014e090       _B_PASS16                  0054f090 f   voxmodel.obj
 0001:0014e0a0       ?setzrange1@@YAXPAHHH@Z    0054f0a0 f   voxmodel.obj
 0001:0014e170       ?loadkv6@@YAHPBD@Z         0054f170 f   voxmodel.obj
 0001:0014e530       _B_UNBUF16                 0054f530 f   voxmodel.obj
 0001:0014e540       _B_UNBUF32                 0054f540 f   voxmodel.obj
 0001:0014ef90       _hictinting_apply          0054ff90 f   voxmodel.obj
 0001:0014f370       _B_PASS32                  00550370 f   dxtfilter.obj
 0001:0014f380       _B_BUF16                   00550380 f   dxtfilter.obj
 0001:0014f390       _B_UNBUF16                 00550390 f   dxtfilter.obj
 0001:0014f3a0       _tabledivide32             005503a0 f   dxtfilter.obj
 0001:0014f430       ?dxt_hicosub@@YAGG@Z       00550430 f   dxtfilter.obj
 0001:0014f480       ?dxt_handle_io@@YAXHHPAXPAD@Z 00550480 f   dxtfilter.obj
 0001:0014f8b0       ?dedxt_hicoadd@@YAGG@Z     005508b0 f   dxtfilter.obj
 0001:0014f900       ?dedxt_handle_io@@YAHHHPAXHPADH@Z 00550900 f   dxtfilter.obj
 0001:0014fbc0       ?LZ4_64bits@@YAIXZ         00550bc0 f   lz4.obj
 0001:0014fbd0       ?LZ4_compress_generic@@YAHQAXQBDQADHHW4limitedOutput_directive@@W4tableType_t@@W4dict_directive@@W4dictIssue_directive@@I@Z 00550bd0 f   lz4.obj
 0001:001502e0       ?LZ4_writeLE16@@YAXPAXG@Z  005512e0 f   lz4.obj
 0001:00150320       ?LZ4_isLittleEndian@@YAIXZ 00551320 f   lz4.obj
 0001:00150340       ?LZ4_read32@@YAIPBX@Z      00551340 f   lz4.obj
 0001:00150360       ?LZ4_wildCopy@@YAXPAXPBX0@Z 00551360 f   lz4.obj
 0001:001503b0       ?LZ4_copy8@@YAXPAXPBX@Z    005513b0 f   lz4.obj
 0001:001503d0       ?LZ4_count@@YAIPBE00@Z     005513d0 f   lz4.obj
 0001:001504f0       ?LZ4_read16@@YAGPBX@Z      005514f0 f   lz4.obj
 0001:00150510       ?LZ4_read_ARCH@@YAIPBX@Z   00551510 f   lz4.obj
 0001:00150540       ?LZ4_read64@@YA_KPBX@Z     00551540 f   lz4.obj
 0001:00150570       ?LZ4_NbCommonBytes@@YAII@Z 00551570 f   lz4.obj
 0001:00150670       ?LZ4_hashPosition@@YAIPBXW4tableType_t@@@Z 00551670 f   lz4.obj
 0001:00150690       ?LZ4_hashSequenceT@@YAIIW4tableType_t@@@Z 00551690 f   lz4.obj
 0001:001506c0       ?LZ4_hashSequence@@YAIIW4tableType_t@@@Z 005516c0 f   lz4.obj
 0001:001506f0       ?LZ4_hashSequence64@@YAIIW4tableType_t@@@Z 005516f0 f   lz4.obj
 0001:00150750       ?LZ4_putPositionOnHash@@YAXPBEIPAXW4tableType_t@@0@Z 00551750 f   lz4.obj
 0001:001507c0       ?LZ4_putPosition@@YAXPBEPAXW4tableType_t@@0@Z 005517c0 f   lz4.obj
 0001:00150800       ?LZ4_getPositionOnHash@@YAPBEIPAXW4tableType_t@@PBE@Z 00551800 f   lz4.obj
 0001:00150850       ?LZ4_getPosition@@YAPBEPBEPAXW4tableType_t@@0@Z 00551850 f   lz4.obj
 0001:00150a20       ?LZ4_compress_destSize_extState@@YAHPAXPBDPADPAHH@Z 00551a20 f   lz4.obj
 0001:00150ac0       ?LZ4_compress_destSize_generic@@YAHQAXQBDQADQAHHW4tableType_t@@@Z 00551ac0 f   lz4.obj
 0001:00151430       ?LZ4_renormDictT@@YAXPAULZ4_stream_t_internal@@PBE@Z 00552430 f   lz4.obj
 0001:00151670       ?LZ4_decompress_generic@@YAHQBDQADHHHHHHQBE2I@Z 00552670 f   lz4.obj
 0001:00151d40       ?LZ4_readLE16@@YAGPBX@Z    00552d40 f   lz4.obj
 0001:00151d80       ?LZ4_copy4@@YAXPAXPBX@Z    00552d80 f   lz4.obj
 0001:001520c0       ?LZ4_decompress_usingDict_generic@@YAHPBDPADHHH0H@Z 005530c0 f   lz4.obj
 0001:001523a0       ?LZ4_init@@YAXPAULZ4_stream_t_internal@@PAE@Z 005533a0 f   lz4.obj
 0001:00152710       ?MD4Transform@@YAXQAIQBE@Z 00553710 f   md4.obj
 0001:00153060       ?Encode@@YAXPAEPBII@Z      00554060 f   md4.obj
 0001:00153100       ?Decode@@YAXPAIPBEI@Z      00554100 f   md4.obj
 0001:00153560       _xrealloc                  00554560 f   osd.obj
 0001:00153830       _xmalloc                   00554830 f   osd.obj
 0001:001539e0       ?swaposdptrs@@YAXXZ        005549e0 f   osd.obj
 0001:00153a40       _swapptr                   00554a40 f   osd.obj
 0001:00153a70       ?_internal_drawosdchar@@YAXHHDHH@Z 00554a70 f   osd.obj
 0001:00153ab0       ?_internal_drawosdstr@@YAXHHPBDHHH@Z 00554ab0 f   osd.obj
 0001:00153b90       ?_internal_drawosdcursor@@YAXHHHH@Z 00554b90 f   osd.obj
 0001:00153c80       _klabs                     00554c80 f   osd.obj
 0001:00153c90       ?_internal_getcolumnwidth@@YAHH@Z 00554c90 f   osd.obj
 0001:00153cb0       ?_internal_getrowheight@@YAHH@Z 00554cb0 f   osd.obj
 0001:00153cd0       ?_internal_clearbackground@@YAXHH@Z 00554cd0 f   osd.obj
 0001:00153ce0       ?_internal_gettime@@YAHXZ  00554ce0 f   osd.obj
 0001:00153cf0       ?_internal_onshowosd@@YAXH@Z 00554cf0 f   osd.obj
 0001:00154420       ?_internal_osdfunc_exec@@YAHPBUosdfuncparm_t@@@Z 00555420 f   osd.obj
 0001:001544a0       ?_internal_osdfunc_echo@@YAHPBUosdfuncparm_t@@@Z 005554a0 f   osd.obj
 0001:001544c0       ?_internal_osdfunc_fileinfo@@YAHPBUosdfuncparm_t@@@Z 005554c0 f   osd.obj
 0001:001546d0       _getticks                  005556d0 f   osd.obj
 0001:001546e0       ?_internal_osdfunc_alias@@YAHPBUosdfuncparm_t@@@Z 005556e0 f   osd.obj
 0001:001548b0       _xstrdup                   005558b0 f   osd.obj
 0001:001548e0       ?_internal_osdfunc_unalias@@YAHPBUosdfuncparm_t@@@Z 005558e0 f   osd.obj
 0001:001549a0       ?_internal_osdfunc_listsymbols@@YAHPBUosdfuncparm_t@@@Z 005559a0 f   osd.obj
 0001:00154bb0       ?OSD_CvarModified@@YAHPBUosdcvar_t@@@Z 00555bb0 f   osd.obj
 0001:00154cf0       ?_internal_osdfunc_help@@YAHPBUosdfuncparm_t@@@Z 00555cf0 f   osd.obj
 0001:00154d50       ?_internal_osdfunc_clear@@YAHPBUosdfuncparm_t@@@Z 00555d50 f   osd.obj
 0001:00154db0       ?_internal_osdfunc_history@@YAHPBUosdfuncparm_t@@@Z 00555db0 f   osd.obj
 0001:00154e50       ?osdcmd_cvar_set_osd@@YAHPBUosdfuncparm_t@@@Z 00555e50 f   osd.obj
 0001:00154f70       ?_internal_osdfunc_toggle@@YAHPBUosdfuncparm_t@@@Z 00555f70 f   osd.obj
 0001:00156130       _OSD_SetHistory            00557130 f   osd.obj
 0001:00156190       _Bstrncpyz                 00557190 f   osd.obj
 0001:001561c0       ?OSD_FindDiffPoint@@YAHPBD0@Z 005571c0 f   osd.obj
 0001:00156230       ?OSD_HistoryPrev@@YAXXZ    00557230 f   osd.obj
 0001:001563f0       ?OSD_HistoryNext@@YAXXZ    005573f0 f   osd.obj
 0001:00157b80       ?OSD_LineFeed@@YAXXZ       00558b80 f   osd.obj
 0001:00157ec0       ?strtoken@@YAPADPADPAPADPAH@Z 00558ec0 f   osd.obj
 0001:001582c0       ?addnewsymbol@@YAPAU_symbol@@PBD@Z 005592c0 f   osd.obj
 0001:00158470       ?findsymbol@@YAPAU_symbol@@PBDPAU1@@Z 00559470 f   osd.obj
 0001:001584e0       ?findexactsymbol@@YAPAU_symbol@@PBD@Z 005594e0 f   osd.obj
 0001:00158d30       _getrendermode             00559d30 f   osd.obj
 0001:001590f0       _divideu32                 0055a0f0 f   pragmas.obj
 0001:00159170       _tabledivide32             0055a170 f   pragmas.obj
 0001:00159220       _tabledivide64             0055a220 f   pragmas.obj
 0001:00159340       ?skipoverws@@YAXPAUscriptfile@@@Z 0055a340 f   scriptfile.obj
 0001:00159370       ?skipovertoken@@YAXPAUscriptfile@@@Z 0055a370 f   scriptfile.obj
 0001:00159660       ?parsedouble@@YANPADPAPAD@Z 0055a660 f   scriptfile.obj
 0001:00159e00       _xmalloc                   0055ae00 f   scriptfile.obj
 0001:00159f30       _xstrdup                   0055af30 f   scriptfile.obj
 0001:0015a130       _B_UNBUF32                 0055b130 f   scriptfile.obj
 0001:0015a220       _B_BUF32                   0055b220 f   scriptfile.obj
 0001:0015a230       ?getsymbtabspace@@YAPADH@Z 0055b230 f   scriptfile.obj
 0001:0015a2f0       _xrealloc                  0055b2f0 f   scriptfile.obj
 0001:0015a680       ?win_printversion@@YAXXZ   0055b680 f   winbits.obj
 0001:0015a8f0       ?ToggleDesktopComposition@@YAXH@Z 0055b8f0 f   winbits.obj
 0001:0015ace0       ?XXH32_endian_align@@YAIPBXIIW4XXH_endianess@@W4XXH_alignment@@@Z 0055bce0 f   xxhash.obj
 0001:0015af80       ?XXH_readLE32_align@@YAIPBXW4XXH_endianess@@W4XXH_alignment@@@Z 0055bf80 f   xxhash.obj
 0001:0015aff0       ?XXH_read32@@YAIPBX@Z      0055bff0 f   xxhash.obj
 0001:0015b070       ?XXH64_endian_align@@YA_KPBXI_KW4XXH_endianess@@W4XXH_alignment@@@Z 0055c070 f   xxhash.obj
 0001:0015b7b0       ?XXH_readLE64_align@@YA_KPBXW4XXH_endianess@@W4XXH_alignment@@@Z 0055c7b0 f   xxhash.obj
 0001:0015b840       ?XXH_read64@@YA_KPBX@Z     0055c840 f   xxhash.obj
 0001:0015b880       ?XXH_malloc@@YAPAXI@Z      0055c880 f   xxhash.obj
 0001:0015b8c0       ?XXH_free@@YAXPAX@Z        0055c8c0 f   xxhash.obj
 0001:0015ba80       ?XXH32_update_endian@@YA?AW4XXH_errorcode@@PAUXXH32_state_s@@PBXIW4XXH_endianess@@@Z 0055ca80 f   xxhash.obj
 0001:0015be40       ?XXH_memcpy@@YAPAXPAXPBXI@Z 0055ce40 f   xxhash.obj
 0001:0015be60       ?XXH_readLE32@@YAIPBXW4XXH_endianess@@@Z 0055ce60 f   xxhash.obj
 0001:0015bec0       ?XXH32_digest_endian@@YAIPBUXXH32_state_s@@W4XXH_endianess@@@Z 0055cec0 f   xxhash.obj
 0001:0015c080       ?XXH64_update_endian@@YA?AW4XXH_errorcode@@PAUXXH64_state_s@@PBXIW4XXH_endianess@@@Z 0055d080 f   xxhash.obj
 0001:0015c5c0       ?XXH_readLE64@@YA_KPBXW4XXH_endianess@@@Z 0055d5c0 f   xxhash.obj
 0001:0015c620       ?XXH64_digest_endian@@YA_KPBUXXH64_state_s@@W4XXH_endianess@@@Z 0055d620 f   xxhash.obj
 0001:0015cda0       _Bstrncpyz                 0055dda0 f   sdlayer.obj
 0001:0015cf40       ?buildkeytranslationtable@@YAHXZ 0055df40 f   sdlayer.obj
 0001:0015d250       ?sighandler@@YAXH@Z        0055e250 f   sdlayer.obj
 0001:0015d2a0       ?attach_debugger_here@@YAXXZ 0055e2a0 f   sdlayer.obj
 0001:0015d950       ?W_SetKeyboardLayoutUS@@YAXH@Z 0055e950 f   sdlayer.obj
 0001:0015d9a0       ?switchlayout@@YAXPBD@Z    0055e9a0 f   sdlayer.obj
 0001:0015db50       ?grabmouse_low@@YADD@Z     0055eb50 f   sdlayer.obj
 0001:0015de40       _tabledivide32             0055ee40 f   sdlayer.obj
 0001:0015e460       ?sortmodes@@YAHPBX0@Z      0055f460 f   sdlayer.obj
 0001:0015e680       _clamp                     0055f680 f   sdlayer.obj
 0001:0015e6c0       _klabs                     0055f6c0 f   sdlayer.obj
 0001:0015f310       ?destroy_window_resources@@YAXXZ 00560310 f   sdlayer.obj
 0001:0015fc40       ?loadappicon@@YAPAUSDL_Surface@@XZ 00560c40 f   sdlayer.obj
 0001:001605c0       _keyascfifo_isfull         005615c0 f   sdlayer.obj
 0001:001605f0       _keyascfifo_insert         005615f0 f   sdlayer.obj
 0001:00160ac0       ?FX_CheckMVErr@@YAHH@Z     00561ac0 f   fx_man.obj
 0001:00160d20       ?FX_AutoDetectFormat@@YA?AW4wavefmt_t@@PBDI@Z 00561d20 f   fx_man.obj
 0001:00161000       ?DisableInterrupts@@YAXXZ  00562000 f   multivoc.obj
 0001:00161030       ?RestoreInterrupts@@YAXXZ  00562030 f   multivoc.obj
 0001:001610a0       ?MV_GetVoice@@YAPAUVoiceNode@@H@Z 005620a0 f   multivoc.obj
 0001:00161250       ?MV_StopVoice@@YAXPAUVoiceNode@@@Z 00562250 f   multivoc.obj
 0001:00161300       ?MV_EndService@@YAXXZ      00562300 f   multivoc.obj
 0001:00161810       _swapptr                   00562810 f   multivoc.obj
 0001:00161840       ?MV_GetVolumeTable@@YAPBFH@Z 00562840 f   multivoc.obj
 0001:00161ca0       ?MV_CalcVolume@@YAXH@Z     00562ca0 f   multivoc.obj
 0001:00161fd0       _xaligned_malloc           00562fd0 f   multivoc.obj
 0001:00162000       ?MV_SetMixMode@@YAHH@Z     00563000 f   multivoc.obj
 0001:00162070       ?MV_StartPlayback@@YAHXZ   00563070 f   multivoc.obj
 0001:00162100       ?MV_ServiceVoc@@YAXXZ      00563100 f   multivoc.obj
 0001:001623a0       ?MV_Mix@@YAXPAUVoiceNode@@H@Z 005633a0 f   multivoc.obj
 0001:00162540       ?MV_CalcPanTable@@YAXXZ    00563540 f   multivoc.obj
 0001:00162740       ?MV_StopPlayback@@YAXXZ    00563740 f   multivoc.obj
 0001:001637b0       ?MV_GetNextWAVBlock@@YA?AW4playbackstatus@@PAUVoiceNode@@@Z 005647b0 f   formats.obj
 0001:00163b20       ?MV_GetNextVOCBlock@@YA?AW4playbackstatus@@PAUVoiceNode@@@Z 00564b20 f   formats.obj
 0001:00164110       ?read_vorbis@@YAIPAXII0@Z  00565110 f   vorbis.obj
 0001:001641e0       ?seek_vorbis@@YAHPAX_JH@Z  005651e0 f   vorbis.obj
 0001:00164260       ?close_vorbis@@YAHPAX@Z    00565260 f   vorbis.obj
 0001:00164270       ?tell_vorbis@@YAJPAX@Z     00565270 f   vorbis.obj
 0001:001646c0       ?MV_GetVorbisCommentLoops@@YAXPAUVoiceNode@@PAUvorbis_comment@@@Z 005656c0 f   vorbis.obj
 0001:001648f0       ?MV_GetNextVorbisBlock@@YA?AW4playbackstatus@@PAUVoiceNode@@@Z 005658f0 f   vorbis.obj
 0001:00165020       ?MV_GetNextXABlock@@YA?AW4playbackstatus@@PAUVoiceNode@@@Z 00566020 f   xa.obj
 0001:00165250       ?decodeSoundSectMono@@YAXPAUXASector@@PAUxa_data@@@Z 00566250 f   xa.obj
 0001:00165510       ?FXD_FixMul@@YAHHH@Z       00566510 f   xa.obj
 0001:00165590       ?getSoundData@@YACPADHH@Z  00566590 f   xa.obj
 0001:00165600       ?getFilter@@YACPADH@Z      00566600 f   xa.obj
 0001:00165620       ?getRange@@YACPADH@Z       00566620 f   xa.obj
 0001:00165640       ?decodeSoundSectStereo@@YAXPAUXASector@@PAUxa_data@@@Z 00566640 f   xa.obj
 0001:00166060       ?TeardownDSound@@YAXJ@Z    00567060 f   driver_directsound.obj
 0001:001662d0       ?FillBuffer@@YAXH@Z        005672d0 f   driver_directsound.obj
 0001:001663e0       ?FillBufferPortion@@YAXPADH@Z 005673e0 f   driver_directsound.obj
 0001:001664e0       ?fillDataThread@@YGKPAX@Z  005674e0 f   driver_directsound.obj
 0001:00167870       ?initialize_crc32@@YAXXZ   00568870 f   packet.obj
 0001:00167910       ?reflect_crc@@YAIHH@Z      00568910 f   packet.obj
 0001:00167fd0       ?enet_peer_reset_outgoing_commands@@YAXPAU_ENetList@@@Z 00568fd0 f   peer.obj
 0001:00168040       ?enet_peer_reset_incoming_commands@@YAXPAU_ENetList@@@Z 00569040 f   peer.obj
 0001:00168060       ?enet_peer_remove_incoming_commands@@YAXPAU_ENetList@@PAU_ENetListNode@@1@Z 00569060 f   peer.obj
 0001:00169270       ?enet_protocol_send_outgoing_commands@@YAHPAU_ENetHost@@PAU_ENetEvent@@H@Z 0056a270 f   protocol.obj
 0001:00169830       ?enet_protocol_remove_sent_unreliable_commands@@YAXPAU_ENetPeer@@@Z 0056a830 f   protocol.obj
 0001:001698d0       ?enet_protocol_send_acknowledgements@@YAXPAU_ENetHost@@PAU_ENetPeer@@@Z 0056a8d0 f   protocol.obj
 0001:00169a70       ?enet_protocol_dispatch_state@@YAXPAU_ENetHost@@PAU_ENetPeer@@W4_ENetPeerState@@@Z 0056aa70 f   protocol.obj
 0001:00169ac0       ?enet_protocol_change_state@@YAXPAU_ENetHost@@PAU_ENetPeer@@W4_ENetPeerState@@@Z 0056aac0 f   protocol.obj
 0001:00169b00       ?enet_protocol_send_unreliable_outgoing_commands@@YAXPAU_ENetHost@@PAU_ENetPeer@@@Z 0056ab00 f   protocol.obj
 0001:00169e30       ?enet_protocol_check_timeouts@@YAHPAU_ENetHost@@PAU_ENetPeer@@PAU_ENetEvent@@@Z 0056ae30 f   protocol.obj
 0001:0016a040       ?enet_protocol_notify_disconnect@@YAXPAU_ENetHost@@PAU_ENetPeer@@PAU_ENetEvent@@@Z 0056b040 f   protocol.obj
 0001:0016a0d0       ?enet_protocol_send_reliable_outgoing_commands@@YAHPAU_ENetHost@@PAU_ENetPeer@@@Z 0056b0d0 f   protocol.obj
 0001:0016a560       ?enet_protocol_dispatch_incoming_commands@@YAHPAU_ENetHost@@PAU_ENetEvent@@@Z 0056b560 f   protocol.obj
 0001:0016a930       ?enet_protocol_receive_incoming_commands@@YAHPAU_ENetHost@@PAU_ENetEvent@@@Z 0056b930 f   protocol.obj
 0001:0016aa80       ?enet_protocol_handle_incoming_commands@@YAHPAU_ENetHost@@PAU_ENetEvent@@@Z 0056ba80 f   protocol.obj
 0001:0016b130       ?enet_protocol_handle_connect@@YAPAU_ENetPeer@@PAU_ENetHost@@PAU_ENetProtocolHeader@@PAT_ENetProtocol@@@Z 0056c130 f   protocol.obj
 0001:0016b6c0       ?enet_protocol_handle_send_reliable@@YAHPAU_ENetHost@@PAU_ENetPeer@@PAT_ENetProtocol@@PAPAE@Z 0056c6c0 f   protocol.obj
 0001:0016b780       ?enet_protocol_handle_send_unsequenced@@YAHPAU_ENetHost@@PAU_ENetPeer@@PAT_ENetProtocol@@PAPAE@Z 0056c780 f   protocol.obj
 0001:0016b950       ?enet_protocol_handle_send_unreliable@@YAHPAU_ENetHost@@PAU_ENetPeer@@PAT_ENetProtocol@@PAPAE@Z 0056c950 f   protocol.obj
 0001:0016ba10       ?enet_protocol_handle_send_fragment@@YAHPAU_ENetHost@@PAU_ENetPeer@@PBT_ENetProtocol@@PAPAE@Z 0056ca10 f   protocol.obj
 0001:0016bd90       ?enet_protocol_handle_send_unreliable_fragment@@YAHPAU_ENetHost@@PAU_ENetPeer@@PBT_ENetProtocol@@PAPAE@Z 0056cd90 f   protocol.obj
 0001:0016c120       ?enet_protocol_handle_ping@@YAHPAU_ENetHost@@PAU_ENetPeer@@PBT_ENetProtocol@@@Z 0056d120 f   protocol.obj
 0001:0016c140       ?enet_protocol_handle_bandwidth_limit@@YAHPAU_ENetHost@@PAU_ENetPeer@@PBT_ENetProtocol@@@Z 0056d140 f   protocol.obj
 0001:0016c2a0       ?enet_protocol_handle_throttle_configure@@YAHPAU_ENetHost@@PAU_ENetPeer@@PBT_ENetProtocol@@@Z 0056d2a0 f   protocol.obj
 0001:0016c300       ?enet_protocol_handle_disconnect@@YAHPAU_ENetHost@@PAU_ENetPeer@@PBT_ENetProtocol@@@Z 0056d300 f   protocol.obj
 0001:0016c3f0       ?enet_protocol_handle_acknowledge@@YAHPAU_ENetHost@@PAU_ENetEvent@@PAU_ENetPeer@@PBT_ENetProtocol@@@Z 0056d3f0 f   protocol.obj
 0001:0016c760       ?enet_protocol_notify_connect@@YAXPAU_ENetHost@@PAU_ENetPeer@@PAU_ENetEvent@@@Z 0056d760 f   protocol.obj
 0001:0016c7d0       ?enet_protocol_remove_sent_reliable_command@@YA?AW4_ENetProtocolCommand@@PAU_ENetPeer@@GE@Z 0056d7d0 f   protocol.obj
 0001:0016ca20       ?enet_protocol_handle_verify_connect@@YAHPAU_ENetHost@@PAU_ENetEvent@@PAU_ENetPeer@@PBT_ENetProtocol@@@Z 0056da20 f   protocol.obj
 0001:0016e1b0       ?enet_symbol_rescale@@YAGPAU_ENetSymbol@@@Z 0056f1b0 f   compress.obj
 0001:00170790       _SDL_InitDynamicAPI        00571790 f   libSDL2:SDL_dynapi.o
 0001:00170870       _SDL_JoystickFromInstanceID_DEFAULT 00571870 f   libSDL2:SDL_dynapi.o
 0001:00170890       _SDL_GameControllerFromInstanceID_DEFAULT 00571890 f   libSDL2:SDL_dynapi.o
 0001:001708b0       _SDL_JoystickCurrentPowerLevel_DEFAULT 005718b0 f   libSDL2:SDL_dynapi.o
 0001:001708d0       _SDL_GetDisplayDPI_DEFAULT 005718d0 f   libSDL2:SDL_dynapi.o
 0001:00170910       _SDL_SetWindowsMessageHook_DEFAULT 00571910 f   libSDL2:SDL_dynapi.o
 0001:00170930       _SDL_GetQueuedAudioSize_DEFAULT 00571930 f   libSDL2:SDL_dynapi.o
 0001:00170950       _SDL_QueueAudio_DEFAULT    00571950 f   libSDL2:SDL_dynapi.o
 0001:00170980       _SDL_GetGlobalMouseState_DEFAULT 00571980 f   libSDL2:SDL_dynapi.o
 0001:001709a0       _SDL_SetWindowHitTest_DEFAULT 005719a0 f   libSDL2:SDL_dynapi.o
 0001:001709d0       _SDL_CaptureMouse_DEFAULT  005719d0 f   libSDL2:SDL_dynapi.o
 0001:001709f0       _SDL_tanf_DEFAULT          005719f0 f   libSDL2:SDL_dynapi.o
 0001:00170a20       _SDL_tan_DEFAULT           00571a20 f   libSDL2:SDL_dynapi.o
 0001:00170a50       _SDL_sqrtf_DEFAULT         00571a50 f   libSDL2:SDL_dynapi.o
 0001:00170a80       _SDL_WarpMouseGlobal_DEFAULT 00571a80 f   libSDL2:SDL_dynapi.o
 0001:00170aa0       _SDL_RenderIsClipEnabled_DEFAULT 00571aa0 f   libSDL2:SDL_dynapi.o
 0001:00170ac0       _SDL_DXGIGetOutputInfo_DEFAULT 00571ac0 f   libSDL2:SDL_dynapi.o
 0001:00170af0       _SDL_GetAssertionHandler_DEFAULT 00571af0 f   libSDL2:SDL_dynapi.o
 0001:00170b10       _SDL_GameControllerAddMappingsFromRW_DEFAULT 00571b10 f   libSDL2:SDL_dynapi.o
 0001:00170b30       _SDL_vsscanf_DEFAULT       00571b30 f   libSDL2:SDL_dynapi.o
 0001:00170b60       _SDL_GL_SwapWindow_DEFAULT 00571b60 f   libSDL2:SDL_dynapi.o
 0001:00170b80       _SDL_GL_SetSwapInterval_DEFAULT 00571b80 f   libSDL2:SDL_dynapi.o
 0001:00170ba0       _SDL_GL_GetDrawableSize_DEFAULT 00571ba0 f   libSDL2:SDL_dynapi.o
 0001:00170bd0       _SDL_GL_MakeCurrent_DEFAULT 00571bd0 f   libSDL2:SDL_dynapi.o
 0001:00170bf0       _SDL_GL_CreateContext_DEFAULT 00571bf0 f   libSDL2:SDL_dynapi.o
 0001:00170c10       _SDL_GL_GetAttribute_DEFAULT 00571c10 f   libSDL2:SDL_dynapi.o
 0001:00170c30       _SDL_GL_SetAttribute_DEFAULT 00571c30 f   libSDL2:SDL_dynapi.o
 0001:00170c50       _SDL_GL_ExtensionSupported_DEFAULT 00571c50 f   libSDL2:SDL_dynapi.o
 0001:00170c70       _SDL_GL_GetProcAddress_DEFAULT 00571c70 f   libSDL2:SDL_dynapi.o
 0001:00170c90       _SDL_GL_LoadLibrary_DEFAULT 00571c90 f   libSDL2:SDL_dynapi.o
 0001:00170cb0       _SDL_GetWindowGammaRamp_DEFAULT 00571cb0 f   libSDL2:SDL_dynapi.o
 0001:00170cf0       _SDL_SetWindowGammaRamp_DEFAULT 00571cf0 f   libSDL2:SDL_dynapi.o
 0001:00170d30       _SDL_GetWindowBrightness_DEFAULT 00571d30 f   libSDL2:SDL_dynapi.o
 0001:00170d50       _SDL_SetWindowBrightness_DEFAULT 00571d50 f   libSDL2:SDL_dynapi.o
 0001:00170d80       _SDL_GetWindowGrab_DEFAULT 00571d80 f   libSDL2:SDL_dynapi.o
 0001:00170da0       _SDL_SetWindowGrab_DEFAULT 00571da0 f   libSDL2:SDL_dynapi.o
 0001:00170dc0       _SDL_UpdateWindowSurfaceRects_DEFAULT 00571dc0 f   libSDL2:SDL_dynapi.o
 0001:00170df0       _SDL_UpdateWindowSurface_DEFAULT 00571df0 f   libSDL2:SDL_dynapi.o
 0001:00170e10       _SDL_GetWindowSurface_DEFAULT 00571e10 f   libSDL2:SDL_dynapi.o
 0001:00170e30       _SDL_SetWindowFullscreen_DEFAULT 00571e30 f   libSDL2:SDL_dynapi.o
 0001:00170e50       _SDL_SetWindowBordered_DEFAULT 00571e50 f   libSDL2:SDL_dynapi.o
 0001:00170e70       _SDL_GetWindowMaximumSize_DEFAULT 00571e70 f   libSDL2:SDL_dynapi.o
 0001:00170ea0       _SDL_SetWindowMaximumSize_DEFAULT 00571ea0 f   libSDL2:SDL_dynapi.o
 0001:00170ed0       _SDL_GetWindowMinimumSize_DEFAULT 00571ed0 f   libSDL2:SDL_dynapi.o
 0001:00170f00       _SDL_SetWindowMinimumSize_DEFAULT 00571f00 f   libSDL2:SDL_dynapi.o
 0001:00170f30       _SDL_GetWindowSize_DEFAULT 00571f30 f   libSDL2:SDL_dynapi.o
 0001:00170f60       _SDL_SetWindowSize_DEFAULT 00571f60 f   libSDL2:SDL_dynapi.o
 0001:00170f90       _SDL_GetWindowPosition_DEFAULT 00571f90 f   libSDL2:SDL_dynapi.o
 0001:00170fc0       _SDL_SetWindowPosition_DEFAULT 00571fc0 f   libSDL2:SDL_dynapi.o
 0001:00170ff0       _SDL_GetWindowData_DEFAULT 00571ff0 f   libSDL2:SDL_dynapi.o
 0001:00171010       _SDL_SetWindowData_DEFAULT 00572010 f   libSDL2:SDL_dynapi.o
 0001:00171040       _SDL_SetWindowIcon_DEFAULT 00572040 f   libSDL2:SDL_dynapi.o
 0001:00171060       _SDL_GetWindowTitle_DEFAULT 00572060 f   libSDL2:SDL_dynapi.o
 0001:00171080       _SDL_SetWindowTitle_DEFAULT 00572080 f   libSDL2:SDL_dynapi.o
 0001:001710a0       _SDL_GetWindowFlags_DEFAULT 005720a0 f   libSDL2:SDL_dynapi.o
 0001:001710c0       _SDL_GetWindowFromID_DEFAULT 005720c0 f   libSDL2:SDL_dynapi.o
 0001:001710e0       _SDL_GetWindowID_DEFAULT   005720e0 f   libSDL2:SDL_dynapi.o
 0001:00171100       _SDL_CreateWindowFrom_DEFAULT 00572100 f   libSDL2:SDL_dynapi.o
 0001:00171120       _SDL_CreateWindow_DEFAULT  00572120 f   libSDL2:SDL_dynapi.o
 0001:00171180       _SDL_GetWindowPixelFormat_DEFAULT 00572180 f   libSDL2:SDL_dynapi.o
 0001:001711a0       _SDL_GetWindowDisplayMode_DEFAULT 005721a0 f   libSDL2:SDL_dynapi.o
 0001:001711c0       _SDL_SetWindowDisplayMode_DEFAULT 005721c0 f   libSDL2:SDL_dynapi.o
 0001:001711e0       _SDL_GetWindowDisplayIndex_DEFAULT 005721e0 f   libSDL2:SDL_dynapi.o
 0001:00171200       _SDL_GetClosestDisplayMode_DEFAULT 00572200 f   libSDL2:SDL_dynapi.o
 0001:00171230       _SDL_GetCurrentDisplayMode_DEFAULT 00572230 f   libSDL2:SDL_dynapi.o
 0001:00171250       _SDL_GetDesktopDisplayMode_DEFAULT 00572250 f   libSDL2:SDL_dynapi.o
 0001:00171270       _SDL_GetDisplayMode_DEFAULT 00572270 f   libSDL2:SDL_dynapi.o
 0001:001712a0       _SDL_GetNumDisplayModes_DEFAULT 005722a0 f   libSDL2:SDL_dynapi.o
 0001:001712c0       _SDL_GetDisplayBounds_DEFAULT 005722c0 f   libSDL2:SDL_dynapi.o
 0001:001712e0       _SDL_GetDisplayName_DEFAULT 005722e0 f   libSDL2:SDL_dynapi.o
 0001:00171300       _SDL_GetNumVideoDisplays_DEFAULT 00572300 f   libSDL2:SDL_dynapi.o
 0001:00171310       _SDL_VideoInit_DEFAULT     00572310 f   libSDL2:SDL_dynapi.o
 0001:00171330       _SDL_GetVideoDriver_DEFAULT 00572330 f   libSDL2:SDL_dynapi.o
 0001:00171350       _SDL_GetTouchFinger_DEFAULT 00572350 f   libSDL2:SDL_dynapi.o
 0001:00171380       _SDL_GetNumTouchFingers_DEFAULT 00572380 f   libSDL2:SDL_dynapi.o
 0001:001713a0       _SDL_GetTouchDevice_DEFAULT 005723a0 f   libSDL2:SDL_dynapi.o
 0001:001713c0       _SDL_RemoveTimer_DEFAULT   005723c0 f   libSDL2:SDL_dynapi.o
 0001:001713e0       _SDL_AddTimer_DEFAULT      005723e0 f   libSDL2:SDL_dynapi.o
 0001:00171410       _SDL_GetPerformanceFrequency_DEFAULT 00572410 f   libSDL2:SDL_dynapi.o
 0001:00171420       _SDL_GetPerformanceCounter_DEFAULT 00572420 f   libSDL2:SDL_dynapi.o
 0001:00171430       _SDL_GetTicks_DEFAULT      00572430 f   libSDL2:SDL_dynapi.o
 0001:00171440       _SDL_TLSSet_DEFAULT        00572440 f   libSDL2:SDL_dynapi.o
 0001:00171470       _SDL_TLSGet_DEFAULT        00572470 f   libSDL2:SDL_dynapi.o
 0001:00171490       _SDL_WaitThread_DEFAULT    00572490 f   libSDL2:SDL_dynapi.o
 0001:001714b0       _SDL_SetThreadPriority_DEFAULT 005724b0 f   libSDL2:SDL_dynapi.o
 0001:001714d0       _SDL_GetThreadID_DEFAULT   005724d0 f   libSDL2:SDL_dynapi.o
 0001:001714f0       _SDL_GetThreadName_DEFAULT 005724f0 f   libSDL2:SDL_dynapi.o
 0001:00171510       _SDL_GetWindowWMInfo_DEFAULT 00572510 f   libSDL2:SDL_dynapi.o
 0001:00171530       _SDL_LowerBlitScaled_DEFAULT 00572530 f   libSDL2:SDL_dynapi.o
 0001:00171570       _SDL_UpperBlitScaled_DEFAULT 00572570 f   libSDL2:SDL_dynapi.o
 0001:001715b0       _SDL_SoftStretch_DEFAULT   005725b0 f   libSDL2:SDL_dynapi.o
 0001:001715f0       _SDL_LowerBlit_DEFAULT     005725f0 f   libSDL2:SDL_dynapi.o
 0001:00171630       _SDL_UpperBlit_DEFAULT     00572630 f   libSDL2:SDL_dynapi.o
 0001:00171670       _SDL_FillRects_DEFAULT     00572670 f   libSDL2:SDL_dynapi.o
 0001:001716b0       _SDL_FillRect_DEFAULT      005726b0 f   libSDL2:SDL_dynapi.o
 0001:001716e0       _SDL_ConvertPixels_DEFAULT 005726e0 f   libSDL2:SDL_dynapi.o
 0001:00171760       _SDL_ConvertSurfaceFormat_DEFAULT 00572760 f   libSDL2:SDL_dynapi.o
 0001:00171790       _SDL_ConvertSurface_DEFAULT 00572790 f   libSDL2:SDL_dynapi.o
 0001:001717c0       _SDL_GetClipRect_DEFAULT   005727c0 f   libSDL2:SDL_dynapi.o
 0001:001717e0       _SDL_SetClipRect_DEFAULT   005727e0 f   libSDL2:SDL_dynapi.o
 0001:00171800       _SDL_GetSurfaceBlendMode_DEFAULT 00572800 f   libSDL2:SDL_dynapi.o
 0001:00171820       _SDL_SetSurfaceBlendMode_DEFAULT 00572820 f   libSDL2:SDL_dynapi.o
 0001:00171840       _SDL_GetSurfaceAlphaMod_DEFAULT 00572840 f   libSDL2:SDL_dynapi.o
 0001:00171860       _SDL_SetSurfaceAlphaMod_DEFAULT 00572860 f   libSDL2:SDL_dynapi.o
 0001:00171890       _SDL_GetSurfaceColorMod_DEFAULT 00572890 f   libSDL2:SDL_dynapi.o
 0001:001718d0       _SDL_SetSurfaceColorMod_DEFAULT 005728d0 f   libSDL2:SDL_dynapi.o
 0001:00171920       _SDL_GetColorKey_DEFAULT   00572920 f   libSDL2:SDL_dynapi.o
 0001:00171940       _SDL_SetColorKey_DEFAULT   00572940 f   libSDL2:SDL_dynapi.o
 0001:00171970       _SDL_SetSurfaceRLE_DEFAULT 00572970 f   libSDL2:SDL_dynapi.o
 0001:00171990       _SDL_SaveBMP_RW_DEFAULT    00572990 f   libSDL2:SDL_dynapi.o
 0001:001719c0       _SDL_LoadBMP_RW_DEFAULT    005729c0 f   libSDL2:SDL_dynapi.o
 0001:001719e0       _SDL_LockSurface_DEFAULT   005729e0 f   libSDL2:SDL_dynapi.o
 0001:00171a00       _SDL_SetSurfacePalette_DEFAULT 00572a00 f   libSDL2:SDL_dynapi.o
 0001:00171a20       _SDL_CreateRGBSurfaceFrom_DEFAULT 00572a20 f   libSDL2:SDL_dynapi.o
 0001:00171ab0       _SDL_CreateRGBSurface_DEFAULT 00572ab0 f   libSDL2:SDL_dynapi.o
 0001:00171b30       _SDL_iconv_string_DEFAULT  00572b30 f   libSDL2:SDL_dynapi.o
 0001:00171b70       _SDL_iconv_DEFAULT         00572b70 f   libSDL2:SDL_dynapi.o
 0001:00171bc0       _SDL_iconv_close_DEFAULT   00572bc0 f   libSDL2:SDL_dynapi.o
 0001:00171be0       _SDL_iconv_open_DEFAULT    00572be0 f   libSDL2:SDL_dynapi.o
 0001:00171c00       _SDL_sqrt_DEFAULT          00572c00 f   libSDL2:SDL_dynapi.o
 0001:00171c30       _SDL_sinf_DEFAULT          00572c30 f   libSDL2:SDL_dynapi.o
 0001:00171c60       _SDL_sin_DEFAULT           00572c60 f   libSDL2:SDL_dynapi.o
 0001:00171c90       _SDL_scalbn_DEFAULT        00572c90 f   libSDL2:SDL_dynapi.o
 0001:00171cc0       _SDL_pow_DEFAULT           00572cc0 f   libSDL2:SDL_dynapi.o
 0001:00171cf0       _SDL_log_DEFAULT           00572cf0 f   libSDL2:SDL_dynapi.o
 0001:00171d20       _SDL_floor_DEFAULT         00572d20 f   libSDL2:SDL_dynapi.o
 0001:00171d50       _SDL_fabs_DEFAULT          00572d50 f   libSDL2:SDL_dynapi.o
 0001:00171d80       _SDL_cosf_DEFAULT          00572d80 f   libSDL2:SDL_dynapi.o
 0001:00171db0       _SDL_cos_DEFAULT           00572db0 f   libSDL2:SDL_dynapi.o
 0001:00171de0       _SDL_copysign_DEFAULT      00572de0 f   libSDL2:SDL_dynapi.o
 0001:00171e10       _SDL_ceil_DEFAULT          00572e10 f   libSDL2:SDL_dynapi.o
 0001:00171e40       _SDL_atan2_DEFAULT         00572e40 f   libSDL2:SDL_dynapi.o
 0001:00171e70       _SDL_atan_DEFAULT          00572e70 f   libSDL2:SDL_dynapi.o
 0001:00171ea0       _SDL_asin_DEFAULT          00572ea0 f   libSDL2:SDL_dynapi.o
 0001:00171ed0       _SDL_acos_DEFAULT          00572ed0 f   libSDL2:SDL_dynapi.o
 0001:00171f00       _SDL_vsnprintf_DEFAULT     00572f00 f   libSDL2:SDL_dynapi.o
 0001:00171f40       _SDL_strncasecmp_DEFAULT   00572f40 f   libSDL2:SDL_dynapi.o
 0001:00171f70       _SDL_strcasecmp_DEFAULT    00572f70 f   libSDL2:SDL_dynapi.o
 0001:00171f90       _SDL_strncmp_DEFAULT       00572f90 f   libSDL2:SDL_dynapi.o
 0001:00171fc0       _SDL_strcmp_DEFAULT        00572fc0 f   libSDL2:SDL_dynapi.o
 0001:00171fe0       _SDL_strtod_DEFAULT        00572fe0 f   libSDL2:SDL_dynapi.o
 0001:00172010       _SDL_strtoull_DEFAULT      00573010 f   libSDL2:SDL_dynapi.o
 0001:00172040       _SDL_strtoll_DEFAULT       00573040 f   libSDL2:SDL_dynapi.o
 0001:00172070       _SDL_strtoul_DEFAULT       00573070 f   libSDL2:SDL_dynapi.o
 0001:001720a0       _SDL_strtol_DEFAULT        005730a0 f   libSDL2:SDL_dynapi.o
 0001:001720d0       _SDL_atof_DEFAULT          005730d0 f   libSDL2:SDL_dynapi.o
 0001:001720f0       _SDL_atoi_DEFAULT          005730f0 f   libSDL2:SDL_dynapi.o
 0001:00172110       _SDL_ulltoa_DEFAULT        00573110 f   libSDL2:SDL_dynapi.o
 0001:00172150       _SDL_lltoa_DEFAULT         00573150 f   libSDL2:SDL_dynapi.o
 0001:00172190       _SDL_ultoa_DEFAULT         00573190 f   libSDL2:SDL_dynapi.o
 0001:001721c0       _SDL_ltoa_DEFAULT          005731c0 f   libSDL2:SDL_dynapi.o
 0001:001721f0       _SDL_uitoa_DEFAULT         005731f0 f   libSDL2:SDL_dynapi.o
 0001:00172220       _SDL_itoa_DEFAULT          00573220 f   libSDL2:SDL_dynapi.o
 0001:00172250       _SDL_strstr_DEFAULT        00573250 f   libSDL2:SDL_dynapi.o
 0001:00172270       _SDL_strrchr_DEFAULT       00573270 f   libSDL2:SDL_dynapi.o
 0001:00172290       _SDL_strchr_DEFAULT        00573290 f   libSDL2:SDL_dynapi.o
 0001:001722b0       _SDL_strlwr_DEFAULT        005732b0 f   libSDL2:SDL_dynapi.o
 0001:001722d0       _SDL_strupr_DEFAULT        005732d0 f   libSDL2:SDL_dynapi.o
 0001:001722f0       _SDL_strrev_DEFAULT        005732f0 f   libSDL2:SDL_dynapi.o
 0001:00172310       _SDL_strdup_DEFAULT        00573310 f   libSDL2:SDL_dynapi.o
 0001:00172330       _SDL_strlcat_DEFAULT       00573330 f   libSDL2:SDL_dynapi.o
 0001:00172360       _SDL_utf8strlcpy_DEFAULT   00573360 f   libSDL2:SDL_dynapi.o
 0001:00172390       _SDL_strlcpy_DEFAULT       00573390 f   libSDL2:SDL_dynapi.o
 0001:001723c0       _SDL_strlen_DEFAULT        005733c0 f   libSDL2:SDL_dynapi.o
 0001:001723e0       _SDL_wcslcat_DEFAULT       005733e0 f   libSDL2:SDL_dynapi.o
 0001:00172410       _SDL_wcslcpy_DEFAULT       00573410 f   libSDL2:SDL_dynapi.o
 0001:00172440       _SDL_wcslen_DEFAULT        00573440 f   libSDL2:SDL_dynapi.o
 0001:00172460       _SDL_memcmp_DEFAULT        00573460 f   libSDL2:SDL_dynapi.o
 0001:00172490       _SDL_memmove_DEFAULT       00573490 f   libSDL2:SDL_dynapi.o
 0001:001724c0       _SDL_memcpy_DEFAULT        005734c0 f   libSDL2:SDL_dynapi.o
 0001:001724f0       _SDL_memset_DEFAULT        005734f0 f   libSDL2:SDL_dynapi.o
 0001:00172520       _SDL_tolower_DEFAULT       00573520 f   libSDL2:SDL_dynapi.o
 0001:00172540       _SDL_toupper_DEFAULT       00573540 f   libSDL2:SDL_dynapi.o
 0001:00172560       _SDL_isspace_DEFAULT       00573560 f   libSDL2:SDL_dynapi.o
 0001:00172580       _SDL_isdigit_DEFAULT       00573580 f   libSDL2:SDL_dynapi.o
 0001:001725a0       _SDL_abs_DEFAULT           005735a0 f   libSDL2:SDL_dynapi.o
 0001:001725c0       _SDL_qsort_DEFAULT         005735c0 f   libSDL2:SDL_dynapi.o
 0001:00172600       _SDL_setenv_DEFAULT        00573600 f   libSDL2:SDL_dynapi.o
 0001:00172630       _SDL_getenv_DEFAULT        00573630 f   libSDL2:SDL_dynapi.o
 0001:00172650       _SDL_realloc_DEFAULT       00573650 f   libSDL2:SDL_dynapi.o
 0001:00172670       _SDL_calloc_DEFAULT        00573670 f   libSDL2:SDL_dynapi.o
 0001:00172690       _SDL_malloc_DEFAULT        00573690 f   libSDL2:SDL_dynapi.o
 0001:001726b0       _SDL_GetShapedWindowMode_DEFAULT 005736b0 f   libSDL2:SDL_dynapi.o
 0001:001726d0       _SDL_SetWindowShape_DEFAULT 005736d0 f   libSDL2:SDL_dynapi.o
 0001:00172700       _SDL_IsShapedWindow_DEFAULT 00573700 f   libSDL2:SDL_dynapi.o
 0001:00172720       _SDL_CreateShapedWindow_DEFAULT 00573720 f   libSDL2:SDL_dynapi.o
 0001:00172780       _SDL_WriteBE64_DEFAULT     00573780 f   libSDL2:SDL_dynapi.o
 0001:001727b0       _SDL_WriteLE64_DEFAULT     005737b0 f   libSDL2:SDL_dynapi.o
 0001:001727e0       _SDL_WriteBE32_DEFAULT     005737e0 f   libSDL2:SDL_dynapi.o
 0001:00172800       _SDL_WriteLE32_DEFAULT     00573800 f   libSDL2:SDL_dynapi.o
 0001:00172820       _SDL_WriteBE16_DEFAULT     00573820 f   libSDL2:SDL_dynapi.o
 0001:00172850       _SDL_WriteLE16_DEFAULT     00573850 f   libSDL2:SDL_dynapi.o
 0001:00172880       _SDL_WriteU8_DEFAULT       00573880 f   libSDL2:SDL_dynapi.o
 0001:001728b0       _SDL_ReadBE64_DEFAULT      005738b0 f   libSDL2:SDL_dynapi.o
 0001:001728d0       _SDL_ReadLE64_DEFAULT      005738d0 f   libSDL2:SDL_dynapi.o
 0001:001728f0       _SDL_ReadBE32_DEFAULT      005738f0 f   libSDL2:SDL_dynapi.o
 0001:00172910       _SDL_ReadLE32_DEFAULT      00573910 f   libSDL2:SDL_dynapi.o
 0001:00172930       _SDL_ReadBE16_DEFAULT      00573930 f   libSDL2:SDL_dynapi.o
 0001:00172950       _SDL_ReadLE16_DEFAULT      00573950 f   libSDL2:SDL_dynapi.o
 0001:00172970       _SDL_ReadU8_DEFAULT        00573970 f   libSDL2:SDL_dynapi.o
 0001:00172990       _SDL_FreeRW_DEFAULT        00573990 f   libSDL2:SDL_dynapi.o
 0001:001729b0       _SDL_RWFromConstMem_DEFAULT 005739b0 f   libSDL2:SDL_dynapi.o
 0001:001729d0       _SDL_RWFromMem_DEFAULT     005739d0 f   libSDL2:SDL_dynapi.o
 0001:001729f0       _SDL_RWFromFile_DEFAULT    005739f0 f   libSDL2:SDL_dynapi.o
 0001:00172a10       _SDL_GL_UnbindTexture_DEFAULT 00573a10 f   libSDL2:SDL_dynapi.o
 0001:00172a30       _SDL_GL_BindTexture_DEFAULT 00573a30 f   libSDL2:SDL_dynapi.o
 0001:00172a60       _SDL_RenderReadPixels_DEFAULT 00573a60 f   libSDL2:SDL_dynapi.o
 0001:00172ab0       _SDL_RenderCopyEx_DEFAULT  00573ab0 f   libSDL2:SDL_dynapi.o
 0001:00172b20       _SDL_RenderCopy_DEFAULT    00573b20 f   libSDL2:SDL_dynapi.o
 0001:00172b60       _SDL_RenderFillRects_DEFAULT 00573b60 f   libSDL2:SDL_dynapi.o
 0001:00172b90       _SDL_RenderFillRect_DEFAULT 00573b90 f   libSDL2:SDL_dynapi.o
 0001:00172bb0       _SDL_RenderDrawRects_DEFAULT 00573bb0 f   libSDL2:SDL_dynapi.o
 0001:00172be0       _SDL_RenderDrawRect_DEFAULT 00573be0 f   libSDL2:SDL_dynapi.o
 0001:00172c00       _SDL_RenderDrawLines_DEFAULT 00573c00 f   libSDL2:SDL_dynapi.o
 0001:00172c30       _SDL_RenderDrawLine_DEFAULT 00573c30 f   libSDL2:SDL_dynapi.o
 0001:00172c80       _SDL_RenderDrawPoints_DEFAULT 00573c80 f   libSDL2:SDL_dynapi.o
 0001:00172cb0       _SDL_RenderDrawPoint_DEFAULT 00573cb0 f   libSDL2:SDL_dynapi.o
 0001:00172ce0       _SDL_RenderClear_DEFAULT   00573ce0 f   libSDL2:SDL_dynapi.o
 0001:00172d00       _SDL_GetRenderDrawBlendMode_DEFAULT 00573d00 f   libSDL2:SDL_dynapi.o
 0001:00172d20       _SDL_SetRenderDrawBlendMode_DEFAULT 00573d20 f   libSDL2:SDL_dynapi.o
 0001:00172d40       _SDL_GetRenderDrawColor_DEFAULT 00573d40 f   libSDL2:SDL_dynapi.o
 0001:00172d90       _SDL_SetRenderDrawColor_DEFAULT 00573d90 f   libSDL2:SDL_dynapi.o
 0001:00172df0       _SDL_RenderGetScale_DEFAULT 00573df0 f   libSDL2:SDL_dynapi.o
 0001:00172e20       _SDL_RenderSetScale_DEFAULT 00573e20 f   libSDL2:SDL_dynapi.o
 0001:00172e70       _SDL_RenderGetClipRect_DEFAULT 00573e70 f   libSDL2:SDL_dynapi.o
 0001:00172e90       _SDL_RenderSetClipRect_DEFAULT 00573e90 f   libSDL2:SDL_dynapi.o
 0001:00172eb0       _SDL_RenderGetViewport_DEFAULT 00573eb0 f   libSDL2:SDL_dynapi.o
 0001:00172ed0       _SDL_RenderSetViewport_DEFAULT 00573ed0 f   libSDL2:SDL_dynapi.o
 0001:00172ef0       _SDL_RenderGetLogicalSize_DEFAULT 00573ef0 f   libSDL2:SDL_dynapi.o
 0001:00172f20       _SDL_RenderSetLogicalSize_DEFAULT 00573f20 f   libSDL2:SDL_dynapi.o
 0001:00172f50       _SDL_GetRenderTarget_DEFAULT 00573f50 f   libSDL2:SDL_dynapi.o
 0001:00172f70       _SDL_SetRenderTarget_DEFAULT 00573f70 f   libSDL2:SDL_dynapi.o
 0001:00172f90       _SDL_RenderTargetSupported_DEFAULT 00573f90 f   libSDL2:SDL_dynapi.o
 0001:00172fb0       _SDL_LockTexture_DEFAULT   00573fb0 f   libSDL2:SDL_dynapi.o
 0001:00172ff0       _SDL_UpdateYUVTexture_DEFAULT 00573ff0 f   libSDL2:SDL_dynapi.o
 0001:00173070       _SDL_UpdateTexture_DEFAULT 00574070 f   libSDL2:SDL_dynapi.o
 0001:001730b0       _SDL_GetTextureBlendMode_DEFAULT 005740b0 f   libSDL2:SDL_dynapi.o
 0001:001730d0       _SDL_SetTextureBlendMode_DEFAULT 005740d0 f   libSDL2:SDL_dynapi.o
 0001:001730f0       _SDL_GetTextureAlphaMod_DEFAULT 005740f0 f   libSDL2:SDL_dynapi.o
 0001:00173110       _SDL_SetTextureAlphaMod_DEFAULT 00574110 f   libSDL2:SDL_dynapi.o
 0001:00173140       _SDL_GetTextureColorMod_DEFAULT 00574140 f   libSDL2:SDL_dynapi.o
 0001:00173180       _SDL_SetTextureColorMod_DEFAULT 00574180 f   libSDL2:SDL_dynapi.o
 0001:001731d0       _SDL_QueryTexture_DEFAULT  005741d0 f   libSDL2:SDL_dynapi.o
 0001:00173220       _SDL_CreateTextureFromSurface_DEFAULT 00574220 f   libSDL2:SDL_dynapi.o
 0001:00173240       _SDL_CreateTexture_DEFAULT 00574240 f   libSDL2:SDL_dynapi.o
 0001:00173290       _SDL_GetRendererOutputSize_DEFAULT 00574290 f   libSDL2:SDL_dynapi.o
 0001:001732c0       _SDL_GetRendererInfo_DEFAULT 005742c0 f   libSDL2:SDL_dynapi.o
 0001:001732e0       _SDL_GetRenderer_DEFAULT   005742e0 f   libSDL2:SDL_dynapi.o
 0001:00173300       _SDL_CreateSoftwareRenderer_DEFAULT 00574300 f   libSDL2:SDL_dynapi.o
 0001:00173320       _SDL_CreateRenderer_DEFAULT 00574320 f   libSDL2:SDL_dynapi.o
 0001:00173350       _SDL_CreateWindowAndRenderer_DEFAULT 00574350 f   libSDL2:SDL_dynapi.o
 0001:001733a0       _SDL_GetRenderDriverInfo_DEFAULT 005743a0 f   libSDL2:SDL_dynapi.o
 0001:001733c0       _SDL_IntersectRectAndLine_DEFAULT 005743c0 f   libSDL2:SDL_dynapi.o
 0001:00173410       _SDL_EnclosePoints_DEFAULT 00574410 f   libSDL2:SDL_dynapi.o
 0001:00173450       _SDL_UnionRect_DEFAULT     00574450 f   libSDL2:SDL_dynapi.o
 0001:00173480       _SDL_IntersectRect_DEFAULT 00574480 f   libSDL2:SDL_dynapi.o
 0001:001734b0       _SDL_HasIntersection_DEFAULT 005744b0 f   libSDL2:SDL_dynapi.o
 0001:001734d0       _SDL_GetPowerInfo_DEFAULT  005744d0 f   libSDL2:SDL_dynapi.o
 0001:001734f0       _SDL_GetPlatform_DEFAULT   005744f0 f   libSDL2:SDL_dynapi.o
 0001:00173500       _SDL_CalculateGammaRamp_DEFAULT 00574500 f   libSDL2:SDL_dynapi.o
 0001:00173530       _SDL_GetRGBA_DEFAULT       00574530 f   libSDL2:SDL_dynapi.o
 0001:00173590       _SDL_GetRGB_DEFAULT        00574590 f   libSDL2:SDL_dynapi.o
 0001:001735e0       _SDL_MapRGBA_DEFAULT       005745e0 f   libSDL2:SDL_dynapi.o
 0001:00173640       _SDL_MapRGB_DEFAULT        00574640 f   libSDL2:SDL_dynapi.o
 0001:00173690       _SDL_SetPaletteColors_DEFAULT 00574690 f   libSDL2:SDL_dynapi.o
 0001:001736d0       _SDL_SetPixelFormatPalette_DEFAULT 005746d0 f   libSDL2:SDL_dynapi.o
 0001:001736f0       _SDL_AllocPalette_DEFAULT  005746f0 f   libSDL2:SDL_dynapi.o
 0001:00173710       _SDL_FreeFormat_DEFAULT    00574710 f   libSDL2:SDL_dynapi.o
 0001:00173730       _SDL_AllocFormat_DEFAULT   00574730 f   libSDL2:SDL_dynapi.o
 0001:00173750       _SDL_MasksToPixelFormatEnum_DEFAULT 00574750 f   libSDL2:SDL_dynapi.o
 0001:001737a0       _SDL_PixelFormatEnumToMasks_DEFAULT 005747a0 f   libSDL2:SDL_dynapi.o
 0001:00173800       _SDL_GetPixelFormatName_DEFAULT 00574800 f   libSDL2:SDL_dynapi.o
 0001:00173820       _SDL_CondWaitTimeout_DEFAULT 00574820 f   libSDL2:SDL_dynapi.o
 0001:00173850       _SDL_CondWait_DEFAULT      00574850 f   libSDL2:SDL_dynapi.o
 0001:00173870       _SDL_CondBroadcast_DEFAULT 00574870 f   libSDL2:SDL_dynapi.o
 0001:00173890       _SDL_CondSignal_DEFAULT    00574890 f   libSDL2:SDL_dynapi.o
 0001:001738b0       _SDL_DestroyCond_DEFAULT   005748b0 f   libSDL2:SDL_dynapi.o
 0001:001738d0       _SDL_SemValue_DEFAULT      005748d0 f   libSDL2:SDL_dynapi.o
 0001:001738f0       _SDL_SemPost_DEFAULT       005748f0 f   libSDL2:SDL_dynapi.o
 0001:00173910       _SDL_SemWaitTimeout_DEFAULT 00574910 f   libSDL2:SDL_dynapi.o
 0001:00173930       _SDL_SemTryWait_DEFAULT    00574930 f   libSDL2:SDL_dynapi.o
 0001:00173950       _SDL_SemWait_DEFAULT       00574950 f   libSDL2:SDL_dynapi.o
 0001:00173970       _SDL_DestroySemaphore_DEFAULT 00574970 f   libSDL2:SDL_dynapi.o
 0001:00173990       _SDL_CreateSemaphore_DEFAULT 00574990 f   libSDL2:SDL_dynapi.o
 0001:001739b0       _SDL_UnlockMutex_DEFAULT   005749b0 f   libSDL2:SDL_dynapi.o
 0001:001739d0       _SDL_TryLockMutex_DEFAULT  005749d0 f   libSDL2:SDL_dynapi.o
 0001:001739f0       _SDL_LockMutex_DEFAULT     005749f0 f   libSDL2:SDL_dynapi.o
 0001:00173a10       _SDL_CreateMutex_DEFAULT   00574a10 f   libSDL2:SDL_dynapi.o
 0001:00173a20       _SDL_ShowCursor_DEFAULT    00574a20 f   libSDL2:SDL_dynapi.o
 0001:00173a40       _SDL_CreateSystemCursor_DEFAULT 00574a40 f   libSDL2:SDL_dynapi.o
 0001:00173a60       _SDL_CreateColorCursor_DEFAULT 00574a60 f   libSDL2:SDL_dynapi.o
 0001:00173a90       _SDL_CreateCursor_DEFAULT  00574a90 f   libSDL2:SDL_dynapi.o
 0001:00173af0       _SDL_GetRelativeMouseMode_DEFAULT 00574af0 f   libSDL2:SDL_dynapi.o
 0001:00173b00       _SDL_SetRelativeMouseMode_DEFAULT 00574b00 f   libSDL2:SDL_dynapi.o
 0001:00173b20       _SDL_WarpMouseInWindow_DEFAULT 00574b20 f   libSDL2:SDL_dynapi.o
 0001:00173b50       _SDL_GetRelativeMouseState_DEFAULT 00574b50 f   libSDL2:SDL_dynapi.o
 0001:00173b70       _SDL_GetMouseState_DEFAULT 00574b70 f   libSDL2:SDL_dynapi.o
 0001:00173b90       _SDL_ShowSimpleMessageBox_DEFAULT 00574b90 f   libSDL2:SDL_dynapi.o
 0001:00173bd0       _SDL_ShowMessageBox_DEFAULT 00574bd0 f   libSDL2:SDL_dynapi.o
 0001:00173bf0       _SDL_LogSetOutputFunction_DEFAULT 00574bf0 f   libSDL2:SDL_dynapi.o
 0001:00173c10       _SDL_LogGetOutputFunction_DEFAULT 00574c10 f   libSDL2:SDL_dynapi.o
 0001:00173c30       _SDL_LogMessageV_DEFAULT   00574c30 f   libSDL2:SDL_dynapi.o
 0001:00173c70       _SDL_LogGetPriority_DEFAULT 00574c70 f   libSDL2:SDL_dynapi.o
 0001:00173c90       _SDL_LogSetPriority_DEFAULT 00574c90 f   libSDL2:SDL_dynapi.o
 0001:00173cb0       _SDL_LogSetAllPriority_DEFAULT 00574cb0 f   libSDL2:SDL_dynapi.o
 0001:00173cd0       _SDL_LoadFunction_DEFAULT  00574cd0 f   libSDL2:SDL_dynapi.o
 0001:00173cf0       _SDL_LoadObject_DEFAULT    00574cf0 f   libSDL2:SDL_dynapi.o
 0001:00173d10       _SDL_IsScreenKeyboardShown_DEFAULT 00574d10 f   libSDL2:SDL_dynapi.o
 0001:00173d30       _SDL_HasScreenKeyboardSupport_DEFAULT 00574d30 f   libSDL2:SDL_dynapi.o
 0001:00173d40       _SDL_IsTextInputActive_DEFAULT 00574d40 f   libSDL2:SDL_dynapi.o
 0001:00173d50       _SDL_GetKeyFromName_DEFAULT 00574d50 f   libSDL2:SDL_dynapi.o
 0001:00173d70       _SDL_GetKeyName_DEFAULT    00574d70 f   libSDL2:SDL_dynapi.o
 0001:00173d90       _SDL_GetScancodeFromName_DEFAULT 00574d90 f   libSDL2:SDL_dynapi.o
 0001:00173db0       _SDL_GetScancodeName_DEFAULT 00574db0 f   libSDL2:SDL_dynapi.o
 0001:00173dd0       _SDL_GetScancodeFromKey_DEFAULT 00574dd0 f   libSDL2:SDL_dynapi.o
 0001:00173df0       _SDL_GetKeyFromScancode_DEFAULT 00574df0 f   libSDL2:SDL_dynapi.o
 0001:00173e10       _SDL_SetModState_DEFAULT   00574e10 f   libSDL2:SDL_dynapi.o
 0001:00173e30       _SDL_GetModState_DEFAULT   00574e30 f   libSDL2:SDL_dynapi.o
 0001:00173e40       _SDL_GetKeyboardState_DEFAULT 00574e40 f   libSDL2:SDL_dynapi.o
 0001:00173e60       _SDL_GetKeyboardFocus_DEFAULT 00574e60 f   libSDL2:SDL_dynapi.o
 0001:00173e70       _SDL_JoystickGetButton_DEFAULT 00574e70 f   libSDL2:SDL_dynapi.o
 0001:00173e90       _SDL_JoystickGetBall_DEFAULT 00574e90 f   libSDL2:SDL_dynapi.o
 0001:00173ed0       _SDL_JoystickGetHat_DEFAULT 00574ed0 f   libSDL2:SDL_dynapi.o
 0001:00173ef0       _SDL_JoystickGetAxis_DEFAULT 00574ef0 f   libSDL2:SDL_dynapi.o
 0001:00173f10       _SDL_JoystickEventState_DEFAULT 00574f10 f   libSDL2:SDL_dynapi.o
 0001:00173f30       _SDL_JoystickNumButtons_DEFAULT 00574f30 f   libSDL2:SDL_dynapi.o
 0001:00173f50       _SDL_JoystickNumHats_DEFAULT 00574f50 f   libSDL2:SDL_dynapi.o
 0001:00173f70       _SDL_JoystickNumBalls_DEFAULT 00574f70 f   libSDL2:SDL_dynapi.o
 0001:00173f90       _SDL_JoystickNumAxes_DEFAULT 00574f90 f   libSDL2:SDL_dynapi.o
 0001:00173fb0       _SDL_JoystickInstanceID_DEFAULT 00574fb0 f   libSDL2:SDL_dynapi.o
 0001:00173fd0       _SDL_JoystickGetAttached_DEFAULT 00574fd0 f   libSDL2:SDL_dynapi.o
 0001:00173ff0       _SDL_JoystickGetGUIDFromString_DEFAULT 00574ff0 f   libSDL2:SDL_dynapi.o
 0001:00174020       _SDL_JoystickGetGUIDString_DEFAULT 00575020 f   libSDL2:SDL_dynapi.o
 0001:00174040       _SDL_JoystickGetGUID_DEFAULT 00575040 f   libSDL2:SDL_dynapi.o
 0001:00174070       _SDL_JoystickGetDeviceGUID_DEFAULT 00575070 f   libSDL2:SDL_dynapi.o
 0001:001740a0       _SDL_JoystickName_DEFAULT  005750a0 f   libSDL2:SDL_dynapi.o
 0001:001740c0       _SDL_JoystickOpen_DEFAULT  005750c0 f   libSDL2:SDL_dynapi.o
 0001:001740e0       _SDL_JoystickNameForIndex_DEFAULT 005750e0 f   libSDL2:SDL_dynapi.o
 0001:00174100       _SDL_NumJoysticks_DEFAULT  00575100 f   libSDL2:SDL_dynapi.o
 0001:00174110       _SDL_DelHintCallback_DEFAULT 00575110 f   libSDL2:SDL_dynapi.o
 0001:00174140       _SDL_AddHintCallback_DEFAULT 00575140 f   libSDL2:SDL_dynapi.o
 0001:00174170       _SDL_GetHint_DEFAULT       00575170 f   libSDL2:SDL_dynapi.o
 0001:00174190       _SDL_SetHint_DEFAULT       00575190 f   libSDL2:SDL_dynapi.o
 0001:001741b0       _SDL_SetHintWithPriority_DEFAULT 005751b0 f   libSDL2:SDL_dynapi.o
 0001:001741e0       _SDL_HapticRumbleStop_DEFAULT 005751e0 f   libSDL2:SDL_dynapi.o
 0001:00174200       _SDL_HapticRumblePlay_DEFAULT 00575200 f   libSDL2:SDL_dynapi.o
 0001:00174240       _SDL_HapticRumbleInit_DEFAULT 00575240 f   libSDL2:SDL_dynapi.o
 0001:00174260       _SDL_HapticRumbleSupported_DEFAULT 00575260 f   libSDL2:SDL_dynapi.o
 0001:00174280       _SDL_HapticStopAll_DEFAULT 00575280 f   libSDL2:SDL_dynapi.o
 0001:001742a0       _SDL_HapticUnpause_DEFAULT 005752a0 f   libSDL2:SDL_dynapi.o
 0001:001742c0       _SDL_HapticPause_DEFAULT   005752c0 f   libSDL2:SDL_dynapi.o
 0001:001742e0       _SDL_HapticSetAutocenter_DEFAULT 005752e0 f   libSDL2:SDL_dynapi.o
 0001:00174300       _SDL_HapticSetGain_DEFAULT 00575300 f   libSDL2:SDL_dynapi.o
 0001:00174320       _SDL_HapticGetEffectStatus_DEFAULT 00575320 f   libSDL2:SDL_dynapi.o
 0001:00174340       _SDL_HapticDestroyEffect_DEFAULT 00575340 f   libSDL2:SDL_dynapi.o
 0001:00174360       _SDL_HapticStopEffect_DEFAULT 00575360 f   libSDL2:SDL_dynapi.o
 0001:00174380       _SDL_HapticRunEffect_DEFAULT 00575380 f   libSDL2:SDL_dynapi.o
 0001:001743b0       _SDL_HapticUpdateEffect_DEFAULT 005753b0 f   libSDL2:SDL_dynapi.o
 0001:001743e0       _SDL_HapticNewEffect_DEFAULT 005753e0 f   libSDL2:SDL_dynapi.o
 0001:00174400       _SDL_HapticEffectSupported_DEFAULT 00575400 f   libSDL2:SDL_dynapi.o
 0001:00174420       _SDL_HapticNumAxes_DEFAULT 00575420 f   libSDL2:SDL_dynapi.o
 0001:00174440       _SDL_HapticQuery_DEFAULT   00575440 f   libSDL2:SDL_dynapi.o
 0001:00174460       _SDL_HapticNumEffectsPlaying_DEFAULT 00575460 f   libSDL2:SDL_dynapi.o
 0001:00174480       _SDL_HapticNumEffects_DEFAULT 00575480 f   libSDL2:SDL_dynapi.o
 0001:001744a0       _SDL_HapticClose_DEFAULT   005754a0 f   libSDL2:SDL_dynapi.o
 0001:001744c0       _SDL_HapticOpenFromJoystick_DEFAULT 005754c0 f   libSDL2:SDL_dynapi.o
 0001:001744e0       _SDL_JoystickIsHaptic_DEFAULT 005754e0 f   libSDL2:SDL_dynapi.o
 0001:00174500       _SDL_HapticOpenFromMouse_DEFAULT 00575500 f   libSDL2:SDL_dynapi.o
 0001:00174510       _SDL_MouseIsHaptic_DEFAULT 00575510 f   libSDL2:SDL_dynapi.o
 0001:00174520       _SDL_HapticIndex_DEFAULT   00575520 f   libSDL2:SDL_dynapi.o
 0001:00174540       _SDL_HapticOpened_DEFAULT  00575540 f   libSDL2:SDL_dynapi.o
 0001:00174560       _SDL_HapticOpen_DEFAULT    00575560 f   libSDL2:SDL_dynapi.o
 0001:00174580       _SDL_HapticName_DEFAULT    00575580 f   libSDL2:SDL_dynapi.o
 0001:001745a0       _SDL_NumHaptics_DEFAULT    005755a0 f   libSDL2:SDL_dynapi.o
 0001:001745b0       _SDL_LoadDollarTemplates_DEFAULT 005755b0 f   libSDL2:SDL_dynapi.o
 0001:001745e0       _SDL_SaveDollarTemplate_DEFAULT 005755e0 f   libSDL2:SDL_dynapi.o
 0001:00174610       _SDL_SaveAllDollarTemplates_DEFAULT 00575610 f   libSDL2:SDL_dynapi.o
 0001:00174630       _SDL_RecordGesture_DEFAULT 00575630 f   libSDL2:SDL_dynapi.o
 0001:00174650       _SDL_GameControllerClose_DEFAULT 00575650 f   libSDL2:SDL_dynapi.o
 0001:00174670       _SDL_GameControllerGetButton_DEFAULT 00575670 f   libSDL2:SDL_dynapi.o
 0001:00174690       _SDL_GameControllerGetBindForButton_DEFAULT 00575690 f   libSDL2:SDL_dynapi.o
 0001:001746c0       _SDL_GameControllerGetStringForButton_DEFAULT 005756c0 f   libSDL2:SDL_dynapi.o
 0001:001746e0       _SDL_GameControllerGetButtonFromString_DEFAULT 005756e0 f   libSDL2:SDL_dynapi.o
 0001:00174700       _SDL_GameControllerGetAxis_DEFAULT 00575700 f   libSDL2:SDL_dynapi.o
 0001:00174720       _SDL_GameControllerGetBindForAxis_DEFAULT 00575720 f   libSDL2:SDL_dynapi.o
 0001:00174750       _SDL_GameControllerGetStringForAxis_DEFAULT 00575750 f   libSDL2:SDL_dynapi.o
 0001:00174770       _SDL_GameControllerGetAxisFromString_DEFAULT 00575770 f   libSDL2:SDL_dynapi.o
 0001:00174790       _SDL_GameControllerEventState_DEFAULT 00575790 f   libSDL2:SDL_dynapi.o
 0001:001747b0       _SDL_GameControllerGetJoystick_DEFAULT 005757b0 f   libSDL2:SDL_dynapi.o
 0001:001747d0       _SDL_GameControllerGetAttached_DEFAULT 005757d0 f   libSDL2:SDL_dynapi.o
 0001:001747f0       _SDL_GameControllerName_DEFAULT 005757f0 f   libSDL2:SDL_dynapi.o
 0001:00174810       _SDL_GameControllerOpen_DEFAULT 00575810 f   libSDL2:SDL_dynapi.o
 0001:00174830       _SDL_GameControllerNameForIndex_DEFAULT 00575830 f   libSDL2:SDL_dynapi.o
 0001:00174850       _SDL_IsGameController_DEFAULT 00575850 f   libSDL2:SDL_dynapi.o
 0001:00174870       _SDL_GameControllerMapping_DEFAULT 00575870 f   libSDL2:SDL_dynapi.o
 0001:00174890       _SDL_GameControllerMappingForGUID_DEFAULT 00575890 f   libSDL2:SDL_dynapi.o
 0001:001748a0       _SDL_GameControllerAddMapping_DEFAULT 005758a0 f   libSDL2:SDL_dynapi.o
 0001:001748c0       _SDL_GetPrefPath_DEFAULT   005758c0 f   libSDL2:SDL_dynapi.o
 0001:001748e0       _SDL_GetBasePath_DEFAULT   005758e0 f   libSDL2:SDL_dynapi.o
 0001:001748f0       _SDL_RegisterEvents_DEFAULT 005758f0 f   libSDL2:SDL_dynapi.o
 0001:00174910       _SDL_EventState_DEFAULT    00575910 f   libSDL2:SDL_dynapi.o
 0001:00174930       _SDL_FilterEvents_DEFAULT  00575930 f   libSDL2:SDL_dynapi.o
 0001:00174950       _SDL_DelEventWatch_DEFAULT 00575950 f   libSDL2:SDL_dynapi.o
 0001:00174970       _SDL_AddEventWatch_DEFAULT 00575970 f   libSDL2:SDL_dynapi.o
 0001:00174990       _SDL_GetEventFilter_DEFAULT 00575990 f   libSDL2:SDL_dynapi.o
 0001:001749b0       _SDL_SetEventFilter_DEFAULT 005759b0 f   libSDL2:SDL_dynapi.o
 0001:001749d0       _SDL_PushEvent_DEFAULT     005759d0 f   libSDL2:SDL_dynapi.o
 0001:001749f0       _SDL_WaitEventTimeout_DEFAULT 005759f0 f   libSDL2:SDL_dynapi.o
 0001:00174a10       _SDL_WaitEvent_DEFAULT     00575a10 f   libSDL2:SDL_dynapi.o
 0001:00174a30       _SDL_PollEvent_DEFAULT     00575a30 f   libSDL2:SDL_dynapi.o
 0001:00174a50       _SDL_FlushEvents_DEFAULT   00575a50 f   libSDL2:SDL_dynapi.o
 0001:00174a70       _SDL_FlushEvent_DEFAULT    00575a70 f   libSDL2:SDL_dynapi.o
 0001:00174a90       _SDL_HasEvents_DEFAULT     00575a90 f   libSDL2:SDL_dynapi.o
 0001:00174ab0       _SDL_HasEvent_DEFAULT      00575ab0 f   libSDL2:SDL_dynapi.o
 0001:00174ad0       _SDL_PeepEvents_DEFAULT    00575ad0 f   libSDL2:SDL_dynapi.o
 0001:00174b20       _SDL_Error_DEFAULT         00575b20 f   libSDL2:SDL_dynapi.o
 0001:00174b40       _SDL_GetSystemRAM_DEFAULT  00575b40 f   libSDL2:SDL_dynapi.o
 0001:00174b50       _SDL_HasSSE2_DEFAULT       00575b50 f   libSDL2:SDL_dynapi.o
 0001:00174b60       _SDL_HasAltiVec_DEFAULT    00575b60 f   libSDL2:SDL_dynapi.o
 0001:00174b70       _SDL_SetClipboardText_DEFAULT 00575b70 f   libSDL2:SDL_dynapi.o
 0001:00174b90       _SDL_MixAudioFormat_DEFAULT 00575b90 f   libSDL2:SDL_dynapi.o
 0001:00174be0       _SDL_MixAudio_DEFAULT      00575be0 f   libSDL2:SDL_dynapi.o
 0001:00174c20       _SDL_ConvertAudio_DEFAULT  00575c20 f   libSDL2:SDL_dynapi.o
 0001:00174c40       _SDL_BuildAudioCVT_DEFAULT 00575c40 f   libSDL2:SDL_dynapi.o
 0001:00174cb0       _SDL_FreeWAV_DEFAULT       00575cb0 f   libSDL2:SDL_dynapi.o
 0001:00174cd0       _SDL_LoadWAV_RW_DEFAULT    00575cd0 f   libSDL2:SDL_dynapi.o
 0001:00174d20       _SDL_PauseAudioDevice_DEFAULT 00575d20 f   libSDL2:SDL_dynapi.o
 0001:00174d40       _SDL_PauseAudio_DEFAULT    00575d40 f   libSDL2:SDL_dynapi.o
 0001:00174d60       _SDL_GetAudioDeviceStatus_DEFAULT 00575d60 f   libSDL2:SDL_dynapi.o
 0001:00174d80       _SDL_OpenAudioDevice_DEFAULT 00575d80 f   libSDL2:SDL_dynapi.o
 0001:00174dd0       _SDL_GetAudioDeviceName_DEFAULT 00575dd0 f   libSDL2:SDL_dynapi.o
 0001:00174df0       _SDL_GetNumAudioDevices_DEFAULT 00575df0 f   libSDL2:SDL_dynapi.o
 0001:00174e10       _SDL_OpenAudio_DEFAULT     00575e10 f   libSDL2:SDL_dynapi.o
 0001:00174e30       _SDL_AudioInit_DEFAULT     00575e30 f   libSDL2:SDL_dynapi.o
 0001:00174e50       _SDL_GetAudioDriver_DEFAULT 00575e50 f   libSDL2:SDL_dynapi.o
 0001:00174e70       _SDL_GetNumAudioDrivers_DEFAULT 00575e70 f   libSDL2:SDL_dynapi.o
 0001:00174e80       _SDL_AtomicGetPtr_DEFAULT  00575e80 f   libSDL2:SDL_dynapi.o
 0001:00174ea0       _SDL_AtomicSetPtr_DEFAULT  00575ea0 f   libSDL2:SDL_dynapi.o
 0001:00174ec0       _SDL_AtomicCASPtr_DEFAULT  00575ec0 f   libSDL2:SDL_dynapi.o
 0001:00174ef0       _SDL_AtomicAdd_DEFAULT     00575ef0 f   libSDL2:SDL_dynapi.o
 0001:00174f10       _SDL_AtomicGet_DEFAULT     00575f10 f   libSDL2:SDL_dynapi.o
 0001:00174f30       _SDL_AtomicSet_DEFAULT     00575f30 f   libSDL2:SDL_dynapi.o
 0001:00174f50       _SDL_AtomicCAS_DEFAULT     00575f50 f   libSDL2:SDL_dynapi.o
 0001:00174f80       _SDL_AtomicUnlock_DEFAULT  00575f80 f   libSDL2:SDL_dynapi.o
 0001:00174fa0       _SDL_AtomicLock_DEFAULT    00575fa0 f   libSDL2:SDL_dynapi.o
 0001:00174fc0       _SDL_AtomicTryLock_DEFAULT 00575fc0 f   libSDL2:SDL_dynapi.o
 0001:00174fe0       _SDL_GetAssertionReport_DEFAULT 00575fe0 f   libSDL2:SDL_dynapi.o
 0001:00174ff0       _SDL_SetAssertionHandler_DEFAULT 00575ff0 f   libSDL2:SDL_dynapi.o
 0001:00175010       _SDL_ReportAssertion_DEFAULT 00576010 f   libSDL2:SDL_dynapi.o
 0001:00175050       _SDL_WasInit_DEFAULT       00576050 f   libSDL2:SDL_dynapi.o
 0001:00175070       _SDL_QuitSubSystem_DEFAULT 00576070 f   libSDL2:SDL_dynapi.o
 0001:00175090       _SDL_InitSubSystem_DEFAULT 00576090 f   libSDL2:SDL_dynapi.o
 0001:001750b0       _SDL_Init_DEFAULT          005760b0 f   libSDL2:SDL_dynapi.o
 0001:001750d0       _SDL_RenderGetD3D9Device_DEFAULT 005760d0 f   libSDL2:SDL_dynapi.o
 0001:001750f0       _SDL_Direct3D9GetAdapterIndex_DEFAULT 005760f0 f   libSDL2:SDL_dynapi.o
 0001:00175110       _SDL_RegisterApp_DEFAULT   00576110 f   libSDL2:SDL_dynapi.o
 0001:00175140       _SDL_RWFromFP_DEFAULT      00576140 f   libSDL2:SDL_dynapi.o
 0001:00175160       _SDL_CreateThread_DEFAULT  00576160 f   libSDL2:SDL_dynapi.o
 0001:001751b0       _SDL_snprintf_DEFAULT      005761b0 f   libSDL2:SDL_dynapi.o
 0001:001751f0       _SDL_sscanf_DEFAULT        005761f0 f   libSDL2:SDL_dynapi.o
 0001:00175220       _SDL_LogMessage_DEFAULT    00576220 f   libSDL2:SDL_dynapi.o
 0001:00175260       _SDL_LogCritical_DEFAULT   00576260 f   libSDL2:SDL_dynapi.o
 0001:001752a0       _SDL_LogError_DEFAULT      005762a0 f   libSDL2:SDL_dynapi.o
 0001:001752e0       _SDL_LogWarn_DEFAULT       005762e0 f   libSDL2:SDL_dynapi.o
 0001:00175320       _SDL_LogInfo_DEFAULT       00576320 f   libSDL2:SDL_dynapi.o
 0001:00175360       _SDL_LogDebug_DEFAULT      00576360 f   libSDL2:SDL_dynapi.o
 0001:001753a0       _SDL_LogVerbose_DEFAULT    005763a0 f   libSDL2:SDL_dynapi.o
 0001:001753e0       _SDL_Log_DEFAULT           005763e0 f   libSDL2:SDL_dynapi.o
 0001:00175420       _SDL_SetError_DEFAULT      00576420 f   libSDL2:SDL_dynapi.o
 0001:00175470       _SDL_GL_ResetAttributes_DEFAULT 00576470 f   libSDL2:SDL_dynapi.o
 0001:00175560       _SDL_GL_UnloadLibrary_DEFAULT 00576560 f   libSDL2:SDL_dynapi.o
 0001:00175650       _SDL_DisableScreenSaver_DEFAULT 00576650 f   libSDL2:SDL_dynapi.o
 0001:00175740       _SDL_SetMainReady_DEFAULT  00576740 f   libSDL2:SDL_dynapi.o
 0001:00175830       _SDL_PumpEvents_DEFAULT    00576830 f   libSDL2:SDL_dynapi.o
 0001:00175920       _SDL_GameControllerUpdate_DEFAULT 00576920 f   libSDL2:SDL_dynapi.o
 0001:00175a10       _SDL_ClearError_DEFAULT    00576a10 f   libSDL2:SDL_dynapi.o
 0001:00175b00       _SDL_ResetAssertionReport_DEFAULT 00576b00 f   libSDL2:SDL_dynapi.o
 0001:00175bf0       _SDL_CloseAudio_DEFAULT    00576bf0 f   libSDL2:SDL_dynapi.o
 0001:00175ce0       _SDL_EnableScreenSaver_DEFAULT 00576ce0 f   libSDL2:SDL_dynapi.o
 0001:00175dd0       _SDL_VideoQuit_DEFAULT     00576dd0 f   libSDL2:SDL_dynapi.o
 0001:00175ec0       _SDL_JoystickUpdate_DEFAULT 00576ec0 f   libSDL2:SDL_dynapi.o
 0001:00175fb0       _SDL_LogResetPriorities_DEFAULT 00576fb0 f   libSDL2:SDL_dynapi.o
 0001:001760a0       _SDL_StartTextInput_DEFAULT 005770a0 f   libSDL2:SDL_dynapi.o
 0001:00176190       _SDL_StopTextInput_DEFAULT 00577190 f   libSDL2:SDL_dynapi.o
 0001:00176280       _SDL_Quit_DEFAULT          00577280 f   libSDL2:SDL_dynapi.o
 0001:00176370       _SDL_UnregisterApp_DEFAULT 00577370 f   libSDL2:SDL_dynapi.o
 0001:00176460       _SDL_ClearHints_DEFAULT    00577460 f   libSDL2:SDL_dynapi.o
 0001:00176550       _SDL_LockAudio_DEFAULT     00577550 f   libSDL2:SDL_dynapi.o
 0001:00176640       _SDL_UnlockAudio_DEFAULT   00577640 f   libSDL2:SDL_dynapi.o
 0001:00176730       _SDL_AudioQuit_DEFAULT     00577730 f   libSDL2:SDL_dynapi.o
 0001:00176820       _SDL_GetError_DEFAULT      00577820 f   libSDL2:SDL_dynapi.o
 0001:00176910       _SDL_HasSSE42_DEFAULT      00577910 f   libSDL2:SDL_dynapi.o
 0001:00176a00       _SDL_CloseAudioDevice_DEFAULT 00577a00 f   libSDL2:SDL_dynapi.o
 0001:00176af0       _SDL_UnlockTexture_DEFAULT 00577af0 f   libSDL2:SDL_dynapi.o
 0001:00176be0       _SDL_GetCPUCacheLineSize_DEFAULT 00577be0 f   libSDL2:SDL_dynapi.o
 0001:00176cd0       _SDL_HasSSE41_DEFAULT      00577cd0 f   libSDL2:SDL_dynapi.o
 0001:00176dc0       _SDL_DetachThread_DEFAULT  00577dc0 f   libSDL2:SDL_dynapi.o
 0001:00176eb0       _SDL_GetNumVideoDrivers_DEFAULT 00577eb0 f   libSDL2:SDL_dynapi.o
 0001:00176fa0       _SDL_GetGrabbedWindow_DEFAULT 00577fa0 f   libSDL2:SDL_dynapi.o
 0001:00177090       _SDL_GetCPUCount_DEFAULT   00578090 f   libSDL2:SDL_dynapi.o
 0001:00177180       _SDL_RestoreWindow_DEFAULT 00578180 f   libSDL2:SDL_dynapi.o
 0001:00177270       _SDL_IsScreenSaverEnabled_DEFAULT 00578270 f   libSDL2:SDL_dynapi.o
 0001:00177360       _SDL_GetNumTouchDevices_DEFAULT 00578360 f   libSDL2:SDL_dynapi.o
 0001:00177450       _SDL_RaiseWindow_DEFAULT   00578450 f   libSDL2:SDL_dynapi.o
 0001:00177540       _SDL_GetCurrentVideoDriver_DEFAULT 00578540 f   libSDL2:SDL_dynapi.o
 0001:00177630       _SDL_GetAudioStatus_DEFAULT 00578630 f   libSDL2:SDL_dynapi.o
 0001:00177720       _SDL_RenderPresent_DEFAULT 00578720 f   libSDL2:SDL_dynapi.o
 0001:00177810       _SDL_Has3DNow_DEFAULT      00578810 f   libSDL2:SDL_dynapi.o
 0001:00177900       _SDL_UnloadObject_DEFAULT  00578900 f   libSDL2:SDL_dynapi.o
 0001:001779f0       _SDL_GetCursor_DEFAULT     005789f0 f   libSDL2:SDL_dynapi.o
 0001:00177ae0       _SDL_FreePalette_DEFAULT   00578ae0 f   libSDL2:SDL_dynapi.o
 0001:00177bd0       _SDL_JoystickClose_DEFAULT 00578bd0 f   libSDL2:SDL_dynapi.o
 0001:00177cc0       _SDL_HasSSE_DEFAULT        00578cc0 f   libSDL2:SDL_dynapi.o
 0001:00177db0       _SDL_FreeCursor_DEFAULT    00578db0 f   libSDL2:SDL_dynapi.o
 0001:00177ea0       _SDL_HideWindow_DEFAULT    00578ea0 f   libSDL2:SDL_dynapi.o
 0001:00177f90       _SDL_GetDefaultCursor_DEFAULT 00578f90 f   libSDL2:SDL_dynapi.o
 0001:00178080       _SDL_GetRevision_DEFAULT   00579080 f   libSDL2:SDL_dynapi.o
 0001:00178170       _SDL_GetMouseFocus_DEFAULT 00579170 f   libSDL2:SDL_dynapi.o
 0001:00178260       _SDL_DestroyWindow_DEFAULT 00579260 f   libSDL2:SDL_dynapi.o
 0001:00178350       _SDL_SetCursor_DEFAULT     00579350 f   libSDL2:SDL_dynapi.o
 0001:00178440       _SDL_DestroyMutex_DEFAULT  00579440 f   libSDL2:SDL_dynapi.o
 0001:00178530       _SDL_GetClipboardText_DEFAULT 00579530 f   libSDL2:SDL_dynapi.o
 0001:00178620       _SDL_FreeSurface_DEFAULT   00579620 f   libSDL2:SDL_dynapi.o
 0001:00178710       _SDL_LockAudioDevice_DEFAULT 00579710 f   libSDL2:SDL_dynapi.o
 0001:00178800       _SDL_CreateCond_DEFAULT    00579800 f   libSDL2:SDL_dynapi.o
 0001:001788f0       _SDL_HasRDTSC_DEFAULT      005798f0 f   libSDL2:SDL_dynapi.o
 0001:001789e0       _SDL_MaximizeWindow_DEFAULT 005799e0 f   libSDL2:SDL_dynapi.o
 0001:00178ad0       _SDL_HasSSE3_DEFAULT       00579ad0 f   libSDL2:SDL_dynapi.o
 0001:00178bc0       _SDL_SetTextInputRect_DEFAULT 00579bc0 f   libSDL2:SDL_dynapi.o
 0001:00178cb0       _SDL_HasMMX_DEFAULT        00579cb0 f   libSDL2:SDL_dynapi.o
 0001:00178da0       _SDL_UnlockSurface_DEFAULT 00579da0 f   libSDL2:SDL_dynapi.o
 0001:00178e90       _SDL_ThreadID_DEFAULT      00579e90 f   libSDL2:SDL_dynapi.o
 0001:00178f80       _SDL_Delay_DEFAULT         00579f80 f   libSDL2:SDL_dynapi.o
 0001:00179070       _SDL_MinimizeWindow_DEFAULT 0057a070 f   libSDL2:SDL_dynapi.o
 0001:00179160       _SDL_ShowWindow_DEFAULT    0057a160 f   libSDL2:SDL_dynapi.o
 0001:00179250       _SDL_HasAVX_DEFAULT        0057a250 f   libSDL2:SDL_dynapi.o
 0001:00179340       _SDL_GL_GetCurrentWindow_DEFAULT 0057a340 f   libSDL2:SDL_dynapi.o
 0001:00179430       _SDL_GetDefaultAssertionHandler_DEFAULT 0057a430 f   libSDL2:SDL_dynapi.o
 0001:00179520       _SDL_HasAVX2_DEFAULT       0057a520 f   libSDL2:SDL_dynapi.o
 0001:00179610       _SDL_GL_GetSwapInterval_DEFAULT 0057a610 f   libSDL2:SDL_dynapi.o
 0001:00179700       _SDL_GL_GetCurrentContext_DEFAULT 0057a700 f   libSDL2:SDL_dynapi.o
 0001:001797f0       _SDL_ClearQueuedAudio_DEFAULT 0057a7f0 f   libSDL2:SDL_dynapi.o
 0001:001798e0       _SDL_GL_DeleteContext_DEFAULT 0057a8e0 f   libSDL2:SDL_dynapi.o
 0001:001799d0       _SDL_UnlockAudioDevice_DEFAULT 0057a9d0 f   libSDL2:SDL_dynapi.o
 0001:00179ac0       _SDL_GetVersion_DEFAULT    0057aac0 f   libSDL2:SDL_dynapi.o
 0001:00179bb0       _SDL_GetNumRenderDrivers_DEFAULT 0057abb0 f   libSDL2:SDL_dynapi.o
 0001:00179ca0       _SDL_GetCurrentAudioDriver_DEFAULT 0057aca0 f   libSDL2:SDL_dynapi.o
 0001:00179d90       _SDL_free_DEFAULT          0057ad90 f   libSDL2:SDL_dynapi.o
 0001:00179e80       _SDL_HasClipboardText_DEFAULT 0057ae80 f   libSDL2:SDL_dynapi.o
 0001:00179f70       _SDL_TLSCreate_DEFAULT     0057af70 f   libSDL2:SDL_dynapi.o
 0001:0017a060       _SDL_AllocRW_DEFAULT       0057b060 f   libSDL2:SDL_dynapi.o
 0001:0017a150       _SDL_DestroyTexture_DEFAULT 0057b150 f   libSDL2:SDL_dynapi.o
 0001:0017a240       _SDL_DestroyRenderer_DEFAULT 0057b240 f   libSDL2:SDL_dynapi.o
 0001:0017a330       _SDL_GetRevisionNumber_DEFAULT 0057b330 f   libSDL2:SDL_dynapi.o
 0001:0017c960       _SDL_PrivateJoystickDetectProc@16 0057d960 f   libSDL2:SDL_windowsjoystick.o
 0001:0017c9d0       _SDL_JoystickThread        0057d9d0 f   libSDL2:SDL_windowsjoystick.o
 0001:0017d530       _SDL_GetErrorMsg.constprop.0 0057e530 f   libSDL2:SDL_error.o
 0001:0017d900       _SDL_LogOutput             0057e900 f   libSDL2:SDL_log.o
 0001:0017e560       _SDL_strncmp_REAL.constprop.7 0057f560 f   libSDL2:SDL_string.o
 0001:0017e5c0       _SDL_ScanFloat             0057f5c0 f   libSDL2:SDL_string.o
 0001:0017e6f0       _SDL_PrintString           0057f6f0 f   libSDL2:SDL_string.o
 0001:0017e870       _SDL_ScanLong              0057f870 f   libSDL2:SDL_string.o
 0001:0017e9c0       _SDL_ScanLongLong          0057f9c0 f   libSDL2:SDL_string.o
 0001:00182200       _mem_size                  00583200 f   libSDL2:SDL_rwops.o
 0001:00182210       _mem_writeconst            00583210 f   libSDL2:SDL_rwops.o
 0001:00182230       _windows_file_close        00583230 f   libSDL2:SDL_rwops.o
 0001:00182280       _mem_close                 00583280 f   libSDL2:SDL_rwops.o
 0001:001822a0       _windows_file_write        005832a0 f   libSDL2:SDL_rwops.o
 0001:001823a0       _mem_write                 005833a0 f   libSDL2:SDL_rwops.o
 0001:00182400       _mem_read                  00583400 f   libSDL2:SDL_rwops.o
 0001:00182480       _windows_file_read         00583480 f   libSDL2:SDL_rwops.o
 0001:001825c0       _windows_file_seek         005835c0 f   libSDL2:SDL_rwops.o
 0001:001826b0       _mem_seek                  005836b0 f   libSDL2:SDL_rwops.o
 0001:00182720       _windows_file_size         00583720 f   libSDL2:SDL_rwops.o
 0001:00182ff0       _WindowsScanCodeToSDLScanCode 00583ff0 f   libSDL2:SDL_windowsevents.o
 0001:00185260       _UpdateWindowsEnableMessageLoop 00586260 f   libSDL2:SDL_windowsvideo.o
 0001:00185290       _UpdateWindowFrameUsableWhileCursorHidden 00586290 f   libSDL2:SDL_windowsvideo.o
 0001:001852c0       _WIN_Available             005862c0 f   libSDL2:SDL_windowsvideo.o
 0001:001852d0       _WIN_CreateDevice          005862d0 f   libSDL2:SDL_windowsvideo.o
 0001:00185570       _WIN_DeleteDevice          00586570 f   libSDL2:SDL_windowsvideo.o
 0001:001855c0       _WIN_VideoQuit             005865c0 f   libSDL2:SDL_windowsvideo.o
 0001:001855f0       _WIN_VideoInit             005865f0 f   libSDL2:SDL_windowsvideo.o
 0001:00185b70       _D3D_WindowEvent           00586b70 f   libSDL2:SDL_render_d3d.o
 0001:00185b90       _D3D_UpdateViewport        00586b90 f   libSDL2:SDL_render_d3d.o
 0001:00185cc0       _D3D_SetError              00586cc0 f   libSDL2:SDL_render_d3d.o
 0001:00185ed0       _D3D_BindTextureRep        00586ed0 f   libSDL2:SDL_render_d3d.o
 0001:00186010       _D3D_UpdateClipRect        00587010 f   libSDL2:SDL_render_d3d.o
 0001:001860e0       _D3D_InitRenderState       005870e0 f   libSDL2:SDL_render_d3d.o
 0001:001863a0       _D3D_RenderReadPixels      005873a0 f   libSDL2:SDL_render_d3d.o
 0001:001865e0       _D3D_DestroyRenderer       005875e0 f   libSDL2:SDL_render_d3d.o
 0001:00186680       _D3D_CreateRenderer        00587680 f   libSDL2:SDL_render_d3d.o
 0001:00186cf0       _D3D_SetBlendMode.isra.3   00587cf0 f   libSDL2:SDL_render_d3d.o
 0001:00186f00       _D3D_LockTexture           00587f00 f   libSDL2:SDL_render_d3d.o
 0001:00187170       _D3D_DestroyTexture        00588170 f   libSDL2:SDL_render_d3d.o
 0001:00187240       _D3D_CreateTexture         00588240 f   libSDL2:SDL_render_d3d.o
 0001:00187600       _D3D_Reset                 00588600 f   libSDL2:SDL_render_d3d.o
 0001:00187a00       _D3D_RenderPresent         00588a00 f   libSDL2:SDL_render_d3d.o
 0001:00187ab0       _D3D_ActivateRenderer      00588ab0 f   libSDL2:SDL_render_d3d.o
 0001:00187c40       _D3D_RenderFillRects       00588c40 f   libSDL2:SDL_render_d3d.o
 0001:00187df0       _D3D_RenderDrawLines       00588df0 f   libSDL2:SDL_render_d3d.o
 0001:00188020       _D3D_RenderDrawPoints      00589020 f   libSDL2:SDL_render_d3d.o
 0001:00188170       _D3D_RenderClear           00589170 f   libSDL2:SDL_render_d3d.o
 0001:00188360       _D3D_SetRenderTarget       00589360 f   libSDL2:SDL_render_d3d.o
 0001:00188580       _D3D_RenderCopy            00589580 f   libSDL2:SDL_render_d3d.o
 0001:00188930       _D3D_UpdateTextureRep      00589930 f   libSDL2:SDL_render_d3d.o
 0001:00188bc0       _D3D_UpdateTextureYUV      00589bc0 f   libSDL2:SDL_render_d3d.o
 0001:00188d10       _D3D_UpdateTexture         00589d10 f   libSDL2:SDL_render_d3d.o
 0001:00188f10       _D3D_UnlockTexture         00589f10 f   libSDL2:SDL_render_d3d.o
 0001:00189160       _D3D_RenderCopyEx          0058a160 f   libSDL2:SDL_render_d3d.o
 0001:0018a290       _debug_print               0058b290 f   libSDL2:SDL_assert.o
 0001:0018a2c0       _SDL_PromptAssertion       0058b2c0 f   libSDL2:SDL_assert.o
 0001:0018a530       _debug_print.constprop.0   0058b530 f   libSDL2:SDL_assert.o
 0001:0018ab20       _SDL_AudioThreadInit_Default 0058bb20 f   libSDL2:SDL_audio.o
 0001:0018ab30       _SDL_AudioWaitDevice_Default 0058bb30 f   libSDL2:SDL_audio.o
 0001:0018ab40       _SDL_AudioPlayDevice_Default 0058bb40 f   libSDL2:SDL_audio.o
 0001:0018ab50       _SDL_AudioGetPendingBytes_Default 0058bb50 f   libSDL2:SDL_audio.o
 0001:0018ab60       _SDL_AudioGetDeviceBuf_Default 0058bb60 f   libSDL2:SDL_audio.o
 0001:0018ab70       _SDL_AudioWaitDone_Default 0058bb70 f   libSDL2:SDL_audio.o
 0001:0018ab80       _SDL_AudioCloseDevice_Default 0058bb80 f   libSDL2:SDL_audio.o
 0001:0018ab90       _SDL_AudioDeinitialize_Default 0058bb90 f   libSDL2:SDL_audio.o
 0001:0018aba0       _SDL_AudioFreeDeviceHandle_Default 0058bba0 f   libSDL2:SDL_audio.o
 0001:0018abb0       _SDL_AudioOpenDevice_Default 0058bbb0 f   libSDL2:SDL_audio.o
 0001:0018abc0       _SDL_BufferQueueDrainCallback 0058bbc0 f   libSDL2:SDL_audio.o
 0001:0018aca0       _SDL_AudioUnlockDevice_Default 0058bca0 f   libSDL2:SDL_audio.o
 0001:0018ace0       _SDL_AudioLockDevice_Default 0058bce0 f   libSDL2:SDL_audio.o
 0001:0018aec0       _close_audio_device        0058bec0 f   libSDL2:SDL_audio.o
 0001:0018afa0       _SDL_AudioDetectDevices_Default 0058bfa0 f   libSDL2:SDL_audio.o
 0001:0018bcc0       _open_audio_device         0058ccc0 f   libSDL2:SDL_audio.o
 0001:0018e6b0       _IMA_ADPCM_nibble          0058f6b0 f   libSDL2:SDL_wave.o
 0001:0018f640       _SDL_ConvertMono           00590640 f   libSDL2:SDL_audiocvt.o
 0001:0018fab0       _SDL_ConvertStrip          00590ab0 f   libSDL2:SDL_audiocvt.o
 0001:0018fbe0       _SDL_ConvertStrip_2        00590be0 f   libSDL2:SDL_audiocvt.o
 0001:0018fdf0       _SDL_ConvertStereo         00590df0 f   libSDL2:SDL_audiocvt.o
 0001:0018ff00       _SDL_ConvertSurround       00590f00 f   libSDL2:SDL_audiocvt.o
 0001:00190590       _SDL_ConvertSurround_4     00591590 f   libSDL2:SDL_audiocvt.o
 0001:00194a70       _SDL_AddEvent              00595a70 f   libSDL2:SDL_events.o
 0001:00199040       _dollarNormalize           0059a040 f   libSDL2:SDL_gesture.o
 0001:001993c0       _dollarDifference          0059a3c0 f   libSDL2:SDL_gesture.o
 0001:001994c0       _SDL_AddDollarGesture      0059a4c0 f   libSDL2:SDL_gesture.o
 0001:0019bbe0       _SDL_JoystickAllowBackgroundEventsChanged 0059cbe0 f   libSDL2:SDL_joystick.o
 0001:0019dc60       _cmpmodes                  0059ec60 f   libSDL2:SDL_video.o
 0001:0019dd00       _SDL_GetClosestDisplayModeForDisplay 0059ed00 f   libSDL2:SDL_video.o
 0001:0019df60       _SDL_SetDisplayModeForDisplay 0059ef60 f   libSDL2:SDL_video.o
 0001:0019e0f0       _SDL_SetDisplayModeForDisplay.constprop.11 0059f0f0 f   libSDL2:SDL_video.o
 0001:0019e1c0       _SDL_DestroyWindowTexture  0059f1c0 f   libSDL2:SDL_video.o
 0001:0019e2b0       _SDL_UpdateWindowTexture   0059f2b0 f   libSDL2:SDL_video.o
 0001:0019f0d0       _SDL_UpdateFullscreenMode  005a00d0 f   libSDL2:SDL_video.o
 0001:0019fd20       _SDL_CreateWindowTexture   005a0d20 f   libSDL2:SDL_video.o
 0001:001a14f0       _SDL_FinishWindowCreation  005a24f0 f   libSDL2:SDL_video.o
 0001:001a48e0       _SDL_UpdateMouseFocus.isra.2 005a58e0 f   libSDL2:SDL_mouse.o
 0001:001a4ee0       _SDL_PrivateSendMouseMotion 005a5ee0 f   libSDL2:SDL_mouse.o
 0001:001a6ca0       _Map1to1                   005a7ca0 f   libSDL2:SDL_pixels.o
 0001:001a6e20       _MapNto1.isra.2            005a7e20 f   libSDL2:SDL_pixels.o
 0001:001ab910       _UpdateLogicalSize         005ac910 f   libSDL2:SDL_render.o
 0001:001abd10       _SDL_RendererEventWatch    005acd10 f   libSDL2:SDL_render.o
 0001:001aedf0       _RecursivelyCalculateShapeTree 005afdf0 f   libSDL2:SDL_shape.o
 0001:001b02e0       _sys_trim.constprop.8      005b12e0 f   libSDL2:SDL_malloc.o
 0001:001b2590       _internal_memalign.constprop.4 005b3590 f   libSDL2:SDL_malloc.o
 0001:001b3b40       _pivot_big                 005b4b40 f   libSDL2:SDL_qsort.o
 0001:001b58e0       _getlocale.constprop.0     005b68e0 f   libSDL2:SDL_iconv.o
 0001:001bb670       _RunThreadViaCreateThread@4 005bc670 f   libSDL2:SDL_systhread.o
 0001:001bb6b0       _RunThreadViaBeginThreadEx@4 005bc6b0 f   libSDL2:SDL_systhread.o
 0001:001bb880       _SDL_TimerResolutionChanged 005bc880 f   libSDL2:SDL_systimer.o
 0001:001bbb80       _SDL_TimerThread           005bcb80 f   libSDL2:SDL_timer.o
 0001:001bcfd0       _IsWindowsVersionOrGreater.constprop.0 005bdfd0 f   libSDL2:SDL_windows.o
 0001:001bdaa0       _SortDevFunc               005beaa0 f   libSDL2:SDL_dinputjoystick.o
 0001:001bdac0       _EnumDevObjectsCallback@8  005beac0 f   libSDL2:SDL_dinputjoystick.o
 0001:001bdd90       _UpdateDINPUTJoystickState_Buffered 005bed90 f   libSDL2:SDL_dinputjoystick.o
 0001:001be000       _EnumJoysticksCallback@8   005bf000 f   libSDL2:SDL_dinputjoystick.o
 0001:001be3a0       _UpdateDINPUTJoystickState_Polled 005bf3a0 f   libSDL2:SDL_dinputjoystick.o
 0001:001beca0       _SDL_RunXInputHaptic       005bfca0 f   libSDL2:SDL_xinputhaptic.o
 0001:001bf740       _DI_EffectCallback@8       005c0740 f   libSDL2:SDL_dinputhaptic.o
 0001:001bf8d0       _SDL_DINPUT_HapticOpenFromDevice 005c08d0 f   libSDL2:SDL_dinputhaptic.o
 0001:001bfc10       _DI_DeviceObjectCallback@8 005c0c10 f   libSDL2:SDL_dinputhaptic.o
 0001:001bfd40       _SDL_SYS_SetDirection.isra.3.part.4 005c0d40 f   libSDL2:SDL_dinputhaptic.o
 0001:001c0140       _EnumHapticsCallback@8     005c1140 f   libSDL2:SDL_dinputhaptic.o
 0001:001c20b0       _WIN_GetGlobalMouseState   005c30b0 f   libSDL2:SDL_windowsmouse.o
 0001:001c2170       _WIN_WarpMouseGlobal       005c3170 f   libSDL2:SDL_windowsmouse.o
 0001:001c2190       _WIN_WarpMouse             005c3190 f   libSDL2:SDL_windowsmouse.o
 0001:001c2210       _WIN_FreeCursor            005c3210 f   libSDL2:SDL_windowsmouse.o
 0001:001c2240       _WIN_ShowCursor            005c3240 f   libSDL2:SDL_windowsmouse.o
 0001:001c2280       _WIN_CreateSystemCursor    005c3280 f   libSDL2:SDL_windowsmouse.o
 0001:001c2370       _WIN_CreateCursor          005c3370 f   libSDL2:SDL_windowsmouse.o
 0001:001c2590       _WIN_SetRelativeMouseMode  005c3590 f   libSDL2:SDL_windowsmouse.o
 0001:001c2650       _WIN_CaptureMouse          005c3650 f   libSDL2:SDL_windowsmouse.o
 0001:001c28a0       _SetupWindowData.isra.1    005c38a0 f   libSDL2:SDL_windowswindow.o
 0001:001c4200       _IME_SetupAPI              005c5200 f   libSDL2:SDL_windowskeyboard.o
 0001:001c4320       _IME_SendEditingEvent      005c5320 f   libSDL2:SDL_windowskeyboard.o
 0001:001c4440       _IME_GetId                 005c5440 f   libSDL2:SDL_windowskeyboard.o
 0001:001c4930       _UILess_GetCandidateList   005c5930 f   libSDL2:SDL_windowskeyboard.o
 0001:001c4bd0       _IME_Disable.isra.5        005c5bd0 f   libSDL2:SDL_windowskeyboard.o
 0001:001c5430       _IME_Init.part.7           005c6430 f   libSDL2:SDL_windowskeyboard.o
 0001:001c5800       _IME_GetReadingString      005c6800 f   libSDL2:SDL_windowskeyboard.o
 0001:001c7b60       _RemovePendingResizedEvents 005c8b60 f   libSDL2:SDL_windowevents.o
 0001:001c7b90       _RemovePendingSizeChangedEvents 005c8b90 f   libSDL2:SDL_windowevents.o
 0001:001c7bc0       _RemovePendingMoveEvents   005c8bc0 f   libSDL2:SDL_windowevents.o
 0001:001c85a0       _WIN_GetMonitorDPI@16      005c95a0 f   libSDL2:SDL_windowsmodes.o
 0001:001c8660       _WIN_GetDisplayMode.isra.0 005c9660 f   libSDL2:SDL_windowsmodes.o
 0001:001c8be0       _WIN_AddDisplay            005c9be0 f   libSDL2:SDL_windowsmodes.o
 0001:001c9a30       _WIN_GL_ChoosePixelFormatARB 005caa30 f   libSDL2:SDL_windowsopengl.o
 0001:001c9cb0       _WIN_GL_SetupWindowInternal.isra.1 005cacb0 f   libSDL2:SDL_windowsopengl.o
 0001:001cbc20       _VoiceCBOnStreamEnd@4      005ccc20 f   libSDL2:SDL_xaudio2.o
 0001:001cbc30       _VoiceCBOnVoiceProcessPassStart@8 005ccc30 f   libSDL2:SDL_xaudio2.o
 0001:001cbc40       _VoiceCBOnVoiceProcessPassEnd@4 005ccc40 f   libSDL2:SDL_xaudio2.o
 0001:001cbc50       _VoiceCBOnBufferStart@8    005ccc50 f   libSDL2:SDL_xaudio2.o
 0001:001cbc60       _VoiceCBOnLoopEnd@8        005ccc60 f   libSDL2:SDL_xaudio2.o
 0001:001cbc70       _XAUDIO2_GetDeviceBuf      005ccc70 f   libSDL2:SDL_xaudio2.o
 0001:001cbc80       _XAUDIO2_Deinitialize      005ccc80 f   libSDL2:SDL_xaudio2.o
 0001:001cbc90       _XAUDIO2_CloseDevice       005ccc90 f   libSDL2:SDL_xaudio2.o
 0001:001cbd70       _XAUDIO2_WaitDone          005ccd70 f   libSDL2:SDL_xaudio2.o
 0001:001cbdd0       _XAUDIO2_PlayDevice        005ccdd0 f   libSDL2:SDL_xaudio2.o
 0001:001cbe80       _VoiceCBOnVoiceError@12    005cce80 f   libSDL2:SDL_xaudio2.o
 0001:001cbea0       _VoiceCBOnBufferEnd@8      005ccea0 f   libSDL2:SDL_xaudio2.o
 0001:001cbec0       _XAUDIO2_WaitDevice        005ccec0 f   libSDL2:SDL_xaudio2.o
 0001:001cbef0       _XAUDIO2_Init              005ccef0 f   libSDL2:SDL_xaudio2.o
 0001:001cbff0       _XAUDIO2_DetectDevices     005ccff0 f   libSDL2:SDL_xaudio2.o
 0001:001cc1a0       _XAUDIO2_OpenDevice        005cd1a0 f   libSDL2:SDL_xaudio2.o
 0001:001ccc60       _DSOUND_DetectDevices      005cdc60 f   libSDL2:SDL_directsound.o
 0001:001ccca0       _DSOUND_PlayDevice         005cdca0 f   libSDL2:SDL_directsound.o
 0001:001cccf0       _DSOUND_FreeDeviceHandle   005cdcf0 f   libSDL2:SDL_directsound.o
 0001:001ccd00       _DSOUND_CloseDevice        005cdd00 f   libSDL2:SDL_directsound.o
 0001:001ccd70       _SetDSerror                005cdd70 f   libSDL2:SDL_directsound.o
 0001:001ccf20       _DSOUND_GetDeviceBuf       005cdf20 f   libSDL2:SDL_directsound.o
 0001:001cd0d0       _DSOUND_WaitDevice         005ce0d0 f   libSDL2:SDL_directsound.o
 0001:001cd240       _FindAllDevs@16            005ce240 f   libSDL2:SDL_directsound.o
 0001:001cd2d0       _DSOUND_Deinitialize       005ce2d0 f   libSDL2:SDL_directsound.o
 0001:001cd320       _DSOUND_Init               005ce320 f   libSDL2:SDL_directsound.o
 0001:001cd480       _DSOUND_WaitDone           005ce480 f   libSDL2:SDL_directsound.o
 0001:001cd510       _DSOUND_OpenDevice         005ce510 f   libSDL2:SDL_directsound.o
 0001:001cd980       _WINMM_GetDeviceBuf        005ce980 f   libSDL2:SDL_winmm.o
 0001:001cd9a0       _WINMM_Init                005ce9a0 f   libSDL2:SDL_winmm.o
 0001:001cd9e0       _WINMM_CloseDevice         005ce9e0 f   libSDL2:SDL_winmm.o
 0001:001cdaf0       _WINMM_WaitDone            005ceaf0 f   libSDL2:SDL_winmm.o
 0001:001cdb20       _WINMM_WaitDevice          005ceb20 f   libSDL2:SDL_winmm.o
 0001:001cdb50       _WINMM_PlayDevice          005ceb50 f   libSDL2:SDL_winmm.o
 0001:001cdbb0       _FillSound@20              005cebb0 f   libSDL2:SDL_winmm.o
 0001:001cdbf0       _CaptureSound@20           005cebf0 f   libSDL2:SDL_winmm.o
 0001:001cdc30       _SetMMerror                005cec30 f   libSDL2:SDL_winmm.o
 0001:001cdd00       _WINMM_OpenDevice          005ced00 f   libSDL2:SDL_winmm.o
 0001:001ce0d0       _WINMM_DetectDevices       005cf0d0 f   libSDL2:SDL_winmm.o
 0001:001ce240       _DISKAUD_GetDeviceBuf      005cf240 f   libSDL2:SDL_diskaudio.o
 0001:001ce250       _DISKAUD_Init              005cf250 f   libSDL2:SDL_diskaudio.o
 0001:001ce290       _DISKAUD_DetectDevices     005cf290 f   libSDL2:SDL_diskaudio.o
 0001:001ce2c0       _DISKAUD_CloseDevice       005cf2c0 f   libSDL2:SDL_diskaudio.o
 0001:001ce320       _DISKAUD_PlayDevice        005cf320 f   libSDL2:SDL_diskaudio.o
 0001:001ce370       _DISKAUD_WaitDevice        005cf370 f   libSDL2:SDL_diskaudio.o
 0001:001ce390       _DISKAUD_OpenDevice        005cf390 f   libSDL2:SDL_diskaudio.o
 0001:001ce510       _DUMMYAUD_OpenDevice       005cf510 f   libSDL2:SDL_dummyaudio.o
 0001:001ce520       _DUMMYAUD_Init             005cf520 f   libSDL2:SDL_dummyaudio.o
 0001:001ce540       _SDL_Convert_U8_to_S8      005cf540 f   libSDL2:SDL_audiotypecvt.o
 0001:001ce590       _SDL_Convert_U8_to_U16LSB  005cf590 f   libSDL2:SDL_audiotypecvt.o
 0001:001ce600       _SDL_Convert_U8_to_S16LSB  005cf600 f   libSDL2:SDL_audiotypecvt.o
 0001:001ce670       _SDL_Convert_U8_to_U16MSB  005cf670 f   libSDL2:SDL_audiotypecvt.o
 0001:001ce6e0       _SDL_Convert_U8_to_S16MSB  005cf6e0 f   libSDL2:SDL_audiotypecvt.o
 0001:001ce750       _SDL_Convert_U8_to_S32LSB  005cf750 f   libSDL2:SDL_audiotypecvt.o
 0001:001ce7d0       _SDL_Convert_U8_to_S32MSB  005cf7d0 f   libSDL2:SDL_audiotypecvt.o
 0001:001ce850       _SDL_Convert_U8_to_F32LSB  005cf850 f   libSDL2:SDL_audiotypecvt.o
 0001:001ce8e0       _SDL_Convert_U8_to_F32MSB  005cf8e0 f   libSDL2:SDL_audiotypecvt.o
 0001:001ce970       _SDL_Convert_S8_to_U8      005cf970 f   libSDL2:SDL_audiotypecvt.o
 0001:001ce9c0       _SDL_Convert_S8_to_U16LSB  005cf9c0 f   libSDL2:SDL_audiotypecvt.o
 0001:001cea30       _SDL_Convert_S8_to_S16LSB  005cfa30 f   libSDL2:SDL_audiotypecvt.o
 0001:001ceaa0       _SDL_Convert_S8_to_U16MSB  005cfaa0 f   libSDL2:SDL_audiotypecvt.o
 0001:001ceb10       _SDL_Convert_S8_to_S16MSB  005cfb10 f   libSDL2:SDL_audiotypecvt.o
 0001:001ceb80       _SDL_Convert_S8_to_S32LSB  005cfb80 f   libSDL2:SDL_audiotypecvt.o
 0001:001cec00       _SDL_Convert_S8_to_S32MSB  005cfc00 f   libSDL2:SDL_audiotypecvt.o
 0001:001cec70       _SDL_Convert_S8_to_F32LSB  005cfc70 f   libSDL2:SDL_audiotypecvt.o
 0001:001ced00       _SDL_Convert_S8_to_F32MSB  005cfd00 f   libSDL2:SDL_audiotypecvt.o
 0001:001ced90       _SDL_Convert_U16LSB_to_U8  005cfd90 f   libSDL2:SDL_audiotypecvt.o
 0001:001cedf0       _SDL_Convert_U16LSB_to_S8  005cfdf0 f   libSDL2:SDL_audiotypecvt.o
 0001:001cee50       _SDL_Convert_U16LSB_to_S16LSB 005cfe50 f   libSDL2:SDL_audiotypecvt.o
 0001:001ceea0       _SDL_Convert_U16LSB_to_U16MSB 005cfea0 f   libSDL2:SDL_audiotypecvt.o
 0001:001ceef0       _SDL_Convert_U16LSB_to_S16MSB 005cfef0 f   libSDL2:SDL_audiotypecvt.o
 0001:001cef40       _SDL_Convert_U16LSB_to_S32LSB 005cff40 f   libSDL2:SDL_audiotypecvt.o
 0001:001cefb0       _SDL_Convert_U16LSB_to_S32MSB 005cffb0 f   libSDL2:SDL_audiotypecvt.o
 0001:001cf020       _SDL_Convert_U16LSB_to_F32LSB 005d0020 f   libSDL2:SDL_audiotypecvt.o
 0001:001cf0b0       _SDL_Convert_U16LSB_to_F32MSB 005d00b0 f   libSDL2:SDL_audiotypecvt.o
 0001:001cf140       _SDL_Convert_S16LSB_to_U8  005d0140 f   libSDL2:SDL_audiotypecvt.o
 0001:001cf1a0       _SDL_Convert_S16LSB_to_S8  005d01a0 f   libSDL2:SDL_audiotypecvt.o
 0001:001cf200       _SDL_Convert_S16LSB_to_U16LSB 005d0200 f   libSDL2:SDL_audiotypecvt.o
 0001:001cf250       _SDL_Convert_S16LSB_to_U16MSB 005d0250 f   libSDL2:SDL_audiotypecvt.o
 0001:001cf2a0       _SDL_Convert_S16LSB_to_S16MSB 005d02a0 f   libSDL2:SDL_audiotypecvt.o
 0001:001cf2f0       _SDL_Convert_S16LSB_to_S32LSB 005d02f0 f   libSDL2:SDL_audiotypecvt.o
 0001:001cf360       _SDL_Convert_S16LSB_to_S32MSB 005d0360 f   libSDL2:SDL_audiotypecvt.o
 0001:001cf3d0       _SDL_Convert_S16LSB_to_F32LSB 005d03d0 f   libSDL2:SDL_audiotypecvt.o
 0001:001cf440       _SDL_Convert_S16LSB_to_F32MSB 005d0440 f   libSDL2:SDL_audiotypecvt.o
 0001:001cf4c0       _SDL_Convert_U16MSB_to_U8  005d04c0 f   libSDL2:SDL_audiotypecvt.o
 0001:001cf520       _SDL_Convert_U16MSB_to_S8  005d0520 f   libSDL2:SDL_audiotypecvt.o
 0001:001cf590       _SDL_Convert_U16MSB_to_U16LSB 005d0590 f   libSDL2:SDL_audiotypecvt.o
 0001:001cf5e0       _SDL_Convert_U16MSB_to_S16LSB 005d05e0 f   libSDL2:SDL_audiotypecvt.o
 0001:001cf630       _SDL_Convert_U16MSB_to_S16MSB 005d0630 f   libSDL2:SDL_audiotypecvt.o
 0001:001cf690       _SDL_Convert_U16MSB_to_S32LSB 005d0690 f   libSDL2:SDL_audiotypecvt.o
 0001:001cf700       _SDL_Convert_U16MSB_to_S32MSB 005d0700 f   libSDL2:SDL_audiotypecvt.o
 0001:001cf770       _SDL_Convert_U16MSB_to_F32LSB 005d0770 f   libSDL2:SDL_audiotypecvt.o
 0001:001cf800       _SDL_Convert_U16MSB_to_F32MSB 005d0800 f   libSDL2:SDL_audiotypecvt.o
 0001:001cf8a0       _SDL_Convert_S16MSB_to_U8  005d08a0 f   libSDL2:SDL_audiotypecvt.o
 0001:001cf910       _SDL_Convert_S16MSB_to_S8  005d0910 f   libSDL2:SDL_audiotypecvt.o
 0001:001cf970       _SDL_Convert_S16MSB_to_U16LSB 005d0970 f   libSDL2:SDL_audiotypecvt.o
 0001:001cf9c0       _SDL_Convert_S16MSB_to_S16LSB 005d09c0 f   libSDL2:SDL_audiotypecvt.o
 0001:001cfa10       _SDL_Convert_S16MSB_to_U16MSB 005d0a10 f   libSDL2:SDL_audiotypecvt.o
 0001:001cfa70       _SDL_Convert_S16MSB_to_S32LSB 005d0a70 f   libSDL2:SDL_audiotypecvt.o
 0001:001cfae0       _SDL_Convert_S16MSB_to_S32MSB 005d0ae0 f   libSDL2:SDL_audiotypecvt.o
 0001:001cfb50       _SDL_Convert_S16MSB_to_F32LSB 005d0b50 f   libSDL2:SDL_audiotypecvt.o
 0001:001cfbd0       _SDL_Convert_S16MSB_to_F32MSB 005d0bd0 f   libSDL2:SDL_audiotypecvt.o
 0001:001cfc60       _SDL_Convert_S32LSB_to_U8  005d0c60 f   libSDL2:SDL_audiotypecvt.o
 0001:001cfcd0       _SDL_Convert_S32LSB_to_S8  005d0cd0 f   libSDL2:SDL_audiotypecvt.o
 0001:001cfd30       _SDL_Convert_S32LSB_to_U16LSB 005d0d30 f   libSDL2:SDL_audiotypecvt.o
 0001:001cfda0       _SDL_Convert_S32LSB_to_S16LSB 005d0da0 f   libSDL2:SDL_audiotypecvt.o
 0001:001cfe10       _SDL_Convert_S32LSB_to_U16MSB 005d0e10 f   libSDL2:SDL_audiotypecvt.o
 0001:001cfe80       _SDL_Convert_S32LSB_to_S16MSB 005d0e80 f   libSDL2:SDL_audiotypecvt.o
 0001:001cfef0       _SDL_Convert_S32LSB_to_S32MSB 005d0ef0 f   libSDL2:SDL_audiotypecvt.o
 0001:001cff40       _SDL_Convert_S32LSB_to_F32LSB 005d0f40 f   libSDL2:SDL_audiotypecvt.o
 0001:001cff90       _SDL_Convert_S32LSB_to_F32MSB 005d0f90 f   libSDL2:SDL_audiotypecvt.o
 0001:001d0000       _SDL_Convert_S32MSB_to_U8  005d1000 f   libSDL2:SDL_audiotypecvt.o
 0001:001d0070       _SDL_Convert_S32MSB_to_S8  005d1070 f   libSDL2:SDL_audiotypecvt.o
 0001:001d00e0       _SDL_Convert_S32MSB_to_U16LSB 005d10e0 f   libSDL2:SDL_audiotypecvt.o
 0001:001d0150       _SDL_Convert_S32MSB_to_S16LSB 005d1150 f   libSDL2:SDL_audiotypecvt.o
 0001:001d01c0       _SDL_Convert_S32MSB_to_U16MSB 005d11c0 f   libSDL2:SDL_audiotypecvt.o
 0001:001d0240       _SDL_Convert_S32MSB_to_S16MSB 005d1240 f   libSDL2:SDL_audiotypecvt.o
 0001:001d02b0       _SDL_Convert_S32MSB_to_S32LSB 005d12b0 f   libSDL2:SDL_audiotypecvt.o
 0001:001d0300       _SDL_Convert_S32MSB_to_F32LSB 005d1300 f   libSDL2:SDL_audiotypecvt.o
 0001:001d0370       _SDL_Convert_S32MSB_to_F32MSB 005d1370 f   libSDL2:SDL_audiotypecvt.o
 0001:001d03e0       _SDL_Convert_F32LSB_to_U8  005d13e0 f   libSDL2:SDL_audiotypecvt.o
 0001:001d0460       _SDL_Convert_F32LSB_to_S8  005d1460 f   libSDL2:SDL_audiotypecvt.o
 0001:001d04e0       _SDL_Convert_F32LSB_to_U16LSB 005d14e0 f   libSDL2:SDL_audiotypecvt.o
 0001:001d0560       _SDL_Convert_F32LSB_to_S16LSB 005d1560 f   libSDL2:SDL_audiotypecvt.o
 0001:001d05e0       _SDL_Convert_F32LSB_to_U16MSB 005d15e0 f   libSDL2:SDL_audiotypecvt.o
 0001:001d0660       _SDL_Convert_F32LSB_to_S16MSB 005d1660 f   libSDL2:SDL_audiotypecvt.o
 0001:001d06e0       _SDL_Convert_F32LSB_to_S32LSB 005d16e0 f   libSDL2:SDL_audiotypecvt.o
 0001:001d0760       _SDL_Convert_F32LSB_to_S32MSB 005d1760 f   libSDL2:SDL_audiotypecvt.o
 0001:001d07e0       _SDL_Convert_F32LSB_to_F32MSB 005d17e0 f   libSDL2:SDL_audiotypecvt.o
 0001:001d0830       _SDL_Convert_F32MSB_to_U8  005d1830 f   libSDL2:SDL_audiotypecvt.o
 0001:001d08c0       _SDL_Convert_F32MSB_to_S8  005d18c0 f   libSDL2:SDL_audiotypecvt.o
 0001:001d0940       _SDL_Convert_F32MSB_to_U16LSB 005d1940 f   libSDL2:SDL_audiotypecvt.o
 0001:001d09d0       _SDL_Convert_F32MSB_to_S16LSB 005d19d0 f   libSDL2:SDL_audiotypecvt.o
 0001:001d0a50       _SDL_Convert_F32MSB_to_U16MSB 005d1a50 f   libSDL2:SDL_audiotypecvt.o
 0001:001d0ae0       _SDL_Convert_F32MSB_to_S16MSB 005d1ae0 f   libSDL2:SDL_audiotypecvt.o
 0001:001d0b60       _SDL_Convert_F32MSB_to_S32LSB 005d1b60 f   libSDL2:SDL_audiotypecvt.o
 0001:001d0be0       _SDL_Convert_F32MSB_to_S32MSB 005d1be0 f   libSDL2:SDL_audiotypecvt.o
 0001:001d0c70       _SDL_Convert_F32MSB_to_F32LSB 005d1c70 f   libSDL2:SDL_audiotypecvt.o
 0001:001d0cc0       _SDL_Upsample_U8_1c        005d1cc0 f   libSDL2:SDL_audiotypecvt.o
 0001:001d0d90       _SDL_Downsample_U8_1c      005d1d90 f   libSDL2:SDL_audiotypecvt.o
 0001:001d0e70       _SDL_Upsample_U8_2c        005d1e70 f   libSDL2:SDL_audiotypecvt.o
 0001:001d0f70       _SDL_Downsample_U8_2c      005d1f70 f   libSDL2:SDL_audiotypecvt.o
 0001:001d1090       _SDL_Upsample_U8_4c        005d2090 f   libSDL2:SDL_audiotypecvt.o
 0001:001d11e0       _SDL_Downsample_U8_4c      005d21e0 f   libSDL2:SDL_audiotypecvt.o
 0001:001d1330       _SDL_Upsample_U8_6c        005d2330 f   libSDL2:SDL_audiotypecvt.o
 0001:001d14d0       _SDL_Downsample_U8_6c      005d24d0 f   libSDL2:SDL_audiotypecvt.o
 0001:001d1670       _SDL_Upsample_U8_8c        005d2670 f   libSDL2:SDL_audiotypecvt.o
 0001:001d1880       _SDL_Downsample_U8_8c      005d2880 f   libSDL2:SDL_audiotypecvt.o
 0001:001d1a90       _SDL_Upsample_S8_1c        005d2a90 f   libSDL2:SDL_audiotypecvt.o
 0001:001d1b60       _SDL_Downsample_S8_1c      005d2b60 f   libSDL2:SDL_audiotypecvt.o
 0001:001d1c40       _SDL_Upsample_S8_2c        005d2c40 f   libSDL2:SDL_audiotypecvt.o
 0001:001d1d40       _SDL_Downsample_S8_2c      005d2d40 f   libSDL2:SDL_audiotypecvt.o
 0001:001d1e60       _SDL_Upsample_S8_4c        005d2e60 f   libSDL2:SDL_audiotypecvt.o
 0001:001d1fb0       _SDL_Downsample_S8_4c      005d2fb0 f   libSDL2:SDL_audiotypecvt.o
 0001:001d2100       _SDL_Upsample_S8_6c        005d3100 f   libSDL2:SDL_audiotypecvt.o
 0001:001d22a0       _SDL_Downsample_S8_6c      005d32a0 f   libSDL2:SDL_audiotypecvt.o
 0001:001d2440       _SDL_Upsample_S8_8c        005d3440 f   libSDL2:SDL_audiotypecvt.o
 0001:001d2650       _SDL_Downsample_S8_8c      005d3650 f   libSDL2:SDL_audiotypecvt.o
 0001:001d2860       _SDL_Upsample_U16LSB_1c    005d3860 f   libSDL2:SDL_audiotypecvt.o
 0001:001d2930       _SDL_Downsample_U16LSB_1c  005d3930 f   libSDL2:SDL_audiotypecvt.o
 0001:001d2a00       _SDL_Upsample_U16LSB_2c    005d3a00 f   libSDL2:SDL_audiotypecvt.o
 0001:001d2b00       _SDL_Downsample_U16LSB_2c  005d3b00 f   libSDL2:SDL_audiotypecvt.o
 0001:001d2c00       _SDL_Upsample_U16LSB_4c    005d3c00 f   libSDL2:SDL_audiotypecvt.o
 0001:001d2d50       _SDL_Downsample_U16LSB_4c  005d3d50 f   libSDL2:SDL_audiotypecvt.o
 0001:001d2ea0       _SDL_Upsample_U16LSB_6c    005d3ea0 f   libSDL2:SDL_audiotypecvt.o
 0001:001d3050       _SDL_Downsample_U16LSB_6c  005d4050 f   libSDL2:SDL_audiotypecvt.o
 0001:001d31f0       _SDL_Upsample_U16LSB_8c    005d41f0 f   libSDL2:SDL_audiotypecvt.o
 0001:001d3410       _SDL_Downsample_U16LSB_8c  005d4410 f   libSDL2:SDL_audiotypecvt.o
 0001:001d3620       _SDL_Upsample_S16LSB_1c    005d4620 f   libSDL2:SDL_audiotypecvt.o
 0001:001d36f0       _SDL_Downsample_S16LSB_1c  005d46f0 f   libSDL2:SDL_audiotypecvt.o
 0001:001d37c0       _SDL_Upsample_S16LSB_2c    005d47c0 f   libSDL2:SDL_audiotypecvt.o
 0001:001d38c0       _SDL_Downsample_S16LSB_2c  005d48c0 f   libSDL2:SDL_audiotypecvt.o
 0001:001d39c0       _SDL_Upsample_S16LSB_4c    005d49c0 f   libSDL2:SDL_audiotypecvt.o
 0001:001d3b10       _SDL_Downsample_S16LSB_4c  005d4b10 f   libSDL2:SDL_audiotypecvt.o
 0001:001d3c60       _SDL_Upsample_S16LSB_6c    005d4c60 f   libSDL2:SDL_audiotypecvt.o
 0001:001d3e10       _SDL_Downsample_S16LSB_6c  005d4e10 f   libSDL2:SDL_audiotypecvt.o
 0001:001d3fb0       _SDL_Upsample_S16LSB_8c    005d4fb0 f   libSDL2:SDL_audiotypecvt.o
 0001:001d41d0       _SDL_Downsample_S16LSB_8c  005d51d0 f   libSDL2:SDL_audiotypecvt.o
 0001:001d43e0       _SDL_Upsample_U16MSB_1c    005d53e0 f   libSDL2:SDL_audiotypecvt.o
 0001:001d44c0       _SDL_Downsample_U16MSB_1c  005d54c0 f   libSDL2:SDL_audiotypecvt.o
 0001:001d45b0       _SDL_Upsample_U16MSB_2c    005d55b0 f   libSDL2:SDL_audiotypecvt.o
 0001:001d46d0       _SDL_Downsample_U16MSB_2c  005d56d0 f   libSDL2:SDL_audiotypecvt.o
 0001:001d47f0       _SDL_Upsample_U16MSB_4c    005d57f0 f   libSDL2:SDL_audiotypecvt.o
 0001:001d4990       _SDL_Downsample_U16MSB_4c  005d5990 f   libSDL2:SDL_audiotypecvt.o
 0001:001d4b30       _SDL_Upsample_U16MSB_6c    005d5b30 f   libSDL2:SDL_audiotypecvt.o
 0001:001d4d40       _SDL_Downsample_U16MSB_6c  005d5d40 f   libSDL2:SDL_audiotypecvt.o
 0001:001d4f50       _SDL_Upsample_U16MSB_8c    005d5f50 f   libSDL2:SDL_audiotypecvt.o
 0001:001d51f0       _SDL_Downsample_U16MSB_8c  005d61f0 f   libSDL2:SDL_audiotypecvt.o
 0001:001d5490       _SDL_Upsample_S16MSB_1c    005d6490 f   libSDL2:SDL_audiotypecvt.o
 0001:001d5570       _SDL_Downsample_S16MSB_1c  005d6570 f   libSDL2:SDL_audiotypecvt.o
 0001:001d5660       _SDL_Upsample_S16MSB_2c    005d6660 f   libSDL2:SDL_audiotypecvt.o
 0001:001d5780       _SDL_Downsample_S16MSB_2c  005d6780 f   libSDL2:SDL_audiotypecvt.o
 0001:001d58a0       _SDL_Upsample_S16MSB_4c    005d68a0 f   libSDL2:SDL_audiotypecvt.o
 0001:001d5a40       _SDL_Downsample_S16MSB_4c  005d6a40 f   libSDL2:SDL_audiotypecvt.o
 0001:001d5be0       _SDL_Upsample_S16MSB_6c    005d6be0 f   libSDL2:SDL_audiotypecvt.o
 0001:001d5df0       _SDL_Downsample_S16MSB_6c  005d6df0 f   libSDL2:SDL_audiotypecvt.o
 0001:001d6000       _SDL_Upsample_S16MSB_8c    005d7000 f   libSDL2:SDL_audiotypecvt.o
 0001:001d62a0       _SDL_Downsample_S16MSB_8c  005d72a0 f   libSDL2:SDL_audiotypecvt.o
 0001:001d6540       _SDL_Upsample_S32LSB_1c    005d7540 f   libSDL2:SDL_audiotypecvt.o
 0001:001d6660       _SDL_Downsample_S32LSB_1c  005d7660 f   libSDL2:SDL_audiotypecvt.o
 0001:001d6770       _SDL_Upsample_S32LSB_2c    005d7770 f   libSDL2:SDL_audiotypecvt.o
 0001:001d68c0       _SDL_Downsample_S32LSB_2c  005d78c0 f   libSDL2:SDL_audiotypecvt.o
 0001:001d69f0       _SDL_Upsample_S32LSB_4c    005d79f0 f   libSDL2:SDL_audiotypecvt.o
 0001:001d6b80       _SDL_Downsample_S32LSB_4c  005d7b80 f   libSDL2:SDL_audiotypecvt.o
 0001:001d6d10       _SDL_Upsample_S32LSB_6c    005d7d10 f   libSDL2:SDL_audiotypecvt.o
 0001:001d6f00       _SDL_Downsample_S32LSB_6c  005d7f00 f   libSDL2:SDL_audiotypecvt.o
 0001:001d70e0       _SDL_Upsample_S32LSB_8c    005d80e0 f   libSDL2:SDL_audiotypecvt.o
 0001:001d7310       _SDL_Downsample_S32LSB_8c  005d8310 f   libSDL2:SDL_audiotypecvt.o
 0001:001d7530       _SDL_Upsample_S32MSB_1c    005d8530 f   libSDL2:SDL_audiotypecvt.o
 0001:001d7630       _SDL_Downsample_S32MSB_1c  005d8630 f   libSDL2:SDL_audiotypecvt.o
 0001:001d7740       _SDL_Upsample_S32MSB_2c    005d8740 f   libSDL2:SDL_audiotypecvt.o
 0001:001d78a0       _SDL_Downsample_S32MSB_2c  005d88a0 f   libSDL2:SDL_audiotypecvt.o
 0001:001d79e0       _SDL_Upsample_S32MSB_4c    005d89e0 f   libSDL2:SDL_audiotypecvt.o
 0001:001d7b90       _SDL_Downsample_S32MSB_4c  005d8b90 f   libSDL2:SDL_audiotypecvt.o
 0001:001d7d30       _SDL_Upsample_S32MSB_6c    005d8d30 f   libSDL2:SDL_audiotypecvt.o
 0001:001d7f40       _SDL_Downsample_S32MSB_6c  005d8f40 f   libSDL2:SDL_audiotypecvt.o
 0001:001d8140       _SDL_Upsample_S32MSB_8c    005d9140 f   libSDL2:SDL_audiotypecvt.o
 0001:001d83a0       _SDL_Downsample_S32MSB_8c  005d93a0 f   libSDL2:SDL_audiotypecvt.o
 0001:001d85f0       _SDL_Upsample_F32LSB_1c    005d95f0 f   libSDL2:SDL_audiotypecvt.o
 0001:001d86e0       _SDL_Downsample_F32LSB_1c  005d96e0 f   libSDL2:SDL_audiotypecvt.o
 0001:001d87c0       _SDL_Upsample_F32LSB_2c    005d97c0 f   libSDL2:SDL_audiotypecvt.o
 0001:001d88d0       _SDL_Downsample_F32LSB_2c  005d98d0 f   libSDL2:SDL_audiotypecvt.o
 0001:001d89d0       _SDL_Upsample_F32LSB_4c    005d99d0 f   libSDL2:SDL_audiotypecvt.o
 0001:001d8b30       _SDL_Downsample_F32LSB_4c  005d9b30 f   libSDL2:SDL_audiotypecvt.o
 0001:001d8c80       _SDL_Upsample_F32LSB_6c    005d9c80 f   libSDL2:SDL_audiotypecvt.o
 0001:001d8e20       _SDL_Downsample_F32LSB_6c  005d9e20 f   libSDL2:SDL_audiotypecvt.o
 0001:001d8fb0       _SDL_Upsample_F32LSB_8c    005d9fb0 f   libSDL2:SDL_audiotypecvt.o
 0001:001d9190       _SDL_Downsample_F32LSB_8c  005da190 f   libSDL2:SDL_audiotypecvt.o
 0001:001d9350       _SDL_Upsample_F32MSB_1c    005da350 f   libSDL2:SDL_audiotypecvt.o
 0001:001d9440       _SDL_Downsample_F32MSB_1c  005da440 f   libSDL2:SDL_audiotypecvt.o
 0001:001d9530       _SDL_Upsample_F32MSB_2c    005da530 f   libSDL2:SDL_audiotypecvt.o
 0001:001d9650       _SDL_Downsample_F32MSB_2c  005da650 f   libSDL2:SDL_audiotypecvt.o
 0001:001d9770       _SDL_Upsample_F32MSB_4c    005da770 f   libSDL2:SDL_audiotypecvt.o
 0001:001d98f0       _SDL_Downsample_F32MSB_4c  005da8f0 f   libSDL2:SDL_audiotypecvt.o
 0001:001d9a70       _SDL_Upsample_F32MSB_6c    005daa70 f   libSDL2:SDL_audiotypecvt.o
 0001:001d9c50       _SDL_Downsample_F32MSB_6c  005dac50 f   libSDL2:SDL_audiotypecvt.o
 0001:001d9e30       _SDL_Upsample_F32MSB_8c    005dae30 f   libSDL2:SDL_audiotypecvt.o
 0001:001da050       _SDL_Downsample_F32MSB_8c  005db050 f   libSDL2:SDL_audiotypecvt.o
 0001:001da270       _SDL_Upsample_U8_1c_x2     005db270 f   libSDL2:SDL_audiotypecvt.o
 0001:001da300       _SDL_Downsample_U8_1c_x2   005db300 f   libSDL2:SDL_audiotypecvt.o
 0001:001da390       _SDL_Upsample_U8_1c_x4     005db390 f   libSDL2:SDL_audiotypecvt.o
 0001:001da460       _SDL_Downsample_U8_1c_x4   005db460 f   libSDL2:SDL_audiotypecvt.o
 0001:001da4f0       _SDL_Upsample_U8_2c_x2     005db4f0 f   libSDL2:SDL_audiotypecvt.o
 0001:001da5b0       _SDL_Downsample_U8_2c_x2   005db5b0 f   libSDL2:SDL_audiotypecvt.o
 0001:001da670       _SDL_Upsample_U8_2c_x4     005db670 f   libSDL2:SDL_audiotypecvt.o
 0001:001da7a0       _SDL_Downsample_U8_2c_x4   005db7a0 f   libSDL2:SDL_audiotypecvt.o
 0001:001da860       _SDL_Upsample_U8_4c_x2     005db860 f   libSDL2:SDL_audiotypecvt.o
 0001:001da9b0       _SDL_Downsample_U8_4c_x2   005db9b0 f   libSDL2:SDL_audiotypecvt.o
 0001:001daaf0       _SDL_Upsample_U8_4c_x4     005dbaf0 f   libSDL2:SDL_audiotypecvt.o
 0001:001dad10       _SDL_Downsample_U8_4c_x4   005dbd10 f   libSDL2:SDL_audiotypecvt.o
 0001:001dae50       _SDL_Upsample_U8_6c_x2     005dbe50 f   libSDL2:SDL_audiotypecvt.o
 0001:001db050       _SDL_Downsample_U8_6c_x2   005dc050 f   libSDL2:SDL_audiotypecvt.o
 0001:001db210       _SDL_Upsample_U8_6c_x4     005dc210 f   libSDL2:SDL_audiotypecvt.o
 0001:001db510       _SDL_Downsample_U8_6c_x4   005dc510 f   libSDL2:SDL_audiotypecvt.o
 0001:001db6d0       _SDL_Upsample_U8_8c_x2     005dc6d0 f   libSDL2:SDL_audiotypecvt.o
 0001:001db900       _SDL_Downsample_U8_8c_x2   005dc900 f   libSDL2:SDL_audiotypecvt.o
 0001:001dbb20       _SDL_Upsample_U8_8c_x4     005dcb20 f   libSDL2:SDL_audiotypecvt.o
 0001:001dbf20       _SDL_Downsample_U8_8c_x4   005dcf20 f   libSDL2:SDL_audiotypecvt.o
 0001:001dc140       _SDL_Upsample_S8_1c_x2     005dd140 f   libSDL2:SDL_audiotypecvt.o
 0001:001dc1d0       _SDL_Downsample_S8_1c_x2   005dd1d0 f   libSDL2:SDL_audiotypecvt.o
 0001:001dc260       _SDL_Upsample_S8_1c_x4     005dd260 f   libSDL2:SDL_audiotypecvt.o
 0001:001dc330       _SDL_Downsample_S8_1c_x4   005dd330 f   libSDL2:SDL_audiotypecvt.o
 0001:001dc3c0       _SDL_Upsample_S8_2c_x2     005dd3c0 f   libSDL2:SDL_audiotypecvt.o
 0001:001dc480       _SDL_Downsample_S8_2c_x2   005dd480 f   libSDL2:SDL_audiotypecvt.o
 0001:001dc540       _SDL_Upsample_S8_2c_x4     005dd540 f   libSDL2:SDL_audiotypecvt.o
 0001:001dc670       _SDL_Downsample_S8_2c_x4   005dd670 f   libSDL2:SDL_audiotypecvt.o
 0001:001dc730       _SDL_Upsample_S8_4c_x2     005dd730 f   libSDL2:SDL_audiotypecvt.o
 0001:001dc880       _SDL_Downsample_S8_4c_x2   005dd880 f   libSDL2:SDL_audiotypecvt.o
 0001:001dc9d0       _SDL_Upsample_S8_4c_x4     005dd9d0 f   libSDL2:SDL_audiotypecvt.o
 0001:001dcbf0       _SDL_Downsample_S8_4c_x4   005ddbf0 f   libSDL2:SDL_audiotypecvt.o
 0001:001dcd40       _SDL_Upsample_S8_6c_x2     005ddd40 f   libSDL2:SDL_audiotypecvt.o
 0001:001dcf40       _SDL_Downsample_S8_6c_x2   005ddf40 f   libSDL2:SDL_audiotypecvt.o
 0001:001dd110       _SDL_Upsample_S8_6c_x4     005de110 f   libSDL2:SDL_audiotypecvt.o
 0001:001dd430       _SDL_Downsample_S8_6c_x4   005de430 f   libSDL2:SDL_audiotypecvt.o
 0001:001dd600       _SDL_Upsample_S8_8c_x2     005de600 f   libSDL2:SDL_audiotypecvt.o
 0001:001dd840       _SDL_Downsample_S8_8c_x2   005de840 f   libSDL2:SDL_audiotypecvt.o
 0001:001dda60       _SDL_Upsample_S8_8c_x4     005dea60 f   libSDL2:SDL_audiotypecvt.o
 0001:001dde70       _SDL_Downsample_S8_8c_x4   005dee70 f   libSDL2:SDL_audiotypecvt.o
 0001:001de090       _SDL_Upsample_U16LSB_1c_x2 005df090 f   libSDL2:SDL_audiotypecvt.o
 0001:001de120       _SDL_Downsample_U16LSB_1c_x2 005df120 f   libSDL2:SDL_audiotypecvt.o
 0001:001de1a0       _SDL_Upsample_U16LSB_1c_x4 005df1a0 f   libSDL2:SDL_audiotypecvt.o
 0001:001de250       _SDL_Downsample_U16LSB_1c_x4 005df250 f   libSDL2:SDL_audiotypecvt.o
 0001:001de2d0       _SDL_Upsample_U16LSB_2c_x2 005df2d0 f   libSDL2:SDL_audiotypecvt.o
 0001:001de380       _SDL_Downsample_U16LSB_2c_x2 005df380 f   libSDL2:SDL_audiotypecvt.o
 0001:001de420       _SDL_Upsample_U16LSB_2c_x4 005df420 f   libSDL2:SDL_audiotypecvt.o
 0001:001de510       _SDL_Downsample_U16LSB_2c_x4 005df510 f   libSDL2:SDL_audiotypecvt.o
 0001:001de5c0       _SDL_Upsample_U16LSB_4c_x2 005df5c0 f   libSDL2:SDL_audiotypecvt.o
 0001:001de6e0       _SDL_Downsample_U16LSB_4c_x2 005df6e0 f   libSDL2:SDL_audiotypecvt.o
 0001:001de7d0       _SDL_Upsample_U16LSB_4c_x4 005df7d0 f   libSDL2:SDL_audiotypecvt.o
 0001:001de980       _SDL_Downsample_U16LSB_4c_x4 005df980 f   libSDL2:SDL_audiotypecvt.o
 0001:001dea70       _SDL_Upsample_U16LSB_6c_x2 005dfa70 f   libSDL2:SDL_audiotypecvt.o
 0001:001dec00       _SDL_Downsample_U16LSB_6c_x2 005dfc00 f   libSDL2:SDL_audiotypecvt.o
 0001:001ded40       _SDL_Upsample_U16LSB_6c_x4 005dfd40 f   libSDL2:SDL_audiotypecvt.o
 0001:001defa0       _SDL_Downsample_U16LSB_6c_x4 005dffa0 f   libSDL2:SDL_audiotypecvt.o
 0001:001df0e0       _SDL_Upsample_U16LSB_8c_x2 005e00e0 f   libSDL2:SDL_audiotypecvt.o
 0001:001df2e0       _SDL_Downsample_U16LSB_8c_x2 005e02e0 f   libSDL2:SDL_audiotypecvt.o
 0001:001df470       _SDL_Upsample_U16LSB_8c_x4 005e0470 f   libSDL2:SDL_audiotypecvt.o
 0001:001df7a0       _SDL_Downsample_U16LSB_8c_x4 005e07a0 f   libSDL2:SDL_audiotypecvt.o
 0001:001df930       _SDL_Upsample_S16LSB_1c_x2 005e0930 f   libSDL2:SDL_audiotypecvt.o
 0001:001df9c0       _SDL_Downsample_S16LSB_1c_x2 005e09c0 f   libSDL2:SDL_audiotypecvt.o
 0001:001dfa40       _SDL_Upsample_S16LSB_1c_x4 005e0a40 f   libSDL2:SDL_audiotypecvt.o
 0001:001dfaf0       _SDL_Downsample_S16LSB_1c_x4 005e0af0 f   libSDL2:SDL_audiotypecvt.o
 0001:001dfb70       _SDL_Upsample_S16LSB_2c_x2 005e0b70 f   libSDL2:SDL_audiotypecvt.o
 0001:001dfc20       _SDL_Downsample_S16LSB_2c_x2 005e0c20 f   libSDL2:SDL_audiotypecvt.o
 0001:001dfcc0       _SDL_Upsample_S16LSB_2c_x4 005e0cc0 f   libSDL2:SDL_audiotypecvt.o
 0001:001dfdb0       _SDL_Downsample_S16LSB_2c_x4 005e0db0 f   libSDL2:SDL_audiotypecvt.o
 0001:001dfe60       _SDL_Upsample_S16LSB_4c_x2 005e0e60 f   libSDL2:SDL_audiotypecvt.o
 0001:001dff80       _SDL_Downsample_S16LSB_4c_x2 005e0f80 f   libSDL2:SDL_audiotypecvt.o
 0001:001e0070       _SDL_Upsample_S16LSB_4c_x4 005e1070 f   libSDL2:SDL_audiotypecvt.o
 0001:001e0220       _SDL_Downsample_S16LSB_4c_x4 005e1220 f   libSDL2:SDL_audiotypecvt.o
 0001:001e0310       _SDL_Upsample_S16LSB_6c_x2 005e1310 f   libSDL2:SDL_audiotypecvt.o
 0001:001e04a0       _SDL_Downsample_S16LSB_6c_x2 005e14a0 f   libSDL2:SDL_audiotypecvt.o
 0001:001e05e0       _SDL_Upsample_S16LSB_6c_x4 005e15e0 f   libSDL2:SDL_audiotypecvt.o
 0001:001e0840       _SDL_Downsample_S16LSB_6c_x4 005e1840 f   libSDL2:SDL_audiotypecvt.o
 0001:001e0980       _SDL_Upsample_S16LSB_8c_x2 005e1980 f   libSDL2:SDL_audiotypecvt.o
 0001:001e0b80       _SDL_Downsample_S16LSB_8c_x2 005e1b80 f   libSDL2:SDL_audiotypecvt.o
 0001:001e0d10       _SDL_Upsample_S16LSB_8c_x4 005e1d10 f   libSDL2:SDL_audiotypecvt.o
 0001:001e1020       _SDL_Downsample_S16LSB_8c_x4 005e2020 f   libSDL2:SDL_audiotypecvt.o
 0001:001e11b0       _SDL_Upsample_U16MSB_1c_x2 005e21b0 f   libSDL2:SDL_audiotypecvt.o
 0001:001e1240       _SDL_Downsample_U16MSB_1c_x2 005e2240 f   libSDL2:SDL_audiotypecvt.o
 0001:001e12d0       _SDL_Upsample_U16MSB_1c_x4 005e22d0 f   libSDL2:SDL_audiotypecvt.o
 0001:001e1390       _SDL_Downsample_U16MSB_1c_x4 005e2390 f   libSDL2:SDL_audiotypecvt.o
 0001:001e1420       _SDL_Upsample_U16MSB_2c_x2 005e2420 f   libSDL2:SDL_audiotypecvt.o
 0001:001e14f0       _SDL_Downsample_U16MSB_2c_x2 005e24f0 f   libSDL2:SDL_audiotypecvt.o
 0001:001e15c0       _SDL_Upsample_U16MSB_2c_x4 005e25c0 f   libSDL2:SDL_audiotypecvt.o
 0001:001e16d0       _SDL_Downsample_U16MSB_2c_x4 005e26d0 f   libSDL2:SDL_audiotypecvt.o
 0001:001e17a0       _SDL_Upsample_U16MSB_4c_x2 005e27a0 f   libSDL2:SDL_audiotypecvt.o
 0001:001e1900       _SDL_Downsample_U16MSB_4c_x2 005e2900 f   libSDL2:SDL_audiotypecvt.o
 0001:001e1a30       _SDL_Upsample_U16MSB_4c_x4 005e2a30 f   libSDL2:SDL_audiotypecvt.o
 0001:001e1c00       _SDL_Downsample_U16MSB_4c_x4 005e2c00 f   libSDL2:SDL_audiotypecvt.o
 0001:001e1d30       _SDL_Upsample_U16MSB_6c_x2 005e2d30 f   libSDL2:SDL_audiotypecvt.o
 0001:001e1f10       _SDL_Downsample_U16MSB_6c_x2 005e2f10 f   libSDL2:SDL_audiotypecvt.o
 0001:001e20a0       _SDL_Upsample_U16MSB_6c_x4 005e30a0 f   libSDL2:SDL_audiotypecvt.o
 0001:001e2340       _SDL_Downsample_U16MSB_6c_x4 005e3340 f   libSDL2:SDL_audiotypecvt.o
 0001:001e24d0       _SDL_Upsample_U16MSB_8c_x2 005e34d0 f   libSDL2:SDL_audiotypecvt.o
 0001:001e2720       _SDL_Downsample_U16MSB_8c_x2 005e3720 f   libSDL2:SDL_audiotypecvt.o
 0001:001e2910       _SDL_Upsample_U16MSB_8c_x4 005e3910 f   libSDL2:SDL_audiotypecvt.o
 0001:001e2ca0       _SDL_Downsample_U16MSB_8c_x4 005e3ca0 f   libSDL2:SDL_audiotypecvt.o
 0001:001e2e90       _SDL_Upsample_S16MSB_1c_x2 005e3e90 f   libSDL2:SDL_audiotypecvt.o
 0001:001e2f20       _SDL_Downsample_S16MSB_1c_x2 005e3f20 f   libSDL2:SDL_audiotypecvt.o
 0001:001e2fb0       _SDL_Upsample_S16MSB_1c_x4 005e3fb0 f   libSDL2:SDL_audiotypecvt.o
 0001:001e3070       _SDL_Downsample_S16MSB_1c_x4 005e4070 f   libSDL2:SDL_audiotypecvt.o
 0001:001e3100       _SDL_Upsample_S16MSB_2c_x2 005e4100 f   libSDL2:SDL_audiotypecvt.o
 0001:001e31d0       _SDL_Downsample_S16MSB_2c_x2 005e41d0 f   libSDL2:SDL_audiotypecvt.o
 0001:001e32a0       _SDL_Upsample_S16MSB_2c_x4 005e42a0 f   libSDL2:SDL_audiotypecvt.o
 0001:001e33b0       _SDL_Downsample_S16MSB_2c_x4 005e43b0 f   libSDL2:SDL_audiotypecvt.o
 0001:001e3480       _SDL_Upsample_S16MSB_4c_x2 005e4480 f   libSDL2:SDL_audiotypecvt.o
 0001:001e35d0       _SDL_Downsample_S16MSB_4c_x2 005e45d0 f   libSDL2:SDL_audiotypecvt.o
 0001:001e3700       _SDL_Upsample_S16MSB_4c_x4 005e4700 f   libSDL2:SDL_audiotypecvt.o
 0001:001e38e0       _SDL_Downsample_S16MSB_4c_x4 005e48e0 f   libSDL2:SDL_audiotypecvt.o
 0001:001e3a10       _SDL_Upsample_S16MSB_6c_x2 005e4a10 f   libSDL2:SDL_audiotypecvt.o
 0001:001e3be0       _SDL_Downsample_S16MSB_6c_x2 005e4be0 f   libSDL2:SDL_audiotypecvt.o
 0001:001e3d70       _SDL_Upsample_S16MSB_6c_x4 005e4d70 f   libSDL2:SDL_audiotypecvt.o
 0001:001e4000       _SDL_Downsample_S16MSB_6c_x4 005e5000 f   libSDL2:SDL_audiotypecvt.o
 0001:001e4190       _SDL_Upsample_S16MSB_8c_x2 005e5190 f   libSDL2:SDL_audiotypecvt.o
 0001:001e43d0       _SDL_Downsample_S16MSB_8c_x2 005e53d0 f   libSDL2:SDL_audiotypecvt.o
 0001:001e45a0       _SDL_Upsample_S16MSB_8c_x4 005e55a0 f   libSDL2:SDL_audiotypecvt.o
 0001:001e48f0       _SDL_Downsample_S16MSB_8c_x4 005e58f0 f   libSDL2:SDL_audiotypecvt.o
 0001:001e4ac0       _SDL_Upsample_S32LSB_1c_x2 005e5ac0 f   libSDL2:SDL_audiotypecvt.o
 0001:001e4b60       _SDL_Downsample_S32LSB_1c_x2 005e5b60 f   libSDL2:SDL_audiotypecvt.o
 0001:001e4c00       _SDL_Upsample_S32LSB_1c_x4 005e5c00 f   libSDL2:SDL_audiotypecvt.o
 0001:001e4d00       _SDL_Downsample_S32LSB_1c_x4 005e5d00 f   libSDL2:SDL_audiotypecvt.o
 0001:001e4da0       _SDL_Upsample_S32LSB_2c_x2 005e5da0 f   libSDL2:SDL_audiotypecvt.o
 0001:001e4e90       _SDL_Downsample_S32LSB_2c_x2 005e5e90 f   libSDL2:SDL_audiotypecvt.o
 0001:001e4f70       _SDL_Upsample_S32LSB_2c_x4 005e5f70 f   libSDL2:SDL_audiotypecvt.o
 0001:001e50f0       _SDL_Downsample_S32LSB_2c_x4 005e60f0 f   libSDL2:SDL_audiotypecvt.o
 0001:001e51e0       _SDL_Upsample_S32LSB_4c_x2 005e61e0 f   libSDL2:SDL_audiotypecvt.o
 0001:001e5370       _SDL_Downsample_S32LSB_4c_x2 005e6370 f   libSDL2:SDL_audiotypecvt.o
 0001:001e54e0       _SDL_Upsample_S32LSB_4c_x4 005e64e0 f   libSDL2:SDL_audiotypecvt.o
 0001:001e57a0       _SDL_Downsample_S32LSB_4c_x4 005e67a0 f   libSDL2:SDL_audiotypecvt.o
 0001:001e5910       _SDL_Upsample_S32LSB_6c_x2 005e6910 f   libSDL2:SDL_audiotypecvt.o
 0001:001e5b60       _SDL_Downsample_S32LSB_6c_x2 005e6b60 f   libSDL2:SDL_audiotypecvt.o
 0001:001e5d50       _SDL_Upsample_S32LSB_6c_x4 005e6d50 f   libSDL2:SDL_audiotypecvt.o
 0001:001e6140       _SDL_Downsample_S32LSB_6c_x4 005e7140 f   libSDL2:SDL_audiotypecvt.o
 0001:001e6330       _SDL_Upsample_S32LSB_8c_x2 005e7330 f   libSDL2:SDL_audiotypecvt.o
 0001:001e6660       _SDL_Downsample_S32LSB_8c_x2 005e7660 f   libSDL2:SDL_audiotypecvt.o
 0001:001e68e0       _SDL_Upsample_S32LSB_8c_x4 005e78e0 f   libSDL2:SDL_audiotypecvt.o
 0001:001e6e50       _SDL_Downsample_S32LSB_8c_x4 005e7e50 f   libSDL2:SDL_audiotypecvt.o
 0001:001e70d0       _SDL_Upsample_S32MSB_1c_x2 005e80d0 f   libSDL2:SDL_audiotypecvt.o
 0001:001e7180       _SDL_Downsample_S32MSB_1c_x2 005e8180 f   libSDL2:SDL_audiotypecvt.o
 0001:001e7220       _SDL_Upsample_S32MSB_1c_x4 005e8220 f   libSDL2:SDL_audiotypecvt.o
 0001:001e7320       _SDL_Downsample_S32MSB_1c_x4 005e8320 f   libSDL2:SDL_audiotypecvt.o
 0001:001e73c0       _SDL_Upsample_S32MSB_2c_x2 005e83c0 f   libSDL2:SDL_audiotypecvt.o
 0001:001e74c0       _SDL_Downsample_S32MSB_2c_x2 005e84c0 f   libSDL2:SDL_audiotypecvt.o
 0001:001e75b0       _SDL_Upsample_S32MSB_2c_x4 005e85b0 f   libSDL2:SDL_audiotypecvt.o
 0001:001e7740       _SDL_Downsample_S32MSB_2c_x4 005e8740 f   libSDL2:SDL_audiotypecvt.o
 0001:001e7830       _SDL_Upsample_S32MSB_4c_x2 005e8830 f   libSDL2:SDL_audiotypecvt.o
 0001:001e79f0       _SDL_Downsample_S32MSB_4c_x2 005e89f0 f   libSDL2:SDL_audiotypecvt.o
 0001:001e7b70       _SDL_Upsample_S32MSB_4c_x4 005e8b70 f   libSDL2:SDL_audiotypecvt.o
 0001:001e7e40       _SDL_Downsample_S32MSB_4c_x4 005e8e40 f   libSDL2:SDL_audiotypecvt.o
 0001:001e7fc0       _SDL_Upsample_S32MSB_6c_x2 005e8fc0 f   libSDL2:SDL_audiotypecvt.o
 0001:001e8230       _SDL_Downsample_S32MSB_6c_x2 005e9230 f   libSDL2:SDL_audiotypecvt.o
 0001:001e8450       _SDL_Upsample_S32MSB_6c_x4 005e9450 f   libSDL2:SDL_audiotypecvt.o
 0001:001e8860       _SDL_Downsample_S32MSB_6c_x4 005e9860 f   libSDL2:SDL_audiotypecvt.o
 0001:001e8a80       _SDL_Upsample_S32MSB_8c_x2 005e9a80 f   libSDL2:SDL_audiotypecvt.o
 0001:001e8df0       _SDL_Downsample_S32MSB_8c_x2 005e9df0 f   libSDL2:SDL_audiotypecvt.o
 0001:001e90b0       _SDL_Upsample_S32MSB_8c_x4 005ea0b0 f   libSDL2:SDL_audiotypecvt.o
 0001:001e9650       _SDL_Downsample_S32MSB_8c_x4 005ea650 f   libSDL2:SDL_audiotypecvt.o
 0001:001e9910       _SDL_Upsample_F32LSB_1c_x2 005ea910 f   libSDL2:SDL_audiotypecvt.o
 0001:001e99a0       _SDL_Downsample_F32LSB_1c_x2 005ea9a0 f   libSDL2:SDL_audiotypecvt.o
 0001:001e9a20       _SDL_Upsample_F32LSB_1c_x4 005eaa20 f   libSDL2:SDL_audiotypecvt.o
 0001:001e9ad0       _SDL_Downsample_F32LSB_1c_x4 005eaad0 f   libSDL2:SDL_audiotypecvt.o
 0001:001e9b50       _SDL_Upsample_F32LSB_2c_x2 005eab50 f   libSDL2:SDL_audiotypecvt.o
 0001:001e9bf0       _SDL_Downsample_F32LSB_2c_x2 005eabf0 f   libSDL2:SDL_audiotypecvt.o
 0001:001e9c90       _SDL_Upsample_F32LSB_2c_x4 005eac90 f   libSDL2:SDL_audiotypecvt.o
 0001:001e9d90       _SDL_Downsample_F32LSB_2c_x4 005ead90 f   libSDL2:SDL_audiotypecvt.o
 0001:001e9e40       _SDL_Upsample_F32LSB_4c_x2 005eae40 f   libSDL2:SDL_audiotypecvt.o
 0001:001e9f20       _SDL_Downsample_F32LSB_4c_x2 005eaf20 f   libSDL2:SDL_audiotypecvt.o
 0001:001e9ff0       _SDL_Upsample_F32LSB_4c_x4 005eaff0 f   libSDL2:SDL_audiotypecvt.o
 0001:001ea190       _SDL_Downsample_F32LSB_4c_x4 005eb190 f   libSDL2:SDL_audiotypecvt.o
 0001:001ea260       _SDL_Upsample_F32LSB_6c_x2 005eb260 f   libSDL2:SDL_audiotypecvt.o
 0001:001ea390       _SDL_Downsample_F32LSB_6c_x2 005eb390 f   libSDL2:SDL_audiotypecvt.o
 0001:001ea4b0       _SDL_Upsample_F32LSB_6c_x4 005eb4b0 f   libSDL2:SDL_audiotypecvt.o
 0001:001ea720       _SDL_Downsample_F32LSB_6c_x4 005eb720 f   libSDL2:SDL_audiotypecvt.o
 0001:001ea840       _SDL_Upsample_F32LSB_8c_x2 005eb840 f   libSDL2:SDL_audiotypecvt.o
 0001:001ea9e0       _SDL_Downsample_F32LSB_8c_x2 005eb9e0 f   libSDL2:SDL_audiotypecvt.o
 0001:001eab50       _SDL_Upsample_F32LSB_8c_x4 005ebb50 f   libSDL2:SDL_audiotypecvt.o
 0001:001eaea0       _SDL_Downsample_F32LSB_8c_x4 005ebea0 f   libSDL2:SDL_audiotypecvt.o
 0001:001eb010       _SDL_Upsample_F32MSB_1c_x2 005ec010 f   libSDL2:SDL_audiotypecvt.o
 0001:001eb0b0       _SDL_Downsample_F32MSB_1c_x2 005ec0b0 f   libSDL2:SDL_audiotypecvt.o
 0001:001eb150       _SDL_Upsample_F32MSB_1c_x4 005ec150 f   libSDL2:SDL_audiotypecvt.o
 0001:001eb220       _SDL_Downsample_F32MSB_1c_x4 005ec220 f   libSDL2:SDL_audiotypecvt.o
 0001:001eb2c0       _SDL_Upsample_F32MSB_2c_x2 005ec2c0 f   libSDL2:SDL_audiotypecvt.o
 0001:001eb390       _SDL_Downsample_F32MSB_2c_x2 005ec390 f   libSDL2:SDL_audiotypecvt.o
 0001:001eb460       _SDL_Upsample_F32MSB_2c_x4 005ec460 f   libSDL2:SDL_audiotypecvt.o
 0001:001eb590       _SDL_Downsample_F32MSB_2c_x4 005ec590 f   libSDL2:SDL_audiotypecvt.o
 0001:001eb660       _SDL_Upsample_F32MSB_4c_x2 005ec660 f   libSDL2:SDL_audiotypecvt.o
 0001:001eb7a0       _SDL_Downsample_F32MSB_4c_x2 005ec7a0 f   libSDL2:SDL_audiotypecvt.o
 0001:001eb8d0       _SDL_Upsample_F32MSB_4c_x4 005ec8d0 f   libSDL2:SDL_audiotypecvt.o
 0001:001ebab0       _SDL_Downsample_F32MSB_4c_x4 005ecab0 f   libSDL2:SDL_audiotypecvt.o
 0001:001ebbe0       _SDL_Upsample_F32MSB_6c_x2 005ecbe0 f   libSDL2:SDL_audiotypecvt.o
 0001:001ebd90       _SDL_Downsample_F32MSB_6c_x2 005ecd90 f   libSDL2:SDL_audiotypecvt.o
 0001:001ebf30       _SDL_Upsample_F32MSB_6c_x4 005ecf30 f   libSDL2:SDL_audiotypecvt.o
 0001:001ec220       _SDL_Downsample_F32MSB_6c_x4 005ed220 f   libSDL2:SDL_audiotypecvt.o
 0001:001ec3c0       _SDL_Upsample_F32MSB_8c_x2 005ed3c0 f   libSDL2:SDL_audiotypecvt.o
 0001:001ec5f0       _SDL_Downsample_F32MSB_8c_x2 005ed5f0 f   libSDL2:SDL_audiotypecvt.o
 0001:001ec800       _SDL_Upsample_F32MSB_8c_x4 005ed800 f   libSDL2:SDL_audiotypecvt.o
 0001:001ecbf0       _SDL_Downsample_F32MSB_8c_x4 005edbf0 f   libSDL2:SDL_audiotypecvt.o
 0001:001ed390       _DUMMY_SetDisplayMode      005ee390 f   libSDL2:SDL_nullvideo.o
 0001:001ed3a0       _DUMMY_VideoQuit           005ee3a0 f   libSDL2:SDL_nullvideo.o
 0001:001ed3b0       _DUMMY_CreateDevice        005ee3b0 f   libSDL2:SDL_nullvideo.o
 0001:001ed420       _DUMMY_DeleteDevice        005ee420 f   libSDL2:SDL_nullvideo.o
 0001:001ed430       _DUMMY_VideoInit           005ee430 f   libSDL2:SDL_nullvideo.o
 0001:001ed4b0       _DUMMY_Available           005ee4b0 f   libSDL2:SDL_nullvideo.o
 0001:001ed4f0       _MessageBoxDialogProc      005ee4f0 f   libSDL2:SDL_windowsmessagebox.o
 0001:001ed530       _AddDialogString           005ee530 f   libSDL2:SDL_windowsmessagebox.o
 0001:001ed650       _AddDialogControl.constprop.1 005ee650 f   libSDL2:SDL_windowsmessagebox.o
 0001:001ee1e0       _SDL_SoftBlit              005ef1e0 f   libSDL2:SDL_blit.o
 0001:001ee6c0       _copy_opaque_16            005ef6c0 f   libSDL2:SDL_RLEaccel.o
 0001:001ee7c0       _uncopy_opaque_16          005ef7c0 f   libSDL2:SDL_RLEaccel.o
 0001:001ee8c0       _copy_transl_565           005ef8c0 f   libSDL2:SDL_RLEaccel.o
 0001:001ee980       _copy_transl_555           005ef980 f   libSDL2:SDL_RLEaccel.o
 0001:001eea40       _uncopy_transl_16          005efa40 f   libSDL2:SDL_RLEaccel.o
 0001:001eeb30       _copy_32                   005efb30 f   libSDL2:SDL_RLEaccel.o
 0001:001eebc0       _uncopy_32                 005efbc0 f   libSDL2:SDL_RLEaccel.o
 0001:001eeca0       _getpix_8                  005efca0 f   libSDL2:SDL_RLEaccel.o
 0001:001eecb0       _getpix_16                 005efcb0 f   libSDL2:SDL_RLEaccel.o
 0001:001eecc0       _getpix_24                 005efcc0 f   libSDL2:SDL_RLEaccel.o
 0001:001eece0       _getpix_32                 005efce0 f   libSDL2:SDL_RLEaccel.o
 0001:001f2ec0       _GL_WindowEvent            005f3ec0 f   libSDL2:SDL_render_gl.o
 0001:001f2ef0       _GL_LockTexture            005f3ef0 f   libSDL2:SDL_render_gl.o
 0001:001f2f80       _GL_HandleDebugMessage@28  005f3f80 f   libSDL2:SDL_render_gl.o
 0001:001f3090       _GL_UpdateClipRect         005f4090 f   libSDL2:SDL_render_gl.o
 0001:001f3160       _GL_UpdateViewport         005f4160 f   libSDL2:SDL_render_gl.o
 0001:001f3450       _GL_ActivateRenderer       005f4450 f   libSDL2:SDL_render_gl.o
 0001:001f3530       _GL_UnbindTexture          005f4530 f   libSDL2:SDL_render_gl.o
 0001:001f35b0       _GL_BindTexture            005f45b0 f   libSDL2:SDL_render_gl.o
 0001:001f3680       _GL_DestroyTexture         005f4680 f   libSDL2:SDL_render_gl.o
 0001:001f3720       _GL_RenderClear            005f4720 f   libSDL2:SDL_render_gl.o
 0001:001f37b0       _GL_UpdateTextureYUV       005f47b0 f   libSDL2:SDL_render_gl.o
 0001:001f3b40       _GL_UpdateTexture          005f4b40 f   libSDL2:SDL_render_gl.o
 0001:001f4040       _GL_UnlockTexture          005f5040 f   libSDL2:SDL_render_gl.o
 0001:001f40d0       _GL_RenderReadPixels       005f50d0 f   libSDL2:SDL_render_gl.o
 0001:001f4460       _GL_SetRenderTarget        005f5460 f   libSDL2:SDL_render_gl.o
 0001:001f4520       _GL_GetOutputSize          005f5520 f   libSDL2:SDL_render_gl.o
 0001:001f4550       _GL_DestroyRenderer        005f5550 f   libSDL2:SDL_render_gl.o
 0001:001f4830       _GL_CreateRenderer         005f5830 f   libSDL2:SDL_render_gl.o
 0001:001f5a80       _GL_CreateTexture          005f6a80 f   libSDL2:SDL_render_gl.o
 0001:001f69d0       _GL_SetupCopy.isra.5       005f79d0 f   libSDL2:SDL_render_gl.o
 0001:001f6df0       _GL_RenderCopyEx           005f7df0 f   libSDL2:SDL_render_gl.o
 0001:001f7230       _GL_RenderCopy             005f8230 f   libSDL2:SDL_render_gl.o
 0001:001f75a0       _GL_SetDrawingState        005f85a0 f   libSDL2:SDL_render_gl.o
 0001:001f77e0       _GL_RenderFillRects        005f87e0 f   libSDL2:SDL_render_gl.o
 0001:001f79e0       _GL_RenderDrawLines        005f89e0 f   libSDL2:SDL_render_gl.o
 0001:001f7cf0       _GL_RenderDrawPoints       005f8cf0 f   libSDL2:SDL_render_gl.o
 0001:001f7d60       _GL_RenderPresent          005f8d60 f   libSDL2:SDL_render_gl.o
 0001:001f7e40       _GLES2_WindowEvent         005f8e40 f   libSDL2:SDL_render_gles2.o
 0001:001f7e80       _GLES2_LockTexture         005f8e80 f   libSDL2:SDL_render_gles2.o
 0001:001f7f00       _GLES2_UpdateClipRect      005f8f00 f   libSDL2:SDL_render_gles2.o
 0001:001f7fe0       _GLES2_SetRenderTarget     005f8fe0 f   libSDL2:SDL_render_gles2.o
 0001:001f80a0       _GLES2_SetOrthographicProjection 005f90a0 f   libSDL2:SDL_render_gles2.o
 0001:001f8240       _GLES2_UpdateViewport      005f9240 f   libSDL2:SDL_render_gles2.o
 0001:001f83a0       _GLES2_GetOutputSize       005f93a0 f   libSDL2:SDL_render_gles2.o
 0001:001f83d0       _GLES2_DestroyRenderer     005f93d0 f   libSDL2:SDL_render_gles2.o
 0001:001f85d0       _GLES2_CacheShader.isra.6  005f95d0 f   libSDL2:SDL_render_gles2.o
 0001:001f8820       _GLES2_RenderPresent       005f9820 f   libSDL2:SDL_render_gles2.o
 0001:001f8890       _GLES2_UnbindTexture       005f9890 f   libSDL2:SDL_render_gles2.o
 0001:001f8920       _GLES2_BindTexture         005f9920 f   libSDL2:SDL_render_gles2.o
 0001:001f89d0       _GLES2_DestroyTexture      005f99d0 f   libSDL2:SDL_render_gles2.o
 0001:001f8ac0       _GLES2_RenderClear         005f9ac0 f   libSDL2:SDL_render_gles2.o
 0001:001f8c70       _GLES2_RenderReadPixels    005f9c70 f   libSDL2:SDL_render_gles2.o
 0001:001f8f20       _GLES2_CreateTexture       005f9f20 f   libSDL2:SDL_render_gles2.o
 0001:001f9cd0       _GLES2_CreateRenderer      005facd0 f   libSDL2:SDL_render_gles2.o
 0001:001fafe0       _GLES2_UpdateTexture       005fbfe0 f   libSDL2:SDL_render_gles2.o
 0001:001fb820       _GLES2_UnlockTexture       005fc820 f   libSDL2:SDL_render_gles2.o
 0001:001fb880       _GLES2_UpdateTextureYUV    005fc880 f   libSDL2:SDL_render_gles2.o
 0001:001fbe30       _GLES2_SelectProgram       005fce30 f   libSDL2:SDL_render_gles2.o
 0001:001fc560       _GLES2_SetupCopy           005fd560 f   libSDL2:SDL_render_gles2.o
 0001:001fc9e0       _GLES2_RenderCopyEx        005fd9e0 f   libSDL2:SDL_render_gles2.o
 0001:001fcdf0       _GLES2_RenderCopy          005fddf0 f   libSDL2:SDL_render_gles2.o
 0001:001fd070       _GLES2_SetDrawingState     005fe070 f   libSDL2:SDL_render_gles2.o
 0001:001fd310       _GLES2_RenderFillRects     005fe310 f   libSDL2:SDL_render_gles2.o
 0001:001fd4b0       _GLES2_RenderDrawLines     005fe4b0 f   libSDL2:SDL_render_gles2.o
 0001:001fd7b0       _GLES2_RenderDrawPoints    005fe7b0 f   libSDL2:SDL_render_gles2.o
 0001:001fd9b0       _SW_WindowEvent            005fe9b0 f   libSDL2:SDL_render_sw.o
 0001:001fd9e0       _SW_LockTexture            005fe9e0 f   libSDL2:SDL_render_sw.o
 0001:001fda20       _SW_UnlockTexture          005fea20 f   libSDL2:SDL_render_sw.o
 0001:001fda30       _SW_SetRenderTarget        005fea30 f   libSDL2:SDL_render_sw.o
 0001:001fda60       _SW_DestroyTexture         005fea60 f   libSDL2:SDL_render_sw.o
 0001:001fda70       _SW_RenderPresent          005fea70 f   libSDL2:SDL_render_sw.o
 0001:001fda90       _SW_SetTextureBlendMode    005fea90 f   libSDL2:SDL_render_sw.o
 0001:001fdae0       _SW_SetTextureAlphaMod     005feae0 f   libSDL2:SDL_render_sw.o
 0001:001fdb30       _SW_SetTextureColorMod     005feb30 f   libSDL2:SDL_render_sw.o
 0001:001fdba0       _SW_DestroyRenderer        005feba0 f   libSDL2:SDL_render_sw.o
 0001:001fdbd0       _SW_UpdateClipRect         005febd0 f   libSDL2:SDL_render_sw.o
 0001:001fdc20       _SW_UpdateViewport         005fec20 f   libSDL2:SDL_render_sw.o
 0001:001fdc50       _SW_UpdateTexture          005fec50 f   libSDL2:SDL_render_sw.o
 0001:001fdcf0       _SW_CreateTexture          005fecf0 f   libSDL2:SDL_render_sw.o
 0001:001fde00       _SW_RenderFillRects        005fee00 f   libSDL2:SDL_render_sw.o
 0001:001fe0b0       _SW_GetOutputSize          005ff0b0 f   libSDL2:SDL_render_sw.o
 0001:001fe1a0       _SW_RenderReadPixels       005ff1a0 f   libSDL2:SDL_render_sw.o
 0001:001fe360       _SW_RenderCopy             005ff360 f   libSDL2:SDL_render_sw.o
 0001:001fe530       _SW_RenderClear            005ff530 f   libSDL2:SDL_render_sw.o
 0001:001fe680       _SW_CreateRenderer         005ff680 f   libSDL2:SDL_render_sw.o
 0001:001fe7c0       _SW_RenderDrawLines        005ff7c0 f   libSDL2:SDL_render_sw.o
 0001:001fea20       _SW_RenderDrawPoints       005ffa20 f   libSDL2:SDL_render_sw.o
 0001:001fec80       _SW_RenderCopyEx           005ffc80 f   libSDL2:SDL_render_sw.o
 0001:001ff750       _Color16DitherYV12Mod1X    00600750 f   libSDL2:SDL_yuv_sw.o
 0001:001ff960       _Color24DitherYV12Mod1X    00600960 f   libSDL2:SDL_yuv_sw.o
 0001:001ffbc0       _Color32DitherYV12Mod1X    00600bc0 f   libSDL2:SDL_yuv_sw.o
 0001:001ffdc0       _Color16DitherYV12Mod2X    00600dc0 f   libSDL2:SDL_yuv_sw.o
 0001:00200000       _Color24DitherYV12Mod2X    00601000 f   libSDL2:SDL_yuv_sw.o
 0001:00200310       _Color32DitherYV12Mod2X    00601310 f   libSDL2:SDL_yuv_sw.o
 0001:00200560       _Color16DitherYUY2Mod1X    00601560 f   libSDL2:SDL_yuv_sw.o
 0001:002006b0       _Color24DitherYUY2Mod1X    006016b0 f   libSDL2:SDL_yuv_sw.o
 0001:00200830       _Color32DitherYUY2Mod1X    00601830 f   libSDL2:SDL_yuv_sw.o
 0001:00200990       _Color16DitherYUY2Mod2X    00601990 f   libSDL2:SDL_yuv_sw.o
 0001:00200b10       _Color24DitherYUY2Mod2X    00601b10 f   libSDL2:SDL_yuv_sw.o
 0001:00200d00       _Color32DitherYUY2Mod2X    00601d00 f   libSDL2:SDL_yuv_sw.o
 0001:00204c80       _SDL_Blit_RGB888_RGB888_Scale 00605c80 f   libSDL2:SDL_blit_auto.o
 0001:00204d80       _SDL_Blit_RGB888_RGB888_Blend 00605d80 f   libSDL2:SDL_blit_auto.o
 0001:00204ef0       _SDL_Blit_RGB888_RGB888_Blend_Scale 00605ef0 f   libSDL2:SDL_blit_auto.o
 0001:00205120       _SDL_Blit_RGB888_RGB888_Modulate 00606120 f   libSDL2:SDL_blit_auto.o
 0001:00205250       _SDL_Blit_RGB888_RGB888_Modulate_Scale 00606250 f   libSDL2:SDL_blit_auto.o
 0001:002054a0       _SDL_Blit_RGB888_RGB888_Modulate_Blend 006064a0 f   libSDL2:SDL_blit_auto.o
 0001:00205770       _SDL_Blit_RGB888_RGB888_Modulate_Blend_Scale 00606770 f   libSDL2:SDL_blit_auto.o
 0001:00205b00       _SDL_Blit_RGB888_BGR888_Scale 00606b00 f   libSDL2:SDL_blit_auto.o
 0001:00205c60       _SDL_Blit_RGB888_BGR888_Blend 00606c60 f   libSDL2:SDL_blit_auto.o
 0001:00205dc0       _SDL_Blit_RGB888_BGR888_Blend_Scale 00606dc0 f   libSDL2:SDL_blit_auto.o
 0001:00205ff0       _SDL_Blit_RGB888_BGR888_Modulate 00606ff0 f   libSDL2:SDL_blit_auto.o
 0001:00206130       _SDL_Blit_RGB888_BGR888_Modulate_Scale 00607130 f   libSDL2:SDL_blit_auto.o
 0001:00206390       _SDL_Blit_RGB888_BGR888_Modulate_Blend 00607390 f   libSDL2:SDL_blit_auto.o
 0001:00206660       _SDL_Blit_RGB888_BGR888_Modulate_Blend_Scale 00607660 f   libSDL2:SDL_blit_auto.o
 0001:002069f0       _SDL_Blit_RGB888_ARGB8888_Scale 006079f0 f   libSDL2:SDL_blit_auto.o
 0001:00206b10       _SDL_Blit_RGB888_ARGB8888_Blend 00607b10 f   libSDL2:SDL_blit_auto.o
 0001:00206ca0       _SDL_Blit_RGB888_ARGB8888_Blend_Scale 00607ca0 f   libSDL2:SDL_blit_auto.o
 0001:00206ef0       _SDL_Blit_RGB888_ARGB8888_Modulate 00607ef0 f   libSDL2:SDL_blit_auto.o
 0001:00207060       _SDL_Blit_RGB888_ARGB8888_Modulate_Scale 00608060 f   libSDL2:SDL_blit_auto.o
 0001:002072e0       _SDL_Blit_RGB888_ARGB8888_Modulate_Blend 006082e0 f   libSDL2:SDL_blit_auto.o
 0001:002075e0       _SDL_Blit_RGB888_ARGB8888_Modulate_Blend_Scale 006085e0 f   libSDL2:SDL_blit_auto.o
 0001:002079a0       _SDL_Blit_BGR888_RGB888_Scale 006089a0 f   libSDL2:SDL_blit_auto.o
 0001:00207b00       _SDL_Blit_BGR888_RGB888_Blend 00608b00 f   libSDL2:SDL_blit_auto.o
 0001:00207c70       _SDL_Blit_BGR888_RGB888_Blend_Scale 00608c70 f   libSDL2:SDL_blit_auto.o
 0001:00207ea0       _SDL_Blit_BGR888_RGB888_Modulate 00608ea0 f   libSDL2:SDL_blit_auto.o
 0001:00207fe0       _SDL_Blit_BGR888_RGB888_Modulate_Scale 00608fe0 f   libSDL2:SDL_blit_auto.o
 0001:00208240       _SDL_Blit_BGR888_RGB888_Modulate_Blend 00609240 f   libSDL2:SDL_blit_auto.o
 0001:00208510       _SDL_Blit_BGR888_RGB888_Modulate_Blend_Scale 00609510 f   libSDL2:SDL_blit_auto.o
 0001:002088a0       _SDL_Blit_BGR888_BGR888_Scale 006098a0 f   libSDL2:SDL_blit_auto.o
 0001:002089a0       _SDL_Blit_BGR888_BGR888_Blend 006099a0 f   libSDL2:SDL_blit_auto.o
 0001:00208b00       _SDL_Blit_BGR888_BGR888_Blend_Scale 00609b00 f   libSDL2:SDL_blit_auto.o
 0001:00208d30       _SDL_Blit_BGR888_BGR888_Modulate 00609d30 f   libSDL2:SDL_blit_auto.o
 0001:00208e60       _SDL_Blit_BGR888_BGR888_Modulate_Scale 00609e60 f   libSDL2:SDL_blit_auto.o
 0001:002090b0       _SDL_Blit_BGR888_BGR888_Modulate_Blend 0060a0b0 f   libSDL2:SDL_blit_auto.o
 0001:00209380       _SDL_Blit_BGR888_BGR888_Modulate_Blend_Scale 0060a380 f   libSDL2:SDL_blit_auto.o
 0001:00209710       _SDL_Blit_BGR888_ARGB8888_Scale 0060a710 f   libSDL2:SDL_blit_auto.o
 0001:00209870       _SDL_Blit_BGR888_ARGB8888_Blend 0060a870 f   libSDL2:SDL_blit_auto.o
 0001:00209a00       _SDL_Blit_BGR888_ARGB8888_Blend_Scale 0060aa00 f   libSDL2:SDL_blit_auto.o
 0001:00209c50       _SDL_Blit_BGR888_ARGB8888_Modulate 0060ac50 f   libSDL2:SDL_blit_auto.o
 0001:00209dc0       _SDL_Blit_BGR888_ARGB8888_Modulate_Scale 0060adc0 f   libSDL2:SDL_blit_auto.o
 0001:0020a040       _SDL_Blit_BGR888_ARGB8888_Modulate_Blend 0060b040 f   libSDL2:SDL_blit_auto.o
 0001:0020a340       _SDL_Blit_BGR888_ARGB8888_Modulate_Blend_Scale 0060b340 f   libSDL2:SDL_blit_auto.o
 0001:0020a700       _SDL_Blit_ARGB8888_RGB888_Scale 0060b700 f   libSDL2:SDL_blit_auto.o
 0001:0020a820       _SDL_Blit_ARGB8888_RGB888_Blend 0060b820 f   libSDL2:SDL_blit_auto.o
 0001:0020aa40       _SDL_Blit_ARGB8888_RGB888_Blend_Scale 0060ba40 f   libSDL2:SDL_blit_auto.o
 0001:0020ad20       _SDL_Blit_ARGB8888_RGB888_Modulate 0060bd20 f   libSDL2:SDL_blit_auto.o
 0001:0020ae50       _SDL_Blit_ARGB8888_RGB888_Modulate_Scale 0060be50 f   libSDL2:SDL_blit_auto.o
 0001:0020b0a0       _SDL_Blit_ARGB8888_RGB888_Modulate_Blend 0060c0a0 f   libSDL2:SDL_blit_auto.o
 0001:0020b370       _SDL_Blit_ARGB8888_RGB888_Modulate_Blend_Scale 0060c370 f   libSDL2:SDL_blit_auto.o
 0001:0020b6e0       _SDL_Blit_ARGB8888_BGR888_Scale 0060c6e0 f   libSDL2:SDL_blit_auto.o
 0001:0020b840       _SDL_Blit_ARGB8888_BGR888_Blend 0060c840 f   libSDL2:SDL_blit_auto.o
 0001:0020ba60       _SDL_Blit_ARGB8888_BGR888_Blend_Scale 0060ca60 f   libSDL2:SDL_blit_auto.o
 0001:0020bd40       _SDL_Blit_ARGB8888_BGR888_Modulate 0060cd40 f   libSDL2:SDL_blit_auto.o
 0001:0020be80       _SDL_Blit_ARGB8888_BGR888_Modulate_Scale 0060ce80 f   libSDL2:SDL_blit_auto.o
 0001:0020c0e0       _SDL_Blit_ARGB8888_BGR888_Modulate_Blend 0060d0e0 f   libSDL2:SDL_blit_auto.o
 0001:0020c3b0       _SDL_Blit_ARGB8888_BGR888_Modulate_Blend_Scale 0060d3b0 f   libSDL2:SDL_blit_auto.o
 0001:0020c720       _SDL_Blit_ARGB8888_ARGB8888_Scale 0060d720 f   libSDL2:SDL_blit_auto.o
 0001:0020c820       _SDL_Blit_ARGB8888_ARGB8888_Blend 0060d820 f   libSDL2:SDL_blit_auto.o
 0001:0020ca60       _SDL_Blit_ARGB8888_ARGB8888_Blend_Scale 0060da60 f   libSDL2:SDL_blit_auto.o
 0001:0020cd70       _SDL_Blit_ARGB8888_ARGB8888_Modulate 0060dd70 f   libSDL2:SDL_blit_auto.o
 0001:0020cf90       _SDL_Blit_ARGB8888_ARGB8888_Modulate_Scale 0060df90 f   libSDL2:SDL_blit_auto.o
 0001:0020d1b0       _SDL_Blit_ARGB8888_ARGB8888_Modulate_Blend 0060e1b0 f   libSDL2:SDL_blit_auto.o
 0001:0020d4b0       _SDL_Blit_ARGB8888_ARGB8888_Modulate_Blend_Scale 0060e4b0 f   libSDL2:SDL_blit_auto.o
 0001:0020d860       _SDL_Blit_RGBA8888_RGB888_Scale 0060e860 f   libSDL2:SDL_blit_auto.o
 0001:0020d9a0       _SDL_Blit_RGBA8888_RGB888_Blend 0060e9a0 f   libSDL2:SDL_blit_auto.o
 0001:0020dbc0       _SDL_Blit_RGBA8888_RGB888_Blend_Scale 0060ebc0 f   libSDL2:SDL_blit_auto.o
 0001:0020dea0       _SDL_Blit_RGBA8888_RGB888_Modulate 0060eea0 f   libSDL2:SDL_blit_auto.o
 0001:0020dfd0       _SDL_Blit_RGBA8888_RGB888_Modulate_Scale 0060efd0 f   libSDL2:SDL_blit_auto.o
 0001:0020e230       _SDL_Blit_RGBA8888_RGB888_Modulate_Blend 0060f230 f   libSDL2:SDL_blit_auto.o
 0001:0020e500       _SDL_Blit_RGBA8888_RGB888_Modulate_Blend_Scale 0060f500 f   libSDL2:SDL_blit_auto.o
 0001:0020e870       _SDL_Blit_RGBA8888_BGR888_Scale 0060f870 f   libSDL2:SDL_blit_auto.o
 0001:0020e9d0       _SDL_Blit_RGBA8888_BGR888_Blend 0060f9d0 f   libSDL2:SDL_blit_auto.o
 0001:0020ebf0       _SDL_Blit_RGBA8888_BGR888_Blend_Scale 0060fbf0 f   libSDL2:SDL_blit_auto.o
 0001:0020eed0       _SDL_Blit_RGBA8888_BGR888_Modulate 0060fed0 f   libSDL2:SDL_blit_auto.o
 0001:0020f010       _SDL_Blit_RGBA8888_BGR888_Modulate_Scale 00610010 f   libSDL2:SDL_blit_auto.o
 0001:0020f270       _SDL_Blit_RGBA8888_BGR888_Modulate_Blend 00610270 f   libSDL2:SDL_blit_auto.o
 0001:0020f540       _SDL_Blit_RGBA8888_BGR888_Modulate_Blend_Scale 00610540 f   libSDL2:SDL_blit_auto.o
 0001:0020f8b0       _SDL_Blit_RGBA8888_ARGB8888_Scale 006108b0 f   libSDL2:SDL_blit_auto.o
 0001:0020fa20       _SDL_Blit_RGBA8888_ARGB8888_Blend 00610a20 f   libSDL2:SDL_blit_auto.o
 0001:0020fc60       _SDL_Blit_RGBA8888_ARGB8888_Blend_Scale 00610c60 f   libSDL2:SDL_blit_auto.o
 0001:0020ff70       _SDL_Blit_RGBA8888_ARGB8888_Modulate 00610f70 f   libSDL2:SDL_blit_auto.o
 0001:002101d0       _SDL_Blit_RGBA8888_ARGB8888_Modulate_Scale 006111d0 f   libSDL2:SDL_blit_auto.o
 0001:00210400       _SDL_Blit_RGBA8888_ARGB8888_Modulate_Blend 00611400 f   libSDL2:SDL_blit_auto.o
 0001:00210710       _SDL_Blit_RGBA8888_ARGB8888_Modulate_Blend_Scale 00611710 f   libSDL2:SDL_blit_auto.o
 0001:00210ac0       _SDL_Blit_ABGR8888_RGB888_Scale 00611ac0 f   libSDL2:SDL_blit_auto.o
 0001:00210c20       _SDL_Blit_ABGR8888_RGB888_Blend 00611c20 f   libSDL2:SDL_blit_auto.o
 0001:00210e30       _SDL_Blit_ABGR8888_RGB888_Blend_Scale 00611e30 f   libSDL2:SDL_blit_auto.o
 0001:00211110       _SDL_Blit_ABGR8888_RGB888_Modulate 00612110 f   libSDL2:SDL_blit_auto.o
 0001:00211250       _SDL_Blit_ABGR8888_RGB888_Modulate_Scale 00612250 f   libSDL2:SDL_blit_auto.o
 0001:002114b0       _SDL_Blit_ABGR8888_RGB888_Modulate_Blend 006124b0 f   libSDL2:SDL_blit_auto.o
 0001:00211780       _SDL_Blit_ABGR8888_RGB888_Modulate_Blend_Scale 00612780 f   libSDL2:SDL_blit_auto.o
 0001:00211af0       _SDL_Blit_ABGR8888_BGR888_Scale 00612af0 f   libSDL2:SDL_blit_auto.o
 0001:00211c10       _SDL_Blit_ABGR8888_BGR888_Blend 00612c10 f   libSDL2:SDL_blit_auto.o
 0001:00211e30       _SDL_Blit_ABGR8888_BGR888_Blend_Scale 00612e30 f   libSDL2:SDL_blit_auto.o
 0001:00212110       _SDL_Blit_ABGR8888_BGR888_Modulate 00613110 f   libSDL2:SDL_blit_auto.o
 0001:00212240       _SDL_Blit_ABGR8888_BGR888_Modulate_Scale 00613240 f   libSDL2:SDL_blit_auto.o
 0001:00212490       _SDL_Blit_ABGR8888_BGR888_Modulate_Blend 00613490 f   libSDL2:SDL_blit_auto.o
 0001:00212760       _SDL_Blit_ABGR8888_BGR888_Modulate_Blend_Scale 00613760 f   libSDL2:SDL_blit_auto.o
 0001:00212ad0       _SDL_Blit_ABGR8888_ARGB8888_Scale 00613ad0 f   libSDL2:SDL_blit_auto.o
 0001:00212c50       _SDL_Blit_ABGR8888_ARGB8888_Blend 00613c50 f   libSDL2:SDL_blit_auto.o
 0001:00212e90       _SDL_Blit_ABGR8888_ARGB8888_Blend_Scale 00613e90 f   libSDL2:SDL_blit_auto.o
 0001:002131a0       _SDL_Blit_ABGR8888_ARGB8888_Modulate 006141a0 f   libSDL2:SDL_blit_auto.o
 0001:00213400       _SDL_Blit_ABGR8888_ARGB8888_Modulate_Scale 00614400 f   libSDL2:SDL_blit_auto.o
 0001:00213620       _SDL_Blit_ABGR8888_ARGB8888_Modulate_Blend 00614620 f   libSDL2:SDL_blit_auto.o
 0001:00213920       _SDL_Blit_ABGR8888_ARGB8888_Modulate_Blend_Scale 00614920 f   libSDL2:SDL_blit_auto.o
 0001:00213cd0       _SDL_Blit_BGRA8888_RGB888_Scale 00614cd0 f   libSDL2:SDL_blit_auto.o
 0001:00213e30       _SDL_Blit_BGRA8888_RGB888_Blend 00614e30 f   libSDL2:SDL_blit_auto.o
 0001:00214050       _SDL_Blit_BGRA8888_RGB888_Blend_Scale 00615050 f   libSDL2:SDL_blit_auto.o
 0001:00214330       _SDL_Blit_BGRA8888_RGB888_Modulate 00615330 f   libSDL2:SDL_blit_auto.o
 0001:00214470       _SDL_Blit_BGRA8888_RGB888_Modulate_Scale 00615470 f   libSDL2:SDL_blit_auto.o
 0001:002146d0       _SDL_Blit_BGRA8888_RGB888_Modulate_Blend 006156d0 f   libSDL2:SDL_blit_auto.o
 0001:002149a0       _SDL_Blit_BGRA8888_RGB888_Modulate_Blend_Scale 006159a0 f   libSDL2:SDL_blit_auto.o
 0001:00214d10       _SDL_Blit_BGRA8888_BGR888_Scale 00615d10 f   libSDL2:SDL_blit_auto.o
 0001:00214e50       _SDL_Blit_BGRA8888_BGR888_Blend 00615e50 f   libSDL2:SDL_blit_auto.o
 0001:00215070       _SDL_Blit_BGRA8888_BGR888_Blend_Scale 00616070 f   libSDL2:SDL_blit_auto.o
 0001:00215350       _SDL_Blit_BGRA8888_BGR888_Modulate 00616350 f   libSDL2:SDL_blit_auto.o
 0001:00215480       _SDL_Blit_BGRA8888_BGR888_Modulate_Scale 00616480 f   libSDL2:SDL_blit_auto.o
 0001:002156e0       _SDL_Blit_BGRA8888_BGR888_Modulate_Blend 006166e0 f   libSDL2:SDL_blit_auto.o
 0001:002159b0       _SDL_Blit_BGRA8888_BGR888_Modulate_Blend_Scale 006169b0 f   libSDL2:SDL_blit_auto.o
 0001:00215d20       _SDL_Blit_BGRA8888_ARGB8888_Scale 00616d20 f   libSDL2:SDL_blit_auto.o
 0001:00215e40       _SDL_Blit_BGRA8888_ARGB8888_Blend 00616e40 f   libSDL2:SDL_blit_auto.o
 0001:00216080       _SDL_Blit_BGRA8888_ARGB8888_Blend_Scale 00617080 f   libSDL2:SDL_blit_auto.o
 0001:00216390       _SDL_Blit_BGRA8888_ARGB8888_Modulate 00617390 f   libSDL2:SDL_blit_auto.o
 0001:002165f0       _SDL_Blit_BGRA8888_ARGB8888_Modulate_Scale 006175f0 f   libSDL2:SDL_blit_auto.o
 0001:00216820       _SDL_Blit_BGRA8888_ARGB8888_Modulate_Blend 00617820 f   libSDL2:SDL_blit_auto.o
 0001:00216b30       _SDL_Blit_BGRA8888_ARGB8888_Modulate_Blend_Scale 00617b30 f   libSDL2:SDL_blit_auto.o
 0001:002171e0       _Blit_RGB888_index8        006181e0 f   libSDL2:SDL_blit_N.o
 0001:002176c0       _Blit_RGB101010_index8     006186c0 f   libSDL2:SDL_blit_N.o
 0001:00217ba0       _Blit_RGB888_RGB555        00618ba0 f   libSDL2:SDL_blit_N.o
 0001:00217e00       _Blit_RGB888_RGB565        00618e00 f   libSDL2:SDL_blit_N.o
 0001:00218060       _Blit_RGB565_RGBA8888      00619060 f   libSDL2:SDL_blit_N.o
 0001:00218220       _BlitNto1                  00619220 f   libSDL2:SDL_blit_N.o
 0001:00219770       _Blit4to4MaskAlpha         0061a770 f   libSDL2:SDL_blit_N.o
 0001:00219940       _Blit4to4CopyAlpha         0061a940 f   libSDL2:SDL_blit_N.o
 0001:00219a20       _BlitNtoN                  0061aa20 f   libSDL2:SDL_blit_N.o
 0001:0021af00       _BlitNtoNCopyAlpha         0061bf00 f   libSDL2:SDL_blit_N.o
 0001:0021b260       _BlitNto1Key               0061c260 f   libSDL2:SDL_blit_N.o
 0001:0021c820       _Blit2to2Key               0061d820 f   libSDL2:SDL_blit_N.o
 0001:0021c9d0       _BlitNtoNKey               0061d9d0 f   libSDL2:SDL_blit_N.o
 0001:0021de40       _BlitNtoNKeyCopyAlpha      0061ee40 f   libSDL2:SDL_blit_N.o
 0001:0021f4f0       _Blit2101010toN            006204f0 f   libSDL2:SDL_blit_N.o
 0001:00220260       _BlitNto2101010            00621260 f   libSDL2:SDL_blit_N.o
 0001:00220fc0       _Blit_RGB565_BGRA8888      00621fc0 f   libSDL2:SDL_blit_N.o
 0001:00221180       _Blit_RGB565_ARGB8888      00622180 f   libSDL2:SDL_blit_N.o
 0001:00221340       _Blit_RGB565_ABGR8888      00622340 f   libSDL2:SDL_blit_N.o
 0001:002217a0       _BlitNto1SurfaceAlpha      006227a0 f   libSDL2:SDL_blit_A.o
 0001:00221fa0       _BlitNto1PixelAlpha        00622fa0 f   libSDL2:SDL_blit_A.o
 0001:002229c0       _BlitNto1SurfaceAlphaKey   006239c0 f   libSDL2:SDL_blit_A.o
 0001:00223920       _BlitRGBtoRGBSurfaceAlpha  00624920 f   libSDL2:SDL_blit_A.o
 0001:00223ce0       _BlitRGBtoRGBPixelAlpha    00624ce0 f   libSDL2:SDL_blit_A.o
 0001:00223fc0       _Blit16to16SurfaceAlpha128 00624fc0 f   libSDL2:SDL_blit_A.o
 0001:00224270       _Blit565to565SurfaceAlpha  00625270 f   libSDL2:SDL_blit_A.o
 0001:00224460       _Blit555to555SurfaceAlpha  00625460 f   libSDL2:SDL_blit_A.o
 0001:00224650       _BlitARGBto565PixelAlpha   00625650 f   libSDL2:SDL_blit_A.o
 0001:00224990       _BlitARGBto555PixelAlpha   00625990 f   libSDL2:SDL_blit_A.o
 0001:00224cd0       _BlitNtoNSurfaceAlpha      00625cd0 f   libSDL2:SDL_blit_A.o
 0001:00225f10       _BlitNtoNSurfaceAlphaKey   00626f10 f   libSDL2:SDL_blit_A.o
 0001:00227120       _BlitNtoNPixelAlpha        00628120 f   libSDL2:SDL_blit_A.o
 0001:00228630       _BlitRGBtoRGBSurfaceAlphaMMX 00629630 f   libSDL2:SDL_blit_A.o
 0001:002288f0       _Blit565to565SurfaceAlphaMMX 006298f0 f   libSDL2:SDL_blit_A.o
 0001:00228bf0       _Blit555to555SurfaceAlphaMMX 00629bf0 f   libSDL2:SDL_blit_A.o
 0001:00228f10       _BlitRGBtoRGBPixelAlphaMMX 00629f10 f   libSDL2:SDL_blit_A.o
 0001:00229270       _BlitRGBtoRGBPixelAlphaMMX3DNOW 0062a270 f   libSDL2:SDL_blit_A.o
 0001:00229890       _Blit1to1                  0062a890 f   libSDL2:SDL_blit_1.o
 0001:002299a0       _Blit1to2                  0062a9a0 f   libSDL2:SDL_blit_1.o
 0001:00229b00       _Blit1to3                  0062ab00 f   libSDL2:SDL_blit_1.o
 0001:00229d00       _Blit1to4                  0062ad00 f   libSDL2:SDL_blit_1.o
 0001:00229e80       _Blit1to1Key               0062ae80 f   libSDL2:SDL_blit_1.o
 0001:0022a140       _Blit1to2Key               0062b140 f   libSDL2:SDL_blit_1.o
 0001:0022a280       _Blit1to3Key               0062b280 f   libSDL2:SDL_blit_1.o
 0001:0022a4e0       _Blit1to4Key               0062b4e0 f   libSDL2:SDL_blit_1.o
 0001:0022a620       _Blit1toNAlpha             0062b620 f   libSDL2:SDL_blit_1.o
 0001:0022b320       _Blit1toNAlphaKey          0062c320 f   libSDL2:SDL_blit_1.o
 0001:0022ccf0       _BlitBto1                  0062dcf0 f   libSDL2:SDL_blit_0.o
 0001:0022cde0       _BlitBto2                  0062dde0 f   libSDL2:SDL_blit_0.o
 0001:0022cea0       _BlitBto3                  0062dea0 f   libSDL2:SDL_blit_0.o
 0001:0022cf80       _BlitBto4                  0062df80 f   libSDL2:SDL_blit_0.o
 0001:0022d040       _BlitBto1Key               0062e040 f   libSDL2:SDL_blit_0.o
 0001:0022d150       _BlitBto2Key               0062e150 f   libSDL2:SDL_blit_0.o
 0001:0022d220       _BlitBto4Key               0062e220 f   libSDL2:SDL_blit_0.o
 0001:0022d2f0       _BlitBtoNAlpha             0062e2f0 f   libSDL2:SDL_blit_0.o
 0001:0022d700       _BlitBtoNAlphaKey          0062e700 f   libSDL2:SDL_blit_0.o
 0001:0022db30       _BlitBto3Key               0062eb30 f   libSDL2:SDL_blit_0.o
 0001:0022e730       _CompileShader             0062f730 f   libSDL2:SDL_shaders_gl.o
 0001:0022ed30       _SDL_BlendFillRect_RGB555  0062fd30 f   libSDL2:SDL_blendfillrect.o
 0001:0022f6a0       _SDL_BlendFillRect_RGB565  006306a0 f   libSDL2:SDL_blendfillrect.o
 0001:00230050       _SDL_BlendFillRect_RGB888  00631050 f   libSDL2:SDL_blendfillrect.o
 0001:00230820       _SDL_BlendFillRect_ARGB8888 00631820 f   libSDL2:SDL_blendfillrect.o
 0001:002310a0       _SDL_BlendFillRect_RGB     006320a0 f   libSDL2:SDL_blendfillrect.o
 0001:002330e0       _SDL_BlendFillRect_RGBA    006340e0 f   libSDL2:SDL_blendfillrect.o
 0001:00234900       _SDL_BlendLine_RGB2        00635900 f   libSDL2:SDL_blendline.o
 0001:00236740       _SDL_BlendLine_RGB555      00637740 f   libSDL2:SDL_blendline.o
 0001:00237c90       _SDL_BlendLine_RGB565      00638c90 f   libSDL2:SDL_blendline.o
 0001:002392a0       _SDL_BlendLine_RGB4        0063a2a0 f   libSDL2:SDL_blendline.o
 0001:0023ad40       _SDL_BlendLine_RGBA4       0063bd40 f   libSDL2:SDL_blendline.o
 0001:0023ccd0       _SDL_BlendLine_RGB888      0063dcd0 f   libSDL2:SDL_blendline.o
 0001:0023dfa0       _SDL_BlendLine_ARGB8888    0063efa0 f   libSDL2:SDL_blendline.o
 0001:0023f780       _SDL_DrawLine4             00640780 f   libSDL2:SDL_drawline.o
 0001:0023fe50       _SDL_DrawLine2             00640e50 f   libSDL2:SDL_drawline.o
 0001:00240660       _SDL_DrawLine1             00641660 f   libSDL2:SDL_drawline.o
 0001:00240c40       _SDL_BlendPoint_RGB555     00641c40 f   libSDL2:SDL_blendpoint.o
 0001:00240e80       _SDL_BlendPoint_RGB565     00641e80 f   libSDL2:SDL_blendpoint.o
 0001:002410e0       _SDL_BlendPoint_RGB888     006420e0 f   libSDL2:SDL_blendpoint.o
 0001:002412b0       _SDL_BlendPoint_ARGB8888   006422b0 f   libSDL2:SDL_blendpoint.o
 0001:002414a0       _SDL_BlendPoint_RGB        006424a0 f   libSDL2:SDL_blendpoint.o
 0001:00241bd0       _SDL_BlendPoint_RGBA       00642bd0 f   libSDL2:SDL_blendpoint.o
 0001:002453c0       __get_next_page            006463c0 f   libvorbisfile:vorbisfile.o
 0001:00245570       __fseek64_wrap             00646570 f   libvorbisfile:vorbisfile.o
 0001:00245590       __initial_pcmoffset        00646590 f   libvorbisfile:vorbisfile.o
 0001:00245790       __get_next_page.constprop.13 00646790 f   libvorbisfile:vorbisfile.o
 0001:00245910       __fetch_headers            00646910 f   libvorbisfile:vorbisfile.o
 0001:00245c70       __fetch_headers.constprop.12 00646c70 f   libvorbisfile:vorbisfile.o
 0001:00245ef0       __get_next_page.constprop.14 00646ef0 f   libvorbisfile:vorbisfile.o
 0001:00246000       __fetch_and_process_packet.constprop.10 00647000 f   libvorbisfile:vorbisfile.o
 0001:00246390       __ov_getlap.isra.1         00647390 f   libvorbisfile:vorbisfile.o
 0001:00246530       _ov_pcm_total.part.2       00647530 f   libvorbisfile:vorbisfile.o
 0001:00246620       __ov_64_seek_lap           00647620 f   libvorbisfile:vorbisfile.o
 0001:002468e0       __get_prev_page_serial     006478e0 f   libvorbisfile:vorbisfile.o
 0001:00246c90       __fetch_and_process_packet.constprop.9 00647c90 f   libvorbisfile:vorbisfile.o
 0001:00247060       _ov_read_filter.part.8     00648060 f   libvorbisfile:vorbisfile.o
 0001:00247a40       __ov_d_seek_lap            00648a40 f   libvorbisfile:vorbisfile.o
 0001:00247d00       __bisect_forward_serialno  00648d00 f   libvorbisfile:vorbisfile.o
 0001:002483f0       __open_seekable2           006493f0 f   libvorbisfile:vorbisfile.o
 0001:00284c90       _png_write_chunk_header.part.0 00685c90 f   libpng_mini:pngwutil.o
 0001:00284d20       _png_write_chunk_end.part.2 00685d20 f   libpng_mini:pngwutil.o
 0001:00284ec0       _png_write_complete_chunk  00685ec0 f   libpng_mini:pngwutil.o
 0001:00285a40       _longest_match             00686a40 f   libz_mini:deflate.o
 0001:00285cc0       _fill_window               00686cc0 f   libz_mini:deflate.o
 0001:00285fb0       _flush_pending             00686fb0 f   libz_mini:deflate.o
 0001:00286020       _deflate_slow              00687020 f   libz_mini:deflate.o
 0001:002864c0       _deflate_fast              006874c0 f   libz_mini:deflate.o
 0001:00286880       _deflate_stored            00687880 f   libz_mini:deflate.o
 0001:002888f0       _gf2_matrix_square         006898f0 f   libz_mini:crc32.o
 0001:00288930       _crc32_combine_            00689930 f   libz_mini:crc32.o
 0001:00288d10       _pqdownheap                00689d10 f   libz_mini:trees.o
 0001:00288e20       _build_tree                00689e20 f   libz_mini:trees.o
 0001:002892a0       _scan_tree                 0068a2a0 f   libz_mini:trees.o
 0001:00289390       _send_tree                 0068a390 f   libz_mini:trees.o
 0001:00289990       _compress_block            0068a990 f   libz_mini:trees.o
 0001:00289e20       _bi_windup                 0068ae20 f   libz_mini:trees.o
 0001:00289e90       _bi_flush                  0068ae90 f   libz_mini:trees.o
 0001:0028a950       _adler32_combine_.part.0   0068b950 f   libz_mini:adler32.o
 0001:0028ae00       ___qdivrem.part.0          0068be00 f   libcompat-to-msvc:dll_math.o
 0001:0028c920       _pre_c_init                0068d920 f   msvcrtd:crtexew.obj
 0001:0028c9b0       _pre_cpp_init              0068d9b0 f   msvcrtd:crtexew.obj
 0001:0028ca30       ___tmainCRTStartup         0068da30 f   msvcrtd:crtexew.obj
 0001:0028cd40       _check_managed_app         0068dd40 f   msvcrtd:crtexew.obj
 0001:0028d3c0       __packetout                0068e3c0 f   libogg:framing.o
 0001:0028d4e0       _ogg_page_checksum_set.part.0 0068e4e0 f   libogg:framing.o
 0001:0028d7d0       __os_body_expand           0068e7d0 f   libogg:framing.o
 0001:0028d840       __os_lacing_expand         0068e840 f   libogg:framing.o
 0001:0028d930       _ogg_stream_flush_i        0068e930 f   libogg:framing.o
 0001:0028eec0       __vorbis_pack_comment      0068fec0 f   libvorbis:info.o
 0001:00290920       __preextrapolate_helper    00691920 f   libvorbis:block.o
 0001:00290f60       __vds_shared_init          00691f60 f   libvorbis:block.o
 0001:00292910       _sort32a                   00693910 f   libvorbis:sharedbook.o
 0001:00292930       __book_unquantize.part.0   00693930 f   libvorbis:sharedbook.o
 0001:00293c90       _apsort                    00694c90 f   libvorbis:psy.o
 0001:00293cc0       _bark_noise_hybridmp       00694cc0 f   libvorbis:psy.o
 0001:002942b0       _seed_chase                006952b0 f   libvorbis:psy.o
 0001:00294460       _setup_tone_curves         00695460 f   libvorbis:psy.o
 0001:00295280       _noise_normalize.isra.0    00696280 f   libvorbis:psy.o
 0001:002956b0       _bark_noise_hybridmp.constprop.1 006966b0 f   libvorbis:psy.o
 0001:00295a70       _noise_normalize.isra.0.constprop.2 00696a70 f   libvorbis:psy.o
 0001:002991e0       __ve_amp                   0069a1e0 f   libvorbis:envelope.o
 0001:00299c30       _mdct_butterflies.isra.0   0069ac30 f   libvorbis:mdct.o
 0001:0029b6a0       _dradf2                    0069c6a0 f   libvorbis:smallft.o
 0001:0029b880       _dradf4                    0069c880 f   libvorbis:smallft.o
 0001:0029bc50       _dradb2                    0069cc50 f   libvorbis:smallft.o
 0001:0029be20       _dradb3                    0069ce20 f   libvorbis:smallft.o
 0001:0029c070       _dradb4                    0069d070 f   libvorbis:smallft.o
 0001:0029c3d0       _dradfg                    0069d3d0 f   libvorbis:smallft.o
 0001:0029d190       _dradbg                    0069e190 f   libvorbis:smallft.o
 0001:0029e7f0       _mapping0_inverse          0069f7f0 f   libvorbis:mapping0.o
 0001:0029ebb0       _mapping0_forward          0069fbb0 f   libvorbis:mapping0.o
 0001:0029f5a0       _mapping0_free_info        006a05a0 f   libvorbis:mapping0.o
 0001:0029f5c0       _mapping0_pack             006a05c0 f   libvorbis:mapping0.o
 0001:0029f7b0       _mapping0_unpack           006a07b0 f   libvorbis:mapping0.o
 0001:002a02a0       __01inverse                006a12a0 f   libvorbis:res0.o
 0001:002a05f0       __encodepart               006a15f0 f   libvorbis:res0.o
 0001:002a1360       __01forward.constprop.1    006a2360 f   libvorbis:res0.o
 0001:002a1a00       _floor0_inverse1           006a2a00 f   libvorbis:floor0.o
 0001:002a1b30       _floor0_free_look          006a2b30 f   libvorbis:floor0.o
 0001:002a1b90       _floor0_free_info          006a2b90 f   libvorbis:floor0.o
 0001:002a1bb0       _floor0_look               006a2bb0 f   libvorbis:floor0.o
 0001:002a1c00       _floor0_inverse2           006a2c00 f   libvorbis:floor0.o
 0001:002a1e80       _floor0_unpack             006a2e80 f   libvorbis:floor0.o
 0001:002a1f90       _icomp                     006a2f90 f   libvorbis:floor1.o
 0001:002a1fb0       _floor1_inverse2           006a2fb0 f   libvorbis:floor1.o
 0001:002a21e0       _floor1_pack               006a31e0 f   libvorbis:floor1.o
 0001:002a2400       _floor1_inverse1           006a3400 f   libvorbis:floor1.o
 0001:002a2740       _floor1_free_look          006a3740 f   libvorbis:floor1.o
 0001:002a2760       _floor1_free_info          006a3760 f   libvorbis:floor1.o
 0001:002a2780       _floor1_look               006a3780 f   libvorbis:floor1.o
 0001:002a2a80       _accumulate_fit.isra.1     006a3a80 f   libvorbis:floor1.o
 0001:002a2cc0       _fit_line.isra.2           006a3cc0 f   libvorbis:floor1.o
 0001:002a2f40       _floor1_unpack             006a3f40 f   libvorbis:floor1.o
 0001:002a4a40       _comp                      006a5a40 f   libvorbis:lsp.o
 0001:002a4a70       _Laguerre_With_Deflation   006a5a70 f   libvorbis:lsp.o
 0001:002a4cb0       _Newton_Raphson            006a5cb0 f   libvorbis:lsp.o
 0001:002a5990       _oggpack_writecopy_helper  006a6990 f   libogg:bitwise.o
 0001:002a6240       ??__Eg_dynTileList@@YAXXZ  006a7240 f   namesdyn.obj
 0001:002aabd0       ??__Esvgm_udnetw@@YAXXZ    006abbd0 f   savegame.obj
 0001:002ab040       ??__Esvgm_secwsp@@YAXXZ    006ac040 f   savegame.obj
 0001:002ab570       ??__Esvgm_script@@YAXXZ    006ac570 f   savegame.obj
 0001:002ab850       ??__Esvgm_anmisc@@YAXXZ    006ac850 f   savegame.obj
 0001:002abe00       ??__Einternalgrpfiles@@YAXXZ 006ace00 f   grpscan.obj
 0001:002ac4e0       ??__Eg_dynSoundList@@YAXXZ 006ad4e0 f   soundsdyn.obj
 0001:002ad600       ??__Eg_dumper@@YAXXZ       006ae600 f   mdump.obj
